 xerces-c_2_3_0

 Timestamp is 3ed313d7 (Tue May 27 03:29:27 2003)

 Preferred load address is 12000000

 Start         Length     Name                   Class
 0001:00000000 000f0af0H .text                   CODE
 0001:000f0af0 00011062H .text$x                 CODE
 0002:00000000 00000164H .idata$5                DATA
 0002:00000168 000319dcH .rdata                  DATA
 0002:00031b48 00000044H .rdata$r                DATA
 0002:00031b90 00015810H .xdata$x                DATA
 0002:000473a0 00000050H .idata$2                DATA
 0002:000473f0 00000014H .idata$3                DATA
 0002:00047404 00000164H .idata$4                DATA
 0002:00047568 0000055aH .idata$6                DATA
 0002:00047ad0 0006dc73H .edata                  DATA
 0003:00000000 00000004H .CRT$XCA                DATA
 0003:00000004 0000005cH .CRT$XCU                DATA
 0003:00000060 00000004H .CRT$XCZ                DATA
 0003:00000064 00000004H .CRT$XIA                DATA
 0003:00000068 00000004H .CRT$XIZ                DATA
 0003:00000070 00023c10H .data                   DATA
 0003:00023c80 00000b54H .bss                    DATA
 0004:00000000 00000a60H .rsrc$01                DATA
 0004:00000a60 000150c0H .rsrc$02                DATA

  Address         Publics by Value              Rva+Base     Lib:Object

 0001:00000000       ??0MemoryManager@xercesc_2_3@@IAE@XZ 12001000 f i Win32PlatformUtils.obj
 0001:00000010       ??_EMemoryManager@xercesc_2_3@@UAEPAXI@Z 12001010 f i Win32PlatformUtils.obj
 0001:00000070       ??0DOMError@xercesc_2_3@@IAE@XZ 12001070 f i Win32PlatformUtils.obj
 0001:00000080       ??1DOMError@xercesc_2_3@@UAE@XZ 12001080 f i Win32PlatformUtils.obj
 0001:00000090       ??_EDOMError@xercesc_2_3@@UAEPAXI@Z 12001090 f i Win32PlatformUtils.obj
 0001:000000f0       ??1XMLErrorReporter@xercesc_2_3@@UAE@XZ 120010f0 f i Win32PlatformUtils.obj
 0001:00000100       ??0XMLErrorReporter@xercesc_2_3@@IAE@XZ 12001100 f i Win32PlatformUtils.obj
 0001:00000110       ??_EXMLErrorReporter@xercesc_2_3@@UAEPAXI@Z 12001110 f i Win32PlatformUtils.obj
 0001:00000170       ?getSrcFile@XMLException@xercesc_2_3@@QBEPBDXZ 12001170 f i Win32PlatformUtils.obj
 0001:00000180       ?getErrorType@XMLException@xercesc_2_3@@QBE?AW4ErrTypes@XMLErrorReporter@2@XZ 12001180 f i Win32PlatformUtils.obj
 0001:000001c0       ??0PanicHandler@xercesc_2_3@@IAE@XZ 120011c0 f i Win32PlatformUtils.obj
 0001:000001d0       ??1DefaultPanicHandler@xercesc_2_3@@UAE@XZ 120011d0 f i Win32PlatformUtils.obj
 0001:000001d0       ??1PanicHandler@xercesc_2_3@@UAE@XZ 120011d0 f i Win32PlatformUtils.obj
 0001:000001e0       ??_EPanicHandler@xercesc_2_3@@UAEPAXI@Z 120011e0 f i Win32PlatformUtils.obj
 0001:00000240       ??0XMLPlatformUtilsException@xercesc_2_3@@QAE@QBDIW4Codes@XMLExcepts@1@@Z 12001240 f i Win32PlatformUtils.obj
 0001:000002a0       ??0XMLPlatformUtilsException@xercesc_2_3@@QAE@ABV01@@Z 120012a0 f i Win32PlatformUtils.obj
 0001:000002c0       ??0XMLPlatformUtilsException@xercesc_2_3@@QAE@QBDIW4Codes@XMLExcepts@1@QBG222@Z 120012c0 f i Win32PlatformUtils.obj
 0001:00000330       ??0XMLPlatformUtilsException@xercesc_2_3@@QAE@QBDIW4Codes@XMLExcepts@1@0000@Z 12001330 f i Win32PlatformUtils.obj
 0001:000003a0       ??1XMLPlatformUtilsException@xercesc_2_3@@UAE@XZ 120013a0 f i Win32PlatformUtils.obj
 0001:000003b0       ?duplicate@XMLPlatformUtilsException@xercesc_2_3@@UBEPAVXMLException@2@XZ 120013b0 f i Win32PlatformUtils.obj
 0001:00000410       ?getType@XMLPlatformUtilsException@xercesc_2_3@@UBEPBGXZ 12001410 f i Win32PlatformUtils.obj
 0001:00000420       ??_EXMLPlatformUtilsException@xercesc_2_3@@UAEPAXI@Z 12001420 f i Win32PlatformUtils.obj
 0001:00000480       ?alignPointerForNewBlockAllocation@XMLPlatformUtils@xercesc_2_3@@SAII@Z 12001480 f i Win32PlatformUtils.obj
 0001:000004a0       ??1XMLDeleter@xercesc_2_3@@UAE@XZ 120014a0 f i Win32PlatformUtils.obj
 0001:000004b0       ??_EXMLDeleter@xercesc_2_3@@UAEPAXI@Z 120014b0 f i Win32PlatformUtils.obj
 0001:00000510       ??0XMLDeleter@xercesc_2_3@@IAE@XZ 12001510 f i Win32PlatformUtils.obj
 0001:00000520       ??0RuntimeException@xercesc_2_3@@QAE@QBDIW4Codes@XMLExcepts@1@@Z 12001520 f i Win32PlatformUtils.obj
 0001:00000580       ??0RuntimeException@xercesc_2_3@@QAE@ABV01@@Z 12001580 f i Win32PlatformUtils.obj
 0001:000005a0       ??0RuntimeException@xercesc_2_3@@QAE@QBDIW4Codes@XMLExcepts@1@QBG222@Z 120015a0 f i Win32PlatformUtils.obj
 0001:00000610       ??0RuntimeException@xercesc_2_3@@QAE@QBDIW4Codes@XMLExcepts@1@0000@Z 12001610 f i Win32PlatformUtils.obj
 0001:00000680       ??1RuntimeException@xercesc_2_3@@UAE@XZ 12001680 f i Win32PlatformUtils.obj
 0001:00000690       ?duplicate@RuntimeException@xercesc_2_3@@UBEPAVXMLException@2@XZ 12001690 f i Win32PlatformUtils.obj
 0001:000006f0       ?getType@RuntimeException@xercesc_2_3@@UBEPBGXZ 120016f0 f i Win32PlatformUtils.obj
 0001:00000700       ??_ERuntimeException@xercesc_2_3@@UAEPAXI@Z 12001700 f i Win32PlatformUtils.obj
 0001:00000760       ??0ArrayIndexOutOfBoundsException@xercesc_2_3@@QAE@QBDIW4Codes@XMLExcepts@1@@Z 12001760 f i Win32PlatformUtils.obj
 0001:000007c0       ??0ArrayIndexOutOfBoundsException@xercesc_2_3@@QAE@ABV01@@Z 120017c0 f i Win32PlatformUtils.obj
 0001:000007e0       ??0ArrayIndexOutOfBoundsException@xercesc_2_3@@QAE@QBDIW4Codes@XMLExcepts@1@QBG222@Z 120017e0 f i Win32PlatformUtils.obj
 0001:00000850       ??0ArrayIndexOutOfBoundsException@xercesc_2_3@@QAE@QBDIW4Codes@XMLExcepts@1@0000@Z 12001850 f i Win32PlatformUtils.obj
 0001:000008c0       ??1ArrayIndexOutOfBoundsException@xercesc_2_3@@UAE@XZ 120018c0 f i Win32PlatformUtils.obj
 0001:000008d0       ?duplicate@ArrayIndexOutOfBoundsException@xercesc_2_3@@UBEPAVXMLException@2@XZ 120018d0 f i Win32PlatformUtils.obj
 0001:00000930       ?getType@ArrayIndexOutOfBoundsException@xercesc_2_3@@UBEPBGXZ 12001930 f i Win32PlatformUtils.obj
 0001:00000940       ??_EArrayIndexOutOfBoundsException@xercesc_2_3@@UAEPAXI@Z 12001940 f i Win32PlatformUtils.obj
 0001:000009a0       ?moveChars@XMLString@xercesc_2_3@@SAXQAGQBGI@Z 120019a0 f i Win32PlatformUtils.obj
 0001:000009d0       ?stringLen@XMLString@xercesc_2_3@@SAIQBG@Z 120019d0 f i Win32PlatformUtils.obj
 0001:00000a00       ?startsWith@XMLString@xercesc_2_3@@SA_NQBG0@Z 12001a00 f i Win32PlatformUtils.obj
 0001:00000a40       ?startsWithI@XMLString@xercesc_2_3@@SA_NQBG0@Z 12001a40 f i Win32PlatformUtils.obj
 0001:00000a80       ?endsWith@XMLString@xercesc_2_3@@SA_NQBG0@Z 12001a80 f i Win32PlatformUtils.obj
 0001:00000b00       ?replicate@XMLString@xercesc_2_3@@SAPAGQBG@Z 12001b00 f i Win32PlatformUtils.obj
 0001:00000b50       ?replicate@XMLString@xercesc_2_3@@SAPAGQBGQAVMemoryManager@2@@Z 12001b50 f i Win32PlatformUtils.obj
 0001:00000ba0       ?validateRegion@XMLString@xercesc_2_3@@CA_NQBGH0HI@Z 12001ba0 f i Win32PlatformUtils.obj
 0001:00000c20       ?equals@XMLString@xercesc_2_3@@SA_NQBG0@Z 12001c20 f i Win32PlatformUtils.obj
 0001:00000c70       ?equals@XMLString@xercesc_2_3@@SA_NQBD0@Z 12001c70 f i Win32PlatformUtils.obj
 0001:00000cc0       ?getErrorHandler@DOMBuilderImpl@xercesc_2_3@@UAEPAVDOMErrorHandler@2@XZ 12001cc0 f i Win32PlatformUtils.obj
 0001:00000cc0       ?getFinalSet@DatatypeValidator@xercesc_2_3@@QBEHXZ 12001cc0 f i Win32PlatformUtils.obj
 0001:00000cc0       ?getCreateReason@XMLElementDecl@xercesc_2_3@@QBE?AW4CreateReasons@12@XZ 12001cc0 f i Win32PlatformUtils.obj
 0001:00000cc0       ?getLocalPart@QName@xercesc_2_3@@QAEPAGXZ 12001cc0 f i Win32PlatformUtils.obj
 0001:00000cc0       ?getValue@KVStringPair@xercesc_2_3@@QBEPBGXZ 12001cc0 f i Win32PlatformUtils.obj
 0001:00000cc0       ?getConditionToken@ConditionToken@xercesc_2_3@@QBEPAVToken@2@XZ 12001cc0 f i Win32PlatformUtils.obj
 0001:00000cc0       ?getErrorHandler@DOMBuilderImpl@xercesc_2_3@@UBEPBVDOMErrorHandler@2@XZ 12001cc0 f i Win32PlatformUtils.obj
 0001:00000cc0       ?getCompleteWildCard@XercesAttGroupInfo@xercesc_2_3@@QBEPAVSchemaAttDef@2@XZ 12001cc0 f i Win32PlatformUtils.obj
 0001:00000cc0       ?getOffset@DOMLocatorImpl@xercesc_2_3@@UBEJXZ 12001cc0 f i Win32PlatformUtils.obj
 0001:00000cc0       ?getLocalPart@QName@xercesc_2_3@@QBEPBGXZ 12001cc0 f i Win32PlatformUtils.obj
 0001:00000cc0       ?getPublicId@InputSource@xercesc_2_3@@UBEPBGXZ 12001cc0 f i Win32PlatformUtils.obj
 0001:00000cc0       ?getReaderMgr@XMLValidator@xercesc_2_3@@IBEPBVReaderMgr@2@XZ 12001cc0 f i Win32PlatformUtils.obj
 0001:00000cc0       ?getReaderMgr@XMLValidator@xercesc_2_3@@IAEPAVReaderMgr@2@XZ 12001cc0 f i Win32PlatformUtils.obj
 0001:00000cc0       ?getHost@XMLURL@xercesc_2_3@@QBEPBGXZ 12001cc0 f i Win32PlatformUtils.obj
 0001:00000cc0       ?getValue@XMLAttr@xercesc_2_3@@QBEPBGXZ 12001cc0 f i Win32PlatformUtils.obj
 0001:00000cc0       ?getValue@XMLEntityDecl@xercesc_2_3@@QBEPBGXZ 12001cc0 f i Win32PlatformUtils.obj
 0001:00000cc0       ?getString@StringToken@xercesc_2_3@@UBEPBGXZ 12001cc0 f i Win32PlatformUtils.obj
 0001:00000cc0       ?getSrcLine@XMLException@xercesc_2_3@@QBEIXZ 12001cc0 f i Win32PlatformUtils.obj
 0001:00000cc0       ?getCategories@RangeTokenMap@xercesc_2_3@@IBEPAVXMLStringPool@2@XZ 12001cc0 f i Win32PlatformUtils.obj
 0001:00000cc0       ?getBlockSet@ComplexTypeInfo@xercesc_2_3@@QBEHXZ 12001cc0 f i Win32PlatformUtils.obj
 0001:00000cc0       ?getOptionsMask@ModifierToken@xercesc_2_3@@QBEHXZ 12001cc0 f i Win32PlatformUtils.obj
 0001:00000cc0       ?getTargetNSURI@SchemaInfo@xercesc_2_3@@QBEHXZ 12001cc0 f i Win32PlatformUtils.obj
 0001:00000cc0       ?getLen@MemBufFormatTarget@xercesc_2_3@@QBEIXZ 12001cc0 f i Win32PlatformUtils.obj
 0001:00000cc0       ?getMemoryManager@XMLTranscoder@xercesc_2_3@@QBEPAVMemoryManager@2@XZ 12001cc0 f i Win32PlatformUtils.obj
 0001:00000cc0       ?getHost@XMLUri@xercesc_2_3@@QBEPBGXZ 12001cc0 f i Win32PlatformUtils.obj
 0001:00000cc0       ?getSystemId@XMLNotationDecl@xercesc_2_3@@QBEPBGXZ 12001cc0 f i Win32PlatformUtils.obj
 0001:00000cc0       ?getSystemId@XSDLocator@xercesc_2_3@@UBEPBGXZ 12001cc0 f i Win32PlatformUtils.obj
 0001:00000cc0       ?getCreateReason@XMLAttDef@xercesc_2_3@@QBE?AW4CreateReasons@12@XZ 12001cc0 f i Win32PlatformUtils.obj
 0001:00000cc0       ?getMax@ClosureToken@xercesc_2_3@@UBEHXZ 12001cc0 f i Win32PlatformUtils.obj
 0001:00000cc0       ?getLocation@DOMErrorImpl@xercesc_2_3@@UBEPAVDOMLocator@2@XZ 12001cc0 f i Win32PlatformUtils.obj
 0001:00000cc0       ?getScale@XMLBigDecimal@xercesc_2_3@@QBEIXZ 12001cc0 f i Win32PlatformUtils.obj
 0001:00000cc0       ?getValue@KVStringPair@xercesc_2_3@@QAEPAGXZ 12001cc0 f i Win32PlatformUtils.obj
 0001:00000cc0       ?getSelector@IdentityConstraint@xercesc_2_3@@QBEPAVIC_Selector@2@XZ 12001cc0 f i Win32PlatformUtils.obj
 0001:00000cd0       ?getSign@XMLBigDecimal@xercesc_2_3@@UBEHXZ 12001cd0 f i Win32PlatformUtils.obj
 0001:00000cd0       ?getPrefix@QName@xercesc_2_3@@QAEPAGXZ 12001cd0 f i Win32PlatformUtils.obj
 0001:00000cd0       ?getLen@XMLBuffer@xercesc_2_3@@QBEIXZ 12001cd0 f i Win32PlatformUtils.obj
 0001:00000cd0       ?getLineNumber@XSDLocator@xercesc_2_3@@UBEJXZ 12001cd0 f i Win32PlatformUtils.obj
 0001:00000cd0       ?getBufMgr@XMLValidator@xercesc_2_3@@IAEPAVXMLBufferMgr@2@XZ 12001cd0 f i Win32PlatformUtils.obj
 0001:00000cd0       ?getMemoryManager@XMLURL@xercesc_2_3@@QBEPAVMemoryManager@2@XZ 12001cd0 f i Win32PlatformUtils.obj
 0001:00000cd0       ?getReaderNum@EndOfEntityException@xercesc_2_3@@QBEIXZ 12001cd0 f i Win32PlatformUtils.obj
 0001:00000cd0       ?getName@XercesNodeTest@xercesc_2_3@@QBEPAVQName@2@XZ 12001cd0 f i Win32PlatformUtils.obj
 0001:00000cd0       ?getMemoryManager@XMLElementDecl@xercesc_2_3@@QBEPAVMemoryManager@2@XZ 12001cd0 f i Win32PlatformUtils.obj
 0001:00000cd0       ?getXPath@IC_Field@xercesc_2_3@@QBEPAVXercesXPath@2@XZ 12001cd0 f i Win32PlatformUtils.obj
 0001:00000cd0       ?getEncodingName@XMLFormatter@xercesc_2_3@@QBEPBGXZ 12001cd0 f i Win32PlatformUtils.obj
 0001:00000cd0       ?getBlockSize@XMLTranscoder@xercesc_2_3@@QBEIXZ 12001cd0 f i Win32PlatformUtils.obj
 0001:00000cd0       ?getLineNumber@DOMLocatorImpl@xercesc_2_3@@UBEJXZ 12001cd0 f i Win32PlatformUtils.obj
 0001:00000cd0       ?getType@XMLAttr@xercesc_2_3@@QBE?AW4AttTypes@XMLAttDef@2@XZ 12001cd0 f i Win32PlatformUtils.obj
 0001:00000cd0       ?getScope@XercesGroupInfo@xercesc_2_3@@QBEHXZ 12001cd0 f i Win32PlatformUtils.obj
 0001:00000cd0       ?getBufMgr@XMLValidator@xercesc_2_3@@IBEPBVXMLBufferMgr@2@XZ 12001cd0 f i Win32PlatformUtils.obj
 0001:00000cd0       ?getScheme@XMLUri@xercesc_2_3@@QBEPBGXZ 12001cd0 f i Win32PlatformUtils.obj
 0001:00000cd0       ?getKey@KVStringPair@xercesc_2_3@@QBEPBGXZ 12001cd0 f i Win32PlatformUtils.obj
 0001:00000cd0       ?getCode@XMLException@xercesc_2_3@@QBE?AW4Codes@XMLExcepts@2@XZ 12001cd0 f i Win32PlatformUtils.obj
 0001:00000cd0       ?getTokenRegistry@RangeTokenMap@xercesc_2_3@@IBEPAV?$RefHashTableOf@VRangeTokenElemMap@xercesc_2_3@@@2@XZ 12001cd0 f i Win32PlatformUtils.obj
 0001:00000cd0       ?getId@XMLEntityDecl@xercesc_2_3@@QBEIXZ 12001cd0 f i Win32PlatformUtils.obj
 0001:00000cd0       ?getBlockDefault@SchemaInfo@xercesc_2_3@@QBEHXZ 12001cd0 f i Win32PlatformUtils.obj
 0001:00000cd0       ?getDefaultType@XMLAttDef@xercesc_2_3@@QBE?AW4DefAttTypes@12@XZ 12001cd0 f i Win32PlatformUtils.obj
 0001:00000cd0       ?getEntityExpansionLimit@SecurityManager@xercesc_2_3@@UBEIXZ 12001cd0 f i Win32PlatformUtils.obj
 0001:00000cd0       ?getKey@KVStringPair@xercesc_2_3@@QAEPAGXZ 12001cd0 f i Win32PlatformUtils.obj
 0001:00000cd0       ?getMemoryManager@InputSource@xercesc_2_3@@QBEPAVMemoryManager@2@XZ 12001cd0 f i Win32PlatformUtils.obj
 0001:00000cd0       ?getMessage@SAXException@xercesc_2_3@@UBEPBGXZ 12001cd0 f i Win32PlatformUtils.obj
 0001:00000cd0       ?getKey@XMLNotationDecl@xercesc_2_3@@QBEPBGXZ 12001cd0 f i Win32PlatformUtils.obj
 0001:00000cd0       ?getIdentityConstraint@IC_Selector@xercesc_2_3@@QBEPAVIdentityConstraint@2@XZ 12001cd0 f i Win32PlatformUtils.obj
 0001:00000cd0       ?getIdentityConstraintName@IdentityConstraint@xercesc_2_3@@QBEPAGXZ 12001cd0 f i Win32PlatformUtils.obj
 0001:00000cd0       ?getName@XMLNotationDecl@xercesc_2_3@@QBEPBGXZ 12001cd0 f i Win32PlatformUtils.obj
 0001:00000cd0       ?getRefName@XMLRefInfo@xercesc_2_3@@QBEPBGXZ 12001cd0 f i Win32PlatformUtils.obj
 0001:00000cd0       ?getMemoryManager@DatatypeValidator@xercesc_2_3@@QBEPAVMemoryManager@2@XZ 12001cd0 f i Win32PlatformUtils.obj
 0001:00000cd0       ?getNodeTest@XercesStep@xercesc_2_3@@QBEPAVXercesNodeTest@2@XZ 12001cd0 f i Win32PlatformUtils.obj
 0001:00000cd0       ?getPrefix@QName@xercesc_2_3@@QBEPBGXZ 12001cd0 f i Win32PlatformUtils.obj
 0001:00000cd0       ?getTargetNamespace@SchemaGrammar@xercesc_2_3@@UBEPBGXZ 12001cd0 f i Win32PlatformUtils.obj
 0001:00000ce0       ?getType@XMLAttDef@xercesc_2_3@@QBE?AW4AttTypes@12@XZ 12001ce0 f i Win32PlatformUtils.obj
 0001:00000ce0       ?getNoParen@ParenToken@xercesc_2_3@@UBEHXZ 12001ce0 f i Win32PlatformUtils.obj
 0001:00000ce0       ?getEncoding@InputSource@xercesc_2_3@@UBEPBGXZ 12001ce0 f i Win32PlatformUtils.obj
 0001:00000ce0       ?getFinalDefault@SchemaInfo@xercesc_2_3@@QBEHXZ 12001ce0 f i Win32PlatformUtils.obj
 0001:00000ce0       ?getChar@CharToken@xercesc_2_3@@UBEHXZ 12001ce0 f i Win32PlatformUtils.obj
 0001:00000ce0       ?getTotalDigit@XMLBigDecimal@xercesc_2_3@@QBEIXZ 12001ce0 f i Win32PlatformUtils.obj
 0001:00000ce0       ?getLocationPaths@XercesXPath@xercesc_2_3@@QBEPAV?$RefVectorOf@VXercesLocationPath@xercesc_2_3@@@2@XZ 12001ce0 f i Win32PlatformUtils.obj
 0001:00000ce0       ?getOptions@ModifierToken@xercesc_2_3@@QBEHXZ 12001ce0 f i Win32PlatformUtils.obj
 0001:00000ce0       ?getElementName@XMLElementDecl@xercesc_2_3@@QAEPAVQName@2@XZ 12001ce0 f i Win32PlatformUtils.obj
 0001:00000ce0       ?getRawData@XMLBigInteger@xercesc_2_3@@QBEPAGXZ 12001ce0 f i Win32PlatformUtils.obj
 0001:00000ce0       ?getRangeMap@RangeTokenMap@xercesc_2_3@@IBEPAV?$RefHashTableOf@VRangeFactory@xercesc_2_3@@@2@XZ 12001ce0 f i Win32PlatformUtils.obj
 0001:00000ce0       ?getColumnNumber@DOMLocatorImpl@xercesc_2_3@@UBEJXZ 12001ce0 f i Win32PlatformUtils.obj
 0001:00000ce0       ?getEncodingName@XMLTranscoder@xercesc_2_3@@QBEPBGXZ 12001ce0 f i Win32PlatformUtils.obj
 0001:00000ce0       ?getDocTypeHandler@DTDScanner@xercesc_2_3@@QAEPAVDocTypeHandler@2@XZ 12001ce0 f i Win32PlatformUtils.obj
 0001:00000ce0       ?getIdentityConstraint@ValueStore@xercesc_2_3@@QBEPAVIdentityConstraint@2@XZ 12001ce0 f i Win32PlatformUtils.obj
 0001:00000ce0       ?getContentSpec@XercesGroupInfo@xercesc_2_3@@QBEPAVContentSpecNode@2@XZ 12001ce0 f i Win32PlatformUtils.obj
 0001:00000ce0       ?curPos@BinHTTPURLInputStream@xercesc_2_3@@UBEIXZ 12001ce0 f i Win32PlatformUtils.obj
 0001:00000ce0       ?getElementName@IdentityConstraint@xercesc_2_3@@QBEPAGXZ 12001ce0 f i Win32PlatformUtils.obj
 0001:00000ce0       ?getEntityResolver@DOMBuilderImpl@xercesc_2_3@@UAEPAVDOMEntityResolver@2@XZ 12001ce0 f i Win32PlatformUtils.obj
 0001:00000ce0       ?getFragment@XMLURL@xercesc_2_3@@QBEPBGXZ 12001ce0 f i Win32PlatformUtils.obj
 0001:00000ce0       ?getIdentityConstraint@IC_Field@xercesc_2_3@@QBEPAVIdentityConstraint@2@XZ 12001ce0 f i Win32PlatformUtils.obj
 0001:00000ce0       ?getUserInfo@XMLUri@xercesc_2_3@@QBEPBGXZ 12001ce0 f i Win32PlatformUtils.obj
 0001:00000ce0       ?getReferenceNo@StringToken@xercesc_2_3@@UBEHXZ 12001ce0 f i Win32PlatformUtils.obj
 0001:00000ce0       ?getValueLen@XMLEntityDecl@xercesc_2_3@@QBEIXZ 12001ce0 f i Win32PlatformUtils.obj
 0001:00000ce0       ?getElementName@XMLElementDecl@xercesc_2_3@@QBEPBVQName@2@XZ 12001ce0 f i Win32PlatformUtils.obj
 0001:00000ce0       ?getReferenceNo@ConditionToken@xercesc_2_3@@UBEHXZ 12001ce0 f i Win32PlatformUtils.obj
 0001:00000ce0       ?getMessage@DOMErrorImpl@xercesc_2_3@@UBEPBGXZ 12001ce0 f i Win32PlatformUtils.obj
 0001:00000ce0       ?getEntityResolver@DOMBuilderImpl@xercesc_2_3@@UBEPBVDOMEntityResolver@2@XZ 12001ce0 f i Win32PlatformUtils.obj
 0001:00000ce0       ?getMin@ClosureToken@xercesc_2_3@@UBEHXZ 12001ce0 f i Win32PlatformUtils.obj
 0001:00000ce0       ?getPublicId@XMLNotationDecl@xercesc_2_3@@QBEPBGXZ 12001ce0 f i Win32PlatformUtils.obj
 0001:00000ce0       ?getColumnNumber@XSDLocator@xercesc_2_3@@UBEJXZ 12001ce0 f i Win32PlatformUtils.obj
 0001:00000ce0       ?getDerivedBy@ComplexTypeInfo@xercesc_2_3@@QBEHXZ 12001ce0 f i Win32PlatformUtils.obj
 0001:00000ce0       ?getDocTypeHandler@DTDScanner@xercesc_2_3@@QBEPBVDocTypeHandler@2@XZ 12001ce0 f i Win32PlatformUtils.obj
 0001:00000ce0       ?getNextOp@Op@xercesc_2_3@@QBEPBV12@XZ 12001ce0 f i Win32PlatformUtils.obj
 0001:00000cf0       ??0HashBase@xercesc_2_3@@QAE@XZ 12001cf0 f i Win32PlatformUtils.obj
 0001:00000d00       ??0IllegalArgumentException@xercesc_2_3@@QAE@QBDIW4Codes@XMLExcepts@1@@Z 12001d00 f i Win32PlatformUtils.obj
 0001:00000d60       ??0IllegalArgumentException@xercesc_2_3@@QAE@ABV01@@Z 12001d60 f i Win32PlatformUtils.obj
 0001:00000d80       ??0IllegalArgumentException@xercesc_2_3@@QAE@QBDIW4Codes@XMLExcepts@1@QBG222@Z 12001d80 f i Win32PlatformUtils.obj
 0001:00000df0       ??0IllegalArgumentException@xercesc_2_3@@QAE@QBDIW4Codes@XMLExcepts@1@0000@Z 12001df0 f i Win32PlatformUtils.obj
 0001:00000e60       ??1IllegalArgumentException@xercesc_2_3@@UAE@XZ 12001e60 f i Win32PlatformUtils.obj
 0001:00000e70       ??4EmptyStackException@xercesc_2_3@@QAEAAV01@ABV01@@Z 12001e70 f i Win32PlatformUtils.obj
 0001:00000e70       ??4XPathException@xercesc_2_3@@QAEAAV01@ABV01@@Z 12001e70 f i Win32PlatformUtils.obj
 0001:00000e70       ??4SchemaDateTimeException@xercesc_2_3@@QAEAAV01@ABV01@@Z 12001e70 f i Win32PlatformUtils.obj
 0001:00000e70       ??4UTFDataFormatException@xercesc_2_3@@QAEAAV01@ABV01@@Z 12001e70 f i Win32PlatformUtils.obj
 0001:00000e70       ??4InvalidCastException@xercesc_2_3@@QAEAAV01@ABV01@@Z 12001e70 f i Win32PlatformUtils.obj
 0001:00000e70       ??4TranscodingException@xercesc_2_3@@QAEAAV01@ABV01@@Z 12001e70 f i Win32PlatformUtils.obj
 0001:00000e70       ??4InvalidDatatypeValueException@xercesc_2_3@@QAEAAV01@ABV01@@Z 12001e70 f i Win32PlatformUtils.obj
 0001:00000e70       ??4ArrayIndexOutOfBoundsException@xercesc_2_3@@QAEAAV01@ABV01@@Z 12001e70 f i Win32PlatformUtils.obj
 0001:00000e70       ??4UnsupportedEncodingException@xercesc_2_3@@QAEAAV01@ABV01@@Z 12001e70 f i Win32PlatformUtils.obj
 0001:00000e70       ??4InvalidDatatypeFacetException@xercesc_2_3@@QAEAAV01@ABV01@@Z 12001e70 f i Win32PlatformUtils.obj
 0001:00000e70       ??4IllegalArgumentException@xercesc_2_3@@QAEAAV01@ABV01@@Z 12001e70 f i Win32PlatformUtils.obj
 0001:00000e70       ??4MalformedURLException@xercesc_2_3@@QAEAAV01@ABV01@@Z 12001e70 f i Win32PlatformUtils.obj
 0001:00000e70       ??4XMLPlatformUtilsException@xercesc_2_3@@QAEAAV01@ABV01@@Z 12001e70 f i Win32PlatformUtils.obj
 0001:00000e70       ??4NoSuchElementException@xercesc_2_3@@QAEAAV01@ABV01@@Z 12001e70 f i Win32PlatformUtils.obj
 0001:00000e70       ??4NetAccessorException@xercesc_2_3@@QAEAAV01@ABV01@@Z 12001e70 f i Win32PlatformUtils.obj
 0001:00000e70       ??4NullPointerException@xercesc_2_3@@QAEAAV01@ABV01@@Z 12001e70 f i Win32PlatformUtils.obj
 0001:00000e70       ??4ParseException@xercesc_2_3@@QAEAAV01@ABV01@@Z 12001e70 f i Win32PlatformUtils.obj
 0001:00000e70       ??4NumberFormatException@xercesc_2_3@@QAEAAV01@ABV01@@Z 12001e70 f i Win32PlatformUtils.obj
 0001:00000e70       ??4UnexpectedEOFException@xercesc_2_3@@QAEAAV01@ABV01@@Z 12001e70 f i Win32PlatformUtils.obj
 0001:00000e70       ??4RuntimeException@xercesc_2_3@@QAEAAV01@ABV01@@Z 12001e70 f i Win32PlatformUtils.obj
 0001:00000e70       ??4IOException@xercesc_2_3@@QAEAAV01@ABV01@@Z 12001e70 f i Win32PlatformUtils.obj
 0001:00000e90       ?duplicate@IllegalArgumentException@xercesc_2_3@@UBEPAVXMLException@2@XZ 12001e90 f i Win32PlatformUtils.obj
 0001:00000ef0       ?getType@IllegalArgumentException@xercesc_2_3@@UBEPBGXZ 12001ef0 f i Win32PlatformUtils.obj
 0001:00000f00       ??_EIllegalArgumentException@xercesc_2_3@@UAEPAXI@Z 12001f00 f i Win32PlatformUtils.obj
 0001:00000f60       ??0NoSuchElementException@xercesc_2_3@@QAE@QBDIW4Codes@XMLExcepts@1@@Z 12001f60 f i Win32PlatformUtils.obj
 0001:00000fc0       ??0NoSuchElementException@xercesc_2_3@@QAE@ABV01@@Z 12001fc0 f i Win32PlatformUtils.obj
 0001:00000fe0       ??0NoSuchElementException@xercesc_2_3@@QAE@QBDIW4Codes@XMLExcepts@1@QBG222@Z 12001fe0 f i Win32PlatformUtils.obj
 0001:00001050       ??0NoSuchElementException@xercesc_2_3@@QAE@QBDIW4Codes@XMLExcepts@1@0000@Z 12002050 f i Win32PlatformUtils.obj
 0001:000010c0       ??1NoSuchElementException@xercesc_2_3@@UAE@XZ 120020c0 f i Win32PlatformUtils.obj
 0001:000010d0       ?duplicate@NoSuchElementException@xercesc_2_3@@UBEPAVXMLException@2@XZ 120020d0 f i Win32PlatformUtils.obj
 0001:00001130       ?getType@NoSuchElementException@xercesc_2_3@@UBEPBGXZ 12002130 f i Win32PlatformUtils.obj
 0001:00001140       ??_ENoSuchElementException@xercesc_2_3@@UAEPAXI@Z 12002140 f i Win32PlatformUtils.obj
 0001:000011a0       ??0NullPointerException@xercesc_2_3@@QAE@QBDIW4Codes@XMLExcepts@1@@Z 120021a0 f i Win32PlatformUtils.obj
 0001:00001200       ??0NullPointerException@xercesc_2_3@@QAE@ABV01@@Z 12002200 f i Win32PlatformUtils.obj
 0001:00001220       ??0NullPointerException@xercesc_2_3@@QAE@QBDIW4Codes@XMLExcepts@1@QBG222@Z 12002220 f i Win32PlatformUtils.obj
 0001:00001290       ??0NullPointerException@xercesc_2_3@@QAE@QBDIW4Codes@XMLExcepts@1@0000@Z 12002290 f i Win32PlatformUtils.obj
 0001:00001300       ??1NullPointerException@xercesc_2_3@@UAE@XZ 12002300 f i Win32PlatformUtils.obj
 0001:00001310       ?duplicate@NullPointerException@xercesc_2_3@@UBEPAVXMLException@2@XZ 12002310 f i Win32PlatformUtils.obj
 0001:00001370       ?getType@NullPointerException@xercesc_2_3@@UBEPBGXZ 12002370 f i Win32PlatformUtils.obj
 0001:00001380       ??_ENullPointerException@xercesc_2_3@@UAEPAXI@Z 12002380 f i Win32PlatformUtils.obj
 0001:000013e0       ??1XMLMsgLoader@xercesc_2_3@@UAE@XZ 120023e0 f i Win32PlatformUtils.obj
 0001:000013f0       ??_EXMLMsgLoader@xercesc_2_3@@UAEPAXI@Z 120023f0 f i Win32PlatformUtils.obj
 0001:00001450       ??0XMLMsgLoader@xercesc_2_3@@IAE@XZ 12002450 f i Win32PlatformUtils.obj
 0001:00001460       ??_FXMLURL@xercesc_2_3@@QAEXXZ 12002460 f i Win32PlatformUtils.obj
 0001:00001470       ??9XMLURL@xercesc_2_3@@QBE_NABV01@@Z 12002470 f i Win32PlatformUtils.obj
 0001:00001490       ?getEntityDeclPool@DTDGrammar@xercesc_2_3@@QBEPBV?$NameIdPool@VDTDEntityDecl@xercesc_2_3@@@2@XZ 12002490 f i Win32PlatformUtils.obj
 0001:00001490       ?getPublicId@XSDLocator@xercesc_2_3@@UBEPBGXZ 12002490 f i Win32PlatformUtils.obj
 0001:00001490       ?getKey@XMLEntityDecl@xercesc_2_3@@QBEPBGXZ 12002490 f i Win32PlatformUtils.obj
 0001:00001490       ?getSystemId@InputSource@xercesc_2_3@@UBEPBGXZ 12002490 f i Win32PlatformUtils.obj
 0001:00001490       ?getName@XMLEntityDecl@xercesc_2_3@@QBEPBGXZ 12002490 f i Win32PlatformUtils.obj
 0001:00001490       ?curPos@BinMemInputStream@xercesc_2_3@@UBEIXZ 12002490 f i Win32PlatformUtils.obj
 0001:00001490       ?getBaseGroup@XercesGroupInfo@xercesc_2_3@@QBEPAV12@XZ 12002490 f i Win32PlatformUtils.obj
 0001:00001490       ?getScopeCount@SchemaInfo@xercesc_2_3@@QBEHXZ 12002490 f i Win32PlatformUtils.obj
 0001:00001490       ?getScanner@XMLValidator@xercesc_2_3@@IAEPAVXMLScanner@2@XZ 12002490 f i Win32PlatformUtils.obj
 0001:00001490       ?getValue@XMLBigDecimal@xercesc_2_3@@QBEPBGXZ 12002490 f i Win32PlatformUtils.obj
 0001:00001490       ?getBaseURI@XMLNotationDecl@xercesc_2_3@@QBEPBGXZ 12002490 f i Win32PlatformUtils.obj
 0001:00001490       ?getAttName@XMLAttr@xercesc_2_3@@QBEPAVQName@2@XZ 12002490 f i Win32PlatformUtils.obj
 0001:00001490       ?getTranscoder@XMLFormatter@xercesc_2_3@@QBEPBVXMLTranscoder@2@XZ 12002490 f i Win32PlatformUtils.obj
 0001:00001490       ?getScanner@XMLValidator@xercesc_2_3@@IBEPBVXMLScanner@2@XZ 12002490 f i Win32PlatformUtils.obj
 0001:00001490       ?getTokenFactory@RangeTokenMap@xercesc_2_3@@QBEPAVTokenFactory@2@XZ 12002490 f i Win32PlatformUtils.obj
 0001:00001490       ?getFilter@DOMBuilderImpl@xercesc_2_3@@UAEPAVDOMBuilderFilter@2@XZ 12002490 f i Win32PlatformUtils.obj
 0001:00001490       ?getType@DOMErrorImpl@xercesc_2_3@@UBEPBGXZ 12002490 f i Win32PlatformUtils.obj
 0001:00001490       ?getOffset@RegxParser@xercesc_2_3@@QBEHXZ 12002490 f i Win32PlatformUtils.obj
 0001:00001490       ?getPort@XMLUri@xercesc_2_3@@QBEHXZ 12002490 f i Win32PlatformUtils.obj
 0001:00001490       ?getFacetsDefined@DatatypeValidator@xercesc_2_3@@IBEHXZ 12002490 f i Win32PlatformUtils.obj
 0001:00001490       ?getId@XMLElementDecl@xercesc_2_3@@QBEIXZ 12002490 f i Win32PlatformUtils.obj
 0001:00001490       ?getEntityDeclPool@DTDGrammar@xercesc_2_3@@QAEPAV?$NameIdPool@VDTDEntityDecl@xercesc_2_3@@@2@XZ 12002490 f i Win32PlatformUtils.obj
 0001:00001490       ?getFinalSet@ComplexTypeInfo@xercesc_2_3@@QBEHXZ 12002490 f i Win32PlatformUtils.obj
 0001:00001490       ?getMessage@XMLException@xercesc_2_3@@QBEPBGXZ 12002490 f i Win32PlatformUtils.obj
 0001:00001490       ?getErrorNode@DOMLocatorImpl@xercesc_2_3@@UBEPAVDOMNode@2@XZ 12002490 f i Win32PlatformUtils.obj
 0001:00001490       ?getFilter@DOMBuilderImpl@xercesc_2_3@@UBEPBVDOMBuilderFilter@2@XZ 12002490 f i Win32PlatformUtils.obj
 0001:00001490       ?getPassword@XMLURL@xercesc_2_3@@QBEPBGXZ 12002490 f i Win32PlatformUtils.obj
 0001:000014a0       ?getRelatedData@DOMErrorImpl@xercesc_2_3@@UBEPAXXZ 120024a0 f i Win32PlatformUtils.obj
 0001:000014a0       ?getLocator@XercesGroupInfo@xercesc_2_3@@QBEPAVXSDLocator@2@XZ 120024a0 f i Win32PlatformUtils.obj
 0001:000014a0       ?getNotationName@XMLEntityDecl@xercesc_2_3@@QBEPBGXZ 120024a0 f i Win32PlatformUtils.obj
 0001:000014a0       ?getScopeDefined@ComplexTypeInfo@xercesc_2_3@@QBEHXZ 120024a0 f i Win32PlatformUtils.obj
 0001:000014a0       ?getURI@DOMLocatorImpl@xercesc_2_3@@UBEPBGXZ 120024a0 f i Win32PlatformUtils.obj
 0001:000014a0       ?getFixed@DatatypeValidator@xercesc_2_3@@IBEHXZ 120024a0 f i Win32PlatformUtils.obj
 0001:000014a0       ?getFormattedString@XMLBigDecimal@xercesc_2_3@@UBEPBGXZ 120024a0 f i Win32PlatformUtils.obj
 0001:000014a0       ?getErrorCount@XMLScanner@xercesc_2_3@@QAEHXZ 120024a0 f i Win32PlatformUtils.obj
 0001:000014a0       ?getRawData@XMLBigDecimal@xercesc_2_3@@UBEPAGXZ 120024a0 f i Win32PlatformUtils.obj
 0001:000014a0       ?getNoParen@RegxParser@xercesc_2_3@@QBEHXZ 120024a0 f i Win32PlatformUtils.obj
 0001:000014a0       ?getPath@XMLUri@xercesc_2_3@@QBEPBGXZ 120024a0 f i Win32PlatformUtils.obj
 0001:000014a0       ?getNamespaceScopeLevel@SchemaInfo@xercesc_2_3@@QBEIXZ 120024a0 f i Win32PlatformUtils.obj
 0001:000014a0       ?getGrammar@DTDValidator@xercesc_2_3@@UBEPAVGrammar@2@XZ 120024a0 f i Win32PlatformUtils.obj
 0001:000014a0       ?getMemoryManager@XMLNotationDecl@xercesc_2_3@@QBEPAVMemoryManager@2@XZ 120024a0 f i Win32PlatformUtils.obj
 0001:000014a0       ?getPath@XMLURL@xercesc_2_3@@QBEPBGXZ 120024a0 f i Win32PlatformUtils.obj
 0001:000014a0       ?getId@XMLAttDef@xercesc_2_3@@QBEIXZ 120024a0 f i Win32PlatformUtils.obj
 0001:000014b0       ?getProtocol@XMLURL@xercesc_2_3@@QBE?AW4Protocols@12@XZ 120024b0 f i Win32PlatformUtils.obj
 0001:000014b0       ?getTargetNSURIString@SchemaInfo@xercesc_2_3@@QBEQBGXZ 120024b0 f i Win32PlatformUtils.obj
 0001:000014b0       ?getEnumeration@XMLAttDef@xercesc_2_3@@QBEPBGXZ 120024b0 f i Win32PlatformUtils.obj
 0001:000014b0       ?getFragment@XMLUri@xercesc_2_3@@QBEPBGXZ 120024b0 f i Win32PlatformUtils.obj
 0001:000014b0       ?getBaseValidator@DatatypeValidator@xercesc_2_3@@QBEPAV12@XZ 120024b0 f i Win32PlatformUtils.obj
 0001:000014b0       ?getSystemId@XMLEntityDecl@xercesc_2_3@@QBEPBGXZ 120024b0 f i Win32PlatformUtils.obj
 0001:000014b0       ?getIdentityConstraint@XPathMatcher@xercesc_2_3@@QBEPAVIdentityConstraint@2@XZ 120024b0 f i Win32PlatformUtils.obj
 0001:000014b0       ?getString@Context@RegularExpression@xercesc_2_3@@QBEPBGXZ 120024b0 f i Win32PlatformUtils.obj
 0001:000014b0       ?getURI@QName@xercesc_2_3@@QBEIXZ 120024b0 f i Win32PlatformUtils.obj
 0001:000014b0       ?getContentType@ComplexTypeInfo@xercesc_2_3@@QBEHXZ 120024b0 f i Win32PlatformUtils.obj
 0001:000014b0       ?getComplexTypeRegistry@SchemaGrammar@xercesc_2_3@@QBEPAV?$RefHashTableOf@VComplexTypeInfo@xercesc_2_3@@@2@XZ 120024b0 f i Win32PlatformUtils.obj
 0001:000014c0       ?getEnclosingScope@SchemaElementDecl@xercesc_2_3@@QBEHXZ 120024c0 f i Win32PlatformUtils.obj
 0001:000014c0       ?getTypeName@ComplexTypeInfo@xercesc_2_3@@QBEPAGXZ 120024c0 f i Win32PlatformUtils.obj
 0001:000014c0       ?getMemoryManager@XMLAttDef@xercesc_2_3@@QBEPAVMemoryManager@2@XZ 120024c0 f i Win32PlatformUtils.obj
 0001:000014c0       ?getMemoryManager@XPathMatcher@xercesc_2_3@@QBEPAVMemoryManager@2@XZ 120024c0 f i Win32PlatformUtils.obj
 0001:000014c0       ?getContentSpec@DTDElementDecl@xercesc_2_3@@UBEPBVContentSpecNode@2@XZ 120024c0 f i Win32PlatformUtils.obj
 0001:000014c0       ?getEmptyNamespaceId@XMLScanner@xercesc_2_3@@QBEIXZ 120024c0 f i Win32PlatformUtils.obj
 0001:000014c0       ?getQuery@XMLURL@xercesc_2_3@@QBEPBGXZ 120024c0 f i Win32PlatformUtils.obj
 0001:000014c0       ?getFacets@DatatypeValidator@xercesc_2_3@@QBEPAV?$RefHashTableOf@VKVStringPair@xercesc_2_3@@@2@XZ 120024c0 f i Win32PlatformUtils.obj
 0001:000014c0       ?getBaseURI@XMLEntityDecl@xercesc_2_3@@QBEPBGXZ 120024c0 f i Win32PlatformUtils.obj
 0001:000014c0       ?getRoot@SchemaInfo@xercesc_2_3@@QBEPBVDOMElement@2@XZ 120024c0 f i Win32PlatformUtils.obj
 0001:000014c0       ?getContentSpec@DTDElementDecl@xercesc_2_3@@UAEPAVContentSpecNode@2@XZ 120024c0 f i Win32PlatformUtils.obj
 0001:000014c0       ?getCurrentNode@AbstractDOMParser@xercesc_2_3@@IAEPAVDOMNode@2@XZ 120024c0 f i Win32PlatformUtils.obj
 0001:000014c0       ?getGroupInfoRegistry@SchemaGrammar@xercesc_2_3@@QBEPAV?$RefHashTableOf@VXercesGroupInfo@xercesc_2_3@@@2@XZ 120024c0 f i Win32PlatformUtils.obj
 0001:000014d0       ?getElemId@DTDAttDef@xercesc_2_3@@QBEIXZ 120024d0 f i Win32PlatformUtils.obj
 0001:000014d0       ?getUnknownNamespaceId@XMLScanner@xercesc_2_3@@QBEIXZ 120024d0 f i Win32PlatformUtils.obj
 0001:000014d0       ?getNodeIDMap@DOMDocumentImpl@xercesc_2_3@@QAEPAVDOMNodeIDMap@2@XZ 120024d0 f i Win32PlatformUtils.obj
 0001:000014d0       ?getUser@XMLURL@xercesc_2_3@@QBEPBGXZ 120024d0 f i Win32PlatformUtils.obj
 0001:000014d0       ?getEntityResolver@DOMParser@xercesc_2_3@@QBEPBVEntityResolver@2@XZ 120024d0 f i Win32PlatformUtils.obj
 0001:000014d0       ?getElemId@SchemaAttDef@xercesc_2_3@@QBEIXZ 120024d0 f i Win32PlatformUtils.obj
 0001:000014d0       ?getFinalSet@SchemaElementDecl@xercesc_2_3@@QBEHXZ 120024d0 f i Win32PlatformUtils.obj
 0001:000014d0       ?getPattern@DatatypeValidator@xercesc_2_3@@IBEPBGXZ 120024d0 f i Win32PlatformUtils.obj
 0001:000014d0       ?getAttGroupInfoRegistry@SchemaGrammar@xercesc_2_3@@QBEPAV?$RefHashTableOf@VXercesAttGroupInfo@xercesc_2_3@@@2@XZ 120024d0 f i Win32PlatformUtils.obj
 0001:000014d0       ?getMemoryManager@XMLAbstractDoubleFloat@xercesc_2_3@@QBEPAVMemoryManager@2@XZ 120024d0 f i Win32PlatformUtils.obj
 0001:000014d0       ?getMemoryManager@XMLEntityDecl@xercesc_2_3@@QBEPAVMemoryManager@2@XZ 120024d0 f i Win32PlatformUtils.obj
 0001:000014d0       ?getModelType@DTDElementDecl@xercesc_2_3@@QBE?AW4ModelTypes@12@XZ 120024d0 f i Win32PlatformUtils.obj
 0001:000014d0       ?getEntityResolver@DOMParser@xercesc_2_3@@QAEPAVEntityResolver@2@XZ 120024d0 f i Win32PlatformUtils.obj
 0001:000014d0       ?getInitialDepth@SelectorMatcher@xercesc_2_3@@UBEHXZ 120024d0 f i Win32PlatformUtils.obj
 0001:000014d0       ?getValueStore@FieldMatcher@xercesc_2_3@@QBEPAVValueStore@2@XZ 120024d0 f i Win32PlatformUtils.obj
 0001:000014d0       ?getCharData@RegxParser@xercesc_2_3@@QBEHXZ 120024d0 f i Win32PlatformUtils.obj
 0001:000014e0       ?getURLText@XMLURL@xercesc_2_3@@QBEPBGXZ 120024e0 f i Win32PlatformUtils.obj
 0001:00001500       ??0MalformedURLException@xercesc_2_3@@QAE@QBDIW4Codes@XMLExcepts@1@@Z 12002500 f i Win32PlatformUtils.obj
 0001:00001560       ??0MalformedURLException@xercesc_2_3@@QAE@ABV01@@Z 12002560 f i Win32PlatformUtils.obj
 0001:00001580       ??0MalformedURLException@xercesc_2_3@@QAE@QBDIW4Codes@XMLExcepts@1@QBG222@Z 12002580 f i Win32PlatformUtils.obj
 0001:000015f0       ??0MalformedURLException@xercesc_2_3@@QAE@QBDIW4Codes@XMLExcepts@1@0000@Z 120025f0 f i Win32PlatformUtils.obj
 0001:00001660       ??1MalformedURLException@xercesc_2_3@@UAE@XZ 12002660 f i Win32PlatformUtils.obj
 0001:00001670       ?duplicate@MalformedURLException@xercesc_2_3@@UBEPAVXMLException@2@XZ 12002670 f i Win32PlatformUtils.obj
 0001:000016d0       ?getType@MalformedURLException@xercesc_2_3@@UBEPBGXZ 120026d0 f i Win32PlatformUtils.obj
 0001:000016e0       ??_EMalformedURLException@xercesc_2_3@@UAEPAXI@Z 120026e0 f i Win32PlatformUtils.obj
 0001:00001740       ??1XMLNetAccessor@xercesc_2_3@@UAE@XZ 12002740 f i Win32PlatformUtils.obj
 0001:00001750       ??0XMLNetAccessor@xercesc_2_3@@IAE@XZ 12002750 f i Win32PlatformUtils.obj
 0001:00001760       ??_EXMLNetAccessor@xercesc_2_3@@UAEPAXI@Z 12002760 f i Win32PlatformUtils.obj
 0001:000017c0       ??0NetAccessorException@xercesc_2_3@@QAE@QBDIW4Codes@XMLExcepts@1@@Z 120027c0 f i Win32PlatformUtils.obj
 0001:00001820       ??0NetAccessorException@xercesc_2_3@@QAE@ABV01@@Z 12002820 f i Win32PlatformUtils.obj
 0001:00001840       ??0NetAccessorException@xercesc_2_3@@QAE@QBDIW4Codes@XMLExcepts@1@QBG222@Z 12002840 f i Win32PlatformUtils.obj
 0001:000018b0       ??0NetAccessorException@xercesc_2_3@@QAE@QBDIW4Codes@XMLExcepts@1@0000@Z 120028b0 f i Win32PlatformUtils.obj
 0001:00001920       ??1NetAccessorException@xercesc_2_3@@UAE@XZ 12002920 f i Win32PlatformUtils.obj
 0001:00001930       ?duplicate@NetAccessorException@xercesc_2_3@@UBEPAVXMLException@2@XZ 12002930 f i Win32PlatformUtils.obj
 0001:00001990       ?getType@NetAccessorException@xercesc_2_3@@UBEPBGXZ 12002990 f i Win32PlatformUtils.obj
 0001:000019a0       ??_ENetAccessorException@xercesc_2_3@@UAEPAXI@Z 120029a0 f i Win32PlatformUtils.obj
 0001:00001a00       ?getId@WinSockNetAccessor@xercesc_2_3@@UBEPBGXZ 12002a00 f i Win32PlatformUtils.obj
 0001:00001a10       ?panic@XMLPlatformUtils@xercesc_2_3@@SAXW4PanicReasons@PanicHandler@2@@Z 12002a10 f   Win32PlatformUtils.obj
 0001:00001a30       ?curFilePos@XMLPlatformUtils@xercesc_2_3@@SAIPAX@Z 12002a30 f   Win32PlatformUtils.obj
 0001:00001a80       ?closeFile@XMLPlatformUtils@xercesc_2_3@@SAXPAX@Z 12002a80 f   Win32PlatformUtils.obj
 0001:00001ac0       ?fileSize@XMLPlatformUtils@xercesc_2_3@@SAIPAX@Z 12002ac0 f   Win32PlatformUtils.obj
 0001:00001b80       ?openFile@XMLPlatformUtils@xercesc_2_3@@SAPAXQBD@Z 12002b80 f   Win32PlatformUtils.obj
 0001:00001bb0       ?openFile@XMLPlatformUtils@xercesc_2_3@@SAPAXQBG@Z 12002bb0 f   Win32PlatformUtils.obj
 0001:00001d40       ?openFileToWrite@XMLPlatformUtils@xercesc_2_3@@SAPAXQBD@Z 12002d40 f   Win32PlatformUtils.obj
 0001:00001d70       ?openFileToWrite@XMLPlatformUtils@xercesc_2_3@@SAPAXQBG@Z 12002d70 f   Win32PlatformUtils.obj
 0001:00001ea0       ?openStdInHandle@XMLPlatformUtils@xercesc_2_3@@SAPAXXZ 12002ea0 f   Win32PlatformUtils.obj
 0001:00001f60       ?readFileBuffer@XMLPlatformUtils@xercesc_2_3@@SAIPAXIQAE@Z 12002f60 f   Win32PlatformUtils.obj
 0001:00001fd0       ?writeBufferToFile@XMLPlatformUtils@xercesc_2_3@@SAXQAXJQBE@Z 12002fd0 f   Win32PlatformUtils.obj
 0001:00002060       ?resetFile@XMLPlatformUtils@xercesc_2_3@@SAXPAX@Z 12003060 f   Win32PlatformUtils.obj
 0001:000020b0       ?getFullPath@XMLPlatformUtils@xercesc_2_3@@SAPAGQBGQAVMemoryManager@2@@Z 120030b0 f   Win32PlatformUtils.obj
 0001:000022b0       ?isRelative@XMLPlatformUtils@xercesc_2_3@@SA_NQBG@Z 120032b0 f   Win32PlatformUtils.obj
 0001:00002310       ?getCurrentDirectory@XMLPlatformUtils@xercesc_2_3@@SAPAGQAVMemoryManager@2@@Z 12003310 f   Win32PlatformUtils.obj
 0001:00002400       ?isAnySlash@XMLPlatformUtils@xercesc_2_3@@SA_NG@Z 12003400 f i Win32PlatformUtils.obj
 0001:00002430       ?getCurrentMillis@XMLPlatformUtils@xercesc_2_3@@SAKXZ 12003430 f   Win32PlatformUtils.obj
 0001:00002440       ?closeMutex@XMLPlatformUtils@xercesc_2_3@@SAXQAX@Z 12003440 f   Win32PlatformUtils.obj
 0001:00002460       ?lockMutex@XMLPlatformUtils@xercesc_2_3@@SAXQAX@Z 12003460 f   Win32PlatformUtils.obj
 0001:00002470       ?makeMutex@XMLPlatformUtils@xercesc_2_3@@SAPAXXZ 12003470 f   Win32PlatformUtils.obj
 0001:00002490       ?unlockMutex@XMLPlatformUtils@xercesc_2_3@@SAXQAX@Z 12003490 f   Win32PlatformUtils.obj
 0001:000024a0       ?compareAndSwap@XMLPlatformUtils@xercesc_2_3@@SAPAXPAPAXQBX1@Z 120034a0 f   Win32PlatformUtils.obj
 0001:000024c0       ?atomicIncrement@XMLPlatformUtils@xercesc_2_3@@SAHAAH@Z 120034c0 f   Win32PlatformUtils.obj
 0001:000024d0       ?atomicDecrement@XMLPlatformUtils@xercesc_2_3@@SAHAAH@Z 120034d0 f   Win32PlatformUtils.obj
 0001:000024e0       ?makeNetAccessor@XMLPlatformUtils@xercesc_2_3@@CAPAVXMLNetAccessor@2@XZ 120034e0 f   Win32PlatformUtils.obj
 0001:00002540       ?loadAMsgSet@XMLPlatformUtils@xercesc_2_3@@CAPAVXMLMsgLoader@2@QBG@Z 12003540 f   Win32PlatformUtils.obj
 0001:000025a0       ?makeTransService@XMLPlatformUtils@xercesc_2_3@@CAPAVXMLTransService@2@XZ 120035a0 f   Win32PlatformUtils.obj
 0001:00002600       ?platformInit@XMLPlatformUtils@xercesc_2_3@@CAXXZ 12003600 f   Win32PlatformUtils.obj
 0001:00002630       ?weavePaths@XMLPlatformUtils@xercesc_2_3@@SAPAGQBG0@Z 12003630 f   Win32PlatformUtils.obj
 0001:00002740       ?removeDotSlash@XMLPlatformUtils@xercesc_2_3@@SAXQAG@Z 12003740 f   Win32PlatformUtils.obj
 0001:00002880       ?removeDotDotSlash@XMLPlatformUtils@xercesc_2_3@@SAXQAG@Z 12003880 f   Win32PlatformUtils.obj
 0001:00002b10       ?searchSlashDotDotSlash@XMLPlatformUtils@xercesc_2_3@@CAHQAG@Z 12003b10 f   Win32PlatformUtils.obj
 0001:00002bc0       _DllMain@12                12003bc0 f   Win32MsgLoader.obj
 0001:00002be0       ??0Win32MsgLoader@xercesc_2_3@@QAE@QBG@Z 12003be0 f   Win32MsgLoader.obj
 0001:00002e00       ??_EWin32MsgLoader@xercesc_2_3@@UAEPAXI@Z 12003e00 f i Win32MsgLoader.obj
 0001:00002e60       ??1Win32MsgLoader@xercesc_2_3@@UAE@XZ 12003e60 f   Win32MsgLoader.obj
 0001:00002eb0       ?loadMsg@Win32MsgLoader@xercesc_2_3@@UAE_NIQAGI@Z 12003eb0 f   Win32MsgLoader.obj
 0001:00002f60       ?loadMsg@Win32MsgLoader@xercesc_2_3@@UAE_NIQAGIQBG111@Z 12003f60 f   Win32MsgLoader.obj
 0001:00002fb0       ?loadMsg@Win32MsgLoader@xercesc_2_3@@UAE_NIQAGIQBD111@Z 12003fb0 f   Win32MsgLoader.obj
 0001:000030a0       ??0TranscodingException@xercesc_2_3@@QAE@QBDIW4Codes@XMLExcepts@1@@Z 120040a0 f i Win32TransService.obj
 0001:00003100       ??0TranscodingException@xercesc_2_3@@QAE@ABV01@@Z 12004100 f i Win32TransService.obj
 0001:00003120       ??0TranscodingException@xercesc_2_3@@QAE@QBDIW4Codes@XMLExcepts@1@QBG222@Z 12004120 f i Win32TransService.obj
 0001:00003190       ??0TranscodingException@xercesc_2_3@@QAE@QBDIW4Codes@XMLExcepts@1@0000@Z 12004190 f i Win32TransService.obj
 0001:00003200       ??1TranscodingException@xercesc_2_3@@UAE@XZ 12004200 f i Win32TransService.obj
 0001:00003210       ?duplicate@TranscodingException@xercesc_2_3@@UBEPAVXMLException@2@XZ 12004210 f i Win32TransService.obj
 0001:00003270       ?getType@TranscodingException@xercesc_2_3@@UBEPBGXZ 12004270 f i Win32TransService.obj
 0001:00003280       ??_ETranscodingException@xercesc_2_3@@UAEPAXI@Z 12004280 f i Win32TransService.obj
 0001:000032e0       ??0Win32TransService@xercesc_2_3@@QAE@XZ 120042e0 f   Win32TransService.obj
 0001:00003a50       ??_EWin32TransService@xercesc_2_3@@UAEPAXI@Z 12004a50 f i Win32TransService.obj
 0001:00003ab0       ??1Win32TransService@xercesc_2_3@@UAE@XZ 12004ab0 f   Win32TransService.obj
 0001:00003ba0       ?compareIString@Win32TransService@xercesc_2_3@@UAEHQBG0@Z 12004ba0 f   Win32TransService.obj
 0001:00003bc0       ?compareNIString@Win32TransService@xercesc_2_3@@UAEHQBG0I@Z 12004bc0 f   Win32TransService.obj
 0001:00003be0       ?getId@Win32TransService@xercesc_2_3@@UBEPBGXZ 12004be0 f   Win32TransService.obj
 0001:00003bf0       ?isSpace@Win32TransService@xercesc_2_3@@UBE_NG@Z 12004bf0 f   Win32TransService.obj
 0001:00003c10       ?makeNewLCPTranscoder@Win32TransService@xercesc_2_3@@UAEPAVXMLLCPTranscoder@2@XZ 12004c10 f   Win32TransService.obj
 0001:00003c60       ?upperCase@Win32TransService@xercesc_2_3@@UBEXQAG@Z 12004c60 f   Win32TransService.obj
 0001:00003c70       ?lowerCase@Win32TransService@xercesc_2_3@@UBEXQAG@Z 12004c70 f   Win32TransService.obj
 0001:00003c80       ?isAlias@Win32TransService@xercesc_2_3@@CA_NQAUHKEY__@@QADI@Z 12004c80 f   Win32TransService.obj
 0001:00003cb0       ?makeNewXMLTranscoder@Win32TransService@xercesc_2_3@@MAEPAVXMLTranscoder@2@QBGAAW4Codes@XMLTransService@2@IQAVMemoryManager@2@@Z 12004cb0 f   Win32TransService.obj
 0001:00003e30       ??0Win32Transcoder@xercesc_2_3@@QAE@QBGIIIQAVMemoryManager@1@@Z 12004e30 f   Win32TransService.obj
 0001:00003e70       ??_EWin32Transcoder@xercesc_2_3@@UAEPAXI@Z 12004e70 f i Win32TransService.obj
 0001:00003ed0       ??1Win32Transcoder@xercesc_2_3@@UAE@XZ 12004ed0 f   Win32TransService.obj
 0001:00003ee0       ?transcodeFrom@Win32Transcoder@xercesc_2_3@@UAEIQBEIQAGIAAIQAE@Z 12004ee0 f   Win32TransService.obj
 0001:00004010       ?transcodeTo@Win32Transcoder@xercesc_2_3@@UAEIQBGIQAEIAAIW4UnRepOpts@XMLTranscoder@2@@Z 12005010 f   Win32TransService.obj
 0001:000040f0       ?canTranscodeTo@Win32Transcoder@xercesc_2_3@@UBE_NI@Z 120050f0 f   Win32TransService.obj
 0001:00004170       ??0Win32LCPTranscoder@xercesc_2_3@@QAE@XZ 12005170 f   Win32TransService.obj
 0001:00004190       ??_EWin32LCPTranscoder@xercesc_2_3@@UAEPAXI@Z 12005190 f i Win32TransService.obj
 0001:000041f0       ??1Win32LCPTranscoder@xercesc_2_3@@UAE@XZ 120051f0 f   Win32TransService.obj
 0001:00004200       ?calcRequiredSize@Win32LCPTranscoder@xercesc_2_3@@UAEIQBD@Z 12005200 f   Win32TransService.obj
 0001:00004260       ?calcRequiredSize@Win32LCPTranscoder@xercesc_2_3@@UAEIQBG@Z 12005260 f   Win32TransService.obj
 0001:00004290       ?transcode@Win32LCPTranscoder@xercesc_2_3@@UAEPADQBG@Z 12005290 f   Win32TransService.obj
 0001:00004310       ?transcode@Win32LCPTranscoder@xercesc_2_3@@UAEPADQBGQAVMemoryManager@2@@Z 12005310 f   Win32TransService.obj
 0001:00004390       ?transcode@Win32LCPTranscoder@xercesc_2_3@@UAEPAGQBD@Z 12005390 f   Win32TransService.obj
 0001:00004410       ?transcode@Win32LCPTranscoder@xercesc_2_3@@UAEPAGQBDQAVMemoryManager@2@@Z 12005410 f   Win32TransService.obj
 0001:00004490       ?transcode@Win32LCPTranscoder@xercesc_2_3@@UAE_NQBDQAGI@Z 12005490 f   Win32TransService.obj
 0001:000044e0       ?transcode@Win32LCPTranscoder@xercesc_2_3@@UAE_NQBGQADI@Z 120054e0 f   Win32TransService.obj
 0001:00004540       ?Initialize@BinHTTPURLInputStream@xercesc_2_3@@CAXXZ 12005540 f   BinHTTPURLInputStream.obj
 0001:000047c0       ?Cleanup@BinHTTPURLInputStream@xercesc_2_3@@SAXXZ 120057c0 f   BinHTTPURLInputStream.obj
 0001:00004860       ?gethostbyname@BinHTTPURLInputStream@xercesc_2_3@@CAPAUhostent@@PBD@Z 12005860 f i BinHTTPURLInputStream.obj
 0001:00004870       ?inet_addr@BinHTTPURLInputStream@xercesc_2_3@@CAKPBD@Z 12005870 f i BinHTTPURLInputStream.obj
 0001:00004880       ?gethostbyaddr@BinHTTPURLInputStream@xercesc_2_3@@CAPAUhostent@@PBDHH@Z 12005880 f i BinHTTPURLInputStream.obj
 0001:000048a0       ?htons@BinHTTPURLInputStream@xercesc_2_3@@CAGG@Z 120058a0 f i BinHTTPURLInputStream.obj
 0001:000048b0       ?socket@BinHTTPURLInputStream@xercesc_2_3@@CAGHHH@Z 120058b0 f i BinHTTPURLInputStream.obj
 0001:000048d0       ?connect@BinHTTPURLInputStream@xercesc_2_3@@CAHGPBUsockaddr@@H@Z 120058d0 f i BinHTTPURLInputStream.obj
 0001:000048f0       ?send@BinHTTPURLInputStream@xercesc_2_3@@CAHGPBDHH@Z 120058f0 f i BinHTTPURLInputStream.obj
 0001:00004910       ?recv@BinHTTPURLInputStream@xercesc_2_3@@CAHGPADHH@Z 12005910 f i BinHTTPURLInputStream.obj
 0001:00004930       ?shutdown@BinHTTPURLInputStream@xercesc_2_3@@CAHIH@Z 12005930 f i BinHTTPURLInputStream.obj
 0001:00004950       ?closesocket@BinHTTPURLInputStream@xercesc_2_3@@CAHI@Z 12005950 f i BinHTTPURLInputStream.obj
 0001:00004960       ??0BinHTTPURLInputStream@xercesc_2_3@@QAE@ABVXMLURL@1@@Z 12005960 f   BinHTTPURLInputStream.obj
 0001:00005320       ??_EBinHTTPURLInputStream@xercesc_2_3@@UAEPAXI@Z 12006320 f i BinHTTPURLInputStream.obj
 0001:00005380       ??1BinHTTPURLInputStream@xercesc_2_3@@UAE@XZ 12006380 f   BinHTTPURLInputStream.obj
 0001:000053e0       ?readBytes@BinHTTPURLInputStream@xercesc_2_3@@UAEIQAEI@Z 120063e0 f   BinHTTPURLInputStream.obj
 0001:00005480       ??0WinSockNetAccessor@xercesc_2_3@@QAE@XZ 12006480 f   WinSockNetAccessor.obj
 0001:00005490       ??_EWinSockNetAccessor@xercesc_2_3@@UAEPAXI@Z 12006490 f i WinSockNetAccessor.obj
 0001:000054f0       ??1WinSockNetAccessor@xercesc_2_3@@UAE@XZ 120064f0 f   WinSockNetAccessor.obj
 0001:00005540       ?makeNew@WinSockNetAccessor@xercesc_2_3@@UAEPAVBinInputStream@2@ABVXMLURL@2@@Z 12006540 f   WinSockNetAccessor.obj
 0001:00005600       ?getTokenType@Token@xercesc_2_3@@QBEGXZ 12006600 f i ASCIIRangeFactory.obj
 0001:00005600       ?getOpType@Op@xercesc_2_3@@QBEFXZ 12006600 f i ASCIIRangeFactory.obj
 0001:00005610       ?getReferenceNo@Token@xercesc_2_3@@UBEHXZ 12006610 f i ASCIIRangeFactory.obj
 0001:00005610       ?getBaseURI@Wrapper4InputSource@xercesc_2_3@@UBEPBGXZ 12006610 f i ASCIIRangeFactory.obj
 0001:00005610       ?getContentLeafNameTypeVector@MixedContentModel@xercesc_2_3@@UBEPAVContentLeafNameTypeVector@2@XZ 12006610 f i ASCIIRangeFactory.obj
 0001:00005610       ?size@Token@xercesc_2_3@@UBEHXZ 12006610 f i ASCIIRangeFactory.obj
 0001:00005610       ?getDOMTypeInfoName@DTDElementDecl@xercesc_2_3@@UBEPBGXZ 12006610 f i ASCIIRangeFactory.obj
 0001:00005610       ?getRelatedException@DOMErrorImpl@xercesc_2_3@@UBEPAXXZ 12006610 f i ASCIIRangeFactory.obj
 0001:00005610       ?getString@Token@xercesc_2_3@@UBEPBGXZ 12006610 f i ASCIIRangeFactory.obj
 0001:00005610       ?getGrammarType@DTDGrammar@xercesc_2_3@@UBE?AW4GrammarType@Grammar@2@XZ 12006610 f i ASCIIRangeFactory.obj
 0001:00005610       ?getContentLeafNameTypeVector@AllContentModel@xercesc_2_3@@UBEPAVContentLeafNameTypeVector@2@XZ 12006610 f i ASCIIRangeFactory.obj
 0001:00005610       ?getNoParen@Token@xercesc_2_3@@UBEHXZ 12006610 f i ASCIIRangeFactory.obj
 0001:00005610       ?getDOMTypeInfoUri@DTDElementDecl@xercesc_2_3@@UBEPBGXZ 12006610 f i ASCIIRangeFactory.obj
 0001:00005610       ?getDOMTypeInfoUri@DTDAttDef@xercesc_2_3@@UBEPBGXZ 12006610 f i ASCIIRangeFactory.obj
 0001:00005620       ?getChild@Token@xercesc_2_3@@UBEPAV12@H@Z 12006620 f i ASCIIRangeFactory.obj
 0001:00005630       ?getMin@Token@xercesc_2_3@@UBEHXZ 12006630 f i ASCIIRangeFactory.obj
 0001:00005630       ?getChar@Token@xercesc_2_3@@UBEHXZ 12006630 f i ASCIIRangeFactory.obj
 0001:00005630       ?getMax@Token@xercesc_2_3@@UBEHXZ 12006630 f i ASCIIRangeFactory.obj
 0001:00005640       ?setTokenType@Token@xercesc_2_3@@QAEXG@Z 12006640 f i ASCIIRangeFactory.obj
 0001:00005640       ?setOpType@Op@xercesc_2_3@@QAEXF@Z 12006640 f i ASCIIRangeFactory.obj
 0001:00005650       ?addChild@Token@xercesc_2_3@@UAEXQAV12@QAVTokenFactory@2@@Z 12006650 f i ASCIIRangeFactory.obj
 0001:00005680       ?addRange@Token@xercesc_2_3@@UAEXHH@Z 12006680 f i ASCIIRangeFactory.obj
 0001:000056b0       ?mergeRanges@Token@xercesc_2_3@@UAEXQBV12@@Z 120066b0 f i ASCIIRangeFactory.obj
 0001:000056e0       ?sortRanges@Token@xercesc_2_3@@UAEXXZ 120066e0 f i ASCIIRangeFactory.obj
 0001:00005710       ?compactRanges@Token@xercesc_2_3@@UAEXXZ 12006710 f i ASCIIRangeFactory.obj
 0001:00005740       ?subtractRanges@Token@xercesc_2_3@@UAEXQAVRangeToken@2@@Z 12006740 f i ASCIIRangeFactory.obj
 0001:00005770       ?intersectRanges@Token@xercesc_2_3@@UAEXQAVRangeToken@2@@Z 12006770 f i ASCIIRangeFactory.obj
 0001:000057a0       ??_FTokenFactory@xercesc_2_3@@QAEXXZ 120067a0 f i ASCIIRangeFactory.obj
 0001:000057b0       ?getXPath@IC_Selector@xercesc_2_3@@QBEPAVXercesXPath@2@XZ 120067b0 f i ASCIIRangeFactory.obj
 0001:000057b0       ?getId@XMLNotationDecl@xercesc_2_3@@QBEIXZ 120067b0 f i ASCIIRangeFactory.obj
 0001:000057b0       ?getUserDefinedRegistry@DatatypeValidatorFactory@xercesc_2_3@@QBEPAV?$RefHashTableOf@VDatatypeValidator@xercesc_2_3@@@2@XZ 120067b0 f i ASCIIRangeFactory.obj
 0001:000057b0       ?getMemoryManager@QName@xercesc_2_3@@QBEPAVMemoryManager@2@XZ 120067b0 f i ASCIIRangeFactory.obj
 0001:000057b0       ?intValue@XMLInteger@xercesc_2_3@@QBEHXZ 120067b0 f i ASCIIRangeFactory.obj
 0001:000057b0       ?getEntity@EndOfEntityException@xercesc_2_3@@QAEAAVXMLEntityDecl@2@XZ 120067b0 f i ASCIIRangeFactory.obj
 0001:000057b0       ?getMatcherCount@XPathMatcherStack@xercesc_2_3@@QBEIXZ 120067b0 f i ASCIIRangeFactory.obj
 0001:000057b0       ?getEntity@EndOfEntityException@xercesc_2_3@@QBEABVXMLEntityDecl@2@XZ 120067b0 f i ASCIIRangeFactory.obj
 0001:000057b0       ?getCategoryId@RangeTokenElemMap@xercesc_2_3@@QBEIXZ 120067b0 f i ASCIIRangeFactory.obj
 0001:000057b0       ?getSign@XMLBigInteger@xercesc_2_3@@QBEHXZ 120067b0 f i ASCIIRangeFactory.obj
 0001:000057c0       ?getRangeToken@RangeTokenElemMap@xercesc_2_3@@QBEPAVRangeToken@2@_N@Z 120067c0 f i ASCIIRangeFactory.obj
 0001:000057e0       ?setId@XMLNotationDecl@xercesc_2_3@@QAEXI@Z 120067e0 f i ASCIIRangeFactory.obj
 0001:000057e0       ?setEscapeFlags@XMLFormatter@xercesc_2_3@@QAEXW4EscapeFlags@12@@Z 120067e0 f i ASCIIRangeFactory.obj
 0001:000057e0       ?setValueStoreCache@FieldActivator@xercesc_2_3@@QAEXQAVValueStoreCache@2@@Z 120067e0 f i ASCIIRangeFactory.obj
 0001:000057e0       ?setCategoryId@RangeTokenElemMap@xercesc_2_3@@QAEXI@Z 120067e0 f i ASCIIRangeFactory.obj
 0001:000057e0       ?setSign@XMLBigInteger@xercesc_2_3@@AAEXH@Z 120067e0 f i ASCIIRangeFactory.obj
 0001:000057f0       ?setRangeToken@RangeTokenElemMap@xercesc_2_3@@QAEXQAVRangeToken@2@_N@Z 120067f0 f i ASCIIRangeFactory.obj
 0001:00005810       ??0ASCIIRangeFactory@xercesc_2_3@@QAE@XZ 12006810 f   ASCIIRangeFactory.obj
 0001:00005830       ??_EASCIIRangeFactory@xercesc_2_3@@UAEPAXI@Z 12006830 f i ASCIIRangeFactory.obj
 0001:00005890       ??1ASCIIRangeFactory@xercesc_2_3@@UAE@XZ 12006890 f   ASCIIRangeFactory.obj
 0001:000058a0       ?buildRanges@ASCIIRangeFactory@xercesc_2_3@@MAEXXZ 120068a0 f   ASCIIRangeFactory.obj
 0001:000059f0       ?initializeKeywordMap@ASCIIRangeFactory@xercesc_2_3@@UAEXXZ 120069f0 f   ASCIIRangeFactory.obj
 0001:00005a60       ??0BlockRangeFactory@xercesc_2_3@@QAE@XZ 12006a60 f   BlockRangeFactory.obj
 0001:00005a80       ??_EBlockRangeFactory@xercesc_2_3@@UAEPAXI@Z 12006a80 f i BlockRangeFactory.obj
 0001:00005ae0       ??1BlockRangeFactory@xercesc_2_3@@UAE@XZ 12006ae0 f   BlockRangeFactory.obj
 0001:00005af0       ?buildRanges@BlockRangeFactory@xercesc_2_3@@MAEXXZ 12006af0 f   BlockRangeFactory.obj
 0001:00005c90       ?initializeKeywordMap@BlockRangeFactory@xercesc_2_3@@UAEXXZ 12006c90 f   BlockRangeFactory.obj
 0001:00005cd0       ??0BMPattern@xercesc_2_3@@QAE@QBG_NQAVMemoryManager@1@@Z 12006cd0 f   BMPattern.obj
 0001:00005db0       ??0BMPattern@xercesc_2_3@@QAE@QBGH_NQAVMemoryManager@1@@Z 12006db0 f   BMPattern.obj
 0001:00005e90       ?cleanUp@BMPattern@xercesc_2_3@@AAEXXZ 12006e90 f   BMPattern.obj
 0001:00005e90       ??1BMPattern@xercesc_2_3@@QAE@XZ 12006e90 f   BMPattern.obj
 0001:00005ec0       ?matches@BMPattern@xercesc_2_3@@QAEHQBGHH@Z 12006ec0 f   BMPattern.obj
 0001:00006090       ?initialize@BMPattern@xercesc_2_3@@AAEXXZ 12007090 f   BMPattern.obj
 0001:00006240       ?match@CharToken@xercesc_2_3@@QAE_NH@Z 12007240 f i CharToken.obj
 0001:00006260       ??0CharToken@xercesc_2_3@@QAE@GH@Z 12007260 f   CharToken.obj
 0001:00006280       ??_ECharToken@xercesc_2_3@@UAEPAXI@Z 12007280 f i CharToken.obj
 0001:000062e0       ??1CharToken@xercesc_2_3@@UAE@XZ 120072e0 f   CharToken.obj
 0001:000062f0       ?size@ParenToken@xercesc_2_3@@UBEHXZ 120072f0 f i ClosureToken.obj
 0001:000062f0       ?size@ClosureToken@xercesc_2_3@@UBEHXZ 120072f0 f i ClosureToken.obj
 0001:000062f0       ?size@ModifierToken@xercesc_2_3@@UBEHXZ 120072f0 f i ClosureToken.obj
 0001:000062f0       ?getTypeType@SchemaAttDef@xercesc_2_3@@QBE?AW4Complexity@PSVIDefs@2@XZ 120072f0 f i ClosureToken.obj
 0001:000062f0       ?getGrammarType@SchemaGrammar@xercesc_2_3@@UBE?AW4GrammarType@Grammar@2@XZ 120072f0 f i ClosureToken.obj
 0001:00006300       ?getChild@ModifierToken@xercesc_2_3@@UBEPAVToken@2@H@Z 12007300 f i ClosureToken.obj
 0001:00006300       ?getChild@ClosureToken@xercesc_2_3@@UBEPAVToken@2@H@Z 12007300 f i ClosureToken.obj
 0001:00006310       ?setBlockSet@ComplexTypeInfo@xercesc_2_3@@QAEXH@Z 12007310 f i ClosureToken.obj
 0001:00006310       ?setCreateReason@XMLElementDecl@xercesc_2_3@@QAEXW4CreateReasons@12@@Z 12007310 f i ClosureToken.obj
 0001:00006310       ?setEntityHandler@ReaderMgr@xercesc_2_3@@QAEXQAVXMLEntityHandler@2@@Z 12007310 f i ClosureToken.obj
 0001:00006310       ?setOffset@DOMLocatorImpl@xercesc_2_3@@UAEXJ@Z 12007310 f i ClosureToken.obj
 0001:00006310       ?setCreateReason@XMLAttDef@xercesc_2_3@@QAEXW4CreateReasons@12@@Z 12007310 f i ClosureToken.obj
 0001:00006310       ?setUnRepFlags@XMLFormatter@xercesc_2_3@@QAEXW4UnRepFlags@12@@Z 12007310 f i ClosureToken.obj
 0001:00006310       ?setMax@ClosureToken@xercesc_2_3@@UAEXH@Z 12007310 f i ClosureToken.obj
 0001:00006320       ??0ClosureToken@xercesc_2_3@@QAE@GQAVToken@1@@Z 12007320 f   ClosureToken.obj
 0001:00006350       ??_EClosureToken@xercesc_2_3@@UAEPAXI@Z 12007350 f i ClosureToken.obj
 0001:000063b0       ??1ClosureToken@xercesc_2_3@@UAE@XZ 120073b0 f   ClosureToken.obj
 0001:000063c0       ?size@ConcatToken@xercesc_2_3@@UBEHXZ 120073c0 f i ConcatToken.obj
 0001:000063d0       ?getChild@ConcatToken@xercesc_2_3@@UBEPAVToken@2@H@Z 120073d0 f i ConcatToken.obj
 0001:000063f0       ??0ConcatToken@xercesc_2_3@@QAE@QAVToken@1@0@Z 120073f0 f   ConcatToken.obj
 0001:00006420       ??_EConcatToken@xercesc_2_3@@UAEPAXI@Z 12007420 f i ConcatToken.obj
 0001:00006480       ??1ConcatToken@xercesc_2_3@@UAE@XZ 12007480 f   ConcatToken.obj
 0001:00006490       ?size@ConditionToken@xercesc_2_3@@UBEHXZ 12007490 f i ConditionToken.obj
 0001:000064a0       ?getChild@ConditionToken@xercesc_2_3@@UBEPAVToken@2@H@Z 120074a0 f i ConditionToken.obj
 0001:000064f0       ??0ConditionToken@xercesc_2_3@@QAE@IQAVToken@1@00@Z 120074f0 f   ConditionToken.obj
 0001:00006530       ??_EConditionToken@xercesc_2_3@@UAEPAXI@Z 12007530 f i ConditionToken.obj
 0001:00006590       ??1ConditionToken@xercesc_2_3@@UAE@XZ 12007590 f   ConditionToken.obj
 0001:000065a0       ??_FMatch@xercesc_2_3@@QAEXXZ 120075a0 f i Match.obj
 0001:000065c0       ?getNoGroups@Match@xercesc_2_3@@QBEHXZ 120075c0 f i Match.obj
 0001:00006600       ?getStartPos@Match@xercesc_2_3@@QBEHH@Z 12007600 f i Match.obj
 0001:00006670       ?getEndPos@Match@xercesc_2_3@@QBEHH@Z 12007670 f i Match.obj
 0001:000066e0       ?setStartPos@Match@xercesc_2_3@@QAEXHH@Z 120076e0 f i Match.obj
 0001:00006750       ?setEndPos@Match@xercesc_2_3@@QAEXHH@Z 12007750 f i Match.obj
 0001:000067c0       ??0Match@xercesc_2_3@@QAE@QAVMemoryManager@1@@Z 120077c0 f   Match.obj
 0001:000067e0       ??_EMatch@xercesc_2_3@@UAEPAXI@Z 120077e0 f i Match.obj
 0001:00006860       ??0Match@xercesc_2_3@@QAE@ABV01@@Z 12007860 f   Match.obj
 0001:00006af0       ??4Match@xercesc_2_3@@QAEAAV01@ABV01@@Z 12007af0 f   Match.obj
 0001:00006d70       ??1Match@xercesc_2_3@@UAE@XZ 12007d70 f   Match.obj
 0001:00006da0       ?setNoGroups@Match@xercesc_2_3@@QAEXH@Z 12007da0 f   Match.obj
 0001:00006e30       ?initialize@Match@xercesc_2_3@@AAEXABV12@@Z 12007e30 f   Match.obj
 0001:000070b0       ?cleanUp@Match@xercesc_2_3@@AAEXXZ 120080b0 f   Match.obj
 0001:000070e0       ??0ModifierToken@xercesc_2_3@@QAE@QAVToken@1@HH@Z 120080e0 f   ModifierToken.obj
 0001:00007110       ??_EModifierToken@xercesc_2_3@@UAEPAXI@Z 12008110 f i ModifierToken.obj
 0001:00007170       ??1ModifierToken@xercesc_2_3@@UAE@XZ 12008170 f   ModifierToken.obj
 0001:00007180       ??0Op@xercesc_2_3@@AAE@ABV01@@Z 12008180 f i Op.obj
 0001:000071b0       ??4Op@xercesc_2_3@@AAEAAV01@ABV01@@Z 120081b0 f i Op.obj
 0001:000071e0       ??_EOp@xercesc_2_3@@UAEPAXI@Z 120081e0 f i Op.obj
 0001:00007240       ??1UnionOp@xercesc_2_3@@UAE@XZ 12008240 f i Op.obj
 0001:00007290       ??_EUnionOp@xercesc_2_3@@UAEPAXI@Z 12008290 f i Op.obj
 0001:000072f0       ??_EModifierOp@xercesc_2_3@@UAEPAXI@Z 120082f0 f i Op.obj
 0001:00007350       ??_ECharOp@xercesc_2_3@@UAEPAXI@Z 12008350 f i Op.obj
 0001:00007350       ??_ERangeOp@xercesc_2_3@@UAEPAXI@Z 12008350 f i Op.obj
 0001:00007350       ??_EChildOp@xercesc_2_3@@UAEPAXI@Z 12008350 f i Op.obj
 0001:000073b0       ??1StringOp@xercesc_2_3@@UAE@XZ 120083b0 f i Op.obj
 0001:00007400       ??_EStringOp@xercesc_2_3@@UAEPAXI@Z 12008400 f i Op.obj
 0001:00007460       ??1ModifierOp@xercesc_2_3@@UAE@XZ 12008460 f i Op.obj
 0001:00007460       ??1ChildOp@xercesc_2_3@@UAE@XZ 12008460 f i Op.obj
 0001:00007460       ??1CharOp@xercesc_2_3@@UAE@XZ 12008460 f i Op.obj
 0001:00007460       ??1ConditionOp@xercesc_2_3@@UAE@XZ 12008460 f i Op.obj
 0001:00007460       ??1Op@xercesc_2_3@@UAE@XZ  12008460 f i Op.obj
 0001:00007460       ??1RangeOp@xercesc_2_3@@UAE@XZ 12008460 f i Op.obj
 0001:00007470       ??_EConditionOp@xercesc_2_3@@UAEPAXI@Z 12008470 f i Op.obj
 0001:000074d0       ??0Op@xercesc_2_3@@IAE@F@Z 120084d0 f   Op.obj
 0001:000074f0       ?getSize@Op@xercesc_2_3@@UBEHXZ 120084f0 f   Op.obj
 0001:00007520       ?getData@Op@xercesc_2_3@@UBEHXZ 12008520 f   Op.obj
 0001:00007550       ?getData2@Op@xercesc_2_3@@UBEHXZ 12008550 f   Op.obj
 0001:00007580       ?getRefNo@Op@xercesc_2_3@@UBEHXZ 12008580 f   Op.obj
 0001:000075b0       ?elementAt@Op@xercesc_2_3@@UBEPBV12@H@Z 120085b0 f   Op.obj
 0001:000075e0       ?getChild@Op@xercesc_2_3@@UBEPBV12@XZ 120085e0 f   Op.obj
 0001:00007610       ?getConditionFlow@Op@xercesc_2_3@@UBEPBV12@XZ 12008610 f   Op.obj
 0001:00007640       ?getYesFlow@Op@xercesc_2_3@@UBEPBV12@XZ 12008640 f   Op.obj
 0001:00007670       ?getNoFlow@Op@xercesc_2_3@@UBEPBV12@XZ 12008670 f   Op.obj
 0001:000076a0       ?getLiteral@Op@xercesc_2_3@@UBEPBGXZ 120086a0 f   Op.obj
 0001:000076d0       ?getToken@Op@xercesc_2_3@@UBEPBVToken@2@XZ 120086d0 f   Op.obj
 0001:00007700       ??0CharOp@xercesc_2_3@@QAE@FH@Z 12008700 f   Op.obj
 0001:00007730       ??0UnionOp@xercesc_2_3@@QAE@FHQAVMemoryManager@1@@Z 12008730 f   Op.obj
 0001:00007800       ?getSize@UnionOp@xercesc_2_3@@UBEHXZ 12008800 f   Op.obj
 0001:00007810       ?elementAt@UnionOp@xercesc_2_3@@UBEPBVOp@2@H@Z 12008810 f   Op.obj
 0001:00007860       ?addElement@UnionOp@xercesc_2_3@@QAEXQAVOp@2@@Z 12008860 f   Op.obj
 0001:000078f0       ??0ChildOp@xercesc_2_3@@QAE@F@Z 120088f0 f   Op.obj
 0001:00007910       ??0ModifierOp@xercesc_2_3@@QAE@FHH@Z 12008910 f   Op.obj
 0001:00007940       ??0RangeOp@xercesc_2_3@@QAE@FQBVToken@1@@Z 12008940 f   Op.obj
 0001:00007970       ??0StringOp@xercesc_2_3@@QAE@FQBG@Z 12008970 f   Op.obj
 0001:00007a10       ??0ConditionOp@xercesc_2_3@@QAE@FHQBVOp@1@00@Z 12008a10 f   Op.obj
 0001:00007a50       ??_G?$RefVectorOf@VOp@xercesc_2_3@@@xercesc_2_3@@UAEPAXI@Z 12008a50 f i Op.obj
 0001:00007a50       ??_E?$RefVectorOf@VOp@xercesc_2_3@@@xercesc_2_3@@UAEPAXI@Z 12008a50 f i Op.obj
 0001:00007a70       ??1?$RefVectorOf@VOp@xercesc_2_3@@@xercesc_2_3@@UAE@XZ 12008a70 f i Op.obj
 0001:00007af0       ??1?$BaseRefVectorOf@VOp@xercesc_2_3@@@xercesc_2_3@@UAE@XZ 12008af0 f i Op.obj
 0001:00007b00       ??_FOpFactory@xercesc_2_3@@QAEXXZ 12008b00 f i OpFactory.obj
 0001:00007b10       ?reset@OpFactory@xercesc_2_3@@QAEXXZ 12008b10 f i OpFactory.obj
 0001:00007b50       ??0OpFactory@xercesc_2_3@@QAE@QAVMemoryManager@1@@Z 12008b50 f   OpFactory.obj
 0001:00007bf0       ??1OpFactory@xercesc_2_3@@QAE@XZ 12008bf0 f   OpFactory.obj
 0001:00007c10       ?createDotOp@OpFactory@xercesc_2_3@@QAEPAVOp@2@XZ 12008c10 f   OpFactory.obj
 0001:00007cf0       ?createCharOp@OpFactory@xercesc_2_3@@QAEPAVCharOp@2@H@Z 12008cf0 f   OpFactory.obj
 0001:00007de0       ?createAnchorOp@OpFactory@xercesc_2_3@@QAEPAVCharOp@2@H@Z 12008de0 f   OpFactory.obj
 0001:00007ed0       ?createCaptureOp@OpFactory@xercesc_2_3@@QAEPAVCharOp@2@HQBVOp@2@@Z 12008ed0 f   OpFactory.obj
 0001:00007fd0       ?createUnionOp@OpFactory@xercesc_2_3@@QAEPAVUnionOp@2@H@Z 12008fd0 f   OpFactory.obj
 0001:000080c0       ?createClosureOp@OpFactory@xercesc_2_3@@QAEPAVChildOp@2@H@Z 120090c0 f   OpFactory.obj
 0001:000081b0       ?createNonGreedyClosureOp@OpFactory@xercesc_2_3@@QAEPAVChildOp@2@XZ 120091b0 f   OpFactory.obj
 0001:000082a0       ?createQuestionOp@OpFactory@xercesc_2_3@@QAEPAVChildOp@2@_N@Z 120092a0 f   OpFactory.obj
 0001:00008390       ?createRangeOp@OpFactory@xercesc_2_3@@QAEPAVRangeOp@2@QBVToken@2@@Z 12009390 f   OpFactory.obj
 0001:00008480       ?createLookOp@OpFactory@xercesc_2_3@@QAEPAVChildOp@2@FQBVOp@2@0@Z 12009480 f   OpFactory.obj
 0001:00008590       ?createBackReferenceOp@OpFactory@xercesc_2_3@@QAEPAVCharOp@2@H@Z 12009590 f   OpFactory.obj
 0001:00008680       ?createStringOp@OpFactory@xercesc_2_3@@QAEPAVStringOp@2@QBG@Z 12009680 f   OpFactory.obj
 0001:00008770       ?createIndependentOp@OpFactory@xercesc_2_3@@QAEPAVChildOp@2@QBVOp@2@0@Z 12009770 f   OpFactory.obj
 0001:00008870       ?createModifierOp@OpFactory@xercesc_2_3@@QAEPAVModifierOp@2@QBVOp@2@0HH@Z 12009870 f   OpFactory.obj
 0001:000088f0       ?createConditionOp@OpFactory@xercesc_2_3@@QAEPAVConditionOp@2@QBVOp@2@H000@Z 120098f0 f   OpFactory.obj
 0001:00008980       ?getChild@ParenToken@xercesc_2_3@@UBEPAVToken@2@H@Z 12009980 f i ParenToken.obj
 0001:00008990       ??0ParenToken@xercesc_2_3@@QAE@GQAVToken@1@H@Z 12009990 f   ParenToken.obj
 0001:000089c0       ??_EParenToken@xercesc_2_3@@UAEPAXI@Z 120099c0 f i ParenToken.obj
 0001:00008a20       ??1ParenToken@xercesc_2_3@@UAE@XZ 12009a20 f   ParenToken.obj
 0001:00008a30       ??_FRegxParser@xercesc_2_3@@QAEXXZ 12009a30 f i ParserForXMLSchema.obj
 0001:00008a40       ?getParseContext@RegxParser@xercesc_2_3@@QBEGXZ 12009a40 f i ParserForXMLSchema.obj
 0001:00008a50       ?getState@RegxParser@xercesc_2_3@@QBEGXZ 12009a50 f i ParserForXMLSchema.obj
 0001:00008a60       ?hasBackReferences@RegxParser@xercesc_2_3@@QBE_NXZ 12009a60 f i ParserForXMLSchema.obj
 0001:00008a60       ?getAnonymous@DatatypeValidator@xercesc_2_3@@QBE_NXZ 12009a60 f i ParserForXMLSchema.obj
 0001:00008a60       ?getValidationConstraintFatal@XMLScanner@xercesc_2_3@@QBE_NXZ 12009a60 f i ParserForXMLSchema.obj
 0001:00008a70       ?getDatatypeValidator@ComplexTypeInfo@xercesc_2_3@@QBEPAVDatatypeValidator@2@XZ 12009a70 f i ParserForXMLSchema.obj
 0001:00008a70       ?getIDRefList@SchemaGrammar@xercesc_2_3@@QBEPAV?$RefHashTableOf@VXMLRefInfo@xercesc_2_3@@@2@XZ 12009a70 f i ParserForXMLSchema.obj
 0001:00008a70       ?getScanner@DOMParser@xercesc_2_3@@QBEABVXMLScanner@2@XZ 12009a70 f i ParserForXMLSchema.obj
 0001:00008a70       ?getDefaultValue@SchemaElementDecl@xercesc_2_3@@QBEPAGXZ 12009a70 f i ParserForXMLSchema.obj
 0001:00008a70       ?getTypeName@DatatypeValidator@xercesc_2_3@@QBEPBGXZ 12009a70 f i ParserForXMLSchema.obj
 0001:00008a70       ?getTokenFactory@RegxParser@xercesc_2_3@@QBEPAVTokenFactory@2@XZ 12009a70 f i ParserForXMLSchema.obj
 0001:00008a70       ?getTypeLocalName@DatatypeValidator@xercesc_2_3@@QBEPBGXZ 12009a70 f i ParserForXMLSchema.obj
 0001:00008a80       ?setParseContext@RegxParser@xercesc_2_3@@QAEXG@Z 12009a80 f i ParserForXMLSchema.obj
 0001:00008a90       ?setDatatypeValidator@ComplexTypeInfo@xercesc_2_3@@QAEXQAVDatatypeValidator@2@@Z 12009a90 f i ParserForXMLSchema.obj
 0001:00008a90       ?setTokenFactory@RegxParser@xercesc_2_3@@QAEXQAVTokenFactory@2@@Z 12009a90 f i ParserForXMLSchema.obj
 0001:00008a90       ?setAnyDatatypeValidator@SchemaAttDef@xercesc_2_3@@QAEXPAVDatatypeValidator@2@@Z 12009a90 f i ParserForXMLSchema.obj
 0001:00008aa0       ?isSet@RegxParser@xercesc_2_3@@AAE_NH@Z 12009aa0 f i ParserForXMLSchema.obj
 0001:00008ac0       ?hexChar@RegxParser@xercesc_2_3@@AAEHH@Z 12009ac0 f i ParserForXMLSchema.obj
 0001:00008b00       ??_FParserForXMLSchema@xercesc_2_3@@QAEXXZ 12009b00 f i ParserForXMLSchema.obj
 0001:00008b10       ?setString@StringToken@xercesc_2_3@@QAEXQBG@Z 12009b10 f i ParserForXMLSchema.obj
 0001:00008b80       ?size@UnionToken@xercesc_2_3@@UBEHXZ 12009b80 f i ParserForXMLSchema.obj
 0001:00008b90       ??0ParseException@xercesc_2_3@@QAE@QBDIW4Codes@XMLExcepts@1@@Z 12009b90 f i ParserForXMLSchema.obj
 0001:00008bf0       ??0ParseException@xercesc_2_3@@QAE@ABV01@@Z 12009bf0 f i ParserForXMLSchema.obj
 0001:00008c10       ??0ParseException@xercesc_2_3@@QAE@QBDIW4Codes@XMLExcepts@1@QBG222@Z 12009c10 f i ParserForXMLSchema.obj
 0001:00008c80       ??0ParseException@xercesc_2_3@@QAE@QBDIW4Codes@XMLExcepts@1@0000@Z 12009c80 f i ParserForXMLSchema.obj
 0001:00008cf0       ??1ParseException@xercesc_2_3@@UAE@XZ 12009cf0 f i ParserForXMLSchema.obj
 0001:00008d00       ?duplicate@ParseException@xercesc_2_3@@UBEPAVXMLException@2@XZ 12009d00 f i ParserForXMLSchema.obj
 0001:00008d60       ?getType@ParseException@xercesc_2_3@@UBEPBGXZ 12009d60 f i ParserForXMLSchema.obj
 0001:00008d70       ??_EParseException@xercesc_2_3@@UAEPAXI@Z 12009d70 f i ParserForXMLSchema.obj
 0001:00008dd0       ??0ParserForXMLSchema@xercesc_2_3@@QAE@QAVMemoryManager@1@@Z 12009dd0 f   ParserForXMLSchema.obj
 0001:00008df0       ??_EParserForXMLSchema@xercesc_2_3@@UAEPAXI@Z 12009df0 f i ParserForXMLSchema.obj
 0001:00008e50       ??1ParserForXMLSchema@xercesc_2_3@@UAE@XZ 12009e50 f   ParserForXMLSchema.obj
 0001:00008e60       ?processCaret@ParserForXMLSchema@xercesc_2_3@@MAEPAVToken@2@XZ 12009e60 f   ParserForXMLSchema.obj
 0001:00008e80       ?processDollar@ParserForXMLSchema@xercesc_2_3@@MAEPAVToken@2@XZ 12009e80 f   ParserForXMLSchema.obj
 0001:00008ea0       ?processPlus@ParserForXMLSchema@xercesc_2_3@@MAEPAVToken@2@QAV32@@Z 12009ea0 f   ParserForXMLSchema.obj
 0001:00008ed0       ?processStar@ParserForXMLSchema@xercesc_2_3@@MAEPAVToken@2@QAV32@@Z 12009ed0 f   ParserForXMLSchema.obj
 0001:00008ef0       ?processQuestion@ParserForXMLSchema@xercesc_2_3@@MAEPAVToken@2@QAV32@@Z 12009ef0 f   ParserForXMLSchema.obj
 0001:00008f30       ?processParen@ParserForXMLSchema@xercesc_2_3@@MAEPAVToken@2@XZ 12009f30 f   ParserForXMLSchema.obj
 0001:00008f90       ?parseCharacterClass@ParserForXMLSchema@xercesc_2_3@@MAEPAVRangeToken@2@_N@Z 12009f90 f   ParserForXMLSchema.obj
 0001:000093f0       ?processCInCharacterClass@ParserForXMLSchema@xercesc_2_3@@MAEHQAVRangeToken@2@H@Z 1200a3f0 f   ParserForXMLSchema.obj
 0001:00009410       ?processLook@ParserForXMLSchema@xercesc_2_3@@MAEPAVToken@2@G@Z 1200a410 f   ParserForXMLSchema.obj
 0001:00009440       ?processBacksolidus_A@ParserForXMLSchema@xercesc_2_3@@MAEPAVToken@2@XZ 1200a440 f   ParserForXMLSchema.obj
 0001:00009470       ?processBacksolidus_B@ParserForXMLSchema@xercesc_2_3@@MAEPAVToken@2@XZ 1200a470 f   ParserForXMLSchema.obj
 0001:000094a0       ?processBacksolidus_b@ParserForXMLSchema@xercesc_2_3@@MAEPAVToken@2@XZ 1200a4a0 f   ParserForXMLSchema.obj
 0001:000094d0       ?processBacksolidus_C@ParserForXMLSchema@xercesc_2_3@@MAEPAVToken@2@XZ 1200a4d0 f   ParserForXMLSchema.obj
 0001:000094f0       ?processBacksolidus_c@ParserForXMLSchema@xercesc_2_3@@MAEPAVToken@2@XZ 1200a4f0 f   ParserForXMLSchema.obj
 0001:00009510       ?processBacksolidus_g@ParserForXMLSchema@xercesc_2_3@@MAEPAVToken@2@XZ 1200a510 f   ParserForXMLSchema.obj
 0001:00009540       ?processBacksolidus_gt@ParserForXMLSchema@xercesc_2_3@@MAEPAVToken@2@XZ 1200a540 f   ParserForXMLSchema.obj
 0001:00009570       ?processBacksolidus_I@ParserForXMLSchema@xercesc_2_3@@MAEPAVToken@2@XZ 1200a570 f   ParserForXMLSchema.obj
 0001:00009590       ?processBacksolidus_i@ParserForXMLSchema@xercesc_2_3@@MAEPAVToken@2@XZ 1200a590 f   ParserForXMLSchema.obj
 0001:000095b0       ?processBacksolidus_lt@ParserForXMLSchema@xercesc_2_3@@MAEPAVToken@2@XZ 1200a5b0 f   ParserForXMLSchema.obj
 0001:000095e0       ?processBacksolidus_X@ParserForXMLSchema@xercesc_2_3@@MAEPAVToken@2@XZ 1200a5e0 f   ParserForXMLSchema.obj
 0001:00009610       ?processBacksolidus_Z@ParserForXMLSchema@xercesc_2_3@@MAEPAVToken@2@XZ 1200a610 f   ParserForXMLSchema.obj
 0001:00009640       ?processBacksolidus_z@ParserForXMLSchema@xercesc_2_3@@MAEPAVToken@2@XZ 1200a640 f   ParserForXMLSchema.obj
 0001:00009670       ?processBackReference@ParserForXMLSchema@xercesc_2_3@@MAEPAVToken@2@XZ 1200a670 f   ParserForXMLSchema.obj
 0001:000096a0       ?processCondition@ParserForXMLSchema@xercesc_2_3@@MAEPAVToken@2@XZ 1200a6a0 f   ParserForXMLSchema.obj
 0001:000096d0       ?processIndependent@ParserForXMLSchema@xercesc_2_3@@MAEPAVToken@2@XZ 1200a6d0 f   ParserForXMLSchema.obj
 0001:00009700       ?processModifiers@ParserForXMLSchema@xercesc_2_3@@MAEPAVToken@2@XZ 1200a700 f   ParserForXMLSchema.obj
 0001:00009730       ?processParen2@ParserForXMLSchema@xercesc_2_3@@MAEPAVToken@2@XZ 1200a730 f   ParserForXMLSchema.obj
 0001:00009760       ?parseSetOperations@ParserForXMLSchema@xercesc_2_3@@MAEPAVRangeToken@2@XZ 1200a760 f   ParserForXMLSchema.obj
 0001:00009790       ?getTokenForShorthand@ParserForXMLSchema@xercesc_2_3@@MAEPAVToken@2@H@Z 1200a790 f   ParserForXMLSchema.obj
 0001:000098d0       ?checkQuestion@ParserForXMLSchema@xercesc_2_3@@MAE_NH@Z 1200a8d0 f   ParserForXMLSchema.obj
 0001:000098e0       ?decodeEscaped@ParserForXMLSchema@xercesc_2_3@@MAEHXZ 1200a8e0 f   ParserForXMLSchema.obj
 0001:00009a00       ??0RangeFactory@xercesc_2_3@@IAE@XZ 1200aa00 f   RangeFactory.obj
 0001:00009a10       ??_ERangeFactory@xercesc_2_3@@UAEPAXI@Z 1200aa10 f i RangeFactory.obj
 0001:00009a70       ??1RangeFactory@xercesc_2_3@@UAE@XZ 1200aa70 f   RangeFactory.obj
 0001:00009a80       ??0RangeToken@xercesc_2_3@@QAE@GQAVMemoryManager@1@@Z 1200aa80 f   RangeToken.obj
 0001:00009ac0       ??_ERangeToken@xercesc_2_3@@UAEPAXI@Z 1200aac0 f i RangeToken.obj
 0001:00009b20       ??1RangeToken@xercesc_2_3@@UAE@XZ 1200ab20 f   RangeToken.obj
 0001:00009b90       ?getCaseInsensitiveToken@RangeToken@xercesc_2_3@@QAEPAV12@QAVTokenFactory@2@@Z 1200ab90 f   RangeToken.obj
 0001:00009bd0       ?setRangeValues@RangeToken@xercesc_2_3@@QAEXQAHI@Z 1200abd0 f   RangeToken.obj
 0001:00009c20       ?addRange@RangeToken@xercesc_2_3@@UAEXHH@Z 1200ac20 f   RangeToken.obj
 0001:00009d50       ?sortRanges@RangeToken@xercesc_2_3@@UAEXXZ 1200ad50 f   RangeToken.obj
 0001:00009e00       ?compactRanges@RangeToken@xercesc_2_3@@UAEXXZ 1200ae00 f   RangeToken.obj
 0001:00009ee0       ?mergeRanges@RangeToken@xercesc_2_3@@UAEXQBVToken@2@@Z 1200aee0 f   RangeToken.obj
 0001:0000a0e0       ?subtractRanges@RangeToken@xercesc_2_3@@UAEXQAV12@@Z 1200b0e0 f   RangeToken.obj
 0001:0000a280       ?intersectRanges@RangeToken@xercesc_2_3@@UAEXQAV12@@Z 1200b280 f   RangeToken.obj
 0001:0000a3e0       ?complementRanges@RangeToken@xercesc_2_3@@SAPAVToken@2@QAV12@QAVTokenFactory@2@@Z 1200b3e0 f   RangeToken.obj
 0001:0000a4b0       ?match@RangeToken@xercesc_2_3@@QAE_NH@Z 1200b4b0 f   RangeToken.obj
 0001:0000a5b0       ?expand@RangeToken@xercesc_2_3@@AAEXI@Z 1200b5b0 f   RangeToken.obj
 0001:0000a640       ?createMap@RangeToken@xercesc_2_3@@AAEXXZ 1200b640 f   RangeToken.obj
 0001:0000a6e0       ??_FXMLStringPool@xercesc_2_3@@QAEXXZ 1200b6e0 f i RangeTokenMap.obj
 0001:0000a6f0       ??0RangeTokenElemMap@xercesc_2_3@@QAE@I@Z 1200b6f0 f   RangeTokenMap.obj
 0001:0000a710       ??0RangeTokenMap@xercesc_2_3@@IAE@XZ 1200b710 f   RangeTokenMap.obj
 0001:0000a730       ??1RangeTokenMap@xercesc_2_3@@IAE@XZ 1200b730 f   RangeTokenMap.obj
 0001:0000a8a0       ?getRange@RangeTokenMap@xercesc_2_3@@IAEPAVRangeToken@2@QBG_N@Z 1200b8a0 f   RangeTokenMap.obj
 0001:0000aa20       ?addCategory@RangeTokenMap@xercesc_2_3@@QAEXQBG@Z 1200ba20 f   RangeTokenMap.obj
 0001:0000aa40       ?addRangeMap@RangeTokenMap@xercesc_2_3@@QAEXQBGQAVRangeFactory@2@@Z 1200ba40 f   RangeTokenMap.obj
 0001:0000aa60       ?addKeywordMap@RangeTokenMap@xercesc_2_3@@QAEXQBG0@Z 1200ba60 f   RangeTokenMap.obj
 0001:0000ad00       ?setRangeToken@RangeTokenMap@xercesc_2_3@@QAEXQBGQAVRangeToken@2@_N@Z 1200bd00 f   RangeTokenMap.obj
 0001:0000ae40       ?initializeRegistry@RangeTokenMap@xercesc_2_3@@AAEXXZ 1200be40 f   RangeTokenMap.obj
 0001:0000b030       ?instance@RangeTokenMap@xercesc_2_3@@SAPAV12@XZ 1200c030 f   RangeTokenMap.obj
 0001:0000b200       ?reinitInstance@RangeTokenMap@xercesc_2_3@@SAXXZ 1200c200 f   RangeTokenMap.obj
 0001:0000b230       ??1?$RefHashTableOf@V?$KeyRefPair@XVDOMUserDataHandler@xercesc_2_3@@@xercesc_2_3@@@xercesc_2_3@@QAE@XZ 1200c230 f i RangeTokenMap.obj
 0001:0000b230       ??1?$RefHashTableOf@VRangeTokenElemMap@xercesc_2_3@@@xercesc_2_3@@QAE@XZ 1200c230 f i RangeTokenMap.obj
 0001:0000b2b0       ??1?$RefHashTableOf@VRangeFactory@xercesc_2_3@@@xercesc_2_3@@QAE@XZ 1200c2b0 f i RangeTokenMap.obj
 0001:0000b330       ?put@?$RefHashTableOf@VRangeFactory@xercesc_2_3@@@xercesc_2_3@@QAEXPAXQAVRangeFactory@2@@Z 1200c330 f i RangeTokenMap.obj
 0001:0000b540       ??_FContext@RegularExpression@xercesc_2_3@@QAEXXZ 1200c540 f i RegularExpression.obj
 0001:0000b570       ?cleanUp@RegularExpression@xercesc_2_3@@AAEXXZ 1200c570 f i RegularExpression.obj
 0001:0000b600       ?isSet@RegularExpression@xercesc_2_3@@AAE_NHH@Z 1200c600 f i RegularExpression.obj
 0001:0000b600       ?isSet@Token@xercesc_2_3@@AAE_NHI@Z 1200c600 f i RegularExpression.obj
 0001:0000b620       ?compileLook@RegularExpression@xercesc_2_3@@AAEPAVOp@2@QBVToken@2@QBV32@_NG@Z 1200c620 f i RegularExpression.obj
 0001:0000b710       ?compileSingle@RegularExpression@xercesc_2_3@@AAEPAVOp@2@QBVToken@2@QAV32@G@Z 1200c710 f i RegularExpression.obj
 0001:0000b7f0       ?compileUnion@RegularExpression@xercesc_2_3@@AAEPAVOp@2@QBVToken@2@QAV32@_N@Z 1200c7f0 f i RegularExpression.obj
 0001:0000b850       ?compileCondition@RegularExpression@xercesc_2_3@@AAEPAVOp@2@QBVToken@2@QAV32@_N@Z 1200c850 f i RegularExpression.obj
 0001:0000b8f0       ?compileParenthesis@RegularExpression@xercesc_2_3@@AAEPAVOp@2@QBVToken@2@QAV32@_N@Z 1200c8f0 f i RegularExpression.obj
 0001:0000b9c0       ?compileConcat@RegularExpression@xercesc_2_3@@AAEPAVOp@2@QBVToken@2@QAV32@_N@Z 1200c9c0 f i RegularExpression.obj
 0001:0000ba40       ?compileClosure@RegularExpression@xercesc_2_3@@AAEPAVOp@2@QBVToken@2@QAV32@_NG@Z 1200ca40 f i RegularExpression.obj
 0001:0000bb70       ?matchUnion@RegularExpression@xercesc_2_3@@AAEHQAVContext@12@QBVOp@2@HF@Z 1200cb70 f i RegularExpression.obj
 0001:0000bbd0       ?matchModifier@RegularExpression@xercesc_2_3@@AAEHQAVContext@12@QBVOp@2@HF@Z 1200cbd0 f i RegularExpression.obj
 0001:0000bc20       ?getWordType@RegularExpression@xercesc_2_3@@AAEGQBGHHH@Z 1200cc20 f i RegularExpression.obj
 0001:0000bc50       ?getPreviousWordType@RegularExpression@xercesc_2_3@@AAEGQBGHHH@Z 1200cc50 f i RegularExpression.obj
 0001:0000bcc0       ?matchIgnoreCase@RegularExpression@xercesc_2_3@@AAE_NHH@Z 1200ccc0 f i RegularExpression.obj
 0001:0000bce0       ?isEOLChar@RegxUtil@xercesc_2_3@@SA_NG@Z 1200cce0 f i RegularExpression.obj
 0001:0000bd10       ?composeFromSurrogate@RegxUtil@xercesc_2_3@@SAHGG@Z 1200cd10 f i RegularExpression.obj
 0001:0000bd30       ?isLowSurrogate@RegxUtil@xercesc_2_3@@SA_NG@Z 1200cd30 f i RegularExpression.obj
 0001:0000bd50       ?isHighSurrogate@RegxUtil@xercesc_2_3@@SA_NG@Z 1200cd50 f i RegularExpression.obj
 0001:0000bd70       ?isWordChar@RegxUtil@xercesc_2_3@@SA_NG@Z 1200cd70 f i RegularExpression.obj
 0001:0000bdb0       ??0XMLBuffer@xercesc_2_3@@QAE@HQAVMemoryManager@1@@Z 1200cdb0 f i RegularExpression.obj
 0001:0000bdf0       ??1XMLBuffer@xercesc_2_3@@QAE@XZ 1200cdf0 f i RegularExpression.obj
 0001:0000be00       ?append@XMLBuffer@xercesc_2_3@@QAEXG@Z 1200ce00 f i RegularExpression.obj
 0001:0000be30       ?getRawBuffer@XMLBuffer@xercesc_2_3@@QBEPBGXZ 1200ce30 f i RegularExpression.obj
 0001:0000be30       ?getRawBuffer@XMLBuffer@xercesc_2_3@@QAEPAGXZ 1200ce30 f i RegularExpression.obj
 0001:0000be40       ?reset@XMLBuffer@xercesc_2_3@@QAEXXZ 1200ce40 f i RegularExpression.obj
 0001:0000be50       ?isEmpty@XMLBuffer@xercesc_2_3@@QBE_NXZ 1200ce50 f i RegularExpression.obj
 0001:0000be60       ??_FXMLBuffer@xercesc_2_3@@QAEXXZ 1200ce60 f i RegularExpression.obj
 0001:0000bea0       ??0Context@RegularExpression@xercesc_2_3@@QAE@QAVMemoryManager@2@@Z 1200cea0 f   RegularExpression.obj
 0001:0000bed0       ??1Context@RegularExpression@xercesc_2_3@@QAE@XZ 1200ced0 f   RegularExpression.obj
 0001:0000bf10       ?reset@Context@RegularExpression@xercesc_2_3@@QAEXQBGHHH@Z 1200cf10 f   RegularExpression.obj
 0001:0000bff0       ?nextCh@Context@RegularExpression@xercesc_2_3@@QAE_NAAH0F@Z 1200cff0 f   RegularExpression.obj
 0001:0000c0d0       ??0RegularExpression@xercesc_2_3@@QAE@QBDQAVMemoryManager@1@@Z 1200d0d0 f   RegularExpression.obj
 0001:0000c230       ??0RegularExpression@xercesc_2_3@@QAE@QBD0QAVMemoryManager@1@@Z 1200d230 f   RegularExpression.obj
 0001:0000c3e0       ??0RegularExpression@xercesc_2_3@@QAE@QBGQAVMemoryManager@1@@Z 1200d3e0 f   RegularExpression.obj
 0001:0000c500       ??0RegularExpression@xercesc_2_3@@QAE@QBG0QAVMemoryManager@1@@Z 1200d500 f   RegularExpression.obj
 0001:0000c630       ??1RegularExpression@xercesc_2_3@@QAE@XZ 1200d630 f   RegularExpression.obj
 0001:0000c710       ?setPattern@RegularExpression@xercesc_2_3@@AAEXQBG0@Z 1200d710 f   RegularExpression.obj
 0001:0000c910       ?matches@RegularExpression@xercesc_2_3@@QAE_NQBD@Z 1200d910 f   RegularExpression.obj
 0001:0000c9d0       ?matches@RegularExpression@xercesc_2_3@@QAE_NQBDHH@Z 1200d9d0 f   RegularExpression.obj
 0001:0000ca70       ?matches@RegularExpression@xercesc_2_3@@QAE_NQBDQAVMatch@2@@Z 1200da70 f   RegularExpression.obj
 0001:0000cb30       ?matches@RegularExpression@xercesc_2_3@@QAE_NQBDHHQAVMatch@2@@Z 1200db30 f   RegularExpression.obj
 0001:0000cbd0       ?matches@RegularExpression@xercesc_2_3@@QAE_NQBG@Z 1200dbd0 f   RegularExpression.obj
 0001:0000cc20       ?matches@RegularExpression@xercesc_2_3@@QAE_NQBGHH@Z 1200dc20 f   RegularExpression.obj
 0001:0000cc40       ?matches@RegularExpression@xercesc_2_3@@QAE_NQBGQAVMatch@2@@Z 1200dc40 f   RegularExpression.obj
 0001:0000cc90       ?matches@RegularExpression@xercesc_2_3@@QAE_NQBGHHQAVMatch@2@@Z 1200dc90 f   RegularExpression.obj
 0001:0000d4a0       ?tokenize@RegularExpression@xercesc_2_3@@QAEPAV?$RefArrayVectorOf@G@2@QBD@Z 1200e4a0 f   RegularExpression.obj
 0001:0000d540       ?tokenize@RegularExpression@xercesc_2_3@@QAEPAV?$RefArrayVectorOf@G@2@QBDHH@Z 1200e540 f   RegularExpression.obj
 0001:0000d5c0       ?tokenize@RegularExpression@xercesc_2_3@@QAEPAV?$RefArrayVectorOf@G@2@QBG@Z 1200e5c0 f   RegularExpression.obj
 0001:0000d610       ?tokenize@RegularExpression@xercesc_2_3@@QAEPAV?$RefArrayVectorOf@G@2@QBGHH@Z 1200e610 f   RegularExpression.obj
 0001:0000d630       ?tokenize@RegularExpression@xercesc_2_3@@AAEPAV?$RefArrayVectorOf@G@2@QBGHHPAV?$RefVectorOf@VMatch@xercesc_2_3@@@2@@Z 1200e630 f   RegularExpression.obj
 0001:0000dd60       ?replace@RegularExpression@xercesc_2_3@@QAEPAGQBD0@Z 1200ed60 f   RegularExpression.obj
 0001:0000de20       ?replace@RegularExpression@xercesc_2_3@@QAEPAGQBD0HH@Z 1200ee20 f   RegularExpression.obj
 0001:0000ded0       ?replace@RegularExpression@xercesc_2_3@@QAEPAGQBG0@Z 1200eed0 f   RegularExpression.obj
 0001:0000df20       ?replace@RegularExpression@xercesc_2_3@@QAEPAGQBG0HH@Z 1200ef20 f   RegularExpression.obj
 0001:0000e280       ?getOptionValue@RegularExpression@xercesc_2_3@@SAHG@Z 1200f280 f   RegularExpression.obj
 0001:0000e360       ?match@RegularExpression@xercesc_2_3@@AAEHQAVContext@12@QBVOp@2@HF@Z 1200f360 f   RegularExpression.obj
 0001:0000ea40       ?matchChar@RegularExpression@xercesc_2_3@@AAE_NQAVContext@12@HAAHF_N@Z 1200fa40 f   RegularExpression.obj
 0001:0000eaf0       ?matchDot@RegularExpression@xercesc_2_3@@AAE_NQAVContext@12@AAHF@Z 1200faf0 f   RegularExpression.obj
 0001:0000eba0       ?matchRange@RegularExpression@xercesc_2_3@@AAE_NQAVContext@12@QBVOp@2@AAHF_N@Z 1200fba0 f   RegularExpression.obj
 0001:0000ec30       ?matchAnchor@RegularExpression@xercesc_2_3@@AAE_NQAVContext@12@HH@Z 1200fc30 f   RegularExpression.obj
 0001:0000f150       ?matchBackReference@RegularExpression@xercesc_2_3@@AAE_NQAVContext@12@HAAHF_N@Z 12010150 f   RegularExpression.obj
 0001:0000f3a0       ?matchString@RegularExpression@xercesc_2_3@@AAE_NQAVContext@12@QBGAAHF_N@Z 120103a0 f   RegularExpression.obj
 0001:0000f440       ?matchCapture@RegularExpression@xercesc_2_3@@AAEHQAVContext@12@QBVOp@2@HF@Z 12010440 f   RegularExpression.obj
 0001:0000f710       ?matchCondition@RegularExpression@xercesc_2_3@@AAE_NQAVContext@12@QBVOp@2@HF@Z 12010710 f   RegularExpression.obj
 0001:0000f840       ?parseOptions@RegularExpression@xercesc_2_3@@AAEHQBG@Z 12010840 f   RegularExpression.obj
 0001:0000f9b0       ?compile@RegularExpression@xercesc_2_3@@AAEXQBVToken@2@@Z 120109b0 f   RegularExpression.obj
 0001:0000f9e0       ?compile@RegularExpression@xercesc_2_3@@AAEPAVOp@2@QBVToken@2@QAV32@_N@Z 120109e0 f   RegularExpression.obj
 0001:0000fda0       ?subInExp@RegularExpression@xercesc_2_3@@AAEPBGQBG0PBVMatch@2@@Z 12010da0 f   RegularExpression.obj
 0001:00010160       ?prepare@RegularExpression@xercesc_2_3@@AAEXXZ 12011160 f   RegularExpression.obj
 0001:00010470       ?getCharType@RegularExpression@xercesc_2_3@@AAEGG@Z 12011470 f   RegularExpression.obj
 0001:000105c0       ??1?$Janitor@VContext@RegularExpression@xercesc_2_3@@@xercesc_2_3@@QAE@XZ 120115c0 f i RegularExpression.obj
 0001:00010610       ??_E?$RefArrayVectorOf@G@xercesc_2_3@@UAEPAXI@Z 12011610 f i RegularExpression.obj
 0001:00010610       ??_G?$RefArrayVectorOf@G@xercesc_2_3@@UAEPAXI@Z 12011610 f i RegularExpression.obj
 0001:00010630       ??1?$RefArrayVectorOf@G@xercesc_2_3@@UAE@XZ 12011630 f i RegularExpression.obj
 0001:000106b0       ??1?$BaseRefVectorOf@G@xercesc_2_3@@UAE@XZ 120116b0 f i RegularExpression.obj
 0001:000106c0       ??_G?$RefVectorOf@VMatch@xercesc_2_3@@@xercesc_2_3@@UAEPAXI@Z 120116c0 f i RegularExpression.obj
 0001:000106c0       ??_E?$RefVectorOf@VMatch@xercesc_2_3@@@xercesc_2_3@@UAEPAXI@Z 120116c0 f i RegularExpression.obj
 0001:000106e0       ??1?$RefVectorOf@VMatch@xercesc_2_3@@@xercesc_2_3@@UAE@XZ 120116e0 f i RegularExpression.obj
 0001:00010760       ??1?$BaseRefVectorOf@VMatch@xercesc_2_3@@@xercesc_2_3@@UAE@XZ 12011760 f i RegularExpression.obj
 0001:00010770       ??0?$BaseRefVectorOf@VMatch@xercesc_2_3@@@xercesc_2_3@@QAE@I_NQAVMemoryManager@1@@Z 12011770 f i RegularExpression.obj
 0001:000107d0       ?ensureExtraCapacity@?$BaseRefVectorOf@VSchemaInfo@xercesc_2_3@@@xercesc_2_3@@QAEXI@Z 120117d0 f i RegularExpression.obj
 0001:000107d0       ?ensureExtraCapacity@?$BaseRefVectorOf@VFieldValueMap@xercesc_2_3@@@xercesc_2_3@@QAEXI@Z 120117d0 f i RegularExpression.obj
 0001:000107d0       ?ensureExtraCapacity@?$BaseRefVectorOf@VXMLElementDecl@xercesc_2_3@@@xercesc_2_3@@QAEXI@Z 120117d0 f i RegularExpression.obj
 0001:000107d0       ?ensureExtraCapacity@?$BaseRefVectorOf@VXercesStep@xercesc_2_3@@@xercesc_2_3@@QAEXI@Z 120117d0 f i RegularExpression.obj
 0001:000107d0       ?ensureExtraCapacity@?$BaseRefVectorOf@VSchemaElementDecl@xercesc_2_3@@@xercesc_2_3@@QAEXI@Z 120117d0 f i RegularExpression.obj
 0001:000107d0       ?ensureExtraCapacity@?$BaseRefVectorOf@VDatatypeValidator@xercesc_2_3@@@xercesc_2_3@@QAEXI@Z 120117d0 f i RegularExpression.obj
 0001:000107d0       ?ensureExtraCapacity@?$BaseRefVectorOf@V?$RefHashTableOf@G@xercesc_2_3@@@xercesc_2_3@@QAEXI@Z 120117d0 f i RegularExpression.obj
 0001:000107d0       ?ensureExtraCapacity@?$BaseRefVectorOf@VMatch@xercesc_2_3@@@xercesc_2_3@@QAEXI@Z 120117d0 f i RegularExpression.obj
 0001:000107d0       ?ensureExtraCapacity@?$BaseRefVectorOf@VXercesLocationPath@xercesc_2_3@@@xercesc_2_3@@QAEXI@Z 120117d0 f i RegularExpression.obj
 0001:000107d0       ?ensureExtraCapacity@?$BaseRefVectorOf@VXMLBuffer@xercesc_2_3@@@xercesc_2_3@@QAEXI@Z 120117d0 f i RegularExpression.obj
 0001:000107d0       ?ensureExtraCapacity@?$BaseRefVectorOf@VXMLReader@xercesc_2_3@@@xercesc_2_3@@QAEXI@Z 120117d0 f i RegularExpression.obj
 0001:000107d0       ?ensureExtraCapacity@?$BaseRefVectorOf@VENameMap@xercesc_2_3@@@xercesc_2_3@@QAEXI@Z 120117d0 f i RegularExpression.obj
 0001:000107d0       ?ensureExtraCapacity@?$BaseRefVectorOf@VNodeImpl@xercesc_2_3@@@xercesc_2_3@@QAEXI@Z 120117d0 f i RegularExpression.obj
 0001:000107d0       ?ensureExtraCapacity@?$BaseRefVectorOf@VXMLAttr@xercesc_2_3@@@xercesc_2_3@@QAEXI@Z 120117d0 f i RegularExpression.obj
 0001:000107d0       ?ensureExtraCapacity@?$BaseRefVectorOf@VToken@xercesc_2_3@@@xercesc_2_3@@QAEXI@Z 120117d0 f i RegularExpression.obj
 0001:000107d0       ?ensureExtraCapacity@?$BaseRefVectorOf@VDOMImplementationSource@xercesc_2_3@@@xercesc_2_3@@QAEXI@Z 120117d0 f i RegularExpression.obj
 0001:000107d0       ?ensureExtraCapacity@?$BaseRefVectorOf@VIC_Field@xercesc_2_3@@@xercesc_2_3@@QAEXI@Z 120117d0 f i RegularExpression.obj
 0001:000107d0       ?ensureExtraCapacity@?$BaseRefVectorOf@VXMLNumber@xercesc_2_3@@@xercesc_2_3@@QAEXI@Z 120117d0 f i RegularExpression.obj
 0001:000107d0       ?ensureExtraCapacity@?$BaseRefVectorOf@VDOMNode@xercesc_2_3@@@xercesc_2_3@@QAEXI@Z 120117d0 f i RegularExpression.obj
 0001:000107d0       ?ensureExtraCapacity@?$BaseRefVectorOf@VReferencePosition@RegxParser@xercesc_2_3@@@xercesc_2_3@@QAEXI@Z 120117d0 f i RegularExpression.obj
 0001:000107d0       ?ensureExtraCapacity@?$BaseRefVectorOf@VXPathMatcher@xercesc_2_3@@@xercesc_2_3@@QAEXI@Z 120117d0 f i RegularExpression.obj
 0001:000107d0       ?ensureExtraCapacity@?$BaseRefVectorOf@G@xercesc_2_3@@QAEXI@Z 120117d0 f i RegularExpression.obj
 0001:00010850       ??0RegxParser@xercesc_2_3@@QAE@QAVMemoryManager@1@@Z 12011850 f   RegxParser.obj
 0001:000108a0       ??_ERegxParser@xercesc_2_3@@UAEPAXI@Z 120118a0 f i RegxParser.obj
 0001:00010900       ??1RegxParser@xercesc_2_3@@UAE@XZ 12011900 f   RegxParser.obj
 0001:00010970       ?parse@RegxParser@xercesc_2_3@@QAEPAVToken@2@QBGH@Z 12011970 f   RegxParser.obj
 0001:00010c30       ?processNext@RegxParser@xercesc_2_3@@IAEXXZ 12011c30 f   RegxParser.obj
 0001:000111f0       ?parseRegx@RegxParser@xercesc_2_3@@IAEPAVToken@2@_N@Z 120121f0 f   RegxParser.obj
 0001:00011260       ?parseTerm@RegxParser@xercesc_2_3@@AAEPAVToken@2@_N@Z 12012260 f   RegxParser.obj
 0001:00011310       ?processCaret@RegxParser@xercesc_2_3@@MAEPAVToken@2@XZ 12012310 f   RegxParser.obj
 0001:00011330       ?processDollar@RegxParser@xercesc_2_3@@MAEPAVToken@2@XZ 12012330 f   RegxParser.obj
 0001:00011350       ?processLook@RegxParser@xercesc_2_3@@MAEPAVToken@2@G@Z 12012350 f   RegxParser.obj
 0001:00011400       ?processBacksolidus_A@RegxParser@xercesc_2_3@@MAEPAVToken@2@XZ 12012400 f   RegxParser.obj
 0001:00011420       ?processBacksolidus_Z@RegxParser@xercesc_2_3@@MAEPAVToken@2@XZ 12012420 f   RegxParser.obj
 0001:00011440       ?processBacksolidus_z@RegxParser@xercesc_2_3@@MAEPAVToken@2@XZ 12012440 f   RegxParser.obj
 0001:00011460       ?processBacksolidus_b@RegxParser@xercesc_2_3@@MAEPAVToken@2@XZ 12012460 f   RegxParser.obj
 0001:00011480       ?processBacksolidus_B@RegxParser@xercesc_2_3@@MAEPAVToken@2@XZ 12012480 f   RegxParser.obj
 0001:000114a0       ?processBacksolidus_lt@RegxParser@xercesc_2_3@@MAEPAVToken@2@XZ 120124a0 f   RegxParser.obj
 0001:000114c0       ?processBacksolidus_gt@RegxParser@xercesc_2_3@@MAEPAVToken@2@XZ 120124c0 f   RegxParser.obj
 0001:000114e0       ?processStar@RegxParser@xercesc_2_3@@MAEPAVToken@2@QAV32@@Z 120124e0 f   RegxParser.obj
 0001:00011520       ?processPlus@RegxParser@xercesc_2_3@@MAEPAVToken@2@QAV32@@Z 12012520 f   RegxParser.obj
 0001:00011560       ?processQuestion@RegxParser@xercesc_2_3@@MAEPAVToken@2@QAV32@@Z 12012560 f   RegxParser.obj
 0001:000115e0       ?processParen@RegxParser@xercesc_2_3@@MAEPAVToken@2@XZ 120125e0 f   RegxParser.obj
 0001:000116a0       ?processParen2@RegxParser@xercesc_2_3@@MAEPAVToken@2@XZ 120126a0 f   RegxParser.obj
 0001:00011750       ?processCondition@RegxParser@xercesc_2_3@@MAEPAVToken@2@XZ 12012750 f   RegxParser.obj
 0001:00011af0       ?processModifiers@RegxParser@xercesc_2_3@@MAEPAVToken@2@XZ 12012af0 f   RegxParser.obj
 0001:00011d40       ?processIndependent@RegxParser@xercesc_2_3@@MAEPAVToken@2@XZ 12012d40 f   RegxParser.obj
 0001:00011df0       ?processBacksolidus_c@RegxParser@xercesc_2_3@@MAEPAVToken@2@XZ 12012df0 f   RegxParser.obj
 0001:00011e60       ?processBacksolidus_i@RegxParser@xercesc_2_3@@MAEPAVToken@2@XZ 12012e60 f   RegxParser.obj
 0001:00011e80       ?processBacksolidus_g@RegxParser@xercesc_2_3@@MAEPAVToken@2@XZ 12012e80 f   RegxParser.obj
 0001:00011ea0       ?processBacksolidus_X@RegxParser@xercesc_2_3@@MAEPAVToken@2@XZ 12012ea0 f   RegxParser.obj
 0001:00011ec0       ?processBackReference@RegxParser@xercesc_2_3@@MAEPAVToken@2@XZ 12012ec0 f   RegxParser.obj
 0001:00012030       ?parseFactor@RegxParser@xercesc_2_3@@AAEPAVToken@2@XZ 12013030 f   RegxParser.obj
 0001:00012490       ?parseAtom@RegxParser@xercesc_2_3@@AAEPAVToken@2@XZ 12013490 f   RegxParser.obj
 0001:00012910       ?processBacksolidus_pP@RegxParser@xercesc_2_3@@IAEPAVRangeToken@2@H@Z 12013910 f   RegxParser.obj
 0001:00012a90       ?processCInCharacterClass@RegxParser@xercesc_2_3@@MAEHQAVRangeToken@2@H@Z 12013a90 f   RegxParser.obj
 0001:00012aa0       ?parseCharacterClass@RegxParser@xercesc_2_3@@MAEPAVRangeToken@2@_N@Z 12013aa0 f   RegxParser.obj
 0001:00012ff0       ?parseSetOperations@RegxParser@xercesc_2_3@@MAEPAVRangeToken@2@XZ 12013ff0 f   RegxParser.obj
 0001:000130f0       ?getTokenForShorthand@RegxParser@xercesc_2_3@@MAEPAVToken@2@H@Z 120140f0 f   RegxParser.obj
 0001:00013220       ?decodeEscaped@RegxParser@xercesc_2_3@@MAEHXZ 12014220 f   RegxParser.obj
 0001:000136a0       ?checkQuestion@RegxParser@xercesc_2_3@@MAE_NH@Z 120146a0 f   RegxParser.obj
 0001:000136c0       ??_G?$RefVectorOf@VReferencePosition@RegxParser@xercesc_2_3@@@xercesc_2_3@@UAEPAXI@Z 120146c0 f i RegxParser.obj
 0001:000136c0       ??_E?$RefVectorOf@VReferencePosition@RegxParser@xercesc_2_3@@@xercesc_2_3@@UAEPAXI@Z 120146c0 f i RegxParser.obj
 0001:000136e0       ??1?$RefVectorOf@VReferencePosition@RegxParser@xercesc_2_3@@@xercesc_2_3@@UAE@XZ 120146e0 f i RegxParser.obj
 0001:00013760       ??1?$BaseRefVectorOf@VReferencePosition@RegxParser@xercesc_2_3@@@xercesc_2_3@@UAE@XZ 12014760 f i RegxParser.obj
 0001:00013770       ??0?$BaseRefVectorOf@VReferencePosition@RegxParser@xercesc_2_3@@@xercesc_2_3@@QAE@I_NQAVMemoryManager@1@@Z 12014770 f i RegxParser.obj
 0001:000137d0       ?decomposeToSurrogates@RegxUtil@xercesc_2_3@@SAPAGHQAVMemoryManager@2@@Z 120147d0 f   RegxUtil.obj
 0001:00013810       ?stripExtendedComment@RegxUtil@xercesc_2_3@@SAPAGQBGQAVMemoryManager@2@@Z 12014810 f   RegxUtil.obj
 0001:00013970       ??0StringToken@xercesc_2_3@@QAE@GQBGHQAVMemoryManager@1@@Z 12014970 f   StringToken.obj
 0001:00013a20       ??_EStringToken@xercesc_2_3@@UAEPAXI@Z 12014a20 f i StringToken.obj
 0001:00013a80       ??1StringToken@xercesc_2_3@@UAE@XZ 12014a80 f   StringToken.obj
 0001:00013ae0       ??0Token@xercesc_2_3@@QAE@G@Z 12014ae0 f   Token.obj
 0001:00013b00       ??_EToken@xercesc_2_3@@UAEPAXI@Z 12014b00 f i Token.obj
 0001:00013b60       ??1Token@xercesc_2_3@@UAE@XZ 12014b60 f   Token.obj
 0001:00013b70       ?getMinLength@Token@xercesc_2_3@@QBEHXZ 12014b70 f   Token.obj
 0001:00013ce0       ?getMaxLength@Token@xercesc_2_3@@QBEHXZ 12014ce0 f   Token.obj
 0001:00013e80       ?analyzeFirstCharacter@Token@xercesc_2_3@@QAEHQAVRangeToken@2@HQAVTokenFactory@2@@Z 12014e80 f   Token.obj
 0001:00014130       ?findFixedString@Token@xercesc_2_3@@QAEPAV12@HAAH@Z 12015130 f   Token.obj
 0001:000142c0       ?isShorterThan@Token@xercesc_2_3@@AAE_NQAV12@@Z 120152c0 f   Token.obj
 0001:00014360       ??0TokenFactory@xercesc_2_3@@QAE@QAVMemoryManager@1@@Z 12015360 f   TokenFactory.obj
 0001:00014440       ??1TokenFactory@xercesc_2_3@@QAE@XZ 12015440 f   TokenFactory.obj
 0001:000144a0       ?createToken@TokenFactory@xercesc_2_3@@QAEPAVToken@2@G@Z 120154a0 f   TokenFactory.obj
 0001:000145b0       ?createLook@TokenFactory@xercesc_2_3@@QAEPAVParenToken@2@GQAVToken@2@@Z 120155b0 f   TokenFactory.obj
 0001:000146a0       ?createParenthesis@TokenFactory@xercesc_2_3@@QAEPAVParenToken@2@QAVToken@2@H@Z 120156a0 f   TokenFactory.obj
 0001:00014790       ?createClosure@TokenFactory@xercesc_2_3@@QAEPAVClosureToken@2@QAVToken@2@_N@Z 12015790 f   TokenFactory.obj
 0001:000148b0       ?createConcat@TokenFactory@xercesc_2_3@@QAEPAVConcatToken@2@QAVToken@2@0@Z 120158b0 f   TokenFactory.obj
 0001:000149a0       ?createUnion@TokenFactory@xercesc_2_3@@QAEPAVUnionToken@2@_N@Z 120159a0 f   TokenFactory.obj
 0001:00014ac0       ?createRange@TokenFactory@xercesc_2_3@@QAEPAVRangeToken@2@_N@Z 12015ac0 f   TokenFactory.obj
 0001:00014be0       ?createChar@TokenFactory@xercesc_2_3@@QAEPAVCharToken@2@I_N@Z 12015be0 f   TokenFactory.obj
 0001:00014d00       ?createBackReference@TokenFactory@xercesc_2_3@@QAEPAVStringToken@2@H@Z 12015d00 f   TokenFactory.obj
 0001:00014df0       ?createString@TokenFactory@xercesc_2_3@@QAEPAVStringToken@2@QBG@Z 12015df0 f   TokenFactory.obj
 0001:00014ee0       ?createModifierGroup@TokenFactory@xercesc_2_3@@QAEPAVModifierToken@2@QAVToken@2@HH@Z 12015ee0 f   TokenFactory.obj
 0001:00014fe0       ?createCondition@TokenFactory@xercesc_2_3@@QAEPAVConditionToken@2@HQAVToken@2@00@Z 12015fe0 f   TokenFactory.obj
 0001:000150e0       ?getRange@TokenFactory@xercesc_2_3@@QAEPAVRangeToken@2@QBG_N@Z 120160e0 f   TokenFactory.obj
 0001:00015110       ?getLineBegin@TokenFactory@xercesc_2_3@@QAEPAVToken@2@XZ 12016110 f   TokenFactory.obj
 0001:00015130       ?getLineBegin2@TokenFactory@xercesc_2_3@@QAEPAVToken@2@XZ 12016130 f   TokenFactory.obj
 0001:00015150       ?getLineEnd@TokenFactory@xercesc_2_3@@QAEPAVToken@2@XZ 12016150 f   TokenFactory.obj
 0001:00015170       ?getStringBegin@TokenFactory@xercesc_2_3@@QAEPAVToken@2@XZ 12016170 f   TokenFactory.obj
 0001:00015190       ?getStringEnd@TokenFactory@xercesc_2_3@@QAEPAVToken@2@XZ 12016190 f   TokenFactory.obj
 0001:000151b0       ?getStringEnd2@TokenFactory@xercesc_2_3@@QAEPAVToken@2@XZ 120161b0 f   TokenFactory.obj
 0001:000151d0       ?getWordEdge@TokenFactory@xercesc_2_3@@QAEPAVToken@2@XZ 120161d0 f   TokenFactory.obj
 0001:000151f0       ?getNotWordEdge@TokenFactory@xercesc_2_3@@QAEPAVToken@2@XZ 120161f0 f   TokenFactory.obj
 0001:00015210       ?getWordBegin@TokenFactory@xercesc_2_3@@QAEPAVToken@2@XZ 12016210 f   TokenFactory.obj
 0001:00015230       ?getWordEnd@TokenFactory@xercesc_2_3@@QAEPAVToken@2@XZ 12016230 f   TokenFactory.obj
 0001:00015250       ?getDot@TokenFactory@xercesc_2_3@@QAEPAVToken@2@XZ 12016250 f   TokenFactory.obj
 0001:00015270       ?getCombiningCharacterSequence@TokenFactory@xercesc_2_3@@QAEPAVToken@2@XZ 12016270 f   TokenFactory.obj
 0001:000152e0       ?getGraphemePattern@TokenFactory@xercesc_2_3@@QAEPAVToken@2@XZ 120162e0 f   TokenFactory.obj
 0001:00015550       ?initializeRegistry@TokenFactory@xercesc_2_3@@AAEXXZ 12016550 f   TokenFactory.obj
 0001:00015710       ??_E?$RefVectorOf@VToken@xercesc_2_3@@@xercesc_2_3@@UAEPAXI@Z 12016710 f i TokenFactory.obj
 0001:00015710       ??_G?$RefVectorOf@VToken@xercesc_2_3@@@xercesc_2_3@@UAEPAXI@Z 12016710 f i TokenFactory.obj
 0001:00015730       ??1?$RefVectorOf@VToken@xercesc_2_3@@@xercesc_2_3@@UAE@XZ 12016730 f i TokenFactory.obj
 0001:000157b0       ??1?$BaseRefVectorOf@VToken@xercesc_2_3@@@xercesc_2_3@@UAE@XZ 120167b0 f i TokenFactory.obj
 0001:000157c0       ??0UnicodeRangeFactory@xercesc_2_3@@QAE@XZ 120167c0 f   UnicodeRangeFactory.obj
 0001:000157e0       ??_EUnicodeRangeFactory@xercesc_2_3@@UAEPAXI@Z 120167e0 f i UnicodeRangeFactory.obj
 0001:00015840       ??1UnicodeRangeFactory@xercesc_2_3@@UAE@XZ 12016840 f   UnicodeRangeFactory.obj
 0001:00015850       ?buildRanges@UnicodeRangeFactory@xercesc_2_3@@MAEXXZ 12016850 f   UnicodeRangeFactory.obj
 0001:00015a80       ?initializeKeywordMap@UnicodeRangeFactory@xercesc_2_3@@UAEXXZ 12016a80 f   UnicodeRangeFactory.obj
 0001:00015b20       ?getUniCategory@UnicodeRangeFactory@xercesc_2_3@@AAEGG@Z 12016b20 f   UnicodeRangeFactory.obj
 0001:00015bb0       ??0UnionToken@xercesc_2_3@@QAE@G@Z 12016bb0 f   UnionToken.obj
 0001:00015bd0       ??_EUnionToken@xercesc_2_3@@UAEPAXI@Z 12016bd0 f i UnionToken.obj
 0001:00015c30       ??1UnionToken@xercesc_2_3@@UAE@XZ 12016c30 f   UnionToken.obj
 0001:00015c90       ?addChild@UnionToken@xercesc_2_3@@UAEXQAVToken@2@QAVTokenFactory@2@@Z 12016c90 f   UnionToken.obj
 0001:00016070       ??0?$BaseRefVectorOf@VToken@xercesc_2_3@@@xercesc_2_3@@QAE@I_NQAVMemoryManager@1@@Z 12017070 f i UnionToken.obj
 0001:000160d0       ??0XMLRangeFactory@xercesc_2_3@@QAE@XZ 120170d0 f   XMLRangeFactory.obj
 0001:000160f0       ??_EXMLRangeFactory@xercesc_2_3@@UAEPAXI@Z 120170f0 f i XMLRangeFactory.obj
 0001:00016150       ??1XMLRangeFactory@xercesc_2_3@@UAE@XZ 12017150 f   XMLRangeFactory.obj
 0001:00016160       ?buildRanges@XMLRangeFactory@xercesc_2_3@@MAEXXZ 12017160 f   XMLRangeFactory.obj
 0001:00016840       ?initializeKeywordMap@XMLRangeFactory@xercesc_2_3@@UAEXXZ 12017840 f   XMLRangeFactory.obj
 0001:000168b0       ?getType@XMLUniCharacter@xercesc_2_3@@SAGG@Z 120178b0 f   XMLUniCharacter.obj
 0001:000168d0       ?isPad@Base64@xercesc_2_3@@CA_NABE@Z 120178d0 f i Base64.obj
 0001:000168f0       ?set1stOctet@Base64@xercesc_2_3@@CAEABE0@Z 120178f0 f i Base64.obj
 0001:00016910       ?set2ndOctet@Base64@xercesc_2_3@@CAEABE0@Z 12017910 f i Base64.obj
 0001:00016930       ?set3rdOctet@Base64@xercesc_2_3@@CAEABE0@Z 12017930 f i Base64.obj
 0001:00016950       ?split1stOctet@Base64@xercesc_2_3@@CAXABEAAE1@Z 12017950 f i Base64.obj
 0001:00016970       ?split2ndOctet@Base64@xercesc_2_3@@CAXABEAAE1@Z 12017970 f i Base64.obj
 0001:000169a0       ?split3rdOctet@Base64@xercesc_2_3@@CAXABEAAE1@Z 120179a0 f i Base64.obj
 0001:000169c0       ?isXMLLetter@XMLChar1_0@xercesc_2_3@@SA_NGG@Z 120179c0 f i Base64.obj
 0001:000169e0       ?isFirstNameChar@XMLChar1_0@xercesc_2_3@@SA_NGG@Z 120179e0 f i Base64.obj
 0001:00016a10       ?isNameChar@XMLChar1_0@xercesc_2_3@@SA_NGG@Z 12017a10 f i Base64.obj
 0001:00016a40       ?isPlainContentChar@XMLChar1_0@xercesc_2_3@@SA_NGG@Z 12017a40 f i Base64.obj
 0001:00016a90       ?isSpecialStartTagChar@XMLChar1_0@xercesc_2_3@@SA_NGG@Z 12017a90 f i Base64.obj
 0001:00016ac0       ?isXMLChar@XMLChar1_0@xercesc_2_3@@SA_NGG@Z 12017ac0 f i Base64.obj
 0001:00016b10       ?isWhitespace@XMLChar1_0@xercesc_2_3@@SA_NGG@Z 12017b10 f i Base64.obj
 0001:00016b40       ?isControlChar@XMLChar1_0@xercesc_2_3@@SA_NGG@Z 12017b40 f i Base64.obj
 0001:00016b70       ?isNELRecognized@XMLChar1_0@xercesc_2_3@@SA_NXZ 12017b70 f i Base64.obj
 0001:00016b80       ?isXMLLetter@XMLChar1_1@xercesc_2_3@@SA_NGG@Z 12017b80 f i Base64.obj
 0001:00016ba0       ?isFirstNameChar@XMLChar1_1@xercesc_2_3@@SA_NGG@Z 12017ba0 f i Base64.obj
 0001:00016bf0       ?isNameChar@XMLChar1_1@xercesc_2_3@@SA_NGG@Z 12017bf0 f i Base64.obj
 0001:00016c40       ?isPlainContentChar@XMLChar1_1@xercesc_2_3@@SA_NGG@Z 12017c40 f i Base64.obj
 0001:00016c90       ?isSpecialStartTagChar@XMLChar1_1@xercesc_2_3@@SA_NGG@Z 12017c90 f i Base64.obj
 0001:00016cc0       ?isXMLChar@XMLChar1_1@xercesc_2_3@@SA_NGG@Z 12017cc0 f i Base64.obj
 0001:00016d10       ?isWhitespace@XMLChar1_1@xercesc_2_3@@SA_NGG@Z 12017d10 f i Base64.obj
 0001:00016d40       ?isControlChar@XMLChar1_1@xercesc_2_3@@SA_NGG@Z 12017d40 f i Base64.obj
 0001:00016d70       ?isNameChar@XMLReader@xercesc_2_3@@QAE_NG@Z 12017d70 f i Base64.obj
 0001:00016d90       ?isPlainContentChar@XMLReader@xercesc_2_3@@QAE_NG@Z 12017d90 f i Base64.obj
 0001:00016db0       ?isFirstNameChar@XMLReader@xercesc_2_3@@QAE_NG@Z 12017db0 f i Base64.obj
 0001:00016dd0       ?isSpecialStartTagChar@XMLReader@xercesc_2_3@@QAE_NG@Z 12017dd0 f i Base64.obj
 0001:00016df0       ?isXMLChar@XMLReader@xercesc_2_3@@QAE_NG@Z 12017df0 f i Base64.obj
 0001:00016e10       ?isXMLLetter@XMLReader@xercesc_2_3@@QAE_NG@Z 12017e10 f i Base64.obj
 0001:00016e30       ?isWhitespace@XMLReader@xercesc_2_3@@QAE_NG@Z 12017e30 f i Base64.obj
 0001:00016e50       ?isControlChar@XMLReader@xercesc_2_3@@QAE_NG@Z 12017e50 f i Base64.obj
 0001:00016e70       ?charsLeftInBuffer@XMLReader@xercesc_2_3@@QBEKXZ 12017e70 f i Base64.obj
 0001:00016e80       ?getColumnNumber@XMLReader@xercesc_2_3@@QBEJXZ 12017e80 f i Base64.obj
 0001:00016e90       ?getEncodingStr@XMLReader@xercesc_2_3@@QBEPBGXZ 12017e90 f i Base64.obj
 0001:00016ea0       ?getLineNumber@XMLReader@xercesc_2_3@@QBEJXZ 12017ea0 f i Base64.obj
 0001:00016eb0       ?getNoMoreFlag@XMLReader@xercesc_2_3@@QBE_NXZ 12017eb0 f i Base64.obj
 0001:00016ec0       ?getPublicId@XMLReader@xercesc_2_3@@QBEPBGXZ 12017ec0 f i Base64.obj
 0001:00016ed0       ?getReaderNum@XMLReader@xercesc_2_3@@QBEIXZ 12017ed0 f i Base64.obj
 0001:00016ee0       ?getRefFrom@XMLReader@xercesc_2_3@@QBE?AW4RefFrom@12@XZ 12017ee0 f i Base64.obj
 0001:00016ef0       ?getSource@XMLReader@xercesc_2_3@@QBE?AW4Sources@12@XZ 12017ef0 f i Base64.obj
 0001:00016f00       ?getSystemId@XMLReader@xercesc_2_3@@QBEPBGXZ 12017f00 f i Base64.obj
 0001:00016f10       ?getThrowAtEnd@XMLReader@xercesc_2_3@@QBE_NXZ 12017f10 f i Base64.obj
 0001:00016f20       ?getType@XMLReader@xercesc_2_3@@QBE?AW4Types@12@XZ 12017f20 f i Base64.obj
 0001:00016f30       ?setReaderNum@XMLReader@xercesc_2_3@@QAEXI@Z 12017f30 f i Base64.obj
 0001:00016f40       ?setThrowAtEnd@XMLReader@xercesc_2_3@@QAEX_N@Z 12017f40 f i Base64.obj
 0001:00016f50       ?setXMLVersion@XMLReader@xercesc_2_3@@QAEXW4XMLVersion@12@@Z 12017f50 f i Base64.obj
 0001:00016f90       ?movePlainContentChars@XMLReader@xercesc_2_3@@QAEXAAVXMLBuffer@2@@Z 12017f90 f i Base64.obj
 0001:00016ff0       ?getNextCharIfNot@XMLReader@xercesc_2_3@@QAE_NGAAG@Z 12017ff0 f i Base64.obj
 0001:00017110       ?getNextChar@XMLReader@xercesc_2_3@@QAE_NAAG@Z 12018110 f i Base64.obj
 0001:00017200       ?peekNextChar@XMLReader@xercesc_2_3@@QAE_NAAG@Z 12018200 f i Base64.obj
 0001:00017270       ?encode@Base64@xercesc_2_3@@SAPAEQBEIPAIQAVMemoryManager@2@@Z 12018270 f   Base64.obj
 0001:000174f0       ?getDataLength@Base64@xercesc_2_3@@SAHQBG@Z 120184f0 f   Base64.obj
 0001:00017530       ?decode@Base64@xercesc_2_3@@SAPAEQBEPAIQAVMemoryManager@2@@Z 12018530 f   Base64.obj
 0001:00017990       ?decode@Base64@xercesc_2_3@@SAPAGQBGPAIQAVMemoryManager@2@@Z 12018990 f   Base64.obj
 0001:00017b40       ?init@Base64@xercesc_2_3@@CAXXZ 12018b40 f   Base64.obj
 0001:00017b80       ?isData@Base64@xercesc_2_3@@CA_NABE@Z 12018b80 f   Base64.obj
 0001:00017ba0       ??1?$ArrayJanitor@_N@xercesc_2_3@@QAE@XZ 12018ba0 f i Base64.obj
 0001:00017ba0       ??1?$ArrayJanitor@D@xercesc_2_3@@QAE@XZ 12018ba0 f i Base64.obj
 0001:00017ba0       ??1?$ArrayJanitor@H@xercesc_2_3@@QAE@XZ 12018ba0 f i Base64.obj
 0001:00017ba0       ??1?$ArrayJanitor@E@xercesc_2_3@@QAE@XZ 12018ba0 f i Base64.obj
 0001:00017ba0       ??1?$ArrayJanitor@G@xercesc_2_3@@QAE@XZ 12018ba0 f i Base64.obj
 0001:00017be0       ?reset@?$ArrayJanitor@G@xercesc_2_3@@QAEXPAG@Z 12018be0 f i Base64.obj
 0001:00017be0       ?reset@?$ArrayJanitor@E@xercesc_2_3@@QAEXPAE@Z 12018be0 f i Base64.obj
 0001:00017c40       ?getIsOpen@BinFileInputStream@xercesc_2_3@@QBE_NXZ 12018c40 f i BinFileInputStream.obj
 0001:00017c50       ??0BinFileInputStream@xercesc_2_3@@QAE@QBG@Z 12018c50 f   BinFileInputStream.obj
 0001:00017cb0       ??_EBinFileInputStream@xercesc_2_3@@UAEPAXI@Z 12018cb0 f i BinFileInputStream.obj
 0001:00017d10       ??0BinFileInputStream@xercesc_2_3@@QAE@QBDQAVMemoryManager@1@@Z 12018d10 f   BinFileInputStream.obj
 0001:00017db0       ??0BinFileInputStream@xercesc_2_3@@QAE@QAX@Z 12018db0 f   BinFileInputStream.obj
 0001:00017dd0       ??1BinFileInputStream@xercesc_2_3@@UAE@XZ 12018dd0 f   BinFileInputStream.obj
 0001:00017e30       ?getSize@BinFileInputStream@xercesc_2_3@@QBEIXZ 12018e30 f   BinFileInputStream.obj
 0001:00017e40       ?reset@BinFileInputStream@xercesc_2_3@@QAEXXZ 12018e40 f   BinFileInputStream.obj
 0001:00017e50       ?curPos@BinFileInputStream@xercesc_2_3@@UBEIXZ 12018e50 f   BinFileInputStream.obj
 0001:00017e60       ?readBytes@BinFileInputStream@xercesc_2_3@@UAEIQAEI@Z 12018e60 f   BinFileInputStream.obj
 0001:00017e80       ??1BinInputStream@xercesc_2_3@@UAE@XZ 12018e80 f   BinInputStream.obj
 0001:00017e90       ??_EBinInputStream@xercesc_2_3@@UAEPAXI@Z 12018e90 f i BinInputStream.obj
 0001:00017ef0       ??0BinInputStream@xercesc_2_3@@IAE@XZ 12018ef0 f   BinInputStream.obj
 0001:00017f00       ?reset@BinMemInputStream@xercesc_2_3@@QAEXXZ 12018f00 f i BinMemInputStream.obj
 0001:00017f10       ??0BinMemInputStream@xercesc_2_3@@QAE@QBEIW4BufOpts@01@QAVMemoryManager@1@@Z 12018f10 f   BinMemInputStream.obj
 0001:00017fc0       ??_EBinMemInputStream@xercesc_2_3@@UAEPAXI@Z 12018fc0 f i BinMemInputStream.obj
 0001:00018020       ??1BinMemInputStream@xercesc_2_3@@UAE@XZ 12019020 f   BinMemInputStream.obj
 0001:00018090       ?readBytes@BinMemInputStream@xercesc_2_3@@UAEIQAEI@Z 12019090 f   BinMemInputStream.obj
 0001:000180e0       ??0BitSet@xercesc_2_3@@QAE@IQAVMemoryManager@1@@Z 120190e0 f   BitSet.obj
 0001:00018110       ??0BitSet@xercesc_2_3@@QAE@ABV01@@Z 12019110 f   BitSet.obj
 0001:00018160       ??1BitSet@xercesc_2_3@@QAE@XZ 12019160 f   BitSet.obj
 0001:00018170       ?equals@BitSet@xercesc_2_3@@QBE_NABV12@@Z 12019170 f   BitSet.obj
 0001:000181b0       ?get@BitSet@xercesc_2_3@@QBE_NI@Z 120191b0 f   BitSet.obj
 0001:000181e0       ?size@BitSet@xercesc_2_3@@QBEIXZ 120191e0 f   BitSet.obj
 0001:000181f0       ?allAreCleared@BitSet@xercesc_2_3@@QBE_NXZ 120191f0 f   BitSet.obj
 0001:00018210       ?allAreSet@BitSet@xercesc_2_3@@QBE_NXZ 12019210 f   BitSet.obj
 0001:00018230       ?clearAll@BitSet@xercesc_2_3@@QAEXXZ 12019230 f   BitSet.obj
 0001:00018250       ?clear@BitSet@xercesc_2_3@@QAEXI@Z 12019250 f   BitSet.obj
 0001:00018290       ?set@BitSet@xercesc_2_3@@QAEXI@Z 12019290 f   BitSet.obj
 0001:000182d0       ?andWith@BitSet@xercesc_2_3@@QAEXABV12@@Z 120192d0 f   BitSet.obj
 0001:00018320       ?orWith@BitSet@xercesc_2_3@@QAEXABV12@@Z 12019320 f   BitSet.obj
 0001:00018370       ?xorWith@BitSet@xercesc_2_3@@QAEXABV12@@Z 12019370 f   BitSet.obj
 0001:000183c0       ?hash@BitSet@xercesc_2_3@@QBEII@Z 120193c0 f   BitSet.obj
 0001:000183f0       ?ensureCapacity@BitSet@xercesc_2_3@@AAEXI@Z 120193f0 f   BitSet.obj
 0001:00018470       ??0DefaultPanicHandler@xercesc_2_3@@QAE@XZ 12019470 f i DefaultPanicHandler.obj
 0001:00018480       ??_EDefaultPanicHandler@xercesc_2_3@@UAEPAXI@Z 12019480 f i DefaultPanicHandler.obj
 0001:000184e0       ?panic@DefaultPanicHandler@xercesc_2_3@@UAEXW4PanicReasons@PanicHandler@2@@Z 120194e0 f   DefaultPanicHandler.obj
 0001:00018510       ??4EncodingValidator@xercesc_2_3@@QAEAAV01@ABV01@@Z 12019510 f i EncodingValidator.obj
 0001:00018520       ??0EncodingValidator@xercesc_2_3@@AAE@XZ 12019520 f   EncodingValidator.obj
 0001:00018540       ??1EncodingValidator@xercesc_2_3@@AAE@XZ 12019540 f   EncodingValidator.obj
 0001:000185c0       ?isValidEncoding@EncodingValidator@xercesc_2_3@@QAE_NQBG@Z 120195c0 f   EncodingValidator.obj
 0001:00018640       ?initializeRegistry@EncodingValidator@xercesc_2_3@@AAEXXZ 12019640 f   EncodingValidator.obj
 0001:000187f0       ?instance@EncodingValidator@xercesc_2_3@@SAPAV12@XZ 120197f0 f   EncodingValidator.obj
 0001:00018a10       ?reinitInstance@EncodingValidator@xercesc_2_3@@SAXXZ 12019a10 f   EncodingValidator.obj
 0001:00018ab0       ?put@?$ValueHashTableOf@_N@xercesc_2_3@@QAEXPAXAB_N@Z 12019ab0 f i EncodingValidator.obj
 0001:00018bb0       ?initialize@?$ValueHashTableOf@_N@xercesc_2_3@@AAEXI@Z 12019bb0 f i EncodingValidator.obj
 0001:00018bb0       ?initialize@?$ValueHashTableOf@G@xercesc_2_3@@AAEXI@Z 12019bb0 f i EncodingValidator.obj
 0001:00018c20       ??0HashPtr@xercesc_2_3@@QAE@XZ 12019c20 f   HashPtr.obj
 0001:00018c30       ??_EHashPtr@xercesc_2_3@@UAEPAXI@Z 12019c30 f i HashPtr.obj
 0001:00018c90       ??1HashPtr@xercesc_2_3@@UAE@XZ 12019c90 f   HashPtr.obj
 0001:00018ca0       ?getHashVal@HashPtr@xercesc_2_3@@UAEIQBXI@Z 12019ca0 f   HashPtr.obj
 0001:00018cb0       ?equals@HashPtr@xercesc_2_3@@UAE_NQBX0@Z 12019cb0 f   HashPtr.obj
 0001:00018cd0       ??0HashXMLCh@xercesc_2_3@@QAE@XZ 12019cd0 f   HashXMLCh.obj
 0001:00018ce0       ??_EHashXMLCh@xercesc_2_3@@UAEPAXI@Z 12019ce0 f i HashXMLCh.obj
 0001:00018d40       ??1HashXMLCh@xercesc_2_3@@UAE@XZ 12019d40 f   HashXMLCh.obj
 0001:00018d50       ?getHashVal@HashXMLCh@xercesc_2_3@@UAEIQBXI@Z 12019d50 f   HashXMLCh.obj
 0001:00018d70       ?equals@HashXMLCh@xercesc_2_3@@UAE_NQBX0@Z 12019d70 f   HashXMLCh.obj
 0001:00018dd0       ?swapBytes@BitOps@xercesc_2_3@@SAGG@Z 12019dd0 f i HeaderDummy.obj
 0001:00018df0       ?swapBytes@BitOps@xercesc_2_3@@SAII@Z 12019df0 f i HeaderDummy.obj
 0001:00018e20       ??0EmptyStackException@xercesc_2_3@@QAE@QBDIW4Codes@XMLExcepts@1@@Z 12019e20 f i HeaderDummy.obj
 0001:00018e80       ??0EmptyStackException@xercesc_2_3@@QAE@ABV01@@Z 12019e80 f i HeaderDummy.obj
 0001:00018ea0       ??0EmptyStackException@xercesc_2_3@@QAE@QBDIW4Codes@XMLExcepts@1@QBG222@Z 12019ea0 f i HeaderDummy.obj
 0001:00018f10       ??0EmptyStackException@xercesc_2_3@@QAE@QBDIW4Codes@XMLExcepts@1@0000@Z 12019f10 f i HeaderDummy.obj
 0001:00018f80       ??1EmptyStackException@xercesc_2_3@@UAE@XZ 12019f80 f i HeaderDummy.obj
 0001:00018f90       ?duplicate@EmptyStackException@xercesc_2_3@@UBEPAVXMLException@2@XZ 12019f90 f i HeaderDummy.obj
 0001:00018ff0       ?getType@EmptyStackException@xercesc_2_3@@UBEPBGXZ 12019ff0 f i HeaderDummy.obj
 0001:00019000       ??_EEmptyStackException@xercesc_2_3@@UAEPAXI@Z 1201a000 f i HeaderDummy.obj
 0001:00019060       ??0InvalidCastException@xercesc_2_3@@QAE@QBDIW4Codes@XMLExcepts@1@@Z 1201a060 f i HeaderDummy.obj
 0001:000190c0       ??0InvalidCastException@xercesc_2_3@@QAE@ABV01@@Z 1201a0c0 f i HeaderDummy.obj
 0001:000190e0       ??0InvalidCastException@xercesc_2_3@@QAE@QBDIW4Codes@XMLExcepts@1@QBG222@Z 1201a0e0 f i HeaderDummy.obj
 0001:00019150       ??0InvalidCastException@xercesc_2_3@@QAE@QBDIW4Codes@XMLExcepts@1@0000@Z 1201a150 f i HeaderDummy.obj
 0001:000191c0       ??1InvalidCastException@xercesc_2_3@@UAE@XZ 1201a1c0 f i HeaderDummy.obj
 0001:000191d0       ?duplicate@InvalidCastException@xercesc_2_3@@UBEPAVXMLException@2@XZ 1201a1d0 f i HeaderDummy.obj
 0001:00019230       ?getType@InvalidCastException@xercesc_2_3@@UBEPBGXZ 1201a230 f i HeaderDummy.obj
 0001:00019240       ??_EInvalidCastException@xercesc_2_3@@UAEPAXI@Z 1201a240 f i HeaderDummy.obj
 0001:000192a0       ??0IOException@xercesc_2_3@@QAE@QBDIW4Codes@XMLExcepts@1@@Z 1201a2a0 f i HeaderDummy.obj
 0001:00019300       ??0IOException@xercesc_2_3@@QAE@ABV01@@Z 1201a300 f i HeaderDummy.obj
 0001:00019320       ??0IOException@xercesc_2_3@@QAE@QBDIW4Codes@XMLExcepts@1@QBG222@Z 1201a320 f i HeaderDummy.obj
 0001:00019390       ??0IOException@xercesc_2_3@@QAE@QBDIW4Codes@XMLExcepts@1@0000@Z 1201a390 f i HeaderDummy.obj
 0001:00019400       ??1IOException@xercesc_2_3@@UAE@XZ 1201a400 f i HeaderDummy.obj
 0001:00019410       ?duplicate@IOException@xercesc_2_3@@UBEPAVXMLException@2@XZ 1201a410 f i HeaderDummy.obj
 0001:00019470       ?getType@IOException@xercesc_2_3@@UBEPBGXZ 1201a470 f i HeaderDummy.obj
 0001:00019480       ??_EIOException@xercesc_2_3@@UAEPAXI@Z 1201a480 f i HeaderDummy.obj
 0001:000194e0       ??0UnexpectedEOFException@xercesc_2_3@@QAE@QBDIW4Codes@XMLExcepts@1@@Z 1201a4e0 f i HeaderDummy.obj
 0001:00019540       ??0UnexpectedEOFException@xercesc_2_3@@QAE@ABV01@@Z 1201a540 f i HeaderDummy.obj
 0001:00019560       ??0UnexpectedEOFException@xercesc_2_3@@QAE@QBDIW4Codes@XMLExcepts@1@QBG222@Z 1201a560 f i HeaderDummy.obj
 0001:000195d0       ??0UnexpectedEOFException@xercesc_2_3@@QAE@QBDIW4Codes@XMLExcepts@1@0000@Z 1201a5d0 f i HeaderDummy.obj
 0001:00019640       ??1UnexpectedEOFException@xercesc_2_3@@UAE@XZ 1201a640 f i HeaderDummy.obj
 0001:00019650       ?duplicate@UnexpectedEOFException@xercesc_2_3@@UBEPAVXMLException@2@XZ 1201a650 f i HeaderDummy.obj
 0001:000196b0       ?getType@UnexpectedEOFException@xercesc_2_3@@UBEPBGXZ 1201a6b0 f i HeaderDummy.obj
 0001:000196c0       ??_EUnexpectedEOFException@xercesc_2_3@@UAEPAXI@Z 1201a6c0 f i HeaderDummy.obj
 0001:00019720       ??0UnsupportedEncodingException@xercesc_2_3@@QAE@QBDIW4Codes@XMLExcepts@1@@Z 1201a720 f i HeaderDummy.obj
 0001:00019780       ??0UnsupportedEncodingException@xercesc_2_3@@QAE@ABV01@@Z 1201a780 f i HeaderDummy.obj
 0001:000197a0       ??0UnsupportedEncodingException@xercesc_2_3@@QAE@QBDIW4Codes@XMLExcepts@1@QBG222@Z 1201a7a0 f i HeaderDummy.obj
 0001:00019810       ??0UnsupportedEncodingException@xercesc_2_3@@QAE@QBDIW4Codes@XMLExcepts@1@0000@Z 1201a810 f i HeaderDummy.obj
 0001:00019880       ??1UnsupportedEncodingException@xercesc_2_3@@UAE@XZ 1201a880 f i HeaderDummy.obj
 0001:00019890       ?duplicate@UnsupportedEncodingException@xercesc_2_3@@UBEPAVXMLException@2@XZ 1201a890 f i HeaderDummy.obj
 0001:000198f0       ?getType@UnsupportedEncodingException@xercesc_2_3@@UBEPBGXZ 1201a8f0 f i HeaderDummy.obj
 0001:00019900       ??_EUnsupportedEncodingException@xercesc_2_3@@UAEPAXI@Z 1201a900 f i HeaderDummy.obj
 0001:00019960       ??0UTFDataFormatException@xercesc_2_3@@QAE@QBDIW4Codes@XMLExcepts@1@@Z 1201a960 f i HeaderDummy.obj
 0001:000199c0       ??0UTFDataFormatException@xercesc_2_3@@QAE@ABV01@@Z 1201a9c0 f i HeaderDummy.obj
 0001:000199e0       ??0UTFDataFormatException@xercesc_2_3@@QAE@QBDIW4Codes@XMLExcepts@1@QBG222@Z 1201a9e0 f i HeaderDummy.obj
 0001:00019a50       ??0UTFDataFormatException@xercesc_2_3@@QAE@QBDIW4Codes@XMLExcepts@1@0000@Z 1201aa50 f i HeaderDummy.obj
 0001:00019ac0       ??1UTFDataFormatException@xercesc_2_3@@UAE@XZ 1201aac0 f i HeaderDummy.obj
 0001:00019ad0       ?duplicate@UTFDataFormatException@xercesc_2_3@@UBEPAVXMLException@2@XZ 1201aad0 f i HeaderDummy.obj
 0001:00019b30       ?getType@UTFDataFormatException@xercesc_2_3@@UBEPBGXZ 1201ab30 f i HeaderDummy.obj
 0001:00019b40       ??_EUTFDataFormatException@xercesc_2_3@@UAEPAXI@Z 1201ab40 f i HeaderDummy.obj
 0001:00019ba0       ?getDataLength@HexBin@xercesc_2_3@@SAHQBG@Z 1201aba0 f   HexBin.obj
 0001:00019c80       ?isArrayByteHex@HexBin@xercesc_2_3@@SA_NQBG@Z 1201ac80 f   HexBin.obj
 0001:00019d40       ?isHex@HexBin@xercesc_2_3@@CA_NABG@Z 1201ad40 f   HexBin.obj
 0001:00019d60       ?init@HexBin@xercesc_2_3@@CAXXZ 1201ad60 f   HexBin.obj
 0001:00019dc0       ??_FKVStringPair@xercesc_2_3@@QAEXXZ 1201adc0 f i KVStringPair.obj
 0001:00019de0       ??0KVStringPair@xercesc_2_3@@QAE@QAVMemoryManager@1@@Z 1201ade0 f   KVStringPair.obj
 0001:00019e00       ??0KVStringPair@xercesc_2_3@@QAE@QBG0QAVMemoryManager@1@@Z 1201ae00 f   KVStringPair.obj
 0001:00019ed0       ??0KVStringPair@xercesc_2_3@@QAE@ABV01@@Z 1201aed0 f   KVStringPair.obj
 0001:00019fb0       ??1KVStringPair@xercesc_2_3@@QAE@XZ 1201afb0 f   KVStringPair.obj
 0001:00019fd0       ?setKey@KVStringPair@xercesc_2_3@@QAEXQBG@Z 1201afd0 f   KVStringPair.obj
 0001:0001a040       ?setValue@KVStringPair@xercesc_2_3@@QAEXQBG@Z 1201b040 f   KVStringPair.obj
 0001:0001a0b0       ?set@KVStringPair@xercesc_2_3@@QAEXQBG0@Z 1201b0b0 f   KVStringPair.obj
 0001:0001a180       ??0XMLMutex@xercesc_2_3@@QAE@XZ 1201b180 f   Mutexes.obj
 0001:0001a1a0       ??1XMLMutex@xercesc_2_3@@QAE@XZ 1201b1a0 f   Mutexes.obj
 0001:0001a1c0       ?lock@XMLMutex@xercesc_2_3@@QAEXXZ 1201b1c0 f   Mutexes.obj
 0001:0001a1d0       ?unlock@XMLMutex@xercesc_2_3@@QAEXXZ 1201b1d0 f   Mutexes.obj
 0001:0001a1e0       ??0XMLMutexLock@xercesc_2_3@@QAE@QAVXMLMutex@1@@Z 1201b1e0 f   Mutexes.obj
 0001:0001a200       ??1XMLMutexLock@xercesc_2_3@@QAE@XZ 1201b200 f   Mutexes.obj
 0001:0001a210       ?getPanicReasonString@PanicHandler@xercesc_2_3@@SAPBDW4PanicReasons@12@@Z 1201b210 f   PanicHandler.obj
 0001:0001a270       ??0MemoryManagerImpl@xercesc_2_3@@QAE@XZ 1201b270 f i PlatformUtils.obj
 0001:0001a280       ??1MemoryManagerImpl@xercesc_2_3@@UAE@XZ 1201b280 f i PlatformUtils.obj
 0001:0001a280       ??1MemoryManager@xercesc_2_3@@UAE@XZ 1201b280 f i PlatformUtils.obj
 0001:0001a290       ??_EMemoryManagerImpl@xercesc_2_3@@UAEPAXI@Z 1201b290 f i PlatformUtils.obj
 0001:0001a2f0       ?Initialize@XMLPlatformUtils@xercesc_2_3@@SAXQBD0QAVPanicHandler@2@QAVMemoryManager@2@@Z 1201b2f0 f   PlatformUtils.obj
 0001:0001a480       ?Terminate@XMLPlatformUtils@xercesc_2_3@@SAXXZ 1201b480 f   PlatformUtils.obj
 0001:0001a5d0       ?loadMsgSet@XMLPlatformUtils@xercesc_2_3@@SAPAVXMLMsgLoader@2@QBG@Z 1201b5d0 f   PlatformUtils.obj
 0001:0001a5e0       ?recognizeNEL@XMLPlatformUtils@xercesc_2_3@@SAX_N@Z 1201b5e0 f   PlatformUtils.obj
 0001:0001a640       ?isNELRecognized@XMLPlatformUtils@xercesc_2_3@@SA_NXZ 1201b640 f   PlatformUtils.obj
 0001:0001a650       ?strictIANAEncoding@XMLPlatformUtils@xercesc_2_3@@SAX_N@Z 1201b650 f   PlatformUtils.obj
 0001:0001a670       ?isStrictIANAEncoding@XMLPlatformUtils@xercesc_2_3@@SA_NXZ 1201b670 f   PlatformUtils.obj
 0001:0001a690       ??_FQName@xercesc_2_3@@QAEXXZ 1201b690 f i QName.obj
 0001:0001a6b0       ??0QName@xercesc_2_3@@QAE@QAVMemoryManager@1@@Z 1201b6b0 f   QName.obj
 0001:0001a6e0       ??0QName@xercesc_2_3@@QAE@QBG0IQAVMemoryManager@1@@Z 1201b6e0 f   QName.obj
 0001:0001a860       ??0QName@xercesc_2_3@@QAE@QBGIQAVMemoryManager@1@@Z 1201b860 f   QName.obj
 0001:0001a910       ??0QName@xercesc_2_3@@QAE@ABV01@@Z 1201b910 f   QName.obj
 0001:0001a9f0       ?getRawName@QName@xercesc_2_3@@QAEPAGXZ 1201b9f0 f   QName.obj
 0001:0001a9f0       ?getRawName@QName@xercesc_2_3@@QBEPBGXZ 1201b9f0 f   QName.obj
 0001:0001aab0       ?setName@QName@xercesc_2_3@@QAEXQBG0I@Z 1201bab0 f   QName.obj
 0001:0001abc0       ?setName@QName@xercesc_2_3@@QAEXQBGI@Z 1201bbc0 f   QName.obj
 0001:0001ad90       ?setPrefix@QName@xercesc_2_3@@QAEXPBG@Z 1201bd90 f   QName.obj
 0001:0001ae10       ?setNPrefix@QName@xercesc_2_3@@QAEXPBGI@Z 1201be10 f   QName.obj
 0001:0001ae70       ?setLocalPart@QName@xercesc_2_3@@QAEXPBG@Z 1201be70 f   QName.obj
 0001:0001aef0       ?setNLocalPart@QName@xercesc_2_3@@QAEXPBGI@Z 1201bef0 f   QName.obj
 0001:0001af50       ?setValues@QName@xercesc_2_3@@QAEXABV12@@Z 1201bf50 f   QName.obj
 0001:0001b040       ??8QName@xercesc_2_3@@QBE_NABV01@@Z 1201c040 f   QName.obj
 0001:0001b110       ?cleanUp@QName@xercesc_2_3@@QAEXXZ 1201c110 f   QName.obj
 0001:0001b110       ??1QName@xercesc_2_3@@QAE@XZ 1201c110 f   QName.obj
 0001:0001b150       ??0XMLStringPool@xercesc_2_3@@QAE@IQAVMemoryManager@1@@Z 1201c150 f   StringPool.obj
 0001:0001b2b0       ??1XMLStringPool@xercesc_2_3@@QAE@XZ 1201c2b0 f   StringPool.obj
 0001:0001b370       ?addOrFind@XMLStringPool@xercesc_2_3@@QAEIQBG@Z 1201c370 f   StringPool.obj
 0001:0001b400       ?exists@XMLStringPool@xercesc_2_3@@QBE_NQBG@Z 1201c400 f   StringPool.obj
 0001:0001b480       ?exists@XMLStringPool@xercesc_2_3@@QBE_NI@Z 1201c480 f   StringPool.obj
 0001:0001b4a0       ?flushAll@XMLStringPool@xercesc_2_3@@QAEXXZ 1201c4a0 f   StringPool.obj
 0001:0001b530       ?getId@XMLStringPool@xercesc_2_3@@QBEIQBG@Z 1201c530 f   StringPool.obj
 0001:0001b5c0       ?getValueForId@XMLStringPool@xercesc_2_3@@QBEPBGI@Z 1201c5c0 f   StringPool.obj
 0001:0001b610       ?addNewEntry@XMLStringPool@xercesc_2_3@@AAEIQBG@Z 1201c610 f   StringPool.obj
 0001:0001b920       ??0XMLTransService@xercesc_2_3@@IAE@XZ 1201c920 f   TransService.obj
 0001:0001bcd0       ??_EXMLTransService@xercesc_2_3@@UAEPAXI@Z 1201ccd0 f i TransService.obj
 0001:0001bd30       ??1XMLTransService@xercesc_2_3@@UAE@XZ 1201cd30 f   TransService.obj
 0001:0001bd40       ?addEncoding@XMLTransService@xercesc_2_3@@SAXQBGQAVENameMap@2@@Z 1201cd40 f   TransService.obj
 0001:0001bd60       ?makeNewTranscoderFor@XMLTransService@xercesc_2_3@@QAEPAVXMLTranscoder@2@QBDAAW4Codes@12@IQAVMemoryManager@2@@Z 1201cd60 f   TransService.obj
 0001:0001bdf0       ?makeNewTranscoderFor@XMLTransService@xercesc_2_3@@QAEPAVXMLTranscoder@2@QBGAAW4Codes@12@IQAVMemoryManager@2@@Z 1201cdf0 f   TransService.obj
 0001:0001bf70       ?makeNewTranscoderFor@XMLTransService@xercesc_2_3@@QAEPAVXMLTranscoder@2@W4Encodings@XMLRecognizer@2@AAW4Codes@12@IQAVMemoryManager@2@@Z 1201cf70 f   TransService.obj
 0001:0001c040       ?initTransService@XMLTransService@xercesc_2_3@@AAEXXZ 1201d040 f   TransService.obj
 0001:0001d8b0       ??0ENameMap@xercesc_2_3@@IAE@QBG@Z 1201e8b0 f i TransService.obj
 0001:0001d910       ??_GENameMap@xercesc_2_3@@UAEPAXI@Z 1201e910 f i TransService.obj
 0001:0001d910       ??_EENameMap@xercesc_2_3@@UAEPAXI@Z 1201e910 f i TransService.obj
 0001:0001d940       ?strictIANAEncoding@XMLTransService@xercesc_2_3@@AAEX_N@Z 1201e940 f   TransService.obj
 0001:0001d950       ?isStrictIANAEncoding@XMLTransService@xercesc_2_3@@AAE_NXZ 1201e950 f   TransService.obj
 0001:0001d960       ??1XMLTranscoder@xercesc_2_3@@UAE@XZ 1201e960 f   TransService.obj
 0001:0001d980       ??_EXMLTranscoder@xercesc_2_3@@UAEPAXI@Z 1201e980 f i TransService.obj
 0001:0001d9e0       ??0XMLTranscoder@xercesc_2_3@@IAE@QBGIQAVMemoryManager@1@@Z 1201e9e0 f   TransService.obj
 0001:0001da60       ??0XMLLCPTranscoder@xercesc_2_3@@IAE@XZ 1201ea60 f   TransService.obj
 0001:0001da70       ??_EXMLLCPTranscoder@xercesc_2_3@@UAEPAXI@Z 1201ea70 f i TransService.obj
 0001:0001dad0       ??1XMLLCPTranscoder@xercesc_2_3@@UAE@XZ 1201ead0 f   TransService.obj
 0001:0001dae0       ?put@?$RefHashTableOf@VENameMap@xercesc_2_3@@@xercesc_2_3@@QAEXPAXQAVENameMap@2@@Z 1201eae0 f i TransService.obj
 0001:0001dcf0       ?makeNew@?$ENameMapFor@VXMLChTranscoder@xercesc_2_3@@@xercesc_2_3@@UBEPAVXMLTranscoder@2@IQAVMemoryManager@2@@Z 1201ecf0 f i TransService.obj
 0001:0001dd60       ?makeNew@?$ENameMapFor@VXMLASCIITranscoder@xercesc_2_3@@@xercesc_2_3@@UBEPAVXMLTranscoder@2@IQAVMemoryManager@2@@Z 1201ed60 f i TransService.obj
 0001:0001ddd0       ?makeNew@?$ENameMapFor@VXMLUTF8Transcoder@xercesc_2_3@@@xercesc_2_3@@UBEPAVXMLTranscoder@2@IQAVMemoryManager@2@@Z 1201edd0 f i TransService.obj
 0001:0001de40       ??0?$ENameMapFor@VXML88591Transcoder@xercesc_2_3@@@xercesc_2_3@@QAE@QBG@Z 1201ee40 f i TransService.obj
 0001:0001dea0       ?makeNew@?$ENameMapFor@VXML88591Transcoder@xercesc_2_3@@@xercesc_2_3@@UBEPAVXMLTranscoder@2@IQAVMemoryManager@2@@Z 1201eea0 f i TransService.obj
 0001:0001df10       ??0?$EEndianNameMapFor@VXMLUTF16Transcoder@xercesc_2_3@@@xercesc_2_3@@QAE@QBG_N@Z 1201ef10 f i TransService.obj
 0001:0001df80       ?makeNew@?$EEndianNameMapFor@VXMLUTF16Transcoder@xercesc_2_3@@@xercesc_2_3@@UBEPAVXMLTranscoder@2@IQAVMemoryManager@2@@Z 1201ef80 f i TransService.obj
 0001:0001e000       ??0?$EEndianNameMapFor@VXMLUCS4Transcoder@xercesc_2_3@@@xercesc_2_3@@QAE@QBG_N@Z 1201f000 f i TransService.obj
 0001:0001e070       ?makeNew@?$EEndianNameMapFor@VXMLUCS4Transcoder@xercesc_2_3@@@xercesc_2_3@@UBEPAVXMLTranscoder@2@IQAVMemoryManager@2@@Z 1201f070 f i TransService.obj
 0001:0001e0f0       ??0?$ENameMapFor@VXMLEBCDICTranscoder@xercesc_2_3@@@xercesc_2_3@@QAE@QBG@Z 1201f0f0 f i TransService.obj
 0001:0001e150       ?makeNew@?$ENameMapFor@VXMLEBCDICTranscoder@xercesc_2_3@@@xercesc_2_3@@UBEPAVXMLTranscoder@2@IQAVMemoryManager@2@@Z 1201f150 f i TransService.obj
 0001:0001e1c0       ??0?$ENameMapFor@VXMLIBM1140Transcoder@xercesc_2_3@@@xercesc_2_3@@QAE@QBG@Z 1201f1c0 f i TransService.obj
 0001:0001e220       ?makeNew@?$ENameMapFor@VXMLIBM1140Transcoder@xercesc_2_3@@@xercesc_2_3@@UBEPAVXMLTranscoder@2@IQAVMemoryManager@2@@Z 1201f220 f i TransService.obj
 0001:0001e290       ??0?$ENameMapFor@VXMLWin1252Transcoder@xercesc_2_3@@@xercesc_2_3@@QAE@QBG@Z 1201f290 f i TransService.obj
 0001:0001e2f0       ?makeNew@?$ENameMapFor@VXMLWin1252Transcoder@xercesc_2_3@@@xercesc_2_3@@UBEPAVXMLTranscoder@2@IQAVMemoryManager@2@@Z 1201f2f0 f i TransService.obj
 0001:0001e360       ??_G?$RefVectorOf@VENameMap@xercesc_2_3@@@xercesc_2_3@@UAEPAXI@Z 1201f360 f i TransService.obj
 0001:0001e360       ??_E?$RefVectorOf@VENameMap@xercesc_2_3@@@xercesc_2_3@@UAEPAXI@Z 1201f360 f i TransService.obj
 0001:0001e380       ??1?$RefVectorOf@VENameMap@xercesc_2_3@@@xercesc_2_3@@UAE@XZ 1201f380 f i TransService.obj
 0001:0001e400       ??1?$BaseRefVectorOf@VENameMap@xercesc_2_3@@@xercesc_2_3@@UAE@XZ 1201f400 f i TransService.obj
 0001:0001e410       ??1?$ENameMapFor@VXMLWin1252Transcoder@xercesc_2_3@@@xercesc_2_3@@UAE@XZ 1201f410 f i TransService.obj
 0001:0001e410       ??1?$ENameMapFor@VXMLIBM1140Transcoder@xercesc_2_3@@@xercesc_2_3@@UAE@XZ 1201f410 f i TransService.obj
 0001:0001e410       ??1?$ENameMapFor@VXMLEBCDICTranscoder@xercesc_2_3@@@xercesc_2_3@@UAE@XZ 1201f410 f i TransService.obj
 0001:0001e410       ??1?$ENameMapFor@VXML88591Transcoder@xercesc_2_3@@@xercesc_2_3@@UAE@XZ 1201f410 f i TransService.obj
 0001:0001e410       ??1?$ENameMapFor@VXMLChTranscoder@xercesc_2_3@@@xercesc_2_3@@UAE@XZ 1201f410 f i TransService.obj
 0001:0001e410       ??1?$ENameMapFor@VXMLASCIITranscoder@xercesc_2_3@@@xercesc_2_3@@UAE@XZ 1201f410 f i TransService.obj
 0001:0001e410       ??1?$EEndianNameMapFor@VXMLUCS4Transcoder@xercesc_2_3@@@xercesc_2_3@@UAE@XZ 1201f410 f i TransService.obj
 0001:0001e410       ??1?$ENameMapFor@VXMLUTF8Transcoder@xercesc_2_3@@@xercesc_2_3@@UAE@XZ 1201f410 f i TransService.obj
 0001:0001e410       ??1?$EEndianNameMapFor@VXMLUTF16Transcoder@xercesc_2_3@@@xercesc_2_3@@UAE@XZ 1201f410 f i TransService.obj
 0001:0001e430       ??_E?$ENameMapFor@VXMLIBM1140Transcoder@xercesc_2_3@@@xercesc_2_3@@UAEPAXI@Z 1201f430 f i TransService.obj
 0001:0001e430       ??_E?$ENameMapFor@VXMLASCIITranscoder@xercesc_2_3@@@xercesc_2_3@@UAEPAXI@Z 1201f430 f i TransService.obj
 0001:0001e430       ??_G?$ENameMapFor@VXMLIBM1140Transcoder@xercesc_2_3@@@xercesc_2_3@@UAEPAXI@Z 1201f430 f i TransService.obj
 0001:0001e430       ??_G?$EEndianNameMapFor@VXMLUCS4Transcoder@xercesc_2_3@@@xercesc_2_3@@UAEPAXI@Z 1201f430 f i TransService.obj
 0001:0001e430       ??_E?$EEndianNameMapFor@VXMLUTF16Transcoder@xercesc_2_3@@@xercesc_2_3@@UAEPAXI@Z 1201f430 f i TransService.obj
 0001:0001e430       ??_E?$ENameMapFor@VXMLChTranscoder@xercesc_2_3@@@xercesc_2_3@@UAEPAXI@Z 1201f430 f i TransService.obj
 0001:0001e430       ??_G?$ENameMapFor@VXMLEBCDICTranscoder@xercesc_2_3@@@xercesc_2_3@@UAEPAXI@Z 1201f430 f i TransService.obj
 0001:0001e430       ??_G?$ENameMapFor@VXML88591Transcoder@xercesc_2_3@@@xercesc_2_3@@UAEPAXI@Z 1201f430 f i TransService.obj
 0001:0001e430       ??_E?$ENameMapFor@VXMLWin1252Transcoder@xercesc_2_3@@@xercesc_2_3@@UAEPAXI@Z 1201f430 f i TransService.obj
 0001:0001e430       ??_G?$ENameMapFor@VXMLUTF8Transcoder@xercesc_2_3@@@xercesc_2_3@@UAEPAXI@Z 1201f430 f i TransService.obj
 0001:0001e430       ??_E?$ENameMapFor@VXML88591Transcoder@xercesc_2_3@@@xercesc_2_3@@UAEPAXI@Z 1201f430 f i TransService.obj
 0001:0001e430       ??_E?$EEndianNameMapFor@VXMLUCS4Transcoder@xercesc_2_3@@@xercesc_2_3@@UAEPAXI@Z 1201f430 f i TransService.obj
 0001:0001e430       ??_E?$ENameMapFor@VXMLEBCDICTranscoder@xercesc_2_3@@@xercesc_2_3@@UAEPAXI@Z 1201f430 f i TransService.obj
 0001:0001e430       ??_G?$ENameMapFor@VXMLASCIITranscoder@xercesc_2_3@@@xercesc_2_3@@UAEPAXI@Z 1201f430 f i TransService.obj
 0001:0001e430       ??_G?$EEndianNameMapFor@VXMLUTF16Transcoder@xercesc_2_3@@@xercesc_2_3@@UAEPAXI@Z 1201f430 f i TransService.obj
 0001:0001e430       ??_E?$ENameMapFor@VXMLUTF8Transcoder@xercesc_2_3@@@xercesc_2_3@@UAEPAXI@Z 1201f430 f i TransService.obj
 0001:0001e430       ??_G?$ENameMapFor@VXMLWin1252Transcoder@xercesc_2_3@@@xercesc_2_3@@UAEPAXI@Z 1201f430 f i TransService.obj
 0001:0001e430       ??_G?$ENameMapFor@VXMLChTranscoder@xercesc_2_3@@@xercesc_2_3@@UAEPAXI@Z 1201f430 f i TransService.obj
 0001:0001e450       ??2XMemory@xercesc_2_3@@SAPAXI@Z 1201f450 f   XMemory.obj
 0001:0001e470       ??2XMemory@xercesc_2_3@@SAPAXIPAVMemoryManager@1@@Z 1201f470 f   XMemory.obj
 0001:0001e490       ??3XMemory@xercesc_2_3@@SAXPAX@Z 1201f490 f   XMemory.obj
 0001:0001e490       ??3XMemory@xercesc_2_3@@SAXPAXPAVMemoryManager@1@@Z 1201f490 f   XMemory.obj
 0001:0001e4b0       ??1XML256TableTranscoder@xercesc_2_3@@UAE@XZ 1201f4b0 f   XML256TableTranscoder.obj
 0001:0001e4c0       ??_EXML256TableTranscoder@xercesc_2_3@@UAEPAXI@Z 1201f4c0 f i XML256TableTranscoder.obj
 0001:0001e520       ?transcodeFrom@XML256TableTranscoder@xercesc_2_3@@UAEIQBEIQAGIAAIQAE@Z 1201f520 f   XML256TableTranscoder.obj
 0001:0001e590       ?transcodeTo@XML256TableTranscoder@xercesc_2_3@@UAEIQBGIQAEIAAIW4UnRepOpts@XMLTranscoder@2@@Z 1201f590 f   XML256TableTranscoder.obj
 0001:0001e650       ?canTranscodeTo@XML256TableTranscoder@xercesc_2_3@@UBE_NI@Z 1201f650 f   XML256TableTranscoder.obj
 0001:0001e670       ??0XML256TableTranscoder@xercesc_2_3@@IAE@QBGI0QBUTransRec@XMLTransService@1@I@Z 1201f670 f   XML256TableTranscoder.obj
 0001:0001e6b0       ?xlatOneTo@XML256TableTranscoder@xercesc_2_3@@IBEEG@Z 1201f6b0 f   XML256TableTranscoder.obj
 0001:0001e710       ??0XML88591Transcoder@xercesc_2_3@@QAE@QBGI@Z 1201f710 f   XML88591Transcoder.obj
 0001:0001e740       ??_EXML88591Transcoder@xercesc_2_3@@UAEPAXI@Z 1201f740 f i XML88591Transcoder.obj
 0001:0001e7a0       ??1XML88591Transcoder@xercesc_2_3@@UAE@XZ 1201f7a0 f   XML88591Transcoder.obj
 0001:0001e7b0       ?transcodeFrom@XML88591Transcoder@xercesc_2_3@@UAEIQBEIQAGIAAIQAE@Z 1201f7b0 f   XML88591Transcoder.obj
 0001:0001e810       ?transcodeTo@XML88591Transcoder@xercesc_2_3@@UAEIQBGIQAEIAAIW4UnRepOpts@XMLTranscoder@2@@Z 1201f810 f   XML88591Transcoder.obj
 0001:0001e8c0       ?canTranscodeTo@XML88591Transcoder@xercesc_2_3@@UBE_NI@Z 1201f8c0 f   XML88591Transcoder.obj
 0001:0001e8d0       ??_FXMLAbstractDoubleFloat@xercesc_2_3@@QAEXXZ 1201f8d0 f i XMLAbstractDoubleFloat.obj
 0001:0001e8e0       ?isSpecialValue@XMLAbstractDoubleFloat@xercesc_2_3@@ABE_NXZ 1201f8e0 f i XMLAbstractDoubleFloat.obj
 0001:0001e8f0       ??0NumberFormatException@xercesc_2_3@@QAE@QBDIW4Codes@XMLExcepts@1@@Z 1201f8f0 f i XMLAbstractDoubleFloat.obj
 0001:0001e950       ??0NumberFormatException@xercesc_2_3@@QAE@ABV01@@Z 1201f950 f i XMLAbstractDoubleFloat.obj
 0001:0001e970       ??0NumberFormatException@xercesc_2_3@@QAE@QBDIW4Codes@XMLExcepts@1@QBG222@Z 1201f970 f i XMLAbstractDoubleFloat.obj
 0001:0001e9e0       ??0NumberFormatException@xercesc_2_3@@QAE@QBDIW4Codes@XMLExcepts@1@0000@Z 1201f9e0 f i XMLAbstractDoubleFloat.obj
 0001:0001ea50       ??1NumberFormatException@xercesc_2_3@@UAE@XZ 1201fa50 f i XMLAbstractDoubleFloat.obj
 0001:0001ea60       ?duplicate@NumberFormatException@xercesc_2_3@@UBEPAVXMLException@2@XZ 1201fa60 f i XMLAbstractDoubleFloat.obj
 0001:0001eac0       ?getType@NumberFormatException@xercesc_2_3@@UBEPBGXZ 1201fac0 f i XMLAbstractDoubleFloat.obj
 0001:0001ead0       ??_ENumberFormatException@xercesc_2_3@@UAEPAXI@Z 1201fad0 f i XMLAbstractDoubleFloat.obj
 0001:0001eb30       ??0XMLAbstractDoubleFloat@xercesc_2_3@@IAE@QAVMemoryManager@1@@Z 1201fb30 f   XMLAbstractDoubleFloat.obj
 0001:0001eb70       ??_EXMLAbstractDoubleFloat@xercesc_2_3@@UAEPAXI@Z 1201fb70 f i XMLAbstractDoubleFloat.obj
 0001:0001ebd0       ??1XMLAbstractDoubleFloat@xercesc_2_3@@UAE@XZ 1201fbd0 f   XMLAbstractDoubleFloat.obj
 0001:0001ec40       ?init@XMLAbstractDoubleFloat@xercesc_2_3@@IAEXQBG@Z 1201fc40 f   XMLAbstractDoubleFloat.obj
 0001:0001eed0       ?toString@XMLAbstractDoubleFloat@xercesc_2_3@@UBEPAGXZ 1201fed0 f   XMLAbstractDoubleFloat.obj
 0001:0001ef20       ?getFormattedString@XMLAbstractDoubleFloat@xercesc_2_3@@UBEPBGXZ 1201ff20 f   XMLAbstractDoubleFloat.obj
 0001:0001ef50       ?formatString@XMLAbstractDoubleFloat@xercesc_2_3@@AAEXXZ 1201ff50 f   XMLAbstractDoubleFloat.obj
 0001:0001f040       ?compareValues@XMLAbstractDoubleFloat@xercesc_2_3@@KAHQBV12@0@Z 12020040 f   XMLAbstractDoubleFloat.obj
 0001:0001f1a0       ?compareSpecial@XMLAbstractDoubleFloat@xercesc_2_3@@CAHQBV12@0@Z 120201a0 f   XMLAbstractDoubleFloat.obj
 0001:0001f220       ?normalizeZero@XMLAbstractDoubleFloat@xercesc_2_3@@AAEXQAG@Z 12020220 f   XMLAbstractDoubleFloat.obj
 0001:0001f350       ??0XMLASCIITranscoder@xercesc_2_3@@QAE@QBGI@Z 12020350 f   XMLASCIITranscoder.obj
 0001:0001f380       ??_EXMLASCIITranscoder@xercesc_2_3@@UAEPAXI@Z 12020380 f i XMLASCIITranscoder.obj
 0001:0001f3e0       ??1XMLASCIITranscoder@xercesc_2_3@@UAE@XZ 120203e0 f   XMLASCIITranscoder.obj
 0001:0001f3f0       ?transcodeFrom@XMLASCIITranscoder@xercesc_2_3@@UAEIQBEIQAGIAAIQAE@Z 120203f0 f   XMLASCIITranscoder.obj
 0001:0001f4b0       ?transcodeTo@XMLASCIITranscoder@xercesc_2_3@@UAEIQBGIQAEIAAIW4UnRepOpts@XMLTranscoder@2@@Z 120204b0 f   XMLASCIITranscoder.obj
 0001:0001f560       ?canTranscodeTo@XMLASCIITranscoder@xercesc_2_3@@UBE_NI@Z 12020560 f   XMLASCIITranscoder.obj
 0001:0001f570       ?toString@XMLBigDecimal@xercesc_2_3@@UBEPAGXZ 12020570 f i XMLBigDecimal.obj
 0001:0001f5c0       ??0XMLBigDecimal@xercesc_2_3@@QAE@QBGQAVMemoryManager@1@@Z 120205c0 f   XMLBigDecimal.obj
 0001:0001f6f0       ??_EXMLBigDecimal@xercesc_2_3@@UAEPAXI@Z 120206f0 f i XMLBigDecimal.obj
 0001:0001f750       ??1XMLBigDecimal@xercesc_2_3@@UAE@XZ 12020750 f   XMLBigDecimal.obj
 0001:0001f7c0       ?cleanUp@XMLBigDecimal@xercesc_2_3@@AAEXXZ 120207c0 f   XMLBigDecimal.obj
 0001:0001f7f0       ?parseBigDecimal@XMLBigDecimal@xercesc_2_3@@AAEXQBG@Z 120207f0 f   XMLBigDecimal.obj
 0001:0001f9f0       ?compareValues@XMLBigDecimal@xercesc_2_3@@SAHQBV12@0@Z 120209f0 f   XMLBigDecimal.obj
 0001:0001fa40       ?toCompare@XMLBigDecimal@xercesc_2_3@@QBEHABV12@@Z 12020a40 f   XMLBigDecimal.obj
 0001:0001fae0       ?getTotalDigit@XMLBigInteger@xercesc_2_3@@QBEHXZ 12020ae0 f i XMLBigInteger.obj
 0001:0001fb10       ??8XMLBigInteger@xercesc_2_3@@QBE_NABV01@@Z 12020b10 f i XMLBigInteger.obj
 0001:0001fb30       ?toString@XMLBigInteger@xercesc_2_3@@QBEPAGXZ 12020b30 f i XMLBigInteger.obj
 0001:0001fb80       ?parseBigInteger@XMLBigInteger@xercesc_2_3@@SAXQBGQAGAAH@Z 12020b80 f   XMLBigInteger.obj
 0001:0001fd10       ??0XMLBigInteger@xercesc_2_3@@QAE@QBGQAVMemoryManager@1@@Z 12020d10 f   XMLBigInteger.obj
 0001:0001ff00       ??1XMLBigInteger@xercesc_2_3@@QAE@XZ 12020f00 f   XMLBigInteger.obj
 0001:0001ff30       ??0XMLBigInteger@xercesc_2_3@@QAE@ABV01@@Z 12020f30 f   XMLBigInteger.obj
 0001:0001fff0       ?compareValues@XMLBigInteger@xercesc_2_3@@SAHQBV12@0@Z 12020ff0 f   XMLBigInteger.obj
 0001:00020110       ?multiply@XMLBigInteger@xercesc_2_3@@QAEXI@Z 12021110 f   XMLBigInteger.obj
 0001:000201d0       ?divide@XMLBigInteger@xercesc_2_3@@QAEXI@Z 120211d0 f   XMLBigInteger.obj
 0001:00020260       ?intValue@XMLBigInteger@xercesc_2_3@@QBEHXZ 12021260 f   XMLBigInteger.obj
 0001:00020280       ?isAllSpaces@XMLChar1_0@xercesc_2_3@@SA_NQBGI@Z 12021280 f   XMLChar.obj
 0001:000202b0       ?containsWhiteSpace@XMLChar1_0@xercesc_2_3@@SA_NQBGI@Z 120212b0 f   XMLChar.obj
 0001:000202e0       ?isValidNCName@XMLChar1_0@xercesc_2_3@@SA_NQBGI@Z 120212e0 f   XMLChar.obj
 0001:00020340       ?isValidName@XMLChar1_0@xercesc_2_3@@SA_NQBGI@Z 12021340 f   XMLChar.obj
 0001:00020380       ?isValidQName@XMLChar1_0@xercesc_2_3@@SA_NQBGI@Z 12021380 f   XMLChar.obj
 0001:00020460       ?isPublicIdChar@XMLChar1_0@xercesc_2_3@@SA_NGG@Z 12021460 f   XMLChar.obj
 0001:000204d0       ?enableNELWS@XMLChar1_0@xercesc_2_3@@SAXXZ 120214d0 f   XMLChar.obj
 0001:000204f0       ?isAllSpaces@XMLChar1_1@xercesc_2_3@@SA_NQBGI@Z 120214f0 f   XMLChar.obj
 0001:00020520       ?containsWhiteSpace@XMLChar1_1@xercesc_2_3@@SA_NQBGI@Z 12021520 f   XMLChar.obj
 0001:00020550       ?isValidNCName@XMLChar1_1@xercesc_2_3@@SA_NQBGI@Z 12021550 f   XMLChar.obj
 0001:00020600       ?isValidName@XMLChar1_1@xercesc_2_3@@SA_NQBGI@Z 12021600 f   XMLChar.obj
 0001:000206a0       ?isValidQName@XMLChar1_1@xercesc_2_3@@SA_NQBGI@Z 120216a0 f   XMLChar.obj
 0001:00020700       ?isPublicIdChar@XMLChar1_1@xercesc_2_3@@SA_NGG@Z 12021700 f   XMLChar.obj
 0001:00020770       ??0XMLChTranscoder@xercesc_2_3@@QAE@QBGI@Z 12021770 f   XMLChTranscoder.obj
 0001:000207a0       ??_EXMLChTranscoder@xercesc_2_3@@UAEPAXI@Z 120217a0 f i XMLChTranscoder.obj
 0001:00020800       ??1XMLChTranscoder@xercesc_2_3@@UAE@XZ 12021800 f   XMLChTranscoder.obj
 0001:00020810       ?transcodeFrom@XMLChTranscoder@xercesc_2_3@@UAEIQBEIQAGIAAIQAE@Z 12021810 f   XMLChTranscoder.obj
 0001:00020870       ?transcodeTo@XMLChTranscoder@xercesc_2_3@@UAEIQBGIQAEIAAIW4UnRepOpts@XMLTranscoder@2@@Z 12021870 f   XMLChTranscoder.obj
 0001:000208b0       ??0SchemaDateTimeException@xercesc_2_3@@QAE@QBDIW4Codes@XMLExcepts@1@@Z 120218b0 f i XMLDateTime.obj
 0001:00020910       ??0SchemaDateTimeException@xercesc_2_3@@QAE@ABV01@@Z 12021910 f i XMLDateTime.obj
 0001:00020930       ??0SchemaDateTimeException@xercesc_2_3@@QAE@QBDIW4Codes@XMLExcepts@1@QBG222@Z 12021930 f i XMLDateTime.obj
 0001:000209a0       ??0SchemaDateTimeException@xercesc_2_3@@QAE@QBDIW4Codes@XMLExcepts@1@0000@Z 120219a0 f i XMLDateTime.obj
 0001:00020a10       ??1SchemaDateTimeException@xercesc_2_3@@UAE@XZ 12021a10 f i XMLDateTime.obj
 0001:00020a20       ?duplicate@SchemaDateTimeException@xercesc_2_3@@UBEPAVXMLException@2@XZ 12021a20 f i XMLDateTime.obj
 0001:00020a80       ?getType@SchemaDateTimeException@xercesc_2_3@@UBEPBGXZ 12021a80 f i XMLDateTime.obj
 0001:00020a90       ??_ESchemaDateTimeException@xercesc_2_3@@UAEPAXI@Z 12021a90 f i XMLDateTime.obj
 0001:00020af0       ??_FXMLDateTime@xercesc_2_3@@QAEXXZ 12021af0 f i XMLDateTime.obj
 0001:00020b00       ?setBuffer@XMLDateTime@xercesc_2_3@@QAEXQBG@Z 12021b00 f i XMLDateTime.obj
 0001:00020bb0       ?reset@XMLDateTime@xercesc_2_3@@AAEXXZ 12021bb0 f i XMLDateTime.obj
 0001:00020bf0       ?copy@XMLDateTime@xercesc_2_3@@AAEXABV12@@Z 12021bf0 f i XMLDateTime.obj
 0001:00020ca0       ?assertBuffer@XMLDateTime@xercesc_2_3@@ABEXXZ 12021ca0 f i XMLDateTime.obj
 0001:00020ce0       ?initParser@XMLDateTime@xercesc_2_3@@AAEXXZ 12021ce0 f i XMLDateTime.obj
 0001:00020d30       ?isNormalized@XMLDateTime@xercesc_2_3@@ABE_NXZ 12021d30 f i XMLDateTime.obj
 0001:00020d40       ?getRetVal@XMLDateTime@xercesc_2_3@@CAHHH@Z 12021d40 f i XMLDateTime.obj
 0001:00020d70       ?compare@XMLDateTime@xercesc_2_3@@SAHQBV12@0_N@Z 12021d70 f   XMLDateTime.obj
 0001:000210e0       ?addDuration@XMLDateTime@xercesc_2_3@@CAXPAV12@QBV12@H@Z 120220e0 f   XMLDateTime.obj
 0001:00021340       ?compareResult@XMLDateTime@xercesc_2_3@@CAHFF_N@Z 12022340 f   XMLDateTime.obj
 0001:00021390       ?compare@XMLDateTime@xercesc_2_3@@SAHQBV12@0@Z 12022390 f   XMLDateTime.obj
 0001:00021440       ?compareResult@XMLDateTime@xercesc_2_3@@CAHQBV12@0_NH@Z 12022440 f   XMLDateTime.obj
 0001:000215b0       ?compareOrder@XMLDateTime@xercesc_2_3@@SAHQBV12@0@Z 120225b0 f   XMLDateTime.obj
 0001:00021800       ??1XMLDateTime@xercesc_2_3@@UAE@XZ 12022800 f   XMLDateTime.obj
 0001:00021860       ??_EXMLDateTime@xercesc_2_3@@UAEPAXI@Z 12022860 f i XMLDateTime.obj
 0001:000218c0       ??0XMLDateTime@xercesc_2_3@@QAE@QAVMemoryManager@1@@Z 120228c0 f   XMLDateTime.obj
 0001:00021940       ??0XMLDateTime@xercesc_2_3@@QAE@QBGQAVMemoryManager@1@@Z 12022940 f   XMLDateTime.obj
 0001:00021a30       ??0XMLDateTime@xercesc_2_3@@QAE@ABV01@@Z 12022a30 f   XMLDateTime.obj
 0001:00021b20       ??4XMLDateTime@xercesc_2_3@@QAEAAV01@ABV01@@Z 12022b20 f   XMLDateTime.obj
 0001:00021be0       ?toString@XMLDateTime@xercesc_2_3@@UBEPAGXZ 12022be0 f   XMLDateTime.obj
 0001:00021c70       ?getRawData@XMLDateTime@xercesc_2_3@@UBEPAGXZ 12022c70 f   XMLDateTime.obj
 0001:00021cb0       ?getFormattedString@XMLDateTime@xercesc_2_3@@UBEPBGXZ 12022cb0 f   XMLDateTime.obj
 0001:00021cc0       ?parseDateTime@XMLDateTime@xercesc_2_3@@QAEXXZ 12022cc0 f   XMLDateTime.obj
 0001:00021d70       ?parseDate@XMLDateTime@xercesc_2_3@@QAEXXZ 12022d70 f   XMLDateTime.obj
 0001:00021e50       ?parseTime@XMLDateTime@xercesc_2_3@@QAEXXZ 12022e50 f   XMLDateTime.obj
 0001:00021ec0       ?parseDay@XMLDateTime@xercesc_2_3@@QAEXXZ 12022ec0 f   XMLDateTime.obj
 0001:00022000       ?parseMonth@XMLDateTime@xercesc_2_3@@QAEXXZ 12023000 f   XMLDateTime.obj
 0001:00022160       ?parseYear@XMLDateTime@xercesc_2_3@@QAEXXZ 12023160 f   XMLDateTime.obj
 0001:00022240       ?parseMonthDay@XMLDateTime@xercesc_2_3@@QAEXXZ 12023240 f   XMLDateTime.obj
 0001:00022390       ?parseYearMonth@XMLDateTime@xercesc_2_3@@QAEXXZ 12023390 f   XMLDateTime.obj
 0001:00022470       ?parseDuration@XMLDateTime@xercesc_2_3@@QAEXXZ 12023470 f   XMLDateTime.obj
 0001:000228a0       ?getDate@XMLDateTime@xercesc_2_3@@AAEXXZ 120238a0 f   XMLDateTime.obj
 0001:00022950       ?getTime@XMLDateTime@xercesc_2_3@@AAEXXZ 12023950 f   XMLDateTime.obj
 0001:00022b20       ?getYearMonth@XMLDateTime@xercesc_2_3@@AAEXXZ 12023b20 f   XMLDateTime.obj
 0001:00022c30       ?parseTimeZone@XMLDateTime@xercesc_2_3@@AAEXXZ 12023c30 f   XMLDateTime.obj
 0001:00022cb0       ?getTimeZone@XMLDateTime@xercesc_2_3@@AAEXH@Z 12023cb0 f   XMLDateTime.obj
 0001:00022d70       ?normalize@XMLDateTime@xercesc_2_3@@AAEXXZ 12023d70 f   XMLDateTime.obj
 0001:00022f50       ?validateDateTime@XMLDateTime@xercesc_2_3@@ABEXXZ 12023f50 f   XMLDateTime.obj
 0001:00023200       ?indexOf@XMLDateTime@xercesc_2_3@@ABEHHHG@Z 12024200 f   XMLDateTime.obj
 0001:00023230       ?findUTCSign@XMLDateTime@xercesc_2_3@@AAEHH@Z 12024230 f   XMLDateTime.obj
 0001:00023280       ?parseInt@XMLDateTime@xercesc_2_3@@ABEHHH@Z 12024280 f   XMLDateTime.obj
 0001:00023330       ?parseIntYear@XMLDateTime@xercesc_2_3@@ABEHH@Z 12024330 f   XMLDateTime.obj
 0001:000233e0       ?compareValues@XMLDouble@xercesc_2_3@@SAHQBV12@0@Z 120243e0 f i XMLDouble.obj
 0001:000233e0       ?compareValues@XMLFloat@xercesc_2_3@@SAHQBV12@0@Z 120243e0 f i XMLDouble.obj
 0001:00023400       ??0XMLDouble@xercesc_2_3@@QAE@QBGQAVMemoryManager@1@@Z 12024400 f   XMLDouble.obj
 0001:00023460       ??_EXMLDouble@xercesc_2_3@@UAEPAXI@Z 12024460 f i XMLDouble.obj
 0001:000234c0       ??1XMLDouble@xercesc_2_3@@UAE@XZ 120244c0 f   XMLDouble.obj
 0001:000234d0       ?checkBoundary@XMLDouble@xercesc_2_3@@MAEXQBG@Z 120244d0 f   XMLDouble.obj
 0001:00023640       ?xlatThisOne@XMLEBCDICTranscoder@xercesc_2_3@@SAGE@Z 12024640 f   XMLEBCDICTranscoder.obj
 0001:00023660       ??0XMLEBCDICTranscoder@xercesc_2_3@@QAE@QBGI@Z 12024660 f   XMLEBCDICTranscoder.obj
 0001:00023690       ??_EXMLEBCDICTranscoder@xercesc_2_3@@UAEPAXI@Z 12024690 f i XMLEBCDICTranscoder.obj
 0001:000236f0       ??1XMLEBCDICTranscoder@xercesc_2_3@@UAE@XZ 120246f0 f   XMLEBCDICTranscoder.obj
 0001:00023700       ?registerCleanup@XMLRegisterCleanup@xercesc_2_3@@QAEXP6AXXZ@Z 12024700 f i XMLException.obj
 0001:00023790       ??1XMLException@xercesc_2_3@@UAE@XZ 12024790 f   XMLException.obj
 0001:000237c0       ??_EXMLException@xercesc_2_3@@UAEPAXI@Z 120247c0 f i XMLException.obj
 0001:00023840       ?setPosition@XMLException@xercesc_2_3@@QAEXQBDI@Z 12024840 f   XMLException.obj
 0001:00023880       ??0XMLException@xercesc_2_3@@QAE@XZ 12024880 f   XMLException.obj
 0001:000238a0       ??0XMLException@xercesc_2_3@@QAE@QBDI@Z 120248a0 f   XMLException.obj
 0001:000238e0       ??0XMLException@xercesc_2_3@@QAE@ABV01@@Z 120248e0 f   XMLException.obj
 0001:00023980       ??4XMLException@xercesc_2_3@@QAEAAV01@ABV01@@Z 12024980 f   XMLException.obj
 0001:00023a40       ?loadExceptText@XMLException@xercesc_2_3@@IAEXW4Codes@XMLExcepts@2@@Z 12024a40 f   XMLException.obj
 0001:00023cc0       ?loadExceptText@XMLException@xercesc_2_3@@IAEXW4Codes@XMLExcepts@2@QBG111@Z 12024cc0 f   XMLException.obj
 0001:00023dd0       ?loadExceptText@XMLException@xercesc_2_3@@IAEXW4Codes@XMLExcepts@2@QBD111@Z 12024dd0 f   XMLException.obj
 0001:00023ee0       ?reinitMsgMutex@XMLException@xercesc_2_3@@SAXXZ 12024ee0 f   XMLException.obj
 0001:00023f10       ?reinitMsgLoader@XMLException@xercesc_2_3@@SAXXZ 12024f10 f   XMLException.obj
 0001:00023f30       ??0XMLFloat@xercesc_2_3@@QAE@QBGQAVMemoryManager@1@@Z 12024f30 f   XMLFloat.obj
 0001:00023f90       ??_EXMLFloat@xercesc_2_3@@UAEPAXI@Z 12024f90 f i XMLFloat.obj
 0001:00023ff0       ??1XMLFloat@xercesc_2_3@@UAE@XZ 12024ff0 f   XMLFloat.obj
 0001:00024000       ?checkBoundary@XMLFloat@xercesc_2_3@@MAEXQBG@Z 12025000 f   XMLFloat.obj
 0001:00024210       ?xlatThisOne@XMLIBM1140Transcoder@xercesc_2_3@@SAGE@Z 12025210 f   XMLIBM1140Transcoder.obj
 0001:00024230       ??0XMLIBM1140Transcoder@xercesc_2_3@@QAE@QBGI@Z 12025230 f   XMLIBM1140Transcoder.obj
 0001:00024260       ??_EXMLIBM1140Transcoder@xercesc_2_3@@UAEPAXI@Z 12025260 f i XMLIBM1140Transcoder.obj
 0001:000242c0       ??1XMLIBM1140Transcoder@xercesc_2_3@@UAE@XZ 120252c0 f   XMLIBM1140Transcoder.obj
 0001:000242d0       ?setLocale@XMLMsgLoader@xercesc_2_3@@SAXQBD@Z 120252d0 f   XMLMsgLoader.obj
 0001:00024330       ?getLocale@XMLMsgLoader@xercesc_2_3@@SAPBDXZ 12025330 f   XMLMsgLoader.obj
 0001:00024340       ?setNLSHome@XMLMsgLoader@xercesc_2_3@@SAXQBD@Z 12025340 f   XMLMsgLoader.obj
 0001:00024380       ?getNLSHome@XMLMsgLoader@xercesc_2_3@@SAPBDXZ 12025380 f   XMLMsgLoader.obj
 0001:00024390       ?getLanguageName@XMLMsgLoader@xercesc_2_3@@UBEPBGXZ 12025390 f   XMLMsgLoader.obj
 0001:000243a0       ??0XMLNumber@xercesc_2_3@@IAE@XZ 120253a0 f   XMLNumber.obj
 0001:000243b0       ??_EXMLNumber@xercesc_2_3@@UAEPAXI@Z 120253b0 f i XMLNumber.obj
 0001:00024410       ??1XMLNumber@xercesc_2_3@@UAE@XZ 12025410 f   XMLNumber.obj
 0001:00024420       ?binToText@XMLString@xercesc_2_3@@SAXKQADII@Z 12025420 f   XMLString.obj
 0001:00024560       ?binToText@XMLString@xercesc_2_3@@SAXIQADII@Z 12025560 f   XMLString.obj
 0001:00024580       ?binToText@XMLString@xercesc_2_3@@SAXJQADII@Z 12025580 f   XMLString.obj
 0001:00024580       ?binToText@XMLString@xercesc_2_3@@SAXHQADII@Z 12025580 f   XMLString.obj
 0001:000245c0       ?catString@XMLString@xercesc_2_3@@SAXQADQBD@Z 120255c0 f   XMLString.obj
 0001:000245f0       ?compareIString@XMLString@xercesc_2_3@@SAHQBD0@Z 120255f0 f   XMLString.obj
 0001:00024610       ?compareNString@XMLString@xercesc_2_3@@SAHQBD0I@Z 12025610 f   XMLString.obj
 0001:00024630       ?compareNIString@XMLString@xercesc_2_3@@SAHQBD0I@Z 12025630 f   XMLString.obj
 0001:00024650       ?compareString@XMLString@xercesc_2_3@@SAHQBD0@Z 12025650 f   XMLString.obj
 0001:00024690       ?copyString@XMLString@xercesc_2_3@@SAXQADQBD@Z 12025690 f   XMLString.obj
 0001:000246c0       ?cut@XMLString@xercesc_2_3@@SAXQAGI@Z 120256c0 f   XMLString.obj
 0001:000246f0       ?hash@XMLString@xercesc_2_3@@SAIQBDI@Z 120256f0 f   XMLString.obj
 0001:00024760       ?indexOf@XMLString@xercesc_2_3@@SAHQBDD@Z 12025760 f   XMLString.obj
 0001:00024790       ?indexOf@XMLString@xercesc_2_3@@SAHQBDDI@Z 12025790 f   XMLString.obj
 0001:000247f0       ?lastIndexOf@XMLString@xercesc_2_3@@SAHQBDD@Z 120257f0 f   XMLString.obj
 0001:00024820       ?lastIndexOf@XMLString@xercesc_2_3@@SAHQBDDI@Z 12025820 f   XMLString.obj
 0001:00024880       ?replaceTokens@XMLString@xercesc_2_3@@SAIQAGIQBG111@Z 12025880 f   XMLString.obj
 0001:000249e0       ?replicate@XMLString@xercesc_2_3@@SAPADQBD@Z 120259e0 f   XMLString.obj
 0001:00024a20       ?replicate@XMLString@xercesc_2_3@@SAPADQBDQAVMemoryManager@2@@Z 12025a20 f   XMLString.obj
 0001:00024a60       ?startsWith@XMLString@xercesc_2_3@@SA_NQBD0@Z 12025a60 f   XMLString.obj
 0001:00024a90       ?startsWithI@XMLString@xercesc_2_3@@SA_NQBD0@Z 12025a90 f   XMLString.obj
 0001:00024ac0       ?stringLen@XMLString@xercesc_2_3@@SAIQBD@Z 12025ac0 f   XMLString.obj
 0001:00024ae0       ?transcode@XMLString@xercesc_2_3@@SAPADQBG@Z 12025ae0 f   XMLString.obj
 0001:00024b00       ?transcode@XMLString@xercesc_2_3@@SAPADQBGQAVMemoryManager@2@@Z 12025b00 f   XMLString.obj
 0001:00024b20       ?transcode@XMLString@xercesc_2_3@@SA_NQBGQADI@Z 12025b20 f   XMLString.obj
 0001:00024b40       ?transcode@XMLString@xercesc_2_3@@SAPAGQBD@Z 12025b40 f   XMLString.obj
 0001:00024b60       ?transcode@XMLString@xercesc_2_3@@SAPAGQBDQAVMemoryManager@2@@Z 12025b60 f   XMLString.obj
 0001:00024b80       ?transcode@XMLString@xercesc_2_3@@SA_NQBDQAGI@Z 12025b80 f   XMLString.obj
 0001:00024ba0       ?trim@XMLString@xercesc_2_3@@SAXQAD@Z 12025ba0 f   XMLString.obj
 0001:00024c20       ?subString@XMLString@xercesc_2_3@@SAXQADQBDHH@Z 12025c20 f   XMLString.obj
 0001:00024cd0       ?isValidNCName@XMLString@xercesc_2_3@@SA_NQBG@Z 12025cd0 f   XMLString.obj
 0001:00024d10       ?isValidName@XMLString@xercesc_2_3@@SA_NQBG@Z 12025d10 f   XMLString.obj
 0001:00024d50       ?isValidEncName@XMLString@xercesc_2_3@@SA_NQBG@Z 12025d50 f   XMLString.obj
 0001:00024df0       ?isValidQName@XMLString@xercesc_2_3@@SA_NQBG@Z 12025df0 f   XMLString.obj
 0001:00024e30       ?isAlpha@XMLString@xercesc_2_3@@SA_NG@Z 12025e30 f   XMLString.obj
 0001:00024e60       ?isDigit@XMLString@xercesc_2_3@@SA_NG@Z 12025e60 f   XMLString.obj
 0001:00024e80       ?isAlphaNum@XMLString@xercesc_2_3@@SA_NG@Z 12025e80 f   XMLString.obj
 0001:00024ec0       ?isHex@XMLString@xercesc_2_3@@SA_NG@Z 12025ec0 f   XMLString.obj
 0001:00024f00       ?isAllWhiteSpace@XMLString@xercesc_2_3@@SA_NQBG@Z 12025f00 f   XMLString.obj
 0001:00024f40       ?binToText@XMLString@xercesc_2_3@@SAXKQAGII@Z 12025f40 f   XMLString.obj
 0001:000250b0       ?binToText@XMLString@xercesc_2_3@@SAXIQAGII@Z 120260b0 f   XMLString.obj
 0001:000250d0       ?binToText@XMLString@xercesc_2_3@@SAXHQAGII@Z 120260d0 f   XMLString.obj
 0001:000250d0       ?binToText@XMLString@xercesc_2_3@@SAXJQAGII@Z 120260d0 f   XMLString.obj
 0001:00025110       ?catString@XMLString@xercesc_2_3@@SAXQAGQBG@Z 12026110 f   XMLString.obj
 0001:00025170       ?compareIString@XMLString@xercesc_2_3@@SAHQBG0@Z 12026170 f   XMLString.obj
 0001:00025190       ?compareNString@XMLString@xercesc_2_3@@SAHQBG0I@Z 12026190 f   XMLString.obj
 0001:000251d0       ?compareNIString@XMLString@xercesc_2_3@@SAHQBG0I@Z 120261d0 f   XMLString.obj
 0001:000251f0       ?compareString@XMLString@xercesc_2_3@@SAHQBG0@Z 120261f0 f   XMLString.obj
 0001:00025270       ?regionMatches@XMLString@xercesc_2_3@@SA_NQBGH0HI@Z 12026270 f   XMLString.obj
 0001:00025330       ?regionIMatches@XMLString@xercesc_2_3@@SA_NQBGH0HI@Z 12026330 f   XMLString.obj
 0001:000253d0       ?copyString@XMLString@xercesc_2_3@@SAXQAGQBG@Z 120263d0 f   XMLString.obj
 0001:00025410       ?copyNString@XMLString@xercesc_2_3@@SA_NQAGQBGI@Z 12026410 f   XMLString.obj
 0001:00025450       ?hash@XMLString@xercesc_2_3@@SAIQBGI@Z 12026450 f   XMLString.obj
 0001:000254d0       ?findAny@XMLString@xercesc_2_3@@SAPBGQBG0@Z 120264d0 f   XMLString.obj
 0001:000254d0       ?findAny@XMLString@xercesc_2_3@@SAPAGQAGQBG@Z 120264d0 f   XMLString.obj
 0001:00025520       ?patternMatch@XMLString@xercesc_2_3@@SAHQBG0@Z 12026520 f   XMLString.obj
 0001:000255a0       ?hashN@XMLString@xercesc_2_3@@SAIQBGII@Z 120265a0 f   XMLString.obj
 0001:00025610       ?indexOf@XMLString@xercesc_2_3@@SAHQBGG@Z 12026610 f   XMLString.obj
 0001:00025650       ?indexOf@XMLString@xercesc_2_3@@SAHQBGGI@Z 12026650 f   XMLString.obj
 0001:000256d0       ?lastIndexOf@XMLString@xercesc_2_3@@SAHQBGG@Z 120266d0 f   XMLString.obj
 0001:00025720       ?lastIndexOf@XMLString@xercesc_2_3@@SAHQBGGI@Z 12026720 f   XMLString.obj
 0001:000257a0       ?makeUName@XMLString@xercesc_2_3@@SAPAGQBG0@Z 120267a0 f   XMLString.obj
 0001:00025990       ?textToBin@XMLString@xercesc_2_3@@SA_NQBGAAI@Z 12026990 f   XMLString.obj
 0001:00025bb0       ?parseInt@XMLString@xercesc_2_3@@SAHQBG@Z 12026bb0 f   XMLString.obj
 0001:00025df0       ?trim@XMLString@xercesc_2_3@@SAXQAG@Z 12026df0 f   XMLString.obj
 0001:00025ec0       ?upperCase@XMLString@xercesc_2_3@@SAXQAG@Z 12026ec0 f   XMLString.obj
 0001:00025ee0       ?lowerCase@XMLString@xercesc_2_3@@SAXQAG@Z 12026ee0 f   XMLString.obj
 0001:00025f00       ?subString@XMLString@xercesc_2_3@@SAXQAGQBGHH@Z 12026f00 f   XMLString.obj
 0001:00025fd0       ?tokenizeString@XMLString@xercesc_2_3@@SAPAV?$BaseRefVectorOf@G@2@QBG@Z 12026fd0 f   XMLString.obj
 0001:00026260       ?isInList@XMLString@xercesc_2_3@@SA_NQBG0@Z 12027260 f   XMLString.obj
 0001:00026310       ?isWSReplaced@XMLString@xercesc_2_3@@SA_NQBG@Z 12027310 f   XMLString.obj
 0001:00026350       ?replaceWS@XMLString@xercesc_2_3@@SAXQAG@Z 12027350 f   XMLString.obj
 0001:00026400       ?isWSCollapsed@XMLString@xercesc_2_3@@SA_NQBG@Z 12027400 f   XMLString.obj
 0001:00026490       ?collapseWS@XMLString@xercesc_2_3@@SAXQAG@Z 12027490 f   XMLString.obj
 0001:00026620       ?removeWS@XMLString@xercesc_2_3@@SAXQAG@Z 12027620 f   XMLString.obj
 0001:000266e0       ?fixURI@XMLString@xercesc_2_3@@SAXQBGQAG@Z 120276e0 f   XMLString.obj
 0001:00026880       ?release@XMLString@xercesc_2_3@@SAXPAPAE@Z 12027880 f   XMLString.obj
 0001:00026880       ?release@XMLString@xercesc_2_3@@SAXPAPAD@Z 12027880 f   XMLString.obj
 0001:00026880       ?release@XMLString@xercesc_2_3@@SAXPAPAG@Z 12027880 f   XMLString.obj
 0001:000268a0       ?initString@XMLString@xercesc_2_3@@CAXQAVXMLLCPTranscoder@2@QAVMemoryManager@2@@Z 120278a0 f   XMLString.obj
 0001:000268c0       ?termString@XMLString@xercesc_2_3@@CAXXZ 120278c0 f   XMLString.obj
 0001:000268f0       ?cleanUp@XMLStringTokenizer@xercesc_2_3@@AAEXXZ 120278f0 f i XMLStringTokenizer.obj
 0001:00026920       ?isDelimeter@XMLStringTokenizer@xercesc_2_3@@AAE_NG@Z 12027920 f i XMLStringTokenizer.obj
 0001:00026940       ?countTokens@XMLStringTokenizer@xercesc_2_3@@QAEHXZ 12027940 f i XMLStringTokenizer.obj
 0001:00026990       ??0XMLStringTokenizer@xercesc_2_3@@QAE@QBGQAVMemoryManager@1@@Z 12027990 f   XMLStringTokenizer.obj
 0001:00026b60       ??0XMLStringTokenizer@xercesc_2_3@@QAE@QBG0QAVMemoryManager@1@@Z 12027b60 f   XMLStringTokenizer.obj
 0001:00026d20       ??1XMLStringTokenizer@xercesc_2_3@@QAE@XZ 12027d20 f   XMLStringTokenizer.obj
 0001:00026d50       ?nextToken@XMLStringTokenizer@xercesc_2_3@@QAEPAGXZ 12027d50 f   XMLStringTokenizer.obj
 0001:00026e70       ?hasMoreTokens@XMLStringTokenizer@xercesc_2_3@@QAE_NXZ 12027e70 f   XMLStringTokenizer.obj
 0001:00026ed0       ??0XMLUCS4Transcoder@xercesc_2_3@@QAE@QBGI_N@Z 12027ed0 f   XMLUCSTranscoder.obj
 0001:00026f00       ??_EXMLUCS4Transcoder@xercesc_2_3@@UAEPAXI@Z 12027f00 f i XMLUCSTranscoder.obj
 0001:00026f60       ??1XMLUCS4Transcoder@xercesc_2_3@@UAE@XZ 12027f60 f   XMLUCSTranscoder.obj
 0001:00026f70       ?transcodeFrom@XMLUCS4Transcoder@xercesc_2_3@@UAEIQBEIQAGIAAIQAE@Z 12027f70 f   XMLUCSTranscoder.obj
 0001:00027060       ?transcodeTo@XMLUCS4Transcoder@xercesc_2_3@@UAEIQBGIQAEIAAIW4UnRepOpts@XMLTranscoder@2@@Z 12028060 f   XMLUCSTranscoder.obj
 0001:000271a0       ?canTranscodeTo@XMLUCS4Transcoder@xercesc_2_3@@UBE_NI@Z 120281a0 f   XMLUCSTranscoder.obj
 0001:000271a0       ?canTranscodeTo@XMLChTranscoder@xercesc_2_3@@UBE_NI@Z 120281a0 f   XMLUCSTranscoder.obj
 0001:000271a0       ?canTranscodeTo@XMLUTF16Transcoder@xercesc_2_3@@UBE_NI@Z 120281a0 f   XMLUCSTranscoder.obj
 0001:000271b0       ?getUriText@XMLUri@xercesc_2_3@@QBEPBGXZ 120281b0 f i XMLUri.obj
 0001:000271d0       ?isReservedCharacter@XMLUri@xercesc_2_3@@CA_NG@Z 120281d0 f i XMLUri.obj
 0001:000271f0       ?isUnreservedCharacter@XMLUri@xercesc_2_3@@CA_NG@Z 120281f0 f i XMLUri.obj
 0001:00027220       ??0XMLUri@xercesc_2_3@@QAE@QBGQAVMemoryManager@1@@Z 12028220 f   XMLUri.obj
 0001:000272b0       ??_EXMLUri@xercesc_2_3@@UAEPAXI@Z 120282b0 f i XMLUri.obj
 0001:00027310       ??0XMLUri@xercesc_2_3@@QAE@QBV01@QBGQAVMemoryManager@1@@Z 12028310 f   XMLUri.obj
 0001:000273a0       ??0XMLUri@xercesc_2_3@@QAE@ABV01@@Z 120283a0 f   XMLUri.obj
 0001:00027430       ??4XMLUri@xercesc_2_3@@QAEAAV01@ABV01@@Z 12028430 f   XMLUri.obj
 0001:00027490       ??1XMLUri@xercesc_2_3@@UAE@XZ 12028490 f   XMLUri.obj
 0001:000274a0       ?cleanUp@XMLUri@xercesc_2_3@@AAEXXZ 120284a0 f   XMLUri.obj
 0001:00027520       ?initialize@XMLUri@xercesc_2_3@@AAEXABV12@@Z 12028520 f   XMLUri.obj
 0001:00027700       ?initialize@XMLUri@xercesc_2_3@@AAEXQBV12@QBG@Z 12028700 f   XMLUri.obj
 0001:00028440       ?initializeAuthority@XMLUri@xercesc_2_3@@AAEXQBG@Z 12029440 f   XMLUri.obj
 0001:00028690       ?initializeScheme@XMLUri@xercesc_2_3@@AAEXQBG@Z 12029690 f   XMLUri.obj
 0001:000287c0       ?initializePath@XMLUri@xercesc_2_3@@AAEXQBG@Z 120297c0 f   XMLUri.obj
 0001:00028cd0       ?setScheme@XMLUri@xercesc_2_3@@QAEXQBG@Z 12029cd0 f   XMLUri.obj
 0001:00028e00       ?setUserInfo@XMLUri@xercesc_2_3@@QAEXQBG@Z 12029e00 f   XMLUri.obj
 0001:00028f10       ?setHost@XMLUri@xercesc_2_3@@QAEXQBG@Z 12029f10 f   XMLUri.obj
 0001:00029000       ?setPort@XMLUri@xercesc_2_3@@QAEXH@Z 1202a000 f   XMLUri.obj
 0001:000290c0       ?setPath@XMLUri@xercesc_2_3@@QAEXQBG@Z 1202a0c0 f   XMLUri.obj
 0001:00029110       ?setFragment@XMLUri@xercesc_2_3@@QAEXQBG@Z 1202a110 f   XMLUri.obj
 0001:000292c0       ?setQueryString@XMLUri@xercesc_2_3@@QAEXQBG@Z 1202a2c0 f   XMLUri.obj
 0001:00029470       ?isConformantSchemeName@XMLUri@xercesc_2_3@@CA_NQBG@Z 1202a470 f   XMLUri.obj
 0001:000294e0       ?isConformantUserInfo@XMLUri@xercesc_2_3@@CAXQBG@Z 1202a4e0 f   XMLUri.obj
 0001:00029610       ?isURIString@XMLUri@xercesc_2_3@@SA_NQBG@Z 1202a610 f   XMLUri.obj
 0001:000296a0       ?isWellFormedAddress@XMLUri@xercesc_2_3@@CA_NQBG@Z 1202a6a0 f   XMLUri.obj
 0001:000299f0       ?isGenericURI@XMLUri@xercesc_2_3@@AAE_NXZ 1202a9f0 f   XMLUri.obj
 0001:00029a00       ?buildFullText@XMLUri@xercesc_2_3@@AAEXXZ 1202aa00 f   XMLUri.obj
 0001:00029d60       ?lookupByName@XMLURL@xercesc_2_3@@SA?AW4Protocols@12@QBG@Z 1202ad60 f   XMLURL.obj
 0001:00029db0       ??0XMLURL@xercesc_2_3@@QAE@QAVMemoryManager@1@@Z 1202adb0 f   XMLURL.obj
 0001:00029df0       ??_EXMLURL@xercesc_2_3@@UAEPAXI@Z 1202adf0 f i XMLURL.obj
 0001:00029e50       ??0XMLURL@xercesc_2_3@@QAE@QBG0QAVMemoryManager@1@@Z 1202ae50 f   XMLURL.obj
 0001:00029f80       ??0XMLURL@xercesc_2_3@@QAE@QBGQBDQAVMemoryManager@1@@Z 1202af80 f   XMLURL.obj
 0001:0002a0f0       ??0XMLURL@xercesc_2_3@@QAE@ABV01@QBG@Z 1202b0f0 f   XMLURL.obj
 0001:0002a1a0       ??0XMLURL@xercesc_2_3@@QAE@ABV01@QBD@Z 1202b1a0 f   XMLURL.obj
 0001:0002a2a0       ??0XMLURL@xercesc_2_3@@QAE@QBGQAVMemoryManager@1@@Z 1202b2a0 f   XMLURL.obj
 0001:0002a330       ??0XMLURL@xercesc_2_3@@QAE@QBDQAVMemoryManager@1@@Z 1202b330 f   XMLURL.obj
 0001:0002a400       ??0XMLURL@xercesc_2_3@@QAE@ABV01@@Z 1202b400 f   XMLURL.obj
 0001:0002a690       ??1XMLURL@xercesc_2_3@@UAE@XZ 1202b690 f   XMLURL.obj
 0001:0002a6a0       ??4XMLURL@xercesc_2_3@@QAEAAV01@ABV01@@Z 1202b6a0 f   XMLURL.obj
 0001:0002a8d0       ??8XMLURL@xercesc_2_3@@QBE_NABV01@@Z 1202b8d0 f   XMLURL.obj
 0001:0002a950       ?getPortNum@XMLURL@xercesc_2_3@@QBEIXZ 1202b950 f   XMLURL.obj
 0001:0002a970       ?getProtocolName@XMLURL@xercesc_2_3@@QBEPBGXZ 1202b970 f   XMLURL.obj
 0001:0002a9b0       ?setURL@XMLURL@xercesc_2_3@@QAEXQBG@Z 1202b9b0 f   XMLURL.obj
 0001:0002a9d0       ?setURL@XMLURL@xercesc_2_3@@QAEXQBG0@Z 1202b9d0 f   XMLURL.obj
 0001:0002aad0       ?setURL@XMLURL@xercesc_2_3@@QAEXABV12@QBG@Z 1202bad0 f   XMLURL.obj
 0001:0002ab10       ?isRelative@XMLURL@xercesc_2_3@@QBE_NXZ 1202bb10 f   XMLURL.obj
 0001:0002ab30       ?hasInvalidChar@XMLURL@xercesc_2_3@@QBE_NXZ 1202bb30 f   XMLURL.obj
 0001:0002ab40       ?makeNewStream@XMLURL@xercesc_2_3@@QBEPAVBinInputStream@2@XZ 1202bb40 f   XMLURL.obj
 0001:0002af00       ?makeRelativeTo@XMLURL@xercesc_2_3@@QAEXQBG@Z 1202bf00 f   XMLURL.obj
 0001:0002af90       ?makeRelativeTo@XMLURL@xercesc_2_3@@QAEXABV12@@Z 1202bf90 f   XMLURL.obj
 0001:0002afc0       ?buildFullText@XMLURL@xercesc_2_3@@AAEXXZ 1202bfc0 f   XMLURL.obj
 0001:0002b370       ?cleanup@XMLURL@xercesc_2_3@@AAEXXZ 1202c370 f   XMLURL.obj
 0001:0002b3f0       ?conglomerateWithBase@XMLURL@xercesc_2_3@@AAE_NABV12@_N@Z 1202c3f0 f   XMLURL.obj
 0001:0002b820       ?parse@XMLURL@xercesc_2_3@@AAEXQBG@Z 1202c820 f   XMLURL.obj
 0001:0002c010       ??0XMLUTF16Transcoder@xercesc_2_3@@QAE@QBGI_N@Z 1202d010 f   XMLUTF16Transcoder.obj
 0001:0002c040       ??_EXMLUTF16Transcoder@xercesc_2_3@@UAEPAXI@Z 1202d040 f i XMLUTF16Transcoder.obj
 0001:0002c0a0       ??1XMLUTF16Transcoder@xercesc_2_3@@UAE@XZ 1202d0a0 f   XMLUTF16Transcoder.obj
 0001:0002c0b0       ?transcodeFrom@XMLUTF16Transcoder@xercesc_2_3@@UAEIQBEIQAGIAAIQAE@Z 1202d0b0 f   XMLUTF16Transcoder.obj
 0001:0002c130       ?transcodeTo@XMLUTF16Transcoder@xercesc_2_3@@UAEIQBGIQAEIAAIW4UnRepOpts@XMLTranscoder@2@@Z 1202d130 f   XMLUTF16Transcoder.obj
 0001:0002c1b0       ??0XMLUTF8Transcoder@xercesc_2_3@@QAE@QBGI@Z 1202d1b0 f   XMLUTF8Transcoder.obj
 0001:0002c1e0       ??_EXMLUTF8Transcoder@xercesc_2_3@@UAEPAXI@Z 1202d1e0 f i XMLUTF8Transcoder.obj
 0001:0002c240       ??1XMLUTF8Transcoder@xercesc_2_3@@UAE@XZ 1202d240 f   XMLUTF8Transcoder.obj
 0001:0002c250       ?transcodeFrom@XMLUTF8Transcoder@xercesc_2_3@@UAEIQBEIQAGIAAIQAE@Z 1202d250 f   XMLUTF8Transcoder.obj
 0001:0002c530       ?transcodeTo@XMLUTF8Transcoder@xercesc_2_3@@UAEIQBGIQAEIAAIW4UnRepOpts@XMLTranscoder@2@@Z 1202d530 f   XMLUTF8Transcoder.obj
 0001:0002c720       ?canTranscodeTo@XMLUTF8Transcoder@xercesc_2_3@@UBE_NI@Z 1202d720 f   XMLUTF8Transcoder.obj
 0001:0002c740       ??0XMLWin1252Transcoder@xercesc_2_3@@QAE@QBGI@Z 1202d740 f   XMLWin1252Transcoder.obj
 0001:0002c770       ??_EXMLWin1252Transcoder@xercesc_2_3@@UAEPAXI@Z 1202d770 f i XMLWin1252Transcoder.obj
 0001:0002c7d0       ??1XMLWin1252Transcoder@xercesc_2_3@@UAE@XZ 1202d7d0 f   XMLWin1252Transcoder.obj
 0001:0002c7e0       ??1XMLFormatTarget@xercesc_2_3@@UAE@XZ 1202d7e0 f i LocalFileFormatTarget.obj
 0001:0002c7f0       ??0XMLFormatTarget@xercesc_2_3@@IAE@XZ 1202d7f0 f i LocalFileFormatTarget.obj
 0001:0002c800       ??0XMLFormatTarget@xercesc_2_3@@IAE@ABV01@@Z 1202d800 f i LocalFileFormatTarget.obj
 0001:0002c810       ??_EXMLFormatTarget@xercesc_2_3@@UAEPAXI@Z 1202d810 f i LocalFileFormatTarget.obj
 0001:0002c870       ??6XMLFormatter@xercesc_2_3@@QAEAAV01@W4UnRepFlags@01@@Z 1202d870 f i LocalFileFormatTarget.obj
 0001:0002c880       ??0LocalFileFormatTarget@xercesc_2_3@@QAE@QBGQAVMemoryManager@1@@Z 1202d880 f   LocalFileFormatTarget.obj
 0001:0002c950       ??_ELocalFileFormatTarget@xercesc_2_3@@UAEPAXI@Z 1202d950 f i LocalFileFormatTarget.obj
 0001:0002c9b0       ??0LocalFileFormatTarget@xercesc_2_3@@QAE@QBDQAVMemoryManager@1@@Z 1202d9b0 f   LocalFileFormatTarget.obj
 0001:0002ca80       ??1LocalFileFormatTarget@xercesc_2_3@@UAE@XZ 1202da80 f   LocalFileFormatTarget.obj
 0001:0002cb20       ?writeChars@LocalFileFormatTarget@xercesc_2_3@@UAEXQBEIQAVXMLFormatter@2@@Z 1202db20 f   LocalFileFormatTarget.obj
 0001:0002cc00       ?flush@LocalFileFormatTarget@xercesc_2_3@@UAEXXZ 1202dc00 f   LocalFileFormatTarget.obj
 0001:0002cc00       ?flushBuffer@LocalFileFormatTarget@xercesc_2_3@@AAEXXZ 1202dc00 f   LocalFileFormatTarget.obj
 0001:0002cc50       ?insureCapacity@LocalFileFormatTarget@xercesc_2_3@@AAEXI@Z 1202dc50 f   LocalFileFormatTarget.obj
 0001:0002ccf0       ??_FInputSource@xercesc_2_3@@QAEXXZ 1202dcf0 f i LocalFileInputSource.obj
 0001:0002cd00       ??0LocalFileInputSource@xercesc_2_3@@QAE@QBG0QAVMemoryManager@1@@Z 1202dd00 f   LocalFileInputSource.obj
 0001:0002cdf0       ??_ELocalFileInputSource@xercesc_2_3@@UAEPAXI@Z 1202ddf0 f i LocalFileInputSource.obj
 0001:0002ce50       ??0LocalFileInputSource@xercesc_2_3@@QAE@QBGQAVMemoryManager@1@@Z 1202de50 f   LocalFileInputSource.obj
 0001:0002cfc0       ??1LocalFileInputSource@xercesc_2_3@@UAE@XZ 1202dfc0 f   LocalFileInputSource.obj
 0001:0002cfd0       ?makeStream@LocalFileInputSource@xercesc_2_3@@UBEPAVBinInputStream@2@XZ 1202dfd0 f   LocalFileInputSource.obj
 0001:0002d060       ??_FMemBufFormatTarget@xercesc_2_3@@QAEXXZ 1202e060 f i MemBufFormatTarget.obj
 0001:0002d080       ??0MemBufFormatTarget@xercesc_2_3@@QAE@HQAVMemoryManager@1@@Z 1202e080 f   MemBufFormatTarget.obj
 0001:0002d0f0       ??_EMemBufFormatTarget@xercesc_2_3@@UAEPAXI@Z 1202e0f0 f i MemBufFormatTarget.obj
 0001:0002d150       ??1MemBufFormatTarget@xercesc_2_3@@UAE@XZ 1202e150 f   MemBufFormatTarget.obj
 0001:0002d1a0       ?writeChars@MemBufFormatTarget@xercesc_2_3@@UAEXQBEIQAVXMLFormatter@2@@Z 1202e1a0 f   MemBufFormatTarget.obj
 0001:0002d230       ?getRawBuffer@MemBufFormatTarget@xercesc_2_3@@QBEPBEXZ 1202e230 f   MemBufFormatTarget.obj
 0001:0002d260       ?reset@MemBufFormatTarget@xercesc_2_3@@QAEXXZ 1202e260 f   MemBufFormatTarget.obj
 0001:0002d290       ?insureCapacity@MemBufFormatTarget@xercesc_2_3@@AAEXI@Z 1202e290 f   MemBufFormatTarget.obj
 0001:0002d2f0       ?setCopyBufToStream@MemBufInputSource@xercesc_2_3@@QAEX_N@Z 1202e2f0 f i MemBufInputSource.obj
 0001:0002d300       ??0MemBufInputSource@xercesc_2_3@@QAE@QBEIQBG_NQAVMemoryManager@1@@Z 1202e300 f   MemBufInputSource.obj
 0001:0002d340       ??_EMemBufInputSource@xercesc_2_3@@UAEPAXI@Z 1202e340 f i MemBufInputSource.obj
 0001:0002d3a0       ??0MemBufInputSource@xercesc_2_3@@QAE@QBEIQBD_NQAVMemoryManager@1@@Z 1202e3a0 f   MemBufInputSource.obj
 0001:0002d3e0       ??1MemBufInputSource@xercesc_2_3@@UAE@XZ 1202e3e0 f   MemBufInputSource.obj
 0001:0002d440       ?makeStream@MemBufInputSource@xercesc_2_3@@UBEPAVBinInputStream@2@XZ 1202e440 f   MemBufInputSource.obj
 0001:0002d4c0       ??_FStdInInputSource@xercesc_2_3@@QAEXXZ 1202e4c0 f i StdInInputSource.obj
 0001:0002d4d0       ??0StdInInputSource@xercesc_2_3@@QAE@QAVMemoryManager@1@@Z 1202e4d0 f i StdInInputSource.obj
 0001:0002d4f0       ??_EStdInInputSource@xercesc_2_3@@UAEPAXI@Z 1202e4f0 f i StdInInputSource.obj
 0001:0002d550       ??1StdInInputSource@xercesc_2_3@@UAE@XZ 1202e550 f i StdInInputSource.obj
 0001:0002d560       ?makeStream@StdInInputSource@xercesc_2_3@@UBEPAVBinInputStream@2@XZ 1202e560 f   StdInInputSource.obj
 0001:0002d5e0       ??0StdOutFormatTarget@xercesc_2_3@@QAE@XZ 1202e5e0 f   StdOutFormatTarget.obj
 0001:0002d5f0       ??_EStdOutFormatTarget@xercesc_2_3@@UAEPAXI@Z 1202e5f0 f i StdOutFormatTarget.obj
 0001:0002d650       ??1StdOutFormatTarget@xercesc_2_3@@UAE@XZ 1202e650 f   StdOutFormatTarget.obj
 0001:0002d660       ?flush@StdOutFormatTarget@xercesc_2_3@@UAEXXZ 1202e660 f   StdOutFormatTarget.obj
 0001:0002d670       ?writeChars@StdOutFormatTarget@xercesc_2_3@@UAEXQBEIQAVXMLFormatter@2@@Z 1202e670 f   StdOutFormatTarget.obj
 0001:0002d6a0       ?urlSrc@URLInputSource@xercesc_2_3@@QBEABVXMLURL@2@XZ 1202e6a0 f i URLInputSource.obj
 0001:0002d6b0       ??0URLInputSource@xercesc_2_3@@QAE@ABVXMLURL@1@QAVMemoryManager@1@@Z 1202e6b0 f   URLInputSource.obj
 0001:0002d730       ??_EURLInputSource@xercesc_2_3@@UAEPAXI@Z 1202e730 f i URLInputSource.obj
 0001:0002d790       ??0URLInputSource@xercesc_2_3@@QAE@QBG0QAVMemoryManager@1@@Z 1202e790 f   URLInputSource.obj
 0001:0002d820       ??0URLInputSource@xercesc_2_3@@QAE@QBG00QAVMemoryManager@1@@Z 1202e820 f   URLInputSource.obj
 0001:0002d8b0       ??0URLInputSource@xercesc_2_3@@QAE@QBGQBDQAVMemoryManager@1@@Z 1202e8b0 f   URLInputSource.obj
 0001:0002d940       ??0URLInputSource@xercesc_2_3@@QAE@QBGQBD1QAVMemoryManager@1@@Z 1202e940 f   URLInputSource.obj
 0001:0002d9d0       ??1URLInputSource@xercesc_2_3@@UAE@XZ 1202e9d0 f   URLInputSource.obj
 0001:0002da30       ?makeStream@URLInputSource@xercesc_2_3@@UBEPAVBinInputStream@2@XZ 1202ea30 f   URLInputSource.obj
 0001:0002da40       ??0DOMInputSource@xercesc_2_3@@IAE@XZ 1202ea40 f i Wrapper4DOMInputSource.obj
 0001:0002da50       ??1DOMInputSource@xercesc_2_3@@UAE@XZ 1202ea50 f i Wrapper4DOMInputSource.obj
 0001:0002da60       ??_EDOMInputSource@xercesc_2_3@@UAEPAXI@Z 1202ea60 f i Wrapper4DOMInputSource.obj
 0001:0002dac0       ??0Wrapper4DOMInputSource@xercesc_2_3@@QAE@QAVDOMInputSource@1@_NQAVMemoryManager@1@@Z 1202eac0 f   Wrapper4DOMInputSource.obj
 0001:0002db60       ??_EWrapper4DOMInputSource@xercesc_2_3@@UAEPAXI@Z 1202eb60 f i Wrapper4DOMInputSource.obj
 0001:0002dbc0       ??1Wrapper4DOMInputSource@xercesc_2_3@@UAE@XZ 1202ebc0 f   Wrapper4DOMInputSource.obj
 0001:0002dc20       ?getIssueFatalErrorIfNotFound@Wrapper4DOMInputSource@xercesc_2_3@@UBE?B_NXZ 1202ec20 f   Wrapper4DOMInputSource.obj
 0001:0002dc30       ?getEncoding@Wrapper4DOMInputSource@xercesc_2_3@@UBEPBGXZ 1202ec30 f   Wrapper4DOMInputSource.obj
 0001:0002dc40       ?getSystemId@Wrapper4DOMInputSource@xercesc_2_3@@UBEPBGXZ 1202ec40 f   Wrapper4DOMInputSource.obj
 0001:0002dc50       ?getPublicId@Wrapper4DOMInputSource@xercesc_2_3@@UBEPBGXZ 1202ec50 f   Wrapper4DOMInputSource.obj
 0001:0002dc60       ?setIssueFatalErrorIfNotFound@Wrapper4DOMInputSource@xercesc_2_3@@UAEX_N@Z 1202ec60 f   Wrapper4DOMInputSource.obj
 0001:0002dc70       ?setEncoding@Wrapper4DOMInputSource@xercesc_2_3@@UAEXQBG@Z 1202ec70 f   Wrapper4DOMInputSource.obj
 0001:0002dc80       ?setPublicId@Wrapper4DOMInputSource@xercesc_2_3@@UAEXQBG@Z 1202ec80 f   Wrapper4DOMInputSource.obj
 0001:0002dc90       ?setSystemId@Wrapper4DOMInputSource@xercesc_2_3@@UAEXQBG@Z 1202ec90 f   Wrapper4DOMInputSource.obj
 0001:0002dca0       ?makeStream@Wrapper4DOMInputSource@xercesc_2_3@@UBEPAVBinInputStream@2@XZ 1202eca0 f   Wrapper4DOMInputSource.obj
 0001:0002dcb0       ??0Wrapper4InputSource@xercesc_2_3@@QAE@QAVInputSource@1@_N@Z 1202ecb0 f   Wrapper4InputSource.obj
 0001:0002dd40       ??_EWrapper4InputSource@xercesc_2_3@@UAEPAXI@Z 1202ed40 f i Wrapper4InputSource.obj
 0001:0002dda0       ??1Wrapper4InputSource@xercesc_2_3@@UAE@XZ 1202eda0 f   Wrapper4InputSource.obj
 0001:0002de00       ?getIssueFatalErrorIfNotFound@Wrapper4InputSource@xercesc_2_3@@UBE?B_NXZ 1202ee00 f   Wrapper4InputSource.obj
 0001:0002de10       ?getEncoding@Wrapper4InputSource@xercesc_2_3@@UBEPBGXZ 1202ee10 f   Wrapper4InputSource.obj
 0001:0002de20       ?getSystemId@Wrapper4InputSource@xercesc_2_3@@UBEPBGXZ 1202ee20 f   Wrapper4InputSource.obj
 0001:0002de30       ?getPublicId@Wrapper4InputSource@xercesc_2_3@@UBEPBGXZ 1202ee30 f   Wrapper4InputSource.obj
 0001:0002de40       ?setIssueFatalErrorIfNotFound@Wrapper4InputSource@xercesc_2_3@@UAEX_N@Z 1202ee40 f   Wrapper4InputSource.obj
 0001:0002de50       ?setEncoding@Wrapper4InputSource@xercesc_2_3@@UAEXQBG@Z 1202ee50 f   Wrapper4InputSource.obj
 0001:0002de60       ?setPublicId@Wrapper4InputSource@xercesc_2_3@@UAEXQBG@Z 1202ee60 f   Wrapper4InputSource.obj
 0001:0002de70       ?setSystemId@Wrapper4InputSource@xercesc_2_3@@UAEXQBG@Z 1202ee70 f   Wrapper4InputSource.obj
 0001:0002de80       ?makeStream@Wrapper4InputSource@xercesc_2_3@@UBEPAVBinInputStream@2@XZ 1202ee80 f   Wrapper4InputSource.obj
 0001:0002de90       ??_FXMLAttDef@xercesc_2_3@@QAEXXZ 1202ee90 f i XMLAttDef.obj
 0001:0002ded0       ?setEnumeration@XMLAttDef@xercesc_2_3@@QAEXQBG@Z 1202eed0 f i XMLAttDef.obj
 0001:0002df40       ?setValue@XMLAttDef@xercesc_2_3@@QAEXQBG@Z 1202ef40 f i XMLAttDef.obj
 0001:0002dfb0       ?getAttTypeString@XMLAttDef@xercesc_2_3@@SAPBGW4AttTypes@12@@Z 1202efb0 f   XMLAttDef.obj
 0001:0002dff0       ?getDefAttTypeString@XMLAttDef@xercesc_2_3@@SAPBGW4DefAttTypes@12@@Z 1202eff0 f   XMLAttDef.obj
 0001:0002e030       ??1XMLAttDef@xercesc_2_3@@UAE@XZ 1202f030 f   XMLAttDef.obj
 0001:0002e060       ??_EXMLAttDef@xercesc_2_3@@UAEPAXI@Z 1202f060 f i XMLAttDef.obj
 0001:0002e0e0       ??0XMLAttDef@xercesc_2_3@@IAE@W4AttTypes@01@W4DefAttTypes@01@QAVMemoryManager@1@@Z 1202f0e0 f   XMLAttDef.obj
 0001:0002e120       ??0XMLAttDef@xercesc_2_3@@IAE@QBGW4AttTypes@01@W4DefAttTypes@01@0QAVMemoryManager@1@@Z 1202f120 f   XMLAttDef.obj
 0001:0002e250       ?cleanUp@XMLAttDef@xercesc_2_3@@AAEXXZ 1202f250 f   XMLAttDef.obj
 0001:0002e280       ??_FXMLAttr@xercesc_2_3@@QAEXXZ 1202f280 f i XMLAttr.obj
 0001:0002e290       ??1XMLAttr@xercesc_2_3@@QAE@XZ 1202f290 f i XMLAttr.obj
 0001:0002e2c0       ?getName@XMLAttr@xercesc_2_3@@QBEPBGXZ 1202f2c0 f i XMLAttr.obj
 0001:0002e2d0       ?getPrefix@XMLAttr@xercesc_2_3@@QBEPBGXZ 1202f2d0 f i XMLAttr.obj
 0001:0002e2e0       ?getURIId@XMLAttr@xercesc_2_3@@QBEIXZ 1202f2e0 f i XMLAttr.obj
 0001:0002e2f0       ?set@XMLAttr@xercesc_2_3@@QAEXIQBG00W4AttTypes@XMLAttDef@2@@Z 1202f2f0 f i XMLAttr.obj
 0001:0002e390       ?set@XMLAttr@xercesc_2_3@@QAEXIQBG0W4AttTypes@XMLAttDef@2@@Z 1202f390 f i XMLAttr.obj
 0001:0002e430       ??0XMLAttr@xercesc_2_3@@QAE@QAVMemoryManager@1@@Z 1202f430 f   XMLAttr.obj
 0001:0002e4b0       ??0XMLAttr@xercesc_2_3@@QAE@IQBG00W4AttTypes@XMLAttDef@1@_NQAVMemoryManager@1@@Z 1202f4b0 f   XMLAttr.obj
 0001:0002e5e0       ??0XMLAttr@xercesc_2_3@@QAE@IQBG0W4AttTypes@XMLAttDef@1@_NQAVMemoryManager@1@@Z 1202f5e0 f   XMLAttr.obj
 0001:0002e700       ?getQName@XMLAttr@xercesc_2_3@@QBEPBGXZ 1202f700 f   XMLAttr.obj
 0001:0002e710       ?setName@XMLAttr@xercesc_2_3@@QAEXIQBG0@Z 1202f710 f   XMLAttr.obj
 0001:0002e730       ?setURIId@XMLAttr@xercesc_2_3@@QAEXI@Z 1202f730 f   XMLAttr.obj
 0001:0002e740       ?setValue@XMLAttr@xercesc_2_3@@QAEXQBG@Z 1202f740 f   XMLAttr.obj
 0001:0002e7c0       ?cleanUp@XMLAttr@xercesc_2_3@@AAEXXZ 1202f7c0 f   XMLAttr.obj
 0001:0002e7f0       ?append@XMLBuffer@xercesc_2_3@@QAEXQBGI@Z 1202f7f0 f   XMLBuffer.obj
 0001:0002e8c0       ?set@XMLBuffer@xercesc_2_3@@QAEXQBGI@Z 1202f8c0 f   XMLBuffer.obj
 0001:0002e970       ?expand@XMLBuffer@xercesc_2_3@@AAEXXZ 1202f970 f   XMLBuffer.obj
 0001:0002e9f0       ?insureCapacity@XMLBuffer@xercesc_2_3@@AAEXI@Z 1202f9f0 f   XMLBuffer.obj
 0001:0002ea50       ??_FXMLBufferMgr@xercesc_2_3@@QAEXXZ 1202fa50 f i XMLBufferMgr.obj
 0001:0002eaa0       ??0XMLBufferMgr@xercesc_2_3@@QAE@QAVMemoryManager@1@@Z 1202faa0 f   XMLBufferMgr.obj
 0001:0002eaf0       ??1XMLBufferMgr@xercesc_2_3@@QAE@XZ 1202faf0 f   XMLBufferMgr.obj
 0001:0002eb40       ?bidOnBuffer@XMLBufferMgr@xercesc_2_3@@QAEAAVXMLBuffer@2@XZ 1202fb40 f   XMLBufferMgr.obj
 0001:0002ec70       ?releaseBuffer@XMLBufferMgr@xercesc_2_3@@QAEXAAVXMLBuffer@2@@Z 1202fc70 f   XMLBufferMgr.obj
 0001:0002ecc0       ??1XMLContentModel@xercesc_2_3@@UAE@XZ 1202fcc0 f i XMLContentModel.obj
 0001:0002ecd0       ??0XMLContentModel@xercesc_2_3@@IAE@XZ 1202fcd0 f i XMLContentModel.obj
 0001:0002ece0       ??_EXMLContentModel@xercesc_2_3@@UAEPAXI@Z 1202fce0 f i XMLContentModel.obj
 0001:0002ed40       ??1XMLAttDefList@xercesc_2_3@@UAE@XZ 1202fd40 f i XMLElementDecl.obj
 0001:0002ed50       ??_EXMLAttDefList@xercesc_2_3@@UAEPAXI@Z 1202fd50 f i XMLElementDecl.obj
 0001:0002edb0       ??0XMLAttDefList@xercesc_2_3@@IAE@XZ 1202fdb0 f i XMLElementDecl.obj
 0001:0002edc0       ??0XMLAttDefList@xercesc_2_3@@IAE@ABV01@@Z 1202fdc0 f i XMLElementDecl.obj
 0001:0002edd0       ??_FXMLElementDecl@xercesc_2_3@@QAEXXZ 1202fdd0 f i XMLElementDecl.obj
 0001:0002ee00       ?getBaseName@XMLElementDecl@xercesc_2_3@@QAEPAGXZ 1202fe00 f i XMLElementDecl.obj
 0001:0002ee00       ?getBaseName@XMLElementDecl@xercesc_2_3@@QBEPBGXZ 1202fe00 f i XMLElementDecl.obj
 0001:0002ee10       ?getURI@XMLElementDecl@xercesc_2_3@@QBEIXZ 1202fe10 f i XMLElementDecl.obj
 0001:0002ee20       ?getFullName@XMLElementDecl@xercesc_2_3@@QBEPBGXZ 1202fe20 f i XMLElementDecl.obj
 0001:0002ee20       ?getKey@DTDElementDecl@xercesc_2_3@@QBEPBGXZ 1202fe20 f i XMLElementDecl.obj
 0001:0002ee30       ?isDeclared@XMLElementDecl@xercesc_2_3@@QBE_NXZ 1202fe30 f i XMLElementDecl.obj
 0001:0002ee40       ??1XMLElementDecl@xercesc_2_3@@UAE@XZ 1202fe40 f   XMLElementDecl.obj
 0001:0002ee60       ??_EXMLElementDecl@xercesc_2_3@@UAEPAXI@Z 1202fe60 f i XMLElementDecl.obj
 0001:0002eed0       ?setElementName@XMLElementDecl@xercesc_2_3@@QAEXQBG0H@Z 1202fed0 f   XMLElementDecl.obj
 0001:0002ef70       ?setElementName@XMLElementDecl@xercesc_2_3@@QAEXQBGH@Z 1202ff70 f   XMLElementDecl.obj
 0001:0002f010       ?setElementName@XMLElementDecl@xercesc_2_3@@QAEXQBVQName@2@@Z 12030010 f   XMLElementDecl.obj
 0001:0002f0a0       ??0XMLElementDecl@xercesc_2_3@@IAE@QAVMemoryManager@1@@Z 120300a0 f   XMLElementDecl.obj
 0001:0002f0d0       ??_FXMLEntityDecl@xercesc_2_3@@QAEXXZ 120300d0 f i XMLEntityDecl.obj
 0001:0002f100       ?isExternal@XMLEntityDecl@xercesc_2_3@@QBE_NXZ 12030100 f i XMLEntityDecl.obj
 0001:0002f120       ?isUnparsed@XMLEntityDecl@xercesc_2_3@@QBE_NXZ 12030120 f i XMLEntityDecl.obj
 0001:0002f130       ?setNotationName@XMLEntityDecl@xercesc_2_3@@QAEXQBG@Z 12030130 f i XMLEntityDecl.obj
 0001:0002f1a0       ?setPublicId@XMLEntityDecl@xercesc_2_3@@QAEXQBG@Z 120301a0 f i XMLEntityDecl.obj
 0001:0002f210       ?setSystemId@XMLEntityDecl@xercesc_2_3@@QAEXQBG@Z 12030210 f i XMLEntityDecl.obj
 0001:0002f280       ?setBaseURI@XMLEntityDecl@xercesc_2_3@@QAEXQBG@Z 12030280 f i XMLEntityDecl.obj
 0001:0002f2f0       ?setValue@XMLEntityDecl@xercesc_2_3@@QAEXQBG@Z 120302f0 f i XMLEntityDecl.obj
 0001:0002f390       ??0XMLEntityDecl@xercesc_2_3@@QAE@QAVMemoryManager@1@@Z 12030390 f   XMLEntityDecl.obj
 0001:0002f3c0       ??_EXMLEntityDecl@xercesc_2_3@@UAEPAXI@Z 120303c0 f i XMLEntityDecl.obj
 0001:0002f460       ??0XMLEntityDecl@xercesc_2_3@@QAE@QBGQAVMemoryManager@1@@Z 12030460 f   XMLEntityDecl.obj
 0001:0002f4f0       ??0XMLEntityDecl@xercesc_2_3@@QAE@QBG0QAVMemoryManager@1@@Z 120304f0 f   XMLEntityDecl.obj
 0001:0002f660       ??0XMLEntityDecl@xercesc_2_3@@QAE@QBGGQAVMemoryManager@1@@Z 12030660 f   XMLEntityDecl.obj
 0001:0002f7c0       ??1XMLEntityDecl@xercesc_2_3@@UAE@XZ 120307c0 f   XMLEntityDecl.obj
 0001:0002f820       ?setName@XMLEntityDecl@xercesc_2_3@@QAEXQBG@Z 12030820 f   XMLEntityDecl.obj
 0001:0002f890       ?cleanUp@XMLEntityDecl@xercesc_2_3@@AAEXXZ 12030890 f   XMLEntityDecl.obj
 0001:0002f8e0       ?inEscapeList@XMLFormatter@xercesc_2_3@@AAE_NW4EscapeFlags@12@G@Z 120308e0 f   XMLFormatter.obj
 0001:0002f940       ??0XMLFormatter@xercesc_2_3@@QAE@QBD0QAVXMLFormatTarget@1@W4EscapeFlags@01@W4UnRepFlags@01@QAVMemoryManager@1@@Z 12030940 f   XMLFormatter.obj
 0001:0002fb00       ??0XMLFormatter@xercesc_2_3@@QAE@QBG0QAVXMLFormatTarget@1@W4EscapeFlags@01@W4UnRepFlags@01@QAVMemoryManager@1@@Z 12030b00 f   XMLFormatter.obj
 0001:0002fc80       ??1XMLFormatter@xercesc_2_3@@QAE@XZ 12030c80 f   XMLFormatter.obj
 0001:0002fd00       ?formatBuf@XMLFormatter@xercesc_2_3@@QAEXQBGIW4EscapeFlags@12@W4UnRepFlags@12@@Z 12030d00 f   XMLFormatter.obj
 0001:0002ff70       ?handleUnEscapedChars@XMLFormatter@xercesc_2_3@@AAEIPBGIW4UnRepFlags@12@@Z 12030f70 f   XMLFormatter.obj
 0001:00030000       ??6XMLFormatter@xercesc_2_3@@QAEAAV01@QBG@Z 12031000 f   XMLFormatter.obj
 0001:00030050       ??6XMLFormatter@xercesc_2_3@@QAEAAV01@G@Z 12031050 f   XMLFormatter.obj
 0001:00030090       ?writeBOM@XMLFormatter@xercesc_2_3@@QAEXQBEI@Z 12031090 f   XMLFormatter.obj
 0001:000300b0       ?writeCharRef@XMLFormatter@xercesc_2_3@@AAEXABG@Z 120310b0 f   XMLFormatter.obj
 0001:00030140       ?getCharRef@XMLFormatter@xercesc_2_3@@AAEPBEAAIAAPAEPBG@Z 12031140 f   XMLFormatter.obj
 0001:000301f0       ?specialFormat@XMLFormatter@xercesc_2_3@@AAEXQBGIW4EscapeFlags@12@@Z 120311f0 f   XMLFormatter.obj
 0001:00030300       ??_FXMLNotationDecl@xercesc_2_3@@QAEXXZ 12031300 f i XMLNotationDecl.obj
 0001:00030320       ?setPublicId@XMLNotationDecl@xercesc_2_3@@QAEXQBG@Z 12031320 f i XMLNotationDecl.obj
 0001:00030390       ?setSystemId@XMLNotationDecl@xercesc_2_3@@QAEXQBG@Z 12031390 f i XMLNotationDecl.obj
 0001:00030400       ?setBaseURI@XMLNotationDecl@xercesc_2_3@@QAEXQBG@Z 12031400 f i XMLNotationDecl.obj
 0001:00030470       ??0XMLNotationDecl@xercesc_2_3@@QAE@QAVMemoryManager@1@@Z 12031470 f   XMLNotationDecl.obj
 0001:00030490       ??0XMLNotationDecl@xercesc_2_3@@QAE@QBG000QAVMemoryManager@1@@Z 12031490 f   XMLNotationDecl.obj
 0001:00030640       ?setName@XMLNotationDecl@xercesc_2_3@@QAEXQBG@Z 12031640 f   XMLNotationDecl.obj
 0001:000306b0       ?cleanUp@XMLNotationDecl@xercesc_2_3@@AAEXXZ 120316b0 f   XMLNotationDecl.obj
 0001:000306b0       ??1XMLNotationDecl@xercesc_2_3@@QAE@XZ 120316b0 f   XMLNotationDecl.obj
 0001:000306f0       ?basicEncodingProbe@XMLRecognizer@xercesc_2_3@@SA?AW4Encodings@12@QBEI@Z 120316f0 f   XMLRecognizer.obj
 0001:00030860       ?encodingForName@XMLRecognizer@xercesc_2_3@@SA?AW4Encodings@12@QBG@Z 12031860 f   XMLRecognizer.obj
 0001:000309e0       ?nameForEncoding@XMLRecognizer@xercesc_2_3@@SAPBGW4Encodings@12@@Z 120319e0 f   XMLRecognizer.obj
 0001:00030a20       ??1XMLValidator@xercesc_2_3@@UAE@XZ 12031a20 f i XMLValidator.obj
 0001:00030a30       ??_FXMLValidator@xercesc_2_3@@QAEXXZ 12031a30 f i XMLValidator.obj
 0001:00030a50       ??_EXMLValidator@xercesc_2_3@@UAEPAXI@Z 12031a50 f i XMLValidator.obj
 0001:00030ab0       ?setScannerInfo@XMLValidator@xercesc_2_3@@QAEXQAVXMLScanner@2@QAVReaderMgr@2@QAVXMLBufferMgr@2@@Z 12031ab0 f i XMLValidator.obj
 0001:00030ad0       ??0XMLRefInfo@xercesc_2_3@@QAE@QBG_N1QAVMemoryManager@1@@Z 12031ad0 f i XMLValidator.obj
 0001:00030b50       ??1XMLRefInfo@xercesc_2_3@@QAE@XZ 12031b50 f i XMLValidator.obj
 0001:00030b60       ??0SecurityManager@xercesc_2_3@@QAE@XZ 12031b60 f i XMLValidator.obj
 0001:00030b70       ??1SecurityManager@xercesc_2_3@@UAE@XZ 12031b70 f i XMLValidator.obj
 0001:00030b80       ??_ESecurityManager@xercesc_2_3@@UAEPAXI@Z 12031b80 f i XMLValidator.obj
 0001:00030be0       ??0Locator@xercesc_2_3@@QAE@XZ 12031be0 f i XMLValidator.obj
 0001:00030bf0       ??_ELocator@xercesc_2_3@@UAEPAXI@Z 12031bf0 f i XMLValidator.obj
 0001:00030c50       ??_FReaderMgr@xercesc_2_3@@QAEXXZ 12031c50 f i XMLValidator.obj
 0001:00030c60       ?getCurrentReaderNum@ReaderMgr@xercesc_2_3@@QBEIXZ 12031c60 f i XMLValidator.obj
 0001:00030c70       ?getName@ReaderMgr@xercesc_2_3@@QAE_NAAVXMLBuffer@2@@Z 12031c70 f i XMLValidator.obj
 0001:00030ca0       ?getNameToken@ReaderMgr@xercesc_2_3@@QAE_NAAVXMLBuffer@2@@Z 12031ca0 f i XMLValidator.obj
 0001:00030cd0       ?getNextCharIfNot@ReaderMgr@xercesc_2_3@@QAE_NGAAG@Z 12031cd0 f i XMLValidator.obj
 0001:00030df0       ?movePlainContentChars@ReaderMgr@xercesc_2_3@@QAEXAAVXMLBuffer@2@@Z 12031df0 f i XMLValidator.obj
 0001:00030e50       ?getValidated@DTDGrammar@xercesc_2_3@@UBE_NXZ 12031e50 f i XMLValidator.obj
 0001:00030e50       ?getThrowEOE@ReaderMgr@xercesc_2_3@@QBE_NXZ 12031e50 f i XMLValidator.obj
 0001:00030e60       ?getSrcOffset@ReaderMgr@xercesc_2_3@@QBEIXZ 12031e60 f i XMLValidator.obj
 0001:00030e70       ?lookingAtChar@ReaderMgr@xercesc_2_3@@QAE_NG@Z 12031e70 f i XMLValidator.obj
 0001:00030e90       ?lookingAtSpace@ReaderMgr@xercesc_2_3@@QAE_NXZ 12031e90 f i XMLValidator.obj
 0001:00030ec0       ?setThrowEOE@ReaderMgr@xercesc_2_3@@QAEX_N@Z 12031ec0 f i XMLValidator.obj
 0001:00030ec0       ?setValidated@DTDGrammar@xercesc_2_3@@UAEX_N@Z 12031ec0 f i XMLValidator.obj
 0001:00030ed0       ?skippedString@ReaderMgr@xercesc_2_3@@QAE_NQBG@Z 12031ed0 f i XMLValidator.obj
 0001:00030ee0       ?skipPastChar@ReaderMgr@xercesc_2_3@@QAEXG@Z 12031ee0 f i XMLValidator.obj
 0001:00030ee0       ?skipToChar@ReaderMgr@xercesc_2_3@@QAEXG@Z 12031ee0 f i XMLValidator.obj
 0001:00030f00       ?peekString@ReaderMgr@xercesc_2_3@@QAE_NQBG@Z 12031f00 f i XMLValidator.obj
 0001:00030f10       ?setXMLVersion@ReaderMgr@xercesc_2_3@@QAEXW4XMLVersion@XMLReader@2@@Z 12031f10 f i XMLValidator.obj
 0001:00030f60       ??0ThrowEOEJanitor@xercesc_2_3@@QAE@PAVReaderMgr@1@_N@Z 12031f60 f i XMLValidator.obj
 0001:00030f80       ??1ThrowEOEJanitor@xercesc_2_3@@QAE@XZ 12031f80 f i XMLValidator.obj
 0001:00030f90       ??_FDTDEntityDecl@xercesc_2_3@@QAEXXZ 12031f90 f i XMLValidator.obj
 0001:00030fa0       ??0DTDEntityDecl@xercesc_2_3@@QAE@QAVMemoryManager@1@@Z 12031fa0 f i XMLValidator.obj
 0001:00030fd0       ??_EDTDEntityDecl@xercesc_2_3@@UAEPAXI@Z 12031fd0 f i XMLValidator.obj
 0001:00031030       ??0DTDEntityDecl@xercesc_2_3@@QAE@QBG_NQAVMemoryManager@1@@Z 12032030 f i XMLValidator.obj
 0001:00031060       ??0DTDEntityDecl@xercesc_2_3@@QAE@QBG0_NQAVMemoryManager@1@@Z 12032060 f i XMLValidator.obj
 0001:000310a0       ??0DTDEntityDecl@xercesc_2_3@@QAE@QBGG_N1@Z 120320a0 f i XMLValidator.obj
 0001:000310e0       ??1DTDEntityDecl@xercesc_2_3@@UAE@XZ 120320e0 f i XMLValidator.obj
 0001:000310f0       ?getDeclaredInIntSubset@DTDEntityDecl@xercesc_2_3@@UBE_NXZ 120320f0 f i XMLValidator.obj
 0001:00031100       ?getIsParameter@DTDEntityDecl@xercesc_2_3@@UBE_NXZ 12032100 f i XMLValidator.obj
 0001:00031110       ?getIsSpecialChar@DTDEntityDecl@xercesc_2_3@@UBE_NXZ 12032110 f i XMLValidator.obj
 0001:00031120       ?setDeclaredInIntSubset@DTDEntityDecl@xercesc_2_3@@QAEX_N@Z 12032120 f i XMLValidator.obj
 0001:00031130       ?setIsParameter@DTDEntityDecl@xercesc_2_3@@QAEX_N@Z 12032130 f i XMLValidator.obj
 0001:00031140       ?setIsSpecialChar@DTDEntityDecl@xercesc_2_3@@QAEX_N@Z 12032140 f i XMLValidator.obj
 0001:00031150       ?getDoNamespaces@XMLScanner@xercesc_2_3@@QBE_NXZ 12032150 f i XMLValidator.obj
 0001:00031160       ?getExitOnFirstFatal@XMLScanner@xercesc_2_3@@QBE_NXZ 12032160 f i XMLValidator.obj
 0001:00031170       ?getInException@XMLScanner@xercesc_2_3@@QBE_NXZ 12032170 f i XMLValidator.obj
 0001:00031180       ?getLocator@XMLScanner@xercesc_2_3@@QBEPBVLocator@2@XZ 12032180 f i XMLValidator.obj
 0001:00031180       ?getReaderMgr@XMLScanner@xercesc_2_3@@QBEPBVReaderMgr@2@XZ 12032180 f i XMLValidator.obj
 0001:00031190       ?getSrcOffset@XMLScanner@xercesc_2_3@@QBEIXZ 12032190 f i XMLValidator.obj
 0001:000311a0       ?getStandalone@XMLScanner@xercesc_2_3@@QBE_NXZ 120321a0 f i XMLValidator.obj
 0001:000311b0       ?getValidationScheme@XMLScanner@xercesc_2_3@@QBE?AW4ValSchemes@12@XZ 120321b0 f i XMLValidator.obj
 0001:000311c0       ?getValidator@XMLScanner@xercesc_2_3@@QAEPAVXMLValidator@2@XZ 120321c0 f i XMLValidator.obj
 0001:000311c0       ?getValidator@XMLScanner@xercesc_2_3@@QBEPBVXMLValidator@2@XZ 120321c0 f i XMLValidator.obj
 0001:000311d0       ?getDoSchema@XMLScanner@xercesc_2_3@@QBE_NXZ 120321d0 f i XMLValidator.obj
 0001:000311e0       ?getValidationSchemaFullChecking@XMLScanner@xercesc_2_3@@QBE_NXZ 120321e0 f i XMLValidator.obj
 0001:000311f0       ?isValidatorFromUser@XMLScanner@xercesc_2_3@@QAE_NXZ 120321f0 f i XMLValidator.obj
 0001:00031200       ?getURIStringPool@XMLScanner@xercesc_2_3@@QBEPBVXMLStringPool@2@XZ 12032200 f i XMLValidator.obj
 0001:00031200       ?getURIStringPool@XMLScanner@xercesc_2_3@@QAEPAVXMLStringPool@2@XZ 12032200 f i XMLValidator.obj
 0001:00031210       ?getHasNoDTD@XMLScanner@xercesc_2_3@@QBE_NXZ 12032210 f i XMLValidator.obj
 0001:00031220       ?getExternalSchemaLocation@XMLScanner@xercesc_2_3@@QBEPAGXZ 12032220 f i XMLValidator.obj
 0001:00031230       ?getExternalNoNamespaceSchemaLocation@XMLScanner@xercesc_2_3@@QBEPAGXZ 12032230 f i XMLValidator.obj
 0001:00031240       ?getSecurityManager@XMLScanner@xercesc_2_3@@QBEPAVSecurityManager@2@XZ 12032240 f i XMLValidator.obj
 0001:00031250       ?getLoadExternalDTD@XMLScanner@xercesc_2_3@@QBE_NXZ 12032250 f i XMLValidator.obj
 0001:00031250       ?getIncludeIgnorableWhitespace@DOMParser@xercesc_2_3@@QBE_NXZ 12032250 f i XMLValidator.obj
 0001:00031260       ?getCalculateSrcOfs@XMLScanner@xercesc_2_3@@QBE_NXZ 12032260 f i XMLValidator.obj
 0001:00031270       ?getRootGrammar@XMLScanner@xercesc_2_3@@QBEPAVGrammar@2@XZ 12032270 f i XMLValidator.obj
 0001:00031280       ?getXMLVersion@XMLScanner@xercesc_2_3@@QBE?AW4XMLVersion@XMLReader@2@XZ 12032280 f i XMLValidator.obj
 0001:00031290       ?getMemoryManager@XMLScanner@xercesc_2_3@@QBEPAVMemoryManager@2@XZ 12032290 f i XMLValidator.obj
 0001:000312a0       ?setDocTypeHandler@XMLScanner@xercesc_2_3@@QAEXQAVDocTypeHandler@2@@Z 120322a0 f i XMLValidator.obj
 0001:000312b0       ?setEntityHandler@XMLScanner@xercesc_2_3@@QAEXQAVXMLEntityHandler@2@@Z 120322b0 f i XMLValidator.obj
 0001:000312c0       ?setGrammarResolver@XMLScanner@xercesc_2_3@@QAEXQAVGrammarResolver@2@@Z 120322c0 f i XMLValidator.obj
 0001:000312d0       ?setExitOnFirstFatal@XMLScanner@xercesc_2_3@@QAEX_N@Z 120322d0 f i XMLValidator.obj
 0001:000312e0       ?setValidationConstraintFatal@XMLScanner@xercesc_2_3@@QAEX_N@Z 120322e0 f i XMLValidator.obj
 0001:000312f0       ?setValidationScheme@XMLScanner@xercesc_2_3@@QAEXW4ValSchemes@12@@Z 120322f0 f i XMLValidator.obj
 0001:00031310       ?setDoSchema@XMLScanner@xercesc_2_3@@QAEX_N@Z 12032310 f i XMLValidator.obj
 0001:00031320       ?setDoNamespaces@XMLScanner@xercesc_2_3@@QAEX_N@Z 12032320 f i XMLValidator.obj
 0001:00031330       ?setValidationSchemaFullChecking@XMLScanner@xercesc_2_3@@QAEX_N@Z 12032330 f i XMLValidator.obj
 0001:00031340       ?setHasNoDTD@XMLScanner@xercesc_2_3@@QAEX_N@Z 12032340 f i XMLValidator.obj
 0001:00031350       ?setRootElemName@XMLScanner@xercesc_2_3@@QAEXPAG@Z 12032350 f i XMLValidator.obj
 0001:000313d0       ?setExternalSchemaLocation@XMLScanner@xercesc_2_3@@QAEXQBG@Z 120323d0 f i XMLValidator.obj
 0001:00031450       ?setExternalNoNamespaceSchemaLocation@XMLScanner@xercesc_2_3@@QAEXQBG@Z 12032450 f i XMLValidator.obj
 0001:000314d0       ?setExternalSchemaLocation@XMLScanner@xercesc_2_3@@QAEXQBD@Z 120324d0 f i XMLValidator.obj
 0001:00031510       ?setExternalNoNamespaceSchemaLocation@XMLScanner@xercesc_2_3@@QAEXQBD@Z 12032510 f i XMLValidator.obj
 0001:00031550       ?setSecurityManager@XMLScanner@xercesc_2_3@@QAEXQAVSecurityManager@2@@Z 12032550 f i XMLValidator.obj
 0001:00031580       ?setLoadExternalDTD@XMLScanner@xercesc_2_3@@QAEX_N@Z 12032580 f i XMLValidator.obj
 0001:00031580       ?setIncludeIgnorableWhitespace@DOMParser@xercesc_2_3@@QAEX_N@Z 12032580 f i XMLValidator.obj
 0001:00031590       ?setCalculateSrcOfs@XMLScanner@xercesc_2_3@@QAEX_N@Z 12032590 f i XMLValidator.obj
 0001:000315a0       ?setStandardUriConformant@XMLScanner@xercesc_2_3@@QAEX_N@Z 120325a0 f i XMLValidator.obj
 0001:000315b0       ?incrementErrorCount@XMLScanner@xercesc_2_3@@QAEXXZ 120325b0 f i XMLValidator.obj
 0001:000315c0       ?setDoValidation@XMLScanner@xercesc_2_3@@QAEX_N@Z 120325c0 f i XMLValidator.obj
 0001:00031630       ?emitError@XMLValidator@xercesc_2_3@@QAEXW4Codes@XMLValid@2@@Z 12032630 f   XMLValidator.obj
 0001:000318c0       ?emitError@XMLValidator@xercesc_2_3@@QAEXW4Codes@XMLValid@2@QBG111@Z 120328c0 f   XMLValidator.obj
 0001:000319e0       ?emitError@XMLValidator@xercesc_2_3@@QAEXW4Codes@XMLValid@2@QBD111@Z 120329e0 f   XMLValidator.obj
 0001:00031b00       ??0XMLValidator@xercesc_2_3@@IAE@QAVXMLErrorReporter@1@@Z 12032b00 f   XMLValidator.obj
 0001:00031b20       ?reinitMsgMutex@XMLValidator@xercesc_2_3@@SAXXZ 12032b20 f   XMLValidator.obj
 0001:00031b50       ?reinitMsgLoader@XMLValidator@xercesc_2_3@@SAXXZ 12032b50 f   XMLValidator.obj
 0001:00031b70       ??_FElemStack@xercesc_2_3@@QAEXXZ 12032b70 f i DGXMLScanner.obj
 0001:00031b80       ??_FWFElemStack@xercesc_2_3@@QAEXXZ 12032b80 f i DGXMLScanner.obj
 0001:00031b90       ?isEmpty@ElemStack@xercesc_2_3@@QBE_NXZ 12032b90 f i DGXMLScanner.obj
 0001:00031ba0       ?getValidationFlag@ElemStack@xercesc_2_3@@QAE_NXZ 12032ba0 f i DGXMLScanner.obj
 0001:00031bb0       ?setValidationFlag@ElemStack@xercesc_2_3@@QAEX_N@Z 12032bb0 f i DGXMLScanner.obj
 0001:00031bd0       ?getCurrentScope@ElemStack@xercesc_2_3@@QAEHXZ 12032bd0 f i DGXMLScanner.obj
 0001:00031be0       ?setCurrentScope@ElemStack@xercesc_2_3@@QAEXH@Z 12032be0 f i DGXMLScanner.obj
 0001:00031c00       ?getCurrentGrammar@ElemStack@xercesc_2_3@@QAEPAVGrammar@2@XZ 12032c00 f i DGXMLScanner.obj
 0001:00031c10       ?setCurrentGrammar@ElemStack@xercesc_2_3@@QAEXPAVGrammar@2@@Z 12032c10 f i DGXMLScanner.obj
 0001:00031c30       ?getCurrentURI@ElemStack@xercesc_2_3@@QAEIXZ 12032c30 f i DGXMLScanner.obj
 0001:00031c40       ?setCurrentURI@ElemStack@xercesc_2_3@@QAEXI@Z 12032c40 f i DGXMLScanner.obj
 0001:00031c60       ?isEmpty@WFElemStack@xercesc_2_3@@QBE_NXZ 12032c60 f i DGXMLScanner.obj
 0001:00031c70       ?getCurrentURI@WFElemStack@xercesc_2_3@@QAEIXZ 12032c70 f i DGXMLScanner.obj
 0001:00031c80       ?setCurrentURI@WFElemStack@xercesc_2_3@@QAEXI@Z 12032c80 f i DGXMLScanner.obj
 0001:00031ca0       ??1Grammar@xercesc_2_3@@UAE@XZ 12032ca0 f i DGXMLScanner.obj
 0001:00031cb0       ??0Grammar@xercesc_2_3@@IAE@XZ 12032cb0 f i DGXMLScanner.obj
 0001:00031cc0       ??_EGrammar@xercesc_2_3@@UAEPAXI@Z 12032cc0 f i DGXMLScanner.obj
 0001:00031d20       ?getName@DGXMLScanner@xercesc_2_3@@UBEPBGXZ 12032d20 f i DGXMLScanner.obj
 0001:00031d30       ??1XMLDocumentHandler@xercesc_2_3@@UAE@XZ 12032d30 f i DGXMLScanner.obj
 0001:00031d40       ??0XMLDocumentHandler@xercesc_2_3@@IAE@XZ 12032d40 f i DGXMLScanner.obj
 0001:00031d50       ??_EXMLDocumentHandler@xercesc_2_3@@UAEPAXI@Z 12032d50 f i DGXMLScanner.obj
 0001:00031db0       ??1XMLEntityHandler@xercesc_2_3@@UAE@XZ 12032db0 f i DGXMLScanner.obj
 0001:00031dc0       ??0XMLEntityHandler@xercesc_2_3@@IAE@XZ 12032dc0 f i DGXMLScanner.obj
 0001:00031dd0       ??_EXMLEntityHandler@xercesc_2_3@@UAEPAXI@Z 12032dd0 f i DGXMLScanner.obj
 0001:00031e30       ??0XMLPScanToken@xercesc_2_3@@QAE@XZ 12032e30 f i DGXMLScanner.obj
 0001:00031e40       ??4DOMNodeImpl@xercesc_2_3@@QAEAAV01@ABV01@@Z 12032e40 f i DGXMLScanner.obj
 0001:00031e40       ??4DOMChildNode@xercesc_2_3@@QAEAAV01@ABV01@@Z 12032e40 f i DGXMLScanner.obj
 0001:00031e40       ??4EndOfEntityException@xercesc_2_3@@QAEAAV01@ABV01@@Z 12032e40 f i DGXMLScanner.obj
 0001:00031e40       ??4ThrowEOEJanitor@xercesc_2_3@@QAEAAV01@ABV01@@Z 12032e40 f i DGXMLScanner.obj
 0001:00031e40       ??4DOMCharacterDataImpl@xercesc_2_3@@QAEAAV01@ABV01@@Z 12032e40 f i DGXMLScanner.obj
 0001:00031e40       ??0XMLPScanToken@xercesc_2_3@@QAE@ABV01@@Z 12032e40 f i DGXMLScanner.obj
 0001:00031e40       ??0EndOfEntityException@xercesc_2_3@@QAE@ABV01@@Z 12032e40 f i DGXMLScanner.obj
 0001:00031e60       ??4XMLPScanToken@xercesc_2_3@@QAEAAV01@ABV01@@Z 12032e60 f i DGXMLScanner.obj
 0001:00031e80       ?set@XMLPScanToken@xercesc_2_3@@IAEXII@Z 12032e80 f i DGXMLScanner.obj
 0001:00031e90       ??0EndOfEntityException@xercesc_2_3@@QAE@PAVXMLEntityDecl@1@I@Z 12032e90 f i DGXMLScanner.obj
 0001:00031e90       ??0SubstitutionGroupComparator@xercesc_2_3@@QAE@QAVGrammarResolver@1@QAVXMLStringPool@1@@Z 12032e90 f i DGXMLScanner.obj
 0001:00031e90       ??0?$NameIdPoolBucketElem@VDTDEntityDecl@xercesc_2_3@@@xercesc_2_3@@QAE@QAVDTDEntityDecl@1@QAU01@@Z 12032e90 f i DGXMLScanner.obj
 0001:00031eb0       ??_FGrammarResolver@xercesc_2_3@@QAEXXZ 12032eb0 f i DGXMLScanner.obj
 0001:00031ec0       ?getStringPool@GrammarResolver@xercesc_2_3@@QAEPAVXMLStringPool@2@XZ 12032ec0 f i DGXMLScanner.obj
 0001:00031ed0       ?orphanGrammar@GrammarResolver@xercesc_2_3@@QAEPAVGrammar@2@QBG@Z 12032ed0 f i DGXMLScanner.obj
 0001:00032060       ??_FDTDAttDef@xercesc_2_3@@QAEXXZ 12033060 f i DGXMLScanner.obj
 0001:00032070       ?getDOMTypeInfoName@DTDAttDef@xercesc_2_3@@UBEPBGXZ 12033070 f i DGXMLScanner.obj
 0001:00032080       ?setElemId@SchemaAttDef@xercesc_2_3@@QAEXI@Z 12033080 f i DGXMLScanner.obj
 0001:00032080       ?setModelType@DTDElementDecl@xercesc_2_3@@QAEXW4ModelTypes@12@@Z 12033080 f i DGXMLScanner.obj
 0001:00032080       ?setAttGroupInfoRegistry@SchemaGrammar@xercesc_2_3@@QAEXQAV?$RefHashTableOf@VXercesAttGroupInfo@xercesc_2_3@@@2@@Z 12033080 f i DGXMLScanner.obj
 0001:00032080       ?setFinalSet@SchemaElementDecl@xercesc_2_3@@QAEXH@Z 12033080 f i DGXMLScanner.obj
 0001:00032080       ?setElemId@DTDAttDef@xercesc_2_3@@QAEXI@Z 12033080 f i DGXMLScanner.obj
 0001:00032090       ??_FDTDElementDecl@xercesc_2_3@@QAEXXZ 12033090 f i DGXMLScanner.obj
 0001:000320a0       ?getContentModel@DTDElementDecl@xercesc_2_3@@UAEPAVXMLContentModel@2@XZ 120330a0 f i DGXMLScanner.obj
 0001:000320c0       ?setContentModel@DTDElementDecl@xercesc_2_3@@UAEXQAVXMLContentModel@2@@Z 120330c0 f i DGXMLScanner.obj
 0001:000320f0       ??0DocTypeHandler@xercesc_2_3@@QAE@XZ 120330f0 f i DGXMLScanner.obj
 0001:00032100       ??1DocTypeHandler@xercesc_2_3@@UAE@XZ 12033100 f i DGXMLScanner.obj
 0001:00032110       ??_EDocTypeHandler@xercesc_2_3@@UAEPAXI@Z 12033110 f i DGXMLScanner.obj
 0001:00032170       ??_FDTDGrammar@xercesc_2_3@@QAEXXZ 12033170 f i DGXMLScanner.obj
 0001:00032180       ?getElemEnumerator@DTDGrammar@xercesc_2_3@@QBE?AV?$NameIdPoolEnumerator@VDTDElementDecl@xercesc_2_3@@@2@XZ 12033180 f i DGXMLScanner.obj
 0001:000321b0       ?getEntityEnumerator@DTDGrammar@xercesc_2_3@@QBE?AV?$NameIdPoolEnumerator@VDTDEntityDecl@xercesc_2_3@@@2@XZ 120331b0 f i DGXMLScanner.obj
 0001:000321e0       ?getNotationEnumerator@DTDGrammar@xercesc_2_3@@QBE?AV?$NameIdPoolEnumerator@VXMLNotationDecl@xercesc_2_3@@@2@XZ 120331e0 f i DGXMLScanner.obj
 0001:00032210       ?getEntityDecl@DTDGrammar@xercesc_2_3@@QAEPAVDTDEntityDecl@2@QBG@Z 12033210 f i DGXMLScanner.obj
 0001:00032210       ?getEntityDecl@DTDGrammar@xercesc_2_3@@QBEPBVDTDEntityDecl@2@QBG@Z 12033210 f i DGXMLScanner.obj
 0001:000322c0       ?putEntityDecl@DTDGrammar@xercesc_2_3@@QBEIQAVDTDEntityDecl@2@@Z 120332c0 f i DGXMLScanner.obj
 0001:000322d0       ?getTargetNamespace@DTDGrammar@xercesc_2_3@@UBEPBGXZ 120332d0 f i DGXMLScanner.obj
 0001:000322e0       ?getElemId@DTDGrammar@xercesc_2_3@@UBEIIQBG0I@Z 120332e0 f i DGXMLScanner.obj
 0001:000323b0       ?getElemDecl@DTDGrammar@xercesc_2_3@@UBEPBVXMLElementDecl@2@IQBG0I@Z 120333b0 f i DGXMLScanner.obj
 0001:000323b0       ?getElemDecl@DTDGrammar@xercesc_2_3@@UAEPAVXMLElementDecl@2@IQBG0I@Z 120333b0 f i DGXMLScanner.obj
 0001:00032510       ?getElemDecl@DTDGrammar@xercesc_2_3@@UBEPBVXMLElementDecl@2@I@Z 12033510 f i DGXMLScanner.obj
 0001:00032510       ?getElemDecl@DTDGrammar@xercesc_2_3@@UAEPAVXMLElementDecl@2@I@Z 12033510 f i DGXMLScanner.obj
 0001:00032560       ?putElemDecl@DTDGrammar@xercesc_2_3@@UBEIQAVXMLElementDecl@2@_N@Z 12033560 f i DGXMLScanner.obj
 0001:00032590       ?getNotationDecl@DTDGrammar@xercesc_2_3@@UAEPAVXMLNotationDecl@2@QBG@Z 12033590 f i DGXMLScanner.obj
 0001:00032590       ?getNotationDecl@DTDGrammar@xercesc_2_3@@UBEPBVXMLNotationDecl@2@QBG@Z 12033590 f i DGXMLScanner.obj
 0001:00032590       ?getNotationDecl@SchemaGrammar@xercesc_2_3@@UBEPBVXMLNotationDecl@2@QBG@Z 12033590 f i DGXMLScanner.obj
 0001:00032590       ?getNotationDecl@SchemaGrammar@xercesc_2_3@@UAEPAVXMLNotationDecl@2@QBG@Z 12033590 f i DGXMLScanner.obj
 0001:00032640       ?putNotationDecl@DTDGrammar@xercesc_2_3@@UBEIQAVXMLNotationDecl@2@@Z 12033640 f i DGXMLScanner.obj
 0001:00032640       ?putNotationDecl@SchemaGrammar@xercesc_2_3@@UBEIQAVXMLNotationDecl@2@@Z 12033640 f i DGXMLScanner.obj
 0001:00032650       ?isReadingExternalEntity@DTDScanner@xercesc_2_3@@AAE_NXZ 12033650 f i DGXMLScanner.obj
 0001:00032670       ??_FDTDValidator@xercesc_2_3@@QAEXXZ 12033670 f i DGXMLScanner.obj
 0001:00032680       ?isAtomic@DatatypeValidator@xercesc_2_3@@UBE_NXZ 12033680 f i DGXMLScanner.obj
 0001:00032680       ?handlesSchema@SchemaValidator@xercesc_2_3@@UBE_NXZ 12033680 f i DGXMLScanner.obj
 0001:00032680       ?handlesDTD@DTDValidator@xercesc_2_3@@UBE_NXZ 12033680 f i DGXMLScanner.obj
 0001:00032690       ??0DGXMLScanner@xercesc_2_3@@QAE@QAVXMLValidator@1@QAVMemoryManager@1@@Z 12033690 f   DGXMLScanner.obj
 0001:00032840       ??_EDGXMLScanner@xercesc_2_3@@UAEPAXI@Z 12033840 f i DGXMLScanner.obj
 0001:000328a0       ??0DGXMLScanner@xercesc_2_3@@QAE@QAVXMLDocumentHandler@1@QAVDocTypeHandler@1@QAVXMLEntityHandler@1@QAVXMLErrorReporter@1@QAVXMLValidator@1@QAVMemoryManager@1@@Z 120338a0 f   DGXMLScanner.obj
 0001:00032a60       ??1DGXMLScanner@xercesc_2_3@@UAE@XZ 12033a60 f   DGXMLScanner.obj
 0001:00032af0       ?getEntityDeclPool@DGXMLScanner@xercesc_2_3@@UBEPBV?$NameIdPool@VDTDEntityDecl@xercesc_2_3@@@2@XZ 12033af0 f   DGXMLScanner.obj
 0001:00032af0       ?getEntityDeclPool@DGXMLScanner@xercesc_2_3@@UAEPAV?$NameIdPool@VDTDEntityDecl@xercesc_2_3@@@2@XZ 12033af0 f   DGXMLScanner.obj
 0001:00032b00       ?scanDocument@DGXMLScanner@xercesc_2_3@@UAEXABVInputSource@2@@Z 12033b00 f   DGXMLScanner.obj
 0001:00032cc0       ?scanNext@DGXMLScanner@xercesc_2_3@@UAE_NAAVXMLPScanToken@2@@Z 12033cc0 f   DGXMLScanner.obj
 0001:00032ff0       ?scanContent@DGXMLScanner@xercesc_2_3@@AAE_N_N@Z 12033ff0 f   DGXMLScanner.obj
 0001:00033190       ?scanEndTag@DGXMLScanner@xercesc_2_3@@AAEXAA_N@Z 12034190 f   DGXMLScanner.obj
 0001:00033470       ?scanDocTypeDecl@DGXMLScanner@xercesc_2_3@@EAEXXZ 12034470 f   DGXMLScanner.obj
 0001:00033e90       ??1XMLBufBid@xercesc_2_3@@QAE@XZ 12034e90 f i DGXMLScanner.obj
 0001:00033ea0       ?scanStartTag@DGXMLScanner@xercesc_2_3@@AAE_NAA_N@Z 12034ea0 f   DGXMLScanner.obj
 0001:000348d0       ?resolveQName@DGXMLScanner@xercesc_2_3@@UAEIQBGAAVXMLBuffer@2@FAAH@Z 120358d0 f   DGXMLScanner.obj
 0001:00034a60       ?loadGrammar@DGXMLScanner@xercesc_2_3@@UAEPAVGrammar@2@ABVInputSource@2@F_N@Z 12035a60 f   DGXMLScanner.obj
 0001:00034be0       ?loadDTDGrammar@DGXMLScanner@xercesc_2_3@@AAEPAVGrammar@2@ABVInputSource@2@_N@Z 12035be0 f   DGXMLScanner.obj
 0001:000350d0       ?commonInit@DGXMLScanner@xercesc_2_3@@AAEXXZ 120360d0 f   DGXMLScanner.obj
 0001:000351c0       ?cleanUp@DGXMLScanner@xercesc_2_3@@AAEXXZ 120361c0 f   DGXMLScanner.obj
 0001:00035200       ?buildAttList@DGXMLScanner@xercesc_2_3@@AAEIIPAVXMLElementDecl@2@AAV?$RefVectorOf@VXMLAttr@xercesc_2_3@@@2@@Z 12036200 f   DGXMLScanner.obj
 0001:000356d0       ?resolvePrefix@DGXMLScanner@xercesc_2_3@@AAEIQBGW4MapModes@ElemStack@2@@Z 120366d0 f   DGXMLScanner.obj
 0001:000357c0       ?scanReset@DGXMLScanner@xercesc_2_3@@EAEXABVInputSource@2@@Z 120367c0 f   DGXMLScanner.obj
 0001:00035a80       ?sendCharData@DGXMLScanner@xercesc_2_3@@EAEXAAVXMLBuffer@2@@Z 12036a80 f   DGXMLScanner.obj
 0001:00035b80       ?updateNSMap@DGXMLScanner@xercesc_2_3@@AAEXQBG00@Z 12036b80 f   DGXMLScanner.obj
 0001:00035df0       ?scanAttrListforNameSpaces@DGXMLScanner@xercesc_2_3@@AAEXPAV?$RefVectorOf@VXMLAttr@xercesc_2_3@@@2@H@Z 12036df0 f   DGXMLScanner.obj
 0001:00035ff0       ?resolveSystemId@DGXMLScanner@xercesc_2_3@@AAEPAVInputSource@2@QBG@Z 12036ff0 f   DGXMLScanner.obj
 0001:00036260       ?scanAttValue@DGXMLScanner@xercesc_2_3@@AAE_NQBVXMLAttDef@2@AAVXMLBuffer@2@@Z 12037260 f   DGXMLScanner.obj
 0001:000366b0       ?scanCDSection@DGXMLScanner@xercesc_2_3@@EAEXXZ 120376b0 f   DGXMLScanner.obj
 0001:00036960       ?scanCharData@DGXMLScanner@xercesc_2_3@@EAEXAAVXMLBuffer@2@@Z 12037960 f   DGXMLScanner.obj
 0001:00036ca0       ?scanEntityRef@DGXMLScanner@xercesc_2_3@@EAE?AW4EntityExpRes@XMLScanner@2@_NAAG1AA_N@Z 12037ca0 f   DGXMLScanner.obj
 0001:00037210       ?orphanKey@?$RefHashTableOf@VGrammar@xercesc_2_3@@@xercesc_2_3@@QAEPAVGrammar@2@QBX@Z 12038210 f i DGXMLScanner.obj
 0001:000372e0       ?nextElement@?$NameIdPoolEnumerator@VDTDEntityDecl@xercesc_2_3@@@xercesc_2_3@@UAEAAVDTDEntityDecl@2@XZ 120382e0 f i DGXMLScanner.obj
 0001:000372e0       ?nextElement@?$NameIdPoolEnumerator@VXMLNotationDecl@xercesc_2_3@@@xercesc_2_3@@UAEAAVXMLNotationDecl@2@XZ 120382e0 f i DGXMLScanner.obj
 0001:000372e0       ?nextElement@?$NameIdPoolEnumerator@VDTDElementDecl@xercesc_2_3@@@xercesc_2_3@@UAEAAVDTDElementDecl@2@XZ 120382e0 f i DGXMLScanner.obj
 0001:00037330       ?hasMoreElements@?$NameIdPoolEnumerator@VDTDElementDecl@xercesc_2_3@@@xercesc_2_3@@UBE_NXZ 12038330 f i DGXMLScanner.obj
 0001:00037330       ?hasMoreElements@?$NameIdPoolEnumerator@VDTDEntityDecl@xercesc_2_3@@@xercesc_2_3@@UBE_NXZ 12038330 f i DGXMLScanner.obj
 0001:00037330       ?hasMoreElements@?$NameIdPoolEnumerator@VXMLNotationDecl@xercesc_2_3@@@xercesc_2_3@@UBE_NXZ 12038330 f i DGXMLScanner.obj
 0001:00037350       ?Reset@?$NameIdPoolEnumerator@VXMLNotationDecl@xercesc_2_3@@@xercesc_2_3@@UAEXXZ 12038350 f i DGXMLScanner.obj
 0001:00037350       ?Reset@?$NameIdPoolEnumerator@VDTDElementDecl@xercesc_2_3@@@xercesc_2_3@@UAEXXZ 12038350 f i DGXMLScanner.obj
 0001:00037350       ?Reset@?$NameIdPoolEnumerator@VDTDEntityDecl@xercesc_2_3@@@xercesc_2_3@@UAEXXZ 12038350 f i DGXMLScanner.obj
 0001:00037360       ?put@?$NameIdPool@VDTDEntityDecl@xercesc_2_3@@@xercesc_2_3@@QAEIQAVDTDEntityDecl@2@@Z 12038360 f i DGXMLScanner.obj
 0001:00037520       ?put@?$NameIdPool@VDTDElementDecl@xercesc_2_3@@@xercesc_2_3@@QAEIQAVDTDElementDecl@2@@Z 12038520 f i DGXMLScanner.obj
 0001:00037700       ?put@?$NameIdPool@VXMLNotationDecl@xercesc_2_3@@@xercesc_2_3@@QAEIQAVXMLNotationDecl@2@@Z 12038700 f i DGXMLScanner.obj
 0001:000378c0       ??1?$Janitor@VXMLDateTime@xercesc_2_3@@@xercesc_2_3@@QAE@XZ 120388c0 f i DGXMLScanner.obj
 0001:000378c0       ??1?$Janitor@VIC_KeyRef@xercesc_2_3@@@xercesc_2_3@@QAE@XZ 120388c0 f i DGXMLScanner.obj
 0001:000378c0       ??1?$Janitor@V?$RefVectorOf@VDatatypeValidator@xercesc_2_3@@@xercesc_2_3@@@xercesc_2_3@@QAE@XZ 120388c0 f i DGXMLScanner.obj
 0001:000378c0       ??1?$Janitor@VRegxParser@xercesc_2_3@@@xercesc_2_3@@QAE@XZ 120388c0 f i DGXMLScanner.obj
 0001:000378c0       ??1?$Janitor@VSchemaAttDef@xercesc_2_3@@@xercesc_2_3@@QAE@XZ 120388c0 f i DGXMLScanner.obj
 0001:000378c0       ??1?$Janitor@VDTDElementDecl@xercesc_2_3@@@xercesc_2_3@@QAE@XZ 120388c0 f i DGXMLScanner.obj
 0001:000378c0       ??1?$Janitor@V?$RefArrayVectorOf@G@xercesc_2_3@@@xercesc_2_3@@QAE@XZ 120388c0 f i DGXMLScanner.obj
 0001:000378c0       ??1?$Janitor@V?$RefVectorOf@VMatch@xercesc_2_3@@@xercesc_2_3@@@xercesc_2_3@@QAE@XZ 120388c0 f i DGXMLScanner.obj
 0001:000378c0       ??1?$Janitor@VInputSource@xercesc_2_3@@@xercesc_2_3@@QAE@XZ 120388c0 f i DGXMLScanner.obj
 0001:000378c0       ??1?$Janitor@V?$RefVectorOf@VXercesStep@xercesc_2_3@@@xercesc_2_3@@@xercesc_2_3@@QAE@XZ 120388c0 f i DGXMLScanner.obj
 0001:000378c0       ??1?$Janitor@VIC_Key@xercesc_2_3@@@xercesc_2_3@@QAE@XZ 120388c0 f i DGXMLScanner.obj
 0001:000378c0       ??1?$Janitor@V?$BaseRefVectorOf@G@xercesc_2_3@@@xercesc_2_3@@QAE@XZ 120388c0 f i DGXMLScanner.obj
 0001:000378c0       ??1?$Janitor@VDTDEntityDecl@xercesc_2_3@@@xercesc_2_3@@QAE@XZ 120388c0 f i DGXMLScanner.obj
 0001:000378c0       ??1?$Janitor@VIC_Unique@xercesc_2_3@@@xercesc_2_3@@QAE@XZ 120388c0 f i DGXMLScanner.obj
 0001:000378e0       ??_E?$NameIdPoolEnumerator@VDTDElementDecl@xercesc_2_3@@@xercesc_2_3@@UAEPAXI@Z 120388e0 f i DGXMLScanner.obj
 0001:000378e0       ??_G?$NameIdPoolEnumerator@VDTDElementDecl@xercesc_2_3@@@xercesc_2_3@@UAEPAXI@Z 120388e0 f i DGXMLScanner.obj
 0001:00037900       ??1?$NameIdPoolEnumerator@VDTDElementDecl@xercesc_2_3@@@xercesc_2_3@@UAE@XZ 12038900 f i DGXMLScanner.obj
 0001:00037910       ??_E?$XMLEnumerator@VDTDElementDecl@xercesc_2_3@@@xercesc_2_3@@UAEPAXI@Z 12038910 f i DGXMLScanner.obj
 0001:00037910       ??_G?$XMLEnumerator@VDTDElementDecl@xercesc_2_3@@@xercesc_2_3@@UAEPAXI@Z 12038910 f i DGXMLScanner.obj
 0001:00037930       ??_E?$NameIdPoolEnumerator@VDTDEntityDecl@xercesc_2_3@@@xercesc_2_3@@UAEPAXI@Z 12038930 f i DGXMLScanner.obj
 0001:00037930       ??_G?$NameIdPoolEnumerator@VDTDEntityDecl@xercesc_2_3@@@xercesc_2_3@@UAEPAXI@Z 12038930 f i DGXMLScanner.obj
 0001:00037950       ??1?$NameIdPoolEnumerator@VDTDEntityDecl@xercesc_2_3@@@xercesc_2_3@@UAE@XZ 12038950 f i DGXMLScanner.obj
 0001:00037960       ??_E?$XMLEnumerator@VDTDEntityDecl@xercesc_2_3@@@xercesc_2_3@@UAEPAXI@Z 12038960 f i DGXMLScanner.obj
 0001:00037960       ??_G?$XMLEnumerator@VDTDEntityDecl@xercesc_2_3@@@xercesc_2_3@@UAEPAXI@Z 12038960 f i DGXMLScanner.obj
 0001:00037980       ??_E?$NameIdPoolEnumerator@VXMLNotationDecl@xercesc_2_3@@@xercesc_2_3@@UAEPAXI@Z 12038980 f i DGXMLScanner.obj
 0001:00037980       ??_G?$NameIdPoolEnumerator@VXMLNotationDecl@xercesc_2_3@@@xercesc_2_3@@UAEPAXI@Z 12038980 f i DGXMLScanner.obj
 0001:000379a0       ??1?$NameIdPoolEnumerator@VXMLNotationDecl@xercesc_2_3@@@xercesc_2_3@@UAE@XZ 120389a0 f i DGXMLScanner.obj
 0001:000379b0       ??_E?$XMLEnumerator@VXMLNotationDecl@xercesc_2_3@@@xercesc_2_3@@UAEPAXI@Z 120389b0 f i DGXMLScanner.obj
 0001:000379b0       ??_G?$XMLEnumerator@VXMLNotationDecl@xercesc_2_3@@@xercesc_2_3@@UAEPAXI@Z 120389b0 f i DGXMLScanner.obj
 0001:000379d0       ?findBucketElem@?$NameIdPool@VDTDEntityDecl@xercesc_2_3@@@xercesc_2_3@@AAEPAU?$NameIdPoolBucketElem@VDTDEntityDecl@xercesc_2_3@@@2@QBGAAI@Z 120389d0 f i DGXMLScanner.obj
 0001:00037a80       ??0ElemStack@xercesc_2_3@@QAE@QAVMemoryManager@1@@Z 12038a80 f   ElemStack.obj
 0001:00037b20       ??1ElemStack@xercesc_2_3@@QAE@XZ 12038b20 f   ElemStack.obj
 0001:00037bc0       ?addLevel@ElemStack@xercesc_2_3@@QAEIXZ 12038bc0 f   ElemStack.obj
 0001:00037d30       ?addLevel@ElemStack@xercesc_2_3@@QAEIQAVXMLElementDecl@2@I@Z 12038d30 f   ElemStack.obj
 0001:00037eb0       ?popTop@ElemStack@xercesc_2_3@@QAEPBUStackElem@12@XZ 12038eb0 f   ElemStack.obj
 0001:00037ef0       ?setElement@ElemStack@xercesc_2_3@@QAEXQAVXMLElementDecl@2@I@Z 12038ef0 f   ElemStack.obj
 0001:00037f50       ?addChild@ElemStack@xercesc_2_3@@QAEIQAVQName@2@_N@Z 12038f50 f   ElemStack.obj
 0001:00038070       ?topElement@ElemStack@xercesc_2_3@@QBEPBUStackElem@12@XZ 12039070 f   ElemStack.obj
 0001:000380b0       ?addPrefix@ElemStack@xercesc_2_3@@QAEXQBGI@Z 120390b0 f   ElemStack.obj
 0001:000381e0       ?mapPrefixToURI@ElemStack@xercesc_2_3@@QBEIQBGW4MapModes@12@AA_N@Z 120391e0 f   ElemStack.obj
 0001:000382d0       ?reset@ElemStack@xercesc_2_3@@QAEXIIII@Z 120392d0 f   ElemStack.obj
 0001:00038340       ?expandMap@ElemStack@xercesc_2_3@@AAEXQAUStackElem@12@@Z 12039340 f   ElemStack.obj
 0001:000383e0       ?expandStack@ElemStack@xercesc_2_3@@AAEXXZ 120393e0 f   ElemStack.obj
 0001:00038480       ??0WFElemStack@xercesc_2_3@@QAE@QAVMemoryManager@1@@Z 12039480 f   ElemStack.obj
 0001:00038520       ??1WFElemStack@xercesc_2_3@@QAE@XZ 12039520 f   ElemStack.obj
 0001:000385c0       ?addLevel@WFElemStack@xercesc_2_3@@QAEIXZ 120395c0 f   ElemStack.obj
 0001:00038700       ?addLevel@WFElemStack@xercesc_2_3@@QAEIQBGII@Z 12039700 f   ElemStack.obj
 0001:000388a0       ?popTop@WFElemStack@xercesc_2_3@@QAEPBUStackElem@12@XZ 120398a0 f   ElemStack.obj
 0001:000388e0       ?setElement@WFElemStack@xercesc_2_3@@QAEXQBGII@Z 120398e0 f   ElemStack.obj
 0001:000389a0       ?topElement@WFElemStack@xercesc_2_3@@QBEPBUStackElem@12@XZ 120399a0 f   ElemStack.obj
 0001:000389e0       ?addPrefix@WFElemStack@xercesc_2_3@@QAEXQBGI@Z 120399e0 f   ElemStack.obj
 0001:00038b10       ?mapPrefixToURI@WFElemStack@xercesc_2_3@@QBEIQBGW4MapModes@12@AA_N@Z 12039b10 f   ElemStack.obj
 0001:00038bb0       ?reset@WFElemStack@xercesc_2_3@@QAEXIIII@Z 12039bb0 f   ElemStack.obj
 0001:00038c20       ?expandMap@WFElemStack@xercesc_2_3@@AAEXXZ 12039c20 f   ElemStack.obj
 0001:00038cd0       ?expandStack@WFElemStack@xercesc_2_3@@AAEXXZ 12039cd0 f   ElemStack.obj
 0001:00038d70       ?setFacetsDefined@DatatypeValidator@xercesc_2_3@@IAEXH@Z 12039d70 f i IGXMLScanner.obj
 0001:00038d80       ?setFixed@DatatypeValidator@xercesc_2_3@@IAEXH@Z 12039d80 f i IGXMLScanner.obj
 0001:00038d90       ?setPattern@DatatypeValidator@xercesc_2_3@@IAEXPBG@Z 12039d90 f i IGXMLScanner.obj
 0001:00038e00       ?setAnonymous@DatatypeValidator@xercesc_2_3@@QAEXXZ 12039e00 f i IGXMLScanner.obj
 0001:00038e10       ?compare@DatatypeValidator@xercesc_2_3@@UAEHQBG0@Z 12039e10 f i IGXMLScanner.obj
 0001:00038e30       ?isSubstitutableBy@DatatypeValidator@xercesc_2_3@@UAE_NQBV12@@Z 12039e30 f i IGXMLScanner.obj
 0001:00038e50       ??_FUnionDatatypeValidator@xercesc_2_3@@QAEXXZ 12039e50 f i IGXMLScanner.obj
 0001:00038e60       ?newInstance@UnionDatatypeValidator@xercesc_2_3@@UAEPAVDatatypeValidator@2@QAV?$RefHashTableOf@VKVStringPair@xercesc_2_3@@@2@QAV?$RefArrayVectorOf@G@2@HQAVMemoryManager@2@@Z 12039e60 f i IGXMLScanner.obj
 0001:00038ee0       ?validate@UnionDatatypeValidator@xercesc_2_3@@UAEXQBG@Z 12039ee0 f i IGXMLScanner.obj
 0001:00038ef0       ?cleanUp@UnionDatatypeValidator@xercesc_2_3@@AAEXXZ 12039ef0 f i IGXMLScanner.obj
 0001:00038f20       ?setEnumeration@UnionDatatypeValidator@xercesc_2_3@@AAEXPAV?$RefArrayVectorOf@G@2@_N@Z 12039f20 f i IGXMLScanner.obj
 0001:00038f60       ?getMemberTypeValidators@UnionDatatypeValidator@xercesc_2_3@@QBEPAV?$RefVectorOf@VDatatypeValidator@xercesc_2_3@@@2@XZ 12039f60 f i IGXMLScanner.obj
 0001:00038f80       ?isAtomic@UnionDatatypeValidator@xercesc_2_3@@UBE_NXZ 12039f80 f i IGXMLScanner.obj
 0001:00039000       ?isSubstitutableBy@UnionDatatypeValidator@xercesc_2_3@@UAE_NQBVDatatypeValidator@2@@Z 1203a000 f i IGXMLScanner.obj
 0001:00039080       ?getMemberTypeName@UnionDatatypeValidator@xercesc_2_3@@QBEPBGXZ 1203a080 f i IGXMLScanner.obj
 0001:00039090       ?getMemberTypeUri@UnionDatatypeValidator@xercesc_2_3@@QBEPBGXZ 1203a090 f i IGXMLScanner.obj
 0001:000390a0       ?getMemberTypeAnonymous@UnionDatatypeValidator@xercesc_2_3@@QBE_NXZ 1203a0a0 f i IGXMLScanner.obj
 0001:000390b0       ?reset@UnionDatatypeValidator@xercesc_2_3@@QAEXXZ 1203a0b0 f i IGXMLScanner.obj
 0001:000390c0       ??_FSchemaAttDef@xercesc_2_3@@QAEXXZ 1203a0c0 f i IGXMLScanner.obj
 0001:000390d0       ?getTypeName@SchemaAttDef@xercesc_2_3@@QBEPBGXZ 1203a0d0 f i IGXMLScanner.obj
 0001:00039100       ?getTypeUri@SchemaAttDef@xercesc_2_3@@QBEPBGXZ 1203a100 f i IGXMLScanner.obj
 0001:00039130       ?getMemberTypeName@SchemaAttDef@xercesc_2_3@@QBEPBGXZ 1203a130 f i IGXMLScanner.obj
 0001:00039140       ?getMemberTypeUri@SchemaAttDef@xercesc_2_3@@QBEPBGXZ 1203a140 f i IGXMLScanner.obj
 0001:00039150       ?getDOMTypeInfoName@SchemaAttDef@xercesc_2_3@@UBEPBGXZ 1203a150 f i IGXMLScanner.obj
 0001:000391c0       ?getDOMTypeInfoUri@SchemaAttDef@xercesc_2_3@@UBEPBGXZ 1203a1c0 f i IGXMLScanner.obj
 0001:00039230       ?getTypeAnonymous@SchemaAttDef@xercesc_2_3@@QBE_NXZ 1203a230 f i IGXMLScanner.obj
 0001:00039250       ?getMemberTypeAnonymous@SchemaAttDef@xercesc_2_3@@QBE_NXZ 1203a250 f i IGXMLScanner.obj
 0001:00039260       ?isTypeDefinitionUnion@SchemaAttDef@xercesc_2_3@@QBE_NXZ 1203a260 f i IGXMLScanner.obj
 0001:00039290       ?resetNamespaceList@SchemaAttDef@xercesc_2_3@@QAEXXZ 1203a290 f i IGXMLScanner.obj
 0001:000392b0       ?setNamespaceList@SchemaAttDef@xercesc_2_3@@QAEXQBV?$ValueVectorOf@I@2@@Z 1203a2b0 f i IGXMLScanner.obj
 0001:00039410       ?reset@SchemaAttDef@xercesc_2_3@@UAEXXZ 1203a410 f i IGXMLScanner.obj
 0001:00039450       ??_FComplexTypeInfo@xercesc_2_3@@QAEXXZ 1203a450 f i IGXMLScanner.obj
 0001:00039460       ?getAbstract@ComplexTypeInfo@xercesc_2_3@@QBE_NXZ 1203a460 f i IGXMLScanner.obj
 0001:00039460       ?getProcessed@SchemaInfo@xercesc_2_3@@QBE_NXZ 1203a460 f i IGXMLScanner.obj
 0001:00039460       ?getUsed@XMLRefInfo@xercesc_2_3@@QBE_NXZ 1203a460 f i IGXMLScanner.obj
 0001:00039470       ?getAdoptContentSpec@ComplexTypeInfo@xercesc_2_3@@QBE_NXZ 1203a470 f i IGXMLScanner.obj
 0001:00039480       ?containsAttWithTypeId@ComplexTypeInfo@xercesc_2_3@@QBE_NXZ 1203a480 f i IGXMLScanner.obj
 0001:00039490       ?getAttDef@ComplexTypeInfo@xercesc_2_3@@QAEPAVSchemaAttDef@2@QBGH@Z 1203a490 f i IGXMLScanner.obj
 0001:00039490       ?getAttDef@ComplexTypeInfo@xercesc_2_3@@QBEPBVSchemaAttDef@2@QBGH@Z 1203a490 f i IGXMLScanner.obj
 0001:00039540       ?elementAt@ComplexTypeInfo@xercesc_2_3@@QAEPAVSchemaElementDecl@2@I@Z 1203a540 f i IGXMLScanner.obj
 0001:00039540       ?elementAt@ComplexTypeInfo@xercesc_2_3@@QBEPBVSchemaElementDecl@2@I@Z 1203a540 f i IGXMLScanner.obj
 0001:00039590       ?getContentModel@ComplexTypeInfo@xercesc_2_3@@QAEPAVXMLContentModel@2@_N@Z 1203a590 f i IGXMLScanner.obj
 0001:000395b0       ?getLocator@ComplexTypeInfo@xercesc_2_3@@QBEPAVXSDLocator@2@XZ 1203a5b0 f i IGXMLScanner.obj
 0001:000395c0       ?getTypeLocalName@ComplexTypeInfo@xercesc_2_3@@QBEPBGXZ 1203a5c0 f i IGXMLScanner.obj
 0001:00039640       ?getTypeUri@ComplexTypeInfo@xercesc_2_3@@QBEPBGXZ 1203a640 f i IGXMLScanner.obj
 0001:00039690       ?setAdoptContentSpec@ComplexTypeInfo@xercesc_2_3@@QAEX_N@Z 1203a690 f i IGXMLScanner.obj
 0001:000396a0       ?setAttWithTypeId@ComplexTypeInfo@xercesc_2_3@@QAEX_N@Z 1203a6a0 f i IGXMLScanner.obj
 0001:000396b0       ?setTypeName@ComplexTypeInfo@xercesc_2_3@@QAEXQBG@Z 1203a6b0 f i IGXMLScanner.obj
 0001:00039740       ?addElement@ComplexTypeInfo@xercesc_2_3@@QAEXQAVSchemaElementDecl@2@@Z 1203a740 f i IGXMLScanner.obj
 0001:00039890       ?setAttWildCard@ComplexTypeInfo@xercesc_2_3@@QAEXQAVSchemaAttDef@2@@Z 1203a890 f i IGXMLScanner.obj
 0001:000398c0       ?setContentModel@ComplexTypeInfo@xercesc_2_3@@QAEXQAVXMLContentModel@2@@Z 1203a8c0 f i IGXMLScanner.obj
 0001:000398f0       ?setAnonymous@ComplexTypeInfo@xercesc_2_3@@QAEXXZ 1203a8f0 f i IGXMLScanner.obj
 0001:00039900       ?hasAttDefs@ComplexTypeInfo@xercesc_2_3@@QBE_NXZ 1203a900 f i IGXMLScanner.obj
 0001:00039940       ?contains@ComplexTypeInfo@xercesc_2_3@@QAE_NQBG@Z 1203a940 f i IGXMLScanner.obj
 0001:00039b40       ?cleanUp@XPathMatcher@xercesc_2_3@@AAEXXZ 1203ab40 f i IGXMLScanner.obj
 0001:00039b80       ??1FieldMatcher@xercesc_2_3@@UAE@XZ 1203ab80 f i IGXMLScanner.obj
 0001:00039b90       ??_EFieldMatcher@xercesc_2_3@@UAEPAXI@Z 1203ab90 f i IGXMLScanner.obj
 0001:00039bf0       ?getFieldCount@IdentityConstraint@xercesc_2_3@@QBEHXZ 1203abf0 f i IGXMLScanner.obj
 0001:00039c00       ?addField@IdentityConstraint@xercesc_2_3@@QAEXQAVIC_Field@2@@Z 1203ac00 f i IGXMLScanner.obj
 0001:00039d30       ?getFieldAt@IdentityConstraint@xercesc_2_3@@QBEPBVIC_Field@2@I@Z 1203ad30 f i IGXMLScanner.obj
 0001:00039d30       ?getFieldAt@IdentityConstraint@xercesc_2_3@@QAEPAVIC_Field@2@I@Z 1203ad30 f i IGXMLScanner.obj
 0001:00039d80       ??_FSchemaElementDecl@xercesc_2_3@@QAEXXZ 1203ad80 f i IGXMLScanner.obj
 0001:00039d90       ?getContentSpec@SchemaElementDecl@xercesc_2_3@@UAEPAVContentSpecNode@2@XZ 1203ad90 f i IGXMLScanner.obj
 0001:00039d90       ?getContentSpec@SchemaElementDecl@xercesc_2_3@@UBEPBVContentSpecNode@2@XZ 1203ad90 f i IGXMLScanner.obj
 0001:00039db0       ?getContentModel@SchemaElementDecl@xercesc_2_3@@UAEPAVXMLContentModel@2@XZ 1203adb0 f i IGXMLScanner.obj
 0001:00039de0       ?getModelType@SchemaElementDecl@xercesc_2_3@@QBE?AW4ModelTypes@12@XZ 1203ade0 f i IGXMLScanner.obj
 0001:00039e00       ?getDatatypeValidator@SchemaElementDecl@xercesc_2_3@@QBEPAVDatatypeValidator@2@XZ 1203ae00 f i IGXMLScanner.obj
 0001:00039e10       ?getComplexTypeInfo@SchemaElementDecl@xercesc_2_3@@QBEPAVComplexTypeInfo@2@XZ 1203ae10 f i IGXMLScanner.obj
 0001:00039e20       ?getAttWildCard@SchemaElementDecl@xercesc_2_3@@QAEPAVSchemaAttDef@2@XZ 1203ae20 f i IGXMLScanner.obj
 0001:00039e20       ?getAttWildCard@SchemaElementDecl@xercesc_2_3@@QBEPBVSchemaAttDef@2@XZ 1203ae20 f i IGXMLScanner.obj
 0001:00039e40       ?isGlobalDecl@SchemaElementDecl@xercesc_2_3@@UBE_NXZ 1203ae40 f i IGXMLScanner.obj
 0001:00039e50       ?getTypeName@SchemaElementDecl@xercesc_2_3@@QBEPBGXZ 1203ae50 f i IGXMLScanner.obj
 0001:00039fb0       ?getTypeType@SchemaElementDecl@xercesc_2_3@@QBE?AW4Complexity@PSVIDefs@2@XZ 1203afb0 f i IGXMLScanner.obj
 0001:00039ff0       ?getTypeUri@SchemaElementDecl@xercesc_2_3@@QBEPBGXZ 1203aff0 f i IGXMLScanner.obj
 0001:0003a0e0       ?getMemberTypeName@SchemaElementDecl@xercesc_2_3@@QBEPBGXZ 1203b0e0 f i IGXMLScanner.obj
 0001:0003a120       ?getMemberTypeUri@SchemaElementDecl@xercesc_2_3@@QBEPBGXZ 1203b120 f i IGXMLScanner.obj
 0001:0003a160       ?getMemberTypeAnonymous@SchemaElementDecl@xercesc_2_3@@QBE_NXZ 1203b160 f i IGXMLScanner.obj
 0001:0003a1a0       ?isTypeDefinitionUnion@SchemaElementDecl@xercesc_2_3@@QBE_NXZ 1203b1a0 f i IGXMLScanner.obj
 0001:0003a1d0       ?getValidationAttempted@SchemaElementDecl@xercesc_2_3@@QBE?AW4Validation@PSVIDefs@2@XZ 1203b1d0 f i IGXMLScanner.obj
 0001:0003a210       ?getTypeAnonymous@SchemaElementDecl@xercesc_2_3@@QBE_NXZ 1203b210 f i IGXMLScanner.obj
 0001:0003a240       ?getDOMTypeInfoName@SchemaElementDecl@xercesc_2_3@@UBEPBGXZ 1203b240 f i IGXMLScanner.obj
 0001:0003a420       ?getDOMTypeInfoUri@SchemaElementDecl@xercesc_2_3@@UBEPBGXZ 1203b420 f i IGXMLScanner.obj
 0001:0003a5c0       ?setDefaultValue@SchemaElementDecl@xercesc_2_3@@QAEXQBG@Z 1203b5c0 f i IGXMLScanner.obj
 0001:0003a630       ?setMembertypeValidator@SchemaAttDef@xercesc_2_3@@QAEXPBVDatatypeValidator@2@@Z 1203b630 f i IGXMLScanner.obj
 0001:0003a630       ?setComplexTypeInfo@SchemaElementDecl@xercesc_2_3@@QAEXQAVComplexTypeInfo@2@@Z 1203b630 f i IGXMLScanner.obj
 0001:0003a630       ?setBaseComplexTypeInfo@ComplexTypeInfo@xercesc_2_3@@QAEXQAV12@@Z 1203b630 f i IGXMLScanner.obj
 0001:0003a640       ?setAttWildCard@SchemaElementDecl@xercesc_2_3@@QAEXQAVSchemaAttDef@2@@Z 1203b640 f i IGXMLScanner.obj
 0001:0003a670       ?setValidationAttempted@SchemaElementDecl@xercesc_2_3@@QAEXW4Validation@PSVIDefs@2@@Z 1203b670 f i IGXMLScanner.obj
 0001:0003a680       ?updateValidityFromAttribute@SchemaElementDecl@xercesc_2_3@@QAEXPBVSchemaAttDef@2@@Z 1203b680 f i IGXMLScanner.obj
 0001:0003a6c0       ?updateValidityFromElement@SchemaElementDecl@xercesc_2_3@@QAEXPBVXMLElementDecl@2@W4GrammarType@Grammar@2@@Z 1203b6c0 f i IGXMLScanner.obj
 0001:0003a730       ?reset@SchemaElementDecl@xercesc_2_3@@QAEXXZ 1203b730 f i IGXMLScanner.obj
 0001:0003a770       ?addIdentityConstraint@SchemaElementDecl@xercesc_2_3@@QAEXQAVIdentityConstraint@2@@Z 1203b770 f i IGXMLScanner.obj
 0001:0003a8a0       ?elementCount@ComplexTypeInfo@xercesc_2_3@@QBEIXZ 1203b8a0 f i IGXMLScanner.obj
 0001:0003a8a0       ?getIdentityConstraintCount@SchemaElementDecl@xercesc_2_3@@QBEIXZ 1203b8a0 f i IGXMLScanner.obj
 0001:0003a8b0       ?getIdentityConstraintAt@SchemaElementDecl@xercesc_2_3@@QBEPAVIdentityConstraint@2@I@Z 1203b8b0 f i IGXMLScanner.obj
 0001:0003a900       ?getName@IGXMLScanner@xercesc_2_3@@UBEPBGXZ 1203b900 f i IGXMLScanner.obj
 0001:0003a910       ?setLength@AbstractStringValidator@xercesc_2_3@@IAEXI@Z 1203b910 f i IGXMLScanner.obj
 0001:0003a920       ?setMaxLength@AbstractStringValidator@xercesc_2_3@@IAEXI@Z 1203b920 f i IGXMLScanner.obj
 0001:0003a920       ?setValidity@SchemaAttDef@xercesc_2_3@@QAEXW4Validity@PSVIDefs@2@@Z 1203b920 f i IGXMLScanner.obj
 0001:0003a920       ?setXsiComplexTypeInfo@SchemaElementDecl@xercesc_2_3@@QAEXQAVComplexTypeInfo@2@@Z 1203b920 f i IGXMLScanner.obj
 0001:0003a930       ?setMinLength@AbstractStringValidator@xercesc_2_3@@IAEXI@Z 1203b930 f i IGXMLScanner.obj
 0001:0003a930       ?setXsiSimpleTypeInfo@SchemaElementDecl@xercesc_2_3@@QAEXQBVDatatypeValidator@2@@Z 1203b930 f i IGXMLScanner.obj
 0001:0003a930       ?setValidationAttempted@SchemaAttDef@xercesc_2_3@@QAEXW4Validation@PSVIDefs@2@@Z 1203b930 f i IGXMLScanner.obj
 0001:0003a930       ?setDocHandler@XMLScanner@xercesc_2_3@@QAEXQAVXMLDocumentHandler@2@@Z 1203b930 f i IGXMLScanner.obj
 0001:0003a940       ?setEnumeration@AbstractStringValidator@xercesc_2_3@@IAEXPAV?$RefArrayVectorOf@G@2@_N@Z 1203b940 f i IGXMLScanner.obj
 0001:0003a980       ??_FStringDatatypeValidator@xercesc_2_3@@QAEXXZ 1203b980 f i IGXMLScanner.obj
 0001:0003a990       ?setWhiteSpace@StringDatatypeValidator@xercesc_2_3@@AAEXF@Z 1203b990 f i IGXMLScanner.obj
 0001:0003a9a0       ??_FIDDatatypeValidator@xercesc_2_3@@QAEXXZ 1203b9a0 f i IGXMLScanner.obj
 0001:0003a9b0       ??_FDatatypeValidatorFactory@xercesc_2_3@@QAEXXZ 1203b9b0 f i IGXMLScanner.obj
 0001:0003a9c0       ?getDatatypeValidator@DatatypeValidatorFactory@xercesc_2_3@@QBEPAVDatatypeValidator@2@QBG@Z 1203b9c0 f i IGXMLScanner.obj
 0001:0003aba0       ?getBuiltInRegistry@DatatypeValidatorFactory@xercesc_2_3@@QBEPAV?$RefHashTableOf@VDatatypeValidator@xercesc_2_3@@@2@XZ 1203bba0 f i IGXMLScanner.obj
 0001:0003abb0       ?cleanUp@DatatypeValidatorFactory@xercesc_2_3@@AAEXXZ 1203bbb0 f i IGXMLScanner.obj
 0001:0003ac50       ??_FSchemaGrammar@xercesc_2_3@@QAEXXZ 1203bc50 f i IGXMLScanner.obj
 0001:0003ac60       ?getElemEnumerator@SchemaGrammar@xercesc_2_3@@QBE?AV?$RefHash3KeysIdPoolEnumerator@VSchemaElementDecl@xercesc_2_3@@@2@XZ 1203bc60 f i IGXMLScanner.obj
 0001:0003ad00       ?getDatatypeRegistry@SchemaGrammar@xercesc_2_3@@QAEPAVDatatypeValidatorFactory@2@XZ 1203bd00 f i IGXMLScanner.obj
 0001:0003ad10       ?getRegex@DatatypeValidator@xercesc_2_3@@IBEPAVRegularExpression@2@XZ 1203bd10 f i IGXMLScanner.obj
 0001:0003ad10       ?getNamespaceScope@SchemaGrammar@xercesc_2_3@@QBEPAVNamespaceScope@2@XZ 1203bd10 f i IGXMLScanner.obj
 0001:0003ad10       ?getXMLNamespaceId@XMLScanner@xercesc_2_3@@QBEIXZ 1203bd10 f i IGXMLScanner.obj
 0001:0003ad10       ?getErrorHandler@DOMParser@xercesc_2_3@@QBEPBVErrorHandler@2@XZ 1203bd10 f i IGXMLScanner.obj
 0001:0003ad10       ?getField@FieldMatcher@xercesc_2_3@@QBEPAVIC_Field@2@XZ 1203bd10 f i IGXMLScanner.obj
 0001:0003ad10       ?getFullName@DTDAttDef@xercesc_2_3@@UBEPBGXZ 1203bd10 f i IGXMLScanner.obj
 0001:0003ad10       ?getBlockSet@SchemaElementDecl@xercesc_2_3@@QBEHXZ 1203bd10 f i IGXMLScanner.obj
 0001:0003ad10       ?getAttName@SchemaAttDef@xercesc_2_3@@QBEPAVQName@2@XZ 1203bd10 f i IGXMLScanner.obj
 0001:0003ad10       ?getErrorHandler@DOMParser@xercesc_2_3@@QAEPAVErrorHandler@2@XZ 1203bd10 f i IGXMLScanner.obj
 0001:0003ad20       ?getXMLNSNamespaceId@XMLScanner@xercesc_2_3@@QBEIXZ 1203bd20 f i IGXMLScanner.obj
 0001:0003ad20       ?getBaseDatatypeValidator@ComplexTypeInfo@xercesc_2_3@@QBEPAVDatatypeValidator@2@XZ 1203bd20 f i IGXMLScanner.obj
 0001:0003ad20       ?getMiscFlags@SchemaElementDecl@xercesc_2_3@@QBEHXZ 1203bd20 f i IGXMLScanner.obj
 0001:0003ad20       ?getDatatypeValidator@SchemaAttDef@xercesc_2_3@@QBEPAVDatatypeValidator@2@XZ 1203bd20 f i IGXMLScanner.obj
 0001:0003ad20       ?getValidSubstitutionGroups@SchemaGrammar@xercesc_2_3@@QBEPAV?$RefHash2KeysTableOf@V?$ValueVectorOf@PAVSchemaElementDecl@xercesc_2_3@@@xercesc_2_3@@@2@XZ 1203bd20 f i IGXMLScanner.obj
 0001:0003ad30       ?setTargetNamespace@SchemaGrammar@xercesc_2_3@@QAEXQBG@Z 1203bd30 f i IGXMLScanner.obj
 0001:0003ada0       ?setDatatypeValidator@SchemaAttDef@xercesc_2_3@@QAEXPAVDatatypeValidator@2@@Z 1203bda0 f i IGXMLScanner.obj
 0001:0003ada0       ?setValidSubstitutionGroups@SchemaGrammar@xercesc_2_3@@QAEXQAV?$RefHash2KeysTableOf@V?$ValueVectorOf@PAVSchemaElementDecl@xercesc_2_3@@@xercesc_2_3@@@2@@Z 1203bda0 f i IGXMLScanner.obj
 0001:0003ada0       ?setMiscFlags@SchemaElementDecl@xercesc_2_3@@QAEXH@Z 1203bda0 f i IGXMLScanner.obj
 0001:0003ada0       ?setBaseDatatypeValidator@ComplexTypeInfo@xercesc_2_3@@QAEXQAVDatatypeValidator@2@@Z 1203bda0 f i IGXMLScanner.obj
 0001:0003adb0       ?getElemId@SchemaGrammar@xercesc_2_3@@UBEIIQBG0I@Z 1203bdb0 f i IGXMLScanner.obj
 0001:0003aee0       ?getElemDecl@SchemaGrammar@xercesc_2_3@@UBEPBVXMLElementDecl@2@IQBG0I@Z 1203bee0 f i IGXMLScanner.obj
 0001:0003aee0       ?getElemDecl@SchemaGrammar@xercesc_2_3@@UAEPAVXMLElementDecl@2@IQBG0I@Z 1203bee0 f i IGXMLScanner.obj
 0001:0003b080       ?getElemDecl@SchemaGrammar@xercesc_2_3@@UBEPBVXMLElementDecl@2@I@Z 1203c080 f i IGXMLScanner.obj
 0001:0003b080       ?getElemDecl@SchemaGrammar@xercesc_2_3@@UAEPAVXMLElementDecl@2@I@Z 1203c080 f i IGXMLScanner.obj
 0001:0003b100       ?putElemDecl@SchemaGrammar@xercesc_2_3@@UBEIQAVXMLElementDecl@2@_N@Z 1203c100 f i IGXMLScanner.obj
 0001:0003b140       ?putGroupElemDecl@SchemaGrammar@xercesc_2_3@@QBEIQAVXMLElementDecl@2@@Z 1203c140 f i IGXMLScanner.obj
 0001:0003b170       ?getValidated@SchemaGrammar@xercesc_2_3@@UBE_NXZ 1203c170 f i IGXMLScanner.obj
 0001:0003b180       ?setValidated@SchemaGrammar@xercesc_2_3@@UAEX_N@Z 1203c180 f i IGXMLScanner.obj
 0001:0003b190       ??1XSDErrorReporter@xercesc_2_3@@UAE@XZ 1203c190 f i IGXMLScanner.obj
 0001:0003b1a0       ??_FXSDErrorReporter@xercesc_2_3@@QAEXXZ 1203c1a0 f i IGXMLScanner.obj
 0001:0003b1b0       ??_EXSDErrorReporter@xercesc_2_3@@UAEPAXI@Z 1203c1b0 f i IGXMLScanner.obj
 0001:0003b210       ?getStandardUriConformant@XMLScanner@xercesc_2_3@@QBE_NXZ 1203c210 f i IGXMLScanner.obj
 0001:0003b210       ?getExitOnFirstFatal@XSDErrorReporter@xercesc_2_3@@QBE_NXZ 1203c210 f i IGXMLScanner.obj
 0001:0003b210       ?getPreprocessed@ComplexTypeInfo@xercesc_2_3@@QBE_NXZ 1203c210 f i IGXMLScanner.obj
 0001:0003b220       ??_FSchemaValidator@xercesc_2_3@@QAEXXZ 1203c220 f i IGXMLScanner.obj
 0001:0003b230       ?setURI@QName@xercesc_2_3@@QAEXI@Z 1203c230 f i IGXMLScanner.obj
 0001:0003b230       ?setDatatypeValidator@SchemaElementDecl@xercesc_2_3@@QAEXPAVDatatypeValidator@2@@Z 1203c230 f i IGXMLScanner.obj
 0001:0003b230       ?setComplexTypeRegistry@SchemaGrammar@xercesc_2_3@@QAEXQAV?$RefHashTableOf@VComplexTypeInfo@xercesc_2_3@@@2@@Z 1203c230 f i IGXMLScanner.obj
 0001:0003b230       ?setContentType@ComplexTypeInfo@xercesc_2_3@@QAEXH@Z 1203c230 f i IGXMLScanner.obj
 0001:0003b230       ?setGrammarResolver@SchemaValidator@xercesc_2_3@@QAEXPAVGrammarResolver@2@@Z 1203c230 f i IGXMLScanner.obj
 0001:0003b240       ?setXsiType@SchemaValidator@xercesc_2_3@@QAEXQBG0I@Z 1203c240 f i IGXMLScanner.obj
 0001:0003b2d0       ?setNillable@SchemaValidator@xercesc_2_3@@QAEX_N@Z 1203c2d0 f i IGXMLScanner.obj
 0001:0003b2d0       ?setStandardUriConformant@ReaderMgr@xercesc_2_3@@QAEX_N@Z 1203c2d0 f i IGXMLScanner.obj
 0001:0003b2e0       ?setExitOnFirstFatal@SchemaValidator@xercesc_2_3@@QAEX_N@Z 1203c2e0 f i IGXMLScanner.obj
 0001:0003b2f0       ?setDatatypeBuffer@SchemaValidator@xercesc_2_3@@QAEXQBG@Z 1203c2f0 f i IGXMLScanner.obj
 0001:0003b310       ?getCurrentTypeInfo@SchemaValidator@xercesc_2_3@@QBEPAVComplexTypeInfo@2@XZ 1203c310 f i IGXMLScanner.obj
 0001:0003b380       ?setRootElemId@DTDGrammar@xercesc_2_3@@QAEXI@Z 1203c380 f i IGXMLScanner.obj
 0001:0003b380       ?setModelType@SchemaElementDecl@xercesc_2_3@@QAEXW4ModelTypes@12@@Z 1203c380 f i IGXMLScanner.obj
 0001:0003b380       ?setGrammar@SchemaValidator@xercesc_2_3@@UAEXPAVGrammar@2@@Z 1203c380 f i IGXMLScanner.obj
 0001:0003b380       ?setType@DatatypeValidator@xercesc_2_3@@IAEXW4ValidatorType@12@@Z 1203c380 f i IGXMLScanner.obj
 0001:0003b380       ?setElementId@ComplexTypeInfo@xercesc_2_3@@QAEXI@Z 1203c380 f i IGXMLScanner.obj
 0001:0003b380       ?setAttributeDeclRegistry@SchemaGrammar@xercesc_2_3@@QAEXQAV?$RefHashTableOf@VXMLAttDef@xercesc_2_3@@@2@@Z 1203c380 f i IGXMLScanner.obj
 0001:0003b390       ?setErrorReporter@SchemaValidator@xercesc_2_3@@QAEXQAVXMLErrorReporter@2@@Z 1203c390 f i IGXMLScanner.obj
 0001:0003b3a0       ?isOccurrenceRangeOK@SchemaValidator@xercesc_2_3@@AAE_NHHHH@Z 1203c3a0 f i IGXMLScanner.obj
 0001:0003b3d0       ??_FXPathMatcherStack@xercesc_2_3@@QAEXXZ 1203c3d0 f i IGXMLScanner.obj
 0001:0003b3e0       ?size@XPathMatcherStack@xercesc_2_3@@QBEIXZ 1203c3e0 f i IGXMLScanner.obj
 0001:0003b3f0       ?getMatcherAt@XPathMatcherStack@xercesc_2_3@@QBEPAVXPathMatcher@2@I@Z 1203c3f0 f i IGXMLScanner.obj
 0001:0003b3f0       ?getChild@UnionToken@xercesc_2_3@@UBEPAVToken@2@H@Z 1203c3f0 f i IGXMLScanner.obj
 0001:0003b440       ?pushContext@XPathMatcherStack@xercesc_2_3@@QAEXXZ 1203c440 f i IGXMLScanner.obj
 0001:0003b4e0       ?popContext@XPathMatcherStack@xercesc_2_3@@QAEXXZ 1203c4e0 f i IGXMLScanner.obj
 0001:0003b5a0       ?addMatcher@XPathMatcherStack@xercesc_2_3@@QAEXQAVXPathMatcher@2@@Z 1203c5a0 f i IGXMLScanner.obj
 0001:0003b6a0       ??_FValueStoreCache@xercesc_2_3@@QAEXXZ 1203c6a0 f i IGXMLScanner.obj
 0001:0003b6b0       ?getValueStoreFor@ValueStoreCache@xercesc_2_3@@QAEPAVValueStore@2@QBVIC_Field@2@H@Z 1203c6b0 f i IGXMLScanner.obj
 0001:0003b750       ?getValueStoreFor@ValueStoreCache@xercesc_2_3@@QAEPAVValueStore@2@QBVIdentityConstraint@2@H@Z 1203c750 f i IGXMLScanner.obj
 0001:0003b7f0       ?getGlobalValueStoreFor@ValueStoreCache@xercesc_2_3@@QAEPAVValueStore@2@QBVIdentityConstraint@2@@Z 1203c7f0 f i IGXMLScanner.obj
 0001:0003b880       ??1SelectorMatcher@xercesc_2_3@@UAE@XZ 1203c880 f i IGXMLScanner.obj
 0001:0003b890       ??_ESelectorMatcher@xercesc_2_3@@UAEPAXI@Z 1203c890 f i IGXMLScanner.obj
 0001:0003b8f0       ??_FFieldValueMap@xercesc_2_3@@QAEXXZ 1203c8f0 f i IGXMLScanner.obj
 0001:0003b900       ?getDatatypeValidatorAt@FieldValueMap@xercesc_2_3@@QBEPAVDatatypeValidator@2@I@Z 1203c900 f i IGXMLScanner.obj
 0001:0003b950       ?getDatatypeValidatorFor@FieldValueMap@xercesc_2_3@@QBEPAVDatatypeValidator@2@QBVIC_Field@2@@Z 1203c950 f i IGXMLScanner.obj
 0001:0003b9b0       ?getValueAt@FieldValueMap@xercesc_2_3@@QBEPAGI@Z 1203c9b0 f i IGXMLScanner.obj
 0001:0003b9b0       ?anyAttributeAt@XercesAttGroupInfo@xercesc_2_3@@QBEPBVSchemaAttDef@2@I@Z 1203c9b0 f i IGXMLScanner.obj
 0001:0003b9b0       ?anyAttributeAt@XercesAttGroupInfo@xercesc_2_3@@QAEPAVSchemaAttDef@2@I@Z 1203c9b0 f i IGXMLScanner.obj
 0001:0003ba00       ?getValueFor@FieldValueMap@xercesc_2_3@@QBEPAGQBVIC_Field@2@@Z 1203ca00 f i IGXMLScanner.obj
 0001:0003ba60       ?keyAt@FieldValueMap@xercesc_2_3@@QBEPAVIC_Field@2@I@Z 1203ca60 f i IGXMLScanner.obj
 0001:0003bab0       ?size@FieldValueMap@xercesc_2_3@@QBEIXZ 1203cab0 f i IGXMLScanner.obj
 0001:0003bac0       ?put@FieldValueMap@xercesc_2_3@@QAEXQAVIC_Field@2@QAVDatatypeValidator@2@QBG@Z 1203cac0 f i IGXMLScanner.obj
 0001:0003bd60       ??0IGXMLScanner@xercesc_2_3@@QAE@QAVXMLValidator@1@QAVMemoryManager@1@@Z 1203cd60 f   IGXMLScanner.obj
 0001:0003be70       ??_EIGXMLScanner@xercesc_2_3@@UAEPAXI@Z 1203ce70 f i IGXMLScanner.obj
 0001:0003bed0       ??0IGXMLScanner@xercesc_2_3@@QAE@QAVXMLDocumentHandler@1@QAVDocTypeHandler@1@QAVXMLEntityHandler@1@QAVXMLErrorReporter@1@QAVXMLValidator@1@QAVMemoryManager@1@@Z 1203ced0 f   IGXMLScanner.obj
 0001:0003bff0       ??1IGXMLScanner@xercesc_2_3@@UAE@XZ 1203cff0 f   IGXMLScanner.obj
 0001:0003c070       ?getEntityDeclPool@IGXMLScanner@xercesc_2_3@@UBEPBV?$NameIdPool@VDTDEntityDecl@xercesc_2_3@@@2@XZ 1203d070 f   IGXMLScanner.obj
 0001:0003c070       ?getEntityDeclPool@IGXMLScanner@xercesc_2_3@@UAEPAV?$NameIdPool@VDTDEntityDecl@xercesc_2_3@@@2@XZ 1203d070 f   IGXMLScanner.obj
 0001:0003c080       ?scanDocument@IGXMLScanner@xercesc_2_3@@UAEXABVInputSource@2@@Z 1203d080 f   IGXMLScanner.obj
 0001:0003c240       ?scanNext@IGXMLScanner@xercesc_2_3@@UAE_NAAVXMLPScanToken@2@@Z 1203d240 f   IGXMLScanner.obj
 0001:0003c580       ?commonInit@IGXMLScanner@xercesc_2_3@@AAEXXZ 1203d580 f   IGXMLScanner.obj
 0001:0003c7b0       ?cleanUp@IGXMLScanner@xercesc_2_3@@AAEXXZ 1203d7b0 f   IGXMLScanner.obj
 0001:0003c850       ?rawAttrScan@IGXMLScanner@xercesc_2_3@@AAEIQBGAAV?$RefVectorOf@VKVStringPair@xercesc_2_3@@@2@AA_N@Z 1203d850 f   IGXMLScanner.obj
 0001:0003cd70       ?scanContent@IGXMLScanner@xercesc_2_3@@AAE_N_N@Z 1203dd70 f   IGXMLScanner.obj
 0001:0003cf30       ?scanEndTag@IGXMLScanner@xercesc_2_3@@AAEXAA_N@Z 1203df30 f   IGXMLScanner.obj
 0001:0003d750       ?scanDocTypeDecl@IGXMLScanner@xercesc_2_3@@EAEXXZ 1203e750 f   IGXMLScanner.obj
 0001:0003e170       ?scanStartTag@IGXMLScanner@xercesc_2_3@@AAE_NAA_N@Z 1203f170 f   IGXMLScanner.obj
 0001:0003ebb0       ?scanStartTagNS@IGXMLScanner@xercesc_2_3@@AAE_NAA_N@Z 1203fbb0 f   IGXMLScanner.obj
 0001:000400e0       ?resizeElemState@SGXMLScanner@xercesc_2_3@@AAEXXZ 120410e0 f   IGXMLScanner.obj
 0001:000400e0       ?resizeElemState@IGXMLScanner@xercesc_2_3@@AAEXXZ 120410e0 f   IGXMLScanner.obj
 0001:00040160       ?loadGrammar@IGXMLScanner@xercesc_2_3@@UAEPAVGrammar@2@ABVInputSource@2@F_N@Z 12041160 f   IGXMLScanner.obj
 0001:00040300       ?loadDTDGrammar@IGXMLScanner@xercesc_2_3@@AAEPAVGrammar@2@ABVInputSource@2@_N@Z 12041300 f   IGXMLScanner.obj
 0001:00040870       ??1?$XMLEnumerator@VSchemaAttDef@xercesc_2_3@@@xercesc_2_3@@UAE@XZ 12041870 f i IGXMLScanner.obj
 0001:00040880       ??1?$XMLEnumerator@VSchemaElementDecl@xercesc_2_3@@@xercesc_2_3@@UAE@XZ 12041880 f i IGXMLScanner.obj
 0001:00040890       ??_E?$XMLEnumerator@VSchemaAttDef@xercesc_2_3@@@xercesc_2_3@@UAEPAXI@Z 12041890 f i IGXMLScanner.obj
 0001:00040890       ??_G?$XMLEnumerator@VSchemaAttDef@xercesc_2_3@@@xercesc_2_3@@UAEPAXI@Z 12041890 f i IGXMLScanner.obj
 0001:000408b0       ??_E?$XMLEnumerator@VSchemaElementDecl@xercesc_2_3@@@xercesc_2_3@@UAEPAXI@Z 120418b0 f i IGXMLScanner.obj
 0001:000408b0       ??_G?$XMLEnumerator@VSchemaElementDecl@xercesc_2_3@@@xercesc_2_3@@UAEPAXI@Z 120418b0 f i IGXMLScanner.obj
 0001:000408d0       ?setElementAt@?$BaseRefVectorOf@G@xercesc_2_3@@QAEXQAGI@Z 120418d0 f i IGXMLScanner.obj
 0001:00040930       ??1?$RefHash2KeysTableOfEnumerator@VSchemaAttDef@xercesc_2_3@@@xercesc_2_3@@UAE@XZ 12041930 f i IGXMLScanner.obj
 0001:00040a10       ?nextElement@?$RefHash2KeysTableOfEnumerator@VSchemaAttDef@xercesc_2_3@@@xercesc_2_3@@UAEAAVSchemaAttDef@2@XZ 12041a10 f i IGXMLScanner.obj
 0001:00040a90       ?hasMoreElements@?$RefHash3KeysIdPoolEnumerator@VSchemaElementDecl@xercesc_2_3@@@xercesc_2_3@@UBE_NXZ 12041a90 f i IGXMLScanner.obj
 0001:00040ab0       ?nextElement@?$RefHash3KeysIdPoolEnumerator@VSchemaElementDecl@xercesc_2_3@@@xercesc_2_3@@UAEAAVSchemaElementDecl@2@XZ 12041ab0 f i IGXMLScanner.obj
 0001:00040b00       ?put@?$RefHash3KeysIdPool@VSchemaElementDecl@xercesc_2_3@@@xercesc_2_3@@QAEIPAXHHQAVSchemaElementDecl@2@@Z 12041b00 f i IGXMLScanner.obj
 0001:00040cc0       ?setElementAt@?$BaseRefVectorOf@VXPathMatcher@xercesc_2_3@@@xercesc_2_3@@QAEXQAVXPathMatcher@2@I@Z 12041cc0 f i IGXMLScanner.obj
 0001:00040cc0       ?setElementAt@?$BaseRefVectorOf@VENameMap@xercesc_2_3@@@xercesc_2_3@@QAEXQAVENameMap@2@I@Z 12041cc0 f i IGXMLScanner.obj
 0001:00040d20       ??_G?$RefVectorOf@VSchemaElementDecl@xercesc_2_3@@@xercesc_2_3@@UAEPAXI@Z 12041d20 f i IGXMLScanner.obj
 0001:00040d20       ??_E?$RefVectorOf@VSchemaElementDecl@xercesc_2_3@@@xercesc_2_3@@UAEPAXI@Z 12041d20 f i IGXMLScanner.obj
 0001:00040d40       ??1?$RefVectorOf@VSchemaElementDecl@xercesc_2_3@@@xercesc_2_3@@UAE@XZ 12041d40 f i IGXMLScanner.obj
 0001:00040dc0       ??1?$BaseRefVectorOf@VSchemaElementDecl@xercesc_2_3@@@xercesc_2_3@@UAE@XZ 12041dc0 f i IGXMLScanner.obj
 0001:00040dd0       ??_G?$RefHash2KeysTableOfEnumerator@VSchemaAttDef@xercesc_2_3@@@xercesc_2_3@@UAEPAXI@Z 12041dd0 f i IGXMLScanner.obj
 0001:00040dd0       ??_E?$RefHash2KeysTableOfEnumerator@VSchemaAttDef@xercesc_2_3@@@xercesc_2_3@@UAEPAXI@Z 12041dd0 f i IGXMLScanner.obj
 0001:00040df0       ??_E?$RefVectorOf@VIC_Field@xercesc_2_3@@@xercesc_2_3@@UAEPAXI@Z 12041df0 f i IGXMLScanner.obj
 0001:00040df0       ??_G?$RefVectorOf@VIC_Field@xercesc_2_3@@@xercesc_2_3@@UAEPAXI@Z 12041df0 f i IGXMLScanner.obj
 0001:00040e10       ??1?$RefVectorOf@VIC_Field@xercesc_2_3@@@xercesc_2_3@@UAE@XZ 12041e10 f i IGXMLScanner.obj
 0001:00040ea0       ??1?$BaseRefVectorOf@VIC_Field@xercesc_2_3@@@xercesc_2_3@@UAE@XZ 12041ea0 f i IGXMLScanner.obj
 0001:00040eb0       ??_G?$RefVectorOf@VIdentityConstraint@xercesc_2_3@@@xercesc_2_3@@UAEPAXI@Z 12041eb0 f i IGXMLScanner.obj
 0001:00040eb0       ??_E?$RefVectorOf@VIdentityConstraint@xercesc_2_3@@@xercesc_2_3@@UAEPAXI@Z 12041eb0 f i IGXMLScanner.obj
 0001:00040ed0       ??1?$RefVectorOf@VIdentityConstraint@xercesc_2_3@@@xercesc_2_3@@UAE@XZ 12041ed0 f i IGXMLScanner.obj
 0001:00040f50       ??1?$BaseRefVectorOf@VIdentityConstraint@xercesc_2_3@@@xercesc_2_3@@UAE@XZ 12041f50 f i IGXMLScanner.obj
 0001:00040f60       ??_G?$RefHash3KeysIdPoolEnumerator@VSchemaElementDecl@xercesc_2_3@@@xercesc_2_3@@UAEPAXI@Z 12041f60 f i IGXMLScanner.obj
 0001:00040f60       ??_E?$RefHash3KeysIdPoolEnumerator@VSchemaElementDecl@xercesc_2_3@@@xercesc_2_3@@UAEPAXI@Z 12041f60 f i IGXMLScanner.obj
 0001:00040f80       ??1?$RefHash3KeysIdPoolEnumerator@VSchemaElementDecl@xercesc_2_3@@@xercesc_2_3@@UAE@XZ 12041f80 f i IGXMLScanner.obj
 0001:00041080       ??_G?$RefVectorOf@VKVStringPair@xercesc_2_3@@@xercesc_2_3@@UAEPAXI@Z 12042080 f i IGXMLScanner.obj
 0001:00041080       ??_E?$RefVectorOf@VKVStringPair@xercesc_2_3@@@xercesc_2_3@@UAEPAXI@Z 12042080 f i IGXMLScanner.obj
 0001:000410a0       ??1?$RefVectorOf@VKVStringPair@xercesc_2_3@@@xercesc_2_3@@UAE@XZ 120420a0 f i IGXMLScanner.obj
 0001:00041130       ??1?$BaseRefVectorOf@VKVStringPair@xercesc_2_3@@@xercesc_2_3@@UAE@XZ 12042130 f i IGXMLScanner.obj
 0001:00041140       ??0?$BaseRefVectorOf@G@xercesc_2_3@@QAE@I_NQAVMemoryManager@1@@Z 12042140 f i IGXMLScanner.obj
 0001:000411a0       ?removeElementAt@?$ValueVectorOf@PAVComplexTypeInfo@xercesc_2_3@@@xercesc_2_3@@QAEXI@Z 120421a0 f i IGXMLScanner.obj
 0001:000411a0       ?removeElementAt@?$ValueVectorOf@I@xercesc_2_3@@QAEXI@Z 120421a0 f i IGXMLScanner.obj
 0001:000411a0       ?removeElementAt@?$ValueVectorOf@H@xercesc_2_3@@QAEXI@Z 120421a0 f i IGXMLScanner.obj
 0001:00041200       ??0DOMNode@xercesc_2_3@@IAE@XZ 12042200 f i IGXMLScanner2.obj
 0001:00041210       ??_EDOMNode@xercesc_2_3@@UAEPAXI@Z 12042210 f i IGXMLScanner2.obj
 0001:00041270       ??0DOMElement@xercesc_2_3@@IAE@XZ 12042270 f i IGXMLScanner2.obj
 0001:00041280       ??0DOMAttr@xercesc_2_3@@IAE@XZ 12042280 f i IGXMLScanner2.obj
 0001:00041290       ?getElemAttrDefaultQualified@SchemaInfo@xercesc_2_3@@QBEGXZ 12042290 f i IGXMLScanner2.obj
 0001:000412a0       ?getImportingListEnumerator@SchemaInfo@xercesc_2_3@@QBE?AV?$BaseRefVectorEnumerator@VSchemaInfo@xercesc_2_3@@@2@XZ 120422a0 f i IGXMLScanner2.obj
 0001:000412d0       ?setElemAttrDefaultQualified@SchemaInfo@xercesc_2_3@@QAEXG@Z 120422d0 f i IGXMLScanner2.obj
 0001:000412e0       ?setUsed@XMLRefInfo@xercesc_2_3@@QAEX_N@Z 120422e0 f i IGXMLScanner2.obj
 0001:000412e0       ?setAbstract@ComplexTypeInfo@xercesc_2_3@@QAEX_N@Z 120422e0 f i IGXMLScanner2.obj
 0001:000412e0       ?useCachedGrammarInParse@GrammarResolver@xercesc_2_3@@QAEX_N@Z 120422e0 f i IGXMLScanner2.obj
 0001:000412e0       ?setProcessed@SchemaInfo@xercesc_2_3@@QAEX_N@Z 120422e0 f i IGXMLScanner2.obj
 0001:000412f0       ?addImportedNS@SchemaInfo@xercesc_2_3@@QAEXH@Z 120422f0 f i IGXMLScanner2.obj
 0001:00041440       ?addSchemaInfo@SchemaInfo@xercesc_2_3@@QAEXQAV12@W4ListType@12@@Z 12042440 f i IGXMLScanner2.obj
 0001:00041670       ?getImportInfo@SchemaInfo@xercesc_2_3@@QBEPAV12@I@Z 12042670 f i IGXMLScanner2.obj
 0001:000416e0       ?containsInfo@SchemaInfo@xercesc_2_3@@QBE_NQBV12@W4ListType@12@@Z 120426e0 f i IGXMLScanner2.obj
 0001:00041750       ?circularImportExist@SchemaInfo@xercesc_2_3@@QAE_NI@Z 12042750 f i IGXMLScanner2.obj
 0001:000417c0       ?isFailedRedefine@SchemaInfo@xercesc_2_3@@QAE_NQBVDOMElement@2@@Z 120427c0 f i IGXMLScanner2.obj
 0001:00041800       ?addFailedRedefine@SchemaInfo@xercesc_2_3@@QAEXQBVDOMElement@2@@Z 12042800 f i IGXMLScanner2.obj
 0001:00041930       ?isImportingNS@SchemaInfo@xercesc_2_3@@QAE_NH@Z 12042930 f i IGXMLScanner2.obj
 0001:00041970       ?addRecursingType@SchemaInfo@xercesc_2_3@@QAEXQBVDOMElement@2@QBG@Z 12042970 f i IGXMLScanner2.obj
 0001:00041b80       ?clearTopLevelComponents@SchemaInfo@xercesc_2_3@@AAEXXZ 12042b80 f i IGXMLScanner2.obj
 0001:00041bc0       ??_FGeneralAttributeCheck@xercesc_2_3@@QAEXXZ 12042bc0 f i IGXMLScanner2.obj
 0001:00041bd0       ?getFacetId@GeneralAttributeCheck@xercesc_2_3@@QAEGQBG@Z 12042bd0 f i IGXMLScanner2.obj
 0001:00041c70       ?getPrefix@TraverseSchema@xercesc_2_3@@AAEPBGQBG@Z 12042c70 f i IGXMLScanner2.obj
 0001:00041cd0       ?getLocalPart@TraverseSchema@xercesc_2_3@@AAEPBGQBG@Z 12042cd0 f i IGXMLScanner2.obj
 0001:00041d60       ?isValidRefDeclaration@TraverseSchema@xercesc_2_3@@AAE_NQBVDOMElement@2@@Z 12042d60 f i IGXMLScanner2.obj
 0001:00041f30       ?getElementAttValue@TraverseSchema@xercesc_2_3@@AAEPBGQBVDOMElement@2@QBG_N@Z 12042f30 f i IGXMLScanner2.obj
 0001:00041fb0       ?checkForEmptyTargetNamespace@TraverseSchema@xercesc_2_3@@AAEXQBVDOMElement@2@@Z 12042fb0 f i IGXMLScanner2.obj
 0001:00042000       ?isBaseFromAnotherSchema@TraverseSchema@xercesc_2_3@@AAE_NQBG@Z 12043000 f i IGXMLScanner2.obj
 0001:000420b0       ?isAttrOrAttrGroup@TraverseSchema@xercesc_2_3@@AAE_NQBVDOMElement@2@@Z 120430b0 f i IGXMLScanner2.obj
 0001:000421d0       ?genAnonTypeName@TraverseSchema@xercesc_2_3@@AAEPBGQBG@Z 120431d0 f i IGXMLScanner2.obj
 0001:00042240       ?popCurrentTypeNameStack@TraverseSchema@xercesc_2_3@@AAEXXZ 12043240 f i IGXMLScanner2.obj
 0001:000422b0       ?copyWildCardData@TraverseSchema@xercesc_2_3@@AAEXQBVSchemaAttDef@2@QAV32@@Z 120432b0 f i IGXMLScanner2.obj
 0001:000422e0       ?getRedefineNewTypeName@TraverseSchema@xercesc_2_3@@AAEXQBGHAAVXMLBuffer@2@@Z 120432e0 f i IGXMLScanner2.obj
 0001:00042320       ?normalizeURI@TraverseSchema@xercesc_2_3@@AAEXQBGAAVXMLBuffer@2@@Z 12043320 f i IGXMLScanner2.obj
 0001:000423b0       ??0DOMDocumentRange@xercesc_2_3@@IAE@XZ 120433b0 f i IGXMLScanner2.obj
 0001:000423c0       ??1DOMDocumentRange@xercesc_2_3@@UAE@XZ 120433c0 f i IGXMLScanner2.obj
 0001:000423d0       ??_EDOMDocumentRange@xercesc_2_3@@UAEPAXI@Z 120433d0 f i IGXMLScanner2.obj
 0001:00042430       ??0DOMDocumentTraversal@xercesc_2_3@@IAE@XZ 12043430 f i IGXMLScanner2.obj
 0001:00042440       ??1DOMDocumentTraversal@xercesc_2_3@@UAE@XZ 12043440 f i IGXMLScanner2.obj
 0001:00042450       ??_EDOMDocumentTraversal@xercesc_2_3@@UAEPAXI@Z 12043450 f i IGXMLScanner2.obj
 0001:000424b0       ??0DOMDocument@xercesc_2_3@@IAE@XZ 120434b0 f i IGXMLScanner2.obj
 0001:000424e0       ??1DOMDocument@xercesc_2_3@@UAE@XZ 120434e0 f i IGXMLScanner2.obj
 0001:00042520       ??_EDOMDocument@xercesc_2_3@@UAEPAXI@Z 12043520 f i IGXMLScanner2.obj
 0001:00042580       ??0DOMDocumentType@xercesc_2_3@@IAE@XZ 12043580 f i IGXMLScanner2.obj
 0001:00042590       ??_FAbstractDOMParser@xercesc_2_3@@QAEXXZ 12043590 f i IGXMLScanner2.obj
 0001:000425a0       ?getExpandEntityReferences@AbstractDOMParser@xercesc_2_3@@QBE_NXZ 120435a0 f i IGXMLScanner2.obj
 0001:000425b0       ?isCachingGrammarFromParse@XMLScanner@xercesc_2_3@@QBE_NXZ 120435b0 f i IGXMLScanner2.obj
 0001:000425b0       ?getCreateEntityReferenceNodes@AbstractDOMParser@xercesc_2_3@@QBE_NXZ 120435b0 f i IGXMLScanner2.obj
 0001:000425b0       ?getToCreateXMLDeclTypeNode@DOMParser@xercesc_2_3@@QBE_NXZ 120435b0 f i IGXMLScanner2.obj
 0001:000425b0       ?getProvided@XMLAttDef@xercesc_2_3@@QBE_NXZ 120435b0 f i IGXMLScanner2.obj
 0001:000425c0       ?isUsingCachedGrammarInParse@XMLScanner@xercesc_2_3@@QBE_NXZ 120435c0 f i IGXMLScanner2.obj
 0001:000425c0       ?getIncludeIgnorableWhitespace@AbstractDOMParser@xercesc_2_3@@QBE_NXZ 120435c0 f i IGXMLScanner2.obj
 0001:000425c0       ?isExternal@XMLAttDef@xercesc_2_3@@QBE_NXZ 120435c0 f i IGXMLScanner2.obj
 0001:000425c0       ?getCreateEntityReferenceNodes@DOMParser@xercesc_2_3@@QBE_NXZ 120435c0 f i IGXMLScanner2.obj
 0001:000425d0       ?getParseInProgress@AbstractDOMParser@xercesc_2_3@@IBE_NXZ 120435d0 f i IGXMLScanner2.obj
 0001:000425d0       ?getNormalizeData@XMLScanner@xercesc_2_3@@QBE_NXZ 120435d0 f i IGXMLScanner2.obj
 0001:000425e0       ?setExpandEntityReferences@AbstractDOMParser@xercesc_2_3@@QAEX_N@Z 120435e0 f i IGXMLScanner2.obj
 0001:000425f0       ?setCreateEntityReferenceNodes@AbstractDOMParser@xercesc_2_3@@QAEX_N@Z 120435f0 f i IGXMLScanner2.obj
 0001:000425f0       ?cacheGrammarFromParse@XMLScanner@xercesc_2_3@@QAEX_N@Z 120435f0 f i IGXMLScanner2.obj
 0001:000425f0       ?setToCreateXMLDeclTypeNode@DOMParser@xercesc_2_3@@QAEX_N@Z 120435f0 f i IGXMLScanner2.obj
 0001:000425f0       ?setProvided@XMLAttDef@xercesc_2_3@@QAEX_N@Z 120435f0 f i IGXMLScanner2.obj
 0001:00042600       ?setIncludeIgnorableWhitespace@AbstractDOMParser@xercesc_2_3@@QAEX_N@Z 12043600 f i IGXMLScanner2.obj
 0001:00042600       ?setExternalAttDeclaration@XMLAttDef@xercesc_2_3@@QAEX_N@Z 12043600 f i IGXMLScanner2.obj
 0001:00042600       ?setCreateEntityReferenceNodes@DOMParser@xercesc_2_3@@QAEX_N@Z 12043600 f i IGXMLScanner2.obj
 0001:00042600       ?useCachedGrammarInParse@XMLScanner@xercesc_2_3@@QAEX_N@Z 12043600 f i IGXMLScanner2.obj
 0001:00042610       ?setEnclosingScope@SchemaElementDecl@xercesc_2_3@@QAEXH@Z 12043610 f i IGXMLScanner2.obj
 0001:00042610       ?setGroupInfoRegistry@SchemaGrammar@xercesc_2_3@@QAEXQAV?$RefHashTableOf@VXercesGroupInfo@xercesc_2_3@@@2@@Z 12043610 f i IGXMLScanner2.obj
 0001:00042610       ?setCurrentNode@AbstractDOMParser@xercesc_2_3@@IAEXPAVDOMNode@2@@Z 12043610 f i IGXMLScanner2.obj
 0001:00042620       ?setDocument@AbstractDOMParser@xercesc_2_3@@IAEXPAVDOMDocument@2@@Z 12043620 f i IGXMLScanner2.obj
 0001:00042620       ?setNamespaceScope@SchemaGrammar@xercesc_2_3@@QAEXQAVNamespaceScope@2@@Z 12043620 f i IGXMLScanner2.obj
 0001:00042620       ?setRegex@DatatypeValidator@xercesc_2_3@@IAEXQAVRegularExpression@2@@Z 12043620 f i IGXMLScanner2.obj
 0001:00042620       ?setBlockSet@SchemaElementDecl@xercesc_2_3@@QAEXH@Z 12043620 f i IGXMLScanner2.obj
 0001:00042630       ?setParseInProgress@AbstractDOMParser@xercesc_2_3@@IAEX_N@Z 12043630 f i IGXMLScanner2.obj
 0001:00042630       ?setNormalizeData@XMLScanner@xercesc_2_3@@QAEX_N@Z 12043630 f i IGXMLScanner2.obj
 0001:00042640       ??_FXercesDOMParser@xercesc_2_3@@QAEXXZ 12043640 f i IGXMLScanner2.obj
 0001:00042650       ??_FXSDDOMParser@xercesc_2_3@@QAEXXZ 12043650 f i IGXMLScanner2.obj
 0001:00042660       ?getSawFatal@XSDDOMParser@xercesc_2_3@@QBE_NXZ 12043660 f i IGXMLScanner2.obj
 0001:00042670       ?buildAttList@IGXMLScanner@xercesc_2_3@@AAEIABV?$RefVectorOf@VKVStringPair@xercesc_2_3@@@2@IPAVXMLElementDecl@2@AAV?$RefVectorOf@VXMLAttr@xercesc_2_3@@@2@@Z 12043670 f   IGXMLScanner2.obj
 0001:00043580       ?normalizeAttValue@IGXMLScanner@xercesc_2_3@@AAE_NQBVXMLAttDef@2@QBGAAVXMLBuffer@2@@Z 12044580 f   IGXMLScanner2.obj
 0001:00043850       ?resolvePrefix@IGXMLScanner@xercesc_2_3@@AAEIQBGW4MapModes@ElemStack@2@@Z 12044850 f   IGXMLScanner2.obj
 0001:00043850       ?resolvePrefix@SGXMLScanner@xercesc_2_3@@AAEIQBGW4MapModes@ElemStack@2@@Z 12044850 f   IGXMLScanner2.obj
 0001:00043940       ?scanReset@IGXMLScanner@xercesc_2_3@@EAEXABVInputSource@2@@Z 12044940 f   IGXMLScanner2.obj
 0001:00043ce0       ?sendCharData@IGXMLScanner@xercesc_2_3@@EAEXAAVXMLBuffer@2@@Z 12044ce0 f   IGXMLScanner2.obj
 0001:00044130       ?updateNSMap@IGXMLScanner@xercesc_2_3@@AAEXQBG0@Z 12045130 f   IGXMLScanner2.obj
 0001:00044420       ?scanRawAttrListforNameSpaces@IGXMLScanner@xercesc_2_3@@AAEXPBV?$RefVectorOf@VKVStringPair@xercesc_2_3@@@2@H@Z 12045420 f   IGXMLScanner2.obj
 0001:000449b0       ?parseSchemaLocation@IGXMLScanner@xercesc_2_3@@AAEXQBG@Z 120459b0 f   IGXMLScanner2.obj
 0001:00044a70       ?resolveSchemaGrammar@IGXMLScanner@xercesc_2_3@@AAEXQBG0@Z 12045a70 f   IGXMLScanner2.obj
 0001:00045180       ?resolveSystemId@IGXMLScanner@xercesc_2_3@@AAEPAVInputSource@2@QBG@Z 12046180 f   IGXMLScanner2.obj
 0001:000453f0       ?loadXMLSchemaGrammar@IGXMLScanner@xercesc_2_3@@AAEPAVGrammar@2@ABVInputSource@2@_N@Z 120463f0 f   IGXMLScanner2.obj
 0001:000456a0       ?basicAttrValueScan@IGXMLScanner@xercesc_2_3@@AAE_NQBGAAVXMLBuffer@2@@Z 120466a0 f   IGXMLScanner2.obj
 0001:00045940       ?scanAttValue@IGXMLScanner@xercesc_2_3@@AAE_NQBVXMLAttDef@2@AAVXMLBuffer@2@@Z 12046940 f   IGXMLScanner2.obj
 0001:00045e00       ?scanCDSection@IGXMLScanner@xercesc_2_3@@EAEXXZ 12046e00 f   IGXMLScanner2.obj
 0001:000461d0       ?scanCharData@IGXMLScanner@xercesc_2_3@@EAEXAAVXMLBuffer@2@@Z 120471d0 f   IGXMLScanner2.obj
 0001:00046530       ?scanEntityRef@IGXMLScanner@xercesc_2_3@@EAE?AW4EntityExpRes@XMLScanner@2@_NAAG1AA_N@Z 12047530 f   IGXMLScanner2.obj
 0001:00046aa0       ?switchGrammar@IGXMLScanner@xercesc_2_3@@AAE_NQBG@Z 12047aa0 f   IGXMLScanner2.obj
 0001:00046ba0       ?laxElementValidation@IGXMLScanner@xercesc_2_3@@AAE_NPAVQName@2@PAVContentLeafNameTypeVector@2@QBVXMLContentModel@2@I@Z 12047ba0 f   IGXMLScanner2.obj
 0001:00046dd0       ?anyAttributeValidation@IGXMLScanner@xercesc_2_3@@AAE_NPAVSchemaAttDef@2@IAA_N1@Z 12047dd0 f   IGXMLScanner2.obj
 0001:00046eb0       ?normalizeURI@IGXMLScanner@xercesc_2_3@@AAEXQBGAAVXMLBuffer@2@@Z 12047eb0 f   IGXMLScanner2.obj
 0001:00046eb0       ?normalizeURI@SGXMLScanner@xercesc_2_3@@AAEXQBGAAVXMLBuffer@2@@Z 12047eb0 f   IGXMLScanner2.obj
 0001:00046f40       ?hasMoreElements@?$BaseRefVectorEnumerator@VSchemaInfo@xercesc_2_3@@@xercesc_2_3@@UBE_NXZ 12047f40 f i IGXMLScanner2.obj
 0001:00046f50       ?nextElement@?$BaseRefVectorEnumerator@VSchemaInfo@xercesc_2_3@@@xercesc_2_3@@UAEAAVSchemaInfo@2@XZ 12047f50 f i IGXMLScanner2.obj
 0001:00046fa0       ?Reset@?$BaseRefVectorEnumerator@VSchemaInfo@xercesc_2_3@@@xercesc_2_3@@UAEXXZ 12047fa0 f i IGXMLScanner2.obj
 0001:00046fa0       ?Reset@?$RefHash3KeysIdPoolEnumerator@VSchemaElementDecl@xercesc_2_3@@@xercesc_2_3@@UAEXXZ 12047fa0 f i IGXMLScanner2.obj
 0001:00046fb0       ?containsElement@?$ValueVectorOf@H@xercesc_2_3@@QAE_NABHI@Z 12047fb0 f i IGXMLScanner2.obj
 0001:00046fb0       ?containsElement@?$ValueVectorOf@I@xercesc_2_3@@QAE_NABII@Z 12047fb0 f i IGXMLScanner2.obj
 0001:00046fe0       ??_G?$BaseRefVectorEnumerator@VSchemaInfo@xercesc_2_3@@@xercesc_2_3@@UAEPAXI@Z 12047fe0 f i IGXMLScanner2.obj
 0001:00046fe0       ??_E?$BaseRefVectorEnumerator@VSchemaInfo@xercesc_2_3@@@xercesc_2_3@@UAEPAXI@Z 12047fe0 f i IGXMLScanner2.obj
 0001:00047000       ??1?$BaseRefVectorEnumerator@VSchemaInfo@xercesc_2_3@@@xercesc_2_3@@UAE@XZ 12048000 f i IGXMLScanner2.obj
 0001:00047060       ??1?$XMLEnumerator@VSchemaInfo@xercesc_2_3@@@xercesc_2_3@@UAE@XZ 12048060 f i IGXMLScanner2.obj
 0001:00047070       ??_G?$XMLEnumerator@VSchemaInfo@xercesc_2_3@@@xercesc_2_3@@UAEPAXI@Z 12048070 f i IGXMLScanner2.obj
 0001:00047070       ??_E?$XMLEnumerator@VSchemaInfo@xercesc_2_3@@@xercesc_2_3@@UAEPAXI@Z 12048070 f i IGXMLScanner2.obj
 0001:00047090       ??_G?$RefVectorOf@VSchemaInfo@xercesc_2_3@@@xercesc_2_3@@UAEPAXI@Z 12048090 f i IGXMLScanner2.obj
 0001:00047090       ??_E?$RefVectorOf@VSchemaInfo@xercesc_2_3@@@xercesc_2_3@@UAEPAXI@Z 12048090 f i IGXMLScanner2.obj
 0001:000470b0       ??1?$RefVectorOf@VSchemaInfo@xercesc_2_3@@@xercesc_2_3@@UAE@XZ 120480b0 f i IGXMLScanner2.obj
 0001:00047140       ??1?$BaseRefVectorOf@VSchemaInfo@xercesc_2_3@@@xercesc_2_3@@UAE@XZ 12048140 f i IGXMLScanner2.obj
 0001:00047150       ??0?$BaseRefVectorOf@VSchemaInfo@xercesc_2_3@@@xercesc_2_3@@QAE@I_NQAVMemoryManager@1@@Z 12048150 f i IGXMLScanner2.obj
 0001:000471b0       ??_EDOMDocument@xercesc_2_3@@W3AEPAXI@Z 120481b0 f i IGXMLScanner2.obj
 0001:000471c0       ??_EDOMDocument@xercesc_2_3@@W7AEPAXI@Z 120481c0 f i IGXMLScanner2.obj
 0001:000471d0       ?allocate@MemoryManagerImpl@xercesc_2_3@@UAEPAXI@Z 120481d0 f   MemoryManagerImpl.obj
 0001:000471e0       ?deallocate@MemoryManagerImpl@xercesc_2_3@@UAEXPAX@Z 120481e0 f   MemoryManagerImpl.obj
 0001:000471f0       ??0ReaderMgr@xercesc_2_3@@QAE@QAVMemoryManager@1@@Z 120481f0 f   ReaderMgr.obj
 0001:00047230       ??_EReaderMgr@xercesc_2_3@@UAEPAXI@Z 12048230 f i ReaderMgr.obj
 0001:00047290       ??1ReaderMgr@xercesc_2_3@@UAE@XZ 12048290 f   ReaderMgr.obj
 0001:000473b0       ?isEmpty@ReaderMgr@xercesc_2_3@@QBE_NXZ 120483b0 f   ReaderMgr.obj
 0001:000473c0       ?getNextChar@ReaderMgr@xercesc_2_3@@QAEGXZ 120483c0 f   ReaderMgr.obj
 0001:00047590       ?getSpaces@ReaderMgr@xercesc_2_3@@QAEXAAVXMLBuffer@2@@Z 12048590 f   ReaderMgr.obj
 0001:000475d0       ?getUpToCharOrWS@ReaderMgr@xercesc_2_3@@QAEXAAVXMLBuffer@2@G@Z 120485d0 f   ReaderMgr.obj
 0001:00047610       ?peekNextChar@ReaderMgr@xercesc_2_3@@QAEGXZ 12048610 f   ReaderMgr.obj
 0001:000476d0       ?skippedChar@ReaderMgr@xercesc_2_3@@QAE_NG@Z 120486d0 f   ReaderMgr.obj
 0001:00047710       ?skippedSpace@ReaderMgr@xercesc_2_3@@QAE_NXZ 12048710 f   ReaderMgr.obj
 0001:00047750       ?skipIfQuote@ReaderMgr@xercesc_2_3@@QAE_NAAG@Z 12048750 f   ReaderMgr.obj
 0001:00047790       ?skipPastSpaces@ReaderMgr@xercesc_2_3@@QAE_NXZ 12048790 f   ReaderMgr.obj
 0001:000477e0       ?skipQuotedString@ReaderMgr@xercesc_2_3@@QAEXG@Z 120487e0 f   ReaderMgr.obj
 0001:00047960       ?skipUntilIn@ReaderMgr@xercesc_2_3@@QAEGQBG@Z 12048960 f   ReaderMgr.obj
 0001:00047be0       ?skipUntilInOrWS@ReaderMgr@xercesc_2_3@@QAEGQBG@Z 12048be0 f   ReaderMgr.obj
 0001:00047e70       ?atEOF@ReaderMgr@xercesc_2_3@@QBE_NXZ 12048e70 f   ReaderMgr.obj
 0001:00047e90       ?cleanStackBackTo@ReaderMgr@xercesc_2_3@@QAEXI@Z 12048e90 f   ReaderMgr.obj
 0001:00048040       ?createReader@ReaderMgr@xercesc_2_3@@QAEPAVXMLReader@2@ABVInputSource@2@_NW4RefFrom@32@W4Types@32@W4Sources@32@1@Z 12049040 f   ReaderMgr.obj
 0001:000481c0       ?createReader@ReaderMgr@xercesc_2_3@@QAEPAVXMLReader@2@QBG0_NW4RefFrom@32@W4Types@32@W4Sources@32@AAPAVInputSource@2@1@Z 120491c0 f   ReaderMgr.obj
 0001:000484b0       ?createReader@ReaderMgr@xercesc_2_3@@QAEPAVXMLReader@2@QBG00_NW4RefFrom@32@W4Types@32@W4Sources@32@AAPAVInputSource@2@1@Z 120494b0 f   ReaderMgr.obj
 0001:000487b0       ?createIntEntReader@ReaderMgr@xercesc_2_3@@QAEPAVXMLReader@2@QBGW4RefFrom@32@W4Types@32@0I_N3@Z 120497b0 f   ReaderMgr.obj
 0001:000488e0       ?getCurrentEncodingStr@ReaderMgr@xercesc_2_3@@QBEPBGXZ 120498e0 f   ReaderMgr.obj
 0001:00048900       ?getReaderDepth@ReaderMgr@xercesc_2_3@@QBEIXZ 12049900 f   ReaderMgr.obj
 0001:00048920       ?getLastExtEntityInfo@ReaderMgr@xercesc_2_3@@QBEXAAULastExtEntityInfo@12@@Z 12049920 f   ReaderMgr.obj
 0001:00048980       ?isScanningPERefOutOfLiteral@ReaderMgr@xercesc_2_3@@QBE_NXZ 12049980 f   ReaderMgr.obj
 0001:000489b0       ?pushReader@ReaderMgr@xercesc_2_3@@QAE_NQAVXMLReader@2@QAVXMLEntityDecl@2@@Z 120499b0 f   ReaderMgr.obj
 0001:00048c20       ?reset@ReaderMgr@xercesc_2_3@@QAEXXZ 12049c20 f   ReaderMgr.obj
 0001:00048cd0       ?getPublicId@ReaderMgr@xercesc_2_3@@UBEPBGXZ 12049cd0 f   ReaderMgr.obj
 0001:00048d00       ?getSystemId@ReaderMgr@xercesc_2_3@@UBEPBGXZ 12049d00 f   ReaderMgr.obj
 0001:00048d30       ?getColumnNumber@ReaderMgr@xercesc_2_3@@UBEJXZ 12049d30 f   ReaderMgr.obj
 0001:00048d60       ?getLineNumber@ReaderMgr@xercesc_2_3@@UBEJXZ 12049d60 f   ReaderMgr.obj
 0001:00048d90       ?getLastExtEntity@ReaderMgr@xercesc_2_3@@ABEPBVXMLReader@2@AAPBVXMLEntityDecl@2@@Z 12049d90 f   ReaderMgr.obj
 0001:00048f00       ?popReader@ReaderMgr@xercesc_2_3@@AAE_NXZ 12049f00 f   ReaderMgr.obj
 0001:00049180       ??1?$BaseRefVectorOf@VXMLReader@xercesc_2_3@@@xercesc_2_3@@UAE@XZ 1204a180 f i ReaderMgr.obj
 0001:00049190       ??1?$BaseRefVectorOf@VXMLEntityDecl@xercesc_2_3@@@xercesc_2_3@@UAE@XZ 1204a190 f i ReaderMgr.obj
 0001:000491a0       ??_E?$RefVectorOf@VXMLReader@xercesc_2_3@@@xercesc_2_3@@UAEPAXI@Z 1204a1a0 f i ReaderMgr.obj
 0001:000491a0       ??_G?$RefVectorOf@VXMLReader@xercesc_2_3@@@xercesc_2_3@@UAEPAXI@Z 1204a1a0 f i ReaderMgr.obj
 0001:000491c0       ??1?$RefVectorOf@VXMLReader@xercesc_2_3@@@xercesc_2_3@@UAE@XZ 1204a1c0 f i ReaderMgr.obj
 0001:00049250       ??_E?$RefVectorOf@VXMLEntityDecl@xercesc_2_3@@@xercesc_2_3@@UAEPAXI@Z 1204a250 f i ReaderMgr.obj
 0001:00049250       ??_G?$RefVectorOf@VXMLEntityDecl@xercesc_2_3@@@xercesc_2_3@@UAEPAXI@Z 1204a250 f i ReaderMgr.obj
 0001:00049270       ??1?$RefVectorOf@VXMLEntityDecl@xercesc_2_3@@@xercesc_2_3@@UAE@XZ 1204a270 f i ReaderMgr.obj
 0001:000492f0       ?orphanElementAt@?$BaseRefVectorOf@V?$RefHashTableOf@VValueStore@xercesc_2_3@@@xercesc_2_3@@@xercesc_2_3@@QAEPAV?$RefHashTableOf@VValueStore@xercesc_2_3@@@2@I@Z 1204a2f0 f i ReaderMgr.obj
 0001:000492f0       ?orphanElementAt@?$BaseRefVectorOf@VXMLReader@xercesc_2_3@@@xercesc_2_3@@QAEPAVXMLReader@2@I@Z 1204a2f0 f i ReaderMgr.obj
 0001:000492f0       ?orphanElementAt@?$BaseRefVectorOf@VXMLEntityDecl@xercesc_2_3@@@xercesc_2_3@@QAEPAVXMLEntityDecl@2@I@Z 1204a2f0 f i ReaderMgr.obj
 0001:000492f0       ?orphanElementAt@?$BaseRefVectorOf@VXMLBuffer@xercesc_2_3@@@xercesc_2_3@@QAEPAVXMLBuffer@2@I@Z 1204a2f0 f i ReaderMgr.obj
 0001:00049380       ?elementAt@?$BaseRefVectorOf@VXMLEntityDecl@xercesc_2_3@@@xercesc_2_3@@QBEPBVXMLEntityDecl@2@I@Z 1204a380 f i ReaderMgr.obj
 0001:000493c0       ??0?$BaseRefVectorOf@VXMLReader@xercesc_2_3@@@xercesc_2_3@@QAE@I_NQAVMemoryManager@1@@Z 1204a3c0 f i ReaderMgr.obj
 0001:00049420       ??0?$BaseRefVectorOf@VXMLEntityDecl@xercesc_2_3@@@xercesc_2_3@@QAE@I_NQAVMemoryManager@1@@Z 1204a420 f i ReaderMgr.obj
 0001:00049480       ?getName@SGXMLScanner@xercesc_2_3@@UBEPBGXZ 1204a480 f i SGXMLScanner.obj
 0001:00049490       ??0SGXMLScanner@xercesc_2_3@@QAE@QAVXMLValidator@1@QAVMemoryManager@1@@Z 1204a490 f   SGXMLScanner.obj
 0001:000495e0       ??_ESGXMLScanner@xercesc_2_3@@UAEPAXI@Z 1204a5e0 f i SGXMLScanner.obj
 0001:00049640       ??0SGXMLScanner@xercesc_2_3@@QAE@QAVXMLDocumentHandler@1@QAVDocTypeHandler@1@QAVXMLEntityHandler@1@QAVXMLErrorReporter@1@QAVXMLValidator@1@QAVMemoryManager@1@@Z 1204a640 f   SGXMLScanner.obj
 0001:000497a0       ??1SGXMLScanner@xercesc_2_3@@UAE@XZ 1204a7a0 f   SGXMLScanner.obj
 0001:00049820       ?scanDocument@SGXMLScanner@xercesc_2_3@@UAEXABVInputSource@2@@Z 1204a820 f   SGXMLScanner.obj
 0001:000499e0       ?scanNext@SGXMLScanner@xercesc_2_3@@UAE_NAAVXMLPScanToken@2@@Z 1204a9e0 f   SGXMLScanner.obj
 0001:00049d10       ?rawAttrScan@SGXMLScanner@xercesc_2_3@@AAEIQBGAAV?$RefVectorOf@VKVStringPair@xercesc_2_3@@@2@AA_N@Z 1204ad10 f   SGXMLScanner.obj
 0001:0004a270       ?scanContent@SGXMLScanner@xercesc_2_3@@AAE_N_N@Z 1204b270 f   SGXMLScanner.obj
 0001:0004a410       ?scanEndTag@SGXMLScanner@xercesc_2_3@@AAEXAA_N@Z 1204b410 f   SGXMLScanner.obj
 0001:0004ab00       ?scanDocTypeDecl@SGXMLScanner@xercesc_2_3@@EAEXXZ 1204bb00 f   SGXMLScanner.obj
 0001:0004ab40       ?scanStartTag@SGXMLScanner@xercesc_2_3@@AAE_NAA_N@Z 1204bb40 f   SGXMLScanner.obj
 0001:0004c040       ?resolveQName@IGXMLScanner@xercesc_2_3@@UAEIQBGAAVXMLBuffer@2@FAAH@Z 1204d040 f   SGXMLScanner.obj
 0001:0004c040       ?resolveQName@SGXMLScanner@xercesc_2_3@@UAEIQBGAAVXMLBuffer@2@FAAH@Z 1204d040 f   SGXMLScanner.obj
 0001:0004c1d0       ?activateSelectorFor@IGXMLScanner@xercesc_2_3@@AAEXQAVIdentityConstraint@2@H@Z 1204d1d0 f   SGXMLScanner.obj
 0001:0004c1d0       ?activateSelectorFor@SGXMLScanner@xercesc_2_3@@AAEXQAVIdentityConstraint@2@H@Z 1204d1d0 f   SGXMLScanner.obj
 0001:0004c310       ?loadGrammar@SGXMLScanner@xercesc_2_3@@UAEPAVGrammar@2@ABVInputSource@2@F_N@Z 1204d310 f   SGXMLScanner.obj
 0001:0004c490       ?commonInit@SGXMLScanner@xercesc_2_3@@AAEXXZ 1204d490 f   SGXMLScanner.obj
 0001:0004c890       ?cleanUp@SGXMLScanner@xercesc_2_3@@AAEXXZ 1204d890 f   SGXMLScanner.obj
 0001:0004c990       ?buildAttList@SGXMLScanner@xercesc_2_3@@AAEIABV?$RefVectorOf@VKVStringPair@xercesc_2_3@@@2@IPAVXMLElementDecl@2@AAV?$RefVectorOf@VXMLAttr@xercesc_2_3@@@2@@Z 1204d990 f   SGXMLScanner.obj
 0001:0004d730       ?normalizeAttValue@SGXMLScanner@xercesc_2_3@@AAE_NQBVXMLAttDef@2@QBGAAVXMLBuffer@2@@Z 1204e730 f   SGXMLScanner.obj
 0001:0004d9e0       ?normalizeAttRawValue@SGXMLScanner@xercesc_2_3@@AAE_NQBG0AAVXMLBuffer@2@@Z 1204e9e0 f   SGXMLScanner.obj
 0001:0004d9e0       ?normalizeAttRawValue@IGXMLScanner@xercesc_2_3@@AAE_NQBG0AAVXMLBuffer@2@@Z 1204e9e0 f   SGXMLScanner.obj
 0001:0004dab0       ?resolvePrefix@IGXMLScanner@xercesc_2_3@@AAEIQBGAAVXMLBuffer@2@W4MapModes@ElemStack@2@@Z 1204eab0 f   SGXMLScanner.obj
 0001:0004dab0       ?resolvePrefix@SGXMLScanner@xercesc_2_3@@AAEIQBGAAVXMLBuffer@2@W4MapModes@ElemStack@2@@Z 1204eab0 f   SGXMLScanner.obj
 0001:0004dbb0       ?scanReset@SGXMLScanner@xercesc_2_3@@EAEXABVInputSource@2@@Z 1204ebb0 f   SGXMLScanner.obj
 0001:0004de50       ?sendCharData@SGXMLScanner@xercesc_2_3@@EAEXAAVXMLBuffer@2@@Z 1204ee50 f   SGXMLScanner.obj
 0001:0004e240       ?updateNSMap@SGXMLScanner@xercesc_2_3@@AAEXQBG0@Z 1204f240 f   SGXMLScanner.obj
 0001:0004e530       ?scanRawAttrListforNameSpaces@SGXMLScanner@xercesc_2_3@@AAEXPBV?$RefVectorOf@VKVStringPair@xercesc_2_3@@@2@H@Z 1204f530 f   SGXMLScanner.obj
 0001:0004eab0       ?parseSchemaLocation@SGXMLScanner@xercesc_2_3@@AAEXQBG@Z 1204fab0 f   SGXMLScanner.obj
 0001:0004eb70       ?resolveSchemaGrammar@SGXMLScanner@xercesc_2_3@@AAEXQBG0@Z 1204fb70 f   SGXMLScanner.obj
 0001:0004f180       ?resolveSystemId@SGXMLScanner@xercesc_2_3@@AAEPAVInputSource@2@QBG@Z 12050180 f   SGXMLScanner.obj
 0001:0004f3f0       ?loadXMLSchemaGrammar@SGXMLScanner@xercesc_2_3@@AAEPAVGrammar@2@ABVInputSource@2@_N@Z 120503f0 f   SGXMLScanner.obj
 0001:0004f620       ?basicAttrValueScan@SGXMLScanner@xercesc_2_3@@AAE_NQBGAAVXMLBuffer@2@@Z 12050620 f   SGXMLScanner.obj
 0001:0004f8c0       ?scanCDSection@SGXMLScanner@xercesc_2_3@@EAEXXZ 120508c0 f   SGXMLScanner.obj
 0001:0004fc60       ?scanCharData@SGXMLScanner@xercesc_2_3@@EAEXAAVXMLBuffer@2@@Z 12050c60 f   SGXMLScanner.obj
 0001:0004ffb0       ?scanEntityRef@SGXMLScanner@xercesc_2_3@@EAE?AW4EntityExpRes@XMLScanner@2@_NAAG1AA_N@Z 12050fb0 f   SGXMLScanner.obj
 0001:000502e0       ?switchGrammar@SGXMLScanner@xercesc_2_3@@AAE_NQBG@Z 120512e0 f   SGXMLScanner.obj
 0001:00050370       ?laxElementValidation@SGXMLScanner@xercesc_2_3@@AAE_NPAVQName@2@PAVContentLeafNameTypeVector@2@QBVXMLContentModel@2@I@Z 12051370 f   SGXMLScanner.obj
 0001:000505a0       ?anyAttributeValidation@SGXMLScanner@xercesc_2_3@@AAE_NPAVSchemaAttDef@2@IAA_N1@Z 120515a0 f   SGXMLScanner.obj
 0001:00050690       ?put@?$ValueHashTableOf@G@xercesc_2_3@@QAEXPAXABG@Z 12051690 f i SGXMLScanner.obj
 0001:00050790       ?findBucketElem@?$ValueHashTableOf@G@xercesc_2_3@@ABEPBU?$ValueHashTableBucketElem@G@2@QBXAAI@Z 12051790 f i SGXMLScanner.obj
 0001:00050810       ?findBucketElem@?$ValueHashTableOf@G@xercesc_2_3@@AAEPAU?$ValueHashTableBucketElem@G@2@QBXAAI@Z 12051810 f i SGXMLScanner.obj
 0001:00050890       ??0Attributes@xercesc_2_3@@QAE@XZ 12051890 f i VecAttributesImpl.obj
 0001:000508a0       ??1Attributes@xercesc_2_3@@UAE@XZ 120518a0 f i VecAttributesImpl.obj
 0001:000508b0       ??_EAttributes@xercesc_2_3@@UAEPAXI@Z 120518b0 f i VecAttributesImpl.obj
 0001:00050910       ??0VecAttributesImpl@xercesc_2_3@@QAE@XZ 12051910 f   VecAttributesImpl.obj
 0001:00050930       ??_EVecAttributesImpl@xercesc_2_3@@UAEPAXI@Z 12051930 f i VecAttributesImpl.obj
 0001:00050990       ??1VecAttributesImpl@xercesc_2_3@@UAE@XZ 12051990 f   VecAttributesImpl.obj
 0001:000509f0       ?getURI@VecAttributesImpl@xercesc_2_3@@UBEPBGI@Z 120519f0 f   VecAttributesImpl.obj
 0001:00050a50       ?getLocalName@VecAttributesImpl@xercesc_2_3@@UBEPBGI@Z 12051a50 f   VecAttributesImpl.obj
 0001:00050ab0       ?getValue@VecAttributesImpl@xercesc_2_3@@UBEPBGI@Z 12051ab0 f   VecAttributesImpl.obj
 0001:00050ab0       ?getValue@VecAttrListImpl@xercesc_2_3@@UBEPBGI@Z 12051ab0 f   VecAttributesImpl.obj
 0001:00050b10       ?getIndex@VecAttributesImpl@xercesc_2_3@@UBEHQBG0@Z 12051b10 f   VecAttributesImpl.obj
 0001:00050cd0       ?getIndex@VecAttributesImpl@xercesc_2_3@@UBEHQBG@Z 12051cd0 f   VecAttributesImpl.obj
 0001:00050d80       ?getType@VecAttributesImpl@xercesc_2_3@@UBEPBGQBG0@Z 12051d80 f   VecAttributesImpl.obj
 0001:00050db0       ?getType@VecAttributesImpl@xercesc_2_3@@UBEPBGQBG@Z 12051db0 f   VecAttributesImpl.obj
 0001:00050de0       ?getValue@VecAttributesImpl@xercesc_2_3@@UBEPBGQBG0@Z 12051de0 f   VecAttributesImpl.obj
 0001:00050e10       ?getValue@VecAttributesImpl@xercesc_2_3@@UBEPBGQBG@Z 12051e10 f   VecAttributesImpl.obj
 0001:00050e40       ?setVector@VecAttributesImpl@xercesc_2_3@@QAEXQBV?$RefVectorOf@VXMLAttr@xercesc_2_3@@@2@IQBVXMLScanner@2@_N@Z 12051e40 f   VecAttributesImpl.obj
 0001:00050e80       ??0AttributeList@xercesc_2_3@@QAE@XZ 12051e80 f i VecAttrListImpl.obj
 0001:00050e90       ??1AttributeList@xercesc_2_3@@UAE@XZ 12051e90 f i VecAttrListImpl.obj
 0001:00050ea0       ??_EAttributeList@xercesc_2_3@@UAEPAXI@Z 12051ea0 f i VecAttrListImpl.obj
 0001:00050f00       ??0VecAttrListImpl@xercesc_2_3@@QAE@XZ 12051f00 f   VecAttrListImpl.obj
 0001:00050f20       ??_EVecAttrListImpl@xercesc_2_3@@UAEPAXI@Z 12051f20 f i VecAttrListImpl.obj
 0001:00050f80       ??1VecAttrListImpl@xercesc_2_3@@UAE@XZ 12051f80 f   VecAttrListImpl.obj
 0001:00050fe0       ?getQName@VecAttributesImpl@xercesc_2_3@@UBEPBGI@Z 12051fe0 f   VecAttrListImpl.obj
 0001:00050fe0       ?getName@VecAttrListImpl@xercesc_2_3@@UBEPBGI@Z 12051fe0 f   VecAttrListImpl.obj
 0001:00051040       ?getType@VecAttributesImpl@xercesc_2_3@@UBEPBGI@Z 12052040 f   VecAttrListImpl.obj
 0001:00051040       ?getType@VecAttrListImpl@xercesc_2_3@@UBEPBGI@Z 12052040 f   VecAttrListImpl.obj
 0001:000510a0       ?getType@VecAttrListImpl@xercesc_2_3@@UBEPBGQBG@Z 120520a0 f   VecAttrListImpl.obj
 0001:00051160       ?getValue@VecAttrListImpl@xercesc_2_3@@UBEPBGQBG@Z 12052160 f   VecAttrListImpl.obj
 0001:00051210       ?getValue@VecAttrListImpl@xercesc_2_3@@UBEPBGQBD@Z 12052210 f   VecAttrListImpl.obj
 0001:00051370       ?setVector@VecAttrListImpl@xercesc_2_3@@QAEXQBV?$RefVectorOf@VXMLAttr@xercesc_2_3@@@2@I_N@Z 12052370 f   VecAttrListImpl.obj
 0001:000513a0       ?getName@WFXMLScanner@xercesc_2_3@@UBEPBGXZ 120523a0 f i WFXMLScanner.obj
 0001:000513b0       ??0WFXMLScanner@xercesc_2_3@@QAE@QAVXMLValidator@1@QAVMemoryManager@1@@Z 120523b0 f   WFXMLScanner.obj
 0001:00051580       ??_EWFXMLScanner@xercesc_2_3@@UAEPAXI@Z 12052580 f i WFXMLScanner.obj
 0001:000515e0       ??0WFXMLScanner@xercesc_2_3@@QAE@QAVXMLDocumentHandler@1@QAVDocTypeHandler@1@QAVXMLEntityHandler@1@QAVXMLErrorReporter@1@QAVXMLValidator@1@QAVMemoryManager@1@@Z 120525e0 f   WFXMLScanner.obj
 0001:000517c0       ??1WFXMLScanner@xercesc_2_3@@UAE@XZ 120527c0 f   WFXMLScanner.obj
 0001:00051950       ?scanDocument@WFXMLScanner@xercesc_2_3@@UAEXABVInputSource@2@@Z 12052950 f   WFXMLScanner.obj
 0001:00051b00       ?scanNext@WFXMLScanner@xercesc_2_3@@UAE_NAAVXMLPScanToken@2@@Z 12052b00 f   WFXMLScanner.obj
 0001:00051e40       ?commonInit@WFXMLScanner@xercesc_2_3@@AAEXXZ 12052e40 f   WFXMLScanner.obj
 0001:000521e0       ?cleanUp@WFXMLScanner@xercesc_2_3@@AAEXXZ 120531e0 f   WFXMLScanner.obj
 0001:00052320       ?resolvePrefix@WFXMLScanner@xercesc_2_3@@AAEIQBGW4MapModes@ElemStack@2@@Z 12053320 f   WFXMLScanner.obj
 0001:00052410       ?scanReset@WFXMLScanner@xercesc_2_3@@EAEXABVInputSource@2@@Z 12053410 f   WFXMLScanner.obj
 0001:00052580       ?sendCharData@WFXMLScanner@xercesc_2_3@@EAEXAAVXMLBuffer@2@@Z 12053580 f   WFXMLScanner.obj
 0001:000525c0       ?scanContent@WFXMLScanner@xercesc_2_3@@AAE_N_N@Z 120535c0 f   WFXMLScanner.obj
 0001:00052780       ?scanEndTag@WFXMLScanner@xercesc_2_3@@AAEXAA_N@Z 12053780 f   WFXMLScanner.obj
 0001:00052900       ?scanDocTypeDecl@WFXMLScanner@xercesc_2_3@@EAEXXZ 12053900 f   WFXMLScanner.obj
 0001:00052940       ?scanStartTag@WFXMLScanner@xercesc_2_3@@AAE_NAA_N@Z 12053940 f   WFXMLScanner.obj
 0001:000532e0       ?scanStartTagNS@WFXMLScanner@xercesc_2_3@@AAE_NAA_N@Z 120542e0 f   WFXMLScanner.obj
 0001:00054170       ?resolveQName@WFXMLScanner@xercesc_2_3@@UAEIQBGAAVXMLBuffer@2@FAAH@Z 12055170 f   WFXMLScanner.obj
 0001:00054300       ?scanAttValue@WFXMLScanner@xercesc_2_3@@AAE_NQBGAAVXMLBuffer@2@@Z 12055300 f   WFXMLScanner.obj
 0001:000545d0       ?scanCDSection@WFXMLScanner@xercesc_2_3@@EAEXXZ 120555d0 f   WFXMLScanner.obj
 0001:00054800       ?scanCharData@WFXMLScanner@xercesc_2_3@@EAEXAAVXMLBuffer@2@@Z 12055800 f   WFXMLScanner.obj
 0001:00054ae0       ?scanEntityRef@WFXMLScanner@xercesc_2_3@@EAE?AW4EntityExpRes@XMLScanner@2@_NAAG1AA_N@Z 12055ae0 f   WFXMLScanner.obj
 0001:00054e10       ?loadGrammar@WFXMLScanner@xercesc_2_3@@UAEPAVGrammar@2@ABVInputSource@2@F_N@Z 12055e10 f   WFXMLScanner.obj
 0001:00054e20       ??_G?$RefVectorOf@VXMLElementDecl@xercesc_2_3@@@xercesc_2_3@@UAEPAXI@Z 12055e20 f i WFXMLScanner.obj
 0001:00054e20       ??_E?$RefVectorOf@VXMLElementDecl@xercesc_2_3@@@xercesc_2_3@@UAEPAXI@Z 12055e20 f i WFXMLScanner.obj
 0001:00054e40       ??1?$RefVectorOf@VXMLElementDecl@xercesc_2_3@@@xercesc_2_3@@UAE@XZ 12055e40 f i WFXMLScanner.obj
 0001:00054ec0       ??1?$BaseRefVectorOf@VXMLElementDecl@xercesc_2_3@@@xercesc_2_3@@UAE@XZ 12055ec0 f i WFXMLScanner.obj
 0001:00054ed0       ??0?$ValueHashTableBucketElem@G@xercesc_2_3@@QAE@PAXABGPAU01@@Z 12055ed0 f i WFXMLScanner.obj
 0001:00054ef0       ?ensureExtraCapacity@?$ValueVectorOf@PAVQName@xercesc_2_3@@@xercesc_2_3@@QAEXI@Z 12055ef0 f i WFXMLScanner.obj
 0001:00054ef0       ?ensureExtraCapacity@?$ValueVectorOf@PAVSchemaElementDecl@xercesc_2_3@@@xercesc_2_3@@QAEXI@Z 12055ef0 f i WFXMLScanner.obj
 0001:00054ef0       ?ensureExtraCapacity@?$ValueVectorOf@PAVDOMElement@xercesc_2_3@@@xercesc_2_3@@QAEXI@Z 12055ef0 f i WFXMLScanner.obj
 0001:00054ef0       ?ensureExtraCapacity@?$ValueVectorOf@PAVXercesAttGroupInfo@xercesc_2_3@@@xercesc_2_3@@QAEXI@Z 12055ef0 f i WFXMLScanner.obj
 0001:00054ef0       ?ensureExtraCapacity@?$ValueVectorOf@PAG@xercesc_2_3@@QAEXI@Z 12055ef0 f i WFXMLScanner.obj
 0001:00054ef0       ?ensureExtraCapacity@?$ValueVectorOf@PBVDOMElement@xercesc_2_3@@@xercesc_2_3@@QAEXI@Z 12055ef0 f i WFXMLScanner.obj
 0001:00054ef0       ?ensureExtraCapacity@?$ValueVectorOf@PAVIC_Field@xercesc_2_3@@@xercesc_2_3@@QAEXI@Z 12055ef0 f i WFXMLScanner.obj
 0001:00054ef0       ?ensureExtraCapacity@?$ValueVectorOf@PAVDatatypeValidator@xercesc_2_3@@@xercesc_2_3@@QAEXI@Z 12055ef0 f i WFXMLScanner.obj
 0001:00054ef0       ?ensureExtraCapacity@?$ValueVectorOf@H@xercesc_2_3@@QAEXI@Z 12055ef0 f i WFXMLScanner.obj
 0001:00054ef0       ?ensureExtraCapacity@?$ValueVectorOf@PAVComplexTypeInfo@xercesc_2_3@@@xercesc_2_3@@QAEXI@Z 12055ef0 f i WFXMLScanner.obj
 0001:00054ef0       ?ensureExtraCapacity@?$ValueVectorOf@PAVXMLAttr@xercesc_2_3@@@xercesc_2_3@@QAEXI@Z 12055ef0 f i WFXMLScanner.obj
 0001:00054ef0       ?ensureExtraCapacity@?$ValueVectorOf@I@xercesc_2_3@@QAEXI@Z 12055ef0 f i WFXMLScanner.obj
 0001:00054f80       ??0?$BaseRefVectorOf@VXMLElementDecl@xercesc_2_3@@@xercesc_2_3@@QAE@I_NQAVMemoryManager@1@@Z 12055f80 f i WFXMLScanner.obj
 0001:00054fe0       ?isAllSpaces@XMLReader@xercesc_2_3@@QAE_NQBGI@Z 12055fe0 f   XMLReader.obj
 0001:00055020       ?containsWhiteSpace@XMLReader@xercesc_2_3@@QAE_NQBGI@Z 12056020 f   XMLReader.obj
 0001:00055060       ?isPublicIdChar@XMLReader@xercesc_2_3@@QAE_NG@Z 12056060 f   XMLReader.obj
 0001:00055090       ??0XMLReader@xercesc_2_3@@QAE@QBG0QAVBinInputStream@1@W4RefFrom@01@W4Types@01@W4Sources@01@_N5W4XMLVersion@01@QAVMemoryManager@1@@Z 12056090 f   XMLReader.obj
 0001:00055310       ??0XMLReader@xercesc_2_3@@QAE@QBG0QAVBinInputStream@1@0W4RefFrom@01@W4Types@01@W4Sources@01@_N5W4XMLVersion@01@QAVMemoryManager@1@@Z 12056310 f   XMLReader.obj
 0001:00055640       ??0XMLReader@xercesc_2_3@@QAE@QBG0QAVBinInputStream@1@W4Encodings@XMLRecognizer@1@W4RefFrom@01@W4Types@01@W4Sources@01@_N6W4XMLVersion@01@QAVMemoryManager@1@@Z 12056640 f   XMLReader.obj
 0001:00055940       ??1XMLReader@xercesc_2_3@@QAE@XZ 12056940 f   XMLReader.obj
 0001:00055990       ?getSrcOffset@XMLReader@xercesc_2_3@@QBEIXZ 12056990 f   XMLReader.obj
 0001:00055a00       ?refreshCharBuffer@XMLReader@xercesc_2_3@@QAE_NXZ 12056a00 f   XMLReader.obj
 0001:00055c90       ?getName@XMLReader@xercesc_2_3@@QAE_NAAVXMLBuffer@2@_N@Z 12056c90 f   XMLReader.obj
 0001:00055e90       ?getSpaces@XMLReader@xercesc_2_3@@QAE_NAAVXMLBuffer@2@@Z 12056e90 f   XMLReader.obj
 0001:00055fc0       ?getUpToCharOrWS@XMLReader@xercesc_2_3@@QAE_NAAVXMLBuffer@2@G@Z 12056fc0 f   XMLReader.obj
 0001:00056100       ?skipIfQuote@XMLReader@xercesc_2_3@@QAE_NAAG@Z 12057100 f   XMLReader.obj
 0001:00056160       ?skipSpaces@XMLReader@xercesc_2_3@@QAE_NAA_N@Z 12057160 f   XMLReader.obj
 0001:000562e0       ?skippedChar@XMLReader@xercesc_2_3@@QAE_NG@Z 120572e0 f   XMLReader.obj
 0001:00056320       ?skippedSpace@XMLReader@xercesc_2_3@@QAE_NXZ 12057320 f   XMLReader.obj
 0001:00056410       ?skippedString@XMLReader@xercesc_2_3@@QAE_NQBG@Z 12057410 f   XMLReader.obj
 0001:000564b0       ?peekString@XMLReader@xercesc_2_3@@QAE_NQBG@Z 120574b0 f   XMLReader.obj
 0001:00056530       ?setEncoding@XMLReader@xercesc_2_3@@QAE_NQBG@Z 12057530 f   XMLReader.obj
 0001:00056930       ?checkForSwapped@XMLReader@xercesc_2_3@@AAEXXZ 12057930 f   XMLReader.obj
 0001:00056950       ?doInitDecode@XMLReader@xercesc_2_3@@AAEXXZ 12057950 f   XMLReader.obj
 0001:00056d70       ?refreshRawBuffer@XMLReader@xercesc_2_3@@AAEXXZ 12057d70 f   XMLReader.obj
 0001:00056de0       ?xcodeMoreChars@XMLReader@xercesc_2_3@@AAEIQAGQAEI@Z 12057de0 f   XMLReader.obj
 0001:00056ef0       ?reinitMsgLoader@XMLScanner@xercesc_2_3@@SAXXZ 12057ef0 f   XMLScanner.obj
 0001:00056f10       ?reinitScannerMutex@XMLScanner@xercesc_2_3@@SAXXZ 12057f10 f   XMLScanner.obj
 0001:00056f40       ??0XMLScanner@xercesc_2_3@@QAE@QAVXMLValidator@1@QAVMemoryManager@1@@Z 12057f40 f   XMLScanner.obj
 0001:000571d0       ??_EXMLScanner@xercesc_2_3@@UAEPAXI@Z 120581d0 f i XMLScanner.obj
 0001:00057230       ??0XMLScanner@xercesc_2_3@@QAE@QAVXMLDocumentHandler@1@QAVDocTypeHandler@1@QAVXMLEntityHandler@1@QAVXMLErrorReporter@1@QAVXMLValidator@1@QAVMemoryManager@1@@Z 12058230 f   XMLScanner.obj
 0001:000574e0       ??1XMLScanner@xercesc_2_3@@UAE@XZ 120584e0 f   XMLScanner.obj
 0001:00057640       ?setValidator@XMLScanner@xercesc_2_3@@QAEXQAVXMLValidator@2@@Z 12058640 f   XMLScanner.obj
 0001:00057690       ?scanDocument@XMLScanner@xercesc_2_3@@QAEXQBG@Z 12058690 f   XMLScanner.obj
 0001:000579b0       ?scanDocument@XMLScanner@xercesc_2_3@@QAEXQBD@Z 120589b0 f   XMLScanner.obj
 0001:00057a50       ?scanFirst@XMLScanner@xercesc_2_3@@QAE_NQBGAAVXMLPScanToken@2@@Z 12058a50 f   XMLScanner.obj
 0001:00057d70       ?scanFirst@XMLScanner@xercesc_2_3@@QAE_NQBDAAVXMLPScanToken@2@@Z 12058d70 f   XMLScanner.obj
 0001:00057e10       ?scanFirst@XMLScanner@xercesc_2_3@@QAE_NABVInputSource@2@AAVXMLPScanToken@2@@Z 12058e10 f   XMLScanner.obj
 0001:00057fa0       ?scanReset@XMLScanner@xercesc_2_3@@QAEXAAVXMLPScanToken@2@@Z 12058fa0 f   XMLScanner.obj
 0001:00058000       ?setParseSettings@XMLScanner@xercesc_2_3@@QAEXQAV12@@Z 12059000 f   XMLScanner.obj
 0001:00058170       ?commonInit@XMLScanner@xercesc_2_3@@AAEXXZ 12059170 f   XMLScanner.obj
 0001:000583f0       ?initValidator@XMLScanner@xercesc_2_3@@IAEXPAVXMLValidator@2@@Z 120593f0 f   XMLScanner.obj
 0001:00058410       ?emitError@XMLScanner@xercesc_2_3@@QAEXW4Codes@XMLErrs@2@@Z 12059410 f   XMLScanner.obj
 0001:000586c0       ?emitError@XMLScanner@xercesc_2_3@@QAEXW4Codes@XMLErrs@2@QBG111@Z 120596c0 f   XMLScanner.obj
 0001:000587e0       ?emitError@XMLScanner@xercesc_2_3@@QAEXW4Codes@XMLErrs@2@QBD111@Z 120597e0 f   XMLScanner.obj
 0001:00058900       ?scanMiscellaneous@XMLScanner@xercesc_2_3@@IAEXXZ 12059900 f   XMLScanner.obj
 0001:00058ab0       ?scanPI@XMLScanner@xercesc_2_3@@IAEXXZ 12059ab0 f   XMLScanner.obj
 0001:00058e10       ?scanProlog@XMLScanner@xercesc_2_3@@IAEXXZ 12059e10 f   XMLScanner.obj
 0001:00059010       ?scanXMLDecl@XMLScanner@xercesc_2_3@@IAEXW4DeclTypes@12@@Z 1205a010 f   XMLScanner.obj
 0001:000598c0       ?getURIText@XMLScanner@xercesc_2_3@@QBEPBGI@Z 1205a8c0 f   XMLScanner.obj
 0001:00059900       ?getURIText@XMLScanner@xercesc_2_3@@QBE_NIAAVXMLBuffer@2@@Z 1205a900 f   XMLScanner.obj
 0001:00059950       ?checkXMLDecl@XMLScanner@xercesc_2_3@@QAE_N_N@Z 1205a950 f   XMLScanner.obj
 0001:00059ad0       ?loadGrammar@XMLScanner@xercesc_2_3@@QAEPAVGrammar@2@QBGF_N@Z 1205aad0 f   XMLScanner.obj
 0001:00059e10       ?loadGrammar@XMLScanner@xercesc_2_3@@QAEPAVGrammar@2@QBDF_N@Z 1205ae10 f   XMLScanner.obj
 0001:00059eb0       ?setURIStringPool@XMLScanner@xercesc_2_3@@QAEXQAVXMLStringPool@2@@Z 1205aeb0 f   XMLScanner.obj
 0001:00059f10       ?checkIDRefs@XMLScanner@xercesc_2_3@@IAEXXZ 1205af10 f   XMLScanner.obj
 0001:0005a0e0       ?isLegalToken@XMLScanner@xercesc_2_3@@IAE_NABVXMLPScanToken@2@@Z 1205b0e0 f   XMLScanner.obj
 0001:0005a100       ?senseNextToken@XMLScanner@xercesc_2_3@@IAE?AW4XMLTokens@12@AAI@Z 1205b100 f   XMLScanner.obj
 0001:0005a290       ?getQuotedString@XMLScanner@xercesc_2_3@@AAE_NAAVXMLBuffer@2@@Z 1205b290 f   XMLScanner.obj
 0001:0005a300       ?scanCharRef@XMLScanner@xercesc_2_3@@IAE_NAAG0@Z 1205b300 f   XMLScanner.obj
 0001:0005a540       ?scanComment@XMLScanner@xercesc_2_3@@IAEXXZ 1205b540 f   XMLScanner.obj
 0001:0005a7b0       ?scanEq@XMLScanner@xercesc_2_3@@IAE_NXZ 1205b7b0 f   XMLScanner.obj
 0001:0005a7e0       ?scanUpToWSOr@XMLScanner@xercesc_2_3@@AAEIAAVXMLBuffer@2@G@Z 1205b7e0 f   XMLScanner.obj
 0001:0005a800       ??1?$XMLEnumerator@VXMLRefInfo@xercesc_2_3@@@xercesc_2_3@@UAE@XZ 1205b800 f i XMLScanner.obj
 0001:0005a810       ??_G?$XMLEnumerator@VXMLRefInfo@xercesc_2_3@@@xercesc_2_3@@UAEPAXI@Z 1205b810 f i XMLScanner.obj
 0001:0005a810       ??_E?$XMLEnumerator@VXMLRefInfo@xercesc_2_3@@@xercesc_2_3@@UAEPAXI@Z 1205b810 f i XMLScanner.obj
 0001:0005a830       ??1?$RefHashTableOfEnumerator@VXMLRefInfo@xercesc_2_3@@@xercesc_2_3@@UAE@XZ 1205b830 f i XMLScanner.obj
 0001:0005a920       ??_G?$RefVectorOf@VXMLAttr@xercesc_2_3@@@xercesc_2_3@@UAEPAXI@Z 1205b920 f i XMLScanner.obj
 0001:0005a920       ??_E?$RefVectorOf@VXMLAttr@xercesc_2_3@@@xercesc_2_3@@UAEPAXI@Z 1205b920 f i XMLScanner.obj
 0001:0005a940       ??1?$RefVectorOf@VXMLAttr@xercesc_2_3@@@xercesc_2_3@@UAE@XZ 1205b940 f i XMLScanner.obj
 0001:0005a9d0       ??1?$BaseRefVectorOf@VXMLAttr@xercesc_2_3@@@xercesc_2_3@@UAE@XZ 1205b9d0 f i XMLScanner.obj
 0001:0005a9e0       ??_G?$RefHashTableOfEnumerator@VXMLRefInfo@xercesc_2_3@@@xercesc_2_3@@UAEPAXI@Z 1205b9e0 f i XMLScanner.obj
 0001:0005a9e0       ??_E?$RefHashTableOfEnumerator@VXMLRefInfo@xercesc_2_3@@@xercesc_2_3@@UAEPAXI@Z 1205b9e0 f i XMLScanner.obj
 0001:0005aa00       ?removeAll@?$RefHashTableOf@VXMLRefInfo@xercesc_2_3@@@xercesc_2_3@@QAEXXZ 1205ba00 f i XMLScanner.obj
 0001:0005aa90       ?findNext@?$RefHashTableOfEnumerator@VValueStore@xercesc_2_3@@@xercesc_2_3@@AAEXXZ 1205ba90 f i XMLScanner.obj
 0001:0005aa90       ?findNext@?$RefHashTableOfEnumerator@V?$KeyRefPair@XVDOMUserDataHandler@xercesc_2_3@@@xercesc_2_3@@@xercesc_2_3@@AAEXXZ 1205ba90 f i XMLScanner.obj
 0001:0005aa90       ?findNext@?$RefHashTableOfEnumerator@VKVStringPair@xercesc_2_3@@@xercesc_2_3@@AAEXXZ 1205ba90 f i XMLScanner.obj
 0001:0005aa90       ?findNext@?$RefHashTableOfEnumerator@VXercesGroupInfo@xercesc_2_3@@@xercesc_2_3@@AAEXXZ 1205ba90 f i XMLScanner.obj
 0001:0005aa90       ?findNext@?$RefHashTableOfEnumerator@VGrammar@xercesc_2_3@@@xercesc_2_3@@AAEXXZ 1205ba90 f i XMLScanner.obj
 0001:0005aa90       ?findNext@?$RefHashTableOfEnumerator@VComplexTypeInfo@xercesc_2_3@@@xercesc_2_3@@AAEXXZ 1205ba90 f i XMLScanner.obj
 0001:0005aa90       ?findNext@?$RefHashTableOfEnumerator@VXMLRefInfo@xercesc_2_3@@@xercesc_2_3@@AAEXXZ 1205ba90 f i XMLScanner.obj
 0001:0005aa90       ?findNext@?$RefHash2KeysTableOfEnumerator@VSchemaAttDef@xercesc_2_3@@@xercesc_2_3@@AAEXXZ 1205ba90 f i XMLScanner.obj
 0001:0005aa90       ?findNext@?$RefHashTableOfEnumerator@G@xercesc_2_3@@AAEXXZ 1205ba90 f i XMLScanner.obj
 0001:0005aa90       ?findNext@?$RefHashTableOfEnumerator@VDTDAttDef@xercesc_2_3@@@xercesc_2_3@@AAEXXZ 1205ba90 f i XMLScanner.obj
 0001:0005aae0       ??_GXMLRefInfo@xercesc_2_3@@QAEPAXI@Z 1205bae0 f i XMLScanner.obj
 0001:0005ab10       ?getDefaultScanner@XMLScannerResolver@xercesc_2_3@@SAPAVXMLScanner@2@QAVXMLValidator@2@QAVMemoryManager@2@@Z 1205bb10 f   XMLScannerResolver.obj
 0001:0005ab80       ?resolveScanner@XMLScannerResolver@xercesc_2_3@@SAPAVXMLScanner@2@QBGQAVXMLValidator@2@QAVMemoryManager@2@@Z 1205bb80 f   XMLScannerResolver.obj
 0001:0005ae30       ?resolveScanner@XMLScannerResolver@xercesc_2_3@@SAPAVXMLScanner@2@QBGQAVXMLDocumentHandler@2@QAVDocTypeHandler@2@QAVXMLEntityHandler@2@QAVXMLErrorReporter@2@QAVXMLValidator@2@QAVMemoryManager@2@@Z 1205be30 f   XMLScannerResolver.obj
 0001:0005b130       ??0DocumentHandler@xercesc_2_3@@QAE@XZ 1205c130 f i Dummy.obj
 0001:0005b140       ??1DocumentHandler@xercesc_2_3@@UAE@XZ 1205c140 f i Dummy.obj
 0001:0005b150       ??_EDocumentHandler@xercesc_2_3@@UAEPAXI@Z 1205c150 f i Dummy.obj
 0001:0005b1b0       ??0DTDHandler@xercesc_2_3@@QAE@XZ 1205c1b0 f i Dummy.obj
 0001:0005b1c0       ??1DTDHandler@xercesc_2_3@@UAE@XZ 1205c1c0 f i Dummy.obj
 0001:0005b1d0       ??_EDTDHandler@xercesc_2_3@@UAEPAXI@Z 1205c1d0 f i Dummy.obj
 0001:0005b230       ??0EntityResolver@xercesc_2_3@@QAE@XZ 1205c230 f i Dummy.obj
 0001:0005b240       ??1EntityResolver@xercesc_2_3@@UAE@XZ 1205c240 f i Dummy.obj
 0001:0005b250       ??_EEntityResolver@xercesc_2_3@@UAEPAXI@Z 1205c250 f i Dummy.obj
 0001:0005b2b0       ??0ErrorHandler@xercesc_2_3@@QAE@XZ 1205c2b0 f i Dummy.obj
 0001:0005b2c0       ??1ErrorHandler@xercesc_2_3@@UAE@XZ 1205c2c0 f i Dummy.obj
 0001:0005b2d0       ??_EErrorHandler@xercesc_2_3@@UAEPAXI@Z 1205c2d0 f i Dummy.obj
 0001:0005b330       ??0SAXException@xercesc_2_3@@QAE@XZ 1205c330 f i Dummy.obj
 0001:0005b3a0       ??0SAXException@xercesc_2_3@@QAE@QBG@Z 1205c3a0 f i Dummy.obj
 0001:0005b400       ??0SAXException@xercesc_2_3@@QAE@QBD@Z 1205c400 f i Dummy.obj
 0001:0005b420       ??0SAXException@xercesc_2_3@@QAE@ABV01@@Z 1205c420 f i Dummy.obj
 0001:0005b490       ??4SAXException@xercesc_2_3@@QAEAAV01@ABV01@@Z 1205c490 f i Dummy.obj
 0001:0005b490       ??4SAXNotRecognizedException@xercesc_2_3@@QAEAAV01@ABV01@@Z 1205c490 f i Dummy.obj
 0001:0005b490       ??4SAXNotSupportedException@xercesc_2_3@@QAEAAV01@ABV01@@Z 1205c490 f i Dummy.obj
 0001:0005b500       ??_ESAXException@xercesc_2_3@@UAEPAXI@Z 1205c500 f i Dummy.obj
 0001:0005b560       ??0SAXNotSupportedException@xercesc_2_3@@QAE@ABV01@@Z 1205c560 f i Dummy.obj
 0001:0005b5d0       ??0SAXNotRecognizedException@xercesc_2_3@@QAE@ABV01@@Z 1205c5d0 f i Dummy.obj
 0001:0005b640       ??1SAXNotRecognizedException@xercesc_2_3@@UAE@XZ 1205c640 f i Dummy.obj
 0001:0005b640       ??1SAXException@xercesc_2_3@@UAE@XZ 1205c640 f i Dummy.obj
 0001:0005b640       ??1SAXNotSupportedException@xercesc_2_3@@UAE@XZ 1205c640 f i Dummy.obj
 0001:0005b660       ??_ESAXNotRecognizedException@xercesc_2_3@@UAEPAXI@Z 1205c660 f i Dummy.obj
 0001:0005b660       ??_ESAXNotSupportedException@xercesc_2_3@@UAEPAXI@Z 1205c660 f i Dummy.obj
 0001:0005b6c0       ??0HandlerBase@xercesc_2_3@@QAE@XZ 1205c6c0 f i Dummy.obj
 0001:0005b700       ??1HandlerBase@xercesc_2_3@@UAE@XZ 1205c700 f i Dummy.obj
 0001:0005b750       ??_EHandlerBase@xercesc_2_3@@UAEPAXI@Z 1205c750 f i Dummy.obj
 0001:0005b7b0       ??0Parser@xercesc_2_3@@QAE@XZ 1205c7b0 f i Dummy.obj
 0001:0005b7c0       ??1Parser@xercesc_2_3@@UAE@XZ 1205c7c0 f i Dummy.obj
 0001:0005b7d0       ??_EParser@xercesc_2_3@@UAEPAXI@Z 1205c7d0 f i Dummy.obj
 0001:0005b830       ??_EHandlerBase@xercesc_2_3@@W3AEPAXI@Z 1205c830 f i Dummy.obj
 0001:0005b840       ??_EHandlerBase@xercesc_2_3@@W7AEPAXI@Z 1205c840 f i Dummy.obj
 0001:0005b850       ??_EHandlerBase@xercesc_2_3@@WM@AEPAXI@Z 1205c850 f i Dummy.obj
 0001:0005b860       ??1InputSource@xercesc_2_3@@UAE@XZ 1205c860 f   InputSource.obj
 0001:0005b890       ??_EInputSource@xercesc_2_3@@UAEPAXI@Z 1205c890 f i InputSource.obj
 0001:0005b910       ?setEncoding@InputSource@xercesc_2_3@@UAEXQBG@Z 1205c910 f   InputSource.obj
 0001:0005b980       ?setPublicId@InputSource@xercesc_2_3@@UAEXQBG@Z 1205c980 f   InputSource.obj
 0001:0005b9f0       ?setSystemId@InputSource@xercesc_2_3@@UAEXQBG@Z 1205c9f0 f   InputSource.obj
 0001:0005ba60       ??0InputSource@xercesc_2_3@@IAE@QAVMemoryManager@1@@Z 1205ca60 f   InputSource.obj
 0001:0005ba90       ??0InputSource@xercesc_2_3@@IAE@QBGQAVMemoryManager@1@@Z 1205ca90 f   InputSource.obj
 0001:0005bb10       ??0InputSource@xercesc_2_3@@IAE@QBG0QAVMemoryManager@1@@Z 1205cb10 f   InputSource.obj
 0001:0005bbe0       ??0InputSource@xercesc_2_3@@IAE@QBDQAVMemoryManager@1@@Z 1205cbe0 f   InputSource.obj
 0001:0005bc20       ??0InputSource@xercesc_2_3@@IAE@QBD0QAVMemoryManager@1@@Z 1205cc20 f   InputSource.obj
 0001:0005bc70       ??0SAXNotSupportedException@xercesc_2_3@@QAE@XZ 1205cc70 f   SAXException.obj
 0001:0005bce0       ??0SAXNotSupportedException@xercesc_2_3@@QAE@QBG@Z 1205cce0 f   SAXException.obj
 0001:0005bd40       ??0SAXNotSupportedException@xercesc_2_3@@QAE@QBD@Z 1205cd40 f   SAXException.obj
 0001:0005bd60       ??0SAXNotSupportedException@xercesc_2_3@@QAE@ABVSAXException@1@@Z 1205cd60 f   SAXException.obj
 0001:0005bdd0       ??0SAXNotRecognizedException@xercesc_2_3@@QAE@XZ 1205cdd0 f   SAXException.obj
 0001:0005be40       ??0SAXNotRecognizedException@xercesc_2_3@@QAE@QBG@Z 1205ce40 f   SAXException.obj
 0001:0005bea0       ??0SAXNotRecognizedException@xercesc_2_3@@QAE@QBD@Z 1205cea0 f   SAXException.obj
 0001:0005bec0       ??0SAXNotRecognizedException@xercesc_2_3@@QAE@ABVSAXException@1@@Z 1205cec0 f   SAXException.obj
 0001:0005bf30       ??0SAXParseException@xercesc_2_3@@QAE@QBGABVLocator@1@@Z 1205cf30 f   SAXParseException.obj
 0001:0005c090       ??_ESAXParseException@xercesc_2_3@@UAEPAXI@Z 1205d090 f i SAXParseException.obj
 0001:0005c0f0       ??0SAXParseException@xercesc_2_3@@QAE@QBG00JJ@Z 1205d0f0 f   SAXParseException.obj
 0001:0005c230       ??0SAXParseException@xercesc_2_3@@QAE@ABV01@@Z 1205d230 f   SAXParseException.obj
 0001:0005c370       ??1SAXParseException@xercesc_2_3@@UAE@XZ 1205d370 f   SAXParseException.obj
 0001:0005c3e0       ??4SAXParseException@xercesc_2_3@@QAEAAV01@ABV01@@Z 1205d3e0 f   SAXParseException.obj
 0001:0005c510       ??0DOMImplementationLS@xercesc_2_3@@IAE@XZ 1205d510 f i AbstractDOMParser.obj
 0001:0005c520       ??_EDOMImplementationLS@xercesc_2_3@@UAEPAXI@Z 1205d520 f i AbstractDOMParser.obj
 0001:0005c580       ??4DOMRangeException@xercesc_2_3@@QAEAAV01@ABV01@@Z 1205d580 f i AbstractDOMParser.obj
 0001:0005c5a0       ??0DOMImplementation@xercesc_2_3@@IAE@XZ 1205d5a0 f i AbstractDOMParser.obj
 0001:0005c5b0       ??1DOMImplementation@xercesc_2_3@@UAE@XZ 1205d5b0 f i AbstractDOMParser.obj
 0001:0005c5b0       ??1DOMImplementationLS@xercesc_2_3@@UAE@XZ 1205d5b0 f i AbstractDOMParser.obj
 0001:0005c5c0       ??_EDOMImplementation@xercesc_2_3@@UAEPAXI@Z 1205d5c0 f i AbstractDOMParser.obj
 0001:0005c620       ??0DOMNodeList@xercesc_2_3@@IAE@XZ 1205d620 f i AbstractDOMParser.obj
 0001:0005c630       ??1DOMNodeList@xercesc_2_3@@UAE@XZ 1205d630 f i AbstractDOMParser.obj
 0001:0005c640       ??_EDOMNodeList@xercesc_2_3@@UAEPAXI@Z 1205d640 f i AbstractDOMParser.obj
 0001:0005c6a0       ??1DOMParentNode@xercesc_2_3@@QAE@XZ 1205d6a0 f i AbstractDOMParser.obj
 0001:0005c6b0       ??0DOMUserDataHandler@xercesc_2_3@@IAE@XZ 1205d6b0 f i AbstractDOMParser.obj
 0001:0005c6c0       ??1DOMUserDataHandler@xercesc_2_3@@UAE@XZ 1205d6c0 f i AbstractDOMParser.obj
 0001:0005c6d0       ??_EDOMUserDataHandler@xercesc_2_3@@UAEPAXI@Z 1205d6d0 f i AbstractDOMParser.obj
 0001:0005c730       ?isReadOnly@DOMNodeImpl@xercesc_2_3@@QBE_NXZ 1205d730 f i AbstractDOMParser.obj
 0001:0005c750       ?isReadOnly@DOMNodeImpl@xercesc_2_3@@QAEX_N@Z 1205d750 f i AbstractDOMParser.obj
 0001:0005c790       ?needsSyncData@DOMNodeImpl@xercesc_2_3@@QBE_NXZ 1205d790 f i AbstractDOMParser.obj
 0001:0005c7b0       ?needsSyncData@DOMNodeImpl@xercesc_2_3@@QAEX_N@Z 1205d7b0 f i AbstractDOMParser.obj
 0001:0005c7f0       ?needsSyncChildren@DOMNodeImpl@xercesc_2_3@@QBE_NXZ 1205d7f0 f i AbstractDOMParser.obj
 0001:0005c810       ?needsSyncChildren@DOMNodeImpl@xercesc_2_3@@QAEX_N@Z 1205d810 f i AbstractDOMParser.obj
 0001:0005c850       ?isOwned@DOMNodeImpl@xercesc_2_3@@QBE_NXZ 1205d850 f i AbstractDOMParser.obj
 0001:0005c870       ?isOwned@DOMNodeImpl@xercesc_2_3@@QAEX_N@Z 1205d870 f i AbstractDOMParser.obj
 0001:0005c8b0       ?isFirstChild@DOMNodeImpl@xercesc_2_3@@QBE_NXZ 1205d8b0 f i AbstractDOMParser.obj
 0001:0005c8d0       ?isFirstChild@DOMNodeImpl@xercesc_2_3@@QAEX_N@Z 1205d8d0 f i AbstractDOMParser.obj
 0001:0005c910       ?isSpecified@DOMNodeImpl@xercesc_2_3@@QBE_NXZ 1205d910 f i AbstractDOMParser.obj
 0001:0005c930       ?isSpecified@DOMNodeImpl@xercesc_2_3@@QAEX_N@Z 1205d930 f i AbstractDOMParser.obj
 0001:0005c970       ?ignorableWhitespace@DOMNodeImpl@xercesc_2_3@@QBE_NXZ 1205d970 f i AbstractDOMParser.obj
 0001:0005c990       ?ignorableWhitespace@DOMNodeImpl@xercesc_2_3@@QAEX_N@Z 1205d990 f i AbstractDOMParser.obj
 0001:0005c9d0       ?setValue@DOMNodeImpl@xercesc_2_3@@QBE_NXZ 1205d9d0 f i AbstractDOMParser.obj
 0001:0005c9f0       ?setValue@DOMNodeImpl@xercesc_2_3@@QAEX_N@Z 1205d9f0 f i AbstractDOMParser.obj
 0001:0005ca30       ?isIdAttr@DOMNodeImpl@xercesc_2_3@@QBE_NXZ 1205da30 f i AbstractDOMParser.obj
 0001:0005ca50       ?isIdAttr@DOMNodeImpl@xercesc_2_3@@QAEX_N@Z 1205da50 f i AbstractDOMParser.obj
 0001:0005ca90       ?hasUserData@DOMNodeImpl@xercesc_2_3@@QBE_NXZ 1205da90 f i AbstractDOMParser.obj
 0001:0005cab0       ?hasUserData@DOMNodeImpl@xercesc_2_3@@QAEX_N@Z 1205dab0 f i AbstractDOMParser.obj
 0001:0005caf0       ?isLeafNode@DOMNodeImpl@xercesc_2_3@@QBE_NXZ 1205daf0 f i AbstractDOMParser.obj
 0001:0005cb10       ?setIsLeafNode@DOMNodeImpl@xercesc_2_3@@QAEX_N@Z 1205db10 f i AbstractDOMParser.obj
 0001:0005cb50       ?isChildNode@DOMNodeImpl@xercesc_2_3@@QBE_NXZ 1205db50 f i AbstractDOMParser.obj
 0001:0005cb70       ?setIsChildNode@DOMNodeImpl@xercesc_2_3@@QAEX_N@Z 1205db70 f i AbstractDOMParser.obj
 0001:0005cbb0       ?isToBeReleased@DOMNodeImpl@xercesc_2_3@@QBE_NXZ 1205dbb0 f i AbstractDOMParser.obj
 0001:0005cbd0       ?isToBeReleased@DOMNodeImpl@xercesc_2_3@@QAEX_N@Z 1205dbd0 f i AbstractDOMParser.obj
 0001:0005cc10       ?setErrorChecking@DOMDocumentImpl@xercesc_2_3@@QAEX_N@Z 1205dc10 f i AbstractDOMParser.obj
 0001:0005cc20       ?getErrorChecking@DOMDocumentImpl@xercesc_2_3@@QBE_NXZ 1205dc20 f i AbstractDOMParser.obj
 0001:0005cc30       ??_FDOMDocumentImpl@xercesc_2_3@@QAEXXZ 1205dc30 f i AbstractDOMParser.obj
 0001:0005cc40       ?getMemoryManager@DOMDocumentImpl@xercesc_2_3@@QBEPAVMemoryManager@2@XZ 1205dc40 f i AbstractDOMParser.obj
 0001:0005cc50       ??0DOMTypeInfo@xercesc_2_3@@IAE@XZ 1205dc50 f i AbstractDOMParser.obj
 0001:0005cc60       ??_EDOMTypeInfo@xercesc_2_3@@UAEPAXI@Z 1205dc60 f i AbstractDOMParser.obj
 0001:0005ccc0       ??_ODOMAttrImpl@xercesc_2_3@@QAEXABV01@@Z 1205dcc0 f i AbstractDOMParser.obj
 0001:0005ccd0       ?removeAttrFromIDNodeMap@DOMAttrImpl@xercesc_2_3@@UAEXXZ 1205dcd0 f i AbstractDOMParser.obj
 0001:0005cd00       ?addAttrToIDNodeMap@DOMAttrImpl@xercesc_2_3@@UAEXXZ 1205dd00 f i AbstractDOMParser.obj
 0001:0005cd90       ??0DOMCharacterData@xercesc_2_3@@IAE@XZ 1205dd90 f i AbstractDOMParser.obj
 0001:0005cda0       ??0DOMText@xercesc_2_3@@IAE@XZ 1205dda0 f i AbstractDOMParser.obj
 0001:0005cdb0       ??0DOMCDATASection@xercesc_2_3@@IAE@XZ 1205ddb0 f i AbstractDOMParser.obj
 0001:0005cdc0       ??0DOMComment@xercesc_2_3@@IAE@XZ 1205ddc0 f i AbstractDOMParser.obj
 0001:0005cdd0       ??_ODOMTextImpl@xercesc_2_3@@QAEXABV01@@Z 1205ddd0 f i AbstractDOMParser.obj
 0001:0005cde0       ??0DOMNamedNodeMap@xercesc_2_3@@IAE@XZ 1205dde0 f i AbstractDOMParser.obj
 0001:0005cdf0       ??1DOMNamedNodeMap@xercesc_2_3@@UAE@XZ 1205ddf0 f i AbstractDOMParser.obj
 0001:0005ce00       ??_EDOMNamedNodeMap@xercesc_2_3@@UAEPAXI@Z 1205de00 f i AbstractDOMParser.obj
 0001:0005ce60       ?hasDefaults@DOMAttrMapImpl@xercesc_2_3@@UAE_NXZ 1205de60 f i AbstractDOMParser.obj
 0001:0005ce60       ?getDoValidation@XMLScanner@xercesc_2_3@@QBE_NXZ 1205de60 f i AbstractDOMParser.obj
 0001:0005ce70       ?hasDefaults@DOMAttrMapImpl@xercesc_2_3@@UAEX_N@Z 1205de70 f i AbstractDOMParser.obj
 0001:0005ce80       ??_ODOMElementImpl@xercesc_2_3@@QAEXABV01@@Z 1205de80 f i AbstractDOMParser.obj
 0001:0005ce90       ??0DOMEntity@xercesc_2_3@@IAE@XZ 1205de90 f i AbstractDOMParser.obj
 0001:0005cea0       ??_ODOMEntityImpl@xercesc_2_3@@QAEXABV01@@Z 1205dea0 f i AbstractDOMParser.obj
 0001:0005ceb0       ??0DOMEntityReference@xercesc_2_3@@IAE@XZ 1205deb0 f i AbstractDOMParser.obj
 0001:0005cec0       ??_ODOMEntityReferenceImpl@xercesc_2_3@@QAEXABV01@@Z 1205dec0 f i AbstractDOMParser.obj
 0001:0005ced0       ??0DOMNotation@xercesc_2_3@@IAE@XZ 1205ded0 f i AbstractDOMParser.obj
 0001:0005cee0       ??_EDOMProcessingInstruction@xercesc_2_3@@UAEPAXI@Z 1205dee0 f i AbstractDOMParser.obj
 0001:0005cee0       ??_EDOMAttr@xercesc_2_3@@UAEPAXI@Z 1205dee0 f i AbstractDOMParser.obj
 0001:0005cee0       ??_EDOMCDATASection@xercesc_2_3@@UAEPAXI@Z 1205dee0 f i AbstractDOMParser.obj
 0001:0005cee0       ??_EDOMElement@xercesc_2_3@@UAEPAXI@Z 1205dee0 f i AbstractDOMParser.obj
 0001:0005cee0       ??_EDOMEntity@xercesc_2_3@@UAEPAXI@Z 1205dee0 f i AbstractDOMParser.obj
 0001:0005cee0       ??_EDOMDocumentType@xercesc_2_3@@UAEPAXI@Z 1205dee0 f i AbstractDOMParser.obj
 0001:0005cee0       ??_EDOMNotation@xercesc_2_3@@UAEPAXI@Z 1205dee0 f i AbstractDOMParser.obj
 0001:0005cee0       ??_EDOMEntityReference@xercesc_2_3@@UAEPAXI@Z 1205dee0 f i AbstractDOMParser.obj
 0001:0005cee0       ??_EDOMText@xercesc_2_3@@UAEPAXI@Z 1205dee0 f i AbstractDOMParser.obj
 0001:0005cee0       ??_EDOMComment@xercesc_2_3@@UAEPAXI@Z 1205dee0 f i AbstractDOMParser.obj
 0001:0005cee0       ??_EDOMDocumentFragment@xercesc_2_3@@UAEPAXI@Z 1205dee0 f i AbstractDOMParser.obj
 0001:0005cee0       ??_EDOMCharacterData@xercesc_2_3@@UAEPAXI@Z 1205dee0 f i AbstractDOMParser.obj
 0001:0005cf40       ??_ODOMNotationImpl@xercesc_2_3@@QAEXABV01@@Z 1205df40 f i AbstractDOMParser.obj
 0001:0005cf50       ??0DOMProcessingInstruction@xercesc_2_3@@IAE@XZ 1205df50 f i AbstractDOMParser.obj
 0001:0005cf60       ??_ODOMProcessingInstructionImpl@xercesc_2_3@@QAEXABV01@@Z 1205df60 f i AbstractDOMParser.obj
 0001:0005cf70       ??0AbstractDOMParser@xercesc_2_3@@IAE@QAVXMLValidator@1@QAVMemoryManager@1@@Z 1205df70 f   AbstractDOMParser.obj
 0001:0005d060       ??_EAbstractDOMParser@xercesc_2_3@@UAEPAXI@Z 1205e060 f i AbstractDOMParser.obj
 0001:0005d0c0       ??1AbstractDOMParser@xercesc_2_3@@UAE@XZ 1205e0c0 f   AbstractDOMParser.obj
 0001:0005d160       ?initialize@AbstractDOMParser@xercesc_2_3@@AAEXXZ 1205e160 f   AbstractDOMParser.obj
 0001:0005d2b0       ?cleanUp@AbstractDOMParser@xercesc_2_3@@AAEXXZ 1205e2b0 f   AbstractDOMParser.obj
 0001:0005d340       ?reset@AbstractDOMParser@xercesc_2_3@@QAEXXZ 1205e340 f   AbstractDOMParser.obj
 0001:0005d4c0       ?resetPool@AbstractDOMParser@xercesc_2_3@@IAEXXZ 1205e4c0 f   AbstractDOMParser.obj
 0001:0005d560       ?isDocumentAdopted@AbstractDOMParser@xercesc_2_3@@IBE_NXZ 1205e560 f   AbstractDOMParser.obj
 0001:0005d570       ?adoptDocument@AbstractDOMParser@xercesc_2_3@@QAEPAVDOMDocument@2@XZ 1205e570 f   AbstractDOMParser.obj
 0001:0005d580       ?getValidator@AbstractDOMParser@xercesc_2_3@@QBEABVXMLValidator@2@XZ 1205e580 f   AbstractDOMParser.obj
 0001:0005d590       ?getDoNamespaces@AbstractDOMParser@xercesc_2_3@@QBE_NXZ 1205e590 f   AbstractDOMParser.obj
 0001:0005d5a0       ?getExitOnFirstFatalError@AbstractDOMParser@xercesc_2_3@@QBE_NXZ 1205e5a0 f   AbstractDOMParser.obj
 0001:0005d5b0       ?getValidationConstraintFatal@AbstractDOMParser@xercesc_2_3@@QBE_NXZ 1205e5b0 f   AbstractDOMParser.obj
 0001:0005d5c0       ?getValidationScheme@AbstractDOMParser@xercesc_2_3@@QBE?AW4ValSchemes@12@XZ 1205e5c0 f   AbstractDOMParser.obj
 0001:0005d5e0       ?getDoSchema@AbstractDOMParser@xercesc_2_3@@QBE_NXZ 1205e5e0 f   AbstractDOMParser.obj
 0001:0005d5f0       ?getValidationSchemaFullChecking@AbstractDOMParser@xercesc_2_3@@QBE_NXZ 1205e5f0 f   AbstractDOMParser.obj
 0001:0005d600       ?getErrorCount@AbstractDOMParser@xercesc_2_3@@QBEHXZ 1205e600 f   AbstractDOMParser.obj
 0001:0005d610       ?getExternalSchemaLocation@AbstractDOMParser@xercesc_2_3@@QBEPAGXZ 1205e610 f   AbstractDOMParser.obj
 0001:0005d620       ?getExternalNoNamespaceSchemaLocation@AbstractDOMParser@xercesc_2_3@@QBEPAGXZ 1205e620 f   AbstractDOMParser.obj
 0001:0005d630       ?getSecurityManager@AbstractDOMParser@xercesc_2_3@@QBEPAVSecurityManager@2@XZ 1205e630 f   AbstractDOMParser.obj
 0001:0005d640       ?getLoadExternalDTD@AbstractDOMParser@xercesc_2_3@@QBE_NXZ 1205e640 f   AbstractDOMParser.obj
 0001:0005d650       ?getCalculateSrcOfs@AbstractDOMParser@xercesc_2_3@@QBE_NXZ 1205e650 f   AbstractDOMParser.obj
 0001:0005d660       ?getStandardUriConformant@AbstractDOMParser@xercesc_2_3@@QBE_NXZ 1205e660 f   AbstractDOMParser.obj
 0001:0005d670       ?setDoNamespaces@AbstractDOMParser@xercesc_2_3@@QAEX_N@Z 1205e670 f   AbstractDOMParser.obj
 0001:0005d680       ?setExitOnFirstFatalError@AbstractDOMParser@xercesc_2_3@@QAEX_N@Z 1205e680 f   AbstractDOMParser.obj
 0001:0005d690       ?setValidationConstraintFatal@AbstractDOMParser@xercesc_2_3@@QAEX_N@Z 1205e690 f   AbstractDOMParser.obj
 0001:0005d6a0       ?setValidationScheme@AbstractDOMParser@xercesc_2_3@@QAEXW4ValSchemes@12@@Z 1205e6a0 f   AbstractDOMParser.obj
 0001:0005d6f0       ?setDoSchema@AbstractDOMParser@xercesc_2_3@@QAEX_N@Z 1205e6f0 f   AbstractDOMParser.obj
 0001:0005d700       ?setValidationSchemaFullChecking@AbstractDOMParser@xercesc_2_3@@QAEX_N@Z 1205e700 f   AbstractDOMParser.obj
 0001:0005d710       ?setExternalSchemaLocation@AbstractDOMParser@xercesc_2_3@@QAEXQBG@Z 1205e710 f   AbstractDOMParser.obj
 0001:0005d790       ?setExternalNoNamespaceSchemaLocation@AbstractDOMParser@xercesc_2_3@@QAEXQBG@Z 1205e790 f   AbstractDOMParser.obj
 0001:0005d810       ?setExternalSchemaLocation@AbstractDOMParser@xercesc_2_3@@QAEXQBD@Z 1205e810 f   AbstractDOMParser.obj
 0001:0005d850       ?setExternalNoNamespaceSchemaLocation@AbstractDOMParser@xercesc_2_3@@QAEXQBD@Z 1205e850 f   AbstractDOMParser.obj
 0001:0005d890       ?setSecurityManager@AbstractDOMParser@xercesc_2_3@@QAEXQAVSecurityManager@2@@Z 1205e890 f   AbstractDOMParser.obj
 0001:0005d8f0       ?setLoadExternalDTD@AbstractDOMParser@xercesc_2_3@@QAEX_N@Z 1205e8f0 f   AbstractDOMParser.obj
 0001:0005d900       ?setCalculateSrcOfs@AbstractDOMParser@xercesc_2_3@@QAEX_N@Z 1205e900 f   AbstractDOMParser.obj
 0001:0005d910       ?setStandardUriConformant@AbstractDOMParser@xercesc_2_3@@QAEX_N@Z 1205e910 f   AbstractDOMParser.obj
 0001:0005d920       ?useScanner@AbstractDOMParser@xercesc_2_3@@QAEXQBG@Z 1205e920 f   AbstractDOMParser.obj
 0001:0005d980       ?parse@AbstractDOMParser@xercesc_2_3@@QAEXABVInputSource@2@@Z 1205e980 f   AbstractDOMParser.obj
 0001:0005da30       ?parse@AbstractDOMParser@xercesc_2_3@@QAEXQBG@Z 1205ea30 f   AbstractDOMParser.obj
 0001:0005dae0       ?parse@AbstractDOMParser@xercesc_2_3@@QAEXQBD@Z 1205eae0 f   AbstractDOMParser.obj
 0001:0005db90       ?parseFirst@AbstractDOMParser@xercesc_2_3@@QAE_NQBGAAVXMLPScanToken@2@@Z 1205eb90 f   AbstractDOMParser.obj
 0001:0005dbe0       ?parseFirst@AbstractDOMParser@xercesc_2_3@@QAE_NQBDAAVXMLPScanToken@2@@Z 1205ebe0 f   AbstractDOMParser.obj
 0001:0005dc30       ?parseFirst@AbstractDOMParser@xercesc_2_3@@QAE_NABVInputSource@2@AAVXMLPScanToken@2@@Z 1205ec30 f   AbstractDOMParser.obj
 0001:0005dc80       ?parseNext@AbstractDOMParser@xercesc_2_3@@QAE_NAAVXMLPScanToken@2@@Z 1205ec80 f   AbstractDOMParser.obj
 0001:0005dc90       ?parseReset@AbstractDOMParser@xercesc_2_3@@QAEXAAVXMLPScanToken@2@@Z 1205ec90 f   AbstractDOMParser.obj
 0001:0005dcb0       ?docCharacters@AbstractDOMParser@xercesc_2_3@@UAEXQBGI_N@Z 1205ecb0 f   AbstractDOMParser.obj
 0001:0005dd40       ?docComment@AbstractDOMParser@xercesc_2_3@@UAEXQBG@Z 1205ed40 f   AbstractDOMParser.obj
 0001:0005dd70       ?docPI@AbstractDOMParser@xercesc_2_3@@UAEXQBG0@Z 1205ed70 f   AbstractDOMParser.obj
 0001:0005dda0       ?endEntityReference@AbstractDOMParser@xercesc_2_3@@UAEXABVXMLEntityDecl@2@@Z 1205eda0 f   AbstractDOMParser.obj
 0001:0005e0a0       ?endElement@AbstractDOMParser@xercesc_2_3@@UAEXABVXMLElementDecl@2@I_NQBG@Z 1205f0a0 f   AbstractDOMParser.obj
 0001:0005e190       ?ignorableWhitespace@AbstractDOMParser@xercesc_2_3@@UAEXQBGI_N@Z 1205f190 f   AbstractDOMParser.obj
 0001:0005e220       ?resetDocument@AbstractDOMParser@xercesc_2_3@@UAEXXZ 1205f220 f   AbstractDOMParser.obj
 0001:0005e230       ?startDocument@AbstractDOMParser@xercesc_2_3@@UAEXXZ 1205f230 f   AbstractDOMParser.obj
 0001:0005e2a0       ?endDocument@AbstractDOMParser@xercesc_2_3@@UAEXXZ 1205f2a0 f   AbstractDOMParser.obj
 0001:0005e2d0       ?startElement@AbstractDOMParser@xercesc_2_3@@UAEXABVXMLElementDecl@2@IQBGABV?$RefVectorOf@VXMLAttr@xercesc_2_3@@@2@I_N3@Z 1205f2d0 f   AbstractDOMParser.obj
 0001:0005ec00       ?startEntityReference@AbstractDOMParser@xercesc_2_3@@UAEXABVXMLEntityDecl@2@@Z 1205fc00 f   AbstractDOMParser.obj
 0001:0005ed20       ?XMLDecl@AbstractDOMParser@xercesc_2_3@@UAEXQBG000@Z 1205fd20 f   AbstractDOMParser.obj
 0001:0005edc0       ?createElementNSNode@AbstractDOMParser@xercesc_2_3@@MAEPAVDOMElement@2@PBG0@Z 1205fdc0 f   AbstractDOMParser.obj
 0001:0005ede0       ?getDoValidation@AbstractDOMParser@xercesc_2_3@@QBE_NXZ 1205fde0 f   AbstractDOMParser.obj
 0001:0005edf0       ?setDoValidation@AbstractDOMParser@xercesc_2_3@@QAEX_N@Z 1205fdf0 f   AbstractDOMParser.obj
 0001:0005ee20       ?attDef@AbstractDOMParser@xercesc_2_3@@UAEXABVDTDElementDecl@2@ABVDTDAttDef@2@_N@Z 1205fe20 f   AbstractDOMParser.obj
 0001:0005f2c0       ?doctypeComment@AbstractDOMParser@xercesc_2_3@@UAEXQBG@Z 120602c0 f   AbstractDOMParser.obj
 0001:0005f3b0       ?doctypeDecl@AbstractDOMParser@xercesc_2_3@@UAEXABVDTDElementDecl@2@QBG1_N2@Z 120603b0 f   AbstractDOMParser.obj
 0001:0005f3f0       ?doctypePI@AbstractDOMParser@xercesc_2_3@@UAEXQBG0@Z 120603f0 f   AbstractDOMParser.obj
 0001:0005f4d0       ?doctypeWhitespace@AbstractDOMParser@xercesc_2_3@@UAEXQBGI@Z 120604d0 f   AbstractDOMParser.obj
 0001:0005f500       ?elementDecl@AbstractDOMParser@xercesc_2_3@@UAEXABVDTDElementDecl@2@_N@Z 12060500 f   AbstractDOMParser.obj
 0001:0005f610       ?endAttList@AbstractDOMParser@xercesc_2_3@@UAEXABVDTDElementDecl@2@@Z 12060610 f   AbstractDOMParser.obj
 0001:0005f910       ?endIntSubset@AbstractDOMParser@xercesc_2_3@@UAEXXZ 12060910 f   AbstractDOMParser.obj
 0001:0005f940       ?entityDecl@AbstractDOMParser@xercesc_2_3@@UAEXABVDTDEntityDecl@2@_N1@Z 12060940 f   AbstractDOMParser.obj
 0001:0005fce0       ?resetDocType@AbstractDOMParser@xercesc_2_3@@UAEXXZ 12060ce0 f   AbstractDOMParser.obj
 0001:0005fcf0       ?notationDecl@AbstractDOMParser@xercesc_2_3@@UAEXABVXMLNotationDecl@2@_N@Z 12060cf0 f   AbstractDOMParser.obj
 0001:0005ff90       ?startAttList@AbstractDOMParser@xercesc_2_3@@UAEXABVDTDElementDecl@2@@Z 12060f90 f   AbstractDOMParser.obj
 0001:00060040       ?startIntSubset@AbstractDOMParser@xercesc_2_3@@UAEXXZ 12061040 f   AbstractDOMParser.obj
 0001:00060050       ?TextDecl@AbstractDOMParser@xercesc_2_3@@UAEXQBG0@Z 12061050 f   AbstractDOMParser.obj
 0001:00060080       ??_G?$RefVectorOf@VDOMDocumentImpl@xercesc_2_3@@@xercesc_2_3@@UAEPAXI@Z 12061080 f i AbstractDOMParser.obj
 0001:00060080       ??_E?$RefVectorOf@VDOMDocumentImpl@xercesc_2_3@@@xercesc_2_3@@UAEPAXI@Z 12061080 f i AbstractDOMParser.obj
 0001:000600a0       ??1?$RefVectorOf@VDOMDocumentImpl@xercesc_2_3@@@xercesc_2_3@@UAE@XZ 120610a0 f i AbstractDOMParser.obj
 0001:00060120       ??1?$BaseRefVectorOf@VDOMDocumentImpl@xercesc_2_3@@@xercesc_2_3@@UAE@XZ 12061120 f i AbstractDOMParser.obj
 0001:00060130       ??_EAbstractDOMParser@xercesc_2_3@@W3AEPAXI@Z 12061130 f i AbstractDOMParser.obj
 0001:00060140       ??_EAbstractDOMParser@xercesc_2_3@@W7AEPAXI@Z 12061140 f i AbstractDOMParser.obj
 0001:00060150       ??_EAbstractDOMParser@xercesc_2_3@@WM@AEPAXI@Z 12061150 f i AbstractDOMParser.obj
 0001:00060160       ??0DOMBuilder@xercesc_2_3@@IAE@XZ 12061160 f i DOMBuilderImpl.obj
 0001:00060170       ??1DOMBuilder@xercesc_2_3@@UAE@XZ 12061170 f i DOMBuilderImpl.obj
 0001:00060180       ??_EDOMBuilder@xercesc_2_3@@UAEPAXI@Z 12061180 f i DOMBuilderImpl.obj
 0001:000601e0       ??_FDOMBuilderImpl@xercesc_2_3@@QAEXXZ 120611e0 f i DOMBuilderImpl.obj
 0001:000601f0       ?expandSystemId@DOMParser@xercesc_2_3@@UAE_NQBGAAVXMLBuffer@2@@Z 120611f0 f i DOMBuilderImpl.obj
 0001:000601f0       ?expandSystemId@XercesDOMParser@xercesc_2_3@@UAE_NQBGAAVXMLBuffer@2@@Z 120611f0 f i DOMBuilderImpl.obj
 0001:000601f0       ?expandSystemId@DOMBuilderImpl@xercesc_2_3@@UAE_NQBGAAVXMLBuffer@2@@Z 120611f0 f i DOMBuilderImpl.obj
 0001:00060200       ??0DOMEntityResolver@xercesc_2_3@@IAE@XZ 12061200 f i DOMBuilderImpl.obj
 0001:00060210       ??1DOMEntityResolver@xercesc_2_3@@UAE@XZ 12061210 f i DOMBuilderImpl.obj
 0001:00060220       ??_EDOMEntityResolver@xercesc_2_3@@UAEPAXI@Z 12061220 f i DOMBuilderImpl.obj
 0001:00060280       ??0DOMErrorHandler@xercesc_2_3@@IAE@XZ 12061280 f i DOMBuilderImpl.obj
 0001:00060290       ??1DOMErrorHandler@xercesc_2_3@@UAE@XZ 12061290 f i DOMBuilderImpl.obj
 0001:000602a0       ??_EDOMErrorHandler@xercesc_2_3@@UAEPAXI@Z 120612a0 f i DOMBuilderImpl.obj
 0001:00060300       ?getSeverity@DOMErrorImpl@xercesc_2_3@@UBEFXZ 12061300 f i DOMBuilderImpl.obj
 0001:00060310       ?setSeverity@DOMErrorImpl@xercesc_2_3@@UAEXF@Z 12061310 f i DOMBuilderImpl.obj
 0001:00060320       ?setPreprocessed@ComplexTypeInfo@xercesc_2_3@@QAEX_N@Z 12061320 f i DOMBuilderImpl.obj
 0001:00060320       ?setExitOnFirstFatal@XSDErrorReporter@xercesc_2_3@@QAEX_N@Z 12061320 f i DOMBuilderImpl.obj
 0001:00060320       ?setAdoptLocation@DOMErrorImpl@xercesc_2_3@@QAEX_N@Z 12061320 f i DOMBuilderImpl.obj
 0001:00060330       ?setAdoptRelatedData@DOMErrorImpl@xercesc_2_3@@QAEX_N@Z 12061330 f i DOMBuilderImpl.obj
 0001:00060340       ??0DOMLocator@xercesc_2_3@@IAE@XZ 12061340 f i DOMBuilderImpl.obj
 0001:00060350       ??1DOMLocator@xercesc_2_3@@UAE@XZ 12061350 f i DOMBuilderImpl.obj
 0001:00060360       ??_EDOMLocator@xercesc_2_3@@UAEPAXI@Z 12061360 f i DOMBuilderImpl.obj
 0001:000603c0       ?setRelatedData@DOMErrorImpl@xercesc_2_3@@UAEXPAX@Z 120613c0 f i DOMBuilderImpl.obj
 0001:000603c0       ?setScopeDefined@ComplexTypeInfo@xercesc_2_3@@QAEXH@Z 120613c0 f i DOMBuilderImpl.obj
 0001:000603c0       ?setId@XMLAttDef@xercesc_2_3@@QAEXI@Z 120613c0 f i DOMBuilderImpl.obj
 0001:000603c0       ?setGrammar@DTDValidator@xercesc_2_3@@UAEXPAVGrammar@2@@Z 120613c0 f i DOMBuilderImpl.obj
 0001:000603c0       ?setURI@DOMLocatorImpl@xercesc_2_3@@UAEXQBG@Z 120613c0 f i DOMBuilderImpl.obj
 0001:000603d0       ??0DOMBuilderImpl@xercesc_2_3@@QAE@QAVXMLValidator@1@QAVMemoryManager@1@@Z 120613d0 f   DOMBuilderImpl.obj
 0001:00060440       ??_EDOMBuilderImpl@xercesc_2_3@@UAEPAXI@Z 12061440 f i DOMBuilderImpl.obj
 0001:000604a0       ??1DOMBuilderImpl@xercesc_2_3@@UAE@XZ 120614a0 f   DOMBuilderImpl.obj
 0001:000604e0       ?setErrorHandler@DOMBuilderImpl@xercesc_2_3@@UAEXQAVDOMErrorHandler@2@@Z 120614e0 f   DOMBuilderImpl.obj
 0001:00060520       ?setEntityResolver@DOMBuilderImpl@xercesc_2_3@@UAEXQAVDOMEntityResolver@2@@Z 12061520 f   DOMBuilderImpl.obj
 0001:00060550       ?setFeature@DOMBuilderImpl@xercesc_2_3@@UAEXQBG_N@Z 12061550 f   DOMBuilderImpl.obj
 0001:00060930       ?getFeature@DOMBuilderImpl@xercesc_2_3@@UBE_NQBG@Z 12061930 f   DOMBuilderImpl.obj
 0001:00060c20       ?canSetFeature@DOMBuilderImpl@xercesc_2_3@@UBE_NQBG_N@Z 12061c20 f   DOMBuilderImpl.obj
 0001:00060e30       ?setProperty@DOMBuilderImpl@xercesc_2_3@@UAEXQBGPAX@Z 12061e30 f   DOMBuilderImpl.obj
 0001:00060f30       ?getProperty@DOMBuilderImpl@xercesc_2_3@@UBEPAXQBG@Z 12061f30 f   DOMBuilderImpl.obj
 0001:00060fc0       ?release@DOMBuilderImpl@xercesc_2_3@@UAEXXZ 12061fc0 f   DOMBuilderImpl.obj
 0001:00060fd0       ?resetDocumentPool@DOMBuilderImpl@xercesc_2_3@@UAEXXZ 12061fd0 f   DOMBuilderImpl.obj
 0001:00060fe0       ?parse@DOMBuilderImpl@xercesc_2_3@@UAEPAVDOMDocument@2@ABVDOMInputSource@2@@Z 12061fe0 f   DOMBuilderImpl.obj
 0001:00061070       ?parseURI@DOMBuilderImpl@xercesc_2_3@@UAEPAVDOMDocument@2@QBG@Z 12062070 f   DOMBuilderImpl.obj
 0001:000610a0       ?parseURI@DOMBuilderImpl@xercesc_2_3@@UAEPAVDOMDocument@2@QBD@Z 120620a0 f   DOMBuilderImpl.obj
 0001:000610d0       ?error@DOMBuilderImpl@xercesc_2_3@@UAEXIQBGW4ErrTypes@XMLErrorReporter@2@000JJ@Z 120620d0 f   DOMBuilderImpl.obj
 0001:000611c0       ?resolveEntity@DOMBuilderImpl@xercesc_2_3@@UAEPAVInputSource@2@QBG00@Z 120621c0 f   DOMBuilderImpl.obj
 0001:00061250       ?loadGrammar@DOMBuilderImpl@xercesc_2_3@@UAEPAVGrammar@2@QBDF_N@Z 12062250 f   DOMBuilderImpl.obj
 0001:00061320       ?loadGrammar@DOMBuilderImpl@xercesc_2_3@@UAEPAVGrammar@2@QBGF_N@Z 12062320 f   DOMBuilderImpl.obj
 0001:000613f0       ?loadGrammar@DOMBuilderImpl@xercesc_2_3@@UAEPAVGrammar@2@ABVDOMInputSource@2@F_N@Z 120623f0 f   DOMBuilderImpl.obj
 0001:000614e0       ?resetCachedGrammarPool@DOMBuilderImpl@xercesc_2_3@@UAEXXZ 120624e0 f   DOMBuilderImpl.obj
 0001:000614f0       ?getGrammar@DOMBuilderImpl@xercesc_2_3@@UBEPAVGrammar@2@QBG@Z 120624f0 f   DOMBuilderImpl.obj
 0001:00061500       ?getRootGrammar@DOMBuilderImpl@xercesc_2_3@@UBEPAVGrammar@2@XZ 12062500 f   DOMBuilderImpl.obj
 0001:00061510       ?getURIText@DOMBuilderImpl@xercesc_2_3@@UBEPBGI@Z 12062510 f   DOMBuilderImpl.obj
 0001:00061520       ?getSrcOffset@DOMBuilderImpl@xercesc_2_3@@UBEIXZ 12062520 f   DOMBuilderImpl.obj
 0001:00061530       ??_EDOMBuilderImpl@xercesc_2_3@@W3AEPAXI@Z 12062530 f i DOMBuilderImpl.obj
 0001:00061540       ??_EDOMBuilderImpl@xercesc_2_3@@W7AEPAXI@Z 12062540 f i DOMBuilderImpl.obj
 0001:00061550       ??_EDOMBuilderImpl@xercesc_2_3@@WM@AEPAXI@Z 12062550 f i DOMBuilderImpl.obj
 0001:00061560       ??_EDOMBuilderImpl@xercesc_2_3@@WFI@AEPAXI@Z 12062560 f i DOMBuilderImpl.obj
 0001:00061570       ??0ContentHandler@xercesc_2_3@@QAE@XZ 12062570 f i SAX2XMLReaderImpl.obj
 0001:00061580       ??1ContentHandler@xercesc_2_3@@UAE@XZ 12062580 f i SAX2XMLReaderImpl.obj
 0001:00061590       ??_EContentHandler@xercesc_2_3@@UAEPAXI@Z 12062590 f i SAX2XMLReaderImpl.obj
 0001:000615f0       ??0LexicalHandler@xercesc_2_3@@QAE@XZ 120625f0 f i SAX2XMLReaderImpl.obj
 0001:00061600       ??1LexicalHandler@xercesc_2_3@@UAE@XZ 12062600 f i SAX2XMLReaderImpl.obj
 0001:00061610       ??_ELexicalHandler@xercesc_2_3@@UAEPAXI@Z 12062610 f i SAX2XMLReaderImpl.obj
 0001:00061670       ??0DeclHandler@xercesc_2_3@@QAE@XZ 12062670 f i SAX2XMLReaderImpl.obj
 0001:00061680       ??1DeclHandler@xercesc_2_3@@UAE@XZ 12062680 f i SAX2XMLReaderImpl.obj
 0001:00061690       ??_EDeclHandler@xercesc_2_3@@UAEPAXI@Z 12062690 f i SAX2XMLReaderImpl.obj
 0001:000616f0       ??_FSAXParser@xercesc_2_3@@QAEXXZ 120626f0 f i SAX2XMLReaderImpl.obj
 0001:00061700       ?getBaseComplexTypeInfo@ComplexTypeInfo@xercesc_2_3@@QBEPAV12@XZ 12062700 f i SAX2XMLReaderImpl.obj
 0001:00061700       ?getDocumentHandler@SAXParser@xercesc_2_3@@QAEPAVDocumentHandler@2@XZ 12062700 f i SAX2XMLReaderImpl.obj
 0001:00061700       ?getDocumentHandler@SAXParser@xercesc_2_3@@QBEPBVDocumentHandler@2@XZ 12062700 f i SAX2XMLReaderImpl.obj
 0001:00061700       ?getTypeUri@DatatypeValidator@xercesc_2_3@@QBEPBGXZ 12062700 f i SAX2XMLReaderImpl.obj
 0001:00061710       ??0SAX2XMLReader@xercesc_2_3@@QAE@XZ 12062710 f i SAX2XMLReaderImpl.obj
 0001:00061720       ??1SAX2XMLReader@xercesc_2_3@@UAE@XZ 12062720 f i SAX2XMLReaderImpl.obj
 0001:00061730       ??_ESAX2XMLReader@xercesc_2_3@@UAEPAXI@Z 12062730 f i SAX2XMLReaderImpl.obj
 0001:00061790       ??_FSAX2XMLReaderImpl@xercesc_2_3@@QAEXXZ 12062790 f i SAX2XMLReaderImpl.obj
 0001:000617a0       ?getContentHandler@SAX2XMLReaderImpl@xercesc_2_3@@UBEPAVContentHandler@2@XZ 120627a0 f i SAX2XMLReaderImpl.obj
 0001:000617a0       ?getAttWildCard@ComplexTypeInfo@xercesc_2_3@@QBEPBVSchemaAttDef@2@XZ 120627a0 f i SAX2XMLReaderImpl.obj
 0001:000617a0       ?getAttWildCard@ComplexTypeInfo@xercesc_2_3@@QAEPAVSchemaAttDef@2@XZ 120627a0 f i SAX2XMLReaderImpl.obj
 0001:000617a0       ?getValidity@SchemaAttDef@xercesc_2_3@@QBE?AW4Validity@PSVIDefs@2@XZ 120627a0 f i SAX2XMLReaderImpl.obj
 0001:000617a0       ?getMaxLength@AbstractStringValidator@xercesc_2_3@@QBEIXZ 120627a0 f i SAX2XMLReaderImpl.obj
 0001:000617a0       ?getEnumeration@UnionDatatypeValidator@xercesc_2_3@@ABEPAV?$RefArrayVectorOf@G@2@XZ 120627a0 f i SAX2XMLReaderImpl.obj
 0001:000617a0       ?getEntityResolver@SAXParser@xercesc_2_3@@QAEPAVEntityResolver@2@XZ 120627a0 f i SAX2XMLReaderImpl.obj
 0001:000617a0       ?getEntityResolver@SAXParser@xercesc_2_3@@QBEPBVEntityResolver@2@XZ 120627a0 f i SAX2XMLReaderImpl.obj
 0001:000617a0       ?getRecursingTypeNames@SchemaInfo@xercesc_2_3@@QBEPAV?$ValueVectorOf@PBG@2@XZ 120627a0 f i SAX2XMLReaderImpl.obj
 0001:000617b0       ?getExitOnFirstFatalError@SAX2XMLReaderImpl@xercesc_2_3@@UBE_NXZ 120627b0 f i SAX2XMLReaderImpl.obj
 0001:000617c0       ?getValidationConstraintFatal@SAX2XMLReaderImpl@xercesc_2_3@@UBE_NXZ 120627c0 f i SAX2XMLReaderImpl.obj
 0001:000617d0       ?getRootGrammar@SAX2XMLReaderImpl@xercesc_2_3@@UAEPAVGrammar@2@XZ 120627d0 f i SAX2XMLReaderImpl.obj
 0001:000617e0       ?getURIText@SAX2XMLReaderImpl@xercesc_2_3@@UBEPBGI@Z 120627e0 f i SAX2XMLReaderImpl.obj
 0001:000617f0       ?getSrcOffset@SAX2XMLReaderImpl@xercesc_2_3@@UBEIXZ 120627f0 f i SAX2XMLReaderImpl.obj
 0001:00061800       ??0SAX2XMLReaderImpl@xercesc_2_3@@QAE@QAVMemoryManager@1@@Z 12062800 f   SAX2XMLReaderImpl.obj
 0001:00061910       ??_ESAX2XMLReaderImpl@xercesc_2_3@@UAEPAXI@Z 12062910 f i SAX2XMLReaderImpl.obj
 0001:00061970       ??1SAX2XMLReaderImpl@xercesc_2_3@@UAE@XZ 12062970 f   SAX2XMLReaderImpl.obj
 0001:00061a40       ?initialize@SAX2XMLReaderImpl@xercesc_2_3@@AAEXXZ 12062a40 f   SAX2XMLReaderImpl.obj
 0001:00061c80       ?cleanUp@SAX2XMLReaderImpl@xercesc_2_3@@AAEXXZ 12062c80 f   SAX2XMLReaderImpl.obj
 0001:00061d10       ?installAdvDocHandler@SAX2XMLReaderImpl@xercesc_2_3@@UAEXQAVXMLDocumentHandler@2@@Z 12062d10 f   SAX2XMLReaderImpl.obj
 0001:00061df0       ?removeAdvDocHandler@SAX2XMLReaderImpl@xercesc_2_3@@UAE_NQAVXMLDocumentHandler@2@@Z 12062df0 f   SAX2XMLReaderImpl.obj
 0001:00061e70       ?setValidator@SAX2XMLReaderImpl@xercesc_2_3@@UAEXPAVXMLValidator@2@@Z 12062e70 f   SAX2XMLReaderImpl.obj
 0001:00061e90       ?getValidator@SAX2XMLReaderImpl@xercesc_2_3@@UBEPAVXMLValidator@2@XZ 12062e90 f   SAX2XMLReaderImpl.obj
 0001:00061ea0       ?getErrorCount@SAX2XMLReaderImpl@xercesc_2_3@@UBEHXZ 12062ea0 f   SAX2XMLReaderImpl.obj
 0001:00061eb0       ?setContentHandler@SAX2XMLReaderImpl@xercesc_2_3@@UAEXQAVContentHandler@2@@Z 12062eb0 f   SAX2XMLReaderImpl.obj
 0001:00061ef0       ?setDTDHandler@SAX2XMLReaderImpl@xercesc_2_3@@UAEXQAVDTDHandler@2@@Z 12062ef0 f   SAX2XMLReaderImpl.obj
 0001:00061f30       ?setErrorHandler@SAX2XMLReaderImpl@xercesc_2_3@@UAEXQAVErrorHandler@2@@Z 12062f30 f   SAX2XMLReaderImpl.obj
 0001:00061f70       ?setLexicalHandler@SAX2XMLReaderImpl@xercesc_2_3@@UAEXQAVLexicalHandler@2@@Z 12062f70 f   SAX2XMLReaderImpl.obj
 0001:00061fb0       ?setDeclarationHandler@SAX2XMLReaderImpl@xercesc_2_3@@UAEXQAVDeclHandler@2@@Z 12062fb0 f   SAX2XMLReaderImpl.obj
 0001:00061ff0       ?setEntityResolver@SAX2XMLReaderImpl@xercesc_2_3@@UAEXQAVEntityResolver@2@@Z 12062ff0 f   SAX2XMLReaderImpl.obj
 0001:00062010       ?setExitOnFirstFatalError@SAX2XMLReaderImpl@xercesc_2_3@@UAEX_N@Z 12063010 f   SAX2XMLReaderImpl.obj
 0001:00062020       ?setValidationConstraintFatal@SAX2XMLReaderImpl@xercesc_2_3@@UAEX_N@Z 12063020 f   SAX2XMLReaderImpl.obj
 0001:00062030       ?parse@SAX2XMLReaderImpl@xercesc_2_3@@UAEXABVInputSource@2@@Z 12063030 f   SAX2XMLReaderImpl.obj
 0001:000620e0       ?parse@SAX2XMLReaderImpl@xercesc_2_3@@UAEXQBG@Z 120630e0 f   SAX2XMLReaderImpl.obj
 0001:00062190       ?parse@SAX2XMLReaderImpl@xercesc_2_3@@UAEXQBD@Z 12063190 f   SAX2XMLReaderImpl.obj
 0001:00062240       ?parseFirst@SAX2XMLReaderImpl@xercesc_2_3@@UAE_NQBGAAVXMLPScanToken@2@@Z 12063240 f   SAX2XMLReaderImpl.obj
 0001:00062290       ?parseFirst@SAX2XMLReaderImpl@xercesc_2_3@@UAE_NQBDAAVXMLPScanToken@2@@Z 12063290 f   SAX2XMLReaderImpl.obj
 0001:000622e0       ?parseFirst@SAX2XMLReaderImpl@xercesc_2_3@@UAE_NABVInputSource@2@AAVXMLPScanToken@2@@Z 120632e0 f   SAX2XMLReaderImpl.obj
 0001:00062330       ?parseNext@SAX2XMLReaderImpl@xercesc_2_3@@UAE_NAAVXMLPScanToken@2@@Z 12063330 f   SAX2XMLReaderImpl.obj
 0001:00062340       ?parseReset@SAX2XMLReaderImpl@xercesc_2_3@@UAEXAAVXMLPScanToken@2@@Z 12063340 f   SAX2XMLReaderImpl.obj
 0001:00062350       ?docCharacters@SAX2XMLReaderImpl@xercesc_2_3@@UAEXQBGI_N@Z 12063350 f   SAX2XMLReaderImpl.obj
 0001:000623d0       ?docComment@SAX2XMLReaderImpl@xercesc_2_3@@UAEXQBG@Z 120633d0 f   SAX2XMLReaderImpl.obj
 0001:00062430       ?XMLDecl@SAX2XMLReaderImpl@xercesc_2_3@@UAEXQBG000@Z 12063430 f   SAX2XMLReaderImpl.obj
 0001:00062470       ?docPI@SAX2XMLReaderImpl@xercesc_2_3@@UAEXQBG0@Z 12063470 f   SAX2XMLReaderImpl.obj
 0001:000624c0       ?endDocument@SAX2XMLReaderImpl@xercesc_2_3@@UAEXXZ 120634c0 f   SAX2XMLReaderImpl.obj
 0001:000624f0       ?endEntityReference@SAX2XMLReaderImpl@xercesc_2_3@@UAEXABVXMLEntityDecl@2@@Z 120634f0 f   SAX2XMLReaderImpl.obj
 0001:00062530       ?ignorableWhitespace@SAX2XMLReaderImpl@xercesc_2_3@@UAEXQBGI_N@Z 12063530 f   SAX2XMLReaderImpl.obj
 0001:00062580       ?resetDocument@SAX2XMLReaderImpl@xercesc_2_3@@UAEXXZ 12063580 f   SAX2XMLReaderImpl.obj
 0001:00062710       ?startDocument@SAX2XMLReaderImpl@xercesc_2_3@@UAEXXZ 12063710 f   SAX2XMLReaderImpl.obj
 0001:00062750       ?startElement@SAX2XMLReaderImpl@xercesc_2_3@@UAEXABVXMLElementDecl@2@IQBGABV?$RefVectorOf@VXMLAttr@xercesc_2_3@@@2@I_N3@Z 12063750 f   SAX2XMLReaderImpl.obj
 0001:00062cb0       ?endElement@SAX2XMLReaderImpl@xercesc_2_3@@UAEXABVXMLElementDecl@2@I_NQBG@Z 12063cb0 f   SAX2XMLReaderImpl.obj
 0001:00062ef0       ?startEntityReference@SAX2XMLReaderImpl@xercesc_2_3@@UAEXABVXMLEntityDecl@2@@Z 12063ef0 f   SAX2XMLReaderImpl.obj
 0001:00062f30       ?attDef@SAX2XMLReaderImpl@xercesc_2_3@@UAEXABVDTDElementDecl@2@ABVDTDAttDef@2@_N@Z 12063f30 f   SAX2XMLReaderImpl.obj
 0001:00063190       ?doctypeComment@SAX2XMLReaderImpl@xercesc_2_3@@UAEXQBG@Z 12064190 f   SAX2XMLReaderImpl.obj
 0001:000631e0       ?doctypeDecl@SAX2XMLReaderImpl@xercesc_2_3@@UAEXABVDTDElementDecl@2@QBG1_N2@Z 120641e0 f   SAX2XMLReaderImpl.obj
 0001:00063240       ?elementDecl@SAX2XMLReaderImpl@xercesc_2_3@@UAEXABVDTDElementDecl@2@_N@Z 12064240 f   SAX2XMLReaderImpl.obj
 0001:00063280       ?endIntSubset@SAX2XMLReaderImpl@xercesc_2_3@@UAEXXZ 12064280 f   SAX2XMLReaderImpl.obj
 0001:000632a0       ?endExtSubset@SAX2XMLReaderImpl@xercesc_2_3@@UAEXXZ 120642a0 f   SAX2XMLReaderImpl.obj
 0001:000632c0       ?entityDecl@SAX2XMLReaderImpl@xercesc_2_3@@UAEXABVDTDEntityDecl@2@_N1@Z 120642c0 f   SAX2XMLReaderImpl.obj
 0001:00063420       ?resetDocType@SAX2XMLReaderImpl@xercesc_2_3@@UAEXXZ 12064420 f   SAX2XMLReaderImpl.obj
 0001:00063440       ?notationDecl@SAX2XMLReaderImpl@xercesc_2_3@@UAEXABVXMLNotationDecl@2@_N@Z 12064440 f   SAX2XMLReaderImpl.obj
 0001:00063470       ?startExtSubset@SAX2XMLReaderImpl@xercesc_2_3@@UAEXXZ 12064470 f   SAX2XMLReaderImpl.obj
 0001:00063490       ?resolveEntity@SAX2XMLReaderImpl@xercesc_2_3@@UAEPAVInputSource@2@QBG00@Z 12064490 f   SAX2XMLReaderImpl.obj
 0001:000634b0       ?resetErrors@SAX2XMLReaderImpl@xercesc_2_3@@UAEXXZ 120644b0 f   SAX2XMLReaderImpl.obj
 0001:000634c0       ?error@SAX2XMLReaderImpl@xercesc_2_3@@UAEXIQBGW4ErrTypes@XMLErrorReporter@2@000JJ@Z 120644c0 f   SAX2XMLReaderImpl.obj
 0001:00063580       ?setFeature@SAX2XMLReaderImpl@xercesc_2_3@@UAEXQBG_N@Z 12064580 f   SAX2XMLReaderImpl.obj
 0001:00063810       ?getFeature@SAX2XMLReaderImpl@xercesc_2_3@@UBE_NQBG@Z 12064810 f   SAX2XMLReaderImpl.obj
 0001:000639e0       ?setProperty@SAX2XMLReaderImpl@xercesc_2_3@@UAEXQBGPAX@Z 120649e0 f   SAX2XMLReaderImpl.obj
 0001:00063c20       ?getProperty@SAX2XMLReaderImpl@xercesc_2_3@@UBEPAXQBG@Z 12064c20 f   SAX2XMLReaderImpl.obj
 0001:00063d10       ?setValidationScheme@SAX2XMLReaderImpl@xercesc_2_3@@AAEXW4ValSchemes@SAX2XMLReader@2@@Z 12064d10 f   SAX2XMLReaderImpl.obj
 0001:00063d60       ?setDoNamespaces@SAX2XMLReaderImpl@xercesc_2_3@@AAEX_N@Z 12064d60 f   SAX2XMLReaderImpl.obj
 0001:00063d70       ?getDoNamespaces@SAX2XMLReaderImpl@xercesc_2_3@@ABE_NXZ 12064d70 f   SAX2XMLReaderImpl.obj
 0001:00063d80       ?setDoSchema@SAX2XMLReaderImpl@xercesc_2_3@@AAEX_N@Z 12064d80 f   SAX2XMLReaderImpl.obj
 0001:00063d90       ?getDoSchema@SAX2XMLReaderImpl@xercesc_2_3@@ABE_NXZ 12064d90 f   SAX2XMLReaderImpl.obj
 0001:00063da0       ?loadGrammar@SAX2XMLReaderImpl@xercesc_2_3@@UAEPAVGrammar@2@QBDF_N@Z 12064da0 f   SAX2XMLReaderImpl.obj
 0001:00063e50       ?loadGrammar@SAX2XMLReaderImpl@xercesc_2_3@@UAEPAVGrammar@2@QBGF_N@Z 12064e50 f   SAX2XMLReaderImpl.obj
 0001:00063f00       ?loadGrammar@SAX2XMLReaderImpl@xercesc_2_3@@UAEPAVGrammar@2@ABVInputSource@2@F_N@Z 12064f00 f   SAX2XMLReaderImpl.obj
 0001:00063fb0       ?resetCachedGrammarPool@SAX2XMLReaderImpl@xercesc_2_3@@UAEXXZ 12064fb0 f   SAX2XMLReaderImpl.obj
 0001:00063fc0       ?getGrammar@SAX2XMLReaderImpl@xercesc_2_3@@UAEPAVGrammar@2@QBG@Z 12064fc0 f   SAX2XMLReaderImpl.obj
 0001:00063fd0       ??1?$RefStackOf@VXMLBuffer@xercesc_2_3@@@xercesc_2_3@@QAE@XZ 12064fd0 f i SAX2XMLReaderImpl.obj
 0001:00064060       ??1?$BaseRefVectorOf@VXMLBuffer@xercesc_2_3@@@xercesc_2_3@@UAE@XZ 12065060 f i SAX2XMLReaderImpl.obj
 0001:00064070       ??_G?$RefVectorOf@VXMLBuffer@xercesc_2_3@@@xercesc_2_3@@UAEPAXI@Z 12065070 f i SAX2XMLReaderImpl.obj
 0001:00064070       ??_E?$RefVectorOf@VXMLBuffer@xercesc_2_3@@@xercesc_2_3@@UAEPAXI@Z 12065070 f i SAX2XMLReaderImpl.obj
 0001:00064090       ??1?$RefVectorOf@VXMLBuffer@xercesc_2_3@@@xercesc_2_3@@UAE@XZ 12065090 f i SAX2XMLReaderImpl.obj
 0001:00064120       ??_ESAX2XMLReaderImpl@xercesc_2_3@@W3AEPAXI@Z 12065120 f i SAX2XMLReaderImpl.obj
 0001:00064130       ??_ESAX2XMLReaderImpl@xercesc_2_3@@W7AEPAXI@Z 12065130 f i SAX2XMLReaderImpl.obj
 0001:00064140       ??_ESAX2XMLReaderImpl@xercesc_2_3@@WM@AEPAXI@Z 12065140 f i SAX2XMLReaderImpl.obj
 0001:00064150       ??_ESAX2XMLReaderImpl@xercesc_2_3@@WBA@AEPAXI@Z 12065150 f i SAX2XMLReaderImpl.obj
 0001:00064160       ??0SAXParser@xercesc_2_3@@QAE@QAVXMLValidator@1@QAVMemoryManager@1@@Z 12065160 f   SAXParser.obj
 0001:000642c0       ??_ESAXParser@xercesc_2_3@@UAEPAXI@Z 120652c0 f i SAXParser.obj
 0001:00064320       ??1SAXParser@xercesc_2_3@@UAE@XZ 12065320 f   SAXParser.obj
 0001:00064450       ?initialize@SAXParser@xercesc_2_3@@AAEXXZ 12065450 f   SAXParser.obj
 0001:00064540       ?cleanUp@SAXParser@xercesc_2_3@@AAEXXZ 12065540 f   SAXParser.obj
 0001:000645a0       ?installAdvDocHandler@SAXParser@xercesc_2_3@@QAEXQAVXMLDocumentHandler@2@@Z 120655a0 f   SAXParser.obj
 0001:00064680       ?removeAdvDocHandler@SAXParser@xercesc_2_3@@QAE_NQAVXMLDocumentHandler@2@@Z 12065680 f   SAXParser.obj
 0001:00064700       ?getValidator@SAXParser@xercesc_2_3@@QBEABVXMLValidator@2@XZ 12065700 f   SAXParser.obj
 0001:00064710       ?getDoNamespaces@SAXParser@xercesc_2_3@@QBE_NXZ 12065710 f   SAXParser.obj
 0001:00064720       ?getExitOnFirstFatalError@SAXParser@xercesc_2_3@@QBE_NXZ 12065720 f   SAXParser.obj
 0001:00064730       ?getValidationConstraintFatal@SAXParser@xercesc_2_3@@QBE_NXZ 12065730 f   SAXParser.obj
 0001:00064740       ?getValidationScheme@SAXParser@xercesc_2_3@@QBE?AW4ValSchemes@12@XZ 12065740 f   SAXParser.obj
 0001:00064760       ?getDoSchema@SAXParser@xercesc_2_3@@QBE_NXZ 12065760 f   SAXParser.obj
 0001:00064770       ?getValidationSchemaFullChecking@SAXParser@xercesc_2_3@@QBE_NXZ 12065770 f   SAXParser.obj
 0001:00064780       ?getErrorCount@SAXParser@xercesc_2_3@@QBEHXZ 12065780 f   SAXParser.obj
 0001:00064790       ?getExternalSchemaLocation@SAXParser@xercesc_2_3@@QBEPAGXZ 12065790 f   SAXParser.obj
 0001:000647a0       ?getExternalNoNamespaceSchemaLocation@SAXParser@xercesc_2_3@@QBEPAGXZ 120657a0 f   SAXParser.obj
 0001:000647b0       ?getSecurityManager@SAXParser@xercesc_2_3@@QBEPAVSecurityManager@2@XZ 120657b0 f   SAXParser.obj
 0001:000647c0       ?getLoadExternalDTD@SAXParser@xercesc_2_3@@QBE_NXZ 120657c0 f   SAXParser.obj
 0001:000647d0       ?isCachingGrammarFromParse@SAXParser@xercesc_2_3@@QBE_NXZ 120657d0 f   SAXParser.obj
 0001:000647e0       ?isUsingCachedGrammarInParse@SAXParser@xercesc_2_3@@QBE_NXZ 120657e0 f   SAXParser.obj
 0001:000647f0       ?getCalculateSrcOfs@SAXParser@xercesc_2_3@@QBE_NXZ 120657f0 f   SAXParser.obj
 0001:00064800       ?getStandardUriConformant@SAXParser@xercesc_2_3@@QBE_NXZ 12065800 f   SAXParser.obj
 0001:00064810       ?getGrammar@SAXParser@xercesc_2_3@@QAEPAVGrammar@2@QBG@Z 12065810 f   SAXParser.obj
 0001:00064820       ?getRootGrammar@SAXParser@xercesc_2_3@@QAEPAVGrammar@2@XZ 12065820 f   SAXParser.obj
 0001:00064830       ?getURIText@SAXParser@xercesc_2_3@@QBEPBGI@Z 12065830 f   SAXParser.obj
 0001:00064840       ?getSrcOffset@SAXParser@xercesc_2_3@@QBEIXZ 12065840 f   SAXParser.obj
 0001:00064850       ?setDoNamespaces@SAXParser@xercesc_2_3@@QAEX_N@Z 12065850 f   SAXParser.obj
 0001:00064860       ?setExitOnFirstFatalError@SAXParser@xercesc_2_3@@QAEX_N@Z 12065860 f   SAXParser.obj
 0001:00064870       ?setValidationConstraintFatal@SAXParser@xercesc_2_3@@QAEX_N@Z 12065870 f   SAXParser.obj
 0001:00064880       ?setValidationScheme@SAXParser@xercesc_2_3@@QAEXW4ValSchemes@12@@Z 12065880 f   SAXParser.obj
 0001:000648d0       ?setDoSchema@SAXParser@xercesc_2_3@@QAEX_N@Z 120658d0 f   SAXParser.obj
 0001:000648e0       ?setValidationSchemaFullChecking@SAXParser@xercesc_2_3@@QAEX_N@Z 120658e0 f   SAXParser.obj
 0001:000648f0       ?setExternalSchemaLocation@SAXParser@xercesc_2_3@@QAEXQBG@Z 120658f0 f   SAXParser.obj
 0001:00064970       ?setExternalNoNamespaceSchemaLocation@SAXParser@xercesc_2_3@@QAEXQBG@Z 12065970 f   SAXParser.obj
 0001:000649f0       ?setExternalSchemaLocation@SAXParser@xercesc_2_3@@QAEXQBD@Z 120659f0 f   SAXParser.obj
 0001:00064a30       ?setExternalNoNamespaceSchemaLocation@SAXParser@xercesc_2_3@@QAEXQBD@Z 12065a30 f   SAXParser.obj
 0001:00064a70       ?setSecurityManager@SAXParser@xercesc_2_3@@QAEXQAVSecurityManager@2@@Z 12065a70 f   SAXParser.obj
 0001:00064ad0       ?setLoadExternalDTD@SAXParser@xercesc_2_3@@QAEX_N@Z 12065ad0 f   SAXParser.obj
 0001:00064ae0       ?cacheGrammarFromParse@SAXParser@xercesc_2_3@@QAEX_N@Z 12065ae0 f   SAXParser.obj
 0001:00064b00       ?useCachedGrammarInParse@SAXParser@xercesc_2_3@@QAEX_N@Z 12065b00 f   SAXParser.obj
 0001:00064b20       ?setCalculateSrcOfs@SAXParser@xercesc_2_3@@QAEX_N@Z 12065b20 f   SAXParser.obj
 0001:00064b30       ?setStandardUriConformant@SAXParser@xercesc_2_3@@QAEX_N@Z 12065b30 f   SAXParser.obj
 0001:00064b40       ?useScanner@SAXParser@xercesc_2_3@@QAEXQBG@Z 12065b40 f   SAXParser.obj
 0001:00064ba0       ?parse@SAXParser@xercesc_2_3@@UAEXABVInputSource@2@@Z 12065ba0 f   SAXParser.obj
 0001:00064c50       ?parse@SAXParser@xercesc_2_3@@UAEXQBG@Z 12065c50 f   SAXParser.obj
 0001:00064d00       ?parse@SAXParser@xercesc_2_3@@UAEXQBD@Z 12065d00 f   SAXParser.obj
 0001:00064db0       ?setDocumentHandler@SAXParser@xercesc_2_3@@UAEXQAVDocumentHandler@2@@Z 12065db0 f   SAXParser.obj
 0001:00064df0       ?setDTDHandler@SAXParser@xercesc_2_3@@UAEXQAVDTDHandler@2@@Z 12065df0 f   SAXParser.obj
 0001:00064e30       ?setErrorHandler@SAXParser@xercesc_2_3@@UAEXQAVErrorHandler@2@@Z 12065e30 f   SAXParser.obj
 0001:00064e70       ?setEntityResolver@SAXParser@xercesc_2_3@@UAEXQAVEntityResolver@2@@Z 12065e70 f   SAXParser.obj
 0001:00064e90       ?parseFirst@SAXParser@xercesc_2_3@@QAE_NQBGAAVXMLPScanToken@2@@Z 12065e90 f   SAXParser.obj
 0001:00064ee0       ?parseFirst@SAXParser@xercesc_2_3@@QAE_NQBDAAVXMLPScanToken@2@@Z 12065ee0 f   SAXParser.obj
 0001:00064f30       ?parseFirst@SAXParser@xercesc_2_3@@QAE_NABVInputSource@2@AAVXMLPScanToken@2@@Z 12065f30 f   SAXParser.obj
 0001:00064f80       ?parseNext@SAXParser@xercesc_2_3@@QAE_NAAVXMLPScanToken@2@@Z 12065f80 f   SAXParser.obj
 0001:00064f90       ?parseReset@SAXParser@xercesc_2_3@@QAEXAAVXMLPScanToken@2@@Z 12065f90 f   SAXParser.obj
 0001:00064fa0       ?docCharacters@SAXParser@xercesc_2_3@@UAEXQBGI_N@Z 12065fa0 f   SAXParser.obj
 0001:00064ff0       ?docComment@SAXParser@xercesc_2_3@@UAEXQBG@Z 12065ff0 f   SAXParser.obj
 0001:00065020       ?XMLDecl@SAXParser@xercesc_2_3@@UAEXQBG000@Z 12066020 f   SAXParser.obj
 0001:00065060       ?docPI@SAXParser@xercesc_2_3@@UAEXQBG0@Z 12066060 f   SAXParser.obj
 0001:000650b0       ?endDocument@SAXParser@xercesc_2_3@@UAEXXZ 120660b0 f   SAXParser.obj
 0001:000650e0       ?endElement@SAXParser@xercesc_2_3@@UAEXABVXMLElementDecl@2@I_NQBG@Z 120660e0 f   SAXParser.obj
 0001:000651c0       ?endEntityReference@SAXParser@xercesc_2_3@@UAEXABVXMLEntityDecl@2@@Z 120661c0 f   SAXParser.obj
 0001:000651f0       ?ignorableWhitespace@SAXParser@xercesc_2_3@@UAEXQBGI_N@Z 120661f0 f   SAXParser.obj
 0001:00065240       ?resetDocument@SAXParser@xercesc_2_3@@UAEXXZ 12066240 f   SAXParser.obj
 0001:00065280       ?startDocument@SAXParser@xercesc_2_3@@UAEXXZ 12066280 f   SAXParser.obj
 0001:000652c0       ?startElement@SAXParser@xercesc_2_3@@UAEXABVXMLElementDecl@2@IQBGABV?$RefVectorOf@VXMLAttr@xercesc_2_3@@@2@I_N3@Z 120662c0 f   SAXParser.obj
 0001:00065420       ?startEntityReference@SAXParser@xercesc_2_3@@UAEXABVXMLEntityDecl@2@@Z 12066420 f   SAXParser.obj
 0001:00065450       ?doctypeDecl@SAXParser@xercesc_2_3@@UAEXABVDTDElementDecl@2@QBG1_N2@Z 12066450 f   SAXParser.obj
 0001:00065460       ?entityDecl@SAXParser@xercesc_2_3@@UAEXABVDTDEntityDecl@2@_N1@Z 12066460 f   SAXParser.obj
 0001:000654a0       ?resetDocType@SAXParser@xercesc_2_3@@UAEXXZ 120664a0 f   SAXParser.obj
 0001:000654b0       ?notationDecl@SAXParser@xercesc_2_3@@UAEXABVXMLNotationDecl@2@_N@Z 120664b0 f   SAXParser.obj
 0001:000654e0       ?doctypePI@SAX2XMLReaderImpl@xercesc_2_3@@UAEXQBG0@Z 120664e0 f   SAXParser.obj
 0001:000654e0       ?elementDecl@SAXParser@xercesc_2_3@@UAEXABVDTDElementDecl@2@_N@Z 120664e0 f   SAXParser.obj
 0001:000654e0       ?doctypePI@SAXParser@xercesc_2_3@@UAEXQBG0@Z 120664e0 f   SAXParser.obj
 0001:000654e0       ?doctypeWhitespace@SAXParser@xercesc_2_3@@UAEXQBGI@Z 120664e0 f   SAXParser.obj
 0001:000654e0       ?TextDecl@SAXParser@xercesc_2_3@@UAEXQBG0@Z 120664e0 f   SAXParser.obj
 0001:000654e0       ?doctypeWhitespace@SAX2XMLReaderImpl@xercesc_2_3@@UAEXQBGI@Z 120664e0 f   SAXParser.obj
 0001:000654e0       ?TextDecl@SAX2XMLReaderImpl@xercesc_2_3@@UAEXQBG0@Z 120664e0 f   SAXParser.obj
 0001:000654e0       ?TextDecl@DOMParser@xercesc_2_3@@UAEXQBG0@Z 120664e0 f   SAXParser.obj
 0001:000654f0       ?resetErrors@SAXParser@xercesc_2_3@@UAEXXZ 120664f0 f   SAXParser.obj
 0001:00065500       ?error@SAXParser@xercesc_2_3@@UAEXIQBGW4ErrTypes@XMLErrorReporter@2@000JJ@Z 12066500 f   SAXParser.obj
 0001:000655c0       ?expandSystemId@SAX2XMLReaderImpl@xercesc_2_3@@UAE_NQBGAAVXMLBuffer@2@@Z 120665c0 f   SAXParser.obj
 0001:000655c0       ?expandSystemId@SAXParser@xercesc_2_3@@UAE_NQBGAAVXMLBuffer@2@@Z 120665c0 f   SAXParser.obj
 0001:000655d0       ?resolveEntity@SAXParser@xercesc_2_3@@UAEPAVInputSource@2@QBG00@Z 120665d0 f   SAXParser.obj
 0001:000655f0       ?getDoValidation@SAXParser@xercesc_2_3@@QBE_NXZ 120665f0 f   SAXParser.obj
 0001:00065600       ?setDoValidation@SAXParser@xercesc_2_3@@QAEX_N@Z 12066600 f   SAXParser.obj
 0001:00065630       ?loadGrammar@SAXParser@xercesc_2_3@@QAEPAVGrammar@2@QBDF_N@Z 12066630 f   SAXParser.obj
 0001:000656e0       ?loadGrammar@SAXParser@xercesc_2_3@@QAEPAVGrammar@2@QBGF_N@Z 120666e0 f   SAXParser.obj
 0001:00065790       ?loadGrammar@SAXParser@xercesc_2_3@@QAEPAVGrammar@2@ABVInputSource@2@F_N@Z 12066790 f   SAXParser.obj
 0001:00065840       ?resetCachedGrammarPool@SAXParser@xercesc_2_3@@QAEXXZ 12066840 f   SAXParser.obj
 0001:00065850       ??_ESAXParser@xercesc_2_3@@W3AEPAXI@Z 12066850 f i SAXParser.obj
 0001:00065860       ??_ESAXParser@xercesc_2_3@@W7AEPAXI@Z 12066860 f i SAXParser.obj
 0001:00065870       ??_ESAXParser@xercesc_2_3@@WM@AEPAXI@Z 12066870 f i SAXParser.obj
 0001:00065880       ??_ESAXParser@xercesc_2_3@@WBA@AEPAXI@Z 12066880 f i SAXParser.obj
 0001:00065890       ??0XercesDOMParser@xercesc_2_3@@QAE@QAVXMLValidator@1@QAVMemoryManager@1@@Z 12066890 f   XercesDOMParser.obj
 0001:000658d0       ??_EXercesDOMParser@xercesc_2_3@@UAEPAXI@Z 120668d0 f i XercesDOMParser.obj
 0001:00065930       ??1XercesDOMParser@xercesc_2_3@@UAE@XZ 12066930 f   XercesDOMParser.obj
 0001:00065950       ?isCachingGrammarFromParse@XercesDOMParser@xercesc_2_3@@QBE_NXZ 12066950 f   XercesDOMParser.obj
 0001:00065960       ?isUsingCachedGrammarInParse@XercesDOMParser@xercesc_2_3@@QBE_NXZ 12066960 f   XercesDOMParser.obj
 0001:00065970       ?getRootGrammar@XercesDOMParser@xercesc_2_3@@QAEPAVGrammar@2@XZ 12066970 f   XercesDOMParser.obj
 0001:00065980       ?getURIText@XercesDOMParser@xercesc_2_3@@QBEPBGI@Z 12066980 f   XercesDOMParser.obj
 0001:00065990       ?getSrcOffset@XercesDOMParser@xercesc_2_3@@QBEIXZ 12066990 f   XercesDOMParser.obj
 0001:000659a0       ?setErrorHandler@XercesDOMParser@xercesc_2_3@@QAEXQAVErrorHandler@2@@Z 120669a0 f   XercesDOMParser.obj
 0001:000659e0       ?setEntityResolver@XercesDOMParser@xercesc_2_3@@QAEXQAVEntityResolver@2@@Z 120669e0 f   XercesDOMParser.obj
 0001:00065a00       ?cacheGrammarFromParse@XercesDOMParser@xercesc_2_3@@QAEX_N@Z 12066a00 f   XercesDOMParser.obj
 0001:00065a20       ?useCachedGrammarInParse@XercesDOMParser@xercesc_2_3@@QAEX_N@Z 12066a20 f   XercesDOMParser.obj
 0001:00065a40       ?resetDocumentPool@XercesDOMParser@xercesc_2_3@@QAEXXZ 12066a40 f   XercesDOMParser.obj
 0001:00065a50       ?error@XercesDOMParser@xercesc_2_3@@UAEXIQBGW4ErrTypes@XMLErrorReporter@2@000JJ@Z 12066a50 f   XercesDOMParser.obj
 0001:00065b10       ?resolveEntity@XercesDOMParser@xercesc_2_3@@UAEPAVInputSource@2@QBG00@Z 12066b10 f   XercesDOMParser.obj
 0001:00065b30       ?loadGrammar@XercesDOMParser@xercesc_2_3@@QAEPAVGrammar@2@QBDF_N@Z 12066b30 f   XercesDOMParser.obj
 0001:00065be0       ?loadGrammar@XercesDOMParser@xercesc_2_3@@QAEPAVGrammar@2@QBGF_N@Z 12066be0 f   XercesDOMParser.obj
 0001:00065c90       ?loadGrammar@XercesDOMParser@xercesc_2_3@@QAEPAVGrammar@2@ABVInputSource@2@F_N@Z 12066c90 f   XercesDOMParser.obj
 0001:00065d40       ??_EXercesDOMParser@xercesc_2_3@@W3AEPAXI@Z 12066d40 f i XercesDOMParser.obj
 0001:00065d50       ??_EXercesDOMParser@xercesc_2_3@@W7AEPAXI@Z 12066d50 f i XercesDOMParser.obj
 0001:00065d60       ??_EXercesDOMParser@xercesc_2_3@@WM@AEPAXI@Z 12066d60 f i XercesDOMParser.obj
 0001:00065d70       ??0AllContentModel@xercesc_2_3@@QAE@QAVContentSpecNode@1@_NQAVMemoryManager@1@@Z 12066d70 f   AllContentModel.obj
 0001:00065fa0       ??_GAllContentModel@xercesc_2_3@@UAEPAXI@Z 12066fa0 f i AllContentModel.obj
 0001:00065fa0       ??_EAllContentModel@xercesc_2_3@@UAEPAXI@Z 12066fa0 f i AllContentModel.obj
 0001:00065fc0       ??1AllContentModel@xercesc_2_3@@UAE@XZ 12066fc0 f   AllContentModel.obj
 0001:00066020       ?validateContent@AllContentModel@xercesc_2_3@@UBEHQAPAVQName@2@II@Z 12067020 f   AllContentModel.obj
 0001:000661a0       ?validateContentSpecial@AllContentModel@xercesc_2_3@@UBEHQAPAVQName@2@IIQAVGrammarResolver@2@QAVXMLStringPool@2@@Z 120671a0 f   AllContentModel.obj
 0001:000662f0       ?checkUniqueParticleAttribution@AllContentModel@xercesc_2_3@@UAEXQAVSchemaGrammar@2@QAVGrammarResolver@2@QAVXMLStringPool@2@QAVXMLValidator@2@QAI@Z 120672f0 f   AllContentModel.obj
 0001:00066410       ?buildChildList@AllContentModel@xercesc_2_3@@AAEXQAVContentSpecNode@2@AAV?$ValueVectorOf@PAVQName@xercesc_2_3@@@2@AAV?$ValueVectorOf@_N@2@@Z 12067410 f   AllContentModel.obj
 0001:000665f0       ?ensureExtraCapacity@?$ValueVectorOf@_N@xercesc_2_3@@QAEXI@Z 120675f0 f i AllContentModel.obj
 0001:00066670       ??0CMAny@xercesc_2_3@@QAE@W4NodeTypes@ContentSpecNode@1@IIQAVMemoryManager@1@@Z 12067670 f   CMAny.obj
 0001:00066730       ??1CMNode@xercesc_2_3@@UAE@XZ 12067730 f i CMAny.obj
 0001:00066780       ??_GCMNode@xercesc_2_3@@UAEPAXI@Z 12067780 f i CMAny.obj
 0001:00066780       ??_ECMNode@xercesc_2_3@@UAEPAXI@Z 12067780 f i CMAny.obj
 0001:000667f0       ??_ECMAny@xercesc_2_3@@UAEPAXI@Z 120677f0 f i CMAny.obj
 0001:000667f0       ??_GCMAny@xercesc_2_3@@UAEPAXI@Z 120677f0 f i CMAny.obj
 0001:00066810       ??1CMAny@xercesc_2_3@@UAE@XZ 12067810 f   CMAny.obj
 0001:00066860       ?isNullable@CMAny@xercesc_2_3@@UBE_NXZ 12067860 f   CMAny.obj
 0001:00066870       ?calcFirstPos@CMAny@xercesc_2_3@@MBEXAAVCMStateSet@2@@Z 12067870 f   CMAny.obj
 0001:00066870       ?calcLastPos@CMAny@xercesc_2_3@@MBEXAAVCMStateSet@2@@Z 12067870 f   CMAny.obj
 0001:00066960       ??0CMBinaryOp@xercesc_2_3@@QAE@W4NodeTypes@ContentSpecNode@1@QAVCMNode@1@1QAVMemoryManager@1@@Z 12067960 f   CMBinaryOp.obj
 0001:00066a10       ??_ECMBinaryOp@xercesc_2_3@@UAEPAXI@Z 12067a10 f i CMBinaryOp.obj
 0001:00066a10       ??_GCMBinaryOp@xercesc_2_3@@UAEPAXI@Z 12067a10 f i CMBinaryOp.obj
 0001:00066a30       ??1CMBinaryOp@xercesc_2_3@@UAE@XZ 12067a30 f   CMBinaryOp.obj
 0001:00066ae0       ?isNullable@CMBinaryOp@xercesc_2_3@@UBE_NXZ 12067ae0 f   CMBinaryOp.obj
 0001:00066b30       ?calcFirstPos@CMBinaryOp@xercesc_2_3@@MBEXAAVCMStateSet@2@@Z 12067b30 f   CMBinaryOp.obj
 0001:00066cf0       ?getFirstPos@CMNode@xercesc_2_3@@QBEABVCMStateSet@2@XZ 12067cf0 f i CMBinaryOp.obj
 0001:00066dd0       ?calcLastPos@CMBinaryOp@xercesc_2_3@@MBEXAAVCMStateSet@2@@Z 12067dd0 f   CMBinaryOp.obj
 0001:00066f90       ?getLastPos@CMNode@xercesc_2_3@@QBEABVCMStateSet@2@XZ 12067f90 f i CMBinaryOp.obj
 0001:00067070       ??0CMUnaryOp@xercesc_2_3@@QAE@W4NodeTypes@ContentSpecNode@1@QAVCMNode@1@QAVMemoryManager@1@@Z 12068070 f   CMUnaryOp.obj
 0001:00067120       ??_ECMUnaryOp@xercesc_2_3@@UAEPAXI@Z 12068120 f i CMUnaryOp.obj
 0001:00067120       ??_GCMUnaryOp@xercesc_2_3@@UAEPAXI@Z 12068120 f i CMUnaryOp.obj
 0001:00067140       ??1CMUnaryOp@xercesc_2_3@@UAE@XZ 12068140 f   CMUnaryOp.obj
 0001:000671e0       ?isNullable@CMUnaryOp@xercesc_2_3@@UBE_NXZ 120681e0 f   CMUnaryOp.obj
 0001:00067200       ?calcFirstPos@CMUnaryOp@xercesc_2_3@@MBEXAAVCMStateSet@2@@Z 12068200 f   CMUnaryOp.obj
 0001:00067280       ?calcLastPos@CMUnaryOp@xercesc_2_3@@MBEXAAVCMStateSet@2@@Z 12068280 f   CMUnaryOp.obj
 0001:00067300       ??0ContentLeafNameTypeVector@xercesc_2_3@@QAE@QAVMemoryManager@1@@Z 12068300 f   ContentLeafNameTypeVector.obj
 0001:00067320       ??1ContentLeafNameTypeVector@xercesc_2_3@@QAE@XZ 12068320 f   ContentLeafNameTypeVector.obj
 0001:00067340       ?setValues@ContentLeafNameTypeVector@xercesc_2_3@@QAEXQAPAVQName@2@QAW4NodeTypes@ContentSpecNode@2@I@Z 12068340 f   ContentLeafNameTypeVector.obj
 0001:000673c0       ?getLeafNameAt@ContentLeafNameTypeVector@xercesc_2_3@@QBEPAVQName@2@I@Z 120683c0 f   ContentLeafNameTypeVector.obj
 0001:00067400       ?getLeafTypeAt@ContentLeafNameTypeVector@xercesc_2_3@@QBE?BW4NodeTypes@ContentSpecNode@2@I@Z 12068400 f   ContentLeafNameTypeVector.obj
 0001:00067440       ??0ContentSpecNode@xercesc_2_3@@QAE@ABV01@@Z 12068440 f   ContentSpecNode.obj
 0001:00067570       ?formatSpec@ContentSpecNode@xercesc_2_3@@QBEXAAVXMLBuffer@2@@Z 12068570 f   ContentSpecNode.obj
 0001:00067a40       ?getMinTotalRange@ContentSpecNode@xercesc_2_3@@QBEHXZ 12068a40 f   ContentSpecNode.obj
 0001:00067aa0       ?getMaxTotalRange@ContentSpecNode@xercesc_2_3@@QBEHXZ 12068aa0 f   ContentSpecNode.obj
 0001:00067b30       ??0HashCMStateSet@xercesc_2_3@@QAE@XZ 12068b30 f i DFAContentModel.obj
 0001:00067b40       ??_EHashCMStateSet@xercesc_2_3@@UAEPAXI@Z 12068b40 f i DFAContentModel.obj
 0001:00067ba0       ??1HashCMStateSet@xercesc_2_3@@UAE@XZ 12068ba0 f i DFAContentModel.obj
 0001:00067bb0       ?getHashVal@HashCMStateSet@xercesc_2_3@@UAEIQBXI@Z 12068bb0 f i DFAContentModel.obj
 0001:00067c00       ?equals@HashCMStateSet@xercesc_2_3@@UAE_NQBX0@Z 12068c00 f i DFAContentModel.obj
 0001:00067c60       ??0XMLInteger@xercesc_2_3@@QAE@H@Z 12068c60 f i DFAContentModel.obj
 0001:00067c60       ??6XMLFormatter@xercesc_2_3@@QAEAAV01@W4EscapeFlags@01@@Z 12068c60 f i DFAContentModel.obj
 0001:00067c70       ??0DFAContentModel@xercesc_2_3@@QAE@_NQAVContentSpecNode@1@QAVMemoryManager@1@@Z 12068c70 f   DFAContentModel.obj
 0001:00067d00       ?getNextState@DFAContentModel@xercesc_2_3@@UBEIII@Z 12068d00 f i DFAContentModel.obj
 0001:00067d60       ??_EDFAContentModel@xercesc_2_3@@UAEPAXI@Z 12068d60 f i DFAContentModel.obj
 0001:00067d60       ??_GDFAContentModel@xercesc_2_3@@UAEPAXI@Z 12068d60 f i DFAContentModel.obj
 0001:00067d80       ??0DFAContentModel@xercesc_2_3@@QAE@_NQAVContentSpecNode@1@0QAVMemoryManager@1@@Z 12068d80 f   DFAContentModel.obj
 0001:00067e10       ??1DFAContentModel@xercesc_2_3@@UAE@XZ 12068e10 f   DFAContentModel.obj
 0001:00067f00       ?validateContent@DFAContentModel@xercesc_2_3@@UBEHQAPAVQName@2@II@Z 12068f00 f   DFAContentModel.obj
 0001:00068150       ?validateContentSpecial@DFAContentModel@xercesc_2_3@@UBEHQAPAVQName@2@IIQAVGrammarResolver@2@QAVXMLStringPool@2@@Z 12069150 f   DFAContentModel.obj
 0001:000682c0       ?buildDFA@DFAContentModel@xercesc_2_3@@AAEXQAVContentSpecNode@2@@Z 120692c0 f   DFAContentModel.obj
 0001:00069360       ?zeroBits@CMStateSet@xercesc_2_3@@QAEXXZ 1206a360 f i DFAContentModel.obj
 0001:00069390       ??_GCMLeaf@xercesc_2_3@@UAEPAXI@Z 1206a390 f i DFAContentModel.obj
 0001:00069390       ??_ECMLeaf@xercesc_2_3@@UAEPAXI@Z 1206a390 f i DFAContentModel.obj
 0001:000693b0       ??1CMLeaf@xercesc_2_3@@UAE@XZ 1206a3b0 f i DFAContentModel.obj
 0001:00069460       ?isNullable@CMLeaf@xercesc_2_3@@UBE_NXZ 1206a460 f i DFAContentModel.obj
 0001:00069470       ?calcLastPos@CMLeaf@xercesc_2_3@@MBEXAAVCMStateSet@2@@Z 1206a470 f i DFAContentModel.obj
 0001:00069470       ?calcFirstPos@CMLeaf@xercesc_2_3@@MBEXAAVCMStateSet@2@@Z 1206a470 f i DFAContentModel.obj
 0001:00069560       ?buildSyntaxTree@DFAContentModel@xercesc_2_3@@AAEPAVCMNode@2@QAVContentSpecNode@2@@Z 1206a560 f   DFAContentModel.obj
 0001:000697c0       ?calcFollowList@DFAContentModel@xercesc_2_3@@AAEXQAVCMNode@2@@Z 1206a7c0 f   DFAContentModel.obj
 0001:00069a30       ?postTreeBuildInit@DFAContentModel@xercesc_2_3@@AAEHQAVCMNode@2@I@Z 1206aa30 f   DFAContentModel.obj
 0001:00069d30       ?checkUniqueParticleAttribution@DFAContentModel@xercesc_2_3@@UAEXQAVSchemaGrammar@2@QAVGrammarResolver@2@QAVXMLStringPool@2@QAVXMLValidator@2@QAI@Z 1206ad30 f   DFAContentModel.obj
 0001:0006a090       ??0GrammarResolver@xercesc_2_3@@QAE@QAVMemoryManager@1@@Z 1206b090 f   GrammarResolver.obj
 0001:0006a180       ??1GrammarResolver@xercesc_2_3@@QAE@XZ 1206b180 f   GrammarResolver.obj
 0001:0006a2e0       ?getDatatypeValidator@GrammarResolver@xercesc_2_3@@QAEPAVDatatypeValidator@2@QBG0@Z 1206b2e0 f   GrammarResolver.obj
 0001:0006a580       ?getGrammar@GrammarResolver@xercesc_2_3@@QAEPAVGrammar@2@QBG@Z 1206b580 f   GrammarResolver.obj
 0001:0006a6a0       ?getGrammarEnumerator@GrammarResolver@xercesc_2_3@@QBE?AV?$RefHashTableOfEnumerator@VGrammar@xercesc_2_3@@@2@XZ 1206b6a0 f   GrammarResolver.obj
 0001:0006a760       ?containsNameSpace@GrammarResolver@xercesc_2_3@@QAE_NQBG@Z 1206b760 f   GrammarResolver.obj
 0001:0006a7e0       ?putGrammar@GrammarResolver@xercesc_2_3@@QAEXQBGQAVGrammar@2@@Z 1206b7e0 f   GrammarResolver.obj
 0001:0006a810       ?reset@GrammarResolver@xercesc_2_3@@QAEXXZ 1206b810 f   GrammarResolver.obj
 0001:0006a880       ?resetCachedGrammar@GrammarResolver@xercesc_2_3@@QAEXXZ 1206b880 f   GrammarResolver.obj
 0001:0006a8f0       ?cacheGrammars@GrammarResolver@xercesc_2_3@@QAEXXZ 1206b8f0 f   GrammarResolver.obj
 0001:0006ac70       ?cacheGrammarFromParse@GrammarResolver@xercesc_2_3@@QAEX_N@Z 1206bc70 f   GrammarResolver.obj
 0001:0006ade0       ??1?$XMLEnumerator@VGrammar@xercesc_2_3@@@xercesc_2_3@@UAE@XZ 1206bde0 f i GrammarResolver.obj
 0001:0006adf0       ??_G?$XMLEnumerator@VGrammar@xercesc_2_3@@@xercesc_2_3@@UAEPAXI@Z 1206bdf0 f i GrammarResolver.obj
 0001:0006adf0       ??_E?$XMLEnumerator@VGrammar@xercesc_2_3@@@xercesc_2_3@@UAEPAXI@Z 1206bdf0 f i GrammarResolver.obj
 0001:0006ae10       ?get@?$RefHashTableOf@VComplexTypeInfo@xercesc_2_3@@@xercesc_2_3@@QAEPAVComplexTypeInfo@2@QBX@Z 1206be10 f i GrammarResolver.obj
 0001:0006ae10       ?get@?$RefHashTableOf@V?$ValueVectorOf@PAVSchemaElementDecl@xercesc_2_3@@@xercesc_2_3@@@xercesc_2_3@@QAEPAV?$ValueVectorOf@PAVSchemaElementDecl@xercesc_2_3@@@2@QBX@Z 1206be10 f i GrammarResolver.obj
 0001:0006ae10       ?get@?$RefHashTableOf@VDatatypeValidator@xercesc_2_3@@@xercesc_2_3@@QAEPAVDatatypeValidator@2@QBX@Z 1206be10 f i GrammarResolver.obj
 0001:0006ae10       ?get@?$RefHashTableOf@V?$ValueVectorOf@I@xercesc_2_3@@@xercesc_2_3@@QAEPAV?$ValueVectorOf@I@2@QBX@Z 1206be10 f i GrammarResolver.obj
 0001:0006ae10       ?get@?$RefHashTableOf@G@xercesc_2_3@@QAEPAGQBX@Z 1206be10 f i GrammarResolver.obj
 0001:0006ae10       ?get@?$RefHashTableOf@VGrammar@xercesc_2_3@@@xercesc_2_3@@QAEPAVGrammar@2@QBX@Z 1206be10 f i GrammarResolver.obj
 0001:0006ae10       ?get@?$RefHashTableOf@VXercesAttGroupInfo@xercesc_2_3@@@xercesc_2_3@@QAEPAVXercesAttGroupInfo@2@QBX@Z 1206be10 f i GrammarResolver.obj
 0001:0006aea0       ?put@?$RefHashTableOf@VGrammar@xercesc_2_3@@@xercesc_2_3@@QAEXPAXQAVGrammar@2@@Z 1206bea0 f i GrammarResolver.obj
 0001:0006b0b0       ??1?$RefHashTableOfEnumerator@VGrammar@xercesc_2_3@@@xercesc_2_3@@UAE@XZ 1206c0b0 f i GrammarResolver.obj
 0001:0006b1a0       ??_G?$RefHashTableOfEnumerator@VGrammar@xercesc_2_3@@@xercesc_2_3@@UAEPAXI@Z 1206c1a0 f i GrammarResolver.obj
 0001:0006b1a0       ??_E?$RefHashTableOfEnumerator@VGrammar@xercesc_2_3@@@xercesc_2_3@@UAEPAXI@Z 1206c1a0 f i GrammarResolver.obj
 0001:0006b1c0       ??0MixedContentModel@xercesc_2_3@@QAE@_NQAVContentSpecNode@1@0QAVMemoryManager@1@@Z 1206c1c0 f   MixedContentModel.obj
 0001:0006b3f0       ?checkUniqueParticleAttribution@MixedContentModel@xercesc_2_3@@UAEXQAVSchemaGrammar@2@QAVGrammarResolver@2@QAVXMLStringPool@2@QAVXMLValidator@2@QAI@Z 1206c3f0 f i MixedContentModel.obj
 0001:0006b440       ??_GMixedContentModel@xercesc_2_3@@UAEPAXI@Z 1206c440 f i MixedContentModel.obj
 0001:0006b440       ??_EMixedContentModel@xercesc_2_3@@UAEPAXI@Z 1206c440 f i MixedContentModel.obj
 0001:0006b460       ??1MixedContentModel@xercesc_2_3@@UAE@XZ 1206c460 f   MixedContentModel.obj
 0001:0006b4c0       ?hasDups@MixedContentModel@xercesc_2_3@@QBE_NXZ 1206c4c0 f   MixedContentModel.obj
 0001:0006b5d0       ?validateContent@MixedContentModel@xercesc_2_3@@UBEHQAPAVQName@2@II@Z 1206c5d0 f   MixedContentModel.obj
 0001:0006b880       ?validateContentSpecial@MixedContentModel@xercesc_2_3@@UBEHQAPAVQName@2@IIQAVGrammarResolver@2@QAVXMLStringPool@2@@Z 1206c880 f   MixedContentModel.obj
 0001:0006b9f0       ?buildChildList@MixedContentModel@xercesc_2_3@@AAEXQAVContentSpecNode@2@AAV?$ValueVectorOf@PAVQName@xercesc_2_3@@@2@AAV?$ValueVectorOf@W4NodeTypes@ContentSpecNode@xercesc_2_3@@@2@@Z 1206c9f0 f   MixedContentModel.obj
 0001:0006bb80       ?validateContent@SimpleContentModel@xercesc_2_3@@UBEHQAPAVQName@2@II@Z 1206cb80 f   SimpleContentModel.obj
 0001:0006c3b0       ?validateContentSpecial@SimpleContentModel@xercesc_2_3@@UBEHQAPAVQName@2@IIQAVGrammarResolver@2@QAVXMLStringPool@2@@Z 1206d3b0 f   SimpleContentModel.obj
 0001:0006c870       ?checkUniqueParticleAttribution@SimpleContentModel@xercesc_2_3@@UAEXQAVSchemaGrammar@2@QAVGrammarResolver@2@QAVXMLStringPool@2@QAVXMLValidator@2@QAI@Z 1206d870 f   SimpleContentModel.obj
 0001:0006c950       ?getEntityHandler@XMLScanner@xercesc_2_3@@QBEPBVXMLEntityHandler@2@XZ 1206d950 f i AbstractNumericFacetValidator.obj
 0001:0006c950       ?getEnumeration@AbstractStringValidator@xercesc_2_3@@QBEPAV?$RefArrayVectorOf@G@2@XZ 1206d950 f i AbstractNumericFacetValidator.obj
 0001:0006c950       ?getMinInclusive@AbstractNumericFacetValidator@xercesc_2_3@@QBEQAVXMLNumber@2@XZ 1206d950 f i AbstractNumericFacetValidator.obj
 0001:0006c950       ?getScanner@SAXParser@xercesc_2_3@@IBEABVXMLScanner@2@XZ 1206d950 f i AbstractNumericFacetValidator.obj
 0001:0006c950       ?getEntityHandler@XMLScanner@xercesc_2_3@@QAEPAVXMLEntityHandler@2@XZ 1206d950 f i AbstractNumericFacetValidator.obj
 0001:0006c960       ?getErrorHandler@XMLScanner@xercesc_2_3@@QBEPBVErrorHandler@2@XZ 1206d960 f i AbstractNumericFacetValidator.obj
 0001:0006c960       ?getEnumeration@AbstractNumericFacetValidator@xercesc_2_3@@QBEPAV?$RefVectorOf@VXMLNumber@xercesc_2_3@@@2@XZ 1206d960 f i AbstractNumericFacetValidator.obj
 0001:0006c960       ?getEntityResolver@SAX2XMLReaderImpl@xercesc_2_3@@UBEPAVEntityResolver@2@XZ 1206d960 f i AbstractNumericFacetValidator.obj
 0001:0006c960       ?getErrorHandler@XMLScanner@xercesc_2_3@@QAEPAVErrorHandler@2@XZ 1206d960 f i AbstractNumericFacetValidator.obj
 0001:0006c960       ?getValidity@SchemaElementDecl@xercesc_2_3@@QBE?AW4Validity@PSVIDefs@2@XZ 1206d960 f i AbstractNumericFacetValidator.obj
 0001:0006c970       ??0InvalidDatatypeFacetException@xercesc_2_3@@QAE@QBDIW4Codes@XMLExcepts@1@@Z 1206d970 f i AbstractNumericFacetValidator.obj
 0001:0006c9d0       ??0InvalidDatatypeFacetException@xercesc_2_3@@QAE@ABV01@@Z 1206d9d0 f i AbstractNumericFacetValidator.obj
 0001:0006c9f0       ??0InvalidDatatypeFacetException@xercesc_2_3@@QAE@QBDIW4Codes@XMLExcepts@1@QBG222@Z 1206d9f0 f i AbstractNumericFacetValidator.obj
 0001:0006ca60       ??0InvalidDatatypeFacetException@xercesc_2_3@@QAE@QBDIW4Codes@XMLExcepts@1@0000@Z 1206da60 f i AbstractNumericFacetValidator.obj
 0001:0006cad0       ??1InvalidDatatypeFacetException@xercesc_2_3@@UAE@XZ 1206dad0 f i AbstractNumericFacetValidator.obj
 0001:0006cae0       ?duplicate@InvalidDatatypeFacetException@xercesc_2_3@@UBEPAVXMLException@2@XZ 1206dae0 f i AbstractNumericFacetValidator.obj
 0001:0006cb40       ?getType@InvalidDatatypeFacetException@xercesc_2_3@@UBEPBGXZ 1206db40 f i AbstractNumericFacetValidator.obj
 0001:0006cb50       ??_EInvalidDatatypeFacetException@xercesc_2_3@@UAEPAXI@Z 1206db50 f i AbstractNumericFacetValidator.obj
 0001:0006cbb0       ??1AbstractNumericFacetValidator@xercesc_2_3@@UAE@XZ 1206dbb0 f   AbstractNumericFacetValidator.obj
 0001:0006cc80       ??_EAbstractNumericFacetValidator@xercesc_2_3@@UAEPAXI@Z 1206dc80 f i AbstractNumericFacetValidator.obj
 0001:0006cce0       ??0AbstractNumericFacetValidator@xercesc_2_3@@IAE@QAVDatatypeValidator@1@QAV?$RefHashTableOf@VKVStringPair@xercesc_2_3@@@1@HW4ValidatorType@21@QAVMemoryManager@1@@Z 1206dce0 f   AbstractNumericFacetValidator.obj
 0001:0006cd40       ?init@AbstractNumericFacetValidator@xercesc_2_3@@IAEXQAV?$RefArrayVectorOf@G@2@@Z 1206dd40 f   AbstractNumericFacetValidator.obj
 0001:0006cd80       ?assignFacet@AbstractNumericFacetValidator@xercesc_2_3@@AAEXXZ 1206dd80 f   AbstractNumericFacetValidator.obj
 0001:0006d300       ?inspectFacet@AbstractNumericFacetValidator@xercesc_2_3@@AAEXXZ 1206e300 f   AbstractNumericFacetValidator.obj
 0001:0006d530       ?inspectFacetBase@AbstractNumericFacetValidator@xercesc_2_3@@AAEXXZ 1206e530 f   AbstractNumericFacetValidator.obj
 0001:0006e2e0       ?inheritFacet@AbstractNumericFacetValidator@xercesc_2_3@@AAEXXZ 1206f2e0 f   AbstractNumericFacetValidator.obj
 0001:0006e3a0       ?getEnumString@AbstractNumericFacetValidator@xercesc_2_3@@UBEPBV?$RefArrayVectorOf@G@2@XZ 1206f3a0 f   AbstractNumericFacetValidator.obj
 0001:0006e3c0       ??1?$XMLEnumerator@VKVStringPair@xercesc_2_3@@@xercesc_2_3@@UAE@XZ 1206f3c0 f i AbstractNumericFacetValidator.obj
 0001:0006e3d0       ??_E?$XMLEnumerator@VKVStringPair@xercesc_2_3@@@xercesc_2_3@@UAEPAXI@Z 1206f3d0 f i AbstractNumericFacetValidator.obj
 0001:0006e3d0       ??_G?$XMLEnumerator@VKVStringPair@xercesc_2_3@@@xercesc_2_3@@UAEPAXI@Z 1206f3d0 f i AbstractNumericFacetValidator.obj
 0001:0006e3f0       ??1?$RefHashTableOfEnumerator@VKVStringPair@xercesc_2_3@@@xercesc_2_3@@UAE@XZ 1206f3f0 f i AbstractNumericFacetValidator.obj
 0001:0006e4e0       ??_G?$RefHashTableOfEnumerator@VKVStringPair@xercesc_2_3@@@xercesc_2_3@@UAEPAXI@Z 1206f4e0 f i AbstractNumericFacetValidator.obj
 0001:0006e4e0       ??_E?$RefHashTableOfEnumerator@VKVStringPair@xercesc_2_3@@@xercesc_2_3@@UAEPAXI@Z 1206f4e0 f i AbstractNumericFacetValidator.obj
 0001:0006e500       ?init@AbstractNumericValidator@xercesc_2_3@@IAEXQAV?$RefArrayVectorOf@G@2@@Z 1206f500 f i AbstractNumericValidator.obj
 0001:0006e510       ??0InvalidDatatypeValueException@xercesc_2_3@@QAE@QBDIW4Codes@XMLExcepts@1@@Z 1206f510 f i AbstractNumericValidator.obj
 0001:0006e570       ??0InvalidDatatypeValueException@xercesc_2_3@@QAE@ABV01@@Z 1206f570 f i AbstractNumericValidator.obj
 0001:0006e590       ??0InvalidDatatypeValueException@xercesc_2_3@@QAE@QBDIW4Codes@XMLExcepts@1@QBG222@Z 1206f590 f i AbstractNumericValidator.obj
 0001:0006e600       ??0InvalidDatatypeValueException@xercesc_2_3@@QAE@QBDIW4Codes@XMLExcepts@1@0000@Z 1206f600 f i AbstractNumericValidator.obj
 0001:0006e670       ??1InvalidDatatypeValueException@xercesc_2_3@@UAE@XZ 1206f670 f i AbstractNumericValidator.obj
 0001:0006e680       ?duplicate@InvalidDatatypeValueException@xercesc_2_3@@UBEPAVXMLException@2@XZ 1206f680 f i AbstractNumericValidator.obj
 0001:0006e6e0       ?getType@InvalidDatatypeValueException@xercesc_2_3@@UBEPBGXZ 1206f6e0 f i AbstractNumericValidator.obj
 0001:0006e6f0       ??_EInvalidDatatypeValueException@xercesc_2_3@@UAEPAXI@Z 1206f6f0 f i AbstractNumericValidator.obj
 0001:0006e750       ??1AbstractNumericValidator@xercesc_2_3@@UAE@XZ 1206f750 f   AbstractNumericValidator.obj
 0001:0006e760       ??_EAbstractNumericValidator@xercesc_2_3@@UAEPAXI@Z 1206f760 f i AbstractNumericValidator.obj
 0001:0006e7c0       ??0AbstractNumericValidator@xercesc_2_3@@IAE@QAVDatatypeValidator@1@QAV?$RefHashTableOf@VKVStringPair@xercesc_2_3@@@1@HW4ValidatorType@21@QAVMemoryManager@1@@Z 1206f7c0 f   AbstractNumericValidator.obj
 0001:0006e7f0       ?boundsCheck@AbstractNumericValidator@xercesc_2_3@@IAEXQBVXMLNumber@2@@Z 1206f7f0 f   AbstractNumericValidator.obj
 0001:0006ea40       ??1AbstractStringValidator@xercesc_2_3@@UAE@XZ 1206fa40 f   AbstractStringValidator.obj
 0001:0006eab0       ??_EAbstractStringValidator@xercesc_2_3@@UAEPAXI@Z 1206fab0 f i AbstractStringValidator.obj
 0001:0006eb10       ??0AbstractStringValidator@xercesc_2_3@@IAE@QAVDatatypeValidator@1@QAV?$RefHashTableOf@VKVStringPair@xercesc_2_3@@@1@HW4ValidatorType@21@QAVMemoryManager@1@@Z 1206fb10 f   AbstractStringValidator.obj
 0001:0006eb60       ?init@AbstractStringValidator@xercesc_2_3@@IAEXQAV?$RefArrayVectorOf@G@2@@Z 1206fb60 f   AbstractStringValidator.obj
 0001:0006ebc0       ?assignFacet@AbstractStringValidator@xercesc_2_3@@AAEXXZ 1206fbc0 f   AbstractStringValidator.obj
 0001:0006f190       ?inspectFacet@AbstractStringValidator@xercesc_2_3@@AAEXXZ 12070190 f   AbstractStringValidator.obj
 0001:0006f270       ?inspectFacetBase@AbstractStringValidator@xercesc_2_3@@MAEXXZ 12070270 f   AbstractStringValidator.obj
 0001:0006f810       ?inheritFacet@AbstractStringValidator@xercesc_2_3@@MAEXXZ 12070810 f   AbstractStringValidator.obj
 0001:0006f8b0       ?compare@AbstractStringValidator@xercesc_2_3@@UAEHQBG0@Z 120708b0 f   AbstractStringValidator.obj
 0001:0006f8d0       ?validate@AbstractStringValidator@xercesc_2_3@@UAEXQBG@Z 120708d0 f   AbstractStringValidator.obj
 0001:0006f8e0       ?checkContent@AbstractStringValidator@xercesc_2_3@@MAEXQBG_N@Z 120708e0 f   AbstractStringValidator.obj
 0001:0006fd90       ?getRanges@DocumentImpl@xercesc_2_3@@UAEPAV?$RefVectorOf@VRangeImpl@xercesc_2_3@@@2@XZ 12070d90 f   AbstractStringValidator.obj
 0001:0006fd90       ?getEnumString@AbstractStringValidator@xercesc_2_3@@UBEPBV?$RefArrayVectorOf@G@2@XZ 12070d90 f   AbstractStringValidator.obj
 0001:0006fda0       ??_FAnySimpleTypeDatatypeValidator@xercesc_2_3@@QAEXXZ 12070da0 f i AnySimpleTypeDatatypeValidator.obj
 0001:0006fdb0       ?compare@AnySimpleTypeDatatypeValidator@xercesc_2_3@@UAEHQBG0@Z 12070db0 f i AnySimpleTypeDatatypeValidator.obj
 0001:0006fdc0       ?isSubstitutableBy@AnySimpleTypeDatatypeValidator@xercesc_2_3@@UAE_NQBVDatatypeValidator@2@@Z 12070dc0 f i AnySimpleTypeDatatypeValidator.obj
 0001:0006fdc0       ?checkRootElement@XMLValidator@xercesc_2_3@@QAE_NI@Z 12070dc0 f i AnySimpleTypeDatatypeValidator.obj
 0001:0006fdd0       ??0AnySimpleTypeDatatypeValidator@xercesc_2_3@@QAE@QAVMemoryManager@1@@Z 12070dd0 f   AnySimpleTypeDatatypeValidator.obj
 0001:0006fe00       ??_EAnySimpleTypeDatatypeValidator@xercesc_2_3@@UAEPAXI@Z 12070e00 f i AnySimpleTypeDatatypeValidator.obj
 0001:0006fe60       ??1AnySimpleTypeDatatypeValidator@xercesc_2_3@@UAE@XZ 12070e60 f   AnySimpleTypeDatatypeValidator.obj
 0001:0006fe70       ?newInstance@AnySimpleTypeDatatypeValidator@xercesc_2_3@@UAEPAVDatatypeValidator@2@QAV?$RefHashTableOf@VKVStringPair@xercesc_2_3@@@2@QAV?$RefArrayVectorOf@G@2@HQAVMemoryManager@2@@Z 12070e70 f   AnySimpleTypeDatatypeValidator.obj
 0001:0006ff40       ??_FAnyURIDatatypeValidator@xercesc_2_3@@QAEXXZ 12070f40 f i AnyURIDatatypeValidator.obj
 0001:0006ff50       ?cleanUp@AnyURIDatatypeValidator@xercesc_2_3@@AAEXXZ 12070f50 f i AnyURIDatatypeValidator.obj
 0001:0006ff70       ??0AnyURIDatatypeValidator@xercesc_2_3@@QAE@QAVMemoryManager@1@@Z 12070f70 f   AnyURIDatatypeValidator.obj
 0001:0006ffa0       ??_EAnyURIDatatypeValidator@xercesc_2_3@@UAEPAXI@Z 12070fa0 f i AnyURIDatatypeValidator.obj
 0001:00070000       ??1AnyURIDatatypeValidator@xercesc_2_3@@UAE@XZ 12071000 f   AnyURIDatatypeValidator.obj
 0001:00070060       ??0AnyURIDatatypeValidator@xercesc_2_3@@QAE@QAVDatatypeValidator@1@QAV?$RefHashTableOf@VKVStringPair@xercesc_2_3@@@1@QAV?$RefArrayVectorOf@G@1@HQAVMemoryManager@1@@Z 12071060 f   AnyURIDatatypeValidator.obj
 0001:000700f0       ?newInstance@AnyURIDatatypeValidator@xercesc_2_3@@UAEPAVDatatypeValidator@2@QAV?$RefHashTableOf@VKVStringPair@xercesc_2_3@@@2@QAV?$RefArrayVectorOf@G@2@HQAVMemoryManager@2@@Z 120710f0 f   AnyURIDatatypeValidator.obj
 0001:00070170       ?assignAdditionalFacet@AnyURIDatatypeValidator@xercesc_2_3@@MAEXQBG0@Z 12071170 f   AnyURIDatatypeValidator.obj
 0001:000701b0       ?getLength@AnyURIDatatypeValidator@xercesc_2_3@@MBEHQBG@Z 120711b0 f   AnyURIDatatypeValidator.obj
 0001:000701b0       ?getLength@QNameDatatypeValidator@xercesc_2_3@@MBEHQBG@Z 120711b0 f   AnyURIDatatypeValidator.obj
 0001:000701b0       ?getLength@StringDatatypeValidator@xercesc_2_3@@MBEHQBG@Z 120711b0 f   AnyURIDatatypeValidator.obj
 0001:000701b0       ?getLength@NOTATIONDatatypeValidator@xercesc_2_3@@MBEHQBG@Z 120711b0 f   AnyURIDatatypeValidator.obj
 0001:000701e0       ?checkValueSpace@AnyURIDatatypeValidator@xercesc_2_3@@MAEXQBG@Z 120711e0 f   AnyURIDatatypeValidator.obj
 0001:000702e0       ??_FBase64BinaryDatatypeValidator@xercesc_2_3@@QAEXXZ 120712e0 f i Base64BinaryDatatypeValidator.obj
 0001:000702f0       ??0Base64BinaryDatatypeValidator@xercesc_2_3@@QAE@QAVMemoryManager@1@@Z 120712f0 f   Base64BinaryDatatypeValidator.obj
 0001:00070320       ??_EBase64BinaryDatatypeValidator@xercesc_2_3@@UAEPAXI@Z 12071320 f i Base64BinaryDatatypeValidator.obj
 0001:00070380       ??1Base64BinaryDatatypeValidator@xercesc_2_3@@UAE@XZ 12071380 f   Base64BinaryDatatypeValidator.obj
 0001:00070390       ??0Base64BinaryDatatypeValidator@xercesc_2_3@@QAE@QAVDatatypeValidator@1@QAV?$RefHashTableOf@VKVStringPair@xercesc_2_3@@@1@QAV?$RefArrayVectorOf@G@1@HQAVMemoryManager@1@@Z 12071390 f   Base64BinaryDatatypeValidator.obj
 0001:00070400       ?newInstance@Base64BinaryDatatypeValidator@xercesc_2_3@@UAEPAVDatatypeValidator@2@QAV?$RefHashTableOf@VKVStringPair@xercesc_2_3@@@2@QAV?$RefArrayVectorOf@G@2@HQAVMemoryManager@2@@Z 12071400 f   Base64BinaryDatatypeValidator.obj
 0001:00070480       ?assignAdditionalFacet@Base64BinaryDatatypeValidator@xercesc_2_3@@MAEXQBG0@Z 12071480 f   Base64BinaryDatatypeValidator.obj
 0001:000704c0       ?checkValueSpace@Base64BinaryDatatypeValidator@xercesc_2_3@@MAEXQBG@Z 120714c0 f   Base64BinaryDatatypeValidator.obj
 0001:00070510       ?getLength@Base64BinaryDatatypeValidator@xercesc_2_3@@MBEHQBG@Z 12071510 f   Base64BinaryDatatypeValidator.obj
 0001:00070520       ?normalizeEnumeration@Base64BinaryDatatypeValidator@xercesc_2_3@@MAEXXZ 12071520 f   Base64BinaryDatatypeValidator.obj
 0001:00070580       ?normalizeContent@Base64BinaryDatatypeValidator@xercesc_2_3@@MBEXQAG@Z 12071580 f   Base64BinaryDatatypeValidator.obj
 0001:00070590       ??_FBooleanDatatypeValidator@xercesc_2_3@@QAEXXZ 12071590 f i BooleanDatatypeValidator.obj
 0001:000705a0       ??0BooleanDatatypeValidator@xercesc_2_3@@QAE@QAVMemoryManager@1@@Z 120715a0 f i BooleanDatatypeValidator.obj
 0001:000705d0       ??_EBooleanDatatypeValidator@xercesc_2_3@@UAEPAXI@Z 120715d0 f i BooleanDatatypeValidator.obj
 0001:00070630       ??1BooleanDatatypeValidator@xercesc_2_3@@UAE@XZ 12071630 f i BooleanDatatypeValidator.obj
 0001:00070640       ?newInstance@BooleanDatatypeValidator@xercesc_2_3@@UAEPAVDatatypeValidator@2@QAV?$RefHashTableOf@VKVStringPair@xercesc_2_3@@@2@QAV?$RefArrayVectorOf@G@2@HQAVMemoryManager@2@@Z 12071640 f i BooleanDatatypeValidator.obj
 0001:000706c0       ?validate@BooleanDatatypeValidator@xercesc_2_3@@UAEXQBG@Z 120716c0 f i BooleanDatatypeValidator.obj
 0001:000706d0       ??0BooleanDatatypeValidator@xercesc_2_3@@QAE@QAVDatatypeValidator@1@QAV?$RefHashTableOf@VKVStringPair@xercesc_2_3@@@1@QAV?$RefArrayVectorOf@G@1@HQAVMemoryManager@1@@Z 120716d0 f   BooleanDatatypeValidator.obj
 0001:00070990       ?checkContent@BooleanDatatypeValidator@xercesc_2_3@@AAEXQBG_N@Z 12071990 f   BooleanDatatypeValidator.obj
 0001:00070b70       ?compare@BooleanDatatypeValidator@xercesc_2_3@@UAEHQBG0@Z 12071b70 f   BooleanDatatypeValidator.obj
 0001:00070e40       ??1?$RefHashTableOf@VKVStringPair@xercesc_2_3@@@xercesc_2_3@@QAE@XZ 12071e40 f i BooleanDatatypeValidator.obj
 0001:00070ed0       ??0DatatypeValidator@xercesc_2_3@@IAE@QAV01@QAV?$RefHashTableOf@VKVStringPair@xercesc_2_3@@@1@HW4ValidatorType@01@QAVMemoryManager@1@@Z 12071ed0 f   DatatypeValidator.obj
 0001:00070f20       ??_EDatatypeValidator@xercesc_2_3@@UAEPAXI@Z 12071f20 f i DatatypeValidator.obj
 0001:00071060       ??1DatatypeValidator@xercesc_2_3@@UAE@XZ 12072060 f   DatatypeValidator.obj
 0001:00071150       ?getWSstring@DatatypeValidator@xercesc_2_3@@IBEPBGF@Z 12072150 f   DatatypeValidator.obj
 0001:00071180       ?setTypeName@DatatypeValidator@xercesc_2_3@@QAEXQBG0@Z 12072180 f   DatatypeValidator.obj
 0001:00071280       ?setTypeName@DatatypeValidator@xercesc_2_3@@QAEXQBG@Z 12072280 f   DatatypeValidator.obj
 0001:00071340       ?cleanUp@DatatypeValidator@xercesc_2_3@@AAEXXZ 12072340 f   DatatypeValidator.obj
 0001:00071420       ??_FDecimalDatatypeValidator@xercesc_2_3@@QAEXXZ 12072420 f i DatatypeValidatorFactory.obj
 0001:00071430       ?getLexicalHandler@SAX2XMLReaderImpl@xercesc_2_3@@UBEPAVLexicalHandler@2@XZ 12072430 f i DatatypeValidatorFactory.obj
 0001:00071430       ?getTotalDigits@DecimalDatatypeValidator@xercesc_2_3@@QBEIXZ 12072430 f i DatatypeValidatorFactory.obj
 0001:00071430       ?getEntityResolver@XercesDOMParser@xercesc_2_3@@QBEPBVEntityResolver@2@XZ 12072430 f i DatatypeValidatorFactory.obj
 0001:00071430       ?getEntityResolver@XercesDOMParser@xercesc_2_3@@QAEPAVEntityResolver@2@XZ 12072430 f i DatatypeValidatorFactory.obj
 0001:00071440       ?getErrorHandler@XercesDOMParser@xercesc_2_3@@QBEPBVErrorHandler@2@XZ 12072440 f i DatatypeValidatorFactory.obj
 0001:00071440       ?getFractionDigits@DecimalDatatypeValidator@xercesc_2_3@@QBEIXZ 12072440 f i DatatypeValidatorFactory.obj
 0001:00071440       ?getErrorHandler@XercesDOMParser@xercesc_2_3@@QAEPAVErrorHandler@2@XZ 12072440 f i DatatypeValidatorFactory.obj
 0001:00071440       ?getDeclarationHandler@SAX2XMLReaderImpl@xercesc_2_3@@UBEPAVDeclHandler@2@XZ 12072440 f i DatatypeValidatorFactory.obj
 0001:00071450       ?setTotalDigits@DecimalDatatypeValidator@xercesc_2_3@@AAEXI@Z 12072450 f i DatatypeValidatorFactory.obj
 0001:00071460       ?setFractionDigits@DecimalDatatypeValidator@xercesc_2_3@@AAEXI@Z 12072460 f i DatatypeValidatorFactory.obj
 0001:00071470       ??_FHexBinaryDatatypeValidator@xercesc_2_3@@QAEXXZ 12072470 f i DatatypeValidatorFactory.obj
 0001:00071480       ??_FIDREFDatatypeValidator@xercesc_2_3@@QAEXXZ 12072480 f i DatatypeValidatorFactory.obj
 0001:00071490       ??_FNOTATIONDatatypeValidator@xercesc_2_3@@QAEXXZ 12072490 f i DatatypeValidatorFactory.obj
 0001:000714a0       ??_FENTITYDatatypeValidator@xercesc_2_3@@QAEXXZ 120724a0 f i DatatypeValidatorFactory.obj
 0001:000714b0       ?setErrorHandler@XMLScanner@xercesc_2_3@@QAEXQAVErrorHandler@2@@Z 120724b0 f i DatatypeValidatorFactory.obj
 0001:000714b0       ?setEntityDeclPool@ENTITYDatatypeValidator@xercesc_2_3@@QAEXQAV?$NameIdPool@VDTDEntityDecl@xercesc_2_3@@@2@@Z 120724b0 f i DatatypeValidatorFactory.obj
 0001:000714b0       ?setValidity@SchemaElementDecl@xercesc_2_3@@QAEXW4Validity@PSVIDefs@2@@Z 120724b0 f i DatatypeValidatorFactory.obj
 0001:000714b0       ?setIDRefList@IDREFDatatypeValidator@xercesc_2_3@@QAEXPAV?$RefHashTableOf@VXMLRefInfo@xercesc_2_3@@@2@@Z 120724b0 f i DatatypeValidatorFactory.obj
 0001:000714b0       ?setIDRefList@IDDatatypeValidator@xercesc_2_3@@QAEXPAV?$RefHashTableOf@VXMLRefInfo@xercesc_2_3@@@2@@Z 120724b0 f i DatatypeValidatorFactory.obj
 0001:000714c0       ??_FQNameDatatypeValidator@xercesc_2_3@@QAEXXZ 120724c0 f i DatatypeValidatorFactory.obj
 0001:000714d0       ??_FNameDatatypeValidator@xercesc_2_3@@QAEXXZ 120724d0 f i DatatypeValidatorFactory.obj
 0001:000714e0       ??_FNCNameDatatypeValidator@xercesc_2_3@@QAEXXZ 120724e0 f i DatatypeValidatorFactory.obj
 0001:000714f0       ??_FListDatatypeValidator@xercesc_2_3@@QAEXXZ 120724f0 f i DatatypeValidatorFactory.obj
 0001:00071500       ?getSubstitutionGroupElem@SchemaElementDecl@xercesc_2_3@@QBEPAV12@XZ 12072500 f i DatatypeValidatorFactory.obj
 0001:00071500       ?getContent@ListDatatypeValidator@xercesc_2_3@@ABEQBGXZ 12072500 f i DatatypeValidatorFactory.obj
 0001:00071500       ?getDTDHandler@SAX2XMLReaderImpl@xercesc_2_3@@UBEPAVDTDHandler@2@XZ 12072500 f i DatatypeValidatorFactory.obj
 0001:00071500       ?getMinExclusive@AbstractNumericFacetValidator@xercesc_2_3@@QBEQAVXMLNumber@2@XZ 12072500 f i DatatypeValidatorFactory.obj
 0001:00071500       ?getErrorReporter@XMLScanner@xercesc_2_3@@QAEPAVXMLErrorReporter@2@XZ 12072500 f i DatatypeValidatorFactory.obj
 0001:00071500       ?getErrorReporter@XMLScanner@xercesc_2_3@@QBEPBVXMLErrorReporter@2@XZ 12072500 f i DatatypeValidatorFactory.obj
 0001:00071510       ?isAtomic@AnySimpleTypeDatatypeValidator@xercesc_2_3@@UBE_NXZ 12072510 f i DatatypeValidatorFactory.obj
 0001:00071510       ?isAtomic@ListDatatypeValidator@xercesc_2_3@@UBE_NXZ 12072510 f i DatatypeValidatorFactory.obj
 0001:00071510       ?handlesDTD@SchemaValidator@xercesc_2_3@@UBE_NXZ 12072510 f i DatatypeValidatorFactory.obj
 0001:00071510       ?handlesSchema@DTDValidator@xercesc_2_3@@UBE_NXZ 12072510 f i DatatypeValidatorFactory.obj
 0001:00071520       ?setErrorReporter@XMLScanner@xercesc_2_3@@QAEXQAVXMLErrorReporter@2@@Z 12072520 f i DatatypeValidatorFactory.obj
 0001:00071520       ?setSubstitutionGroupElem@SchemaElementDecl@xercesc_2_3@@QAEXQAV12@@Z 12072520 f i DatatypeValidatorFactory.obj
 0001:00071520       ?setContent@ListDatatypeValidator@xercesc_2_3@@AAEXQBG@Z 12072520 f i DatatypeValidatorFactory.obj
 0001:00071530       ??_FDoubleDatatypeValidator@xercesc_2_3@@QAEXXZ 12072530 f i DatatypeValidatorFactory.obj
 0001:00071540       ??_FFloatDatatypeValidator@xercesc_2_3@@QAEXXZ 12072540 f i DatatypeValidatorFactory.obj
 0001:00071550       ??_FDateTimeDatatypeValidator@xercesc_2_3@@QAEXXZ 12072550 f i DatatypeValidatorFactory.obj
 0001:00071560       ??_FDateDatatypeValidator@xercesc_2_3@@QAEXXZ 12072560 f i DatatypeValidatorFactory.obj
 0001:00071570       ??_FTimeDatatypeValidator@xercesc_2_3@@QAEXXZ 12072570 f i DatatypeValidatorFactory.obj
 0001:00071580       ??_FDayDatatypeValidator@xercesc_2_3@@QAEXXZ 12072580 f i DatatypeValidatorFactory.obj
 0001:00071590       ??_FMonthDatatypeValidator@xercesc_2_3@@QAEXXZ 12072590 f i DatatypeValidatorFactory.obj
 0001:000715a0       ??_FMonthDayDatatypeValidator@xercesc_2_3@@QAEXXZ 120725a0 f i DatatypeValidatorFactory.obj
 0001:000715b0       ??_FYearDatatypeValidator@xercesc_2_3@@QAEXXZ 120725b0 f i DatatypeValidatorFactory.obj
 0001:000715c0       ??_FYearMonthDatatypeValidator@xercesc_2_3@@QAEXXZ 120725c0 f i DatatypeValidatorFactory.obj
 0001:000715d0       ??_FDurationDatatypeValidator@xercesc_2_3@@QAEXXZ 120725d0 f i DatatypeValidatorFactory.obj
 0001:000715e0       ??0DatatypeValidatorFactory@xercesc_2_3@@QAE@QAVMemoryManager@1@@Z 120725e0 f   DatatypeValidatorFactory.obj
 0001:00071600       ??1DatatypeValidatorFactory@xercesc_2_3@@QAE@XZ 12072600 f   DatatypeValidatorFactory.obj
 0001:000716a0       ?resetRegistry@DatatypeValidatorFactory@xercesc_2_3@@QAEXXZ 120726a0 f   DatatypeValidatorFactory.obj
 0001:00071700       ?reinitRegistry@DatatypeValidatorFactory@xercesc_2_3@@SAXXZ 12072700 f   DatatypeValidatorFactory.obj
 0001:000717a0       ?expandRegistryToFullSchemaSet@DatatypeValidatorFactory@xercesc_2_3@@QAEXXZ 120727a0 f   DatatypeValidatorFactory.obj
 0001:00074260       ?createDatatypeValidator@DatatypeValidatorFactory@xercesc_2_3@@QAEPAVDatatypeValidator@2@QBGQAV32@QAV?$RefHashTableOf@VKVStringPair@xercesc_2_3@@@2@QAV?$RefArrayVectorOf@G@2@_NH4@Z 12075260 f   DatatypeValidatorFactory.obj
 0001:00074500       ?createDatatypeValidator@DatatypeValidatorFactory@xercesc_2_3@@QAEPAVDatatypeValidator@2@QBGQAV?$RefVectorOf@VDatatypeValidator@xercesc_2_3@@@2@H_N@Z 12075500 f   DatatypeValidatorFactory.obj
 0001:000747f0       ??0?$RefHashTableOf@VDatatypeValidator@xercesc_2_3@@@xercesc_2_3@@QAE@IQAVMemoryManager@1@@Z 120757f0 f i DatatypeValidatorFactory.obj
 0001:000748e0       ?removeAll@?$RefHashTableOf@VDatatypeValidator@xercesc_2_3@@@xercesc_2_3@@QAEXXZ 120758e0 f i DatatypeValidatorFactory.obj
 0001:000748e0       ?removeAll@?$RefHashTableOf@VENameMap@xercesc_2_3@@@xercesc_2_3@@QAEXXZ 120758e0 f i DatatypeValidatorFactory.obj
 0001:000748e0       ?removeAll@?$RefHashTableOf@VGrammar@xercesc_2_3@@@xercesc_2_3@@QAEXXZ 120758e0 f i DatatypeValidatorFactory.obj
 0001:000748e0       ?removeAll@?$RefHashTableOf@VXMLAttDef@xercesc_2_3@@@xercesc_2_3@@QAEXXZ 120758e0 f i DatatypeValidatorFactory.obj
 0001:00074950       ?put@?$RefHashTableOf@VDatatypeValidator@xercesc_2_3@@@xercesc_2_3@@QAEXPAXQAVDatatypeValidator@2@@Z 12075950 f i DatatypeValidatorFactory.obj
 0001:00074b60       ??0?$RefHashTableOf@VKVStringPair@xercesc_2_3@@@xercesc_2_3@@QAE@IQAVMemoryManager@1@@Z 12075b60 f i DatatypeValidatorFactory.obj
 0001:00074c50       ?put@?$RefHashTableOf@VKVStringPair@xercesc_2_3@@@xercesc_2_3@@QAEXPAXQAVKVStringPair@2@@Z 12075c50 f i DatatypeValidatorFactory.obj
 0001:00074e60       ??_GKVStringPair@xercesc_2_3@@QAEPAXI@Z 12075e60 f i DatatypeValidatorFactory.obj
 0001:00074e80       ?findBucketElem@?$RefHashTableOf@VENameMap@xercesc_2_3@@@xercesc_2_3@@AAEPAU?$RefHashTableBucketElem@VENameMap@xercesc_2_3@@@2@QBXAAI@Z 12075e80 f i DatatypeValidatorFactory.obj
 0001:00074e80       ?findBucketElem@?$RefHashTableOf@VSchemaInfo@xercesc_2_3@@@xercesc_2_3@@AAEPAU?$RefHashTableBucketElem@VSchemaInfo@xercesc_2_3@@@2@QBXAAI@Z 12075e80 f i DatatypeValidatorFactory.obj
 0001:00074e80       ?findBucketElem@?$RefHashTableOf@VXMLAttDef@xercesc_2_3@@@xercesc_2_3@@AAEPAU?$RefHashTableBucketElem@VXMLAttDef@xercesc_2_3@@@2@QBXAAI@Z 12075e80 f i DatatypeValidatorFactory.obj
 0001:00074e80       ?findBucketElem@?$RefHashTableOf@VValueStore@xercesc_2_3@@@xercesc_2_3@@AAEPAU?$RefHashTableBucketElem@VValueStore@xercesc_2_3@@@2@QBXAAI@Z 12075e80 f i DatatypeValidatorFactory.obj
 0001:00074e80       ?findBucketElem@?$RefHashTableOf@VXercesAttGroupInfo@xercesc_2_3@@@xercesc_2_3@@AAEPAU?$RefHashTableBucketElem@VXercesAttGroupInfo@xercesc_2_3@@@2@QBXAAI@Z 12075e80 f i DatatypeValidatorFactory.obj
 0001:00074e80       ?findBucketElem@?$RefHashTableOf@V?$ValueVectorOf@I@xercesc_2_3@@@xercesc_2_3@@AAEPAU?$RefHashTableBucketElem@V?$ValueVectorOf@I@xercesc_2_3@@@2@QBXAAI@Z 12075e80 f i DatatypeValidatorFactory.obj
 0001:00074e80       ?findBucketElem@?$RefHashTableOf@VXMLRefInfo@xercesc_2_3@@@xercesc_2_3@@AAEPAU?$RefHashTableBucketElem@VXMLRefInfo@xercesc_2_3@@@2@QBXAAI@Z 12075e80 f i DatatypeValidatorFactory.obj
 0001:00074e80       ?findBucketElem@?$RefHashTableOf@VDatatypeValidator@xercesc_2_3@@@xercesc_2_3@@AAEPAU?$RefHashTableBucketElem@VDatatypeValidator@xercesc_2_3@@@2@QBXAAI@Z 12075e80 f i DatatypeValidatorFactory.obj
 0001:00074e80       ?findBucketElem@?$RefHashTableOf@VXercesGroupInfo@xercesc_2_3@@@xercesc_2_3@@AAEPAU?$RefHashTableBucketElem@VXercesGroupInfo@xercesc_2_3@@@2@QBXAAI@Z 12075e80 f i DatatypeValidatorFactory.obj
 0001:00074e80       ?findBucketElem@?$RefHashTableOf@VXMLElementDecl@xercesc_2_3@@@xercesc_2_3@@AAEPAU?$RefHashTableBucketElem@VXMLElementDecl@xercesc_2_3@@@2@QBXAAI@Z 12075e80 f i DatatypeValidatorFactory.obj
 0001:00074e80       ?findBucketElem@?$RefHashTableOf@G@xercesc_2_3@@AAEPAU?$RefHashTableBucketElem@G@2@QBXAAI@Z 12075e80 f i DatatypeValidatorFactory.obj
 0001:00074e80       ?findBucketElem@?$RefHashTableOf@VComplexTypeInfo@xercesc_2_3@@@xercesc_2_3@@AAEPAU?$RefHashTableBucketElem@VComplexTypeInfo@xercesc_2_3@@@2@QBXAAI@Z 12075e80 f i DatatypeValidatorFactory.obj
 0001:00074e80       ?findBucketElem@?$RefHashTableOf@VXMLInteger@xercesc_2_3@@@xercesc_2_3@@AAEPAU?$RefHashTableBucketElem@VXMLInteger@xercesc_2_3@@@2@QBXAAI@Z 12075e80 f i DatatypeValidatorFactory.obj
 0001:00074e80       ?findBucketElem@?$RefHashTableOf@VCPMapEntry@xercesc_2_3@@@xercesc_2_3@@AAEPAU?$RefHashTableBucketElem@VCPMapEntry@xercesc_2_3@@@2@QBXAAI@Z 12075e80 f i DatatypeValidatorFactory.obj
 0001:00074e80       ?findBucketElem@?$RefHashTableOf@VRangeTokenElemMap@xercesc_2_3@@@xercesc_2_3@@AAEPAU?$RefHashTableBucketElem@VRangeTokenElemMap@xercesc_2_3@@@2@QBXAAI@Z 12075e80 f i DatatypeValidatorFactory.obj
 0001:00074e80       ?findBucketElem@?$RefHashTableOf@VKVStringPair@xercesc_2_3@@@xercesc_2_3@@AAEPAU?$RefHashTableBucketElem@VKVStringPair@xercesc_2_3@@@2@QBXAAI@Z 12075e80 f i DatatypeValidatorFactory.obj
 0001:00074e80       ?findBucketElem@?$RefHashTableOf@V?$RefHashTableOf@V?$KeyRefPair@XVDOMUserDataHandler@xercesc_2_3@@@xercesc_2_3@@@xercesc_2_3@@@xercesc_2_3@@AAEPAU?$RefHashTableBucketElem@V?$RefHashTableOf@V?$KeyRefPair@XVDOMUserDataHandler@xercesc_2_3@@@xercesc_2_3@@@xercesc_2_3@@@2@QBXAAI@Z 12075e80 f i DatatypeValidatorFactory.obj
 0001:00074e80       ?findBucketElem@?$RefHashTableOf@V?$KeyRefPair@XVDOMUserDataHandler@xercesc_2_3@@@xercesc_2_3@@@xercesc_2_3@@AAEPAU?$RefHashTableBucketElem@V?$KeyRefPair@XVDOMUserDataHandler@xercesc_2_3@@@xercesc_2_3@@@2@QBXAAI@Z 12075e80 f i DatatypeValidatorFactory.obj
 0001:00074e80       ?findBucketElem@?$RefHashTableOf@VGrammar@xercesc_2_3@@@xercesc_2_3@@AAEPAU?$RefHashTableBucketElem@VGrammar@xercesc_2_3@@@2@QBXAAI@Z 12075e80 f i DatatypeValidatorFactory.obj
 0001:00074e80       ?findBucketElem@?$RefHashTableOf@V?$ValueVectorOf@PAVSchemaElementDecl@xercesc_2_3@@@xercesc_2_3@@@xercesc_2_3@@AAEPAU?$RefHashTableBucketElem@V?$ValueVectorOf@PAVSchemaElementDecl@xercesc_2_3@@@xercesc_2_3@@@2@QBXAAI@Z 12075e80 f i DatatypeValidatorFactory.obj
 0001:00074e80       ?findBucketElem@?$RefHashTableOf@VDTDAttDef@xercesc_2_3@@@xercesc_2_3@@AAEPAU?$RefHashTableBucketElem@VDTDAttDef@xercesc_2_3@@@2@QBXAAI@Z 12075e80 f i DatatypeValidatorFactory.obj
 0001:00074f00       ?removeBucketElem@?$RefHashTableOf@VKVStringPair@xercesc_2_3@@@xercesc_2_3@@AAEXQBXAAI@Z 12075f00 f i DatatypeValidatorFactory.obj
 0001:00074ff0       ??0DateDatatypeValidator@xercesc_2_3@@QAE@QAVMemoryManager@1@@Z 12075ff0 f   DateDatatypeValidator.obj
 0001:00075020       ??_EDateDatatypeValidator@xercesc_2_3@@UAEPAXI@Z 12076020 f i DateDatatypeValidator.obj
 0001:00075080       ??0DateDatatypeValidator@xercesc_2_3@@QAE@QAVDatatypeValidator@1@QAV?$RefHashTableOf@VKVStringPair@xercesc_2_3@@@1@QAV?$RefArrayVectorOf@G@1@HQAVMemoryManager@1@@Z 12076080 f   DateDatatypeValidator.obj
 0001:000750f0       ??1DateDatatypeValidator@xercesc_2_3@@UAE@XZ 120760f0 f   DateDatatypeValidator.obj
 0001:00075100       ?newInstance@DateDatatypeValidator@xercesc_2_3@@UAEPAVDatatypeValidator@2@QAV?$RefHashTableOf@VKVStringPair@xercesc_2_3@@@2@QAV?$RefArrayVectorOf@G@2@HQAVMemoryManager@2@@Z 12076100 f   DateDatatypeValidator.obj
 0001:00075180       ?parse@DateDatatypeValidator@xercesc_2_3@@MAEPAVXMLDateTime@2@QBG@Z 12076180 f   DateDatatypeValidator.obj
 0001:00075220       ??0DateTimeDatatypeValidator@xercesc_2_3@@QAE@QAVMemoryManager@1@@Z 12076220 f   DateTimeDatatypeValidator.obj
 0001:00075250       ??_EDateTimeDatatypeValidator@xercesc_2_3@@UAEPAXI@Z 12076250 f i DateTimeDatatypeValidator.obj
 0001:000752b0       ??0DateTimeDatatypeValidator@xercesc_2_3@@QAE@QAVDatatypeValidator@1@QAV?$RefHashTableOf@VKVStringPair@xercesc_2_3@@@1@QAV?$RefArrayVectorOf@G@1@HQAVMemoryManager@1@@Z 120762b0 f   DateTimeDatatypeValidator.obj
 0001:00075320       ??1DateTimeDatatypeValidator@xercesc_2_3@@UAE@XZ 12076320 f   DateTimeDatatypeValidator.obj
 0001:00075330       ?newInstance@DateTimeDatatypeValidator@xercesc_2_3@@UAEPAVDatatypeValidator@2@QAV?$RefHashTableOf@VKVStringPair@xercesc_2_3@@@2@QAV?$RefArrayVectorOf@G@2@HQAVMemoryManager@2@@Z 12076330 f   DateTimeDatatypeValidator.obj
 0001:000753b0       ?parse@DateTimeDatatypeValidator@xercesc_2_3@@MAEPAVXMLDateTime@2@QBG@Z 120763b0 f   DateTimeDatatypeValidator.obj
 0001:00075450       ??1DateTimeValidator@xercesc_2_3@@UAE@XZ 12076450 f   DateTimeValidator.obj
 0001:00075460       ??_EDateTimeValidator@xercesc_2_3@@UAEPAXI@Z 12076460 f i DateTimeValidator.obj
 0001:000754c0       ??0DateTimeValidator@xercesc_2_3@@IAE@QAVDatatypeValidator@1@QAV?$RefHashTableOf@VKVStringPair@xercesc_2_3@@@1@HW4ValidatorType@21@QAVMemoryManager@1@@Z 120764c0 f   DateTimeValidator.obj
 0001:000754f0       ?compare@DateTimeValidator@xercesc_2_3@@UAEHQBG0@Z 120764f0 f   DateTimeValidator.obj
 0001:000755b0       ?assignAdditionalFacet@DateTimeValidator@xercesc_2_3@@MAEXQBG0@Z 120765b0 f   DateTimeValidator.obj
 0001:000755f0       ?checkContent@DateTimeValidator@xercesc_2_3@@MAEXQBG_N@Z 120765f0 f   DateTimeValidator.obj
 0001:00075a20       ?compareValues@DateTimeValidator@xercesc_2_3@@MAEHQBVXMLNumber@2@0@Z 12076a20 f   DateTimeValidator.obj
 0001:00075a40       ?compareDates@DateTimeValidator@xercesc_2_3@@MAEHQBVXMLDateTime@2@0_N@Z 12076a40 f   DateTimeValidator.obj
 0001:00075a60       ?setMaxInclusive@DateTimeValidator@xercesc_2_3@@MAEXQBG@Z 12076a60 f   DateTimeValidator.obj
 0001:00075a80       ?setMaxExclusive@DateTimeValidator@xercesc_2_3@@MAEXQBG@Z 12076a80 f   DateTimeValidator.obj
 0001:00075aa0       ?setMinInclusive@DateTimeValidator@xercesc_2_3@@MAEXQBG@Z 12076aa0 f   DateTimeValidator.obj
 0001:00075ac0       ?setMinExclusive@DateTimeValidator@xercesc_2_3@@MAEXQBG@Z 12076ac0 f   DateTimeValidator.obj
 0001:00075ae0       ?setEnumeration@DateTimeValidator@xercesc_2_3@@MAEXXZ 12076ae0 f   DateTimeValidator.obj
 0001:00075d10       ??_E?$RefVectorOf@VXMLNumber@xercesc_2_3@@@xercesc_2_3@@UAEPAXI@Z 12076d10 f i DateTimeValidator.obj
 0001:00075d10       ??_G?$RefVectorOf@VXMLNumber@xercesc_2_3@@@xercesc_2_3@@UAEPAXI@Z 12076d10 f i DateTimeValidator.obj
 0001:00075d30       ??1?$RefVectorOf@VXMLNumber@xercesc_2_3@@@xercesc_2_3@@UAE@XZ 12076d30 f i DateTimeValidator.obj
 0001:00075db0       ??1?$BaseRefVectorOf@VXMLNumber@xercesc_2_3@@@xercesc_2_3@@UAE@XZ 12076db0 f i DateTimeValidator.obj
 0001:00075dc0       ??0DayDatatypeValidator@xercesc_2_3@@QAE@QAVMemoryManager@1@@Z 12076dc0 f   DayDatatypeValidator.obj
 0001:00075df0       ??_EDayDatatypeValidator@xercesc_2_3@@UAEPAXI@Z 12076df0 f i DayDatatypeValidator.obj
 0001:00075e50       ??0DayDatatypeValidator@xercesc_2_3@@QAE@QAVDatatypeValidator@1@QAV?$RefHashTableOf@VKVStringPair@xercesc_2_3@@@1@QAV?$RefArrayVectorOf@G@1@HQAVMemoryManager@1@@Z 12076e50 f   DayDatatypeValidator.obj
 0001:00075ec0       ??1DayDatatypeValidator@xercesc_2_3@@UAE@XZ 12076ec0 f   DayDatatypeValidator.obj
 0001:00075ed0       ?newInstance@DayDatatypeValidator@xercesc_2_3@@UAEPAVDatatypeValidator@2@QAV?$RefHashTableOf@VKVStringPair@xercesc_2_3@@@2@QAV?$RefArrayVectorOf@G@2@HQAVMemoryManager@2@@Z 12076ed0 f   DayDatatypeValidator.obj
 0001:00075f50       ?parse@DayDatatypeValidator@xercesc_2_3@@MAEPAVXMLDateTime@2@QBG@Z 12076f50 f   DayDatatypeValidator.obj
 0001:00075ff0       ??0DecimalDatatypeValidator@xercesc_2_3@@QAE@QAVMemoryManager@1@@Z 12076ff0 f   DecimalDatatypeValidator.obj
 0001:00076020       ??_EDecimalDatatypeValidator@xercesc_2_3@@UAEPAXI@Z 12077020 f i DecimalDatatypeValidator.obj
 0001:00076080       ??0DecimalDatatypeValidator@xercesc_2_3@@QAE@QAVDatatypeValidator@1@QAV?$RefHashTableOf@VKVStringPair@xercesc_2_3@@@1@QAV?$RefArrayVectorOf@G@1@HQAVMemoryManager@1@@Z 12077080 f   DecimalDatatypeValidator.obj
 0001:000760f0       ??1DecimalDatatypeValidator@xercesc_2_3@@UAE@XZ 120770f0 f   DecimalDatatypeValidator.obj
 0001:00076100       ?compare@DecimalDatatypeValidator@xercesc_2_3@@UAEHQBG0@Z 12077100 f   DecimalDatatypeValidator.obj
 0001:000761a0       ?newInstance@DecimalDatatypeValidator@xercesc_2_3@@UAEPAVDatatypeValidator@2@QAV?$RefHashTableOf@VKVStringPair@xercesc_2_3@@@2@QAV?$RefArrayVectorOf@G@2@HQAVMemoryManager@2@@Z 120771a0 f   DecimalDatatypeValidator.obj
 0001:00076250       ??0DecimalDatatypeValidator@xercesc_2_3@@IAE@QAVDatatypeValidator@1@QAV?$RefHashTableOf@VKVStringPair@xercesc_2_3@@@1@HW4ValidatorType@21@QAVMemoryManager@1@@Z 12077250 f   DecimalDatatypeValidator.obj
 0001:00076290       ?assignAdditionalFacet@DecimalDatatypeValidator@xercesc_2_3@@MAEXQBG0@Z 12077290 f   DecimalDatatypeValidator.obj
 0001:00076540       ?inheritAdditionalFacet@DecimalDatatypeValidator@xercesc_2_3@@MAEXXZ 12077540 f   DecimalDatatypeValidator.obj
 0001:00076590       ?checkAdditionalFacetConstraints@DecimalDatatypeValidator@xercesc_2_3@@MBEXXZ 12077590 f   DecimalDatatypeValidator.obj
 0001:00076610       ?checkAdditionalFacetConstraintsBase@DecimalDatatypeValidator@xercesc_2_3@@MBEXXZ 12077610 f   DecimalDatatypeValidator.obj
 0001:00076860       ?compareValues@DecimalDatatypeValidator@xercesc_2_3@@MAEHQBVXMLNumber@2@0@Z 12077860 f   DecimalDatatypeValidator.obj
 0001:00076880       ?setMaxInclusive@DecimalDatatypeValidator@xercesc_2_3@@MAEXQBG@Z 12077880 f   DecimalDatatypeValidator.obj
 0001:000768f0       ?setMaxExclusive@DecimalDatatypeValidator@xercesc_2_3@@MAEXQBG@Z 120778f0 f   DecimalDatatypeValidator.obj
 0001:00076960       ?setMinInclusive@DecimalDatatypeValidator@xercesc_2_3@@MAEXQBG@Z 12077960 f   DecimalDatatypeValidator.obj
 0001:000769d0       ?setMinExclusive@DecimalDatatypeValidator@xercesc_2_3@@MAEXQBG@Z 120779d0 f   DecimalDatatypeValidator.obj
 0001:00076a40       ?setEnumeration@DecimalDatatypeValidator@xercesc_2_3@@MAEXXZ 12077a40 f   DecimalDatatypeValidator.obj
 0001:00076d60       ?checkContent@DecimalDatatypeValidator@xercesc_2_3@@MAEXQBG_N@Z 12077d60 f   DecimalDatatypeValidator.obj
 0001:000771d0       ??0?$BaseRefVectorOf@VXMLNumber@xercesc_2_3@@@xercesc_2_3@@QAE@I_NQAVMemoryManager@1@@Z 120781d0 f i DecimalDatatypeValidator.obj
 0001:00077230       ??0DoubleDatatypeValidator@xercesc_2_3@@QAE@QAVMemoryManager@1@@Z 12078230 f   DoubleDatatypeValidator.obj
 0001:00077260       ??_EDoubleDatatypeValidator@xercesc_2_3@@UAEPAXI@Z 12078260 f i DoubleDatatypeValidator.obj
 0001:000772c0       ??0DoubleDatatypeValidator@xercesc_2_3@@QAE@QAVDatatypeValidator@1@QAV?$RefHashTableOf@VKVStringPair@xercesc_2_3@@@1@QAV?$RefArrayVectorOf@G@1@HQAVMemoryManager@1@@Z 120782c0 f   DoubleDatatypeValidator.obj
 0001:00077330       ??1DoubleDatatypeValidator@xercesc_2_3@@UAE@XZ 12078330 f   DoubleDatatypeValidator.obj
 0001:00077340       ?compare@DoubleDatatypeValidator@xercesc_2_3@@UAEHQBG0@Z 12078340 f   DoubleDatatypeValidator.obj
 0001:000773e0       ?newInstance@DoubleDatatypeValidator@xercesc_2_3@@UAEPAVDatatypeValidator@2@QAV?$RefHashTableOf@VKVStringPair@xercesc_2_3@@@2@QAV?$RefArrayVectorOf@G@2@HQAVMemoryManager@2@@Z 120783e0 f   DoubleDatatypeValidator.obj
 0001:00077460       ??0DoubleDatatypeValidator@xercesc_2_3@@IAE@QAVDatatypeValidator@1@QAV?$RefHashTableOf@VKVStringPair@xercesc_2_3@@@1@HW4ValidatorType@21@QAVMemoryManager@1@@Z 12078460 f   DoubleDatatypeValidator.obj
 0001:00077490       ?assignAdditionalFacet@DoubleDatatypeValidator@xercesc_2_3@@MAEXQBG0@Z 12078490 f   DoubleDatatypeValidator.obj
 0001:000774d0       ?setMaxInclusive@DoubleDatatypeValidator@xercesc_2_3@@MAEXQBG@Z 120784d0 f   DoubleDatatypeValidator.obj
 0001:00077540       ?setMaxExclusive@DoubleDatatypeValidator@xercesc_2_3@@MAEXQBG@Z 12078540 f   DoubleDatatypeValidator.obj
 0001:000775b0       ?setMinInclusive@DoubleDatatypeValidator@xercesc_2_3@@MAEXQBG@Z 120785b0 f   DoubleDatatypeValidator.obj
 0001:00077620       ?setMinExclusive@DoubleDatatypeValidator@xercesc_2_3@@MAEXQBG@Z 12078620 f   DoubleDatatypeValidator.obj
 0001:00077690       ?setEnumeration@DoubleDatatypeValidator@xercesc_2_3@@MAEXXZ 12078690 f   DoubleDatatypeValidator.obj
 0001:000779b0       ?checkContent@DoubleDatatypeValidator@xercesc_2_3@@MAEXQBG_N@Z 120789b0 f   DoubleDatatypeValidator.obj
 0001:00077c50       ??0DurationDatatypeValidator@xercesc_2_3@@QAE@QAVMemoryManager@1@@Z 12078c50 f   DurationDatatypeValidator.obj
 0001:00077c80       ??_EDurationDatatypeValidator@xercesc_2_3@@UAEPAXI@Z 12078c80 f i DurationDatatypeValidator.obj
 0001:00077ce0       ??0DurationDatatypeValidator@xercesc_2_3@@QAE@QAVDatatypeValidator@1@QAV?$RefHashTableOf@VKVStringPair@xercesc_2_3@@@1@QAV?$RefArrayVectorOf@G@1@HQAVMemoryManager@1@@Z 12078ce0 f   DurationDatatypeValidator.obj
 0001:00077d50       ??1DurationDatatypeValidator@xercesc_2_3@@UAE@XZ 12078d50 f   DurationDatatypeValidator.obj
 0001:00077d60       ?newInstance@DurationDatatypeValidator@xercesc_2_3@@UAEPAVDatatypeValidator@2@QAV?$RefHashTableOf@VKVStringPair@xercesc_2_3@@@2@QAV?$RefArrayVectorOf@G@2@HQAVMemoryManager@2@@Z 12078d60 f   DurationDatatypeValidator.obj
 0001:00077de0       ?parse@DurationDatatypeValidator@xercesc_2_3@@MAEPAVXMLDateTime@2@QBG@Z 12078de0 f   DurationDatatypeValidator.obj
 0001:00077e80       ?compareDates@DurationDatatypeValidator@xercesc_2_3@@MAEHQBVXMLDateTime@2@0_N@Z 12078e80 f   DurationDatatypeValidator.obj
 0001:00077ea0       ??0ENTITYDatatypeValidator@xercesc_2_3@@QAE@QAVMemoryManager@1@@Z 12078ea0 f   ENTITYDatatypeValidator.obj
 0001:00077ed0       ??_EENTITYDatatypeValidator@xercesc_2_3@@UAEPAXI@Z 12078ed0 f i ENTITYDatatypeValidator.obj
 0001:00077f30       ??0ENTITYDatatypeValidator@xercesc_2_3@@QAE@QAVDatatypeValidator@1@QAV?$RefHashTableOf@VKVStringPair@xercesc_2_3@@@1@QAV?$RefArrayVectorOf@G@1@HQAVMemoryManager@1@@Z 12078f30 f   ENTITYDatatypeValidator.obj
 0001:00077fa0       ??1ENTITYDatatypeValidator@xercesc_2_3@@UAE@XZ 12078fa0 f   ENTITYDatatypeValidator.obj
 0001:00077fb0       ?newInstance@ENTITYDatatypeValidator@xercesc_2_3@@UAEPAVDatatypeValidator@2@QAV?$RefHashTableOf@VKVStringPair@xercesc_2_3@@@2@QAV?$RefArrayVectorOf@G@2@HQAVMemoryManager@2@@Z 12078fb0 f   ENTITYDatatypeValidator.obj
 0001:00078050       ?validate@ENTITYDatatypeValidator@xercesc_2_3@@UAEXQBG@Z 12079050 f   ENTITYDatatypeValidator.obj
 0001:00078170       ?checkValueSpace@ENTITYDatatypeValidator@xercesc_2_3@@MAEXQBG@Z 12079170 f   ENTITYDatatypeValidator.obj
 0001:000781c0       ??0FloatDatatypeValidator@xercesc_2_3@@QAE@QAVMemoryManager@1@@Z 120791c0 f   FloatDatatypeValidator.obj
 0001:000781f0       ??_EFloatDatatypeValidator@xercesc_2_3@@UAEPAXI@Z 120791f0 f i FloatDatatypeValidator.obj
 0001:00078250       ??0FloatDatatypeValidator@xercesc_2_3@@QAE@QAVDatatypeValidator@1@QAV?$RefHashTableOf@VKVStringPair@xercesc_2_3@@@1@QAV?$RefArrayVectorOf@G@1@HQAVMemoryManager@1@@Z 12079250 f   FloatDatatypeValidator.obj
 0001:000782c0       ??1FloatDatatypeValidator@xercesc_2_3@@UAE@XZ 120792c0 f   FloatDatatypeValidator.obj
 0001:000782d0       ?compare@FloatDatatypeValidator@xercesc_2_3@@UAEHQBG0@Z 120792d0 f   FloatDatatypeValidator.obj
 0001:00078370       ?newInstance@FloatDatatypeValidator@xercesc_2_3@@UAEPAVDatatypeValidator@2@QAV?$RefHashTableOf@VKVStringPair@xercesc_2_3@@@2@QAV?$RefArrayVectorOf@G@2@HQAVMemoryManager@2@@Z 12079370 f   FloatDatatypeValidator.obj
 0001:000783f0       ??0FloatDatatypeValidator@xercesc_2_3@@IAE@QAVDatatypeValidator@1@QAV?$RefHashTableOf@VKVStringPair@xercesc_2_3@@@1@HW4ValidatorType@21@QAVMemoryManager@1@@Z 120793f0 f   FloatDatatypeValidator.obj
 0001:00078420       ?assignAdditionalFacet@FloatDatatypeValidator@xercesc_2_3@@MAEXQBG0@Z 12079420 f   FloatDatatypeValidator.obj
 0001:00078460       ?compareValues@FloatDatatypeValidator@xercesc_2_3@@MAEHQBVXMLNumber@2@0@Z 12079460 f   FloatDatatypeValidator.obj
 0001:00078460       ?compareValues@DoubleDatatypeValidator@xercesc_2_3@@MAEHQBVXMLNumber@2@0@Z 12079460 f   FloatDatatypeValidator.obj
 0001:00078480       ?setMaxInclusive@FloatDatatypeValidator@xercesc_2_3@@MAEXQBG@Z 12079480 f   FloatDatatypeValidator.obj
 0001:000784f0       ?setMaxExclusive@FloatDatatypeValidator@xercesc_2_3@@MAEXQBG@Z 120794f0 f   FloatDatatypeValidator.obj
 0001:00078560       ?setMinInclusive@FloatDatatypeValidator@xercesc_2_3@@MAEXQBG@Z 12079560 f   FloatDatatypeValidator.obj
 0001:000785d0       ?setMinExclusive@FloatDatatypeValidator@xercesc_2_3@@MAEXQBG@Z 120795d0 f   FloatDatatypeValidator.obj
 0001:00078640       ?setEnumeration@FloatDatatypeValidator@xercesc_2_3@@MAEXXZ 12079640 f   FloatDatatypeValidator.obj
 0001:00078960       ?checkContent@FloatDatatypeValidator@xercesc_2_3@@MAEXQBG_N@Z 12079960 f   FloatDatatypeValidator.obj
 0001:00078c00       ??0HexBinaryDatatypeValidator@xercesc_2_3@@QAE@QAVMemoryManager@1@@Z 12079c00 f   HexBinaryDatatypeValidator.obj
 0001:00078c30       ??_EHexBinaryDatatypeValidator@xercesc_2_3@@UAEPAXI@Z 12079c30 f i HexBinaryDatatypeValidator.obj
 0001:00078c90       ??1HexBinaryDatatypeValidator@xercesc_2_3@@UAE@XZ 12079c90 f   HexBinaryDatatypeValidator.obj
 0001:00078ca0       ??0HexBinaryDatatypeValidator@xercesc_2_3@@QAE@QAVDatatypeValidator@1@QAV?$RefHashTableOf@VKVStringPair@xercesc_2_3@@@1@QAV?$RefArrayVectorOf@G@1@HQAVMemoryManager@1@@Z 12079ca0 f   HexBinaryDatatypeValidator.obj
 0001:00078d10       ?newInstance@HexBinaryDatatypeValidator@xercesc_2_3@@UAEPAVDatatypeValidator@2@QAV?$RefHashTableOf@VKVStringPair@xercesc_2_3@@@2@QAV?$RefArrayVectorOf@G@2@HQAVMemoryManager@2@@Z 12079d10 f   HexBinaryDatatypeValidator.obj
 0001:00078d90       ?assignAdditionalFacet@HexBinaryDatatypeValidator@xercesc_2_3@@MAEXQBG0@Z 12079d90 f   HexBinaryDatatypeValidator.obj
 0001:00078dd0       ?checkValueSpace@HexBinaryDatatypeValidator@xercesc_2_3@@MAEXQBG@Z 12079dd0 f   HexBinaryDatatypeValidator.obj
 0001:00078e20       ?getLength@HexBinaryDatatypeValidator@xercesc_2_3@@MBEHQBG@Z 12079e20 f   HexBinaryDatatypeValidator.obj
 0001:00078e30       ??0IDDatatypeValidator@xercesc_2_3@@QAE@QAVMemoryManager@1@@Z 12079e30 f   IDDatatypeValidator.obj
 0001:00078e60       ??_EIDDatatypeValidator@xercesc_2_3@@UAEPAXI@Z 12079e60 f i IDDatatypeValidator.obj
 0001:00078ec0       ??0IDDatatypeValidator@xercesc_2_3@@QAE@QAVDatatypeValidator@1@QAV?$RefHashTableOf@VKVStringPair@xercesc_2_3@@@1@QAV?$RefArrayVectorOf@G@1@HQAVMemoryManager@1@@Z 12079ec0 f   IDDatatypeValidator.obj
 0001:00078f30       ??1IDDatatypeValidator@xercesc_2_3@@UAE@XZ 12079f30 f   IDDatatypeValidator.obj
 0001:00078f40       ?newInstance@IDDatatypeValidator@xercesc_2_3@@UAEPAVDatatypeValidator@2@QAV?$RefHashTableOf@VKVStringPair@xercesc_2_3@@@2@QAV?$RefArrayVectorOf@G@2@HQAVMemoryManager@2@@Z 12079f40 f   IDDatatypeValidator.obj
 0001:00078fe0       ??0IDDatatypeValidator@xercesc_2_3@@IAE@QAVDatatypeValidator@1@QAV?$RefHashTableOf@VKVStringPair@xercesc_2_3@@@1@HW4ValidatorType@21@QAVMemoryManager@1@@Z 12079fe0 f   IDDatatypeValidator.obj
 0001:00079020       ?validate@IDDatatypeValidator@xercesc_2_3@@UAEXQBG@Z 1207a020 f   IDDatatypeValidator.obj
 0001:00079050       ?addId@IDDatatypeValidator@xercesc_2_3@@AAEXQBG@Z 1207a050 f   IDDatatypeValidator.obj
 0001:00079270       ?checkValueSpace@IDDatatypeValidator@xercesc_2_3@@MAEXQBG@Z 1207a270 f   IDDatatypeValidator.obj
 0001:000792c0       ??0IDREFDatatypeValidator@xercesc_2_3@@QAE@QAVMemoryManager@1@@Z 1207a2c0 f   IDREFDatatypeValidator.obj
 0001:000792f0       ??_EIDREFDatatypeValidator@xercesc_2_3@@UAEPAXI@Z 1207a2f0 f i IDREFDatatypeValidator.obj
 0001:00079350       ??0IDREFDatatypeValidator@xercesc_2_3@@QAE@QAVDatatypeValidator@1@QAV?$RefHashTableOf@VKVStringPair@xercesc_2_3@@@1@QAV?$RefArrayVectorOf@G@1@HQAVMemoryManager@1@@Z 1207a350 f   IDREFDatatypeValidator.obj
 0001:000793c0       ??1IDREFDatatypeValidator@xercesc_2_3@@UAE@XZ 1207a3c0 f   IDREFDatatypeValidator.obj
 0001:000793d0       ?newInstance@IDREFDatatypeValidator@xercesc_2_3@@UAEPAVDatatypeValidator@2@QAV?$RefHashTableOf@VKVStringPair@xercesc_2_3@@@2@QAV?$RefArrayVectorOf@G@2@HQAVMemoryManager@2@@Z 1207a3d0 f   IDREFDatatypeValidator.obj
 0001:00079470       ??0IDREFDatatypeValidator@xercesc_2_3@@IAE@QAVDatatypeValidator@1@QAV?$RefHashTableOf@VKVStringPair@xercesc_2_3@@@1@HW4ValidatorType@21@QAVMemoryManager@1@@Z 1207a470 f   IDREFDatatypeValidator.obj
 0001:000794b0       ?validate@IDREFDatatypeValidator@xercesc_2_3@@UAEXQBG@Z 1207a4b0 f   IDREFDatatypeValidator.obj
 0001:000794e0       ?addIdRef@IDREFDatatypeValidator@xercesc_2_3@@AAEXQBG@Z 1207a4e0 f   IDREFDatatypeValidator.obj
 0001:00079700       ?checkValueSpace@IDREFDatatypeValidator@xercesc_2_3@@MAEXQBG@Z 1207a700 f   IDREFDatatypeValidator.obj
 0001:00079750       ??0ListDatatypeValidator@xercesc_2_3@@QAE@QAVMemoryManager@1@@Z 1207a750 f   ListDatatypeValidator.obj
 0001:00079780       ??_EListDatatypeValidator@xercesc_2_3@@UAEPAXI@Z 1207a780 f i ListDatatypeValidator.obj
 0001:000797e0       ??0ListDatatypeValidator@xercesc_2_3@@QAE@QAVDatatypeValidator@1@QAV?$RefHashTableOf@VKVStringPair@xercesc_2_3@@@1@QAV?$RefArrayVectorOf@G@1@HQAVMemoryManager@1@@Z 1207a7e0 f   ListDatatypeValidator.obj
 0001:000798a0       ??1ListDatatypeValidator@xercesc_2_3@@UAE@XZ 1207a8a0 f   ListDatatypeValidator.obj
 0001:000798b0       ?newInstance@ListDatatypeValidator@xercesc_2_3@@UAEPAVDatatypeValidator@2@QAV?$RefHashTableOf@VKVStringPair@xercesc_2_3@@@2@QAV?$RefArrayVectorOf@G@2@HQAVMemoryManager@2@@Z 1207a8b0 f   ListDatatypeValidator.obj
 0001:000799a0       ?compare@ListDatatypeValidator@xercesc_2_3@@UAEHQBG0@Z 1207a9a0 f   ListDatatypeValidator.obj
 0001:00079b60       ?validate@ListDatatypeValidator@xercesc_2_3@@UAEXQBG@Z 1207ab60 f   ListDatatypeValidator.obj
 0001:00079bd0       ?checkContent@ListDatatypeValidator@xercesc_2_3@@MAEXQBG_N@Z 1207abd0 f   ListDatatypeValidator.obj
 0001:00079c40       ?checkContent@ListDatatypeValidator@xercesc_2_3@@AAEXPAV?$BaseRefVectorOf@G@2@QBG_N@Z 1207ac40 f   ListDatatypeValidator.obj
 0001:0007a130       ?valueSpaceCheck@ListDatatypeValidator@xercesc_2_3@@ABE_NPAV?$BaseRefVectorOf@G@2@QBG@Z 1207b130 f   ListDatatypeValidator.obj
 0001:0007a2b0       ?getItemTypeDTV@ListDatatypeValidator@xercesc_2_3@@QBEPAVDatatypeValidator@2@XZ 1207b2b0 f   ListDatatypeValidator.obj
 0001:0007a2d0       ?assignAdditionalFacet@ListDatatypeValidator@xercesc_2_3@@MAEXQBG0@Z 1207b2d0 f   ListDatatypeValidator.obj
 0001:0007a310       ?getLength@ListDatatypeValidator@xercesc_2_3@@MBEHQBG@Z 1207b310 f   ListDatatypeValidator.obj
 0001:0007a340       ?inspectFacetBase@ListDatatypeValidator@xercesc_2_3@@MAEXXZ 1207b340 f   ListDatatypeValidator.obj
 0001:0007a590       ?inheritFacet@ListDatatypeValidator@xercesc_2_3@@MAEXXZ 1207b590 f   ListDatatypeValidator.obj
 0001:0007a5a0       ??0MonthDatatypeValidator@xercesc_2_3@@QAE@QAVMemoryManager@1@@Z 1207b5a0 f   MonthDatatypeValidator.obj
 0001:0007a5d0       ??_EMonthDatatypeValidator@xercesc_2_3@@UAEPAXI@Z 1207b5d0 f i MonthDatatypeValidator.obj
 0001:0007a630       ??0MonthDatatypeValidator@xercesc_2_3@@QAE@QAVDatatypeValidator@1@QAV?$RefHashTableOf@VKVStringPair@xercesc_2_3@@@1@QAV?$RefArrayVectorOf@G@1@HQAVMemoryManager@1@@Z 1207b630 f   MonthDatatypeValidator.obj
 0001:0007a6a0       ??1MonthDatatypeValidator@xercesc_2_3@@UAE@XZ 1207b6a0 f   MonthDatatypeValidator.obj
 0001:0007a6b0       ?newInstance@MonthDatatypeValidator@xercesc_2_3@@UAEPAVDatatypeValidator@2@QAV?$RefHashTableOf@VKVStringPair@xercesc_2_3@@@2@QAV?$RefArrayVectorOf@G@2@HQAVMemoryManager@2@@Z 1207b6b0 f   MonthDatatypeValidator.obj
 0001:0007a730       ?parse@MonthDatatypeValidator@xercesc_2_3@@MAEPAVXMLDateTime@2@QBG@Z 1207b730 f   MonthDatatypeValidator.obj
 0001:0007a7d0       ??0MonthDayDatatypeValidator@xercesc_2_3@@QAE@QAVMemoryManager@1@@Z 1207b7d0 f   MonthDayDatatypeValidator.obj
 0001:0007a800       ??_EMonthDayDatatypeValidator@xercesc_2_3@@UAEPAXI@Z 1207b800 f i MonthDayDatatypeValidator.obj
 0001:0007a860       ??0MonthDayDatatypeValidator@xercesc_2_3@@QAE@QAVDatatypeValidator@1@QAV?$RefHashTableOf@VKVStringPair@xercesc_2_3@@@1@QAV?$RefArrayVectorOf@G@1@HQAVMemoryManager@1@@Z 1207b860 f   MonthDayDatatypeValidator.obj
 0001:0007a8d0       ??1MonthDayDatatypeValidator@xercesc_2_3@@UAE@XZ 1207b8d0 f   MonthDayDatatypeValidator.obj
 0001:0007a8e0       ?newInstance@MonthDayDatatypeValidator@xercesc_2_3@@UAEPAVDatatypeValidator@2@QAV?$RefHashTableOf@VKVStringPair@xercesc_2_3@@@2@QAV?$RefArrayVectorOf@G@2@HQAVMemoryManager@2@@Z 1207b8e0 f   MonthDayDatatypeValidator.obj
 0001:0007a960       ?parse@MonthDayDatatypeValidator@xercesc_2_3@@MAEPAVXMLDateTime@2@QBG@Z 1207b960 f   MonthDayDatatypeValidator.obj
 0001:0007aa00       ??0NameDatatypeValidator@xercesc_2_3@@QAE@QAVMemoryManager@1@@Z 1207ba00 f   NameDatatypeValidator.obj
 0001:0007aa30       ??_ENameDatatypeValidator@xercesc_2_3@@UAEPAXI@Z 1207ba30 f i NameDatatypeValidator.obj
 0001:0007aa90       ??1NameDatatypeValidator@xercesc_2_3@@UAE@XZ 1207ba90 f   NameDatatypeValidator.obj
 0001:0007aaa0       ??0NameDatatypeValidator@xercesc_2_3@@QAE@QAVDatatypeValidator@1@QAV?$RefHashTableOf@VKVStringPair@xercesc_2_3@@@1@QAV?$RefArrayVectorOf@G@1@HQAVMemoryManager@1@@Z 1207baa0 f   NameDatatypeValidator.obj
 0001:0007ab10       ?newInstance@NameDatatypeValidator@xercesc_2_3@@UAEPAVDatatypeValidator@2@QAV?$RefHashTableOf@VKVStringPair@xercesc_2_3@@@2@QAV?$RefArrayVectorOf@G@2@HQAVMemoryManager@2@@Z 1207bb10 f   NameDatatypeValidator.obj
 0001:0007ab90       ??0NameDatatypeValidator@xercesc_2_3@@IAE@QAVDatatypeValidator@1@QAV?$RefHashTableOf@VKVStringPair@xercesc_2_3@@@1@HW4ValidatorType@21@QAVMemoryManager@1@@Z 1207bb90 f   NameDatatypeValidator.obj
 0001:0007abc0       ?checkValueSpace@NameDatatypeValidator@xercesc_2_3@@MAEXQBG@Z 1207bbc0 f   NameDatatypeValidator.obj
 0001:0007ac10       ??0NCNameDatatypeValidator@xercesc_2_3@@QAE@QAVMemoryManager@1@@Z 1207bc10 f   NCNameDatatypeValidator.obj
 0001:0007ac40       ??_ENCNameDatatypeValidator@xercesc_2_3@@UAEPAXI@Z 1207bc40 f i NCNameDatatypeValidator.obj
 0001:0007aca0       ??1NCNameDatatypeValidator@xercesc_2_3@@UAE@XZ 1207bca0 f   NCNameDatatypeValidator.obj
 0001:0007acb0       ??0NCNameDatatypeValidator@xercesc_2_3@@QAE@QAVDatatypeValidator@1@QAV?$RefHashTableOf@VKVStringPair@xercesc_2_3@@@1@QAV?$RefArrayVectorOf@G@1@HQAVMemoryManager@1@@Z 1207bcb0 f   NCNameDatatypeValidator.obj
 0001:0007ad20       ?newInstance@NCNameDatatypeValidator@xercesc_2_3@@UAEPAVDatatypeValidator@2@QAV?$RefHashTableOf@VKVStringPair@xercesc_2_3@@@2@QAV?$RefArrayVectorOf@G@2@HQAVMemoryManager@2@@Z 1207bd20 f   NCNameDatatypeValidator.obj
 0001:0007ada0       ??0NCNameDatatypeValidator@xercesc_2_3@@IAE@QAVDatatypeValidator@1@QAV?$RefHashTableOf@VKVStringPair@xercesc_2_3@@@1@HW4ValidatorType@21@QAVMemoryManager@1@@Z 1207bda0 f   NCNameDatatypeValidator.obj
 0001:0007add0       ?compare@ENTITYDatatypeValidator@xercesc_2_3@@UAEHQBG0@Z 1207bdd0 f   NCNameDatatypeValidator.obj
 0001:0007add0       ?compare@NameDatatypeValidator@xercesc_2_3@@UAEHQBG0@Z 1207bdd0 f   NCNameDatatypeValidator.obj
 0001:0007add0       ?compare@NCNameDatatypeValidator@xercesc_2_3@@UAEHQBG0@Z 1207bdd0 f   NCNameDatatypeValidator.obj
 0001:0007ae40       ?validate@NameDatatypeValidator@xercesc_2_3@@UAEXQBG@Z 1207be40 f   NCNameDatatypeValidator.obj
 0001:0007ae40       ?validate@NCNameDatatypeValidator@xercesc_2_3@@UAEXQBG@Z 1207be40 f   NCNameDatatypeValidator.obj
 0001:0007ae50       ?checkValueSpace@NCNameDatatypeValidator@xercesc_2_3@@MAEXQBG@Z 1207be50 f   NCNameDatatypeValidator.obj
 0001:0007aea0       ??0NOTATIONDatatypeValidator@xercesc_2_3@@QAE@QAVMemoryManager@1@@Z 1207bea0 f   NOTATIONDatatypeValidator.obj
 0001:0007aed0       ??_ENOTATIONDatatypeValidator@xercesc_2_3@@UAEPAXI@Z 1207bed0 f i NOTATIONDatatypeValidator.obj
 0001:0007af30       ??1NOTATIONDatatypeValidator@xercesc_2_3@@UAE@XZ 1207bf30 f   NOTATIONDatatypeValidator.obj
 0001:0007af40       ??0NOTATIONDatatypeValidator@xercesc_2_3@@QAE@QAVDatatypeValidator@1@QAV?$RefHashTableOf@VKVStringPair@xercesc_2_3@@@1@QAV?$RefArrayVectorOf@G@1@HQAVMemoryManager@1@@Z 1207bf40 f   NOTATIONDatatypeValidator.obj
 0001:0007afb0       ?newInstance@NOTATIONDatatypeValidator@xercesc_2_3@@UAEPAVDatatypeValidator@2@QAV?$RefHashTableOf@VKVStringPair@xercesc_2_3@@@2@QAV?$RefArrayVectorOf@G@2@HQAVMemoryManager@2@@Z 1207bfb0 f   NOTATIONDatatypeValidator.obj
 0001:0007b030       ?assignAdditionalFacet@NOTATIONDatatypeValidator@xercesc_2_3@@MAEXQBG0@Z 1207c030 f   NOTATIONDatatypeValidator.obj
 0001:0007b070       ?checkValueSpace@NOTATIONDatatypeValidator@xercesc_2_3@@MAEXQBG@Z 1207c070 f   NOTATIONDatatypeValidator.obj
 0001:0007b2d0       ??0QNameDatatypeValidator@xercesc_2_3@@QAE@QAVMemoryManager@1@@Z 1207c2d0 f   QNameDatatypeValidator.obj
 0001:0007b300       ??_EQNameDatatypeValidator@xercesc_2_3@@UAEPAXI@Z 1207c300 f i QNameDatatypeValidator.obj
 0001:0007b360       ??1QNameDatatypeValidator@xercesc_2_3@@UAE@XZ 1207c360 f   QNameDatatypeValidator.obj
 0001:0007b370       ??0QNameDatatypeValidator@xercesc_2_3@@QAE@QAVDatatypeValidator@1@QAV?$RefHashTableOf@VKVStringPair@xercesc_2_3@@@1@QAV?$RefArrayVectorOf@G@1@HQAVMemoryManager@1@@Z 1207c370 f   QNameDatatypeValidator.obj
 0001:0007b3e0       ?newInstance@QNameDatatypeValidator@xercesc_2_3@@UAEPAVDatatypeValidator@2@QAV?$RefHashTableOf@VKVStringPair@xercesc_2_3@@@2@QAV?$RefArrayVectorOf@G@2@HQAVMemoryManager@2@@Z 1207c3e0 f   QNameDatatypeValidator.obj
 0001:0007b460       ?assignAdditionalFacet@QNameDatatypeValidator@xercesc_2_3@@MAEXQBG0@Z 1207c460 f   QNameDatatypeValidator.obj
 0001:0007b4a0       ?checkValueSpace@QNameDatatypeValidator@xercesc_2_3@@MAEXQBG@Z 1207c4a0 f   QNameDatatypeValidator.obj
 0001:0007b4f0       ??0StringDatatypeValidator@xercesc_2_3@@QAE@QAVMemoryManager@1@@Z 1207c4f0 f   StringDatatypeValidator.obj
 0001:0007b520       ??_EStringDatatypeValidator@xercesc_2_3@@UAEPAXI@Z 1207c520 f i StringDatatypeValidator.obj
 0001:0007b580       ??0StringDatatypeValidator@xercesc_2_3@@QAE@QAVDatatypeValidator@1@QAV?$RefHashTableOf@VKVStringPair@xercesc_2_3@@@1@QAV?$RefArrayVectorOf@G@1@HQAVMemoryManager@1@@Z 1207c580 f   StringDatatypeValidator.obj
 0001:0007b5f0       ??1StringDatatypeValidator@xercesc_2_3@@UAE@XZ 1207c5f0 f   StringDatatypeValidator.obj
 0001:0007b600       ?newInstance@StringDatatypeValidator@xercesc_2_3@@UAEPAVDatatypeValidator@2@QAV?$RefHashTableOf@VKVStringPair@xercesc_2_3@@@2@QAV?$RefArrayVectorOf@G@2@HQAVMemoryManager@2@@Z 1207c600 f   StringDatatypeValidator.obj
 0001:0007b6a0       ??0StringDatatypeValidator@xercesc_2_3@@IAE@QAVDatatypeValidator@1@QAV?$RefHashTableOf@VKVStringPair@xercesc_2_3@@@1@HW4ValidatorType@21@QAVMemoryManager@1@@Z 1207c6a0 f   StringDatatypeValidator.obj
 0001:0007b6e0       ?getWSFacet@StringDatatypeValidator@xercesc_2_3@@UBEFXZ 1207c6e0 f   StringDatatypeValidator.obj
 0001:0007b6f0       ?assignAdditionalFacet@StringDatatypeValidator@xercesc_2_3@@MAEXQBG0@Z 1207c6f0 f   StringDatatypeValidator.obj
 0001:0007b8f0       ?inheritAdditionalFacet@StringDatatypeValidator@xercesc_2_3@@MAEXXZ 1207c8f0 f   StringDatatypeValidator.obj
 0001:0007b920       ?checkAdditionalFacetConstraints@StringDatatypeValidator@xercesc_2_3@@MBEXXZ 1207c920 f   StringDatatypeValidator.obj
 0001:0007ba20       ?checkAdditionalFacet@StringDatatypeValidator@xercesc_2_3@@MBEXQBG@Z 1207ca20 f   StringDatatypeValidator.obj
 0001:0007bad0       ??0TimeDatatypeValidator@xercesc_2_3@@QAE@QAVMemoryManager@1@@Z 1207cad0 f   TimeDatatypeValidator.obj
 0001:0007bb00       ??_ETimeDatatypeValidator@xercesc_2_3@@UAEPAXI@Z 1207cb00 f i TimeDatatypeValidator.obj
 0001:0007bb60       ??0TimeDatatypeValidator@xercesc_2_3@@QAE@QAVDatatypeValidator@1@QAV?$RefHashTableOf@VKVStringPair@xercesc_2_3@@@1@QAV?$RefArrayVectorOf@G@1@HQAVMemoryManager@1@@Z 1207cb60 f   TimeDatatypeValidator.obj
 0001:0007bbd0       ??1TimeDatatypeValidator@xercesc_2_3@@UAE@XZ 1207cbd0 f   TimeDatatypeValidator.obj
 0001:0007bbe0       ?newInstance@TimeDatatypeValidator@xercesc_2_3@@UAEPAVDatatypeValidator@2@QAV?$RefHashTableOf@VKVStringPair@xercesc_2_3@@@2@QAV?$RefArrayVectorOf@G@2@HQAVMemoryManager@2@@Z 1207cbe0 f   TimeDatatypeValidator.obj
 0001:0007bc60       ?parse@TimeDatatypeValidator@xercesc_2_3@@MAEPAVXMLDateTime@2@QBG@Z 1207cc60 f   TimeDatatypeValidator.obj
 0001:0007bd00       ??0UnionDatatypeValidator@xercesc_2_3@@QAE@QAVMemoryManager@1@@Z 1207cd00 f   UnionDatatypeValidator.obj
 0001:0007bd30       ??_EUnionDatatypeValidator@xercesc_2_3@@UAEPAXI@Z 1207cd30 f i UnionDatatypeValidator.obj
 0001:0007bd90       ??1UnionDatatypeValidator@xercesc_2_3@@UAE@XZ 1207cd90 f   UnionDatatypeValidator.obj
 0001:0007be00       ??0UnionDatatypeValidator@xercesc_2_3@@QAE@QAV?$RefVectorOf@VDatatypeValidator@xercesc_2_3@@@1@HQAVMemoryManager@1@@Z 1207ce00 f   UnionDatatypeValidator.obj
 0001:0007beb0       ??0UnionDatatypeValidator@xercesc_2_3@@QAE@QAVDatatypeValidator@1@QAV?$RefHashTableOf@VKVStringPair@xercesc_2_3@@@1@QAV?$RefArrayVectorOf@G@1@HQAVMemoryManager@1@@Z 1207ceb0 f   UnionDatatypeValidator.obj
 0001:0007c000       ?init@UnionDatatypeValidator@xercesc_2_3@@AAEXQAVDatatypeValidator@2@QAV?$RefHashTableOf@VKVStringPair@xercesc_2_3@@@2@QAV?$RefArrayVectorOf@G@2@@Z 1207d000 f   UnionDatatypeValidator.obj
 0001:0007c320       ?checkContent@UnionDatatypeValidator@xercesc_2_3@@AAEXQBG_N@Z 1207d320 f   UnionDatatypeValidator.obj
 0001:0007c740       ?compare@UnionDatatypeValidator@xercesc_2_3@@UAEHQBG0@Z 1207d740 f   UnionDatatypeValidator.obj
 0001:0007c7d0       ??_G?$RefHashTableOf@VKVStringPair@xercesc_2_3@@@xercesc_2_3@@QAEPAXI@Z 1207d7d0 f i UnionDatatypeValidator.obj
 0001:0007c870       ??0YearDatatypeValidator@xercesc_2_3@@QAE@QAVMemoryManager@1@@Z 1207d870 f   YearDatatypeValidator.obj
 0001:0007c8a0       ??_EYearDatatypeValidator@xercesc_2_3@@UAEPAXI@Z 1207d8a0 f i YearDatatypeValidator.obj
 0001:0007c900       ??0YearDatatypeValidator@xercesc_2_3@@QAE@QAVDatatypeValidator@1@QAV?$RefHashTableOf@VKVStringPair@xercesc_2_3@@@1@QAV?$RefArrayVectorOf@G@1@HQAVMemoryManager@1@@Z 1207d900 f   YearDatatypeValidator.obj
 0001:0007c970       ??1YearDatatypeValidator@xercesc_2_3@@UAE@XZ 1207d970 f   YearDatatypeValidator.obj
 0001:0007c980       ?newInstance@YearDatatypeValidator@xercesc_2_3@@UAEPAVDatatypeValidator@2@QAV?$RefHashTableOf@VKVStringPair@xercesc_2_3@@@2@QAV?$RefArrayVectorOf@G@2@HQAVMemoryManager@2@@Z 1207d980 f   YearDatatypeValidator.obj
 0001:0007ca00       ?parse@YearDatatypeValidator@xercesc_2_3@@MAEPAVXMLDateTime@2@QBG@Z 1207da00 f   YearDatatypeValidator.obj
 0001:0007caa0       ??0YearMonthDatatypeValidator@xercesc_2_3@@QAE@QAVMemoryManager@1@@Z 1207daa0 f   YearMonthDatatypeValidator.obj
 0001:0007cad0       ??_EYearMonthDatatypeValidator@xercesc_2_3@@UAEPAXI@Z 1207dad0 f i YearMonthDatatypeValidator.obj
 0001:0007cb30       ??0YearMonthDatatypeValidator@xercesc_2_3@@QAE@QAVDatatypeValidator@1@QAV?$RefHashTableOf@VKVStringPair@xercesc_2_3@@@1@QAV?$RefArrayVectorOf@G@1@HQAVMemoryManager@1@@Z 1207db30 f   YearMonthDatatypeValidator.obj
 0001:0007cba0       ??1YearMonthDatatypeValidator@xercesc_2_3@@UAE@XZ 1207dba0 f   YearMonthDatatypeValidator.obj
 0001:0007cbb0       ?newInstance@YearMonthDatatypeValidator@xercesc_2_3@@UAEPAVDatatypeValidator@2@QAV?$RefHashTableOf@VKVStringPair@xercesc_2_3@@@2@QAV?$RefArrayVectorOf@G@2@HQAVMemoryManager@2@@Z 1207dbb0 f   YearMonthDatatypeValidator.obj
 0001:0007cc30       ?parse@YearMonthDatatypeValidator@xercesc_2_3@@MAEPAVXMLDateTime@2@QBG@Z 1207dc30 f   YearMonthDatatypeValidator.obj
 0001:0007ccd0       ??0DTDAttDef@xercesc_2_3@@QAE@QAVMemoryManager@1@@Z 1207dcd0 f   DTDAttDef.obj
 0001:0007cd00       ??_EDTDAttDef@xercesc_2_3@@UAEPAXI@Z 1207dd00 f i DTDAttDef.obj
 0001:0007cd60       ??0DTDAttDef@xercesc_2_3@@QAE@QBGW4AttTypes@XMLAttDef@1@W4DefAttTypes@31@QAVMemoryManager@1@@Z 1207dd60 f   DTDAttDef.obj
 0001:0007ce30       ??0DTDAttDef@xercesc_2_3@@QAE@QBG0W4AttTypes@XMLAttDef@1@W4DefAttTypes@31@0QAVMemoryManager@1@@Z 1207de30 f   DTDAttDef.obj
 0001:0007cf00       ??1DTDAttDef@xercesc_2_3@@UAE@XZ 1207df00 f   DTDAttDef.obj
 0001:0007cf60       ?setName@DTDAttDef@xercesc_2_3@@QAEXQBG@Z 1207df60 f   DTDAttDef.obj
 0001:0007cfd0       ??0DTDAttDefList@xercesc_2_3@@QAE@ABV01@@Z 1207dfd0 f i DTDAttDefList.obj
 0001:0007d000       ??4DTDAttDefList@xercesc_2_3@@QAEAAV01@ABV01@@Z 1207e000 f i DTDAttDefList.obj
 0001:0007d000       ??4DOMException@xercesc_2_3@@QAEAAV01@ABV01@@Z 1207e000 f i DTDAttDefList.obj
 0001:0007d000       ??4SchemaAttDefList@xercesc_2_3@@QAEAAV01@ABV01@@Z 1207e000 f i DTDAttDefList.obj
 0001:0007d020       ??_EDTDAttDefList@xercesc_2_3@@UAEPAXI@Z 1207e020 f i DTDAttDefList.obj
 0001:0007d080       ??0DTDAttDefList@xercesc_2_3@@QAE@QAV?$RefHashTableOf@VDTDAttDef@xercesc_2_3@@@1@@Z 1207e080 f   DTDAttDefList.obj
 0001:0007d180       ??1DTDAttDefList@xercesc_2_3@@UAE@XZ 1207e180 f   DTDAttDefList.obj
 0001:0007d1d0       ?findAttDef@DTDAttDefList@xercesc_2_3@@UAEPAVXMLAttDef@2@QBG0@Z 1207e1d0 f   DTDAttDefList.obj
 0001:0007d1d0       ?findAttDef@DTDAttDefList@xercesc_2_3@@UAEPAVXMLAttDef@2@KQBG@Z 1207e1d0 f   DTDAttDefList.obj
 0001:0007d1d0       ?findAttDef@DTDAttDefList@xercesc_2_3@@UBEPBVXMLAttDef@2@QBG0@Z 1207e1d0 f   DTDAttDefList.obj
 0001:0007d1d0       ?findAttDef@DTDAttDefList@xercesc_2_3@@UBEPBVXMLAttDef@2@KQBG@Z 1207e1d0 f   DTDAttDefList.obj
 0001:0007d260       ?Reset@DTDAttDefList@xercesc_2_3@@UAEXXZ 1207e260 f   DTDAttDefList.obj
 0001:0007d260       ?Reset@SchemaAttDefList@xercesc_2_3@@UAEXXZ 1207e260 f   DTDAttDefList.obj
 0001:0007d270       ??1?$XMLEnumerator@VDTDAttDef@xercesc_2_3@@@xercesc_2_3@@UAE@XZ 1207e270 f i DTDAttDefList.obj
 0001:0007d280       ??_G?$XMLEnumerator@VDTDAttDef@xercesc_2_3@@@xercesc_2_3@@UAEPAXI@Z 1207e280 f i DTDAttDefList.obj
 0001:0007d280       ??_E?$XMLEnumerator@VDTDAttDef@xercesc_2_3@@@xercesc_2_3@@UAEPAXI@Z 1207e280 f i DTDAttDefList.obj
 0001:0007d2a0       ??_G?$RefHashTableOfEnumerator@VDTDAttDef@xercesc_2_3@@@xercesc_2_3@@UAEPAXI@Z 1207e2a0 f i DTDAttDefList.obj
 0001:0007d2a0       ??_E?$RefHashTableOfEnumerator@VDTDAttDef@xercesc_2_3@@@xercesc_2_3@@UAEPAXI@Z 1207e2a0 f i DTDAttDefList.obj
 0001:0007d2c0       ??1?$RefHashTableOfEnumerator@VDTDAttDef@xercesc_2_3@@@xercesc_2_3@@UAE@XZ 1207e2c0 f i DTDAttDefList.obj
 0001:0007d3b0       ??0DTDElementDecl@xercesc_2_3@@QAE@QAVMemoryManager@1@@Z 1207e3b0 f   DTDElementDecl.obj
 0001:0007d3f0       ??_EDTDElementDecl@xercesc_2_3@@UAEPAXI@Z 1207e3f0 f i DTDElementDecl.obj
 0001:0007d450       ??0DTDElementDecl@xercesc_2_3@@QAE@QBGIW4ModelTypes@01@QAVMemoryManager@1@@Z 1207e450 f   DTDElementDecl.obj
 0001:0007d4c0       ??0DTDElementDecl@xercesc_2_3@@QAE@QAVQName@1@W4ModelTypes@01@QAVMemoryManager@1@@Z 1207e4c0 f   DTDElementDecl.obj
 0001:0007d530       ??1DTDElementDecl@xercesc_2_3@@UAE@XZ 1207e530 f   DTDElementDecl.obj
 0001:0007d670       ??_GContentSpecNode@xercesc_2_3@@QAEPAXI@Z 1207e670 f i DTDElementDecl.obj
 0001:0007d6d0       ?findAttr@DTDElementDecl@xercesc_2_3@@UBEPAVXMLAttDef@2@QBGI00W4LookupOpts@XMLElementDecl@2@AA_N@Z 1207e6d0 f   DTDElementDecl.obj
 0001:0007d9b0       ?getAttDefList@DTDElementDecl@xercesc_2_3@@UBEAAVXMLAttDefList@2@XZ 1207e9b0 f   DTDElementDecl.obj
 0001:0007dae0       ?getCharDataOpts@DTDElementDecl@xercesc_2_3@@UBE?AW4CharDataOpts@XMLElementDecl@2@XZ 1207eae0 f   DTDElementDecl.obj
 0001:0007db00       ?hasAttDefs@DTDElementDecl@xercesc_2_3@@UBE_NXZ 1207eb00 f   DTDElementDecl.obj
 0001:0007db40       ?resetDefs@DTDElementDecl@xercesc_2_3@@UAE_NXZ 1207eb40 f   DTDElementDecl.obj
 0001:0007dd00       ?setContentSpec@DTDElementDecl@xercesc_2_3@@UAEXPAVContentSpecNode@2@@Z 1207ed00 f   DTDElementDecl.obj
 0001:0007dd70       ?getFormattedContentModel@DTDElementDecl@xercesc_2_3@@UBEPBGXZ 1207ed70 f   DTDElementDecl.obj
 0001:0007dd90       ?getAttDef@DTDElementDecl@xercesc_2_3@@QAEPAVDTDAttDef@2@QBG@Z 1207ed90 f   DTDElementDecl.obj
 0001:0007dd90       ?getAttDef@DTDElementDecl@xercesc_2_3@@QBEPBVDTDAttDef@2@QBG@Z 1207ed90 f   DTDElementDecl.obj
 0001:0007de30       ?addAttDef@DTDElementDecl@xercesc_2_3@@QAEXQAVDTDAttDef@2@@Z 1207ee30 f   DTDElementDecl.obj
 0001:0007de60       ?formatContentModel@DTDElementDecl@xercesc_2_3@@ABEPAGXZ 1207ee60 f   DTDElementDecl.obj
 0001:0007e010       ?makeContentModel@DTDElementDecl@xercesc_2_3@@AAEPAVXMLContentModel@2@XZ 1207f010 f   DTDElementDecl.obj
 0001:0007e100       ?createChildModel@DTDElementDecl@xercesc_2_3@@AAEPAVXMLContentModel@2@XZ 1207f100 f   DTDElementDecl.obj
 0001:0007e5b0       ??_GSimpleContentModel@xercesc_2_3@@UAEPAXI@Z 1207f5b0 f i DTDElementDecl.obj
 0001:0007e5b0       ??_ESimpleContentModel@xercesc_2_3@@UAEPAXI@Z 1207f5b0 f i DTDElementDecl.obj
 0001:0007e5d0       ??1SimpleContentModel@xercesc_2_3@@UAE@XZ 1207f5d0 f i DTDElementDecl.obj
 0001:0007e650       ?getNextState@SimpleContentModel@xercesc_2_3@@UBEIII@Z 1207f650 f i DTDElementDecl.obj
 0001:0007e650       ?getNextState@MixedContentModel@xercesc_2_3@@UBEIII@Z 1207f650 f i DTDElementDecl.obj
 0001:0007e650       ?getNextState@AllContentModel@xercesc_2_3@@UBEIII@Z 1207f650 f i DTDElementDecl.obj
 0001:0007e660       ?faultInAttDefList@DTDElementDecl@xercesc_2_3@@ABEXXZ 1207f660 f   DTDElementDecl.obj
 0001:0007e750       ??0?$RefHashTableOf@VDTDAttDef@xercesc_2_3@@@xercesc_2_3@@QAE@I_NQAVMemoryManager@1@@Z 1207f750 f i DTDElementDecl.obj
 0001:0007e840       ?put@?$RefHashTableOf@VDTDAttDef@xercesc_2_3@@@xercesc_2_3@@QAEXPAXQAVDTDAttDef@2@@Z 1207f840 f i DTDElementDecl.obj
 0001:0007ea50       ??0DTDGrammar@xercesc_2_3@@QAE@QAVMemoryManager@1@@Z 1207fa50 f   DTDGrammar.obj
 0001:0007ec90       ??_EDTDGrammar@xercesc_2_3@@UAEPAXI@Z 1207fc90 f i DTDGrammar.obj
 0001:0007ecf0       ??1DTDGrammar@xercesc_2_3@@UAE@XZ 1207fcf0 f   DTDGrammar.obj
 0001:0007ee80       ?findOrAddElemDecl@DTDGrammar@xercesc_2_3@@UAEPAVXMLElementDecl@2@IQBG00IAA_N@Z 1207fe80 f   DTDGrammar.obj
 0001:0007f0b0       ?putElemDecl@DTDGrammar@xercesc_2_3@@UAEPAVXMLElementDecl@2@IQBG00I_N@Z 120800b0 f   DTDGrammar.obj
 0001:0007f390       ?reset@DTDGrammar@xercesc_2_3@@UAEXXZ 12080390 f   DTDGrammar.obj
 0001:0007f4d0       ?resetEntityDeclPool@DTDGrammar@xercesc_2_3@@AAEXXZ 120804d0 f   DTDGrammar.obj
 0001:0007f820       ?removeAll@?$NameIdPool@VDTDElementDecl@xercesc_2_3@@@xercesc_2_3@@QAEXXZ 12080820 f i DTDGrammar.obj
 0001:0007f890       ??0?$NameIdPool@VXMLNotationDecl@xercesc_2_3@@@xercesc_2_3@@QAE@IIQAVMemoryManager@1@@Z 12080890 f i DTDGrammar.obj
 0001:0007f940       ?removeAll@?$NameIdPool@VXMLNotationDecl@xercesc_2_3@@@xercesc_2_3@@QAEXXZ 12080940 f i DTDGrammar.obj
 0001:0007f9c0       ??_GRangeTokenElemMap@xercesc_2_3@@QAEPAXI@Z 120809c0 f i DTDGrammar.obj
 0001:0007f9c0       ??_G?$NameIdPoolBucketElem@VXMLNotationDecl@xercesc_2_3@@@xercesc_2_3@@QAEPAXI@Z 120809c0 f i DTDGrammar.obj
 0001:0007f9c0       ??_G?$NameIdPoolBucketElem@VDTDEntityDecl@xercesc_2_3@@@xercesc_2_3@@QAEPAXI@Z 120809c0 f i DTDGrammar.obj
 0001:0007f9c0       ??_G?$KeyRefPair@XVDOMUserDataHandler@xercesc_2_3@@@xercesc_2_3@@QAEPAXI@Z 120809c0 f i DTDGrammar.obj
 0001:0007f9e0       ??_GXMLNotationDecl@xercesc_2_3@@QAEPAXI@Z 120809e0 f i DTDGrammar.obj
 0001:0007fa00       ?findBucketElem@?$NameIdPool@VDTDElementDecl@xercesc_2_3@@@xercesc_2_3@@AAEPAU?$NameIdPoolBucketElem@VDTDElementDecl@xercesc_2_3@@@2@QBGAAI@Z 12080a00 f i DTDGrammar.obj
 0001:0007fac0       ??0DTDScanner@xercesc_2_3@@QAE@PAVDTDGrammar@1@QAVDocTypeHandler@1@QAVMemoryManager@1@@Z 12080ac0 f   DTDScanner.obj
 0001:0007fbb0       ??_EDTDScanner@xercesc_2_3@@UAEPAXI@Z 12080bb0 f i DTDScanner.obj
 0001:0007fcc0       ??1DTDScanner@xercesc_2_3@@UAE@XZ 12080cc0 f   DTDScanner.obj
 0001:0007fd70       ?setScannerInfo@DTDScanner@xercesc_2_3@@QAEXQAVXMLScanner@2@QAVReaderMgr@2@QAVXMLBufferMgr@2@@Z 12080d70 f   DTDScanner.obj
 0001:0007fdc0       ?checkForPERef@DTDScanner@xercesc_2_3@@AAE_N_N000@Z 12080dc0 f   DTDScanner.obj
 0001:0007fe50       ?expandPERef@DTDScanner@xercesc_2_3@@AAE_N_N000@Z 12080e50 f   DTDScanner.obj
 0001:00080220       ?getQuotedString@DTDScanner@xercesc_2_3@@AAE_NAAVXMLBuffer@2@@Z 12081220 f   DTDScanner.obj
 0001:00080290       ?scanAttDef@DTDScanner@xercesc_2_3@@AAEPAVXMLAttDef@2@AAVDTDElementDecl@2@AAVXMLBuffer@2@@Z 12081290 f   DTDScanner.obj
 0001:00080b80       ?scanAttListDecl@DTDScanner@xercesc_2_3@@AAEXXZ 12081b80 f   DTDScanner.obj
 0001:00080eb0       ?scanAttValue@DTDScanner@xercesc_2_3@@AAE_NQBGAAVXMLBuffer@2@W4AttTypes@XMLAttDef@2@@Z 12081eb0 f   DTDScanner.obj
 0001:000811f0       ?scanCharRef@DTDScanner@xercesc_2_3@@AAE_NAAG0@Z 120821f0 f   DTDScanner.obj
 0001:00081410       ?scanChildren@DTDScanner@xercesc_2_3@@AAEPAVContentSpecNode@2@ABVDTDElementDecl@2@AAVXMLBuffer@2@@Z 12082410 f   DTDScanner.obj
 0001:00081c80       ??1ContentSpecNode@xercesc_2_3@@QAE@XZ 12082c80 f i DTDScanner.obj
 0001:00081ce0       ??_GQName@xercesc_2_3@@QAEPAXI@Z 12082ce0 f i DTDScanner.obj
 0001:00081dd0       ?scanComment@DTDScanner@xercesc_2_3@@AAEXXZ 12082dd0 f   DTDScanner.obj
 0001:00082010       ?scanContentSpec@DTDScanner@xercesc_2_3@@AAE_NAAVDTDElementDecl@2@@Z 12083010 f   DTDScanner.obj
 0001:000821f0       ?scanDefaultDecl@DTDScanner@xercesc_2_3@@AAEXAAVDTDAttDef@2@@Z 120831f0 f   DTDScanner.obj
 0001:000823b0       ?scanElementDecl@DTDScanner@xercesc_2_3@@AAEXXZ 120833b0 f   DTDScanner.obj
 0001:00082680       ?scanEntityDecl@DTDScanner@xercesc_2_3@@AAEXXZ 12083680 f   DTDScanner.obj
 0001:00082b10       ?scanEntityRef@DTDScanner@xercesc_2_3@@AAE?AW4EntityExpRes@12@AAG0AA_N@Z 12083b10 f   DTDScanner.obj
 0001:00082f00       ?scanEntityLiteral@DTDScanner@xercesc_2_3@@AAE_NAAVXMLBuffer@2@_N@Z 12083f00 f   DTDScanner.obj
 0001:00083290       ?scanEntityDef@DTDScanner@xercesc_2_3@@AAE_NAAVDTDEntityDecl@2@_N@Z 12084290 f   DTDScanner.obj
 0001:000836b0       ?scanEnumeration@DTDScanner@xercesc_2_3@@AAE_NABVDTDAttDef@2@AAVXMLBuffer@2@_N@Z 120846b0 f   DTDScanner.obj
 0001:00083840       ?scanEq@DTDScanner@xercesc_2_3@@AAE_NXZ 12084840 f   DTDScanner.obj
 0001:00083870       ?scanExtSubsetDecl@DTDScanner@xercesc_2_3@@QAEX_N0@Z 12084870 f   DTDScanner.obj
 0001:00083c30       ?scanId@DTDScanner@xercesc_2_3@@QAE_NAAVXMLBuffer@2@0W4IDTypes@12@@Z 12084c30 f   DTDScanner.obj
 0001:00083ed0       ?scanIgnoredSection@DTDScanner@xercesc_2_3@@AAEXXZ 12084ed0 f   DTDScanner.obj
 0001:00084050       ?scanInternalSubset@DTDScanner@xercesc_2_3@@QAE_NXZ 12085050 f   DTDScanner.obj
 0001:00084290       ?scanMarkupDecl@DTDScanner@xercesc_2_3@@AAEX_N@Z 12085290 f   DTDScanner.obj
 0001:000845d0       ?scanMixed@DTDScanner@xercesc_2_3@@AAE_NAAVDTDElementDecl@2@@Z 120855d0 f   DTDScanner.obj
 0001:00084b30       ?scanNotationDecl@DTDScanner@xercesc_2_3@@AAEXXZ 12085b30 f   DTDScanner.obj
 0001:00084ea0       ?scanPI@DTDScanner@xercesc_2_3@@AAEXXZ 12085ea0 f   DTDScanner.obj
 0001:000851d0       ?scanPublicLiteral@DTDScanner@xercesc_2_3@@AAE_NAAVXMLBuffer@2@@Z 120861d0 f   DTDScanner.obj
 0001:000852c0       ?scanSystemLiteral@DTDScanner@xercesc_2_3@@AAE_NAAVXMLBuffer@2@@Z 120862c0 f   DTDScanner.obj
 0001:00085370       ?scanTextDecl@DTDScanner@xercesc_2_3@@AAEXXZ 12086370 f   DTDScanner.obj
 0001:000857e0       ??1?$FlagJanitor@_N@xercesc_2_3@@QAE@XZ 120867e0 f i DTDScanner.obj
 0001:000857f0       ??0DTDValidator@xercesc_2_3@@QAE@QAVXMLErrorReporter@1@@Z 120867f0 f   DTDValidator.obj
 0001:00085810       ??_EDTDValidator@xercesc_2_3@@UAEPAXI@Z 12086810 f i DTDValidator.obj
 0001:00085870       ??1DTDValidator@xercesc_2_3@@UAE@XZ 12086870 f   DTDValidator.obj
 0001:00085880       ?checkContent@DTDValidator@xercesc_2_3@@UAEHQAVXMLElementDecl@2@QAPAVQName@2@I@Z 12086880 f   DTDValidator.obj
 0001:00085930       ?faultInAttr@DTDValidator@xercesc_2_3@@UBEXAAVXMLAttr@2@ABVXMLAttDef@2@@Z 12086930 f   DTDValidator.obj
 0001:00085a50       ?validateAttrValue@DTDValidator@xercesc_2_3@@UAEXPBVXMLAttDef@2@QBG_NPBVXMLElementDecl@2@@Z 12086a50 f   DTDValidator.obj
 0001:00086150       ?preContentValidation@DTDValidator@xercesc_2_3@@UAEX_N0@Z 12087150 f   DTDValidator.obj
 0001:00086400       ??0FieldActivator@xercesc_2_3@@QAE@QAVValueStoreCache@1@QAVXPathMatcherStack@1@QAVMemoryManager@1@@Z 12087400 f   FieldActivator.obj
 0001:00086420       ??0FieldActivator@xercesc_2_3@@QAE@ABV01@@Z 12087420 f   FieldActivator.obj
 0001:00086440       ??4FieldActivator@xercesc_2_3@@QAEAAV01@ABV01@@Z 12087440 f   FieldActivator.obj
 0001:00086460       ?activateField@FieldActivator@xercesc_2_3@@QAEPAVXPathMatcher@2@QAVIC_Field@2@H@Z 12087460 f   FieldActivator.obj
 0001:00086600       ?startValueScopeFor@FieldActivator@xercesc_2_3@@QAEXQBVIdentityConstraint@2@H@Z 12087600 f   FieldActivator.obj
 0001:00086700       ?endValueScopeFor@FieldActivator@xercesc_2_3@@QAEXQBVIdentityConstraint@2@H@Z 12087700 f   FieldActivator.obj
 0001:000867b0       ??0FieldValueMap@xercesc_2_3@@QAE@QAVMemoryManager@1@@Z 120877b0 f   FieldValueMap.obj
 0001:000867d0       ??0FieldValueMap@xercesc_2_3@@QAE@ABV01@@Z 120877d0 f   FieldValueMap.obj
 0001:00086a60       ??1FieldValueMap@xercesc_2_3@@QAE@XZ 12087a60 f   FieldValueMap.obj
 0001:00086ab0       ?indexOf@FieldValueMap@xercesc_2_3@@QBEHQBVIC_Field@2@@Z 12087ab0 f   FieldValueMap.obj
 0001:00086b10       ??1XercesNodeTest@xercesc_2_3@@QAE@XZ 12087b10 f i IC_Field.obj
 0001:00086b30       ??1XercesStep@xercesc_2_3@@QAE@XZ 12087b30 f i IC_Field.obj
 0001:00086b60       ?getType@XercesNodeTest@xercesc_2_3@@QBEFXZ 12087b60 f i IC_Field.obj
 0001:00086b60       ?getAxisType@XercesStep@xercesc_2_3@@QBEGXZ 12087b60 f i IC_Field.obj
 0001:00086b70       ??1XercesLocationPath@xercesc_2_3@@QAE@XZ 12087b70 f i IC_Field.obj
 0001:00086b80       ??_EXPathScanner@xercesc_2_3@@UAEPAXI@Z 12087b80 f i IC_Field.obj
 0001:00086be0       ??1XPathScanner@xercesc_2_3@@UAE@XZ 12087be0 f i IC_Field.obj
 0001:00086be0       ??1XPathScannerForSchema@xercesc_2_3@@UAE@XZ 12087be0 f i IC_Field.obj
 0001:00086bf0       ??_EXPathScannerForSchema@xercesc_2_3@@UAEPAXI@Z 12087bf0 f i IC_Field.obj
 0001:00086c50       ?getStepSize@XercesLocationPath@xercesc_2_3@@QBEIXZ 12087c50 f i IC_Field.obj
 0001:00086c60       ?addStep@XercesLocationPath@xercesc_2_3@@QAEXQAVXercesStep@2@@Z 12087c60 f i IC_Field.obj
 0001:00086ce0       ?getStep@XercesLocationPath@xercesc_2_3@@QBEPAVXercesStep@2@I@Z 12087ce0 f i IC_Field.obj
 0001:00086d30       ?addToken@XPathScanner@xercesc_2_3@@MAEXQAV?$ValueVectorOf@H@2@H@Z 12087d30 f i IC_Field.obj
 0001:00086dd0       ??0FieldMatcher@xercesc_2_3@@AAE@QAVXercesXPath@1@QAVIC_Field@1@QAVValueStore@1@QAVMemoryManager@1@@Z 12087dd0 f   IC_Field.obj
 0001:00086e00       ?matched@FieldMatcher@xercesc_2_3@@UAEXQBGQAVDatatypeValidator@2@_N@Z 12087e00 f   IC_Field.obj
 0001:00086e40       ??0IC_Field@xercesc_2_3@@QAE@QAVXercesXPath@1@QAVIdentityConstraint@1@@Z 12087e40 f   IC_Field.obj
 0001:00086e60       ??1IC_Field@xercesc_2_3@@QAE@XZ 12087e60 f   IC_Field.obj
 0001:00086e80       ??8IC_Field@xercesc_2_3@@QBE_NABV01@@Z 12087e80 f   IC_Field.obj
 0001:00086ea0       ??9IC_Field@xercesc_2_3@@QBE_NABV01@@Z 12087ea0 f   IC_Field.obj
 0001:00086ec0       ?createMatcher@IC_Field@xercesc_2_3@@QAEPAVXPathMatcher@2@QAVValueStore@2@QAVMemoryManager@2@@Z 12087ec0 f   IC_Field.obj
 0001:00086f30       ?getType@IC_Key@xercesc_2_3@@UBEFXZ 12087f30 f i IC_Key.obj
 0001:00086f40       ??0IC_Key@xercesc_2_3@@QAE@QBG0QAVMemoryManager@1@@Z 12087f40 f   IC_Key.obj
 0001:00086f70       ??_EIC_Key@xercesc_2_3@@UAEPAXI@Z 12087f70 f i IC_Key.obj
 0001:00086fd0       ??1IC_Key@xercesc_2_3@@UAE@XZ 12087fd0 f   IC_Key.obj
 0001:00086fe0       ?getType@IC_KeyRef@xercesc_2_3@@UBEFXZ 12087fe0 f i IC_KeyRef.obj
 0001:00086fe0       ?getWSFacet@DatatypeValidator@xercesc_2_3@@UBEFXZ 12087fe0 f i IC_KeyRef.obj
 0001:00086ff0       ?getRootElemId@DTDGrammar@xercesc_2_3@@QAEIXZ 12087ff0 f i IC_KeyRef.obj
 0001:00086ff0       ?getPublicId@XMLEntityDecl@xercesc_2_3@@QBEPBGXZ 12087ff0 f i IC_KeyRef.obj
 0001:00086ff0       ?getQueryString@XMLUri@xercesc_2_3@@QBEPBGXZ 12087ff0 f i IC_KeyRef.obj
 0001:00086ff0       ?getGrammar@SchemaValidator@xercesc_2_3@@UBEPAVGrammar@2@XZ 12087ff0 f i IC_KeyRef.obj
 0001:00086ff0       ?getElementId@ComplexTypeInfo@xercesc_2_3@@QBEIXZ 12087ff0 f i IC_KeyRef.obj
 0001:00086ff0       ?getAttributeDeclRegistry@SchemaGrammar@xercesc_2_3@@QBEPAV?$RefHashTableOf@VXMLAttDef@xercesc_2_3@@@2@XZ 12087ff0 f i IC_KeyRef.obj
 0001:00086ff0       ?getValue@XMLAttDef@xercesc_2_3@@QBEPBGXZ 12087ff0 f i IC_KeyRef.obj
 0001:00086ff0       ?getType@DatatypeValidator@xercesc_2_3@@QBE?AW4ValidatorType@12@XZ 12087ff0 f i IC_KeyRef.obj
 0001:00086ff0       ?getCurrentSchemaURL@SchemaInfo@xercesc_2_3@@QBEPAGXZ 12087ff0 f i IC_KeyRef.obj
 0001:00086ff0       ?getKey@IC_KeyRef@xercesc_2_3@@QBEPAVIdentityConstraint@2@XZ 12087ff0 f i IC_KeyRef.obj
 0001:00086ff0       ?getScanner@AbstractDOMParser@xercesc_2_3@@IBEPAVXMLScanner@2@XZ 12087ff0 f i IC_KeyRef.obj
 0001:00087000       ??0IC_KeyRef@xercesc_2_3@@QAE@QBG0QAVIdentityConstraint@1@QAVMemoryManager@1@@Z 12088000 f   IC_KeyRef.obj
 0001:00087030       ??_EIC_KeyRef@xercesc_2_3@@UAEPAXI@Z 12088030 f i IC_KeyRef.obj
 0001:00087090       ??1IC_KeyRef@xercesc_2_3@@UAE@XZ 12088090 f   IC_KeyRef.obj
 0001:000870a0       ??0SelectorMatcher@xercesc_2_3@@AAE@QAVXercesXPath@1@QAVIC_Selector@1@QAVFieldActivator@1@HQAVMemoryManager@1@@Z 120880a0 f   IC_Selector.obj
 0001:000870f0       ?startDocumentFragment@SelectorMatcher@xercesc_2_3@@UAEXXZ 120880f0 f   IC_Selector.obj
 0001:00087110       ?startElement@SelectorMatcher@xercesc_2_3@@UAEXABVXMLElementDecl@2@IQBGABV?$RefVectorOf@VXMLAttr@xercesc_2_3@@@2@I@Z 12088110 f   IC_Selector.obj
 0001:00087210       ?endElement@SelectorMatcher@xercesc_2_3@@UAEXABVXMLElementDecl@2@QBG@Z 12088210 f   IC_Selector.obj
 0001:00087250       ??0IC_Selector@xercesc_2_3@@QAE@QAVXercesXPath@1@QAVIdentityConstraint@1@@Z 12088250 f   IC_Selector.obj
 0001:00087270       ??1IC_Selector@xercesc_2_3@@QAE@XZ 12088270 f   IC_Selector.obj
 0001:00087290       ??8IC_Selector@xercesc_2_3@@QBE_NABV01@@Z 12088290 f   IC_Selector.obj
 0001:000872b0       ??9IC_Selector@xercesc_2_3@@QBE_NABV01@@Z 120882b0 f   IC_Selector.obj
 0001:000872d0       ?createMatcher@IC_Selector@xercesc_2_3@@QAEPAVXPathMatcher@2@QAVFieldActivator@2@HQAVMemoryManager@2@@Z 120882d0 f   IC_Selector.obj
 0001:00087370       ?getType@IC_Unique@xercesc_2_3@@UBEFXZ 12088370 f i IC_Unique.obj
 0001:00087370       ?getWSFacet@AnySimpleTypeDatatypeValidator@xercesc_2_3@@UBEFXZ 12088370 f i IC_Unique.obj
 0001:00087380       ??0IC_Unique@xercesc_2_3@@QAE@QBG0QAVMemoryManager@1@@Z 12088380 f   IC_Unique.obj
 0001:000873b0       ??_EIC_Unique@xercesc_2_3@@UAEPAXI@Z 120883b0 f i IC_Unique.obj
 0001:00087410       ??1IC_Unique@xercesc_2_3@@UAE@XZ 12088410 f   IC_Unique.obj
 0001:00087420       ??0IdentityConstraint@xercesc_2_3@@IAE@QBG0QAVMemoryManager@1@@Z 12088420 f   IdentityConstraint.obj
 0001:00087550       ??_EIdentityConstraint@xercesc_2_3@@UAEPAXI@Z 12088550 f i IdentityConstraint.obj
 0001:000875e0       ??1IdentityConstraint@xercesc_2_3@@UAE@XZ 120885e0 f   IdentityConstraint.obj
 0001:00087630       ??8IdentityConstraint@xercesc_2_3@@QBE_NABV01@@Z 12088630 f   IdentityConstraint.obj
 0001:00087770       ??9IdentityConstraint@xercesc_2_3@@QBE_NABV01@@Z 12088770 f   IdentityConstraint.obj
 0001:00087790       ?setSelector@IdentityConstraint@xercesc_2_3@@QAEXQAVIC_Selector@2@@Z 12088790 f   IdentityConstraint.obj
 0001:000877d0       ?cleanUp@IdentityConstraint@xercesc_2_3@@AAEXXZ 120887d0 f   IdentityConstraint.obj
 0001:00087820       ??0ValueStore@xercesc_2_3@@QAE@QAVIdentityConstraint@1@QAVXMLScanner@1@QAVMemoryManager@1@@Z 12088820 f   ValueStore.obj
 0001:00087880       ??1ValueStore@xercesc_2_3@@QAE@XZ 12088880 f   ValueStore.obj
 0001:000878e0       ?addValue@ValueStore@xercesc_2_3@@QAEXQAVIC_Field@2@QAVDatatypeValidator@2@QBG@Z 120888e0 f   ValueStore.obj
 0001:00087c40       ?append@ValueStore@xercesc_2_3@@QAEXQBV12@@Z 12088c40 f   ValueStore.obj
 0001:00087e50       ?startValueScope@ValueStore@xercesc_2_3@@QAEXXZ 12088e50 f   ValueStore.obj
 0001:00087ed0       ?endValueScope@ValueStore@xercesc_2_3@@QAEXXZ 12088ed0 f   ValueStore.obj
 0001:00087fa0       ?contains@ValueStore@xercesc_2_3@@QAE_NQBVFieldValueMap@2@@Z 12088fa0 f   ValueStore.obj
 0001:00088190       ?isDuplicateOf@ValueStore@xercesc_2_3@@AAE_NQAVDatatypeValidator@2@QBG01@Z 12089190 f   ValueStore.obj
 0001:00088320       ?endDcocumentFragment@ValueStore@xercesc_2_3@@QAEXQAVValueStoreCache@2@@Z 12089320 f   ValueStore.obj
 0001:00088410       ?reportNilError@ValueStore@xercesc_2_3@@QAEXQAVIdentityConstraint@2@@Z 12089410 f   ValueStore.obj
 0001:00088450       ?duplicateValue@ValueStore@xercesc_2_3@@QAEXXZ 12089450 f   ValueStore.obj
 0001:000884b0       ?setElementAt@?$ValueVectorOf@PAVDatatypeValidator@xercesc_2_3@@@xercesc_2_3@@QAEXABQAVDatatypeValidator@2@I@Z 120894b0 f i ValueStore.obj
 0001:00088500       ??0?$ValueVectorOf@PBG@xercesc_2_3@@QAE@IQAVMemoryManager@1@@Z 12089500 f i ValueStore.obj
 0001:00088500       ??0?$ValueVectorOf@PAVDatatypeValidator@xercesc_2_3@@@xercesc_2_3@@QAE@IQAVMemoryManager@1@@Z 12089500 f i ValueStore.obj
 0001:00088500       ??0?$ValueVectorOf@H@xercesc_2_3@@QAE@IQAVMemoryManager@1@@Z 12089500 f i ValueStore.obj
 0001:00088500       ??0?$ValueVectorOf@I@xercesc_2_3@@QAE@IQAVMemoryManager@1@@Z 12089500 f i ValueStore.obj
 0001:00088500       ??0?$ValueVectorOf@PAVSchemaElementDecl@xercesc_2_3@@@xercesc_2_3@@QAE@IQAVMemoryManager@1@@Z 12089500 f i ValueStore.obj
 0001:00088500       ??0?$ValueVectorOf@PAVIC_Field@xercesc_2_3@@@xercesc_2_3@@QAE@IQAVMemoryManager@1@@Z 12089500 f i ValueStore.obj
 0001:00088500       ??0?$ValueVectorOf@PBVDOMElement@xercesc_2_3@@@xercesc_2_3@@QAE@IQAVMemoryManager@1@@Z 12089500 f i ValueStore.obj
 0001:00088550       ?addElement@?$ValueVectorOf@PBG@xercesc_2_3@@QAEXABQBG@Z 12089550 f i ValueStore.obj
 0001:00088550       ?addElement@?$ValueVectorOf@PAVDatatypeValidator@xercesc_2_3@@@xercesc_2_3@@QAEXABQAVDatatypeValidator@2@@Z 12089550 f i ValueStore.obj
 0001:00088550       ?addElement@?$ValueVectorOf@PAVDOMElement@xercesc_2_3@@@xercesc_2_3@@QAEXABQAVDOMElement@2@@Z 12089550 f i ValueStore.obj
 0001:00088550       ?addElement@?$ValueVectorOf@PAVIC_Field@xercesc_2_3@@@xercesc_2_3@@QAEXABQAVIC_Field@2@@Z 12089550 f i ValueStore.obj
 0001:00088550       ?addElement@?$ValueVectorOf@PAVSchemaElementDecl@xercesc_2_3@@@xercesc_2_3@@QAEXABQAVSchemaElementDecl@2@@Z 12089550 f i ValueStore.obj
 0001:00088550       ?addElement@?$ValueVectorOf@I@xercesc_2_3@@QAEXABI@Z 12089550 f i ValueStore.obj
 0001:000885f0       ??_E?$RefVectorOf@VFieldValueMap@xercesc_2_3@@@xercesc_2_3@@UAEPAXI@Z 120895f0 f i ValueStore.obj
 0001:000885f0       ??_G?$RefVectorOf@VFieldValueMap@xercesc_2_3@@@xercesc_2_3@@UAEPAXI@Z 120895f0 f i ValueStore.obj
 0001:00088610       ??1?$RefVectorOf@VFieldValueMap@xercesc_2_3@@@xercesc_2_3@@UAE@XZ 12089610 f i ValueStore.obj
 0001:000886a0       ??1?$BaseRefVectorOf@VFieldValueMap@xercesc_2_3@@@xercesc_2_3@@UAE@XZ 120896a0 f i ValueStore.obj
 0001:000886b0       ??0?$BaseRefVectorOf@VFieldValueMap@xercesc_2_3@@@xercesc_2_3@@QAE@I_NQAVMemoryManager@1@@Z 120896b0 f i ValueStore.obj
 0001:00088710       ??0ValueStoreCache@xercesc_2_3@@QAE@QAVMemoryManager@1@@Z 12089710 f   ValueStoreCache.obj
 0001:00088900       ??1ValueStoreCache@xercesc_2_3@@QAE@XZ 12089900 f   ValueStoreCache.obj
 0001:00088a40       ?startDocument@ValueStoreCache@xercesc_2_3@@QAEXXZ 12089a40 f   ValueStoreCache.obj
 0001:00088c50       ?startElement@ValueStoreCache@xercesc_2_3@@QAEXXZ 12089c50 f   ValueStoreCache.obj
 0001:00088dc0       ?endElement@ValueStoreCache@xercesc_2_3@@QAEXXZ 12089dc0 f   ValueStoreCache.obj
 0001:00089060       ??_G?$RefHashTableOf@VValueStore@xercesc_2_3@@@xercesc_2_3@@QAEPAXI@Z 1208a060 f i ValueStoreCache.obj
 0001:00089100       ?cleanUp@ValueStoreCache@xercesc_2_3@@AAEXXZ 1208a100 f   ValueStoreCache.obj
 0001:00089260       ?init@ValueStoreCache@xercesc_2_3@@AAEXXZ 1208a260 f   ValueStoreCache.obj
 0001:00089480       ?initValueStoresFor@ValueStoreCache@xercesc_2_3@@QAEXQAVSchemaElementDecl@2@H@Z 1208a480 f   ValueStoreCache.obj
 0001:00089700       ?transplant@ValueStoreCache@xercesc_2_3@@QAEXQAVIdentityConstraint@2@H@Z 1208a700 f   ValueStoreCache.obj
 0001:000899d0       ??1?$XMLEnumerator@VValueStore@xercesc_2_3@@@xercesc_2_3@@UAE@XZ 1208a9d0 f i ValueStoreCache.obj
 0001:000899e0       ??_G?$XMLEnumerator@VValueStore@xercesc_2_3@@@xercesc_2_3@@UAEPAXI@Z 1208a9e0 f i ValueStoreCache.obj
 0001:000899e0       ??_E?$XMLEnumerator@VValueStore@xercesc_2_3@@@xercesc_2_3@@UAEPAXI@Z 1208a9e0 f i ValueStoreCache.obj
 0001:00089a00       ??1?$RefHashTableOf@VValueStore@xercesc_2_3@@@xercesc_2_3@@QAE@XZ 1208aa00 f i ValueStoreCache.obj
 0001:00089a90       ??1?$BaseRefVectorOf@V?$RefHashTableOf@VValueStore@xercesc_2_3@@@xercesc_2_3@@@xercesc_2_3@@UAE@XZ 1208aa90 f i ValueStoreCache.obj
 0001:00089aa0       ??1?$RefStackOf@V?$RefHashTableOf@VValueStore@xercesc_2_3@@@xercesc_2_3@@@xercesc_2_3@@QAE@XZ 1208aaa0 f i ValueStoreCache.obj
 0001:00089bc0       ??1?$RefHashTableOfEnumerator@VValueStore@xercesc_2_3@@@xercesc_2_3@@UAE@XZ 1208abc0 f i ValueStoreCache.obj
 0001:00089cb0       ?nextElement@?$RefHashTableOfEnumerator@G@xercesc_2_3@@UAEAAGXZ 1208acb0 f i ValueStoreCache.obj
 0001:00089cb0       ?nextElement@?$RefHashTableOfEnumerator@VXMLRefInfo@xercesc_2_3@@@xercesc_2_3@@UAEAAVXMLRefInfo@2@XZ 1208acb0 f i ValueStoreCache.obj
 0001:00089cb0       ?nextElement@?$RefHashTableOfEnumerator@VDTDAttDef@xercesc_2_3@@@xercesc_2_3@@UAEAAVDTDAttDef@2@XZ 1208acb0 f i ValueStoreCache.obj
 0001:00089cb0       ?nextElement@?$RefHashTableOfEnumerator@VXercesGroupInfo@xercesc_2_3@@@xercesc_2_3@@UAEAAVXercesGroupInfo@2@XZ 1208acb0 f i ValueStoreCache.obj
 0001:00089cb0       ?nextElement@?$RefHashTableOfEnumerator@VGrammar@xercesc_2_3@@@xercesc_2_3@@UAEAAVGrammar@2@XZ 1208acb0 f i ValueStoreCache.obj
 0001:00089cb0       ?nextElement@?$RefHashTableOfEnumerator@V?$KeyRefPair@XVDOMUserDataHandler@xercesc_2_3@@@xercesc_2_3@@@xercesc_2_3@@UAEAAV?$KeyRefPair@XVDOMUserDataHandler@xercesc_2_3@@@2@XZ 1208acb0 f i ValueStoreCache.obj
 0001:00089cb0       ?nextElement@?$RefHashTableOfEnumerator@VKVStringPair@xercesc_2_3@@@xercesc_2_3@@UAEAAVKVStringPair@2@XZ 1208acb0 f i ValueStoreCache.obj
 0001:00089cb0       ?nextElement@?$RefHashTableOfEnumerator@VComplexTypeInfo@xercesc_2_3@@@xercesc_2_3@@UAEAAVComplexTypeInfo@2@XZ 1208acb0 f i ValueStoreCache.obj
 0001:00089cb0       ?nextElement@?$RefHashTableOfEnumerator@VValueStore@xercesc_2_3@@@xercesc_2_3@@UAEAAVValueStore@2@XZ 1208acb0 f i ValueStoreCache.obj
 0001:00089d30       ??_GValueStore@xercesc_2_3@@QAEPAXI@Z 1208ad30 f i ValueStoreCache.obj
 0001:00089d50       ??_G?$RefVectorOf@VValueStore@xercesc_2_3@@@xercesc_2_3@@UAEPAXI@Z 1208ad50 f i ValueStoreCache.obj
 0001:00089d50       ??_E?$RefVectorOf@VValueStore@xercesc_2_3@@@xercesc_2_3@@UAEPAXI@Z 1208ad50 f i ValueStoreCache.obj
 0001:00089d70       ??1?$RefVectorOf@VValueStore@xercesc_2_3@@@xercesc_2_3@@UAE@XZ 1208ad70 f i ValueStoreCache.obj
 0001:00089e00       ??1?$BaseRefVectorOf@VValueStore@xercesc_2_3@@@xercesc_2_3@@UAE@XZ 1208ae00 f i ValueStoreCache.obj
 0001:00089e10       ??_G?$RefVectorOf@V?$RefHashTableOf@VValueStore@xercesc_2_3@@@xercesc_2_3@@@xercesc_2_3@@UAEPAXI@Z 1208ae10 f i ValueStoreCache.obj
 0001:00089e10       ??_E?$RefVectorOf@V?$RefHashTableOf@VValueStore@xercesc_2_3@@@xercesc_2_3@@@xercesc_2_3@@UAEPAXI@Z 1208ae10 f i ValueStoreCache.obj
 0001:00089e30       ??1?$RefVectorOf@V?$RefHashTableOf@VValueStore@xercesc_2_3@@@xercesc_2_3@@@xercesc_2_3@@UAE@XZ 1208ae30 f i ValueStoreCache.obj
 0001:00089f50       ??_E?$RefHashTableOfEnumerator@VValueStore@xercesc_2_3@@@xercesc_2_3@@UAEPAXI@Z 1208af50 f i ValueStoreCache.obj
 0001:00089f50       ??_G?$RefHashTableOfEnumerator@VValueStore@xercesc_2_3@@@xercesc_2_3@@UAEPAXI@Z 1208af50 f i ValueStoreCache.obj
 0001:00089f70       ??0?$BaseRefVectorOf@V?$RefHashTableOf@VValueStore@xercesc_2_3@@@xercesc_2_3@@@xercesc_2_3@@QAE@I_NQAVMemoryManager@1@@Z 1208af70 f i ValueStoreCache.obj
 0001:00089fd0       ??0XPathException@xercesc_2_3@@QAE@QBDIW4Codes@XMLExcepts@1@@Z 1208afd0 f i XercesXPath.obj
 0001:0008a030       ??0XPathException@xercesc_2_3@@QAE@ABV01@@Z 1208b030 f i XercesXPath.obj
 0001:0008a050       ??0XPathException@xercesc_2_3@@QAE@QBDIW4Codes@XMLExcepts@1@QBG222@Z 1208b050 f i XercesXPath.obj
 0001:0008a0c0       ??0XPathException@xercesc_2_3@@QAE@QBDIW4Codes@XMLExcepts@1@0000@Z 1208b0c0 f i XercesXPath.obj
 0001:0008a130       ??1XPathException@xercesc_2_3@@UAE@XZ 1208b130 f i XercesXPath.obj
 0001:0008a140       ?duplicate@XPathException@xercesc_2_3@@UBEPAVXMLException@2@XZ 1208b140 f i XercesXPath.obj
 0001:0008a1a0       ?getType@XPathException@xercesc_2_3@@UBEPBGXZ 1208b1a0 f i XercesXPath.obj
 0001:0008a1b0       ??_EXPathException@xercesc_2_3@@UAEPAXI@Z 1208b1b0 f i XercesXPath.obj
 0001:0008a210       ??_FNamespaceScope@xercesc_2_3@@QAEXXZ 1208b210 f i XercesXPath.obj
 0001:0008a220       ?getNamespaceForPrefix@NamespaceScope@xercesc_2_3@@QBEIQBG@Z 1208b220 f i XercesXPath.obj
 0001:0008a240       ?isEmpty@NamespaceScope@xercesc_2_3@@QBE_NXZ 1208b240 f i XercesXPath.obj
 0001:0008a250       ??0XercesNodeTest@xercesc_2_3@@QAE@FQAVMemoryManager@1@@Z 1208b250 f   XercesXPath.obj
 0001:0008a2c0       ??0XercesNodeTest@xercesc_2_3@@QAE@QBVQName@1@@Z 1208b2c0 f   XercesXPath.obj
 0001:0008a330       ??0XercesNodeTest@xercesc_2_3@@QAE@QBGIQAVMemoryManager@1@@Z 1208b330 f   XercesXPath.obj
 0001:0008a3b0       ??0XercesNodeTest@xercesc_2_3@@QAE@ABV01@@Z 1208b3b0 f   XercesXPath.obj
 0001:0008a420       ??4XercesNodeTest@xercesc_2_3@@QAEAAV01@ABV01@@Z 1208b420 f   XercesXPath.obj
 0001:0008a450       ??8XercesNodeTest@xercesc_2_3@@QBE_NABV01@@Z 1208b450 f   XercesXPath.obj
 0001:0008a480       ??9XercesNodeTest@xercesc_2_3@@QBE_NABV01@@Z 1208b480 f   XercesXPath.obj
 0001:0008a4d0       ??0XercesStep@xercesc_2_3@@QAE@GQAVXercesNodeTest@1@@Z 1208b4d0 f   XercesXPath.obj
 0001:0008a4f0       ??0XercesStep@xercesc_2_3@@QAE@ABV01@@Z 1208b4f0 f   XercesXPath.obj
 0001:0008a5b0       ??4XercesStep@xercesc_2_3@@QAEAAV01@ABV01@@Z 1208b5b0 f   XercesXPath.obj
 0001:0008a5f0       ??8XercesStep@xercesc_2_3@@QBE_NABV01@@Z 1208b5f0 f   XercesXPath.obj
 0001:0008a650       ??9XercesStep@xercesc_2_3@@QBE_NABV01@@Z 1208b650 f   XercesXPath.obj
 0001:0008a6e0       ??0XercesLocationPath@xercesc_2_3@@QAE@QAV?$RefVectorOf@VXercesStep@xercesc_2_3@@@1@@Z 1208b6e0 f   XercesXPath.obj
 0001:0008a6f0       ??8XercesLocationPath@xercesc_2_3@@QBE_NABV01@@Z 1208b6f0 f   XercesXPath.obj
 0001:0008a7d0       ??9XercesLocationPath@xercesc_2_3@@QBE_NABV01@@Z 1208b7d0 f   XercesXPath.obj
 0001:0008a8d0       ??0XercesXPath@xercesc_2_3@@QAE@QBGQAVXMLStringPool@1@QAVNamespaceScope@1@I_NQAVMemoryManager@1@@Z 1208b8d0 f   XercesXPath.obj
 0001:0008aa50       ??8XercesXPath@xercesc_2_3@@QBE_NABV01@@Z 1208ba50 f   XercesXPath.obj
 0001:0008abf0       ??9XercesXPath@xercesc_2_3@@QBE_NABV01@@Z 1208bbf0 f   XercesXPath.obj
 0001:0008ada0       ?cleanUp@XercesXPath@xercesc_2_3@@AAEXXZ 1208bda0 f   XercesXPath.obj
 0001:0008ada0       ??1XercesXPath@xercesc_2_3@@QAE@XZ 1208bda0 f   XercesXPath.obj
 0001:0008adc0       ?checkForSelectedAttributes@XercesXPath@xercesc_2_3@@AAEXXZ 1208bdc0 f   XercesXPath.obj
 0001:0008ae90       ?parseExpression@XercesXPath@xercesc_2_3@@AAEXQAVXMLStringPool@2@QAVNamespaceScope@2@@Z 1208be90 f   XercesXPath.obj
 0001:0008c110       ??0XPathScanner@xercesc_2_3@@QAE@QAVXMLStringPool@1@@Z 1208d110 f   XercesXPath.obj
 0001:0008c170       ?init@XPathScanner@xercesc_2_3@@AAEXXZ 1208d170 f   XercesXPath.obj
 0001:0008c2d0       ?scanExpression@XPathScanner@xercesc_2_3@@QAE_NQBGHHQAV?$ValueVectorOf@H@2@@Z 1208d2d0 f   XercesXPath.obj
 0001:0008d3c0       ?scanNCName@XPathScanner@xercesc_2_3@@AAEHQBGHH@Z 1208e3c0 f   XercesXPath.obj
 0001:0008d420       ?scanNumber@XPathScanner@xercesc_2_3@@AAEHQBGHHQAV?$ValueVectorOf@H@2@@Z 1208e420 f   XercesXPath.obj
 0001:0008d600       ??0XPathScannerForSchema@xercesc_2_3@@QAE@QAVXMLStringPool@1@@Z 1208e600 f   XercesXPath.obj
 0001:0008d620       ?addToken@XPathScannerForSchema@xercesc_2_3@@MAEXQAV?$ValueVectorOf@H@2@H@Z 1208e620 f   XercesXPath.obj
 0001:0008d720       ??_E?$RefVectorOf@VXercesStep@xercesc_2_3@@@xercesc_2_3@@UAEPAXI@Z 1208e720 f i XercesXPath.obj
 0001:0008d720       ??_G?$RefVectorOf@VXercesStep@xercesc_2_3@@@xercesc_2_3@@UAEPAXI@Z 1208e720 f i XercesXPath.obj
 0001:0008d740       ??1?$RefVectorOf@VXercesStep@xercesc_2_3@@@xercesc_2_3@@UAE@XZ 1208e740 f i XercesXPath.obj
 0001:0008d7f0       ??1?$BaseRefVectorOf@VXercesStep@xercesc_2_3@@@xercesc_2_3@@UAE@XZ 1208e7f0 f i XercesXPath.obj
 0001:0008d800       ??_G?$RefVectorOf@VXercesLocationPath@xercesc_2_3@@@xercesc_2_3@@UAEPAXI@Z 1208e800 f i XercesXPath.obj
 0001:0008d800       ??_E?$RefVectorOf@VXercesLocationPath@xercesc_2_3@@@xercesc_2_3@@UAEPAXI@Z 1208e800 f i XercesXPath.obj
 0001:0008d820       ??1?$RefVectorOf@VXercesLocationPath@xercesc_2_3@@@xercesc_2_3@@UAE@XZ 1208e820 f i XercesXPath.obj
 0001:0008d8b0       ??1?$BaseRefVectorOf@VXercesLocationPath@xercesc_2_3@@@xercesc_2_3@@UAE@XZ 1208e8b0 f i XercesXPath.obj
 0001:0008d8c0       ??0?$BaseRefVectorOf@VXercesStep@xercesc_2_3@@@xercesc_2_3@@QAE@I_NQAVMemoryManager@1@@Z 1208e8c0 f i XercesXPath.obj
 0001:0008d920       ??0?$BaseRefVectorOf@VXercesLocationPath@xercesc_2_3@@@xercesc_2_3@@QAE@I_NQAVMemoryManager@1@@Z 1208e920 f i XercesXPath.obj
 0001:0008d980       ??0XPathMatcher@xercesc_2_3@@QAE@QAVXercesXPath@1@QAVMemoryManager@1@@Z 1208e980 f   XPathMatcher.obj
 0001:0008da30       ??_EXPathMatcher@xercesc_2_3@@UAEPAXI@Z 1208ea30 f i XPathMatcher.obj
 0001:0008dac0       ??0XPathMatcher@xercesc_2_3@@QAE@QAVXercesXPath@1@QAVIdentityConstraint@1@QAVMemoryManager@1@@Z 1208eac0 f   XPathMatcher.obj
 0001:0008db70       ??1XPathMatcher@xercesc_2_3@@UAE@XZ 1208eb70 f   XPathMatcher.obj
 0001:0008dbb0       ?init@XPathMatcher@xercesc_2_3@@AAEXQAVXercesXPath@2@@Z 1208ebb0 f   XPathMatcher.obj
 0001:0008ddc0       ?startDocumentFragment@XPathMatcher@xercesc_2_3@@UAEXXZ 1208edc0 f   XPathMatcher.obj
 0001:0008de30       ?startElement@XPathMatcher@xercesc_2_3@@UAEXABVXMLElementDecl@2@IQBGABV?$RefVectorOf@VXMLAttr@xercesc_2_3@@@2@I@Z 1208ee30 f   XPathMatcher.obj
 0001:0008e3e0       ?endElement@XPathMatcher@xercesc_2_3@@UAEXABVXMLElementDecl@2@QBG@Z 1208f3e0 f   XPathMatcher.obj
 0001:0008e560       ?isMatched@XPathMatcher@xercesc_2_3@@QAEHXZ 1208f560 f   XPathMatcher.obj
 0001:0008e5a0       ?attDef@SAXParser@xercesc_2_3@@UAEXABVDTDElementDecl@2@ABVDTDAttDef@2@_N@Z 1208f5a0 f   XPathMatcher.obj
 0001:0008e5a0       ?matched@XPathMatcher@xercesc_2_3@@MAEXQBGQAVDatatypeValidator@2@_N@Z 1208f5a0 f   XPathMatcher.obj
 0001:0008e5b0       ?getInitialDepth@XPathMatcher@xercesc_2_3@@UBEHXZ 1208f5b0 f   XPathMatcher.obj
 0001:0008e5e0       ??_E?$RefVectorOf@V?$ValueStackOf@H@xercesc_2_3@@@xercesc_2_3@@UAEPAXI@Z 1208f5e0 f i XPathMatcher.obj
 0001:0008e5e0       ??_G?$RefVectorOf@V?$ValueStackOf@H@xercesc_2_3@@@xercesc_2_3@@UAEPAXI@Z 1208f5e0 f i XPathMatcher.obj
 0001:0008e600       ??1?$RefVectorOf@V?$ValueStackOf@H@xercesc_2_3@@@xercesc_2_3@@UAE@XZ 1208f600 f i XPathMatcher.obj
 0001:0008e690       ??1?$BaseRefVectorOf@V?$ValueStackOf@H@xercesc_2_3@@@xercesc_2_3@@UAE@XZ 1208f690 f i XPathMatcher.obj
 0001:0008e6a0       ??0XPathMatcherStack@xercesc_2_3@@QAE@QAVMemoryManager@1@@Z 1208f6a0 f   XPathMatcherStack.obj
 0001:0008e7d0       ??1XPathMatcherStack@xercesc_2_3@@QAE@XZ 1208f7d0 f   XPathMatcherStack.obj
 0001:0008e800       ?clear@XPathMatcherStack@xercesc_2_3@@QAEXXZ 1208f800 f   XPathMatcherStack.obj
 0001:0008e860       ??_G?$RefVectorOf@VXPathMatcher@xercesc_2_3@@@xercesc_2_3@@UAEPAXI@Z 1208f860 f i XPathMatcherStack.obj
 0001:0008e860       ??_E?$RefVectorOf@VXPathMatcher@xercesc_2_3@@@xercesc_2_3@@UAEPAXI@Z 1208f860 f i XPathMatcherStack.obj
 0001:0008e880       ??1?$RefVectorOf@VXPathMatcher@xercesc_2_3@@@xercesc_2_3@@UAE@XZ 1208f880 f i XPathMatcherStack.obj
 0001:0008e900       ??1?$BaseRefVectorOf@VXPathMatcher@xercesc_2_3@@@xercesc_2_3@@UAE@XZ 1208f900 f i XPathMatcherStack.obj
 0001:0008e910       ??0SchemaAttDefList@xercesc_2_3@@QAE@ABV01@@Z 1208f910 f i ComplexTypeInfo.obj
 0001:0008e940       ??_ESchemaAttDefList@xercesc_2_3@@UAEPAXI@Z 1208f940 f i ComplexTypeInfo.obj
 0001:0008e9a0       ??1Locator@xercesc_2_3@@UAE@XZ 1208f9a0 f i ComplexTypeInfo.obj
 0001:0008e9a0       ??1XSDLocator@xercesc_2_3@@UAE@XZ 1208f9a0 f i ComplexTypeInfo.obj
 0001:0008e9b0       ??_EXSDLocator@xercesc_2_3@@UAEPAXI@Z 1208f9b0 f i ComplexTypeInfo.obj
 0001:0008ea10       ??0ComplexTypeInfo@xercesc_2_3@@QAE@QAVMemoryManager@1@@Z 1208fa10 f   ComplexTypeInfo.obj
 0001:0008ea90       ??1ComplexTypeInfo@xercesc_2_3@@QAE@XZ 1208fa90 f   ComplexTypeInfo.obj
 0001:0008ec00       ?addAttDef@ComplexTypeInfo@xercesc_2_3@@QAEXQAVSchemaAttDef@2@@Z 1208fc00 f   ComplexTypeInfo.obj
 0001:0008ec40       ?setContentSpec@ComplexTypeInfo@xercesc_2_3@@QAEXQAVContentSpecNode@2@@Z 1208fc40 f   ComplexTypeInfo.obj
 0001:0008ece0       ?setLocator@ComplexTypeInfo@xercesc_2_3@@QAEXQAVXSDLocator@2@@Z 1208fce0 f   ComplexTypeInfo.obj
 0001:0008ed10       ?getAttDefList@ComplexTypeInfo@xercesc_2_3@@QBEAAVXMLAttDefList@2@XZ 1208fd10 f   ComplexTypeInfo.obj
 0001:0008ee40       ?getFormattedContentModel@ComplexTypeInfo@xercesc_2_3@@QBEPBGXZ 1208fe40 f   ComplexTypeInfo.obj
 0001:0008ee60       ?findAttr@ComplexTypeInfo@xercesc_2_3@@QBEPAVXMLAttDef@2@QBGI00W4LookupOpts@XMLElementDecl@2@AA_N@Z 1208fe60 f   ComplexTypeInfo.obj
 0001:0008f070       ?resetDefs@ComplexTypeInfo@xercesc_2_3@@QAE_NXZ 12090070 f   ComplexTypeInfo.obj
 0001:0008f230       ?checkUniqueParticleAttribution@ComplexTypeInfo@xercesc_2_3@@QAEXQAVSchemaGrammar@2@QAVGrammarResolver@2@QAVXMLStringPool@2@QAVXMLValidator@2@@Z 12090230 f   ComplexTypeInfo.obj
 0001:0008f360       ?faultInAttDefList@ComplexTypeInfo@xercesc_2_3@@ABEXXZ 12090360 f   ComplexTypeInfo.obj
 0001:0008f450       ?formatContentModel@ComplexTypeInfo@xercesc_2_3@@ABEPAGXZ 12090450 f   ComplexTypeInfo.obj
 0001:0008f610       ?makeContentModel@ComplexTypeInfo@xercesc_2_3@@AAEPAVXMLContentModel@2@_NQAVContentSpecNode@2@@Z 12090610 f   ComplexTypeInfo.obj
 0001:0008f860       ?createChildModel@ComplexTypeInfo@xercesc_2_3@@AAEPAVXMLContentModel@2@PAVContentSpecNode@2@_N@Z 12090860 f   ComplexTypeInfo.obj
 0001:0008fe00       ?convertContentSpecTree@ComplexTypeInfo@xercesc_2_3@@AAEPAVContentSpecNode@2@QAV32@_N@Z 12090e00 f   ComplexTypeInfo.obj
 0001:0008ff90       ?expandContentModel@ComplexTypeInfo@xercesc_2_3@@AAEPAVContentSpecNode@2@QAV32@HH@Z 12090f90 f   ComplexTypeInfo.obj
 0001:00090380       ?resizeContentSpecOrgURI@ComplexTypeInfo@xercesc_2_3@@AAEXXZ 12091380 f   ComplexTypeInfo.obj
 0001:000903e0       ??0?$RefHash2KeysTableOf@VSchemaAttDef@xercesc_2_3@@@xercesc_2_3@@QAE@I_NQAVMemoryManager@1@@Z 120913e0 f i ComplexTypeInfo.obj
 0001:000904d0       ?put@?$RefHash2KeysTableOf@VSchemaAttDef@xercesc_2_3@@@xercesc_2_3@@QAEXPAXHQAVSchemaAttDef@2@@Z 120914d0 f i ComplexTypeInfo.obj
 0001:000905f0       ??_E?$RefVectorOf@VContentSpecNode@xercesc_2_3@@@xercesc_2_3@@UAEPAXI@Z 120915f0 f i ComplexTypeInfo.obj
 0001:000905f0       ??_G?$RefVectorOf@VContentSpecNode@xercesc_2_3@@@xercesc_2_3@@UAEPAXI@Z 120915f0 f i ComplexTypeInfo.obj
 0001:00090610       ??1?$RefVectorOf@VContentSpecNode@xercesc_2_3@@@xercesc_2_3@@UAE@XZ 12091610 f i ComplexTypeInfo.obj
 0001:000906d0       ??1?$BaseRefVectorOf@VContentSpecNode@xercesc_2_3@@@xercesc_2_3@@UAE@XZ 120916d0 f i ComplexTypeInfo.obj
 0001:00090700       ??0GeneralAttributeCheck@xercesc_2_3@@QAE@QAVMemoryManager@1@@Z 12091700 f   GeneralAttributeCheck.obj
 0001:00090920       ??1GeneralAttributeCheck@xercesc_2_3@@QAE@XZ 12091920 f   GeneralAttributeCheck.obj
 0001:00090930       ?setUpValidators@GeneralAttributeCheck@xercesc_2_3@@AAEXXZ 12091930 f   GeneralAttributeCheck.obj
 0001:00090bd0       ?mapElements@GeneralAttributeCheck@xercesc_2_3@@AAEXXZ 12091bd0 f   GeneralAttributeCheck.obj
 0001:00090e10       ?mapAttributes@GeneralAttributeCheck@xercesc_2_3@@AAEXXZ 12091e10 f   GeneralAttributeCheck.obj
 0001:000918d0       ?reinitGeneralAttCheck@GeneralAttributeCheck@xercesc_2_3@@SAXXZ 120928d0 f   GeneralAttributeCheck.obj
 0001:000919d0       ?checkAttributes@GeneralAttributeCheck@xercesc_2_3@@QAEXQBVDOMElement@2@GQAVTraverseSchema@2@_N@Z 120929d0 f   GeneralAttributeCheck.obj
 0001:00091eb0       ?validate@GeneralAttributeCheck@xercesc_2_3@@AAEXQBVDOMElement@2@QBG1FQAVTraverseSchema@2@@Z 12092eb0 f   GeneralAttributeCheck.obj
 0001:000923c0       ??0?$ValueHashTableOf@G@xercesc_2_3@@QAE@IQAVMemoryManager@1@@Z 120933c0 f i GeneralAttributeCheck.obj
 0001:000924b0       ??0NamespaceScope@xercesc_2_3@@QAE@QAVMemoryManager@1@@Z 120934b0 f   NamespaceScope.obj
 0001:00092550       ??1NamespaceScope@xercesc_2_3@@QAE@XZ 12093550 f   NamespaceScope.obj
 0001:000925e0       ?increaseDepth@NamespaceScope@xercesc_2_3@@QAEIXZ 120935e0 f   NamespaceScope.obj
 0001:000926e0       ?decreaseDepth@NamespaceScope@xercesc_2_3@@QAEIXZ 120936e0 f   NamespaceScope.obj
 0001:00092720       ?addPrefix@NamespaceScope@xercesc_2_3@@QAEXQBGI@Z 12093720 f   NamespaceScope.obj
 0001:00092820       ?getNamespaceForPrefix@NamespaceScope@xercesc_2_3@@QBEIQBGH@Z 12093820 f   NamespaceScope.obj
 0001:00092890       ?reset@NamespaceScope@xercesc_2_3@@QAEXI@Z 12093890 f   NamespaceScope.obj
 0001:000928b0       ?expandMap@NamespaceScope@xercesc_2_3@@AAEXQAUStackElem@12@@Z 120938b0 f   NamespaceScope.obj
 0001:00092950       ?expandStack@NamespaceScope@xercesc_2_3@@AAEXXZ 12093950 f   NamespaceScope.obj
 0001:000929f0       ?getFullName@SchemaAttDef@xercesc_2_3@@UBEPBGXZ 120939f0 f   SchemaAttDef.obj
 0001:00092a00       ??0SchemaAttDef@xercesc_2_3@@QAE@QAVMemoryManager@1@@Z 12093a00 f   SchemaAttDef.obj
 0001:00092a50       ??_ESchemaAttDef@xercesc_2_3@@UAEPAXI@Z 12093a50 f i SchemaAttDef.obj
 0001:00092ab0       ??0SchemaAttDef@xercesc_2_3@@QAE@QBG0HW4AttTypes@XMLAttDef@1@W4DefAttTypes@31@QAVMemoryManager@1@@Z 12093ab0 f   SchemaAttDef.obj
 0001:00092b70       ??0SchemaAttDef@xercesc_2_3@@QAE@QBG0H0W4AttTypes@XMLAttDef@1@W4DefAttTypes@31@0QAVMemoryManager@1@@Z 12093b70 f   SchemaAttDef.obj
 0001:00092c30       ??0SchemaAttDef@xercesc_2_3@@QAE@PBV01@@Z 12093c30 f   SchemaAttDef.obj
 0001:00092d80       ??1SchemaAttDef@xercesc_2_3@@UAE@XZ 12093d80 f   SchemaAttDef.obj
 0001:00092e00       ?setAttName@SchemaAttDef@xercesc_2_3@@QAEXQBG0H@Z 12093e00 f   SchemaAttDef.obj
 0001:00092e20       ??0SchemaAttDefList@xercesc_2_3@@QAE@QAV?$RefHash2KeysTableOf@VSchemaAttDef@xercesc_2_3@@@1@@Z 12093e20 f   SchemaAttDefList.obj
 0001:00092f20       ??1SchemaAttDefList@xercesc_2_3@@UAE@XZ 12093f20 f   SchemaAttDefList.obj
 0001:00092f70       ?hasMoreElements@SchemaAttDefList@xercesc_2_3@@UBE_NXZ 12093f70 f   SchemaAttDefList.obj
 0001:00092f70       ?hasMoreElements@DTDAttDefList@xercesc_2_3@@UBE_NXZ 12093f70 f   SchemaAttDefList.obj
 0001:00092f80       ?isEmpty@SchemaAttDefList@xercesc_2_3@@UBE_NXZ 12093f80 f   SchemaAttDefList.obj
 0001:00092f80       ?isEmpty@DTDAttDefList@xercesc_2_3@@UBE_NXZ 12093f80 f   SchemaAttDefList.obj
 0001:00092fb0       ?findAttDef@SchemaAttDefList@xercesc_2_3@@UAEPAVXMLAttDef@2@KQBG@Z 12093fb0 f   SchemaAttDefList.obj
 0001:000930b0       ?findAttDef@SchemaAttDefList@xercesc_2_3@@UBEPBVXMLAttDef@2@KQBG@Z 120940b0 f   SchemaAttDefList.obj
 0001:000931b0       ?findAttDef@SchemaAttDefList@xercesc_2_3@@UAEPAVXMLAttDef@2@QBG0@Z 120941b0 f   SchemaAttDefList.obj
 0001:000931e0       ?findAttDef@SchemaAttDefList@xercesc_2_3@@UBEPBVXMLAttDef@2@QBG0@Z 120941e0 f   SchemaAttDefList.obj
 0001:00093210       ?nextElement@SchemaAttDefList@xercesc_2_3@@UAEAAVXMLAttDef@2@XZ 12094210 f   SchemaAttDefList.obj
 0001:00093210       ?nextElement@DTDAttDefList@xercesc_2_3@@UAEAAVXMLAttDef@2@XZ 12094210 f   SchemaAttDefList.obj
 0001:00093220       ??0SchemaElementDecl@xercesc_2_3@@QAE@QAVMemoryManager@1@@Z 12094220 f   SchemaElementDecl.obj
 0001:00093280       ??_ESchemaElementDecl@xercesc_2_3@@UAEPAXI@Z 12094280 f i SchemaElementDecl.obj
 0001:000932e0       ??0SchemaElementDecl@xercesc_2_3@@QAE@QBG0HW4ModelTypes@01@HQAVMemoryManager@1@@Z 120942e0 f   SchemaElementDecl.obj
 0001:00093390       ??0SchemaElementDecl@xercesc_2_3@@QAE@QBVQName@1@W4ModelTypes@01@HQAVMemoryManager@1@@Z 12094390 f   SchemaElementDecl.obj
 0001:00093430       ??1SchemaElementDecl@xercesc_2_3@@UAE@XZ 12094430 f   SchemaElementDecl.obj
 0001:00093520       ?findAttr@SchemaElementDecl@xercesc_2_3@@UBEPAVXMLAttDef@2@QBGI00W4LookupOpts@XMLElementDecl@2@AA_N@Z 12094520 f   SchemaElementDecl.obj
 0001:000937c0       ?getAttDefList@SchemaElementDecl@xercesc_2_3@@UBEAAVXMLAttDefList@2@XZ 120947c0 f   SchemaElementDecl.obj
 0001:00093810       ?getCharDataOpts@SchemaElementDecl@xercesc_2_3@@UBE?AW4CharDataOpts@XMLElementDecl@2@XZ 12094810 f   SchemaElementDecl.obj
 0001:00093840       ?hasAttDefs@SchemaElementDecl@xercesc_2_3@@UBE_NXZ 12094840 f   SchemaElementDecl.obj
 0001:000938b0       ?resetDefs@SchemaElementDecl@xercesc_2_3@@UAE_NXZ 120948b0 f   SchemaElementDecl.obj
 0001:00093930       ?getFormattedContentModel@SchemaElementDecl@xercesc_2_3@@UBEPBGXZ 12094930 f   SchemaElementDecl.obj
 0001:00093950       ?getAttDef@SchemaElementDecl@xercesc_2_3@@QBEPBVSchemaAttDef@2@QBGH@Z 12094950 f   SchemaElementDecl.obj
 0001:00093950       ?getAttDef@SchemaElementDecl@xercesc_2_3@@QAEPAVSchemaAttDef@2@QBGH@Z 12094950 f   SchemaElementDecl.obj
 0001:00093aa0       ??_FXercesGroupInfo@xercesc_2_3@@QAEXXZ 12094aa0 f i SchemaGrammar.obj
 0001:00093ab0       ?elementCount@XercesGroupInfo@xercesc_2_3@@QBEIXZ 12094ab0 f i SchemaGrammar.obj
 0001:00093ac0       ?elementAt@XercesGroupInfo@xercesc_2_3@@QAEPAVSchemaElementDecl@2@I@Z 12094ac0 f i SchemaGrammar.obj
 0001:00093ac0       ?elementAt@XercesGroupInfo@xercesc_2_3@@QBEPBVSchemaElementDecl@2@I@Z 12094ac0 f i SchemaGrammar.obj
 0001:00093b10       ?setBlockDefault@SchemaInfo@xercesc_2_3@@QAEXH@Z 12094b10 f i SchemaGrammar.obj
 0001:00093b10       ?setIDRefList@GeneralAttributeCheck@xercesc_2_3@@QAEXQAV?$RefHashTableOf@VXMLRefInfo@xercesc_2_3@@@2@@Z 12094b10 f i SchemaGrammar.obj
 0001:00093b10       ?setScope@XercesGroupInfo@xercesc_2_3@@QAEXH@Z 12094b10 f i SchemaGrammar.obj
 0001:00093b10       ?setMatcherStack@FieldActivator@xercesc_2_3@@QAEXQAVXPathMatcherStack@2@@Z 12094b10 f i SchemaGrammar.obj
 0001:00093b10       ?setType@XMLAttr@xercesc_2_3@@QAEXW4AttTypes@XMLAttDef@2@@Z 12094b10 f i SchemaGrammar.obj
 0001:00093b10       ?setLineNumber@DOMLocatorImpl@xercesc_2_3@@UAEXJ@Z 12094b10 f i SchemaGrammar.obj
 0001:00093b10       ?setEntityExpansionLimit@SecurityManager@xercesc_2_3@@UAEXI@Z 12094b10 f i SchemaGrammar.obj
 0001:00093b10       ?setId@XMLEntityDecl@xercesc_2_3@@QAEXI@Z 12094b10 f i SchemaGrammar.obj
 0001:00093b10       ?setDefaultType@XMLAttDef@xercesc_2_3@@QAEXW4DefAttTypes@12@@Z 12094b10 f i SchemaGrammar.obj
 0001:00093b20       ?setMessage@DOMErrorImpl@xercesc_2_3@@UAEXQBG@Z 12094b20 f i SchemaGrammar.obj
 0001:00093b20       ?setColumnNumber@DOMLocatorImpl@xercesc_2_3@@UAEXJ@Z 12094b20 f i SchemaGrammar.obj
 0001:00093b20       ?setDerivedBy@ComplexTypeInfo@xercesc_2_3@@QAEXH@Z 12094b20 f i SchemaGrammar.obj
 0001:00093b20       ?setNextOp@Op@xercesc_2_3@@QAEXQBV12@@Z 12094b20 f i SchemaGrammar.obj
 0001:00093b20       ?setErrorReporter@XSDErrorReporter@xercesc_2_3@@QAEXQAVXMLErrorReporter@2@@Z 12094b20 f i SchemaGrammar.obj
 0001:00093b20       ?setErrorReporter@XMLValidator@xercesc_2_3@@QAEXQAVXMLErrorReporter@2@@Z 12094b20 f i SchemaGrammar.obj
 0001:00093b20       ?setType@XMLAttDef@xercesc_2_3@@QAEXW4AttTypes@12@@Z 12094b20 f i SchemaGrammar.obj
 0001:00093b20       ?setFinalDefault@SchemaInfo@xercesc_2_3@@QAEXH@Z 12094b20 f i SchemaGrammar.obj
 0001:00093b20       ?setDocTypeHandler@DTDScanner@xercesc_2_3@@QAEXQAVDocTypeHandler@2@@Z 12094b20 f i SchemaGrammar.obj
 0001:00093b20       ?setMin@ClosureToken@xercesc_2_3@@UAEXH@Z 12094b20 f i SchemaGrammar.obj
 0001:00093b20       ?setContentSpec@XercesGroupInfo@xercesc_2_3@@QAEXQAVContentSpecNode@2@@Z 12094b20 f i SchemaGrammar.obj
 0001:00093b30       ?addElement@XercesGroupInfo@xercesc_2_3@@QAEXQAVSchemaElementDecl@2@@Z 12094b30 f i SchemaGrammar.obj
 0001:00093bd0       ?setFinalSet@ComplexTypeInfo@xercesc_2_3@@QAEXH@Z 12094bd0 f i SchemaGrammar.obj
 0001:00093bd0       ?setErrorNode@DOMLocatorImpl@xercesc_2_3@@UAEXQAVDOMNode@2@@Z 12094bd0 f i SchemaGrammar.obj
 0001:00093bd0       ?setId@XMLElementDecl@xercesc_2_3@@QAEXI@Z 12094bd0 f i SchemaGrammar.obj
 0001:00093bd0       ?setScopeCount@SchemaInfo@xercesc_2_3@@QAEXH@Z 12094bd0 f i SchemaGrammar.obj
 0001:00093bd0       ?setType@DOMErrorImpl@xercesc_2_3@@UAEXPBG@Z 12094bd0 f i SchemaGrammar.obj
 0001:00093bd0       ?setScanner@ValueStoreCache@xercesc_2_3@@QAEXQAVXMLScanner@2@@Z 12094bd0 f i SchemaGrammar.obj
 0001:00093bd0       ?setBaseGroup@XercesGroupInfo@xercesc_2_3@@QAEXQAV12@@Z 12094bd0 f i SchemaGrammar.obj
 0001:00093be0       ??_FXercesAttGroupInfo@xercesc_2_3@@QAEXXZ 12094be0 f i SchemaGrammar.obj
 0001:00093bf0       ?getInUse@XMLBuffer@xercesc_2_3@@QBE_NXZ 12094bf0 f i SchemaGrammar.obj
 0001:00093bf0       ?containsTypeWithId@XercesAttGroupInfo@xercesc_2_3@@QBE_NXZ 12094bf0 f i SchemaGrammar.obj
 0001:00093bf0       ?getCheckElementConsistency@XercesGroupInfo@xercesc_2_3@@QBE_NXZ 12094bf0 f i SchemaGrammar.obj
 0001:00093bf0       ?getDeclared@XMLRefInfo@xercesc_2_3@@QBE_NXZ 12094bf0 f i SchemaGrammar.obj
 0001:00093bf0       ?getAnonymous@ComplexTypeInfo@xercesc_2_3@@QBE_NXZ 12094bf0 f i SchemaGrammar.obj
 0001:00093bf0       ?getMayMatch@IC_Field@xercesc_2_3@@QBE_NXZ 12094bf0 f i SchemaGrammar.obj
 0001:00093bf0       ?getSpecified@XMLAttr@xercesc_2_3@@QBE_NXZ 12094bf0 f i SchemaGrammar.obj
 0001:00093c00       ?attributeCount@XercesAttGroupInfo@xercesc_2_3@@QBEIXZ 12094c00 f i SchemaGrammar.obj
 0001:00093c10       ?anyAttributeCount@XercesAttGroupInfo@xercesc_2_3@@QBEIXZ 12094c10 f i SchemaGrammar.obj
 0001:00093c20       ?attributeAt@XercesAttGroupInfo@xercesc_2_3@@QBEPBVSchemaAttDef@2@I@Z 12094c20 f i SchemaGrammar.obj
 0001:00093c20       ?attributeAt@XercesAttGroupInfo@xercesc_2_3@@QAEPAVSchemaAttDef@2@I@Z 12094c20 f i SchemaGrammar.obj
 0001:00093c70       ?setMayMatch@IC_Field@xercesc_2_3@@QAEX_N@Z 12094c70 f i SchemaGrammar.obj
 0001:00093c70       ?setSpecified@XMLAttr@xercesc_2_3@@QAEX_N@Z 12094c70 f i SchemaGrammar.obj
 0001:00093c70       ?setInUse@XMLBuffer@xercesc_2_3@@QAEX_N@Z 12094c70 f i SchemaGrammar.obj
 0001:00093c70       ?setCheckElementConsistency@XercesGroupInfo@xercesc_2_3@@QAEX_N@Z 12094c70 f i SchemaGrammar.obj
 0001:00093c70       ?setTypeWithId@XercesAttGroupInfo@xercesc_2_3@@QAEX_N@Z 12094c70 f i SchemaGrammar.obj
 0001:00093c70       ?setDeclared@XMLRefInfo@xercesc_2_3@@QAEX_N@Z 12094c70 f i SchemaGrammar.obj
 0001:00093c80       ?addAttDef@XercesAttGroupInfo@xercesc_2_3@@QAEXQAVSchemaAttDef@2@_N@Z 12094c80 f i SchemaGrammar.obj
 0001:00093e60       ?addAnyAttDef@XercesAttGroupInfo@xercesc_2_3@@QAEXQAVSchemaAttDef@2@_N@Z 12094e60 f i SchemaGrammar.obj
 0001:00094040       ?setCompleteWildCard@XercesAttGroupInfo@xercesc_2_3@@QAEXQAVSchemaAttDef@2@@Z 12095040 f i SchemaGrammar.obj
 0001:00094070       ??0SchemaGrammar@xercesc_2_3@@QAE@QAVMemoryManager@1@@Z 12095070 f   SchemaGrammar.obj
 0001:000943d0       ??_ESchemaGrammar@xercesc_2_3@@UAEPAXI@Z 120953d0 f i SchemaGrammar.obj
 0001:00094430       ??1SchemaGrammar@xercesc_2_3@@UAE@XZ 12095430 f   SchemaGrammar.obj
 0001:00094490       ?findOrAddElemDecl@SchemaGrammar@xercesc_2_3@@UAEPAVXMLElementDecl@2@IQBG00IAA_N@Z 12095490 f   SchemaGrammar.obj
 0001:000946b0       ?putElemDecl@SchemaGrammar@xercesc_2_3@@UAEPAVXMLElementDecl@2@IQBG00I_N@Z 120956b0 f   SchemaGrammar.obj
 0001:00094960       ?reset@SchemaGrammar@xercesc_2_3@@UAEXXZ 12095960 f   SchemaGrammar.obj
 0001:00094af0       ?cleanUp@SchemaGrammar@xercesc_2_3@@AAEXXZ 12095af0 f   SchemaGrammar.obj
 0001:00094c90       ??1?$RefHash3KeysIdPool@VSchemaElementDecl@xercesc_2_3@@@xercesc_2_3@@QAE@XZ 12095c90 f i SchemaGrammar.obj
 0001:00094d10       ?removeAll@?$RefHash3KeysIdPool@VSchemaElementDecl@xercesc_2_3@@@xercesc_2_3@@QAEXXZ 12095d10 f i SchemaGrammar.obj
 0001:00094d80       ??0?$RefHashTableOf@VXMLRefInfo@xercesc_2_3@@@xercesc_2_3@@QAE@IQAVMemoryManager@1@@Z 12095d80 f i SchemaGrammar.obj
 0001:00094e70       ??1?$RefHashTableOf@VXMLRefInfo@xercesc_2_3@@@xercesc_2_3@@QAE@XZ 12095e70 f i SchemaGrammar.obj
 0001:00094f00       ??1?$RefHashTableOf@VXercesGroupInfo@xercesc_2_3@@@xercesc_2_3@@QAE@XZ 12095f00 f i SchemaGrammar.obj
 0001:00094f90       ??1?$RefHashTableOf@VXercesAttGroupInfo@xercesc_2_3@@@xercesc_2_3@@QAE@XZ 12095f90 f i SchemaGrammar.obj
 0001:00095020       ??_G?$RefVectorOf@VSchemaAttDef@xercesc_2_3@@@xercesc_2_3@@UAEPAXI@Z 12096020 f i SchemaGrammar.obj
 0001:00095020       ??_E?$RefVectorOf@VSchemaAttDef@xercesc_2_3@@@xercesc_2_3@@UAEPAXI@Z 12096020 f i SchemaGrammar.obj
 0001:00095040       ??1?$RefVectorOf@VSchemaAttDef@xercesc_2_3@@@xercesc_2_3@@UAE@XZ 12096040 f i SchemaGrammar.obj
 0001:000950c0       ??1?$BaseRefVectorOf@VSchemaAttDef@xercesc_2_3@@@xercesc_2_3@@UAE@XZ 120960c0 f i SchemaGrammar.obj
 0001:000950d0       ?findBucketElem@?$RefHash3KeysIdPool@VSchemaElementDecl@xercesc_2_3@@@xercesc_2_3@@AAEPAU?$RefHash3KeysTableBucketElem@VSchemaElementDecl@xercesc_2_3@@@2@QBXHHAAI@Z 120960d0 f i SchemaGrammar.obj
 0001:00095170       ?initialize@?$RefHash3KeysIdPool@VSchemaElementDecl@xercesc_2_3@@@xercesc_2_3@@AAEXI@Z 12096170 f i SchemaGrammar.obj
 0001:000951e0       ?removeAll@?$RefHashTableOf@VComplexTypeInfo@xercesc_2_3@@@xercesc_2_3@@QAEXXZ 120961e0 f i SchemaGrammar.obj
 0001:00095260       ?removeAll@?$RefHash2KeysTableOf@V?$ValueVectorOf@PAVSchemaElementDecl@xercesc_2_3@@@xercesc_2_3@@@xercesc_2_3@@QAEXXZ 12096260 f i SchemaGrammar.obj
 0001:000952e0       ??0XUtil@xercesc_2_3@@IAE@XZ 120962e0 f i SchemaInfo.obj
 0001:000952e0       ??0XMemory@xercesc_2_3@@IAE@XZ 120962e0 f i SchemaInfo.obj
 0001:000952f0       ??0SchemaInfo@xercesc_2_3@@QAE@GHHHHIQAGQBGQBVDOMElement@1@QAVMemoryManager@1@@Z 120962f0 f   SchemaInfo.obj
 0001:00095400       ??1SchemaInfo@xercesc_2_3@@QAE@XZ 12096400 f   SchemaInfo.obj
 0001:00095500       ?getTopLevelComponent@SchemaInfo@xercesc_2_3@@QAEPAVDOMElement@2@GQBG0PAPAV12@@Z 12096500 f   SchemaInfo.obj
 0001:000955b0       ?getTopLevelComponent@SchemaInfo@xercesc_2_3@@QAEPAVDOMElement@2@GQBG0@Z 120965b0 f   SchemaInfo.obj
 0001:00095a50       ?updateImportingInfo@SchemaInfo@xercesc_2_3@@QAEXQAV12@@Z 12096a50 f   SchemaInfo.obj
 0001:00095bb0       ?addElement@?$BaseRefVectorOf@G@xercesc_2_3@@QAEXQAG@Z 12096bb0 f i SchemaInfo.obj
 0001:00095bb0       ?addElement@?$BaseRefVectorOf@VSchemaInfo@xercesc_2_3@@@xercesc_2_3@@QAEXQAVSchemaInfo@2@@Z 12096bb0 f i SchemaInfo.obj
 0001:00095bb0       ?addElement@?$BaseRefVectorOf@VIdentityConstraint@xercesc_2_3@@@xercesc_2_3@@QAEXQAVIdentityConstraint@2@@Z 12096bb0 f i SchemaInfo.obj
 0001:00095bb0       ?addElement@?$BaseRefVectorOf@VSchemaElementDecl@xercesc_2_3@@@xercesc_2_3@@QAEXQAVSchemaElementDecl@2@@Z 12096bb0 f i SchemaInfo.obj
 0001:00095bb0       ?addElement@?$BaseRefVectorOf@VSchemaAttDef@xercesc_2_3@@@xercesc_2_3@@QAEXQAVSchemaAttDef@2@@Z 12096bb0 f i SchemaInfo.obj
 0001:00095c30       ??0SchemaValidator@xercesc_2_3@@QAE@QAVXMLErrorReporter@1@QAVMemoryManager@1@@Z 12096c30 f   SchemaValidator.obj
 0001:00095d40       ??_ESchemaValidator@xercesc_2_3@@UAEPAXI@Z 12096d40 f i SchemaValidator.obj
 0001:00095da0       ??1SchemaValidator@xercesc_2_3@@UAE@XZ 12096da0 f   SchemaValidator.obj
 0001:00095e30       ?checkContent@SchemaValidator@xercesc_2_3@@UAEHQAVXMLElementDecl@2@QAPAVQName@2@I@Z 12096e30 f   SchemaValidator.obj
 0001:00096660       ?faultInAttr@SchemaValidator@xercesc_2_3@@UBEXAAVXMLAttr@2@ABVXMLAttDef@2@@Z 12097660 f   SchemaValidator.obj
 0001:000966a0       ?reset@SchemaValidator@xercesc_2_3@@UAEXXZ 120976a0 f   SchemaValidator.obj
 0001:000966e0       ?isDocumentFragmentImpl@DocumentFragmentImpl@xercesc_2_3@@UAE_NXZ 120976e0 f   SchemaValidator.obj
 0001:000966e0       ?isDocumentTypeImpl@DocumentTypeImpl@xercesc_2_3@@UAE_NXZ 120976e0 f   SchemaValidator.obj
 0001:000966e0       ?isElementImpl@ElementImpl@xercesc_2_3@@UAE_NXZ 120976e0 f   SchemaValidator.obj
 0001:000966e0       ?supportsSrcOfs@Win32TransService@xercesc_2_3@@UBE_NXZ 120976e0 f   SchemaValidator.obj
 0001:000966e0       ?isAttrImpl@AttrImpl@xercesc_2_3@@UAE_NXZ 120976e0 f   SchemaValidator.obj
 0001:000966e0       ?isTextImpl@TextImpl@xercesc_2_3@@UAE_NXZ 120976e0 f   SchemaValidator.obj
 0001:000966e0       ?requiresNamespaces@SchemaValidator@xercesc_2_3@@UBE_NXZ 120976e0 f   SchemaValidator.obj
 0001:000966e0       ?isEntityReference@EntityReferenceImpl@xercesc_2_3@@UAE_NXZ 120976e0 f   SchemaValidator.obj
 0001:000966e0       ?isDocumentImpl@DocumentImpl@xercesc_2_3@@UAE_NXZ 120976e0 f   SchemaValidator.obj
 0001:000966e0       ?isCDATASectionImpl@CDATASectionImpl@xercesc_2_3@@UAE_NXZ 120976e0 f   SchemaValidator.obj
 0001:000966f0       ?validateAttrValue@SchemaValidator@xercesc_2_3@@UAEXPBVXMLAttDef@2@QBG_NPBVXMLElementDecl@2@@Z 120976f0 f   SchemaValidator.obj
 0001:00096b70       ?validateElement@SchemaValidator@xercesc_2_3@@UAEXPBVXMLElementDecl@2@@Z 12097b70 f   SchemaValidator.obj
 0001:000971b0       ?preContentValidation@SchemaValidator@xercesc_2_3@@UAEX_N0@Z 120981b0 f   SchemaValidator.obj
 0001:00097840       ?normalizeWhiteSpace@SchemaValidator@xercesc_2_3@@QAEXPAVDatatypeValidator@2@QBGAAVXMLBuffer@2@@Z 12098840 f   SchemaValidator.obj
 0001:000979f0       ?checkRefElementConsistency@SchemaValidator@xercesc_2_3@@AAEXQAVSchemaGrammar@2@QBVComplexTypeInfo@2@QBVXercesGroupInfo@2@@Z 120989f0 f   SchemaValidator.obj
 0001:00097c50       ?checkParticleDerivation@SchemaValidator@xercesc_2_3@@AAEXQAVSchemaGrammar@2@QBVComplexTypeInfo@2@@Z 12098c50 f   SchemaValidator.obj
 0001:00097cf0       ?checkParticleDerivationOk@SchemaValidator@xercesc_2_3@@AAEXQAVSchemaGrammar@2@QAVContentSpecNode@2@H1HQBVComplexTypeInfo@2@_N@Z 12098cf0 f   SchemaValidator.obj
 0001:00098560       ?checkForPointlessOccurrences@SchemaValidator@xercesc_2_3@@AAEPAVContentSpecNode@2@QAV32@W4NodeTypes@32@QAV?$ValueVectorOf@PAVContentSpecNode@xercesc_2_3@@@2@@Z 12099560 f   SchemaValidator.obj
 0001:000985e0       ?gatherChildren@SchemaValidator@xercesc_2_3@@AAEXW4NodeTypes@ContentSpecNode@2@QAV42@QAV?$ValueVectorOf@PAVContentSpecNode@xercesc_2_3@@@2@@Z 120995e0 f   SchemaValidator.obj
 0001:000987d0       ?checkNSCompat@SchemaValidator@xercesc_2_3@@AAEXQBVContentSpecNode@2@0_N@Z 120997d0 f   SchemaValidator.obj
 0001:000988a0       ?wildcardEltAllowsNamespace@SchemaValidator@xercesc_2_3@@AAE_NQBVContentSpecNode@2@I@Z 120998a0 f   SchemaValidator.obj
 0001:000988f0       ?checkNameAndTypeOK@SchemaValidator@xercesc_2_3@@AAEXQAVSchemaGrammar@2@QBVContentSpecNode@2@H1HQBVComplexTypeInfo@2@@Z 120998f0 f   SchemaValidator.obj
 0001:00098bc0       ?findElement@SchemaValidator@xercesc_2_3@@AAEPAVSchemaElementDecl@2@HIQBGQAVSchemaGrammar@2@QBVComplexTypeInfo@2@@Z 12099bc0 f   SchemaValidator.obj
 0001:00098c20       ?checkICRestriction@SchemaValidator@xercesc_2_3@@AAEXQBVSchemaElementDecl@2@0QBG1@Z 12099c20 f   SchemaValidator.obj
 0001:00098d80       ?checkTypesOK@SchemaValidator@xercesc_2_3@@AAEXQBVSchemaElementDecl@2@0QBG@Z 12099d80 f   SchemaValidator.obj
 0001:00098ef0       ?checkRecurseAsIfGroup@SchemaValidator@xercesc_2_3@@AAEXQAVSchemaGrammar@2@QAVContentSpecNode@2@HQBV42@HQAV?$ValueVectorOf@PAVContentSpecNode@xercesc_2_3@@@2@QBVComplexTypeInfo@2@@Z 12099ef0 f   SchemaValidator.obj
 0001:000990e0       ?checkRecurse@SchemaValidator@xercesc_2_3@@AAEXQAVSchemaGrammar@2@QBVContentSpecNode@2@HQAV?$ValueVectorOf@PAVContentSpecNode@xercesc_2_3@@@2@1H2QBVComplexTypeInfo@2@_N@Z 1209a0e0 f   SchemaValidator.obj
 0001:000993b0       ?checkNSSubset@SchemaValidator@xercesc_2_3@@AAEXQBVContentSpecNode@2@0@Z 1209a3b0 f   SchemaValidator.obj
 0001:00099440       ?isWildCardEltSubset@SchemaValidator@xercesc_2_3@@AAE_NQBVContentSpecNode@2@0@Z 1209a440 f   SchemaValidator.obj
 0001:000994b0       ?checkNSRecurseCheckCardinality@SchemaValidator@xercesc_2_3@@AAEXQAVSchemaGrammar@2@QBVContentSpecNode@2@QAV?$ValueVectorOf@PAVContentSpecNode@xercesc_2_3@@@2@HQAV42@_N@Z 1209a4b0 f   SchemaValidator.obj
 0001:00099580       ?checkRecurseUnordered@SchemaValidator@xercesc_2_3@@AAEXQAVSchemaGrammar@2@QBVContentSpecNode@2@QAV?$ValueVectorOf@PAVContentSpecNode@xercesc_2_3@@@2@HQAV42@2HQBVComplexTypeInfo@2@@Z 1209a580 f   SchemaValidator.obj
 0001:000998a0       ?checkMapAndSum@SchemaValidator@xercesc_2_3@@AAEXQAVSchemaGrammar@2@QBVContentSpecNode@2@QAV?$ValueVectorOf@PAVContentSpecNode@xercesc_2_3@@@2@HQAV42@2HQBVComplexTypeInfo@2@@Z 1209a8a0 f   SchemaValidator.obj
 0001:00099ac0       ??1?$XMLEnumerator@VComplexTypeInfo@xercesc_2_3@@@xercesc_2_3@@UAE@XZ 1209aac0 f i SchemaValidator.obj
 0001:00099ad0       ??1?$XMLEnumerator@VXercesGroupInfo@xercesc_2_3@@@xercesc_2_3@@UAE@XZ 1209aad0 f i SchemaValidator.obj
 0001:00099ae0       ??_G?$XMLEnumerator@VComplexTypeInfo@xercesc_2_3@@@xercesc_2_3@@UAEPAXI@Z 1209aae0 f i SchemaValidator.obj
 0001:00099ae0       ??_E?$XMLEnumerator@VComplexTypeInfo@xercesc_2_3@@@xercesc_2_3@@UAEPAXI@Z 1209aae0 f i SchemaValidator.obj
 0001:00099b00       ??_E?$XMLEnumerator@VXercesGroupInfo@xercesc_2_3@@@xercesc_2_3@@UAEPAXI@Z 1209ab00 f i SchemaValidator.obj
 0001:00099b00       ??_G?$XMLEnumerator@VXercesGroupInfo@xercesc_2_3@@@xercesc_2_3@@UAEPAXI@Z 1209ab00 f i SchemaValidator.obj
 0001:00099b20       ?elementAt@?$BaseRefVectorOf@VXercesStep@xercesc_2_3@@@xercesc_2_3@@QAEPAVXercesStep@2@I@Z 1209ab20 f i SchemaValidator.obj
 0001:00099b20       ?elementAt@?$BaseRefVectorOf@VSchemaInfo@xercesc_2_3@@@xercesc_2_3@@QAEPAVSchemaInfo@2@I@Z 1209ab20 f i SchemaValidator.obj
 0001:00099b20       ?elementAt@?$BaseRefVectorOf@VScope@InScopeNamespaces@DOMNormalizer@xercesc_2_3@@@xercesc_2_3@@QAEPAVScope@InScopeNamespaces@DOMNormalizer@2@I@Z 1209ab20 f i SchemaValidator.obj
 0001:00099b20       ?elementAt@?$BaseRefVectorOf@VSchemaElementDecl@xercesc_2_3@@@xercesc_2_3@@QAEPAVSchemaElementDecl@2@I@Z 1209ab20 f i SchemaValidator.obj
 0001:00099b20       ?elementAt@?$BaseRefVectorOf@VSchemaAttDef@xercesc_2_3@@@xercesc_2_3@@QAEPAVSchemaAttDef@2@I@Z 1209ab20 f i SchemaValidator.obj
 0001:00099b20       ?elementAt@?$BaseRefVectorOf@G@xercesc_2_3@@QAEPAGI@Z 1209ab20 f i SchemaValidator.obj
 0001:00099b60       ??1?$RefHashTableOfEnumerator@VComplexTypeInfo@xercesc_2_3@@@xercesc_2_3@@UAE@XZ 1209ab60 f i SchemaValidator.obj
 0001:00099c50       ??1?$RefHashTableOfEnumerator@VXercesGroupInfo@xercesc_2_3@@@xercesc_2_3@@UAE@XZ 1209ac50 f i SchemaValidator.obj
 0001:00099d40       ??_E?$RefHashTableOfEnumerator@VComplexTypeInfo@xercesc_2_3@@@xercesc_2_3@@UAEPAXI@Z 1209ad40 f i SchemaValidator.obj
 0001:00099d40       ??_G?$RefHashTableOfEnumerator@VComplexTypeInfo@xercesc_2_3@@@xercesc_2_3@@UAEPAXI@Z 1209ad40 f i SchemaValidator.obj
 0001:00099d60       ??_G?$RefHashTableOfEnumerator@VXercesGroupInfo@xercesc_2_3@@@xercesc_2_3@@UAEPAXI@Z 1209ad60 f i SchemaValidator.obj
 0001:00099d60       ??_E?$RefHashTableOfEnumerator@VXercesGroupInfo@xercesc_2_3@@@xercesc_2_3@@UAEPAXI@Z 1209ad60 f i SchemaValidator.obj
 0001:00099d80       ?removeAll@?$RefHashTableOf@VXercesGroupInfo@xercesc_2_3@@@xercesc_2_3@@QAEXXZ 1209ad80 f i SchemaValidator.obj
 0001:00099e00       ?isEquivalentTo@SubstitutionGroupComparator@xercesc_2_3@@QAE_NQAVQName@2@0@Z 1209ae00 f   SubstitutionGroupComparator.obj
 0001:0009a060       ?isAllowedByWildcard@SubstitutionGroupComparator@xercesc_2_3@@QAE_NQAVSchemaGrammar@2@QAVQName@2@I_N@Z 1209b060 f   SubstitutionGroupComparator.obj
 0001:0009a1c0       ??_ODOMElementNSImpl@xercesc_2_3@@QAEXABV01@@Z 1209b1c0 f i TraverseSchema.obj
 0001:0009a1d0       ?getDocHandler@XMLScanner@xercesc_2_3@@QAEPAVXMLDocumentHandler@2@XZ 1209b1d0 f i TraverseSchema.obj
 0001:0009a1d0       ?getMaxInclusive@AbstractNumericFacetValidator@xercesc_2_3@@QBEQAVXMLNumber@2@XZ 1209b1d0 f i TraverseSchema.obj
 0001:0009a1d0       ?getErrorHandler@SAXParser@xercesc_2_3@@QAEPAVErrorHandler@2@XZ 1209b1d0 f i TraverseSchema.obj
 0001:0009a1d0       ?getMinLength@AbstractStringValidator@xercesc_2_3@@QBEIXZ 1209b1d0 f i TraverseSchema.obj
 0001:0009a1d0       ?getLineNo@XSDElementNSImpl@xercesc_2_3@@QBEJXZ 1209b1d0 f i TraverseSchema.obj
 0001:0009a1d0       ?getErrorHandler@SAXParser@xercesc_2_3@@QBEPBVErrorHandler@2@XZ 1209b1d0 f i TraverseSchema.obj
 0001:0009a1d0       ?getValidationAttempted@SchemaAttDef@xercesc_2_3@@QBE?AW4Validation@PSVIDefs@2@XZ 1209b1d0 f i TraverseSchema.obj
 0001:0009a1d0       ?getDocHandler@XMLScanner@xercesc_2_3@@QBEPBVXMLDocumentHandler@2@XZ 1209b1d0 f i TraverseSchema.obj
 0001:0009a1d0       ?getMemoryManager@TokenFactory@xercesc_2_3@@QBEPAVMemoryManager@2@XZ 1209b1d0 f i TraverseSchema.obj
 0001:0009a1e0       ?getMemberTypeValidator@UnionDatatypeValidator@xercesc_2_3@@QBEPBVDatatypeValidator@2@XZ 1209b1e0 f i TraverseSchema.obj
 0001:0009a1e0       ?getDocTypeHandler@XMLScanner@xercesc_2_3@@QBEPBVDocTypeHandler@2@XZ 1209b1e0 f i TraverseSchema.obj
 0001:0009a1e0       ?getColumnNo@XSDElementNSImpl@xercesc_2_3@@QBEJXZ 1209b1e0 f i TraverseSchema.obj
 0001:0009a1e0       ?getDocTypeHandler@XMLScanner@xercesc_2_3@@QAEPAVDocTypeHandler@2@XZ 1209b1e0 f i TraverseSchema.obj
 0001:0009a1e0       ?getMaxExclusive@AbstractNumericFacetValidator@xercesc_2_3@@QBEQAVXMLNumber@2@XZ 1209b1e0 f i TraverseSchema.obj
 0001:0009a1e0       ?getMemoryManager@AbstractDOMParser@xercesc_2_3@@IBEPAVMemoryManager@2@XZ 1209b1e0 f i TraverseSchema.obj
 0001:0009a1f0       ??1XSDElementNSImpl@xercesc_2_3@@UAE@XZ 1209b1f0 f i TraverseSchema.obj
 0001:0009a1f0       ??1DOMElementNSImpl@xercesc_2_3@@UAE@XZ 1209b1f0 f i TraverseSchema.obj
 0001:0009a200       ??_OXSDElementNSImpl@xercesc_2_3@@QAEXABV01@@Z 1209b200 f i TraverseSchema.obj
 0001:0009a210       ??0TraverseSchema@xercesc_2_3@@QAE@QAVDOMElement@1@QAVXMLStringPool@1@QAVSchemaGrammar@1@QAVGrammarResolver@1@QAVXMLScanner@1@QBGQAVXMLEntityHandler@1@QAVXMLErrorReporter@1@QAVMemoryManager@1@@Z 1209b210 f   TraverseSchema.obj
 0001:0009a3a0       ??1TraverseSchema@xercesc_2_3@@QAE@XZ 1209b3a0 f   TraverseSchema.obj
 0001:0009a410       ?doTraverseSchema@TraverseSchema@xercesc_2_3@@AAEXQBVDOMElement@2@@Z 1209b410 f   TraverseSchema.obj
 0001:0009a610       ?preprocessSchema@TraverseSchema@xercesc_2_3@@AAEXQAVDOMElement@2@QBG@Z 1209b610 f   TraverseSchema.obj
 0001:0009ad00       ?traverseSchemaHeader@TraverseSchema@xercesc_2_3@@AAEXQBVDOMElement@2@@Z 1209bd00 f   TraverseSchema.obj
 0001:0009aef0       ?traverseAnnotationDecl@TraverseSchema@xercesc_2_3@@AAEXQBVDOMElement@2@_N@Z 1209bef0 f   TraverseSchema.obj
 0001:0009b040       ?preprocessInclude@TraverseSchema@xercesc_2_3@@AAEXQBVDOMElement@2@@Z 1209c040 f   TraverseSchema.obj
 0001:0009b590       ?traverseInclude@TraverseSchema@xercesc_2_3@@AAEXQBVDOMElement@2@@Z 1209c590 f   TraverseSchema.obj
 0001:0009b630       ?preprocessImport@TraverseSchema@xercesc_2_3@@AAEXQBVDOMElement@2@@Z 1209c630 f   TraverseSchema.obj
 0001:0009bc10       ?traverseImport@TraverseSchema@xercesc_2_3@@AAEXQBVDOMElement@2@@Z 1209cc10 f   TraverseSchema.obj
 0001:0009bcc0       ?preprocessRedefine@TraverseSchema@xercesc_2_3@@AAEXQBVDOMElement@2@@Z 1209ccc0 f   TraverseSchema.obj
 0001:0009bf00       ?traverseRedefine@TraverseSchema@xercesc_2_3@@AAEXQBVDOMElement@2@@Z 1209cf00 f   TraverseSchema.obj
 0001:0009bfb0       ?traverseChoiceSequence@TraverseSchema@xercesc_2_3@@AAEPAVContentSpecNode@2@QBVDOMElement@2@H@Z 1209cfb0 f   TraverseSchema.obj
 0001:0009c460       ?traverseSimpleTypeDecl@TraverseSchema@xercesc_2_3@@AAEPAVDatatypeValidator@2@QBVDOMElement@2@_NH@Z 1209d460 f   TraverseSchema.obj
 0001:0009c9d0       ?traverseComplexTypeDecl@TraverseSchema@xercesc_2_3@@AAEHQBVDOMElement@2@_NQBG@Z 1209d9d0 f   TraverseSchema.obj
 0001:0009d240       ?traverseGroupDecl@TraverseSchema@xercesc_2_3@@AAEPAVXercesGroupInfo@2@QBVDOMElement@2@_N@Z 1209e240 f   TraverseSchema.obj
 0001:0009d9e0       ?traverseAttributeGroupDecl@TraverseSchema@xercesc_2_3@@AAEPAVXercesAttGroupInfo@2@QBVDOMElement@2@QAVComplexTypeInfo@2@_N@Z 1209e9e0 f   TraverseSchema.obj
 0001:0009e000       ?traverseAttributeGroupDeclNS@TraverseSchema@xercesc_2_3@@AAEPAVXercesAttGroupInfo@2@QBVDOMElement@2@QBG1@Z 1209f000 f i TraverseSchema.obj
 0001:0009e0f0       ?traverseAny@TraverseSchema@xercesc_2_3@@AAEPAVContentSpecNode@2@QBVDOMElement@2@@Z 1209f0f0 f   TraverseSchema.obj
 0001:0009e7e0       ??0ContentSpecNode@xercesc_2_3@@QAE@QAVQName@1@_NQAVMemoryManager@1@@Z 1209f7e0 f i TraverseSchema.obj
 0001:0009e880       ??0ContentSpecNode@xercesc_2_3@@QAE@W4NodeTypes@01@QAV01@1_N2QAVMemoryManager@1@@Z 1209f880 f i TraverseSchema.obj
 0001:0009e8c0       ?traverseAll@TraverseSchema@xercesc_2_3@@AAEPAVContentSpecNode@2@QBVDOMElement@2@@Z 1209f8c0 f   TraverseSchema.obj
 0001:0009eb40       ?traverseAttributeDecl@TraverseSchema@xercesc_2_3@@AAEXQBVDOMElement@2@QAVComplexTypeInfo@2@_N@Z 1209fb40 f   TraverseSchema.obj
 0001:0009fac0       ?traverseElementDecl@TraverseSchema@xercesc_2_3@@AAEPAVQName@2@QBVDOMElement@2@_N@Z 120a0ac0 f   TraverseSchema.obj
 0001:000a1600       ?traverseNotationDecl@TraverseSchema@xercesc_2_3@@AAEPBGQBVDOMElement@2@@Z 120a2600 f   TraverseSchema.obj
 0001:000a17b0       ?traverseNotationDecl@TraverseSchema@xercesc_2_3@@AAEPBGQBVDOMElement@2@QBG1@Z 120a27b0 f   TraverseSchema.obj
 0001:000a1a10       ?traverseByList@TraverseSchema@xercesc_2_3@@AAEPAVDatatypeValidator@2@QBVDOMElement@2@0QBG1H@Z 120a2a10 f   TraverseSchema.obj
 0001:000a1df0       ?traverseByRestriction@TraverseSchema@xercesc_2_3@@AAEPAVDatatypeValidator@2@QBVDOMElement@2@0QBG1H@Z 120a2df0 f   TraverseSchema.obj
 0001:000a2a50       ?traverseByUnion@TraverseSchema@xercesc_2_3@@AAEPAVDatatypeValidator@2@QBVDOMElement@2@0QBG1HH@Z 120a3a50 f   TraverseSchema.obj
 0001:000a2fa0       ?traverseSimpleContentDecl@TraverseSchema@xercesc_2_3@@AAEXQBG0QBVDOMElement@2@QAVComplexTypeInfo@2@@Z 120a3fa0 f   TraverseSchema.obj
 0001:000a4020       ?traverseComplexContentDecl@TraverseSchema@xercesc_2_3@@AAEXQBGQBVDOMElement@2@QAVComplexTypeInfo@2@_N@Z 120a5020 f   TraverseSchema.obj
 0001:000a4480       ?traverseAnyAttribute@TraverseSchema@xercesc_2_3@@AAEPAVSchemaAttDef@2@QBVDOMElement@2@@Z 120a5480 f   TraverseSchema.obj
 0001:000a4920       ?traverseKey@TraverseSchema@xercesc_2_3@@AAEXQBVDOMElement@2@QAVSchemaElementDecl@2@@Z 120a5920 f   TraverseSchema.obj
 0001:000a4c90       ?traverseUnique@TraverseSchema@xercesc_2_3@@AAEXQBVDOMElement@2@QAVSchemaElementDecl@2@@Z 120a5c90 f   TraverseSchema.obj
 0001:000a4fd0       ?traverseKeyRef@TraverseSchema@xercesc_2_3@@AAEXQBVDOMElement@2@QAVSchemaElementDecl@2@I@Z 120a5fd0 f   TraverseSchema.obj
 0001:000a53d0       ?traverseIdentityConstraint@TraverseSchema@xercesc_2_3@@AAE_NQAVIdentityConstraint@2@QBVDOMElement@2@@Z 120a63d0 f   TraverseSchema.obj
 0001:000a5bc0       ?retrieveNamespaceMapping@TraverseSchema@xercesc_2_3@@AAEXQBVDOMElement@2@@Z 120a6bc0 f   TraverseSchema.obj
 0001:000a5d70       ?processChildren@TraverseSchema@xercesc_2_3@@AAEXQBVDOMElement@2@@Z 120a6d70 f   TraverseSchema.obj
 0001:000a67a0       ?preprocessChildren@TraverseSchema@xercesc_2_3@@AAEXQBVDOMElement@2@@Z 120a77a0 f   TraverseSchema.obj
 0001:000a6950       ?checkContent@TraverseSchema@xercesc_2_3@@AAEPAVDOMElement@2@QBV32@QAV32@_N@Z 120a7950 f   TraverseSchema.obj
 0001:000a6b20       ?getDatatypeValidator@TraverseSchema@xercesc_2_3@@AAEPAVDatatypeValidator@2@QBG0@Z 120a7b20 f   TraverseSchema.obj
 0001:000a6d80       ?checkForSimpleTypeValidator@TraverseSchema@xercesc_2_3@@AAEPAVDatatypeValidator@2@QBVDOMElement@2@H@Z 120a7d80 f   TraverseSchema.obj
 0001:000a6e10       ?checkForComplexTypeInfo@TraverseSchema@xercesc_2_3@@AAEPAVComplexTypeInfo@2@QBVDOMElement@2@@Z 120a7e10 f   TraverseSchema.obj
 0001:000a6f20       ?findDTValidator@TraverseSchema@xercesc_2_3@@AAEPAVDatatypeValidator@2@QBVDOMElement@2@QBG1H@Z 120a7f20 f   TraverseSchema.obj
 0001:000a7150       ?resolvePrefixToURI@TraverseSchema@xercesc_2_3@@AAEPBGQBVDOMElement@2@QBG@Z 120a8150 f   TraverseSchema.obj
 0001:000a71d0       ?resolvePrefixToURI@TraverseSchema@xercesc_2_3@@AAEPBGQBVDOMElement@2@QBGI@Z 120a81d0 f   TraverseSchema.obj
 0001:000a7250       ?processElementDeclRef@TraverseSchema@xercesc_2_3@@AAEPAVQName@2@QBVDOMElement@2@QBG@Z 120a8250 f   TraverseSchema.obj
 0001:000a7630       ?parseBlockSet@TraverseSchema@xercesc_2_3@@AAEHQBVDOMElement@2@H_N@Z 120a8630 f   TraverseSchema.obj
 0001:000a7940       ?parseFinalSet@TraverseSchema@xercesc_2_3@@AAEHQBVDOMElement@2@H_N@Z 120a8940 f   TraverseSchema.obj
 0001:000a7c90       ?checkIdentityConstraintContent@TraverseSchema@xercesc_2_3@@AAEPBVDOMElement@2@QBV32@@Z 120a8c90 f   TraverseSchema.obj
 0001:000a7dc0       ?isIdentityConstraintName@TraverseSchema@xercesc_2_3@@AAE_NQBG@Z 120a8dc0 f   TraverseSchema.obj
 0001:000a7ee0       ?checkTypeFromAnotherSchema@TraverseSchema@xercesc_2_3@@AAEPBGQBVDOMElement@2@QBG@Z 120a8ee0 f   TraverseSchema.obj
 0001:000a8060       ?getElementTypeValidator@TraverseSchema@xercesc_2_3@@AAEPAVDatatypeValidator@2@QBVDOMElement@2@QBGAA_N1@Z 120a9060 f   TraverseSchema.obj
 0001:000a83f0       ?getAttrDatatypeValidatorNS@TraverseSchema@xercesc_2_3@@AAEPAVDatatypeValidator@2@QBVDOMElement@2@PBG1@Z 120a93f0 f   TraverseSchema.obj
 0001:000a85b0       ?getElementComplexTypeInfo@TraverseSchema@xercesc_2_3@@AAEPAVComplexTypeInfo@2@QBVDOMElement@2@QBGAA_N1@Z 120a95b0 f   TraverseSchema.obj
 0001:000a8950       ?getSubstituteGroupElemDecl@TraverseSchema@xercesc_2_3@@AAEPAVSchemaElementDecl@2@QBVDOMElement@2@QBGAA_N@Z 120a9950 f   TraverseSchema.obj
 0001:000a8e90       ?isSubstitutionGroupValid@TraverseSchema@xercesc_2_3@@AAE_NQBVDOMElement@2@QBVSchemaElementDecl@2@QBVComplexTypeInfo@2@QBVDatatypeValidator@2@QBG_N@Z 120a9e90 f   TraverseSchema.obj
 0001:000a9060       ?createSchemaElementDecl@TraverseSchema@xercesc_2_3@@AAEPAVSchemaElementDecl@2@QBVDOMElement@2@_NGAA_N1@Z 120aa060 f   TraverseSchema.obj
 0001:000a9330       ?processAttributeDeclRef@TraverseSchema@xercesc_2_3@@AAEXQBVDOMElement@2@QAVComplexTypeInfo@2@QBG222@Z 120aa330 f   TraverseSchema.obj
 0001:000a9d10       ?checkMinMax@TraverseSchema@xercesc_2_3@@AAEXQAVContentSpecNode@2@QBVDOMElement@2@H@Z 120aad10 f   TraverseSchema.obj
 0001:000aa0d0       ?processComplexContent@TraverseSchema@xercesc_2_3@@AAEXQBVDOMElement@2@QBG0QAVComplexTypeInfo@2@111_N3@Z 120ab0d0 f   TraverseSchema.obj
 0001:000aabc0       ?processBaseTypeInfo@TraverseSchema@xercesc_2_3@@AAEXQBVDOMElement@2@QBG11QAVComplexTypeInfo@2@@Z 120abbc0 f   TraverseSchema.obj
 0001:000ab200       ?getTypeInfoFromNS@TraverseSchema@xercesc_2_3@@AAEPAVComplexTypeInfo@2@QBVDOMElement@2@QBG1@Z 120ac200 f   TraverseSchema.obj
 0001:000ab340       ?processAttributes@TraverseSchema@xercesc_2_3@@AAEXQBVDOMElement@2@0QBG11QAVComplexTypeInfo@2@_N@Z 120ac340 f   TraverseSchema.obj
 0001:000abc20       ?defaultComplexTypeInfo@TraverseSchema@xercesc_2_3@@AAEXQAVComplexTypeInfo@2@@Z 120acc20 f   TraverseSchema.obj
 0001:000abc50       ?resolveSchemaLocation@TraverseSchema@xercesc_2_3@@AAEPAVInputSource@2@QBG@Z 120acc50 f   TraverseSchema.obj
 0001:000abeb0       ?restoreSchemaInfo@TraverseSchema@xercesc_2_3@@AAEXQAVSchemaInfo@2@W4ListType@32@H@Z 120aceb0 f   TraverseSchema.obj
 0001:000abf40       ?emptiableParticle@TraverseSchema@xercesc_2_3@@AAE_NQBVContentSpecNode@2@@Z 120acf40 f   TraverseSchema.obj
 0001:000abf60       ?checkFixedFacet@TraverseSchema@xercesc_2_3@@AAEXQBVDOMElement@2@QBGQBVDatatypeValidator@2@AAI@Z 120acf60 f   TraverseSchema.obj
 0001:000ac2a0       ?buildValidSubstitutionListB@TraverseSchema@xercesc_2_3@@AAEXQBVDOMElement@2@QAVSchemaElementDecl@2@1@Z 120ad2a0 f   TraverseSchema.obj
 0001:000ac580       ?buildValidSubstitutionListF@TraverseSchema@xercesc_2_3@@AAEXQBVDOMElement@2@QAVSchemaElementDecl@2@1@Z 120ad580 f   TraverseSchema.obj
 0001:000ac850       ?checkEnumerationRequiredNotation@TraverseSchema@xercesc_2_3@@AAEXQBVDOMElement@2@QBG1@Z 120ad850 f   TraverseSchema.obj
 0001:000ac970       ?processGroupRef@TraverseSchema@xercesc_2_3@@AAEPAVXercesGroupInfo@2@QBVDOMElement@2@QBG@Z 120ad970 f   TraverseSchema.obj
 0001:000acf60       ?processAttributeGroupRef@TraverseSchema@xercesc_2_3@@AAEPAVXercesAttGroupInfo@2@QBVDOMElement@2@QBGQAVComplexTypeInfo@2@@Z 120adf60 f   TraverseSchema.obj
 0001:000ad410       ?processElements@TraverseSchema@xercesc_2_3@@AAEXQBVDOMElement@2@QAVComplexTypeInfo@2@1@Z 120ae410 f   TraverseSchema.obj
 0001:000ad5f0       ?copyGroupElements@TraverseSchema@xercesc_2_3@@AAEXQBVDOMElement@2@QAVXercesGroupInfo@2@1QAVComplexTypeInfo@2@@Z 120ae5f0 f   TraverseSchema.obj
 0001:000ad830       ?copyAttGroupAttributes@TraverseSchema@xercesc_2_3@@AAEXQBVDOMElement@2@QAVXercesAttGroupInfo@2@1QAVComplexTypeInfo@2@@Z 120ae830 f   TraverseSchema.obj
 0001:000adbc0       ?attWildCardIntersection@TraverseSchema@xercesc_2_3@@AAEXQAVSchemaAttDef@2@QBV32@@Z 120aebc0 f   TraverseSchema.obj
 0001:000adfb0       ?attWildCardUnion@TraverseSchema@xercesc_2_3@@AAEXQAVSchemaAttDef@2@QBV32@@Z 120aefb0 f   TraverseSchema.obj
 0001:000ae3c0       ?checkAttDerivationOK@TraverseSchema@xercesc_2_3@@AAEXQBVDOMElement@2@QBVComplexTypeInfo@2@1@Z 120af3c0 f   TraverseSchema.obj
 0001:000ae750       ?checkAttDerivationOK@TraverseSchema@xercesc_2_3@@AAEXQBVDOMElement@2@QBVXercesAttGroupInfo@2@1@Z 120af750 f   TraverseSchema.obj
 0001:000aeb50       ?wildcardAllowsNamespace@TraverseSchema@xercesc_2_3@@AAE_NQBVSchemaAttDef@2@I@Z 120afb50 f   TraverseSchema.obj
 0001:000aebb0       ?isWildCardSubset@TraverseSchema@xercesc_2_3@@AAE_NQBVSchemaAttDef@2@0@Z 120afbb0 f   TraverseSchema.obj
 0001:000aecd0       ?openRedefinedSchema@TraverseSchema@xercesc_2_3@@AAE_NQBVDOMElement@2@@Z 120afcd0 f   TraverseSchema.obj
 0001:000af2e0       ?renameRedefinedComponents@TraverseSchema@xercesc_2_3@@AAEXQBVDOMElement@2@QAVSchemaInfo@2@1@Z 120b02e0 f   TraverseSchema.obj
 0001:000af4e0       ?validateRedefineNameChange@TraverseSchema@xercesc_2_3@@AAE_NQBVDOMElement@2@QBG1HQAVSchemaInfo@2@@Z 120b04e0 f   TraverseSchema.obj
 0001:000afea0       ?changeRedefineGroup@TraverseSchema@xercesc_2_3@@AAEHQBVDOMElement@2@QBG1H@Z 120b0ea0 f   TraverseSchema.obj
 0001:000b0280       ?fixRedefinedSchema@TraverseSchema@xercesc_2_3@@AAEXQBVDOMElement@2@QAVSchemaInfo@2@QBG2H@Z 120b1280 f   TraverseSchema.obj
 0001:000b07a0       ?isSubstitutionGroupCircular@TraverseSchema@xercesc_2_3@@AAE_NQAVSchemaElementDecl@2@0@Z 120b17a0 f   TraverseSchema.obj
 0001:000b07d0       ?reportSchemaError@TraverseSchema@xercesc_2_3@@AAEXQBVXSDLocator@2@QBGH@Z 120b17d0 f   TraverseSchema.obj
 0001:000b07f0       ?reportSchemaError@TraverseSchema@xercesc_2_3@@AAEXQBVXSDLocator@2@QBGH1111@Z 120b17f0 f   TraverseSchema.obj
 0001:000b0830       ?reportSchemaError@TraverseSchema@xercesc_2_3@@AAEXQBVDOMElement@2@QBGH@Z 120b1830 f   TraverseSchema.obj
 0001:000b0880       ?reportSchemaError@TraverseSchema@xercesc_2_3@@AAEXQBVDOMElement@2@QBGH1111@Z 120b1880 f   TraverseSchema.obj
 0001:000b08e0       ?init@TraverseSchema@xercesc_2_3@@AAEXXZ 120b18e0 f   TraverseSchema.obj
 0001:000b0d40       ?cleanUp@TraverseSchema@xercesc_2_3@@AAEXXZ 120b1d40 f   TraverseSchema.obj
 0001:000b0f50       ??0?$ValueVectorOf@I@xercesc_2_3@@QAE@ABV01@@Z 120b1f50 f i TraverseSchema.obj
 0001:000b0fa0       ??4?$ValueVectorOf@I@xercesc_2_3@@QAEAAV01@ABV01@@Z 120b1fa0 f i TraverseSchema.obj
 0001:000b1000       ?containsElement@?$BaseRefVectorOf@VSchemaInfo@xercesc_2_3@@@xercesc_2_3@@QAE_NQBVSchemaInfo@2@@Z 120b2000 f i TraverseSchema.obj
 0001:000b1000       ?containsElement@?$BaseRefVectorOf@VSchemaElementDecl@xercesc_2_3@@@xercesc_2_3@@QAE_NQBVSchemaElementDecl@2@@Z 120b2000 f i TraverseSchema.obj
 0001:000b1030       ??0?$RefVectorOf@VSchemaElementDecl@xercesc_2_3@@@xercesc_2_3@@QAE@I_NQAVMemoryManager@1@@Z 120b2030 f i TraverseSchema.obj
 0001:000b1090       ?get@?$RefHash2KeysTableOf@G@xercesc_2_3@@QAEPAGQBXH@Z 120b2090 f i TraverseSchema.obj
 0001:000b1090       ?get@?$RefHash2KeysTableOf@VSchemaAttDef@xercesc_2_3@@@xercesc_2_3@@QAEPAVSchemaAttDef@2@QBXH@Z 120b2090 f i TraverseSchema.obj
 0001:000b1130       ??0?$RefVectorOf@VIdentityConstraint@xercesc_2_3@@@xercesc_2_3@@QAE@I_NQAVMemoryManager@1@@Z 120b2130 f i TraverseSchema.obj
 0001:000b1190       ??0?$RefVectorOf@VSchemaInfo@xercesc_2_3@@@xercesc_2_3@@QAE@I_NQAVMemoryManager@1@@Z 120b2190 f i TraverseSchema.obj
 0001:000b11f0       ?elementAt@?$ValueVectorOf@PAVContentSpecNode@xercesc_2_3@@@xercesc_2_3@@QAEAAPAVContentSpecNode@2@I@Z 120b21f0 f i TraverseSchema.obj
 0001:000b11f0       ?elementAt@?$ValueVectorOf@PBG@xercesc_2_3@@QAEAAPBGI@Z 120b21f0 f i TraverseSchema.obj
 0001:000b11f0       ?elementAt@?$ValueVectorOf@H@xercesc_2_3@@QAEAAHI@Z 120b21f0 f i TraverseSchema.obj
 0001:000b11f0       ?elementAt@?$ValueVectorOf@PBVDOMElement@xercesc_2_3@@@xercesc_2_3@@QAEAAPBVDOMElement@2@I@Z 120b21f0 f i TraverseSchema.obj
 0001:000b11f0       ?elementAt@?$ValueVectorOf@I@xercesc_2_3@@QAEAAII@Z 120b21f0 f i TraverseSchema.obj
 0001:000b11f0       ?elementAt@?$ValueVectorOf@PAVComplexTypeInfo@xercesc_2_3@@@xercesc_2_3@@QAEAAPAVComplexTypeInfo@2@I@Z 120b21f0 f i TraverseSchema.obj
 0001:000b1230       ??0?$RefVectorOf@VSchemaAttDef@xercesc_2_3@@@xercesc_2_3@@QAE@I_NQAVMemoryManager@1@@Z 120b2230 f i TraverseSchema.obj
 0001:000b1290       ?put@?$RefHashTableOf@V?$ValueVectorOf@PAVSchemaElementDecl@xercesc_2_3@@@xercesc_2_3@@@xercesc_2_3@@QAEXPAXQAV?$ValueVectorOf@PAVSchemaElementDecl@xercesc_2_3@@@2@@Z 120b2290 f i TraverseSchema.obj
 0001:000b14b0       ??0?$RefHashTableOf@V?$ValueVectorOf@I@xercesc_2_3@@@xercesc_2_3@@QAE@IQAVMemoryManager@1@@Z 120b24b0 f i TraverseSchema.obj
 0001:000b15a0       ??1?$RefHashTableOf@V?$ValueVectorOf@I@xercesc_2_3@@@xercesc_2_3@@QAE@XZ 120b25a0 f i TraverseSchema.obj
 0001:000b1630       ?put@?$RefHashTableOf@V?$ValueVectorOf@I@xercesc_2_3@@@xercesc_2_3@@QAEXPAXQAV?$ValueVectorOf@I@2@@Z 120b2630 f i TraverseSchema.obj
 0001:000b1850       ?put@?$RefHashTableOf@V?$ValueVectorOf@PAVDOMElement@xercesc_2_3@@@xercesc_2_3@@@xercesc_2_3@@QAEXPAXQAV?$ValueVectorOf@PAVDOMElement@xercesc_2_3@@@2@@Z 120b2850 f i TraverseSchema.obj
 0001:000b1a70       ?put@?$RefHashTableOf@VXMLAttDef@xercesc_2_3@@@xercesc_2_3@@QAEXPAXQAVXMLAttDef@2@@Z 120b2a70 f i TraverseSchema.obj
 0001:000b1c80       ??1?$RefHashTableOf@VSchemaInfo@xercesc_2_3@@@xercesc_2_3@@QAE@XZ 120b2c80 f i TraverseSchema.obj
 0001:000b1d10       ?put@?$RefHashTableOf@VSchemaInfo@xercesc_2_3@@@xercesc_2_3@@QAEXPAXQAVSchemaInfo@2@@Z 120b2d10 f i TraverseSchema.obj
 0001:000b1f20       ?put@?$RefHash2KeysTableOf@G@xercesc_2_3@@QAEXPAXHQAG@Z 120b2f20 f i TraverseSchema.obj
 0001:000b2040       ?put@?$RefHash2KeysTableOf@VIdentityConstraint@xercesc_2_3@@@xercesc_2_3@@QAEXPAXHQAVIdentityConstraint@2@@Z 120b3040 f i TraverseSchema.obj
 0001:000b2160       ??1?$Janitor@VQName@xercesc_2_3@@@xercesc_2_3@@QAE@XZ 120b3160 f i TraverseSchema.obj
 0001:000b2190       ??1?$ValueVectorOf@_N@xercesc_2_3@@QAE@XZ 120b3190 f i TraverseSchema.obj
 0001:000b2190       ??1?$ValueStackOf@VDOM_Node@xercesc_2_3@@@xercesc_2_3@@QAE@XZ 120b3190 f i TraverseSchema.obj
 0001:000b2190       ??1?$ValueVectorOf@I@xercesc_2_3@@QAE@XZ 120b3190 f i TraverseSchema.obj
 0001:000b2190       ??1?$ValueStackOf@H@xercesc_2_3@@QAE@XZ 120b3190 f i TraverseSchema.obj
 0001:000b2190       ??1?$ValueVectorOf@PAVXercesAttGroupInfo@xercesc_2_3@@@xercesc_2_3@@QAE@XZ 120b3190 f i TraverseSchema.obj
 0001:000b2190       ??1?$ValueVectorOf@PAVQName@xercesc_2_3@@@xercesc_2_3@@QAE@XZ 120b3190 f i TraverseSchema.obj
 0001:000b2190       ??1?$ValueVectorOf@W4NodeTypes@ContentSpecNode@xercesc_2_3@@@xercesc_2_3@@QAE@XZ 120b3190 f i TraverseSchema.obj
 0001:000b2190       ??1?$ValueVectorOf@PAG@xercesc_2_3@@QAE@XZ 120b3190 f i TraverseSchema.obj
 0001:000b2190       ??1?$ValueVectorOf@H@xercesc_2_3@@QAE@XZ 120b3190 f i TraverseSchema.obj
 0001:000b2190       ??1?$ValueVectorOf@PAVContentSpecNode@xercesc_2_3@@@xercesc_2_3@@QAE@XZ 120b3190 f i TraverseSchema.obj
 0001:000b2190       ??1?$ValueStackOf@PAVDOMNode@xercesc_2_3@@@xercesc_2_3@@QAE@XZ 120b3190 f i TraverseSchema.obj
 0001:000b2190       ??1?$ValueStackOf@I@xercesc_2_3@@QAE@XZ 120b3190 f i TraverseSchema.obj
 0001:000b21a0       ??_G?$RefVectorOf@VDatatypeValidator@xercesc_2_3@@@xercesc_2_3@@UAEPAXI@Z 120b31a0 f i TraverseSchema.obj
 0001:000b21a0       ??_E?$RefVectorOf@VDatatypeValidator@xercesc_2_3@@@xercesc_2_3@@UAEPAXI@Z 120b31a0 f i TraverseSchema.obj
 0001:000b21c0       ??1?$RefVectorOf@VDatatypeValidator@xercesc_2_3@@@xercesc_2_3@@UAE@XZ 120b31c0 f i TraverseSchema.obj
 0001:000b2240       ??1?$BaseRefVectorOf@VDatatypeValidator@xercesc_2_3@@@xercesc_2_3@@UAE@XZ 120b3240 f i TraverseSchema.obj
 0001:000b2250       ??_GSchemaInfo@xercesc_2_3@@QAEPAXI@Z 120b3250 f i TraverseSchema.obj
 0001:000b2270       ??_G?$ValueVectorOf@PAVSchemaElementDecl@xercesc_2_3@@@xercesc_2_3@@QAEPAXI@Z 120b3270 f i TraverseSchema.obj
 0001:000b22a0       ??_GXercesAttGroupInfo@xercesc_2_3@@QAEPAXI@Z 120b32a0 f i TraverseSchema.obj
 0001:000b22c0       ??0?$RefHash2KeysTableBucketElem@VIdentityConstraint@xercesc_2_3@@@xercesc_2_3@@QAE@PAXHQAVIdentityConstraint@1@PAU01@@Z 120b32c0 f i TraverseSchema.obj
 0001:000b22c0       ??0?$RefHash2KeysTableBucketElem@V?$ValueVectorOf@PAVSchemaElementDecl@xercesc_2_3@@@xercesc_2_3@@@xercesc_2_3@@QAE@PAXHQAV?$ValueVectorOf@PAVSchemaElementDecl@xercesc_2_3@@@1@PAU01@@Z 120b32c0 f i TraverseSchema.obj
 0001:000b22c0       ??0?$RefHash2KeysTableBucketElem@VSchemaInfo@xercesc_2_3@@@xercesc_2_3@@QAE@PAXHQAVSchemaInfo@1@PAU01@@Z 120b32c0 f i TraverseSchema.obj
 0001:000b22e0       ??0?$BaseRefVectorOf@VDatatypeValidator@xercesc_2_3@@@xercesc_2_3@@QAE@I_NQAVMemoryManager@1@@Z 120b32e0 f i TraverseSchema.obj
 0001:000b2340       ??0?$BaseRefVectorOf@VIC_Field@xercesc_2_3@@@xercesc_2_3@@QAE@I_NQAVMemoryManager@1@@Z 120b3340 f i TraverseSchema.obj
 0001:000b23a0       ??0?$BaseRefVectorOf@VSchemaAttDef@xercesc_2_3@@@xercesc_2_3@@QAE@I_NQAVMemoryManager@1@@Z 120b33a0 f i TraverseSchema.obj
 0001:000b2400       ?findBucketElem@?$RefHashTableOf@VXercesAttGroupInfo@xercesc_2_3@@@xercesc_2_3@@ABEPBU?$RefHashTableBucketElem@VXercesAttGroupInfo@xercesc_2_3@@@2@QBXAAI@Z 120b3400 f i TraverseSchema.obj
 0001:000b2400       ?findBucketElem@?$RefHashTableOf@VDatatypeValidator@xercesc_2_3@@@xercesc_2_3@@ABEPBU?$RefHashTableBucketElem@VDatatypeValidator@xercesc_2_3@@@2@QBXAAI@Z 120b3400 f i TraverseSchema.obj
 0001:000b2400       ?findBucketElem@?$RefHashTableOf@VComplexTypeInfo@xercesc_2_3@@@xercesc_2_3@@ABEPBU?$RefHashTableBucketElem@VComplexTypeInfo@xercesc_2_3@@@2@QBXAAI@Z 120b3400 f i TraverseSchema.obj
 0001:000b2400       ?findBucketElem@?$RefHashTableOf@G@xercesc_2_3@@ABEPBU?$RefHashTableBucketElem@G@2@QBXAAI@Z 120b3400 f i TraverseSchema.obj
 0001:000b2400       ?findBucketElem@?$RefHashTableOf@V?$ValueVectorOf@PAVSchemaElementDecl@xercesc_2_3@@@xercesc_2_3@@@xercesc_2_3@@ABEPBU?$RefHashTableBucketElem@V?$ValueVectorOf@PAVSchemaElementDecl@xercesc_2_3@@@xercesc_2_3@@@2@QBXAAI@Z 120b3400 f i TraverseSchema.obj
 0001:000b2400       ?findBucketElem@?$RefHashTableOf@VKVStringPair@xercesc_2_3@@@xercesc_2_3@@ABEPBU?$RefHashTableBucketElem@VKVStringPair@xercesc_2_3@@@2@QBXAAI@Z 120b3400 f i TraverseSchema.obj
 0001:000b2400       ?findBucketElem@?$RefHashTableOf@VXercesGroupInfo@xercesc_2_3@@@xercesc_2_3@@ABEPBU?$RefHashTableBucketElem@VXercesGroupInfo@xercesc_2_3@@@2@QBXAAI@Z 120b3400 f i TraverseSchema.obj
 0001:000b2400       ?findBucketElem@?$RefHashTableOf@VGrammar@xercesc_2_3@@@xercesc_2_3@@ABEPBU?$RefHashTableBucketElem@VGrammar@xercesc_2_3@@@2@QBXAAI@Z 120b3400 f i TraverseSchema.obj
 0001:000b2400       ?findBucketElem@?$RefHashTableOf@VSchemaInfo@xercesc_2_3@@@xercesc_2_3@@ABEPBU?$RefHashTableBucketElem@VSchemaInfo@xercesc_2_3@@@2@QBXAAI@Z 120b3400 f i TraverseSchema.obj
 0001:000b2400       ?findBucketElem@?$RefHashTableOf@VXMLAttDef@xercesc_2_3@@@xercesc_2_3@@ABEPBU?$RefHashTableBucketElem@VXMLAttDef@xercesc_2_3@@@2@QBXAAI@Z 120b3400 f i TraverseSchema.obj
 0001:000b2400       ?findBucketElem@?$RefHashTableOf@VRangeTokenElemMap@xercesc_2_3@@@xercesc_2_3@@ABEPBU?$RefHashTableBucketElem@VRangeTokenElemMap@xercesc_2_3@@@2@QBXAAI@Z 120b3400 f i TraverseSchema.obj
 0001:000b2480       ?removeAll@?$RefHashTableOf@V?$ValueVectorOf@PAVDOMElement@xercesc_2_3@@@xercesc_2_3@@@xercesc_2_3@@QAEXXZ 120b3480 f i TraverseSchema.obj
 0001:000b2480       ?removeAll@?$RefHashTableOf@V?$ValueVectorOf@PAVSchemaElementDecl@xercesc_2_3@@@xercesc_2_3@@@xercesc_2_3@@QAEXXZ 120b3480 f i TraverseSchema.obj
 0001:000b2510       ?initialize@?$RefHashTableOf@V?$RefHashTableOf@V?$KeyRefPair@XVDOMUserDataHandler@xercesc_2_3@@@xercesc_2_3@@@xercesc_2_3@@@xercesc_2_3@@AAEXI@Z 120b3510 f i TraverseSchema.obj
 0001:000b2510       ?initialize@?$RefHashTableOf@VXercesAttGroupInfo@xercesc_2_3@@@xercesc_2_3@@AAEXI@Z 120b3510 f i TraverseSchema.obj
 0001:000b2510       ?initialize@?$RefHashTableOf@V?$ValueVectorOf@PAVSchemaElementDecl@xercesc_2_3@@@xercesc_2_3@@@xercesc_2_3@@AAEXI@Z 120b3510 f i TraverseSchema.obj
 0001:000b2510       ?initialize@?$RefHashTableOf@VXercesGroupInfo@xercesc_2_3@@@xercesc_2_3@@AAEXI@Z 120b3510 f i TraverseSchema.obj
 0001:000b2510       ?initialize@?$RefHashTableOf@V?$KeyRefPair@XVDOMUserDataHandler@xercesc_2_3@@@xercesc_2_3@@@xercesc_2_3@@AAEXI@Z 120b3510 f i TraverseSchema.obj
 0001:000b2510       ?initialize@?$RefHashTableOf@VXMLElementDecl@xercesc_2_3@@@xercesc_2_3@@AAEXI@Z 120b3510 f i TraverseSchema.obj
 0001:000b2510       ?initialize@?$RefHashTableOf@VKVStringPair@xercesc_2_3@@@xercesc_2_3@@AAEXI@Z 120b3510 f i TraverseSchema.obj
 0001:000b2510       ?initialize@?$RefHashTableOf@VXMLAttDef@xercesc_2_3@@@xercesc_2_3@@AAEXI@Z 120b3510 f i TraverseSchema.obj
 0001:000b2510       ?initialize@?$RefHashTableOf@VGrammar@xercesc_2_3@@@xercesc_2_3@@AAEXI@Z 120b3510 f i TraverseSchema.obj
 0001:000b2510       ?initialize@?$RefHashTableOf@V?$ValueVectorOf@PAVDOMElement@xercesc_2_3@@@xercesc_2_3@@@xercesc_2_3@@AAEXI@Z 120b3510 f i TraverseSchema.obj
 0001:000b2510       ?initialize@?$RefHashTableOf@G@xercesc_2_3@@AAEXI@Z 120b3510 f i TraverseSchema.obj
 0001:000b2510       ?initialize@?$RefHashTableOf@VComplexTypeInfo@xercesc_2_3@@@xercesc_2_3@@AAEXI@Z 120b3510 f i TraverseSchema.obj
 0001:000b2510       ?initialize@?$RefHashTableOf@VDatatypeValidator@xercesc_2_3@@@xercesc_2_3@@AAEXI@Z 120b3510 f i TraverseSchema.obj
 0001:000b2580       ?removeAll@?$RefHash2KeysTableOf@VSchemaInfo@xercesc_2_3@@@xercesc_2_3@@QAEXXZ 120b3580 f i TraverseSchema.obj
 0001:000b25f0       ?findBucketElem@?$RefHash2KeysTableOf@G@xercesc_2_3@@AAEPAU?$RefHash2KeysTableBucketElem@G@2@QBXHAAI@Z 120b35f0 f i TraverseSchema.obj
 0001:000b25f0       ?findBucketElem@?$RefHash2KeysTableOf@VIdentityConstraint@xercesc_2_3@@@xercesc_2_3@@AAEPAU?$RefHash2KeysTableBucketElem@VIdentityConstraint@xercesc_2_3@@@2@QBXHAAI@Z 120b35f0 f i TraverseSchema.obj
 0001:000b25f0       ?findBucketElem@?$RefHash2KeysTableOf@VSchemaInfo@xercesc_2_3@@@xercesc_2_3@@AAEPAU?$RefHash2KeysTableBucketElem@VSchemaInfo@xercesc_2_3@@@2@QBXHAAI@Z 120b35f0 f i TraverseSchema.obj
 0001:000b25f0       ?findBucketElem@?$RefHash2KeysTableOf@VSchemaAttDef@xercesc_2_3@@@xercesc_2_3@@AAEPAU?$RefHash2KeysTableBucketElem@VSchemaAttDef@xercesc_2_3@@@2@QBXHAAI@Z 120b35f0 f i TraverseSchema.obj
 0001:000b25f0       ?findBucketElem@?$RefHash2KeysTableOf@V?$ValueVectorOf@PAVSchemaElementDecl@xercesc_2_3@@@xercesc_2_3@@@xercesc_2_3@@AAEPAU?$RefHash2KeysTableBucketElem@V?$ValueVectorOf@PAVSchemaElementDecl@xercesc_2_3@@@xercesc_2_3@@@2@QBXHAAI@Z 120b35f0 f i TraverseSchema.obj
 0001:000b2680       ?removeAll@?$RefHash2KeysTableOf@G@xercesc_2_3@@QAEXXZ 120b3680 f i TraverseSchema.obj
 0001:000b26e0       ?findBucketElem@?$RefHash2KeysTableOf@VIdentityConstraint@xercesc_2_3@@@xercesc_2_3@@ABEPBU?$RefHash2KeysTableBucketElem@VIdentityConstraint@xercesc_2_3@@@2@QBXHAAI@Z 120b36e0 f i TraverseSchema.obj
 0001:000b26e0       ?findBucketElem@?$RefHash2KeysTableOf@G@xercesc_2_3@@ABEPBU?$RefHash2KeysTableBucketElem@G@2@QBXHAAI@Z 120b36e0 f i TraverseSchema.obj
 0001:000b2770       ?removeAll@?$RefHash2KeysTableOf@VIdentityConstraint@xercesc_2_3@@@xercesc_2_3@@QAEXXZ 120b3770 f i TraverseSchema.obj
 0001:000b2770       ?removeAll@?$RefHash2KeysTableOf@VSchemaAttDef@xercesc_2_3@@@xercesc_2_3@@QAEXXZ 120b3770 f i TraverseSchema.obj
 0001:000b27d0       ?initialize@?$RefHash2KeysTableOf@VSchemaAttDef@xercesc_2_3@@@xercesc_2_3@@AAEXI@Z 120b37d0 f i TraverseSchema.obj
 0001:000b27d0       ?initialize@?$RefHash2KeysTableOf@VIdentityConstraint@xercesc_2_3@@@xercesc_2_3@@AAEXI@Z 120b37d0 f i TraverseSchema.obj
 0001:000b2840       ?reset@?$Janitor@V?$RefVectorOf@VDatatypeValidator@xercesc_2_3@@@xercesc_2_3@@@xercesc_2_3@@QAEXPAV?$RefVectorOf@VDatatypeValidator@xercesc_2_3@@@2@@Z 120b3840 f i TraverseSchema.obj
 0001:000b2840       ?reset@?$Janitor@VInputSource@xercesc_2_3@@@xercesc_2_3@@QAEXPAVInputSource@2@@Z 120b3840 f i TraverseSchema.obj
 0001:000b2840       ?reset@?$Janitor@VIC_KeyRef@xercesc_2_3@@@xercesc_2_3@@QAEXPAVIC_KeyRef@2@@Z 120b3840 f i TraverseSchema.obj
 0001:000b2840       ?reset@?$Janitor@VIC_Key@xercesc_2_3@@@xercesc_2_3@@QAEXPAVIC_Key@2@@Z 120b3840 f i TraverseSchema.obj
 0001:000b2840       ?reset@?$Janitor@VIC_Unique@xercesc_2_3@@@xercesc_2_3@@QAEXPAVIC_Unique@2@@Z 120b3840 f i TraverseSchema.obj
 0001:000b2870       ??0XercesAttGroupInfo@xercesc_2_3@@QAE@QAVMemoryManager@1@@Z 120b3870 f   XercesAttGroupInfo.obj
 0001:000b2890       ??1XercesAttGroupInfo@xercesc_2_3@@QAE@XZ 120b3890 f   XercesAttGroupInfo.obj
 0001:000b28c0       ?containsAttribute@XercesAttGroupInfo@xercesc_2_3@@QAE_NQBGI@Z 120b38c0 f   XercesAttGroupInfo.obj
 0001:000b2990       ?getAttDef@XercesAttGroupInfo@xercesc_2_3@@QBEPBVSchemaAttDef@2@QBGH@Z 120b3990 f   XercesAttGroupInfo.obj
 0001:000b2a50       ?conflict@XercesElementWildcard@xercesc_2_3@@SA_NQAVSchemaGrammar@2@W4NodeTypes@ContentSpecNode@2@PAVQName@2@12PAVSubstitutionGroupComparator@2@@Z 120b3a50 f   XercesElementWildcard.obj
 0001:000b2ba0       ?uriInWildcard@XercesElementWildcard@xercesc_2_3@@CA_NQAVSchemaGrammar@2@PAVQName@2@IW4NodeTypes@ContentSpecNode@2@PAVSubstitutionGroupComparator@2@@Z 120b3ba0 f   XercesElementWildcard.obj
 0001:000b2be0       ?wildcardIntersect@XercesElementWildcard@xercesc_2_3@@CA_NW4NodeTypes@ContentSpecNode@2@I0I@Z 120b3be0 f   XercesElementWildcard.obj
 0001:000b2c40       ??0XercesGroupInfo@xercesc_2_3@@QAE@QAVMemoryManager@1@@Z 120b3c40 f   XercesGroupInfo.obj
 0001:000b2cf0       ??1XercesGroupInfo@xercesc_2_3@@QAE@XZ 120b3cf0 f   XercesGroupInfo.obj
 0001:000b2d70       ?setLocator@XercesGroupInfo@xercesc_2_3@@QAEXQAVXSDLocator@2@@Z 120b3d70 f   XercesGroupInfo.obj
 0001:000b2da0       ??0XSDDOMParser@xercesc_2_3@@QAE@QAVXMLValidator@1@QAVMemoryManager@1@@Z 120b3da0 f   XSDDOMParser.obj
 0001:000b2de0       ??_EXSDDOMParser@xercesc_2_3@@UAEPAXI@Z 120b3de0 f i XSDDOMParser.obj
 0001:000b2e40       ??1XSDDOMParser@xercesc_2_3@@UAE@XZ 120b3e40 f   XSDDOMParser.obj
 0001:000b2e60       ?createElementNSNode@XSDDOMParser@xercesc_2_3@@MAEPAVDOMElement@2@PBG0@Z 120b3e60 f   XSDDOMParser.obj
 0001:000b2ea0       ?setUserErrorReporter@XSDDOMParser@xercesc_2_3@@QAEXQAVXMLErrorReporter@2@@Z 120b3ea0 f   XSDDOMParser.obj
 0001:000b2ed0       ?setUserEntityHandler@XSDDOMParser@xercesc_2_3@@QAEXQAVXMLEntityHandler@2@@Z 120b3ed0 f   XSDDOMParser.obj
 0001:000b2f00       ?error@XSDDOMParser@xercesc_2_3@@UAEXIQBGW4ErrTypes@XMLErrorReporter@2@000JJ@Z 120b3f00 f   XSDDOMParser.obj
 0001:000b2f50       ?resolveEntity@XSDDOMParser@xercesc_2_3@@UAEPAVInputSource@2@QBG00@Z 120b3f50 f   XSDDOMParser.obj
 0001:000b2f80       ??_EXSDDOMParser@xercesc_2_3@@W3AEPAXI@Z 120b3f80 f i XSDDOMParser.obj
 0001:000b2f90       ??_EXSDDOMParser@xercesc_2_3@@W7AEPAXI@Z 120b3f90 f i XSDDOMParser.obj
 0001:000b2fa0       ??_EXSDDOMParser@xercesc_2_3@@WM@AEPAXI@Z 120b3fa0 f i XSDDOMParser.obj
 0001:000b2fb0       ??0XSDErrorReporter@xercesc_2_3@@QAE@QAVXMLErrorReporter@1@@Z 120b3fb0 f   XSDErrorReporter.obj
 0001:000b2fd0       ?emitError@XSDErrorReporter@xercesc_2_3@@QAEXIQBGQBVLocator@2@@Z 120b3fd0 f   XSDErrorReporter.obj
 0001:000b3350       ?emitError@XSDErrorReporter@xercesc_2_3@@QAEXIQBGQBVLocator@2@0000@Z 120b4350 f   XSDErrorReporter.obj
 0001:000b3690       ??0XSDLocator@xercesc_2_3@@QAE@XZ 120b4690 f   XSDLocator.obj
 0001:000b36b0       ?setValues@XSDLocator@xercesc_2_3@@QAEXQBG0JJ@Z 120b46b0 f   XSDLocator.obj
 0001:000b36d0       ?getFirstChildElement@XUtil@xercesc_2_3@@SAPAVDOMElement@2@QBVDOMNode@2@@Z 120b46d0 f   XUtil.obj
 0001:000b3710       ?getFirstChildElementNS@XUtil@xercesc_2_3@@SAPAVDOMElement@2@QBVDOMNode@2@QAPBGQBGI@Z 120b4710 f   XUtil.obj
 0001:000b3820       ?getNextSiblingElement@XUtil@xercesc_2_3@@SAPAVDOMElement@2@QBVDOMNode@2@@Z 120b4820 f   XUtil.obj
 0001:000b3860       ?getNextSiblingElementNS@XUtil@xercesc_2_3@@SAPAVDOMElement@2@QBVDOMNode@2@QAPBGQBGI@Z 120b4860 f   XUtil.obj
 0001:000b3970       ??4SchemaSymbols@xercesc_2_3@@QAEAAV01@ABV01@@Z 120b4970 f i sax2Dummy.obj
 0001:000b3970       ??4XMLUniCharacter@xercesc_2_3@@QAEAAV01@ABV01@@Z 120b4970 f i sax2Dummy.obj
 0001:000b3970       ??4HexBin@xercesc_2_3@@QAEAAV01@ABV01@@Z 120b4970 f i sax2Dummy.obj
 0001:000b3970       ??4XMLString@xercesc_2_3@@QAEAAV01@ABV01@@Z 120b4970 f i sax2Dummy.obj
 0001:000b3970       ??4XMLChar1_1@xercesc_2_3@@QAEAAV01@ABV01@@Z 120b4970 f i sax2Dummy.obj
 0001:000b3970       ??4Base64@xercesc_2_3@@QAEAAV01@ABV01@@Z 120b4970 f i sax2Dummy.obj
 0001:000b3970       ??4XPathSymbols@xercesc_2_3@@QAEAAV01@ABV01@@Z 120b4970 f i sax2Dummy.obj
 0001:000b3970       ??4DOMImplementationRegistry@xercesc_2_3@@QAEAAV01@ABV01@@Z 120b4970 f i sax2Dummy.obj
 0001:000b3970       ??4PSVIDefs@xercesc_2_3@@QAEAAV01@ABV01@@Z 120b4970 f i sax2Dummy.obj
 0001:000b3970       ??4RegxUtil@xercesc_2_3@@QAEAAV01@ABV01@@Z 120b4970 f i sax2Dummy.obj
 0001:000b3970       ??4XMLScannerResolver@xercesc_2_3@@QAEAAV01@ABV01@@Z 120b4970 f i sax2Dummy.obj
 0001:000b3970       ??4XMLUni@xercesc_2_3@@QAEAAV01@ABV01@@Z 120b4970 f i sax2Dummy.obj
 0001:000b3970       ??4XMLReaderFactory@xercesc_2_3@@QAEAAV01@ABV01@@Z 120b4970 f i sax2Dummy.obj
 0001:000b3970       ??4XMLChar1_0@xercesc_2_3@@QAEAAV01@ABV01@@Z 120b4970 f i sax2Dummy.obj
 0001:000b3970       ??4XercesElementWildcard@xercesc_2_3@@QAEAAV01@ABV01@@Z 120b4970 f i sax2Dummy.obj
 0001:000b3970       ??4XMLPlatformUtils@xercesc_2_3@@QAEAAV01@ABV01@@Z 120b4970 f i sax2Dummy.obj
 0001:000b3970       ??4XUtil@xercesc_2_3@@QAEAAV01@ABV01@@Z 120b4970 f i sax2Dummy.obj
 0001:000b3980       ?createXMLReader@XMLReaderFactory@xercesc_2_3@@SAPAVSAX2XMLReader@2@QAVMemoryManager@2@@Z 120b4980 f i sax2Dummy.obj
 0001:000b39f0       ?createXMLReader@XMLReaderFactory@xercesc_2_3@@SAPAVSAX2XMLReader@2@PBG@Z 120b49f0 f i sax2Dummy.obj
 0001:000b3a10       ??0DefaultHandler@xercesc_2_3@@QAE@XZ 120b4a10 f i sax2Dummy.obj
 0001:000b3a60       ??1DefaultHandler@xercesc_2_3@@UAE@XZ 120b4a60 f i sax2Dummy.obj
 0001:000b3ad0       ??_EDefaultHandler@xercesc_2_3@@UAEPAXI@Z 120b4ad0 f i sax2Dummy.obj
 0001:000b3b30       ?fatalError@HandlerBase@xercesc_2_3@@UAEXABVSAXParseException@2@@Z 120b4b30 f i sax2Dummy.obj
 0001:000b3b30       ?fatalError@DefaultHandler@xercesc_2_3@@UAEXABVSAXParseException@2@@Z 120b4b30 f i sax2Dummy.obj
 0001:000b3b50       ?resolveEntity@HandlerBase@xercesc_2_3@@UAEPAVInputSource@2@QBG0@Z 120b4b50 f i sax2Dummy.obj
 0001:000b3b50       ?resolveEntity@DefaultHandler@xercesc_2_3@@UAEPAVInputSource@2@QBG0@Z 120b4b50 f i sax2Dummy.obj
 0001:000b3b60       ?unparsedEntityDecl@HandlerBase@xercesc_2_3@@UAEXQBG000@Z 120b4b60 f i sax2Dummy.obj
 0001:000b3b60       ?startElement@DefaultHandler@xercesc_2_3@@UAEXQBG00ABVAttributes@2@@Z 120b4b60 f i sax2Dummy.obj
 0001:000b3b60       ?unparsedEntityDecl@DefaultHandler@xercesc_2_3@@UAEXQBG000@Z 120b4b60 f i sax2Dummy.obj
 0001:000b3b70       ?resetEntities@DOMBuilderImpl@xercesc_2_3@@UAEXXZ 120b4b70 f i sax2Dummy.obj
 0001:000b3b70       ?resetEntities@DOMParser@xercesc_2_3@@UAEXXZ 120b4b70 f i sax2Dummy.obj
 0001:000b3b70       ?startCDATA@DefaultHandler@xercesc_2_3@@UAEXXZ 120b4b70 f i sax2Dummy.obj
 0001:000b3b70       ?endDocument@ValueStoreCache@xercesc_2_3@@QAEXXZ 120b4b70 f i sax2Dummy.obj
 0001:000b3b70       ??1RegxUtil@xercesc_2_3@@QAE@XZ 120b4b70 f i sax2Dummy.obj
 0001:000b3b70       ?resetDocType@DefaultHandler@xercesc_2_3@@UAEXXZ 120b4b70 f i sax2Dummy.obj
 0001:000b3b70       ?endDocument@HandlerBase@xercesc_2_3@@UAEXXZ 120b4b70 f i sax2Dummy.obj
 0001:000b3b70       ??1XMLPScanToken@xercesc_2_3@@QAE@XZ 120b4b70 f i sax2Dummy.obj
 0001:000b3b70       ?endCDATA@DefaultHandler@xercesc_2_3@@UAEXXZ 120b4b70 f i sax2Dummy.obj
 0001:000b3b70       ?endDTD@DefaultHandler@xercesc_2_3@@UAEXXZ 120b4b70 f i sax2Dummy.obj
 0001:000b3b70       ?resetDocument@DefaultHandler@xercesc_2_3@@UAEXXZ 120b4b70 f i sax2Dummy.obj
 0001:000b3b70       ??1SubstitutionGroupComparator@xercesc_2_3@@QAE@XZ 120b4b70 f i sax2Dummy.obj
 0001:000b3b70       ?startDocument@DefaultHandler@xercesc_2_3@@UAEXXZ 120b4b70 f i sax2Dummy.obj
 0001:000b3b70       ?endDocument@DefaultHandler@xercesc_2_3@@UAEXXZ 120b4b70 f i sax2Dummy.obj
 0001:000b3b70       ?resetDocument@HandlerBase@xercesc_2_3@@UAEXXZ 120b4b70 f i sax2Dummy.obj
 0001:000b3b70       ??3@YAXPAXPAVDOMDocument@xercesc_2_3@@@Z 120b4b70 f i sax2Dummy.obj
 0001:000b3b70       ?resetEntities@XercesDOMParser@xercesc_2_3@@UAEXXZ 120b4b70 f i sax2Dummy.obj
 0001:000b3b70       ??3@YAXPAXPAVDOMDocument@xercesc_2_3@@W4NodeObjectType@DOMDocumentImpl@1@@Z 120b4b70 f i sax2Dummy.obj
 0001:000b3b70       ??1XMLUniCharacter@xercesc_2_3@@QAE@XZ 120b4b70 f i sax2Dummy.obj
 0001:000b3b70       ??1XUtil@xercesc_2_3@@IAE@XZ 120b4b70 f i sax2Dummy.obj
 0001:000b3b70       ?resetDocType@HandlerBase@xercesc_2_3@@UAEXXZ 120b4b70 f i sax2Dummy.obj
 0001:000b3b70       ?flush@XMLFormatTarget@xercesc_2_3@@UAEXXZ 120b4b70 f i sax2Dummy.obj
 0001:000b3b70       ??1XMLInteger@xercesc_2_3@@QAE@XZ 120b4b70 f i sax2Dummy.obj
 0001:000b3b70       ?resetErrors@HandlerBase@xercesc_2_3@@UAEXXZ 120b4b70 f i sax2Dummy.obj
 0001:000b3b70       ?startDocument@HandlerBase@xercesc_2_3@@UAEXXZ 120b4b70 f i sax2Dummy.obj
 0001:000b3b70       ?reset@DTDAttDef@xercesc_2_3@@UAEXXZ 120b4b70 f i sax2Dummy.obj
 0001:000b3b70       ??1EndOfEntityException@xercesc_2_3@@QAE@XZ 120b4b70 f i sax2Dummy.obj
 0001:000b3b70       ?resetErrors@DefaultHandler@xercesc_2_3@@UAEXXZ 120b4b70 f i sax2Dummy.obj
 0001:000b3b80       ?endEntity@DefaultHandler@xercesc_2_3@@UAEXQBG@Z 120b4b80 f i sax2Dummy.obj
 0001:000b3b80       ?endInputSource@XercesDOMParser@xercesc_2_3@@UAEXABVInputSource@2@@Z 120b4b80 f i sax2Dummy.obj
 0001:000b3b80       ?setContentSpec@SchemaElementDecl@xercesc_2_3@@UAEXPAVContentSpecNode@2@@Z 120b4b80 f i sax2Dummy.obj
 0001:000b3b80       ?endPrefixMapping@DefaultHandler@xercesc_2_3@@UAEXQBG@Z 120b4b80 f i sax2Dummy.obj
 0001:000b3b80       ?setMin@Token@xercesc_2_3@@UAEXH@Z 120b4b80 f i sax2Dummy.obj
 0001:000b3b80       ??4XMLFormatTarget@xercesc_2_3@@IAEXABV01@@Z 120b4b80 f i sax2Dummy.obj
 0001:000b3b80       ?validate@AnySimpleTypeDatatypeValidator@xercesc_2_3@@UAEXQBG@Z 120b4b80 f i sax2Dummy.obj
 0001:000b3b80       ?endElement@HandlerBase@xercesc_2_3@@UAEXQBG@Z 120b4b80 f i sax2Dummy.obj
 0001:000b3b80       ?error@DefaultHandler@xercesc_2_3@@UAEXABVSAXParseException@2@@Z 120b4b80 f i sax2Dummy.obj
 0001:000b3b80       ?endInputSource@DOMParser@xercesc_2_3@@UAEXABVInputSource@2@@Z 120b4b80 f i sax2Dummy.obj
 0001:000b3b80       ?startEntity@DefaultHandler@xercesc_2_3@@UAEXQBG@Z 120b4b80 f i sax2Dummy.obj
 0001:000b3b80       ?startInputSource@XercesDOMParser@xercesc_2_3@@UAEXABVInputSource@2@@Z 120b4b80 f i sax2Dummy.obj
 0001:000b3b80       ?startInputSource@DOMBuilderImpl@xercesc_2_3@@UAEXABVInputSource@2@@Z 120b4b80 f i sax2Dummy.obj
 0001:000b3b80       ?endInputSource@DOMBuilderImpl@xercesc_2_3@@UAEXABVInputSource@2@@Z 120b4b80 f i sax2Dummy.obj
 0001:000b3b80       ?setMax@Token@xercesc_2_3@@UAEXH@Z 120b4b80 f i sax2Dummy.obj
 0001:000b3b80       ?error@HandlerBase@xercesc_2_3@@UAEXABVSAXParseException@2@@Z 120b4b80 f i sax2Dummy.obj
 0001:000b3b80       ?setDocumentLocator@HandlerBase@xercesc_2_3@@UAEXQBVLocator@2@@Z 120b4b80 f i sax2Dummy.obj
 0001:000b3b80       ?setContentModel@SchemaElementDecl@xercesc_2_3@@UAEXQAVXMLContentModel@2@@Z 120b4b80 f i sax2Dummy.obj
 0001:000b3b80       ?skippedEntity@DefaultHandler@xercesc_2_3@@UAEXQBG@Z 120b4b80 f i sax2Dummy.obj
 0001:000b3b80       ?setDocumentLocator@DefaultHandler@xercesc_2_3@@UAEXQBVLocator@2@@Z 120b4b80 f i sax2Dummy.obj
 0001:000b3b80       ?warning@HandlerBase@xercesc_2_3@@UAEXABVSAXParseException@2@@Z 120b4b80 f i sax2Dummy.obj
 0001:000b3b80       ?warning@DefaultHandler@xercesc_2_3@@UAEXABVSAXParseException@2@@Z 120b4b80 f i sax2Dummy.obj
 0001:000b3b80       ?validateElement@DTDValidator@xercesc_2_3@@UAEXPBVXMLElementDecl@2@@Z 120b4b80 f i sax2Dummy.obj
 0001:000b3b80       ?setBaseURI@Wrapper4InputSource@xercesc_2_3@@UAEXQBG@Z 120b4b80 f i sax2Dummy.obj
 0001:000b3b80       ?startInputSource@DOMParser@xercesc_2_3@@UAEXABVInputSource@2@@Z 120b4b80 f i sax2Dummy.obj
 0001:000b3b90       ?attributeDecl@DefaultHandler@xercesc_2_3@@UAEXQBG0000@Z 120b4b90 f i sax2Dummy.obj
 0001:000b3ba0       ?notationDecl@DefaultHandler@xercesc_2_3@@UAEXQBG00@Z 120b4ba0 f i sax2Dummy.obj
 0001:000b3ba0       ?endElement@DefaultHandler@xercesc_2_3@@UAEXQBG00@Z 120b4ba0 f i sax2Dummy.obj
 0001:000b3ba0       ?startDTD@DefaultHandler@xercesc_2_3@@UAEXQBG00@Z 120b4ba0 f i sax2Dummy.obj
 0001:000b3ba0       ?externalEntityDecl@DefaultHandler@xercesc_2_3@@UAEXQBG00@Z 120b4ba0 f i sax2Dummy.obj
 0001:000b3ba0       ?notationDecl@HandlerBase@xercesc_2_3@@UAEXQBG00@Z 120b4ba0 f i sax2Dummy.obj
 0001:000b3bb0       ?elementDecl@DefaultHandler@xercesc_2_3@@UAEXQBG0@Z 120b4bb0 f i sax2Dummy.obj
 0001:000b3bb0       ?startPrefixMapping@DefaultHandler@xercesc_2_3@@UAEXQBG0@Z 120b4bb0 f i sax2Dummy.obj
 0001:000b3bb0       ?startElement@HandlerBase@xercesc_2_3@@UAEXQBGAAVAttributeList@2@@Z 120b4bb0 f i sax2Dummy.obj
 0001:000b3bb0       ?comment@DefaultHandler@xercesc_2_3@@UAEXQBGI@Z 120b4bb0 f i sax2Dummy.obj
 0001:000b3bb0       ?internalEntityDecl@DefaultHandler@xercesc_2_3@@UAEXQBG0@Z 120b4bb0 f i sax2Dummy.obj
 0001:000b3bb0       ?characters@DefaultHandler@xercesc_2_3@@UAEXQBGI@Z 120b4bb0 f i sax2Dummy.obj
 0001:000b3bb0       ?processingInstruction@DefaultHandler@xercesc_2_3@@UAEXQBG0@Z 120b4bb0 f i sax2Dummy.obj
 0001:000b3bb0       ?characters@HandlerBase@xercesc_2_3@@UAEXQBGI@Z 120b4bb0 f i sax2Dummy.obj
 0001:000b3bb0       ?ignorableWhitespace@HandlerBase@xercesc_2_3@@UAEXQBGI@Z 120b4bb0 f i sax2Dummy.obj
 0001:000b3bb0       ?ignorableWhitespace@DefaultHandler@xercesc_2_3@@UAEXQBGI@Z 120b4bb0 f i sax2Dummy.obj
 0001:000b3bb0       ?processingInstruction@HandlerBase@xercesc_2_3@@UAEXQBG0@Z 120b4bb0 f i sax2Dummy.obj
 0001:000b3bc0       ??_EDefaultHandler@xercesc_2_3@@W3AEPAXI@Z 120b4bc0 f i sax2Dummy.obj
 0001:000b3bd0       ??_EDefaultHandler@xercesc_2_3@@W7AEPAXI@Z 120b4bd0 f i sax2Dummy.obj
 0001:000b3be0       ??_EDefaultHandler@xercesc_2_3@@WM@AEPAXI@Z 120b4be0 f i sax2Dummy.obj
 0001:000b3bf0       ??_EDefaultHandler@xercesc_2_3@@WBA@AEPAXI@Z 120b4bf0 f i sax2Dummy.obj
 0001:000b3c00       ??_EDefaultHandler@xercesc_2_3@@WBE@AEPAXI@Z 120b4c00 f i sax2Dummy.obj
 0001:000b3c10       ??1DOMTypeInfoImpl@xercesc_2_3@@UAE@XZ 120b4c10 f i DOMAttrImpl.obj
 0001:000b3c10       ??1DOMTypeInfo@xercesc_2_3@@UAE@XZ 120b4c10 f i DOMAttrImpl.obj
 0001:000b3c20       ??0DOMAttrImpl@xercesc_2_3@@QAE@PAVDOMDocument@1@PBG@Z 120b4c20 f   DOMAttrImpl.obj
 0001:000b3cc0       ??_EDOMAttrImpl@xercesc_2_3@@UAEPAXI@Z 120b4cc0 f i DOMAttrImpl.obj
 0001:000b3d20       ??0DOMAttrImpl@xercesc_2_3@@QAE@ABV01@_N@Z 120b4d20 f   DOMAttrImpl.obj
 0001:000b3de0       ??1DOMAttrImpl@xercesc_2_3@@UAE@XZ 120b4de0 f   DOMAttrImpl.obj
 0001:000b3e40       ?cloneNode@DOMAttrImpl@xercesc_2_3@@UBEPAVDOMNode@2@_N@Z 120b4e40 f   DOMAttrImpl.obj
 0001:000b3ec0       ?getRight@CMBinaryOp@xercesc_2_3@@QAEPAVCMNode@2@XZ 120b4ec0 f   DOMAttrImpl.obj
 0001:000b3ec0       ?getPosition@CMAny@xercesc_2_3@@QBEIXZ 120b4ec0 f   DOMAttrImpl.obj
 0001:000b3ec0       ?getTarget@DOMProcessingInstructionImpl@xercesc_2_3@@UBEPBGXZ 120b4ec0 f   DOMAttrImpl.obj
 0001:000b3ec0       ?getNodeName@DOMAttrImpl@xercesc_2_3@@UBEPBGXZ 120b4ec0 f   DOMAttrImpl.obj
 0001:000b3ec0       ?getRawData@XMLAbstractDoubleFloat@xercesc_2_3@@UBEPAGXZ 120b4ec0 f   DOMAttrImpl.obj
 0001:000b3ec0       ?getNodeName@DOMEntityImpl@xercesc_2_3@@UBEPBGXZ 120b4ec0 f   DOMAttrImpl.obj
 0001:000b3ec0       ?getName@DOMAttrImpl@xercesc_2_3@@UBEPBGXZ 120b4ec0 f   DOMAttrImpl.obj
 0001:000b3ec0       ?getFirstChild@ParentNode@xercesc_2_3@@UAEPAVNodeImpl@2@XZ 120b4ec0 f   DOMAttrImpl.obj
 0001:000b3ec0       ?getNodeName@DOMProcessingInstructionImpl@xercesc_2_3@@UBEPBGXZ 120b4ec0 f   DOMAttrImpl.obj
 0001:000b3ed0       ?getNodeType@AttrImpl@xercesc_2_3@@UAEFXZ 120b4ed0 f   DOMAttrImpl.obj
 0001:000b3ed0       ?getNodeType@DOMAttrImpl@xercesc_2_3@@UBEFXZ 120b4ed0 f   DOMAttrImpl.obj
 0001:000b3ee0       ?getNodeValue@DOMAttrImpl@xercesc_2_3@@UBEPBGXZ 120b4ee0 f   DOMAttrImpl.obj
 0001:000b3ef0       ?getSpecified@DOMAttrImpl@xercesc_2_3@@UBE_NXZ 120b4ef0 f   DOMAttrImpl.obj
 0001:000b3f10       ?getValue@DOMAttrImpl@xercesc_2_3@@UBEPBGXZ 120b4f10 f   DOMAttrImpl.obj
 0001:000b4070       ?getTextValue@DOMAttrImpl@xercesc_2_3@@ABEXPAVDOMNode@2@AAVXMLBuffer@2@@Z 120b5070 f   DOMAttrImpl.obj
 0001:000b40f0       ?setNodeValue@DOMAttrImpl@xercesc_2_3@@UAEXPBG@Z 120b50f0 f   DOMAttrImpl.obj
 0001:000b4100       ?setSpecified@DOMAttrImpl@xercesc_2_3@@UAEX_N@Z 120b5100 f   DOMAttrImpl.obj
 0001:000b4140       ?setValue@DOMAttrImpl@xercesc_2_3@@UAEXPBG@Z 120b5140 f   DOMAttrImpl.obj
 0001:000b4200       ?getOwnerElement@DOMAttrImpl@xercesc_2_3@@UBEPAVDOMElement@2@XZ 120b5200 f   DOMAttrImpl.obj
 0001:000b4220       ?setOwnerElement@DOMAttrImpl@xercesc_2_3@@QAEXPAVDOMElement@2@@Z 120b5220 f   DOMAttrImpl.obj
 0001:000b4240       ?release@DOMAttrImpl@xercesc_2_3@@UAEXXZ 120b5240 f   DOMAttrImpl.obj
 0001:000b42d0       ?isId@DOMAttrImpl@xercesc_2_3@@UBE_NXZ 120b52d0 f   DOMAttrImpl.obj
 0001:000b42f0       ?rename@DOMAttrImpl@xercesc_2_3@@UAEPAVDOMNode@2@PBG0@Z 120b52f0 f   DOMAttrImpl.obj
 0001:000b43c0       ?getTypeInfo@DOMAttrImpl@xercesc_2_3@@UBEPBVDOMTypeInfo@2@XZ 120b53c0 f   DOMAttrImpl.obj
 0001:000b4460       ?setTypeInfo@DOMAttrImpl@xercesc_2_3@@UAEXPBG0@Z 120b5460 f   DOMAttrImpl.obj
 0001:000b44d0       ?getLiteral@StringOp@xercesc_2_3@@UBEPBGXZ 120b54d0 f   DOMAttrImpl.obj
 0001:000b44d0       ?getOwnerDocument@DOMElementImpl@xercesc_2_3@@UBEPAVDOMDocument@2@XZ 120b54d0 f   DOMAttrImpl.obj
 0001:000b44d0       ?getFilter@TreeWalkerImpl@xercesc_2_3@@QAEPAVDOM_NodeFilter@2@XZ 120b54d0 f   DOMAttrImpl.obj
 0001:000b44d0       ?getLeafCount@ContentLeafNameTypeVector@xercesc_2_3@@QBE?BIXZ 120b54d0 f   DOMAttrImpl.obj
 0001:000b44d0       ?getOwnerDocument@DOMAttrImpl@xercesc_2_3@@UBEPAVDOMDocument@2@XZ 120b54d0 f   DOMAttrImpl.obj
 0001:000b44d0       ?getOwnerDocument@DOMDocumentFragmentImpl@xercesc_2_3@@UBEPAVDOMDocument@2@XZ 120b54d0 f   DOMAttrImpl.obj
 0001:000b44d0       ?getLineNumber@SAXParseException@xercesc_2_3@@QBEJXZ 120b54d0 f   DOMAttrImpl.obj
 0001:000b44d0       ?getOwnerDocument@DOMEntityReferenceImpl@xercesc_2_3@@UBEPAVDOMDocument@2@XZ 120b54d0 f   DOMAttrImpl.obj
 0001:000b44d0       ?getNodeName@DOMNotationImpl@xercesc_2_3@@UBEPBGXZ 120b54d0 f   DOMAttrImpl.obj
 0001:000b44d0       ?getOwnerDocument@DOMDocumentTypeImpl@xercesc_2_3@@UBEPAVDOMDocument@2@XZ 120b54d0 f   DOMAttrImpl.obj
 0001:000b44d0       ?getWhatToShow@NodeIteratorImpl@xercesc_2_3@@QAEKXZ 120b54d0 f   DOMAttrImpl.obj
 0001:000b44d0       ?getOwnerDocument@DOMEntityImpl@xercesc_2_3@@UBEPAVDOMDocument@2@XZ 120b54d0 f   DOMAttrImpl.obj
 0001:000b44d0       ?getChild@ChildOp@xercesc_2_3@@UBEPBVOp@2@XZ 120b54d0 f   DOMAttrImpl.obj
 0001:000b44d0       ?getCurrentNode@DOMTreeWalkerImpl@xercesc_2_3@@UAEPAVDOMNode@2@XZ 120b54d0 f   DOMAttrImpl.obj
 0001:000b44d0       ?getStartOffset@RangeImpl@xercesc_2_3@@QBEIXZ 120b54d0 f   DOMAttrImpl.obj
 0001:000b44d0       ?getWhatToShow@DOMNodeIteratorImpl@xercesc_2_3@@UAEKXZ 120b54d0 f   DOMAttrImpl.obj
 0001:000b44d0       ?getRefNo@ConditionOp@xercesc_2_3@@UBEHXZ 120b54d0 f   DOMAttrImpl.obj
 0001:000b44d0       ?getOwnerDocument@DOMCDATASectionImpl@xercesc_2_3@@UBEPAVDOMDocument@2@XZ 120b54d0 f   DOMAttrImpl.obj
 0001:000b44d0       ?getToken@RangeOp@xercesc_2_3@@UBEPBVToken@2@XZ 120b54d0 f   DOMAttrImpl.obj
 0001:000b44d0       ?getSchemaType@DOMConfigurationImpl@xercesc_2_3@@QBEPBGXZ 120b54d0 f   DOMAttrImpl.obj
 0001:000b44d0       ?getData@CharOp@xercesc_2_3@@UBEHXZ 120b54d0 f   DOMAttrImpl.obj
 0001:000b44d0       ?getNewLine@DOMWriterImpl@xercesc_2_3@@UBEPBGXZ 120b54d0 f   DOMAttrImpl.obj
 0001:000b44e0       ??0DOMAttrMapImpl@xercesc_2_3@@QAE@PAVDOMNode@1@@Z 120b54e0 f   DOMAttrMapImpl.obj
 0001:000b4500       ??_EDOMAttrMapImpl@xercesc_2_3@@UAEPAXI@Z 120b5500 f i DOMAttrMapImpl.obj
 0001:000b4560       ??0DOMAttrMapImpl@xercesc_2_3@@QAE@PAVDOMNode@1@PBVDOMNamedNodeMapImpl@1@@Z 120b5560 f   DOMAttrMapImpl.obj
 0001:000b45d0       ??1DOMAttrMapImpl@xercesc_2_3@@UAE@XZ 120b55d0 f   DOMAttrMapImpl.obj
 0001:000b45e0       ?cloneAttrMap@DOMAttrMapImpl@xercesc_2_3@@UAEPAV12@PAVDOMNode@2@@Z 120b55e0 f   DOMAttrMapImpl.obj
 0001:000b4670       ?setNamedItem@DOMAttrMapImpl@xercesc_2_3@@UAEPAVDOMNode@2@PAV32@@Z 120b5670 f   DOMAttrMapImpl.obj
 0001:000b46c0       ?setNamedItemNS@DOMAttrMapImpl@xercesc_2_3@@UAEPAVDOMNode@2@PAV32@@Z 120b56c0 f   DOMAttrMapImpl.obj
 0001:000b4710       ?removeNamedItem@DOMAttrMapImpl@xercesc_2_3@@UAEPAVDOMNode@2@PBG@Z 120b5710 f   DOMAttrMapImpl.obj
 0001:000b4760       ?removeNamedItemNS@DOMAttrMapImpl@xercesc_2_3@@UAEPAVDOMNode@2@PBG0@Z 120b5760 f   DOMAttrMapImpl.obj
 0001:000b47c0       ?removeNamedItemAt@DOMAttrMapImpl@xercesc_2_3@@UAEPAVDOMNode@2@K@Z 120b57c0 f   DOMAttrMapImpl.obj
 0001:000b4840       ?reconcileDefaultAttributes@DOMAttrMapImpl@xercesc_2_3@@QAEXPBV12@@Z 120b5840 f   DOMAttrMapImpl.obj
 0001:000b48f0       ?moveSpecifiedAttributes@DOMAttrMapImpl@xercesc_2_3@@QAEXPAV12@@Z 120b58f0 f   DOMAttrMapImpl.obj
 0001:000b4950       ??1DOMAttrNSImpl@xercesc_2_3@@UAE@XZ 120b5950 f i DOMAttrNSImpl.obj
 0001:000b4960       ??_ODOMAttrNSImpl@xercesc_2_3@@QAEXABV01@@Z 120b5960 f i DOMAttrNSImpl.obj
 0001:000b4970       ??0DOMAttrNSImpl@xercesc_2_3@@QAE@PAVDOMDocument@1@PBG@Z 120b5970 f   DOMAttrNSImpl.obj
 0001:000b49a0       ??_EDOMAttrNSImpl@xercesc_2_3@@UAEPAXI@Z 120b59a0 f i DOMAttrNSImpl.obj
 0001:000b4a00       ??0DOMAttrNSImpl@xercesc_2_3@@QAE@PAVDOMDocument@1@PBG1@Z 120b5a00 f   DOMAttrNSImpl.obj
 0001:000b4a60       ??0DOMAttrNSImpl@xercesc_2_3@@QAE@ABV01@_N@Z 120b5a60 f   DOMAttrNSImpl.obj
 0001:000b4aa0       ?cloneNode@DOMAttrNSImpl@xercesc_2_3@@UBEPAVDOMNode@2@_N@Z 120b5aa0 f   DOMAttrNSImpl.obj
 0001:000b4b40       ?getNodeName@DOMDocumentTypeImpl@xercesc_2_3@@UBEPBGXZ 120b5b40 f   DOMAttrNSImpl.obj
 0001:000b4b40       ?getNodeName@DOMEntityReferenceImpl@xercesc_2_3@@UBEPBGXZ 120b5b40 f   DOMAttrNSImpl.obj
 0001:000b4b40       ?getNamespaceURI@DOMAttrNSImpl@xercesc_2_3@@UBEPBGXZ 120b5b40 f   DOMAttrNSImpl.obj
 0001:000b4b40       ?getSystemId@DOMEntityImpl@xercesc_2_3@@UBEPBGXZ 120b5b40 f   DOMAttrNSImpl.obj
 0001:000b4b40       ?getName@DOMDocumentTypeImpl@xercesc_2_3@@UBEPBGXZ 120b5b40 f   DOMAttrNSImpl.obj
 0001:000b4b40       ?getAttributes@DOMElementImpl@xercesc_2_3@@UBEPAVDOMNamedNodeMap@2@XZ 120b5b40 f   DOMAttrNSImpl.obj
 0001:000b4b50       ?getNotations@DOMDocumentTypeImpl@xercesc_2_3@@UBEPAVDOMNamedNodeMap@2@XZ 120b5b50 f   DOMAttrNSImpl.obj
 0001:000b4b50       ?getPrefix@DOMAttrNSImpl@xercesc_2_3@@UBEPBGXZ 120b5b50 f   DOMAttrNSImpl.obj
 0001:000b4b50       ?getEncoding@DOMDocumentImpl@xercesc_2_3@@UBEPBGXZ 120b5b50 f   DOMAttrNSImpl.obj
 0001:000b4b50       ?getTagName@DOMElementImpl@xercesc_2_3@@UBEPBGXZ 120b5b50 f   DOMAttrNSImpl.obj
 0001:000b4b50       ?getDoctype@DocumentImpl@xercesc_2_3@@UAEPAVDocumentTypeImpl@2@XZ 120b5b50 f   DOMAttrNSImpl.obj
 0001:000b4b50       ?getNodeName@DOMElementImpl@xercesc_2_3@@UBEPBGXZ 120b5b50 f   DOMAttrNSImpl.obj
 0001:000b4b50       ?getEntityRef@DOMEntityImpl@xercesc_2_3@@UBEPAVDOMEntityReference@2@XZ 120b5b50 f   DOMAttrNSImpl.obj
 0001:000b4b60       ?setPrefix@DOMAttrNSImpl@xercesc_2_3@@UAEXPBG@Z 120b5b60 f   DOMAttrNSImpl.obj
 0001:000b4e90       ?release@DOMAttrNSImpl@xercesc_2_3@@UAEXXZ 120b5e90 f   DOMAttrNSImpl.obj
 0001:000b4f20       ?rename@DOMAttrNSImpl@xercesc_2_3@@UAEPAVDOMNode@2@PBG0@Z 120b5f20 f   DOMAttrNSImpl.obj
 0001:000b4f70       ?setName@DOMAttrNSImpl@xercesc_2_3@@QAEXPBG0@Z 120b5f70 f   DOMAttrNSImpl.obj
 0001:000b51e0       ??_ODOMCDATASectionImpl@xercesc_2_3@@QAEXABV01@@Z 120b61e0 f i DOMCDATASectionImpl.obj
 0001:000b51f0       ??0DOMRange@xercesc_2_3@@IAE@XZ 120b61f0 f i DOMCDATASectionImpl.obj
 0001:000b5200       ??1DOMRange@xercesc_2_3@@UAE@XZ 120b6200 f i DOMCDATASectionImpl.obj
 0001:000b5210       ??_EDOMRange@xercesc_2_3@@UAEPAXI@Z 120b6210 f i DOMCDATASectionImpl.obj
 0001:000b5270       ??0DOMCDATASectionImpl@xercesc_2_3@@QAE@PAVDOMDocument@1@PBG@Z 120b6270 f   DOMCDATASectionImpl.obj
 0001:000b5300       ??_EDOMCDATASectionImpl@xercesc_2_3@@UAEPAXI@Z 120b6300 f i DOMCDATASectionImpl.obj
 0001:000b5360       ??0DOMCDATASectionImpl@xercesc_2_3@@QAE@ABV01@_N@Z 120b6360 f   DOMCDATASectionImpl.obj
 0001:000b5400       ??1DOMCDATASectionImpl@xercesc_2_3@@UAE@XZ 120b6400 f   DOMCDATASectionImpl.obj
 0001:000b5470       ?cloneNode@DOMCDATASectionImpl@xercesc_2_3@@UBEPAVDOMNode@2@_N@Z 120b6470 f   DOMCDATASectionImpl.obj
 0001:000b54f0       ?getNodeName@DOMCDATASectionImpl@xercesc_2_3@@UBEPBGXZ 120b64f0 f   DOMCDATASectionImpl.obj
 0001:000b5500       ?getNodeType@CDATASectionImpl@xercesc_2_3@@UAEFXZ 120b6500 f   DOMCDATASectionImpl.obj
 0001:000b5500       ?getNodeType@DOMCDATASectionImpl@xercesc_2_3@@UBEFXZ 120b6500 f   DOMCDATASectionImpl.obj
 0001:000b5510       ?splitText@DOMCDATASectionImpl@xercesc_2_3@@UAEPAVDOMText@2@K@Z 120b6510 f   DOMCDATASectionImpl.obj
 0001:000b5650       ?getIsWhitespaceInElementContent@DOMCDATASectionImpl@xercesc_2_3@@UBE_NXZ 120b6650 f   DOMCDATASectionImpl.obj
 0001:000b5650       ?getIsWhitespaceInElementContent@DOMTextImpl@xercesc_2_3@@UBE_NXZ 120b6650 f   DOMCDATASectionImpl.obj
 0001:000b5660       ?release@DOMCDATASectionImpl@xercesc_2_3@@UAEXXZ 120b6660 f   DOMCDATASectionImpl.obj
 0001:000b56f0       ?getNextSibling@DOMDocumentTypeImpl@xercesc_2_3@@UBEPAVDOMNode@2@XZ 120b66f0 f   DOMCDATASectionImpl.obj
 0001:000b56f0       ?getNextSibling@DOMCDATASectionImpl@xercesc_2_3@@UBEPAVDOMNode@2@XZ 120b66f0 f   DOMCDATASectionImpl.obj
 0001:000b56f0       ?getNextSibling@DOMEntityReferenceImpl@xercesc_2_3@@UBEPAVDOMNode@2@XZ 120b66f0 f   DOMCDATASectionImpl.obj
 0001:000b56f0       ?getNextSibling@DOMElementImpl@xercesc_2_3@@UBEPAVDOMNode@2@XZ 120b66f0 f   DOMCDATASectionImpl.obj
 0001:000b5700       ?getParentNode@DOMDocumentTypeImpl@xercesc_2_3@@UBEPAVDOMNode@2@XZ 120b6700 f   DOMCDATASectionImpl.obj
 0001:000b5700       ?getParentNode@DOMCDATASectionImpl@xercesc_2_3@@UBEPAVDOMNode@2@XZ 120b6700 f   DOMCDATASectionImpl.obj
 0001:000b5700       ?getParentNode@DOMElementImpl@xercesc_2_3@@UBEPAVDOMNode@2@XZ 120b6700 f   DOMCDATASectionImpl.obj
 0001:000b5700       ?getParentNode@DOMEntityReferenceImpl@xercesc_2_3@@UBEPAVDOMNode@2@XZ 120b6700 f   DOMCDATASectionImpl.obj
 0001:000b5710       ?getPreviousSibling@DOMEntityReferenceImpl@xercesc_2_3@@UBEPAVDOMNode@2@XZ 120b6710 f   DOMCDATASectionImpl.obj
 0001:000b5710       ?getPreviousSibling@DOMElementImpl@xercesc_2_3@@UBEPAVDOMNode@2@XZ 120b6710 f   DOMCDATASectionImpl.obj
 0001:000b5710       ?getPreviousSibling@DOMDocumentTypeImpl@xercesc_2_3@@UBEPAVDOMNode@2@XZ 120b6710 f   DOMCDATASectionImpl.obj
 0001:000b5710       ?getPreviousSibling@DOMCDATASectionImpl@xercesc_2_3@@UBEPAVDOMNode@2@XZ 120b6710 f   DOMCDATASectionImpl.obj
 0001:000b5720       ?getData@DOMCDATASectionImpl@xercesc_2_3@@UBEPBGXZ 120b6720 f   DOMCDATASectionImpl.obj
 0001:000b5720       ?getNodeValue@DOMCDATASectionImpl@xercesc_2_3@@UBEPBGXZ 120b6720 f   DOMCDATASectionImpl.obj
 0001:000b5730       ?getLength@DOMCDATASectionImpl@xercesc_2_3@@UBEKXZ 120b6730 f   DOMCDATASectionImpl.obj
 0001:000b5740       ?substringData@DOMCDATASectionImpl@xercesc_2_3@@UBEPBGKK@Z 120b6740 f   DOMCDATASectionImpl.obj
 0001:000b5760       ?appendData@DOMCDATASectionImpl@xercesc_2_3@@UAEXPBG@Z 120b6760 f   DOMCDATASectionImpl.obj
 0001:000b5780       ?insertData@DOMCDATASectionImpl@xercesc_2_3@@UAEXKPBG@Z 120b6780 f   DOMCDATASectionImpl.obj
 0001:000b57a0       ?deleteData@DOMCDATASectionImpl@xercesc_2_3@@UAEXKK@Z 120b67a0 f   DOMCDATASectionImpl.obj
 0001:000b57c0       ?replaceData@DOMCDATASectionImpl@xercesc_2_3@@UAEXKKPBG@Z 120b67c0 f   DOMCDATASectionImpl.obj
 0001:000b57e0       ?setData@DOMCDATASectionImpl@xercesc_2_3@@UAEXPBG@Z 120b67e0 f   DOMCDATASectionImpl.obj
 0001:000b5800       ?setNodeValue@DOMCDATASectionImpl@xercesc_2_3@@UAEXPBG@Z 120b6800 f   DOMCDATASectionImpl.obj
 0001:000b5820       ??0DOMCharacterDataImpl@xercesc_2_3@@QAE@PAVDOMDocument@1@PBG@Z 120b6820 f   DOMCharacterDataImpl.obj
 0001:000b58d0       ??0DOMCharacterDataImpl@xercesc_2_3@@QAE@ABV01@@Z 120b68d0 f   DOMCharacterDataImpl.obj
 0001:000b5980       ?setNodeValue@DOMCharacterDataImpl@xercesc_2_3@@QAEXPBVDOMNode@2@PBG@Z 120b6980 f   DOMCharacterDataImpl.obj
 0001:000b5a40       ?appendData@DOMCharacterDataImpl@xercesc_2_3@@QAEXPBVDOMNode@2@PBG@Z 120b6a40 f   DOMCharacterDataImpl.obj
 0001:000b5a90       ?deleteData@DOMCharacterDataImpl@xercesc_2_3@@QAEXPBVDOMNode@2@KK@Z 120b6a90 f   DOMCharacterDataImpl.obj
 0001:000b5c30       ?getData@DOMCharacterDataImpl@xercesc_2_3@@QBEPBGXZ 120b6c30 f   DOMCharacterDataImpl.obj
 0001:000b5c30       ?getNodeValue@DOMCharacterDataImpl@xercesc_2_3@@QBEPBGXZ 120b6c30 f   DOMCharacterDataImpl.obj
 0001:000b5c40       ?getLength@DOMCharacterDataImpl@xercesc_2_3@@QBEKXZ 120b6c40 f   DOMCharacterDataImpl.obj
 0001:000b5c50       ?insertData@DOMCharacterDataImpl@xercesc_2_3@@QAEXPBVDOMNode@2@KPBG@Z 120b6c50 f   DOMCharacterDataImpl.obj
 0001:000b5e20       ?replaceData@DOMCharacterDataImpl@xercesc_2_3@@QAEXPBVDOMNode@2@KKPBG@Z 120b6e20 f   DOMCharacterDataImpl.obj
 0001:000b5e80       ?setData@DOMCharacterDataImpl@xercesc_2_3@@QAEXPBVDOMNode@2@PBG@Z 120b6e80 f   DOMCharacterDataImpl.obj
 0001:000b5ea0       ?substringData@DOMCharacterDataImpl@xercesc_2_3@@QBEPBGPBVDOMNode@2@KK@Z 120b6ea0 f   DOMCharacterDataImpl.obj
 0001:000b5f70       ?releaseBuffer@DOMCharacterDataImpl@xercesc_2_3@@QAEXXZ 120b6f70 f   DOMCharacterDataImpl.obj
 0001:000b5f80       ??0DOMChildNode@xercesc_2_3@@QAE@XZ 120b6f80 f   DOMChildNode.obj
 0001:000b5f90       ??0DOMChildNode@xercesc_2_3@@QAE@ABV01@@Z 120b6f90 f   DOMChildNode.obj
 0001:000b5fb0       ?checkAdditionalFacetConstraints@NOTATIONDatatypeValidator@xercesc_2_3@@MBEXXZ 120b6fb0 f   DOMChildNode.obj
 0001:000b5fb0       ?normalize@DOMNodeImpl@xercesc_2_3@@QAEXXZ 120b6fb0 f   DOMChildNode.obj
 0001:000b5fb0       ?checkAdditionalFacetConstraintsBase@DateTimeValidator@xercesc_2_3@@MBEXXZ 120b6fb0 f   DOMChildNode.obj
 0001:000b5fb0       ?normalize@NodeImpl@xercesc_2_3@@UAEXXZ 120b6fb0 f   DOMChildNode.obj
 0001:000b5fb0       ??1DOM_DOMImplementation@xercesc_2_3@@QAE@XZ 120b6fb0 f   DOMChildNode.obj
 0001:000b5fb0       ?inheritAdditionalFacet@QNameDatatypeValidator@xercesc_2_3@@MAEXXZ 120b6fb0 f   DOMChildNode.obj
 0001:000b5fb0       ?normalizeEnumeration@AbstractStringValidator@xercesc_2_3@@MAEXXZ 120b6fb0 f   DOMChildNode.obj
 0001:000b5fb0       ??1DOMCharacterDataImpl@xercesc_2_3@@QAE@XZ 120b6fb0 f   DOMChildNode.obj
 0001:000b5fb0       ??1DomMemDebug@xercesc_2_3@@QAE@XZ 120b6fb0 f   DOMChildNode.obj
 0001:000b5fb0       ?endIntSubset@SAXParser@xercesc_2_3@@UAEXXZ 120b6fb0 f   DOMChildNode.obj
 0001:000b5fb0       ?resetEntities@SAX2XMLReaderImpl@xercesc_2_3@@UAEXXZ 120b6fb0 f   DOMChildNode.obj
 0001:000b5fb0       ?resetErrors@DOMBuilderImpl@xercesc_2_3@@UAEXXZ 120b6fb0 f   DOMChildNode.obj
 0001:000b5fb0       ?inheritAdditionalFacet@AnyURIDatatypeValidator@xercesc_2_3@@MAEXXZ 120b6fb0 f   DOMChildNode.obj
 0001:000b5fb0       ?startExtSubset@AbstractDOMParser@xercesc_2_3@@UAEXXZ 120b6fb0 f   DOMChildNode.obj
 0001:000b5fb0       ??1RangeTokenElemMap@xercesc_2_3@@QAE@XZ 120b6fb0 f   DOMChildNode.obj
 0001:000b5fb0       ?inheritAdditionalFacet@FloatDatatypeValidator@xercesc_2_3@@MAEXXZ 120b6fb0 f   DOMChildNode.obj
 0001:000b5fb0       ?endExtSubset@DOMParser@xercesc_2_3@@UAEXXZ 120b6fb0 f   DOMChildNode.obj
 0001:000b5fb0       ?resetEntities@SAXParser@xercesc_2_3@@UAEXXZ 120b6fb0 f   DOMChildNode.obj
 0001:000b5fb0       ?startIntSubset@SAX2XMLReaderImpl@xercesc_2_3@@UAEXXZ 120b6fb0 f   DOMChildNode.obj
 0001:000b5fb0       ?checkAdditionalFacetConstraints@AnyURIDatatypeValidator@xercesc_2_3@@MBEXXZ 120b6fb0 f   DOMChildNode.obj
 0001:000b5fb0       ?referenced@RefCountedImpl@xercesc_2_3@@UAEXXZ 120b6fb0 f   DOMChildNode.obj
 0001:000b5fb0       ?checkAdditionalFacetConstraintsBase@DoubleDatatypeValidator@xercesc_2_3@@MBEXXZ 120b6fb0 f   DOMChildNode.obj
 0001:000b5fb0       ?inheritAdditionalFacet@ListDatatypeValidator@xercesc_2_3@@MAEXXZ 120b6fb0 f   DOMChildNode.obj
 0001:000b5fb0       ??1DOMChildNode@xercesc_2_3@@QAE@XZ 120b6fb0 f   DOMChildNode.obj
 0001:000b5fb0       ?checkAdditionalFacetConstraints@QNameDatatypeValidator@xercesc_2_3@@MBEXXZ 120b6fb0 f   DOMChildNode.obj
 0001:000b5fb0       ?unreferenced@RefCountedImpl@xercesc_2_3@@UAEXXZ 120b6fb0 f   DOMChildNode.obj
 0001:000b5fb0       ?checkAdditionalFacetConstraints@ListDatatypeValidator@xercesc_2_3@@MBEXXZ 120b6fb0 f   DOMChildNode.obj
 0001:000b5fb0       ?resetErrors@XercesDOMParser@xercesc_2_3@@UAEXXZ 120b6fb0 f   DOMChildNode.obj
 0001:000b5fb0       ?inheritAdditionalFacet@Base64BinaryDatatypeValidator@xercesc_2_3@@MAEXXZ 120b6fb0 f   DOMChildNode.obj
 0001:000b5fb0       ?startIntSubset@SAXParser@xercesc_2_3@@UAEXXZ 120b6fb0 f   DOMChildNode.obj
 0001:000b5fb0       ?inheritAdditionalFacet@NOTATIONDatatypeValidator@xercesc_2_3@@MAEXXZ 120b6fb0 f   DOMChildNode.obj
 0001:000b5fb0       ??1FieldActivator@xercesc_2_3@@QAE@XZ 120b6fb0 f   DOMChildNode.obj
 0001:000b5fb0       ?checkAdditionalFacetConstraints@DateTimeValidator@xercesc_2_3@@MBEXXZ 120b6fb0 f   DOMChildNode.obj
 0001:000b5fb0       ?startExtSubset@SAXParser@xercesc_2_3@@UAEXXZ 120b6fb0 f   DOMChildNode.obj
 0001:000b5fb0       ?startExtSubset@DOMParser@xercesc_2_3@@UAEXXZ 120b6fb0 f   DOMChildNode.obj
 0001:000b5fb0       ?checkAdditionalFacetConstraints@HexBinaryDatatypeValidator@xercesc_2_3@@MBEXXZ 120b6fb0 f   DOMChildNode.obj
 0001:000b5fb0       ?checkAdditionalFacetConstraintsBase@FloatDatatypeValidator@xercesc_2_3@@MBEXXZ 120b6fb0 f   DOMChildNode.obj
 0001:000b5fb0       ??1DOMNodeImpl@xercesc_2_3@@QAE@XZ 120b6fb0 f   DOMChildNode.obj
 0001:000b5fb0       ?checkAdditionalFacetConstraints@Base64BinaryDatatypeValidator@xercesc_2_3@@MBEXXZ 120b6fb0 f   DOMChildNode.obj
 0001:000b5fb0       ?endExtSubset@SAXParser@xercesc_2_3@@UAEXXZ 120b6fb0 f   DOMChildNode.obj
 0001:000b5fb0       ?inheritAdditionalFacet@DateTimeValidator@xercesc_2_3@@MAEXXZ 120b6fb0 f   DOMChildNode.obj
 0001:000b5fb0       ?reset@DTDValidator@xercesc_2_3@@UAEXXZ 120b6fb0 f   DOMChildNode.obj
 0001:000b5fb0       ?inheritAdditionalFacet@HexBinaryDatatypeValidator@xercesc_2_3@@MAEXXZ 120b6fb0 f   DOMChildNode.obj
 0001:000b5fb0       ?platformTerm@XMLPlatformUtils@xercesc_2_3@@CAXXZ 120b6fb0 f   DOMChildNode.obj
 0001:000b5fb0       ?postParseValidation@DTDValidator@xercesc_2_3@@UAEXXZ 120b6fb0 f   DOMChildNode.obj
 0001:000b5fb0       ?endExtSubset@AbstractDOMParser@xercesc_2_3@@UAEXXZ 120b6fb0 f   DOMChildNode.obj
 0001:000b5fb0       ?postParseValidation@SchemaValidator@xercesc_2_3@@UAEXXZ 120b6fb0 f   DOMChildNode.obj
 0001:000b5fb0       ?inheritAdditionalFacet@DoubleDatatypeValidator@xercesc_2_3@@MAEXXZ 120b6fb0 f   DOMChildNode.obj
 0001:000b5fb0       ?referenced@DocumentImpl@xercesc_2_3@@UAEXXZ 120b6fb0 f   DOMChildNode.obj
 0001:000b5fb0       ?release@DOMTreeWalkerImpl@xercesc_2_3@@UAEXXZ 120b6fb0 f   DOMChildNode.obj
 0001:000b5fb0       ?checkAdditionalFacetConstraints@FloatDatatypeValidator@xercesc_2_3@@MBEXXZ 120b6fb0 f   DOMChildNode.obj
 0001:000b5fb0       ?resetErrors@DOMParser@xercesc_2_3@@UAEXXZ 120b6fb0 f   DOMChildNode.obj
 0001:000b5fb0       ?checkAdditionalFacetConstraints@DoubleDatatypeValidator@xercesc_2_3@@MBEXXZ 120b6fb0 f   DOMChildNode.obj
 0001:000b5fc0       ?getFirstChild@DOMParentNode@xercesc_2_3@@QBEPAVDOMNode@2@XZ 120b6fc0 f   DOMChildNode.obj
 0001:000b5fc0       ?getWhatToShow@DOMTreeWalkerImpl@xercesc_2_3@@UAEKXZ 120b6fc0 f   DOMChildNode.obj
 0001:000b5fc0       ?getName@DOMTypeInfoImpl@xercesc_2_3@@UBEPBGXZ 120b6fc0 f   DOMChildNode.obj
 0001:000b5fc0       ?getCurrentEntity@ReaderMgr@xercesc_2_3@@QAEPAVXMLEntityDecl@2@XZ 120b6fc0 f   DOMChildNode.obj
 0001:000b5fc0       ?getCurrentEntity@ReaderMgr@xercesc_2_3@@QBEPBVXMLEntityDecl@2@XZ 120b6fc0 f   DOMChildNode.obj
 0001:000b5fc0       ?getRoot@DOMNodeIteratorImpl@xercesc_2_3@@UAEPAVDOMNode@2@XZ 120b6fc0 f   DOMChildNode.obj
 0001:000b5fc0       ?getNextSibling@DOMChildNode@xercesc_2_3@@QBEPAVDOMNode@2@XZ 120b6fc0 f   DOMChildNode.obj
 0001:000b5fd0       ?getParentNode@DOMChildNode@xercesc_2_3@@QBEPAVDOMNode@2@PBV32@@Z 120b6fd0 f   DOMChildNode.obj
 0001:000b5ff0       ?getPreviousSibling@DOMChildNode@xercesc_2_3@@QBEPAVDOMNode@2@PBV32@@Z 120b6ff0 f   DOMChildNode.obj
 0001:000b6010       ??0DOMCommentImpl@xercesc_2_3@@QAE@PAVDOMDocument@1@PBG@Z 120b7010 f   DOMCommentImpl.obj
 0001:000b60a0       ??_EDOMCommentImpl@xercesc_2_3@@UAEPAXI@Z 120b70a0 f i DOMCommentImpl.obj
 0001:000b6100       ??0DOMCommentImpl@xercesc_2_3@@QAE@ABV01@_N@Z 120b7100 f   DOMCommentImpl.obj
 0001:000b6190       ??1DOMCommentImpl@xercesc_2_3@@UAE@XZ 120b7190 f   DOMCommentImpl.obj
 0001:000b6200       ?cloneNode@DOMCommentImpl@xercesc_2_3@@UBEPAVDOMNode@2@_N@Z 120b7200 f   DOMCommentImpl.obj
 0001:000b62c0       ?getNodeName@DOMCommentImpl@xercesc_2_3@@UBEPBGXZ 120b72c0 f   DOMCommentImpl.obj
 0001:000b62d0       ?getNodeType@DOMCommentImpl@xercesc_2_3@@UBEFXZ 120b72d0 f   DOMCommentImpl.obj
 0001:000b62d0       ?getNodeType@CommentImpl@xercesc_2_3@@UAEFXZ 120b72d0 f   DOMCommentImpl.obj
 0001:000b62e0       ?release@DOMCommentImpl@xercesc_2_3@@UAEXXZ 120b72e0 f   DOMCommentImpl.obj
 0001:000b6370       ?splitText@DOMCommentImpl@xercesc_2_3@@QAEPAVDOMComment@2@K@Z 120b7370 f   DOMCommentImpl.obj
 0001:000b64b0       ?appendChild@DOMCommentImpl@xercesc_2_3@@UAEPAVDOMNode@2@PAV32@@Z 120b74b0 f   DOMCommentImpl.obj
 0001:000b64b0       ?appendChild@DOMNotationImpl@xercesc_2_3@@UAEPAVDOMNode@2@PAV32@@Z 120b74b0 f   DOMCommentImpl.obj
 0001:000b64b0       ?appendChild@DOMProcessingInstructionImpl@xercesc_2_3@@UAEPAVDOMNode@2@PAV32@@Z 120b74b0 f   DOMCommentImpl.obj
 0001:000b64b0       ?appendChild@DOMTextImpl@xercesc_2_3@@UAEPAVDOMNode@2@PAV32@@Z 120b74b0 f   DOMCommentImpl.obj
 0001:000b64c0       ?getChildNodes@DOMProcessingInstructionImpl@xercesc_2_3@@UBEPAVDOMNodeList@2@XZ 120b74c0 f   DOMCommentImpl.obj
 0001:000b64c0       ?getChildNodes@DOMNotationImpl@xercesc_2_3@@UBEPAVDOMNodeList@2@XZ 120b74c0 f   DOMCommentImpl.obj
 0001:000b64c0       ?getChildNodes@DOMTextImpl@xercesc_2_3@@UBEPAVDOMNodeList@2@XZ 120b74c0 f   DOMCommentImpl.obj
 0001:000b64c0       ?getChildNodes@DOMCommentImpl@xercesc_2_3@@UBEPAVDOMNodeList@2@XZ 120b74c0 f   DOMCommentImpl.obj
 0001:000b64d0       ?getOwnerDocument@DOMTextImpl@xercesc_2_3@@UBEPAVDOMDocument@2@XZ 120b74d0 f   DOMCommentImpl.obj
 0001:000b64d0       ?getOwnerDocument@DOMCommentImpl@xercesc_2_3@@UBEPAVDOMDocument@2@XZ 120b74d0 f   DOMCommentImpl.obj
 0001:000b64d0       ?getOwnerDocument@DOMProcessingInstructionImpl@xercesc_2_3@@UBEPAVDOMDocument@2@XZ 120b74d0 f   DOMCommentImpl.obj
 0001:000b64d0       ?getOwnerDocument@DOMNotationImpl@xercesc_2_3@@UBEPAVDOMDocument@2@XZ 120b74d0 f   DOMCommentImpl.obj
 0001:000b64e0       ?getParentNode@DOMTextImpl@xercesc_2_3@@UBEPAVDOMNode@2@XZ 120b74e0 f   DOMCommentImpl.obj
 0001:000b64e0       ?getParentNode@DOMCommentImpl@xercesc_2_3@@UBEPAVDOMNode@2@XZ 120b74e0 f   DOMCommentImpl.obj
 0001:000b64e0       ?getParentNode@DOMProcessingInstructionImpl@xercesc_2_3@@UBEPAVDOMNode@2@XZ 120b74e0 f   DOMCommentImpl.obj
 0001:000b64f0       ?getPreviousSibling@DOMCommentImpl@xercesc_2_3@@UBEPAVDOMNode@2@XZ 120b74f0 f   DOMCommentImpl.obj
 0001:000b64f0       ?getPreviousSibling@DOMTextImpl@xercesc_2_3@@UBEPAVDOMNode@2@XZ 120b74f0 f   DOMCommentImpl.obj
 0001:000b64f0       ?getPreviousSibling@DOMProcessingInstructionImpl@xercesc_2_3@@UBEPAVDOMNode@2@XZ 120b74f0 f   DOMCommentImpl.obj
 0001:000b6500       ?normalize@DOMCommentImpl@xercesc_2_3@@UAEXXZ 120b7500 f   DOMCommentImpl.obj
 0001:000b6500       ?normalize@DOMNotationImpl@xercesc_2_3@@UAEXXZ 120b7500 f   DOMCommentImpl.obj
 0001:000b6500       ?normalize@DOMCDATASectionImpl@xercesc_2_3@@UAEXXZ 120b7500 f   DOMCommentImpl.obj
 0001:000b6500       ?normalize@DOMProcessingInstructionImpl@xercesc_2_3@@UAEXXZ 120b7500 f   DOMCommentImpl.obj
 0001:000b6500       ?normalize@DOMTextImpl@xercesc_2_3@@UAEXXZ 120b7500 f   DOMCommentImpl.obj
 0001:000b6510       ?removeChild@DOMProcessingInstructionImpl@xercesc_2_3@@UAEPAVDOMNode@2@PAV32@@Z 120b7510 f   DOMCommentImpl.obj
 0001:000b6510       ?removeChild@DOMTextImpl@xercesc_2_3@@UAEPAVDOMNode@2@PAV32@@Z 120b7510 f   DOMCommentImpl.obj
 0001:000b6510       ?removeChild@DOMNotationImpl@xercesc_2_3@@UAEPAVDOMNode@2@PAV32@@Z 120b7510 f   DOMCommentImpl.obj
 0001:000b6510       ?removeChild@DOMCommentImpl@xercesc_2_3@@UAEPAVDOMNode@2@PAV32@@Z 120b7510 f   DOMCommentImpl.obj
 0001:000b6520       ?isEqualNode@DOMProcessingInstructionImpl@xercesc_2_3@@UBE_NPBVDOMNode@2@@Z 120b7520 f   DOMCommentImpl.obj
 0001:000b6520       ?isEqualNode@DOMCommentImpl@xercesc_2_3@@UBE_NPBVDOMNode@2@@Z 120b7520 f   DOMCommentImpl.obj
 0001:000b6520       ?isEqualNode@DOMTextImpl@xercesc_2_3@@UBE_NPBVDOMNode@2@@Z 120b7520 f   DOMCommentImpl.obj
 0001:000b6520       ?isEqualNode@DOMNotationImpl@xercesc_2_3@@UBE_NPBVDOMNode@2@@Z 120b7520 f   DOMCommentImpl.obj
 0001:000b6530       ?getData@DOMTextImpl@xercesc_2_3@@UBEPBGXZ 120b7530 f   DOMCommentImpl.obj
 0001:000b6530       ?getData@DOMCommentImpl@xercesc_2_3@@UBEPBGXZ 120b7530 f   DOMCommentImpl.obj
 0001:000b6530       ?getData@DOMProcessingInstructionImpl@xercesc_2_3@@UBEPBGXZ 120b7530 f   DOMCommentImpl.obj
 0001:000b6530       ?getNodeValue@DOMProcessingInstructionImpl@xercesc_2_3@@UBEPBGXZ 120b7530 f   DOMCommentImpl.obj
 0001:000b6530       ?getNodeValue@DOMTextImpl@xercesc_2_3@@UBEPBGXZ 120b7530 f   DOMCommentImpl.obj
 0001:000b6530       ?getNodeValue@DOMCommentImpl@xercesc_2_3@@UBEPBGXZ 120b7530 f   DOMCommentImpl.obj
 0001:000b6540       ?getLength@DOMCommentImpl@xercesc_2_3@@UBEKXZ 120b7540 f   DOMCommentImpl.obj
 0001:000b6540       ?getLength@DOMTextImpl@xercesc_2_3@@UBEKXZ 120b7540 f   DOMCommentImpl.obj
 0001:000b6550       ?appendData@DOMTextImpl@xercesc_2_3@@UAEXPBG@Z 120b7550 f   DOMCommentImpl.obj
 0001:000b6550       ?appendData@DOMCommentImpl@xercesc_2_3@@UAEXPBG@Z 120b7550 f   DOMCommentImpl.obj
 0001:000b6570       ?insertData@DOMTextImpl@xercesc_2_3@@UAEXKPBG@Z 120b7570 f   DOMCommentImpl.obj
 0001:000b6570       ?insertData@DOMCommentImpl@xercesc_2_3@@UAEXKPBG@Z 120b7570 f   DOMCommentImpl.obj
 0001:000b6590       ?replaceData@DOMCommentImpl@xercesc_2_3@@UAEXKKPBG@Z 120b7590 f   DOMCommentImpl.obj
 0001:000b6590       ?replaceData@DOMTextImpl@xercesc_2_3@@UAEXKKPBG@Z 120b7590 f   DOMCommentImpl.obj
 0001:000b65b0       ??0DOMConfiguration@xercesc_2_3@@IAE@XZ 120b75b0 f i DOMConfigurationImpl.obj
 0001:000b65c0       ??0DOMConfiguration@xercesc_2_3@@IAE@ABV01@@Z 120b75c0 f i DOMConfigurationImpl.obj
 0001:000b65d0       ??4DOMConfigurationImpl@xercesc_2_3@@IAEAAV01@ABVDOMConfiguration@1@@Z 120b75d0 f i DOMConfigurationImpl.obj
 0001:000b65d0       ??4DOMConfiguration@xercesc_2_3@@IAEAAV01@ABV01@@Z 120b75d0 f i DOMConfigurationImpl.obj
 0001:000b65d0       ??4XMLAttDefList@xercesc_2_3@@IAEAAV01@ABV01@@Z 120b75d0 f i DOMConfigurationImpl.obj
 0001:000b65e0       ??0DOMConfigurationImpl@xercesc_2_3@@IAE@ABVDOMConfiguration@1@@Z 120b75e0 f i DOMConfigurationImpl.obj
 0001:000b65f0       ??0DOMConfigurationImpl@xercesc_2_3@@QAE@ABV01@@Z 120b75f0 f i DOMConfigurationImpl.obj
 0001:000b6630       ??4DOMConfigurationImpl@xercesc_2_3@@QAEAAV01@ABV01@@Z 120b7630 f i DOMConfigurationImpl.obj
 0001:000b6660       ??0DOMConfigurationImpl@xercesc_2_3@@QAE@XZ 120b7660 f   DOMConfigurationImpl.obj
 0001:000b66d0       ??1DOMConfigurationImpl@xercesc_2_3@@QAE@XZ 120b76d0 f   DOMConfigurationImpl.obj
 0001:000b66f0       ?setParameter@DOMConfigurationImpl@xercesc_2_3@@UAEXPBGPBX@Z 120b76f0 f   DOMConfigurationImpl.obj
 0001:000b6950       ?getParameter@DOMConfigurationImpl@xercesc_2_3@@UBEPBXPBG@Z 120b7950 f   DOMConfigurationImpl.obj
 0001:000b6b90       ?canSetParameter@DOMConfigurationImpl@xercesc_2_3@@UBE_NPBGPBX@Z 120b7b90 f   DOMConfigurationImpl.obj
 0001:000b6e30       ?getFeatureFlag@DOMConfigurationImpl@xercesc_2_3@@ABE?AW4DOMConfigurationFeature@12@PBG@Z 120b7e30 f   DOMConfigurationImpl.obj
 0001:000b71d0       ?getErrorHandler@DOMConfigurationImpl@xercesc_2_3@@QBEPAVDOMErrorHandler@2@XZ 120b81d0 f   DOMConfigurationImpl.obj
 0001:000b71d0       ?size@NodeVector@xercesc_2_3@@QAEIXZ 120b81d0 f   DOMConfigurationImpl.obj
 0001:000b71d0       ?getCurrentReader@ReaderMgr@xercesc_2_3@@QBEPBVXMLReader@2@XZ 120b81d0 f   DOMConfigurationImpl.obj
 0001:000b71d0       ?getLength@VecAttrListImpl@xercesc_2_3@@UBEIXZ 120b81d0 f   DOMConfigurationImpl.obj
 0001:000b71d0       ?getEncoding@DOMWriterImpl@xercesc_2_3@@UBEPBGXZ 120b81d0 f   DOMConfigurationImpl.obj
 0001:000b71d0       ?getWhatToShow@TreeWalkerImpl@xercesc_2_3@@QAEKXZ 120b81d0 f   DOMConfigurationImpl.obj
 0001:000b71d0       ?getLength@VecAttributesImpl@xercesc_2_3@@UBEIXZ 120b81d0 f   DOMConfigurationImpl.obj
 0001:000b71d0       ?getColumnNumber@SAXParseException@xercesc_2_3@@QBEJXZ 120b81d0 f   DOMConfigurationImpl.obj
 0001:000b71d0       ?getFilter@DOMTreeWalkerImpl@xercesc_2_3@@UAEPAVDOMNodeFilter@2@XZ 120b81d0 f   DOMConfigurationImpl.obj
 0001:000b71d0       ?getCurrentReader@ReaderMgr@xercesc_2_3@@QAEPAVXMLReader@2@XZ 120b81d0 f   DOMConfigurationImpl.obj
 0001:000b71d0       ?size@DOMNodeVector@xercesc_2_3@@QAEKXZ 120b81d0 f   DOMConfigurationImpl.obj
 0001:000b71d0       ?getNamespace@DOMTypeInfoImpl@xercesc_2_3@@UBEPBGXZ 120b81d0 f   DOMConfigurationImpl.obj
 0001:000b71e0       ?getConditionFlow@ConditionOp@xercesc_2_3@@UBEPBVOp@2@XZ 120b81e0 f   DOMConfigurationImpl.obj
 0001:000b71e0       ?getErrorHandler@DOMWriterImpl@xercesc_2_3@@UBEPAVDOMErrorHandler@2@XZ 120b81e0 f   DOMConfigurationImpl.obj
 0001:000b71e0       ?getRoot@DOMTreeWalkerImpl@xercesc_2_3@@UAEPAVDOMNode@2@XZ 120b81e0 f   DOMConfigurationImpl.obj
 0001:000b71e0       ?getSchemaLocation@DOMConfigurationImpl@xercesc_2_3@@QBEPBGXZ 120b81e0 f   DOMConfigurationImpl.obj
 0001:000b71e0       ?getData@ModifierOp@xercesc_2_3@@UBEHXZ 120b81e0 f   DOMConfigurationImpl.obj
 0001:000b71e0       ?getPublicId@DOMNotationImpl@xercesc_2_3@@UBEPBGXZ 120b81e0 f   DOMConfigurationImpl.obj
 0001:000b71e0       ?getPublicId@SAXParseException@xercesc_2_3@@QBEPBGXZ 120b81e0 f   DOMConfigurationImpl.obj
 0001:000b71e0       ?getFilter@DOMNodeIteratorImpl@xercesc_2_3@@UAEPAVDOMNodeFilter@2@XZ 120b81e0 f   DOMConfigurationImpl.obj
 0001:000b71e0       ?getFilter@NodeIteratorImpl@xercesc_2_3@@QAEPAVDOM_NodeFilter@2@XZ 120b81e0 f   DOMConfigurationImpl.obj
 0001:000b71f0       ?setErrorHandler@DOMConfigurationImpl@xercesc_2_3@@QAEXPAVDOMErrorHandler@2@@Z 120b81f0 f   DOMConfigurationImpl.obj
 0001:000b7200       ?setChild@ChildOp@xercesc_2_3@@QAEXQBVOp@2@@Z 120b8200 f   DOMConfigurationImpl.obj
 0001:000b7200       ?setSchemaType@DOMConfigurationImpl@xercesc_2_3@@QAEXPBG@Z 120b8200 f   DOMConfigurationImpl.obj
 0001:000b7210       ?setSchemaLocation@DOMConfigurationImpl@xercesc_2_3@@QAEXPBG@Z 120b8210 f   DOMConfigurationImpl.obj
 0001:000b7210       ?setErrorHandler@DOMWriterImpl@xercesc_2_3@@UAEXPAVDOMErrorHandler@2@@Z 120b8210 f   DOMConfigurationImpl.obj
 0001:000b7220       ??0DOMDeepNodeListImpl@xercesc_2_3@@QAE@PBVDOMNode@1@PBG@Z 120b8220 f   DOMDeepNodeListImpl.obj
 0001:000b72f0       ??_EDOMDeepNodeListImpl@xercesc_2_3@@UAEPAXI@Z 120b82f0 f i DOMDeepNodeListImpl.obj
 0001:000b7350       ??0DOMDeepNodeListImpl@xercesc_2_3@@QAE@PBVDOMNode@1@PBG1@Z 120b8350 f   DOMDeepNodeListImpl.obj
 0001:000b7490       ??1DOMDeepNodeListImpl@xercesc_2_3@@UAE@XZ 120b8490 f   DOMDeepNodeListImpl.obj
 0001:000b7490       ??1DOMNodeListImpl@xercesc_2_3@@UAE@XZ 120b8490 f   DOMDeepNodeListImpl.obj
 0001:000b74a0       ?getLength@DOMDeepNodeListImpl@xercesc_2_3@@UBEKXZ 120b84a0 f   DOMDeepNodeListImpl.obj
 0001:000b74c0       ?item@DOMDeepNodeListImpl@xercesc_2_3@@UBEPAVDOMNode@2@K@Z 120b84c0 f   DOMDeepNodeListImpl.obj
 0001:000b74d0       ?cacheItem@DOMDeepNodeListImpl@xercesc_2_3@@QAEPAVDOMNode@2@K@Z 120b84d0 f   DOMDeepNodeListImpl.obj
 0001:000b7550       ?nextMatchingElementAfter@DOMDeepNodeListImpl@xercesc_2_3@@AAEPAVDOMNode@2@PAV32@@Z 120b8550 f   DOMDeepNodeListImpl.obj
 0001:000b7700       ??0DOMDocumentFragment@xercesc_2_3@@IAE@XZ 120b8700 f i DOMDocumentFragmentImpl.obj
 0001:000b7710       ??1DOMComment@xercesc_2_3@@UAE@XZ 120b8710 f i DOMDocumentFragmentImpl.obj
 0001:000b7710       ??1DOMNode@xercesc_2_3@@UAE@XZ 120b8710 f i DOMDocumentFragmentImpl.obj
 0001:000b7710       ??1DOMEntity@xercesc_2_3@@UAE@XZ 120b8710 f i DOMDocumentFragmentImpl.obj
 0001:000b7710       ??1DOMNotation@xercesc_2_3@@UAE@XZ 120b8710 f i DOMDocumentFragmentImpl.obj
 0001:000b7710       ??1DOMProcessingInstruction@xercesc_2_3@@UAE@XZ 120b8710 f i DOMDocumentFragmentImpl.obj
 0001:000b7710       ??1DOMElement@xercesc_2_3@@UAE@XZ 120b8710 f i DOMDocumentFragmentImpl.obj
 0001:000b7710       ??1DOMText@xercesc_2_3@@UAE@XZ 120b8710 f i DOMDocumentFragmentImpl.obj
 0001:000b7710       ??1DOMCharacterData@xercesc_2_3@@UAE@XZ 120b8710 f i DOMDocumentFragmentImpl.obj
 0001:000b7710       ??1DOMAttr@xercesc_2_3@@UAE@XZ 120b8710 f i DOMDocumentFragmentImpl.obj
 0001:000b7710       ??1DOMEntityReference@xercesc_2_3@@UAE@XZ 120b8710 f i DOMDocumentFragmentImpl.obj
 0001:000b7710       ??1DOMDocumentFragment@xercesc_2_3@@UAE@XZ 120b8710 f i DOMDocumentFragmentImpl.obj
 0001:000b7710       ??1DOMCDATASection@xercesc_2_3@@UAE@XZ 120b8710 f i DOMDocumentFragmentImpl.obj
 0001:000b7710       ??1DOMDocumentType@xercesc_2_3@@UAE@XZ 120b8710 f i DOMDocumentFragmentImpl.obj
 0001:000b7720       ??0DOMDocumentFragmentImpl@xercesc_2_3@@IAE@PAVDOMDocument@1@@Z 120b8720 f   DOMDocumentFragmentImpl.obj
 0001:000b7790       ??_EDOMDocumentFragmentImpl@xercesc_2_3@@UAEPAXI@Z 120b8790 f i DOMDocumentFragmentImpl.obj
 0001:000b77f0       ??0DOMDocumentFragmentImpl@xercesc_2_3@@AAE@ABV01@_N@Z 120b87f0 f   DOMDocumentFragmentImpl.obj
 0001:000b7880       ??1DOMDocumentFragmentImpl@xercesc_2_3@@UAE@XZ 120b8880 f   DOMDocumentFragmentImpl.obj
 0001:000b78e0       ?cloneNode@DOMDocumentFragmentImpl@xercesc_2_3@@UBEPAVDOMNode@2@_N@Z 120b88e0 f   DOMDocumentFragmentImpl.obj
 0001:000b79a0       ?getNodeName@DOMDocumentFragmentImpl@xercesc_2_3@@UBEPBGXZ 120b89a0 f   DOMDocumentFragmentImpl.obj
 0001:000b79b0       ?getNodeType@DOMDocumentFragmentImpl@xercesc_2_3@@UBEFXZ 120b89b0 f   DOMDocumentFragmentImpl.obj
 0001:000b79b0       ?getNodeType@DocumentFragmentImpl@xercesc_2_3@@UAEFXZ 120b89b0 f   DOMDocumentFragmentImpl.obj
 0001:000b79c0       ?release@DOMDocumentFragmentImpl@xercesc_2_3@@UAEXXZ 120b89c0 f   DOMDocumentFragmentImpl.obj
 0001:000b7a50       ?appendChild@DOMDocumentFragmentImpl@xercesc_2_3@@UAEPAVDOMNode@2@PAV32@@Z 120b8a50 f   DOMDocumentFragmentImpl.obj
 0001:000b7a50       ?appendChild@DOMAttrImpl@xercesc_2_3@@UAEPAVDOMNode@2@PAV32@@Z 120b8a50 f   DOMDocumentFragmentImpl.obj
 0001:000b7a50       ?appendChild@DOMEntityReferenceImpl@xercesc_2_3@@UAEPAVDOMNode@2@PAV32@@Z 120b8a50 f   DOMDocumentFragmentImpl.obj
 0001:000b7a50       ?appendChild@DOMCDATASectionImpl@xercesc_2_3@@UAEPAVDOMNode@2@PAV32@@Z 120b8a50 f   DOMDocumentFragmentImpl.obj
 0001:000b7a50       ?appendChild@DOMDocumentTypeImpl@xercesc_2_3@@UAEPAVDOMNode@2@PAV32@@Z 120b8a50 f   DOMDocumentFragmentImpl.obj
 0001:000b7a50       ?appendChild@DOMElementImpl@xercesc_2_3@@UAEPAVDOMNode@2@PAV32@@Z 120b8a50 f   DOMDocumentFragmentImpl.obj
 0001:000b7a60       ?hasChildNodes@DOMCDATASectionImpl@xercesc_2_3@@UBE_NXZ 120b8a60 f   DOMDocumentFragmentImpl.obj
 0001:000b7a60       ?hasChildNodes@DOMDocumentImpl@xercesc_2_3@@UBE_NXZ 120b8a60 f   DOMDocumentFragmentImpl.obj
 0001:000b7a60       ?hasChildNodes@DOMDocumentFragmentImpl@xercesc_2_3@@UBE_NXZ 120b8a60 f   DOMDocumentFragmentImpl.obj
 0001:000b7a60       ?hasChildNodes@DOMAttrImpl@xercesc_2_3@@UBE_NXZ 120b8a60 f   DOMDocumentFragmentImpl.obj
 0001:000b7a60       ?hasChildNodes@DOMDocumentTypeImpl@xercesc_2_3@@UBE_NXZ 120b8a60 f   DOMDocumentFragmentImpl.obj
 0001:000b7a60       ?hasChildNodes@DOMElementImpl@xercesc_2_3@@UBE_NXZ 120b8a60 f   DOMDocumentFragmentImpl.obj
 0001:000b7a60       ?hasChildNodes@DOMEntityReferenceImpl@xercesc_2_3@@UBE_NXZ 120b8a60 f   DOMDocumentFragmentImpl.obj
 0001:000b7a70       ?normalize@DOMEntityReferenceImpl@xercesc_2_3@@UAEXXZ 120b8a70 f   DOMDocumentFragmentImpl.obj
 0001:000b7a70       ?normalize@DOMDocumentFragmentImpl@xercesc_2_3@@UAEXXZ 120b8a70 f   DOMDocumentFragmentImpl.obj
 0001:000b7a70       ?normalize@DOMDocumentImpl@xercesc_2_3@@UAEXXZ 120b8a70 f   DOMDocumentFragmentImpl.obj
 0001:000b7a70       ?normalize@DOMDocumentTypeImpl@xercesc_2_3@@UAEXXZ 120b8a70 f   DOMDocumentFragmentImpl.obj
 0001:000b7a70       ?normalize@DOMAttrImpl@xercesc_2_3@@UAEXXZ 120b8a70 f   DOMDocumentFragmentImpl.obj
 0001:000b7a70       ?normalize@DOMElementImpl@xercesc_2_3@@UAEXXZ 120b8a70 f   DOMDocumentFragmentImpl.obj
 0001:000b7a80       ?removeChild@DOMElementImpl@xercesc_2_3@@UAEPAVDOMNode@2@PAV32@@Z 120b8a80 f   DOMDocumentFragmentImpl.obj
 0001:000b7a80       ?removeChild@DOMDocumentTypeImpl@xercesc_2_3@@UAEPAVDOMNode@2@PAV32@@Z 120b8a80 f   DOMDocumentFragmentImpl.obj
 0001:000b7a80       ?removeChild@DOMDocumentFragmentImpl@xercesc_2_3@@UAEPAVDOMNode@2@PAV32@@Z 120b8a80 f   DOMDocumentFragmentImpl.obj
 0001:000b7a80       ?removeChild@DOMEntityReferenceImpl@xercesc_2_3@@UAEPAVDOMNode@2@PAV32@@Z 120b8a80 f   DOMDocumentFragmentImpl.obj
 0001:000b7a80       ?removeChild@DOMAttrImpl@xercesc_2_3@@UAEPAVDOMNode@2@PAV32@@Z 120b8a80 f   DOMDocumentFragmentImpl.obj
 0001:000b7a80       ?removeChild@DOMCDATASectionImpl@xercesc_2_3@@UAEPAVDOMNode@2@PAV32@@Z 120b8a80 f   DOMDocumentFragmentImpl.obj
 0001:000b7a90       ?setPrefix@DOMDocumentTypeImpl@xercesc_2_3@@UAEXPBG@Z 120b8a90 f   DOMDocumentFragmentImpl.obj
 0001:000b7a90       ?setPrefix@DOMDocumentImpl@xercesc_2_3@@UAEXPBG@Z 120b8a90 f   DOMDocumentFragmentImpl.obj
 0001:000b7a90       ?setPrefix@DOMEntityImpl@xercesc_2_3@@UAEXPBG@Z 120b8a90 f   DOMDocumentFragmentImpl.obj
 0001:000b7a90       ?setPrefix@DOMCommentImpl@xercesc_2_3@@UAEXPBG@Z 120b8a90 f   DOMDocumentFragmentImpl.obj
 0001:000b7a90       ?setPrefix@DOMDocumentFragmentImpl@xercesc_2_3@@UAEXPBG@Z 120b8a90 f   DOMDocumentFragmentImpl.obj
 0001:000b7a90       ?setPrefix@DOMNotationImpl@xercesc_2_3@@UAEXPBG@Z 120b8a90 f   DOMDocumentFragmentImpl.obj
 0001:000b7a90       ?setPrefix@DOMEntityReferenceImpl@xercesc_2_3@@UAEXPBG@Z 120b8a90 f   DOMDocumentFragmentImpl.obj
 0001:000b7a90       ?setPrefix@DOMElementImpl@xercesc_2_3@@UAEXPBG@Z 120b8a90 f   DOMDocumentFragmentImpl.obj
 0001:000b7a90       ?setPrefix@DOMAttrImpl@xercesc_2_3@@UAEXPBG@Z 120b8a90 f   DOMDocumentFragmentImpl.obj
 0001:000b7a90       ?setPrefix@DOMTextImpl@xercesc_2_3@@UAEXPBG@Z 120b8a90 f   DOMDocumentFragmentImpl.obj
 0001:000b7a90       ?setPrefix@DOMProcessingInstructionImpl@xercesc_2_3@@UAEXPBG@Z 120b8a90 f   DOMDocumentFragmentImpl.obj
 0001:000b7a90       ?setPrefix@DOMCDATASectionImpl@xercesc_2_3@@UAEXPBG@Z 120b8a90 f   DOMDocumentFragmentImpl.obj
 0001:000b7aa0       ?hasAttributes@DOMProcessingInstructionImpl@xercesc_2_3@@UBE_NXZ 120b8aa0 f   DOMDocumentFragmentImpl.obj
 0001:000b7aa0       ?hasAttributes@DOMCommentImpl@xercesc_2_3@@UBE_NXZ 120b8aa0 f   DOMDocumentFragmentImpl.obj
 0001:000b7aa0       ?hasChildNodes@DOMTextImpl@xercesc_2_3@@UBE_NXZ 120b8aa0 f   DOMDocumentFragmentImpl.obj
 0001:000b7aa0       ?hasChildNodes@DOMNotationImpl@xercesc_2_3@@UBE_NXZ 120b8aa0 f   DOMDocumentFragmentImpl.obj
 0001:000b7aa0       ?hasChildNodes@DOMCommentImpl@xercesc_2_3@@UBE_NXZ 120b8aa0 f   DOMDocumentFragmentImpl.obj
 0001:000b7aa0       ?hasAttributes@DOMDocumentTypeImpl@xercesc_2_3@@UBE_NXZ 120b8aa0 f   DOMDocumentFragmentImpl.obj
 0001:000b7aa0       ?hasAttributes@DOMTextImpl@xercesc_2_3@@UBE_NXZ 120b8aa0 f   DOMDocumentFragmentImpl.obj
 0001:000b7aa0       ?hasAttributes@DOMDocumentFragmentImpl@xercesc_2_3@@UBE_NXZ 120b8aa0 f   DOMDocumentFragmentImpl.obj
 0001:000b7aa0       ?hasAttributes@DOMEntityImpl@xercesc_2_3@@UBE_NXZ 120b8aa0 f   DOMDocumentFragmentImpl.obj
 0001:000b7aa0       ?hasAttributes@DOMDocumentImpl@xercesc_2_3@@UBE_NXZ 120b8aa0 f   DOMDocumentFragmentImpl.obj
 0001:000b7aa0       ?hasChildNodes@DOMProcessingInstructionImpl@xercesc_2_3@@UBE_NXZ 120b8aa0 f   DOMDocumentFragmentImpl.obj
 0001:000b7aa0       ?hasAttributes@DOMAttrImpl@xercesc_2_3@@UBE_NXZ 120b8aa0 f   DOMDocumentFragmentImpl.obj
 0001:000b7aa0       ?hasAttributes@DOMCDATASectionImpl@xercesc_2_3@@UBE_NXZ 120b8aa0 f   DOMDocumentFragmentImpl.obj
 0001:000b7aa0       ?hasAttributes@DOMEntityReferenceImpl@xercesc_2_3@@UBE_NXZ 120b8aa0 f   DOMDocumentFragmentImpl.obj
 0001:000b7aa0       ?hasAttributes@DOMNotationImpl@xercesc_2_3@@UBE_NXZ 120b8aa0 f   DOMDocumentFragmentImpl.obj
 0001:000b7ab0       ?isSameNode@DOMAttrImpl@xercesc_2_3@@UBE_NPBVDOMNode@2@@Z 120b8ab0 f   DOMDocumentFragmentImpl.obj
 0001:000b7ab0       ?isSameNode@DOMElementImpl@xercesc_2_3@@UBE_NPBVDOMNode@2@@Z 120b8ab0 f   DOMDocumentFragmentImpl.obj
 0001:000b7ab0       ?isSameNode@DOMCommentImpl@xercesc_2_3@@UBE_NPBVDOMNode@2@@Z 120b8ab0 f   DOMDocumentFragmentImpl.obj
 0001:000b7ab0       ?isSameNode@DOMEntityReferenceImpl@xercesc_2_3@@UBE_NPBVDOMNode@2@@Z 120b8ab0 f   DOMDocumentFragmentImpl.obj
 0001:000b7ab0       ?isSameNode@DOMProcessingInstructionImpl@xercesc_2_3@@UBE_NPBVDOMNode@2@@Z 120b8ab0 f   DOMDocumentFragmentImpl.obj
 0001:000b7ab0       ?isSameNode@DOMDocumentTypeImpl@xercesc_2_3@@UBE_NPBVDOMNode@2@@Z 120b8ab0 f   DOMDocumentFragmentImpl.obj
 0001:000b7ab0       ?isSameNode@DOMDocumentFragmentImpl@xercesc_2_3@@UBE_NPBVDOMNode@2@@Z 120b8ab0 f   DOMDocumentFragmentImpl.obj
 0001:000b7ab0       ?isSameNode@DOMCDATASectionImpl@xercesc_2_3@@UBE_NPBVDOMNode@2@@Z 120b8ab0 f   DOMDocumentFragmentImpl.obj
 0001:000b7ab0       ?isSameNode@DOMNotationImpl@xercesc_2_3@@UBE_NPBVDOMNode@2@@Z 120b8ab0 f   DOMDocumentFragmentImpl.obj
 0001:000b7ab0       ?isSameNode@DOMEntityImpl@xercesc_2_3@@UBE_NPBVDOMNode@2@@Z 120b8ab0 f   DOMDocumentFragmentImpl.obj
 0001:000b7ab0       ?isSameNode@DOMTextImpl@xercesc_2_3@@UBE_NPBVDOMNode@2@@Z 120b8ab0 f   DOMDocumentFragmentImpl.obj
 0001:000b7ab0       ?isSameNode@DOMDocumentImpl@xercesc_2_3@@UBE_NPBVDOMNode@2@@Z 120b8ab0 f   DOMDocumentFragmentImpl.obj
 0001:000b7ac0       ?isEqualNode@DOMDocumentImpl@xercesc_2_3@@UBE_NPBVDOMNode@2@@Z 120b8ac0 f   DOMDocumentFragmentImpl.obj
 0001:000b7ac0       ?isEqualNode@DOMEntityReferenceImpl@xercesc_2_3@@UBE_NPBVDOMNode@2@@Z 120b8ac0 f   DOMDocumentFragmentImpl.obj
 0001:000b7ac0       ?isEqualNode@DOMCDATASectionImpl@xercesc_2_3@@UBE_NPBVDOMNode@2@@Z 120b8ac0 f   DOMDocumentFragmentImpl.obj
 0001:000b7ac0       ?isEqualNode@DOMDocumentFragmentImpl@xercesc_2_3@@UBE_NPBVDOMNode@2@@Z 120b8ac0 f   DOMDocumentFragmentImpl.obj
 0001:000b7ac0       ?isEqualNode@DOMAttrImpl@xercesc_2_3@@UBE_NPBVDOMNode@2@@Z 120b8ac0 f   DOMDocumentFragmentImpl.obj
 0001:000b7ad0       ?getUserData@DOMDocumentTypeImpl@xercesc_2_3@@UBEPAXPBG@Z 120b8ad0 f   DOMDocumentFragmentImpl.obj
 0001:000b7ad0       ?getUserData@DOMProcessingInstructionImpl@xercesc_2_3@@UBEPAXPBG@Z 120b8ad0 f   DOMDocumentFragmentImpl.obj
 0001:000b7ad0       ?getUserData@DOMNotationImpl@xercesc_2_3@@UBEPAXPBG@Z 120b8ad0 f   DOMDocumentFragmentImpl.obj
 0001:000b7ad0       ?getUserData@DOMDocumentImpl@xercesc_2_3@@UBEPAXPBG@Z 120b8ad0 f   DOMDocumentFragmentImpl.obj
 0001:000b7ad0       ?getUserData@DOMAttrImpl@xercesc_2_3@@UBEPAXPBG@Z 120b8ad0 f   DOMDocumentFragmentImpl.obj
 0001:000b7ad0       ?getUserData@DOMEntityReferenceImpl@xercesc_2_3@@UBEPAXPBG@Z 120b8ad0 f   DOMDocumentFragmentImpl.obj
 0001:000b7ad0       ?getUserData@DOMCommentImpl@xercesc_2_3@@UBEPAXPBG@Z 120b8ad0 f   DOMDocumentFragmentImpl.obj
 0001:000b7ad0       ?getUserData@DOMEntityImpl@xercesc_2_3@@UBEPAXPBG@Z 120b8ad0 f   DOMDocumentFragmentImpl.obj
 0001:000b7ad0       ?getUserData@DOMDocumentFragmentImpl@xercesc_2_3@@UBEPAXPBG@Z 120b8ad0 f   DOMDocumentFragmentImpl.obj
 0001:000b7ad0       ?getUserData@DOMTextImpl@xercesc_2_3@@UBEPAXPBG@Z 120b8ad0 f   DOMDocumentFragmentImpl.obj
 0001:000b7ad0       ?getUserData@DOMElementImpl@xercesc_2_3@@UBEPAXPBG@Z 120b8ad0 f   DOMDocumentFragmentImpl.obj
 0001:000b7ad0       ?getUserData@DOMCDATASectionImpl@xercesc_2_3@@UBEPAXPBG@Z 120b8ad0 f   DOMDocumentFragmentImpl.obj
 0001:000b7ae0       ?getBaseURI@DOMTextImpl@xercesc_2_3@@UBEPBGXZ 120b8ae0 f   DOMDocumentFragmentImpl.obj
 0001:000b7ae0       ?getBaseURI@DOMDocumentFragmentImpl@xercesc_2_3@@UBEPBGXZ 120b8ae0 f   DOMDocumentFragmentImpl.obj
 0001:000b7ae0       ?getBaseURI@DOMCommentImpl@xercesc_2_3@@UBEPBGXZ 120b8ae0 f   DOMDocumentFragmentImpl.obj
 0001:000b7ae0       ?getBaseURI@DOMDocumentTypeImpl@xercesc_2_3@@UBEPBGXZ 120b8ae0 f   DOMDocumentFragmentImpl.obj
 0001:000b7ae0       ?getBaseURI@DOMCDATASectionImpl@xercesc_2_3@@UBEPBGXZ 120b8ae0 f   DOMDocumentFragmentImpl.obj
 0001:000b7ae0       ?getBaseURI@DOMAttrImpl@xercesc_2_3@@UBEPBGXZ 120b8ae0 f   DOMDocumentFragmentImpl.obj
 0001:000b7af0       ?compareTreePosition@DOMCommentImpl@xercesc_2_3@@UBEFPBVDOMNode@2@@Z 120b8af0 f   DOMDocumentFragmentImpl.obj
 0001:000b7af0       ?compareTreePosition@DOMEntityReferenceImpl@xercesc_2_3@@UBEFPBVDOMNode@2@@Z 120b8af0 f   DOMDocumentFragmentImpl.obj
 0001:000b7af0       ?compareTreePosition@DOMDocumentTypeImpl@xercesc_2_3@@UBEFPBVDOMNode@2@@Z 120b8af0 f   DOMDocumentFragmentImpl.obj
 0001:000b7af0       ?compareTreePosition@DOMElementImpl@xercesc_2_3@@UBEFPBVDOMNode@2@@Z 120b8af0 f   DOMDocumentFragmentImpl.obj
 0001:000b7af0       ?compareTreePosition@DOMCDATASectionImpl@xercesc_2_3@@UBEFPBVDOMNode@2@@Z 120b8af0 f   DOMDocumentFragmentImpl.obj
 0001:000b7af0       ?compareTreePosition@DOMDocumentFragmentImpl@xercesc_2_3@@UBEFPBVDOMNode@2@@Z 120b8af0 f   DOMDocumentFragmentImpl.obj
 0001:000b7af0       ?compareTreePosition@DOMProcessingInstructionImpl@xercesc_2_3@@UBEFPBVDOMNode@2@@Z 120b8af0 f   DOMDocumentFragmentImpl.obj
 0001:000b7af0       ?compareTreePosition@DOMEntityImpl@xercesc_2_3@@UBEFPBVDOMNode@2@@Z 120b8af0 f   DOMDocumentFragmentImpl.obj
 0001:000b7af0       ?compareTreePosition@DOMAttrImpl@xercesc_2_3@@UBEFPBVDOMNode@2@@Z 120b8af0 f   DOMDocumentFragmentImpl.obj
 0001:000b7af0       ?compareTreePosition@DOMTextImpl@xercesc_2_3@@UBEFPBVDOMNode@2@@Z 120b8af0 f   DOMDocumentFragmentImpl.obj
 0001:000b7af0       ?compareTreePosition@DOMNotationImpl@xercesc_2_3@@UBEFPBVDOMNode@2@@Z 120b8af0 f   DOMDocumentFragmentImpl.obj
 0001:000b7af0       ?compareTreePosition@DOMDocumentImpl@xercesc_2_3@@UBEFPBVDOMNode@2@@Z 120b8af0 f   DOMDocumentFragmentImpl.obj
 0001:000b7b00       ?getTextContent@DOMProcessingInstructionImpl@xercesc_2_3@@UBEPBGXZ 120b8b00 f   DOMDocumentFragmentImpl.obj
 0001:000b7b00       ?getTextContent@DOMDocumentFragmentImpl@xercesc_2_3@@UBEPBGXZ 120b8b00 f   DOMDocumentFragmentImpl.obj
 0001:000b7b00       ?getTextContent@DOMEntityReferenceImpl@xercesc_2_3@@UBEPBGXZ 120b8b00 f   DOMDocumentFragmentImpl.obj
 0001:000b7b00       ?getTextContent@DOMCommentImpl@xercesc_2_3@@UBEPBGXZ 120b8b00 f   DOMDocumentFragmentImpl.obj
 0001:000b7b00       ?getTextContent@DOMDocumentTypeImpl@xercesc_2_3@@UBEPBGXZ 120b8b00 f   DOMDocumentFragmentImpl.obj
 0001:000b7b00       ?getTextContent@DOMDocumentImpl@xercesc_2_3@@UBEPBGXZ 120b8b00 f   DOMDocumentFragmentImpl.obj
 0001:000b7b00       ?getTextContent@DOMTextImpl@xercesc_2_3@@UBEPBGXZ 120b8b00 f   DOMDocumentFragmentImpl.obj
 0001:000b7b00       ?getTextContent@DOMEntityImpl@xercesc_2_3@@UBEPBGXZ 120b8b00 f   DOMDocumentFragmentImpl.obj
 0001:000b7b00       ?getTextContent@DOMElementImpl@xercesc_2_3@@UBEPBGXZ 120b8b00 f   DOMDocumentFragmentImpl.obj
 0001:000b7b00       ?getTextContent@DOMCDATASectionImpl@xercesc_2_3@@UBEPBGXZ 120b8b00 f   DOMDocumentFragmentImpl.obj
 0001:000b7b00       ?getTextContent@DOMAttrImpl@xercesc_2_3@@UBEPBGXZ 120b8b00 f   DOMDocumentFragmentImpl.obj
 0001:000b7b00       ?getTextContent@DOMNotationImpl@xercesc_2_3@@UBEPBGXZ 120b8b00 f   DOMDocumentFragmentImpl.obj
 0001:000b7b10       ?isDefaultNamespace@DOMCDATASectionImpl@xercesc_2_3@@UBE_NPBG@Z 120b8b10 f   DOMDocumentFragmentImpl.obj
 0001:000b7b10       ?isDefaultNamespace@DOMCommentImpl@xercesc_2_3@@UBE_NPBG@Z 120b8b10 f   DOMDocumentFragmentImpl.obj
 0001:000b7b10       ?isDefaultNamespace@DOMEntityImpl@xercesc_2_3@@UBE_NPBG@Z 120b8b10 f   DOMDocumentFragmentImpl.obj
 0001:000b7b10       ?isDefaultNamespace@DOMEntityReferenceImpl@xercesc_2_3@@UBE_NPBG@Z 120b8b10 f   DOMDocumentFragmentImpl.obj
 0001:000b7b10       ?isDefaultNamespace@DOMDocumentFragmentImpl@xercesc_2_3@@UBE_NPBG@Z 120b8b10 f   DOMDocumentFragmentImpl.obj
 0001:000b7b10       ?isDefaultNamespace@DOMTextImpl@xercesc_2_3@@UBE_NPBG@Z 120b8b10 f   DOMDocumentFragmentImpl.obj
 0001:000b7b10       ?isDefaultNamespace@DOMNotationImpl@xercesc_2_3@@UBE_NPBG@Z 120b8b10 f   DOMDocumentFragmentImpl.obj
 0001:000b7b10       ?isDefaultNamespace@DOMProcessingInstructionImpl@xercesc_2_3@@UBE_NPBG@Z 120b8b10 f   DOMDocumentFragmentImpl.obj
 0001:000b7b10       ?isDefaultNamespace@DOMDocumentTypeImpl@xercesc_2_3@@UBE_NPBG@Z 120b8b10 f   DOMDocumentFragmentImpl.obj
 0001:000b7b10       ?isDefaultNamespace@DOMDocumentImpl@xercesc_2_3@@UBE_NPBG@Z 120b8b10 f   DOMDocumentFragmentImpl.obj
 0001:000b7b10       ?isDefaultNamespace@DOMElementImpl@xercesc_2_3@@UBE_NPBG@Z 120b8b10 f   DOMDocumentFragmentImpl.obj
 0001:000b7b10       ?isDefaultNamespace@DOMAttrImpl@xercesc_2_3@@UBE_NPBG@Z 120b8b10 f   DOMDocumentFragmentImpl.obj
 0001:000b7b20       ?lookupNamespaceURI@DOMDocumentImpl@xercesc_2_3@@UBEPBGPBG@Z 120b8b20 f   DOMDocumentFragmentImpl.obj
 0001:000b7b20       ?lookupNamespaceURI@DOMEntityImpl@xercesc_2_3@@UBEPBGPBG@Z 120b8b20 f   DOMDocumentFragmentImpl.obj
 0001:000b7b20       ?lookupNamespaceURI@DOMDocumentFragmentImpl@xercesc_2_3@@UBEPBGPBG@Z 120b8b20 f   DOMDocumentFragmentImpl.obj
 0001:000b7b20       ?lookupNamespaceURI@DOMElementImpl@xercesc_2_3@@UBEPBGPBG@Z 120b8b20 f   DOMDocumentFragmentImpl.obj
 0001:000b7b20       ?lookupNamespaceURI@DOMCDATASectionImpl@xercesc_2_3@@UBEPBGPBG@Z 120b8b20 f   DOMDocumentFragmentImpl.obj
 0001:000b7b20       ?lookupNamespaceURI@DOMEntityReferenceImpl@xercesc_2_3@@UBEPBGPBG@Z 120b8b20 f   DOMDocumentFragmentImpl.obj
 0001:000b7b20       ?lookupNamespaceURI@DOMCommentImpl@xercesc_2_3@@UBEPBGPBG@Z 120b8b20 f   DOMDocumentFragmentImpl.obj
 0001:000b7b20       ?lookupNamespaceURI@DOMTextImpl@xercesc_2_3@@UBEPBGPBG@Z 120b8b20 f   DOMDocumentFragmentImpl.obj
 0001:000b7b20       ?lookupNamespaceURI@DOMDocumentTypeImpl@xercesc_2_3@@UBEPBGPBG@Z 120b8b20 f   DOMDocumentFragmentImpl.obj
 0001:000b7b20       ?lookupNamespaceURI@DOMAttrImpl@xercesc_2_3@@UBEPBGPBG@Z 120b8b20 f   DOMDocumentFragmentImpl.obj
 0001:000b7b20       ?lookupNamespaceURI@DOMProcessingInstructionImpl@xercesc_2_3@@UBEPBGPBG@Z 120b8b20 f   DOMDocumentFragmentImpl.obj
 0001:000b7b20       ?lookupNamespaceURI@DOMNotationImpl@xercesc_2_3@@UBEPBGPBG@Z 120b8b20 f   DOMDocumentFragmentImpl.obj
 0001:000b7b30       ?setTextContent@DOMEntityReferenceImpl@xercesc_2_3@@UAEXPBG@Z 120b8b30 f   DOMDocumentFragmentImpl.obj
 0001:000b7b30       ?getInterface@DOMAttrImpl@xercesc_2_3@@UAEPAVDOMNode@2@PBG@Z 120b8b30 f   DOMDocumentFragmentImpl.obj
 0001:000b7b30       ?getInterface@DOMDocumentFragmentImpl@xercesc_2_3@@UAEPAVDOMNode@2@PBG@Z 120b8b30 f   DOMDocumentFragmentImpl.obj
 0001:000b7b30       ?setTextContent@DOMElementImpl@xercesc_2_3@@UAEXPBG@Z 120b8b30 f   DOMDocumentFragmentImpl.obj
 0001:000b7b30       ?setTextContent@DOMAttrImpl@xercesc_2_3@@UAEXPBG@Z 120b8b30 f   DOMDocumentFragmentImpl.obj
 0001:000b7b30       ?setTextContent@DOMProcessingInstructionImpl@xercesc_2_3@@UAEXPBG@Z 120b8b30 f   DOMDocumentFragmentImpl.obj
 0001:000b7b30       ?getInterface@DOMCommentImpl@xercesc_2_3@@UAEPAVDOMNode@2@PBG@Z 120b8b30 f   DOMDocumentFragmentImpl.obj
 0001:000b7b30       ?setTextContent@DOMNotationImpl@xercesc_2_3@@UAEXPBG@Z 120b8b30 f   DOMDocumentFragmentImpl.obj
 0001:000b7b30       ?setTextContent@DOMEntityImpl@xercesc_2_3@@UAEXPBG@Z 120b8b30 f   DOMDocumentFragmentImpl.obj
 0001:000b7b30       ?setTextContent@DOMDocumentFragmentImpl@xercesc_2_3@@UAEXPBG@Z 120b8b30 f   DOMDocumentFragmentImpl.obj
 0001:000b7b30       ?setTextContent@DOMCommentImpl@xercesc_2_3@@UAEXPBG@Z 120b8b30 f   DOMDocumentFragmentImpl.obj
 0001:000b7b30       ?setTextContent@DOMTextImpl@xercesc_2_3@@UAEXPBG@Z 120b8b30 f   DOMDocumentFragmentImpl.obj
 0001:000b7b30       ?getInterface@DOMDocumentImpl@xercesc_2_3@@UAEPAVDOMNode@2@PBG@Z 120b8b30 f   DOMDocumentFragmentImpl.obj
 0001:000b7b30       ?getInterface@DOMDocumentTypeImpl@xercesc_2_3@@UAEPAVDOMNode@2@PBG@Z 120b8b30 f   DOMDocumentFragmentImpl.obj
 0001:000b7b30       ?getInterface@DOMTextImpl@xercesc_2_3@@UAEPAVDOMNode@2@PBG@Z 120b8b30 f   DOMDocumentFragmentImpl.obj
 0001:000b7b30       ?getInterface@DOMProcessingInstructionImpl@xercesc_2_3@@UAEPAVDOMNode@2@PBG@Z 120b8b30 f   DOMDocumentFragmentImpl.obj
 0001:000b7b30       ?getInterface@DOMCDATASectionImpl@xercesc_2_3@@UAEPAVDOMNode@2@PBG@Z 120b8b30 f   DOMDocumentFragmentImpl.obj
 0001:000b7b30       ?setTextContent@DOMDocumentImpl@xercesc_2_3@@UAEXPBG@Z 120b8b30 f   DOMDocumentFragmentImpl.obj
 0001:000b7b30       ?setTextContent@DOMCDATASectionImpl@xercesc_2_3@@UAEXPBG@Z 120b8b30 f   DOMDocumentFragmentImpl.obj
 0001:000b7b30       ?getInterface@DOMNotationImpl@xercesc_2_3@@UAEPAVDOMNode@2@PBG@Z 120b8b30 f   DOMDocumentFragmentImpl.obj
 0001:000b7b30       ?getInterface@DOMElementImpl@xercesc_2_3@@UAEPAVDOMNode@2@PBG@Z 120b8b30 f   DOMDocumentFragmentImpl.obj
 0001:000b7b30       ?getInterface@DOMEntityImpl@xercesc_2_3@@UAEPAVDOMNode@2@PBG@Z 120b8b30 f   DOMDocumentFragmentImpl.obj
 0001:000b7b30       ?setTextContent@DOMDocumentTypeImpl@xercesc_2_3@@UAEXPBG@Z 120b8b30 f   DOMDocumentFragmentImpl.obj
 0001:000b7b30       ?getInterface@DOMEntityReferenceImpl@xercesc_2_3@@UAEPAVDOMNode@2@PBG@Z 120b8b30 f   DOMDocumentFragmentImpl.obj
 0001:000b7b40       ??0DOMNodeFilter@xercesc_2_3@@IAE@XZ 120b8b40 f i DOMDocumentImpl.obj
 0001:000b7b50       ??1DOMNodeFilter@xercesc_2_3@@UAE@XZ 120b8b50 f i DOMDocumentImpl.obj
 0001:000b7b50       ??1DOMWriterFilter@xercesc_2_3@@UAE@XZ 120b8b50 f i DOMDocumentImpl.obj
 0001:000b7b60       ??_EDOMNodeFilter@xercesc_2_3@@UAEPAXI@Z 120b8b60 f i DOMDocumentImpl.obj
 0001:000b7bc0       ??0DOMTreeWalker@xercesc_2_3@@IAE@XZ 120b8bc0 f i DOMDocumentImpl.obj
 0001:000b7bd0       ??_EDOMTreeWalker@xercesc_2_3@@UAEPAXI@Z 120b8bd0 f i DOMDocumentImpl.obj
 0001:000b7c30       ??1DOMTreeWalker@xercesc_2_3@@UAE@XZ 120b8c30 f i DOMDocumentImpl.obj
 0001:000b7c30       ??1DOMTreeWalkerImpl@xercesc_2_3@@UAE@XZ 120b8c30 f i DOMDocumentImpl.obj
 0001:000b7c40       ??0DOMNodeIterator@xercesc_2_3@@IAE@XZ 120b8c40 f i DOMDocumentImpl.obj
 0001:000b7c50       ??1DOMNodeIterator@xercesc_2_3@@UAE@XZ 120b8c50 f i DOMDocumentImpl.obj
 0001:000b7c60       ??_EDOMNodeIterator@xercesc_2_3@@UAEPAXI@Z 120b8c60 f i DOMDocumentImpl.obj
 0001:000b7cc0       ??0DOMDocumentImpl@xercesc_2_3@@QAE@QAVMemoryManager@1@@Z 120b8cc0 f   DOMDocumentImpl.obj
 0001:000b7dd0       ??_EDOMDocumentImpl@xercesc_2_3@@UAEPAXI@Z 120b8dd0 f i DOMDocumentImpl.obj
 0001:000b7e30       ??0DOMDocumentImpl@xercesc_2_3@@QAE@PBG0PAVDOMDocumentType@1@QAVMemoryManager@1@@Z 120b8e30 f   DOMDocumentImpl.obj
 0001:000b8080       ?setDocumentType@DOMDocumentImpl@xercesc_2_3@@QAEXPAVDOMDocumentType@2@@Z 120b9080 f   DOMDocumentImpl.obj
 0001:000b80e0       ??1DOMDocumentImpl@xercesc_2_3@@UAE@XZ 120b90e0 f   DOMDocumentImpl.obj
 0001:000b82a0       ?cloneNode@DOMDocumentImpl@xercesc_2_3@@UBEPAVDOMNode@2@_N@Z 120b92a0 f   DOMDocumentImpl.obj
 0001:000b8390       ?getNodeName@DOMDocumentImpl@xercesc_2_3@@UBEPBGXZ 120b9390 f   DOMDocumentImpl.obj
 0001:000b83a0       ?getNodeType@DOMDocumentImpl@xercesc_2_3@@UBEFXZ 120b93a0 f   DOMDocumentImpl.obj
 0001:000b83a0       ?getNodeType@DocumentImpl@xercesc_2_3@@UAEFXZ 120b93a0 f   DOMDocumentImpl.obj
 0001:000b83b0       ?getOwnerDocument@DOMDocumentImpl@xercesc_2_3@@UBEPAVDOMDocument@2@XZ 120b93b0 f   DOMDocumentImpl.obj
 0001:000b83b0       ?getEntityDeclPool@WFXMLScanner@xercesc_2_3@@UAEPAV?$NameIdPool@VDTDEntityDecl@xercesc_2_3@@@2@XZ 120b93b0 f   DOMDocumentImpl.obj
 0001:000b83b0       ?getEntityDeclPool@SGXMLScanner@xercesc_2_3@@UBEPBV?$NameIdPool@VDTDEntityDecl@xercesc_2_3@@@2@XZ 120b93b0 f   DOMDocumentImpl.obj
 0001:000b83b0       ?getNextSibling@NodeImpl@xercesc_2_3@@UAEPAV12@XZ 120b93b0 f   DOMDocumentImpl.obj
 0001:000b83b0       ?getPrefix@DOMNodeImpl@xercesc_2_3@@QBEPBGXZ 120b93b0 f   DOMDocumentImpl.obj
 0001:000b83b0       ?getEnumString@AnySimpleTypeDatatypeValidator@xercesc_2_3@@UBEPBV?$RefArrayVectorOf@G@2@XZ 120b93b0 f   DOMDocumentImpl.obj
 0001:000b83b0       ?getOwnerDocument@DocumentImpl@xercesc_2_3@@UAEPAV12@XZ 120b93b0 f   DOMDocumentImpl.obj
 0001:000b83b0       ?getEntityDeclPool@WFXMLScanner@xercesc_2_3@@UBEPBV?$NameIdPool@VDTDEntityDecl@xercesc_2_3@@@2@XZ 120b93b0 f   DOMDocumentImpl.obj
 0001:000b83b0       ?getLastChild@DOMNodeImpl@xercesc_2_3@@QBEPAVDOMNode@2@XZ 120b93b0 f   DOMDocumentImpl.obj
 0001:000b83b0       ?getSign@XMLDateTime@xercesc_2_3@@UBEHXZ 120b93b0 f   DOMDocumentImpl.obj
 0001:000b83b0       ?getLocalName@DOMNodeImpl@xercesc_2_3@@QBEPBGXZ 120b93b0 f   DOMDocumentImpl.obj
 0001:000b83b0       ?getNextSibling@DOMNodeImpl@xercesc_2_3@@QBEPAVDOMNode@2@XZ 120b93b0 f   DOMDocumentImpl.obj
 0001:000b83b0       ?getParentNode@NotationImpl@xercesc_2_3@@UAEPAVNodeImpl@2@XZ 120b93b0 f   DOMDocumentImpl.obj
 0001:000b83b0       ?getLastChild@NodeImpl@xercesc_2_3@@UAEPAV12@XZ 120b93b0 f   DOMDocumentImpl.obj
 0001:000b83b0       ?getFirstChild@DOMNodeImpl@xercesc_2_3@@QBEPAVDOMNode@2@XZ 120b93b0 f   DOMDocumentImpl.obj
 0001:000b83b0       ?getNodeValue@DOMNodeImpl@xercesc_2_3@@QBEPBGXZ 120b93b0 f   DOMDocumentImpl.obj
 0001:000b83b0       ?getEnumString@BooleanDatatypeValidator@xercesc_2_3@@UBEPBV?$RefArrayVectorOf@G@2@XZ 120b93b0 f   DOMDocumentImpl.obj
 0001:000b83b0       ?getPreviousSibling@NodeImpl@xercesc_2_3@@UAEPAV12@XZ 120b93b0 f   DOMDocumentImpl.obj
 0001:000b83b0       ?getParentNode@DOMNodeImpl@xercesc_2_3@@QBEPAVDOMNode@2@XZ 120b93b0 f   DOMDocumentImpl.obj
 0001:000b83b0       ?processBacksolidus_I@RegxParser@xercesc_2_3@@MAEPAVToken@2@XZ 120b93b0 f   DOMDocumentImpl.obj
 0001:000b83b0       ?getFirstChild@NodeImpl@xercesc_2_3@@UAEPAV12@XZ 120b93b0 f   DOMDocumentImpl.obj
 0001:000b83b0       ?getNamespaceURI@DOMNodeImpl@xercesc_2_3@@QBEPBGXZ 120b93b0 f   DOMDocumentImpl.obj
 0001:000b83b0       ?getLength@NodeImpl@xercesc_2_3@@UAEIXZ 120b93b0 f   DOMDocumentImpl.obj
 0001:000b83b0       ?getEntityDeclPool@SGXMLScanner@xercesc_2_3@@UAEPAV?$NameIdPool@VDTDEntityDecl@xercesc_2_3@@@2@XZ 120b93b0 f   DOMDocumentImpl.obj
 0001:000b83b0       ?getAttributes@DOMNodeImpl@xercesc_2_3@@QBEPAVDOMNamedNodeMap@2@XZ 120b93b0 f   DOMDocumentImpl.obj
 0001:000b83b0       ?getAttributes@NodeImpl@xercesc_2_3@@UAEPAVNamedNodeMapImpl@2@XZ 120b93b0 f   DOMDocumentImpl.obj
 0001:000b83b0       ?getParentNode@NodeImpl@xercesc_2_3@@UAEPAV12@XZ 120b93b0 f   DOMDocumentImpl.obj
 0001:000b83b0       ?processBacksolidus_C@RegxParser@xercesc_2_3@@MAEPAVToken@2@XZ 120b93b0 f   DOMDocumentImpl.obj
 0001:000b83b0       ?getPreviousSibling@DOMNodeImpl@xercesc_2_3@@QBEPAVDOMNode@2@XZ 120b93b0 f   DOMDocumentImpl.obj
 0001:000b83b0       ?getContentLeafNameTypeVector@SimpleContentModel@xercesc_2_3@@UBEPAVContentLeafNameTypeVector@2@XZ 120b93b0 f   DOMDocumentImpl.obj
 0001:000b83c0       ?createAttribute@DOMDocumentImpl@xercesc_2_3@@UAEPAVDOMAttr@2@PBG@Z 120b93c0 f   DOMDocumentImpl.obj
 0001:000b8640       ?createCDATASection@DOMDocumentImpl@xercesc_2_3@@UAEPAVDOMCDATASection@2@PBG@Z 120b9640 f   DOMDocumentImpl.obj
 0001:000b8800       ?createComment@DOMDocumentImpl@xercesc_2_3@@UAEPAVDOMComment@2@PBG@Z 120b9800 f   DOMDocumentImpl.obj
 0001:000b89c0       ?createDocumentFragment@DOMDocumentImpl@xercesc_2_3@@UAEPAVDOMDocumentFragment@2@XZ 120b99c0 f   DOMDocumentImpl.obj
 0001:000b8b70       ?createDocumentType@DOMDocumentImpl@xercesc_2_3@@UAEPAVDOMDocumentType@2@PBG@Z 120b9b70 f   DOMDocumentImpl.obj
 0001:000b8df0       ?createDocumentType@DOMDocumentImpl@xercesc_2_3@@UAEPAVDOMDocumentType@2@PBG00@Z 120b9df0 f   DOMDocumentImpl.obj
 0001:000b9080       ?createElement@DOMDocumentImpl@xercesc_2_3@@UAEPAVDOMElement@2@PBG@Z 120ba080 f   DOMDocumentImpl.obj
 0001:000b9300       ?createElementNoCheck@DOMDocumentImpl@xercesc_2_3@@UAEPAVDOMElement@2@PBG@Z 120ba300 f   DOMDocumentImpl.obj
 0001:000b94c0       ?createEntity@DOMDocumentImpl@xercesc_2_3@@UAEPAVDOMEntity@2@PBG@Z 120ba4c0 f   DOMDocumentImpl.obj
 0001:000b9740       ?createEntityReference@DOMDocumentImpl@xercesc_2_3@@UAEPAVDOMEntityReference@2@PBG@Z 120ba740 f   DOMDocumentImpl.obj
 0001:000b99c0       ?createEntityReferenceByParser@DOMDocumentImpl@xercesc_2_3@@QAEPAVDOMEntityReference@2@PBG@Z 120ba9c0 f   DOMDocumentImpl.obj
 0001:000b9c40       ?createNotation@DOMDocumentImpl@xercesc_2_3@@UAEPAVDOMNotation@2@PBG@Z 120bac40 f   DOMDocumentImpl.obj
 0001:000b9ec0       ?createProcessingInstruction@DOMDocumentImpl@xercesc_2_3@@UAEPAVDOMProcessingInstruction@2@PBG0@Z 120baec0 f   DOMDocumentImpl.obj
 0001:000ba140       ?createTextNode@DOMDocumentImpl@xercesc_2_3@@UAEPAVDOMText@2@PBG@Z 120bb140 f   DOMDocumentImpl.obj
 0001:000ba300       ?createNodeIterator@DOMDocumentImpl@xercesc_2_3@@UAEPAVDOMNodeIterator@2@PAVDOMNode@2@KPAVDOMNodeFilter@2@_N@Z 120bb300 f   DOMDocumentImpl.obj
 0001:000ba470       ?getNodeIterators@DOMDocumentImpl@xercesc_2_3@@UBEPAV?$RefVectorOf@VDOMNodeIteratorImpl@xercesc_2_3@@@2@XZ 120bb470 f   DOMDocumentImpl.obj
 0001:000ba480       ?removeNodeIterator@DOMDocumentImpl@xercesc_2_3@@UAEXPAVDOMNodeIteratorImpl@2@@Z 120bb480 f   DOMDocumentImpl.obj
 0001:000ba590       ?createTreeWalker@DOMDocumentImpl@xercesc_2_3@@UAEPAVDOMTreeWalker@2@PAVDOMNode@2@KPAVDOMNodeFilter@2@_N@Z 120bb590 f   DOMDocumentImpl.obj
 0001:000ba630       ?getDoctype@DOMDocumentImpl@xercesc_2_3@@UBEPAVDOMDocumentType@2@XZ 120bb630 f   DOMDocumentImpl.obj
 0001:000ba640       ?getDocumentElement@DOMDocumentImpl@xercesc_2_3@@UBEPAVDOMElement@2@XZ 120bb640 f   DOMDocumentImpl.obj
 0001:000ba650       ?getElementsByTagName@DOMDocumentImpl@xercesc_2_3@@UBEPAVDOMNodeList@2@PBG@Z 120bb650 f   DOMDocumentImpl.obj
 0001:000ba680       ?getImplementation@DOMDocumentImpl@xercesc_2_3@@UBEPAVDOMImplementation@2@XZ 120bb680 f   DOMDocumentImpl.obj
 0001:000ba690       ?insertBefore@DOMDocumentImpl@xercesc_2_3@@UAEPAVDOMNode@2@PAV32@0@Z 120bb690 f   DOMDocumentImpl.obj
 0001:000ba750       ?replaceChild@DOMDocumentImpl@xercesc_2_3@@UAEPAVDOMNode@2@PAV32@0@Z 120bb750 f   DOMDocumentImpl.obj
 0001:000ba830       ?isXMLName@DOMDocumentImpl@xercesc_2_3@@QAE_NPBG@Z 120bb830 f   DOMDocumentImpl.obj
 0001:000ba910       ?removeChild@DOMDocumentImpl@xercesc_2_3@@UAEPAVDOMNode@2@PAV32@@Z 120bb910 f   DOMDocumentImpl.obj
 0001:000ba960       ?setNodeValue@DOMDocumentImpl@xercesc_2_3@@UAEXPBG@Z 120bb960 f   DOMDocumentImpl.obj
 0001:000ba960       ?setNodeValue@DOMEntityImpl@xercesc_2_3@@UAEXPBG@Z 120bb960 f   DOMDocumentImpl.obj
 0001:000ba960       ?setNodeValue@DOMEntityReferenceImpl@xercesc_2_3@@UAEXPBG@Z 120bb960 f   DOMDocumentImpl.obj
 0001:000ba960       ?setNodeValue@DOMNotationImpl@xercesc_2_3@@UAEXPBG@Z 120bb960 f   DOMDocumentImpl.obj
 0001:000ba960       ?setNodeValue@DOMDocumentTypeImpl@xercesc_2_3@@UAEXPBG@Z 120bb960 f   DOMDocumentImpl.obj
 0001:000ba960       ?setNodeValue@DOMDocumentFragmentImpl@xercesc_2_3@@UAEXPBG@Z 120bb960 f   DOMDocumentImpl.obj
 0001:000ba960       ?setNodeValue@DOMElementImpl@xercesc_2_3@@UAEXPBG@Z 120bb960 f   DOMDocumentImpl.obj
 0001:000ba970       ?importNode@DOMDocumentImpl@xercesc_2_3@@UAEPAVDOMNode@2@PAV32@_N@Z 120bb970 f   DOMDocumentImpl.obj
 0001:000ba990       ?createElementNS@DOMDocumentImpl@xercesc_2_3@@UAEPAVDOMElement@2@PBG0@Z 120bb990 f   DOMDocumentImpl.obj
 0001:000bac10       ?createElementNS@DOMDocumentImpl@xercesc_2_3@@UAEPAVDOMElement@2@PBG0JJ@Z 120bbc10 f   DOMDocumentImpl.obj
 0001:000bad60       ?createAttributeNS@DOMDocumentImpl@xercesc_2_3@@UAEPAVDOMAttr@2@PBG0@Z 120bbd60 f   DOMDocumentImpl.obj
 0001:000bafe0       ?getElementsByTagNameNS@DOMDocumentImpl@xercesc_2_3@@UBEPAVDOMNodeList@2@PBG0@Z 120bbfe0 f   DOMDocumentImpl.obj
 0001:000bb010       ?getElementById@DOMDocumentImpl@xercesc_2_3@@UBEPAVDOMElement@2@PBG@Z 120bc010 f   DOMDocumentImpl.obj
 0001:000bb040       ?indexofQualifiedName@DOMDocumentImpl@xercesc_2_3@@SAHPBG@Z 120bc040 f   DOMDocumentImpl.obj
 0001:000bb0b0       ?createRange@DOMDocumentImpl@xercesc_2_3@@UAEPAVDOMRange@2@XZ 120bc0b0 f   DOMDocumentImpl.obj
 0001:000bb1f0       ?getRanges@DOMDocumentImpl@xercesc_2_3@@UBEPAV?$RefVectorOf@VDOMRangeImpl@xercesc_2_3@@@2@XZ 120bc1f0 f   DOMDocumentImpl.obj
 0001:000bb200       ?removeRange@DOMDocumentImpl@xercesc_2_3@@UAEXPAVDOMRangeImpl@2@@Z 120bc200 f   DOMDocumentImpl.obj
 0001:000bb310       ?isKidOK@DOMDocumentImpl@xercesc_2_3@@SA_NPAVDOMNode@2@0@Z 120bc310 f   DOMDocumentImpl.obj
 0001:000bb3a0       ?changed@DOMDocumentImpl@xercesc_2_3@@UAEXXZ 120bc3a0 f   DOMDocumentImpl.obj
 0001:000bb3b0       ?changes@DOMDocumentImpl@xercesc_2_3@@UBEHXZ 120bc3b0 f   DOMDocumentImpl.obj
 0001:000bb3c0       ?appendChild@DOMDocumentImpl@xercesc_2_3@@UAEPAVDOMNode@2@PAV32@@Z 120bc3c0 f   DOMDocumentImpl.obj
 0001:000bb3c0       ?validate@DateTimeValidator@xercesc_2_3@@UAEXQBG@Z 120bc3c0 f   DOMDocumentImpl.obj
 0001:000bb3c0       ?validate@AbstractNumericValidator@xercesc_2_3@@UAEXQBG@Z 120bc3c0 f   DOMDocumentImpl.obj
 0001:000bb3d0       ?getPrefix@DOMElementImpl@xercesc_2_3@@UBEPBGXZ 120bc3d0 f   DOMDocumentImpl.obj
 0001:000bb3d0       ?getAttributes@DOMDocumentFragmentImpl@xercesc_2_3@@UBEPAVDOMNamedNodeMap@2@XZ 120bc3d0 f   DOMDocumentImpl.obj
 0001:000bb3d0       ?getNodeValue@DOMElementImpl@xercesc_2_3@@UBEPBGXZ 120bc3d0 f   DOMDocumentImpl.obj
 0001:000bb3d0       ?getPreviousSibling@DOMAttrImpl@xercesc_2_3@@UBEPAVDOMNode@2@XZ 120bc3d0 f   DOMDocumentImpl.obj
 0001:000bb3d0       ?getParentNode@DOMDocumentImpl@xercesc_2_3@@UBEPAVDOMNode@2@XZ 120bc3d0 f   DOMDocumentImpl.obj
 0001:000bb3d0       ?getPrefix@DOMProcessingInstructionImpl@xercesc_2_3@@UBEPBGXZ 120bc3d0 f   DOMDocumentImpl.obj
 0001:000bb3d0       ?getPrefix@DOMNotationImpl@xercesc_2_3@@UBEPBGXZ 120bc3d0 f   DOMDocumentImpl.obj
 0001:000bb3d0       ?getNextSibling@DOMNotationImpl@xercesc_2_3@@UBEPAVDOMNode@2@XZ 120bc3d0 f   DOMDocumentImpl.obj
 0001:000bb3d0       ?getParentNode@DOMEntityImpl@xercesc_2_3@@UBEPAVDOMNode@2@XZ 120bc3d0 f   DOMDocumentImpl.obj
 0001:000bb3d0       ?getPrefix@DOMEntityImpl@xercesc_2_3@@UBEPBGXZ 120bc3d0 f   DOMDocumentImpl.obj
 0001:000bb3d0       ?getNamespaceURI@DOMCommentImpl@xercesc_2_3@@UBEPBGXZ 120bc3d0 f   DOMDocumentImpl.obj
 0001:000bb3d0       ?getLocalName@DOMProcessingInstructionImpl@xercesc_2_3@@UBEPBGXZ 120bc3d0 f   DOMDocumentImpl.obj
 0001:000bb3d0       ?getNodeValue@DOMEntityReferenceImpl@xercesc_2_3@@UBEPBGXZ 120bc3d0 f   DOMDocumentImpl.obj
 0001:000bb3d0       ?getAttributes@DOMDocumentTypeImpl@xercesc_2_3@@UBEPAVDOMNamedNodeMap@2@XZ 120bc3d0 f   DOMDocumentImpl.obj
 0001:000bb3d0       ?getLastChild@DOMTextImpl@xercesc_2_3@@UBEPAVDOMNode@2@XZ 120bc3d0 f   DOMDocumentImpl.obj
 0001:000bb3d0       ?getAttributes@DOMCDATASectionImpl@xercesc_2_3@@UBEPAVDOMNamedNodeMap@2@XZ 120bc3d0 f   DOMDocumentImpl.obj
 0001:000bb3d0       ?getNamespaceURI@DOMDocumentFragmentImpl@xercesc_2_3@@UBEPBGXZ 120bc3d0 f   DOMDocumentImpl.obj
 0001:000bb3d0       ?getNamespaceURI@DOMProcessingInstructionImpl@xercesc_2_3@@UBEPBGXZ 120bc3d0 f   DOMDocumentImpl.obj
 0001:000bb3d0       ?getAttributes@DOMAttrImpl@xercesc_2_3@@UBEPAVDOMNamedNodeMap@2@XZ 120bc3d0 f   DOMDocumentImpl.obj
 0001:000bb3d0       ?getNamespaceURI@DOMNotationImpl@xercesc_2_3@@UBEPBGXZ 120bc3d0 f   DOMDocumentImpl.obj
 0001:000bb3d0       ?getPrefix@DOMEntityReferenceImpl@xercesc_2_3@@UBEPBGXZ 120bc3d0 f   DOMDocumentImpl.obj
 0001:000bb3d0       ?getAttributes@DOMTextImpl@xercesc_2_3@@UBEPAVDOMNamedNodeMap@2@XZ 120bc3d0 f   DOMDocumentImpl.obj
 0001:000bb3d0       ?getNamespaceURI@DOMEntityReferenceImpl@xercesc_2_3@@UBEPBGXZ 120bc3d0 f   DOMDocumentImpl.obj
 0001:000bb3d0       ?getNextSibling@DOMDocumentImpl@xercesc_2_3@@UBEPAVDOMNode@2@XZ 120bc3d0 f   DOMDocumentImpl.obj
 0001:000bb3d0       ?getPrefix@DOMAttrImpl@xercesc_2_3@@UBEPBGXZ 120bc3d0 f   DOMDocumentImpl.obj
 0001:000bb3d0       ?getPreviousSibling@DOMEntityImpl@xercesc_2_3@@UBEPAVDOMNode@2@XZ 120bc3d0 f   DOMDocumentImpl.obj
 0001:000bb3d0       ?getNamespaceURI@DOMCDATASectionImpl@xercesc_2_3@@UBEPBGXZ 120bc3d0 f   DOMDocumentImpl.obj
 0001:000bb3d0       ?getPrefix@DOMDocumentFragmentImpl@xercesc_2_3@@UBEPBGXZ 120bc3d0 f   DOMDocumentImpl.obj
 0001:000bb3d0       ?getParentNode@DOMNotationImpl@xercesc_2_3@@UBEPAVDOMNode@2@XZ 120bc3d0 f   DOMDocumentImpl.obj
 0001:000bb3d0       ?getNodeValue@DOMDocumentFragmentImpl@xercesc_2_3@@UBEPBGXZ 120bc3d0 f   DOMDocumentImpl.obj
 0001:000bb3d0       ?getLocalName@DOMEntityImpl@xercesc_2_3@@UBEPBGXZ 120bc3d0 f   DOMDocumentImpl.obj
 0001:000bb3d0       ?getNodeValue@DOMDocumentImpl@xercesc_2_3@@UBEPBGXZ 120bc3d0 f   DOMDocumentImpl.obj
 0001:000bb3d0       ?getNodeValue@DOMEntityImpl@xercesc_2_3@@UBEPBGXZ 120bc3d0 f   DOMDocumentImpl.obj
 0001:000bb3d0       ?getNodeValue@DOMDocumentTypeImpl@xercesc_2_3@@UBEPBGXZ 120bc3d0 f   DOMDocumentImpl.obj
 0001:000bb3d0       ?getLocalName@DOMAttrImpl@xercesc_2_3@@UBEPBGXZ 120bc3d0 f   DOMDocumentImpl.obj
 0001:000bb3d0       ?getNextSibling@DOMEntityImpl@xercesc_2_3@@UBEPAVDOMNode@2@XZ 120bc3d0 f   DOMDocumentImpl.obj
 0001:000bb3d0       ?getNamespaceURI@DOMAttrImpl@xercesc_2_3@@UBEPBGXZ 120bc3d0 f   DOMDocumentImpl.obj
 0001:000bb3d0       ?getLocalName@DOMCDATASectionImpl@xercesc_2_3@@UBEPBGXZ 120bc3d0 f   DOMDocumentImpl.obj
 0001:000bb3d0       ?getNextSibling@DOMAttrImpl@xercesc_2_3@@UBEPAVDOMNode@2@XZ 120bc3d0 f   DOMDocumentImpl.obj
 0001:000bb3d0       ?getAttributes@DOMEntityReferenceImpl@xercesc_2_3@@UBEPAVDOMNamedNodeMap@2@XZ 120bc3d0 f   DOMDocumentImpl.obj
 0001:000bb3d0       ?getNamespaceURI@DOMElementImpl@xercesc_2_3@@UBEPBGXZ 120bc3d0 f   DOMDocumentImpl.obj
 0001:000bb3d0       ?getPreviousSibling@DOMNotationImpl@xercesc_2_3@@UBEPAVDOMNode@2@XZ 120bc3d0 f   DOMDocumentImpl.obj
 0001:000bb3d0       ?getAttributes@DOMProcessingInstructionImpl@xercesc_2_3@@UBEPAVDOMNamedNodeMap@2@XZ 120bc3d0 f   DOMDocumentImpl.obj
 0001:000bb3d0       ?getPrefix@DOMDocumentImpl@xercesc_2_3@@UBEPBGXZ 120bc3d0 f   DOMDocumentImpl.obj
 0001:000bb3d0       ?getFirstChild@DOMProcessingInstructionImpl@xercesc_2_3@@UBEPAVDOMNode@2@XZ 120bc3d0 f   DOMDocumentImpl.obj
 0001:000bb3d0       ?getLastChild@DOMCommentImpl@xercesc_2_3@@UBEPAVDOMNode@2@XZ 120bc3d0 f   DOMDocumentImpl.obj
 0001:000bb3d0       ?getNamespaceURI@DOMTextImpl@xercesc_2_3@@UBEPBGXZ 120bc3d0 f   DOMDocumentImpl.obj
 0001:000bb3d0       ?getPreviousSibling@DOMDocumentFragmentImpl@xercesc_2_3@@UBEPAVDOMNode@2@XZ 120bc3d0 f   DOMDocumentImpl.obj
 0001:000bb3d0       ?getNamespaceURI@DOMDocumentTypeImpl@xercesc_2_3@@UBEPBGXZ 120bc3d0 f   DOMDocumentImpl.obj
 0001:000bb3d0       ?getFirstChild@DOMNotationImpl@xercesc_2_3@@UBEPAVDOMNode@2@XZ 120bc3d0 f   DOMDocumentImpl.obj
 0001:000bb3d0       ?getLocalName@DOMElementImpl@xercesc_2_3@@UBEPBGXZ 120bc3d0 f   DOMDocumentImpl.obj
 0001:000bb3d0       ?getPrefix@DOMCommentImpl@xercesc_2_3@@UBEPBGXZ 120bc3d0 f   DOMDocumentImpl.obj
 0001:000bb3d0       ?getLocalName@DOMCommentImpl@xercesc_2_3@@UBEPBGXZ 120bc3d0 f   DOMDocumentImpl.obj
 0001:000bb3d0       ?getLocalName@DOMNotationImpl@xercesc_2_3@@UBEPBGXZ 120bc3d0 f   DOMDocumentImpl.obj
 0001:000bb3d0       ?getPreviousSibling@DOMDocumentImpl@xercesc_2_3@@UBEPAVDOMNode@2@XZ 120bc3d0 f   DOMDocumentImpl.obj
 0001:000bb3d0       ?getAttributes@DOMEntityImpl@xercesc_2_3@@UBEPAVDOMNamedNodeMap@2@XZ 120bc3d0 f   DOMDocumentImpl.obj
 0001:000bb3d0       ?getFirstChild@DOMCommentImpl@xercesc_2_3@@UBEPAVDOMNode@2@XZ 120bc3d0 f   DOMDocumentImpl.obj
 0001:000bb3d0       ?getNamespaceURI@DOMDocumentImpl@xercesc_2_3@@UBEPBGXZ 120bc3d0 f   DOMDocumentImpl.obj
 0001:000bb3d0       ?getPrefix@DOMDocumentTypeImpl@xercesc_2_3@@UBEPBGXZ 120bc3d0 f   DOMDocumentImpl.obj
 0001:000bb3d0       ?getFirstChild@DOMTextImpl@xercesc_2_3@@UBEPAVDOMNode@2@XZ 120bc3d0 f   DOMDocumentImpl.obj
 0001:000bb3d0       ?getLastChild@DOMProcessingInstructionImpl@xercesc_2_3@@UBEPAVDOMNode@2@XZ 120bc3d0 f   DOMDocumentImpl.obj
 0001:000bb3d0       ?getAttributes@DOMNotationImpl@xercesc_2_3@@UBEPAVDOMNamedNodeMap@2@XZ 120bc3d0 f   DOMDocumentImpl.obj
 0001:000bb3d0       ?getNamespaceURI@DOMEntityImpl@xercesc_2_3@@UBEPBGXZ 120bc3d0 f   DOMDocumentImpl.obj
 0001:000bb3d0       ?getLocalName@DOMEntityReferenceImpl@xercesc_2_3@@UBEPBGXZ 120bc3d0 f   DOMDocumentImpl.obj
 0001:000bb3d0       ?getNextSibling@DOMDocumentFragmentImpl@xercesc_2_3@@UBEPAVDOMNode@2@XZ 120bc3d0 f   DOMDocumentImpl.obj
 0001:000bb3d0       ?getNodeValue@DOMNotationImpl@xercesc_2_3@@UBEPBGXZ 120bc3d0 f   DOMDocumentImpl.obj
 0001:000bb3d0       ?getLocalName@DOMDocumentFragmentImpl@xercesc_2_3@@UBEPBGXZ 120bc3d0 f   DOMDocumentImpl.obj
 0001:000bb3d0       ?getLastChild@DOMNotationImpl@xercesc_2_3@@UBEPAVDOMNode@2@XZ 120bc3d0 f   DOMDocumentImpl.obj
 0001:000bb3d0       ?getAttributes@DOMCommentImpl@xercesc_2_3@@UBEPAVDOMNamedNodeMap@2@XZ 120bc3d0 f   DOMDocumentImpl.obj
 0001:000bb3d0       ?getAttributes@DOMDocumentImpl@xercesc_2_3@@UBEPAVDOMNamedNodeMap@2@XZ 120bc3d0 f   DOMDocumentImpl.obj
 0001:000bb3d0       ?getParentNode@DOMDocumentFragmentImpl@xercesc_2_3@@UBEPAVDOMNode@2@XZ 120bc3d0 f   DOMDocumentImpl.obj
 0001:000bb3d0       ?getLocalName@DOMDocumentImpl@xercesc_2_3@@UBEPBGXZ 120bc3d0 f   DOMDocumentImpl.obj
 0001:000bb3d0       ?getPrefix@DOMCDATASectionImpl@xercesc_2_3@@UBEPBGXZ 120bc3d0 f   DOMDocumentImpl.obj
 0001:000bb3d0       ?getParentNode@DOMAttrImpl@xercesc_2_3@@UBEPAVDOMNode@2@XZ 120bc3d0 f   DOMDocumentImpl.obj
 0001:000bb3d0       ?getPrefix@DOMTextImpl@xercesc_2_3@@UBEPBGXZ 120bc3d0 f   DOMDocumentImpl.obj
 0001:000bb3d0       ?getLocalName@DOMDocumentTypeImpl@xercesc_2_3@@UBEPBGXZ 120bc3d0 f   DOMDocumentImpl.obj
 0001:000bb3d0       ?getLocalName@DOMTextImpl@xercesc_2_3@@UBEPBGXZ 120bc3d0 f   DOMDocumentImpl.obj
 0001:000bb3e0       ?getChildNodes@DOMDocumentFragmentImpl@xercesc_2_3@@UBEPAVDOMNodeList@2@XZ 120bc3e0 f   DOMDocumentImpl.obj
 0001:000bb3e0       ?getChildNodes@DOMDocumentTypeImpl@xercesc_2_3@@UBEPAVDOMNodeList@2@XZ 120bc3e0 f   DOMDocumentImpl.obj
 0001:000bb3e0       ?getChildNodes@DOMDocumentImpl@xercesc_2_3@@UBEPAVDOMNodeList@2@XZ 120bc3e0 f   DOMDocumentImpl.obj
 0001:000bb3e0       ?getChildNodes@DOMElementImpl@xercesc_2_3@@UBEPAVDOMNodeList@2@XZ 120bc3e0 f   DOMDocumentImpl.obj
 0001:000bb3e0       ?getChildNodes@DOMCDATASectionImpl@xercesc_2_3@@UBEPAVDOMNodeList@2@XZ 120bc3e0 f   DOMDocumentImpl.obj
 0001:000bb3e0       ?getChildNodes@DOMEntityReferenceImpl@xercesc_2_3@@UBEPAVDOMNodeList@2@XZ 120bc3e0 f   DOMDocumentImpl.obj
 0001:000bb3e0       ?getChildNodes@DOMAttrImpl@xercesc_2_3@@UBEPAVDOMNodeList@2@XZ 120bc3e0 f   DOMDocumentImpl.obj
 0001:000bb3f0       ?getNextSibling@DOMProcessingInstructionImpl@xercesc_2_3@@UBEPAVDOMNode@2@XZ 120bc3f0 f   DOMDocumentImpl.obj
 0001:000bb3f0       ?getFirstChild@DOMEntityReferenceImpl@xercesc_2_3@@UBEPAVDOMNode@2@XZ 120bc3f0 f   DOMDocumentImpl.obj
 0001:000bb3f0       ?getFirstChild@DOMElementImpl@xercesc_2_3@@UBEPAVDOMNode@2@XZ 120bc3f0 f   DOMDocumentImpl.obj
 0001:000bb3f0       ?getNextSibling@DOMTextImpl@xercesc_2_3@@UBEPAVDOMNode@2@XZ 120bc3f0 f   DOMDocumentImpl.obj
 0001:000bb3f0       ?getFirstChild@DOMDocumentImpl@xercesc_2_3@@UBEPAVDOMNode@2@XZ 120bc3f0 f   DOMDocumentImpl.obj
 0001:000bb3f0       ?getFirstChild@DOMAttrImpl@xercesc_2_3@@UBEPAVDOMNode@2@XZ 120bc3f0 f   DOMDocumentImpl.obj
 0001:000bb3f0       ?getFirstChild@DOMDocumentFragmentImpl@xercesc_2_3@@UBEPAVDOMNode@2@XZ 120bc3f0 f   DOMDocumentImpl.obj
 0001:000bb3f0       ?getNextSibling@DOMCommentImpl@xercesc_2_3@@UBEPAVDOMNode@2@XZ 120bc3f0 f   DOMDocumentImpl.obj
 0001:000bb3f0       ?getFirstChild@DOMDocumentTypeImpl@xercesc_2_3@@UBEPAVDOMNode@2@XZ 120bc3f0 f   DOMDocumentImpl.obj
 0001:000bb3f0       ?getFirstChild@DOMCDATASectionImpl@xercesc_2_3@@UBEPAVDOMNode@2@XZ 120bc3f0 f   DOMDocumentImpl.obj
 0001:000bb400       ?getLastChild@DOMCDATASectionImpl@xercesc_2_3@@UBEPAVDOMNode@2@XZ 120bc400 f   DOMDocumentImpl.obj
 0001:000bb400       ?getLastChild@DOMDocumentTypeImpl@xercesc_2_3@@UBEPAVDOMNode@2@XZ 120bc400 f   DOMDocumentImpl.obj
 0001:000bb400       ?getLastChild@DOMDocumentFragmentImpl@xercesc_2_3@@UBEPAVDOMNode@2@XZ 120bc400 f   DOMDocumentImpl.obj
 0001:000bb400       ?getLastChild@DOMElementImpl@xercesc_2_3@@UBEPAVDOMNode@2@XZ 120bc400 f   DOMDocumentImpl.obj
 0001:000bb400       ?getLastChild@DOMDocumentImpl@xercesc_2_3@@UBEPAVDOMNode@2@XZ 120bc400 f   DOMDocumentImpl.obj
 0001:000bb400       ?getLastChild@DOMEntityReferenceImpl@xercesc_2_3@@UBEPAVDOMNode@2@XZ 120bc400 f   DOMDocumentImpl.obj
 0001:000bb400       ?getLastChild@DOMAttrImpl@xercesc_2_3@@UBEPAVDOMNode@2@XZ 120bc400 f   DOMDocumentImpl.obj
 0001:000bb410       ?cloneString@DOMDocumentImpl@xercesc_2_3@@QAEPAGPBG@Z 120bc410 f   DOMDocumentImpl.obj
 0001:000bb470       ?getPooledString@DOMDocumentImpl@xercesc_2_3@@QAEPBGPBG@Z 120bc470 f   DOMDocumentImpl.obj
 0001:000bb490       ?allocate@DOMDocumentImpl@xercesc_2_3@@QAEPAXI@Z 120bc490 f   DOMDocumentImpl.obj
 0001:000bb680       ?deleteHeap@DOMDocumentImpl@xercesc_2_3@@QAEXXZ 120bc680 f   DOMDocumentImpl.obj
 0001:000bb6b0       ?getDeepNodeList@DOMDocumentImpl@xercesc_2_3@@QAEPAVDOMNodeList@2@PBVDOMNode@2@PBG@Z 120bc6b0 f   DOMDocumentImpl.obj
 0001:000bb9c0       ?getDeepNodeList@DOMDocumentImpl@xercesc_2_3@@QAEPAVDOMNodeList@2@PBVDOMNode@2@PBG1@Z 120bc9c0 f   DOMDocumentImpl.obj
 0001:000bbce0       ?getDocument@AbstractDOMParser@xercesc_2_3@@QAEPAVDOMDocument@2@XZ 120bcce0 f   DOMDocumentImpl.obj
 0001:000bbce0       ?getBaseURI@DOMEntityReferenceImpl@xercesc_2_3@@UBEPBGXZ 120bcce0 f   DOMDocumentImpl.obj
 0001:000bbce0       ?getEntities@DOMDocumentTypeImpl@xercesc_2_3@@UBEPAVDOMNamedNodeMap@2@XZ 120bcce0 f   DOMDocumentImpl.obj
 0001:000bbce0       ?getActualEncoding@DOMDocumentImpl@xercesc_2_3@@UBEPBGXZ 120bcce0 f   DOMDocumentImpl.obj
 0001:000bbce0       ?getLocalName@DOMAttrNSImpl@xercesc_2_3@@UBEPBGXZ 120bcce0 f   DOMDocumentImpl.obj
 0001:000bbce0       ?getNotationName@DOMEntityImpl@xercesc_2_3@@UBEPBGXZ 120bcce0 f   DOMDocumentImpl.obj
 0001:000bbce0       ?getDefaultAttributes@DOMElementImpl@xercesc_2_3@@UBEPAVDOMAttrMapImpl@2@XZ 120bcce0 f   DOMDocumentImpl.obj
 0001:000bbcf0       ?setActualEncoding@DOMDocumentImpl@xercesc_2_3@@UAEXPBG@Z 120bccf0 f   DOMDocumentImpl.obj
 0001:000bbd50       ?setEncoding@DOMDocumentImpl@xercesc_2_3@@UAEXPBG@Z 120bcd50 f   DOMDocumentImpl.obj
 0001:000bbdb0       ?getStandalone@DOMDocumentImpl@xercesc_2_3@@UBE_NXZ 120bcdb0 f   DOMDocumentImpl.obj
 0001:000bbdc0       ?setStandalone@DOMDocumentImpl@xercesc_2_3@@UAEX_N@Z 120bcdc0 f   DOMDocumentImpl.obj
 0001:000bbdd0       ?setVersion@DOMDocumentImpl@xercesc_2_3@@UAEXPBG@Z 120bcdd0 f   DOMDocumentImpl.obj
 0001:000bbec0       ?setDocumentURI@DOMDocumentImpl@xercesc_2_3@@UAEXPBG@Z 120bcec0 f   DOMDocumentImpl.obj
 0001:000bbf20       ?getStrictErrorChecking@DOMDocumentImpl@xercesc_2_3@@UBE_NXZ 120bcf20 f   DOMDocumentImpl.obj
 0001:000bbf30       ?setStrictErrorChecking@DOMDocumentImpl@xercesc_2_3@@UAEX_N@Z 120bcf30 f   DOMDocumentImpl.obj
 0001:000bbf40       ?normalizeDocument@DOMDocumentImpl@xercesc_2_3@@UAEXXZ 120bcf40 f   DOMDocumentImpl.obj
 0001:000bbfc0       ?getDOMConfiguration@DOMDocumentImpl@xercesc_2_3@@UBEPAVDOMConfiguration@2@XZ 120bcfc0 f   DOMDocumentImpl.obj
 0001:000bc020       ?setDOMConfiguration@DOMDocumentImpl@xercesc_2_3@@UAEXPAVDOMConfiguration@2@@Z 120bd020 f   DOMDocumentImpl.obj
 0001:000bc030       ?importNode@DOMDocumentImpl@xercesc_2_3@@EAEPAVDOMNode@2@PAV32@_N1@Z 120bd030 f   DOMDocumentImpl.obj
 0001:000bc570       ?setUserData@DOMDocumentImpl@xercesc_2_3@@QAEPAXPAVDOMNodeImpl@2@PBGPAXPAVDOMUserDataHandler@2@@Z 120bd570 f   DOMDocumentImpl.obj
 0001:000bc8e0       ?getUserData@DOMDocumentImpl@xercesc_2_3@@QBEPAXPBVDOMNodeImpl@2@PBG@Z 120bd8e0 f   DOMDocumentImpl.obj
 0001:000bc9e0       ?callUserDataHandlers@DOMDocumentImpl@xercesc_2_3@@QBEXPBVDOMNodeImpl@2@W4DOMOperationType@DOMUserDataHandler@2@PBVDOMNode@2@2@Z 120bd9e0 f   DOMDocumentImpl.obj
 0001:000bcb70       ?transferUserData@DOMDocumentImpl@xercesc_2_3@@QAEXPAVDOMNodeImpl@2@0@Z 120bdb70 f   DOMDocumentImpl.obj
 0001:000bcc70       ?renameNode@DOMDocumentImpl@xercesc_2_3@@UAEPAVDOMNode@2@PAV32@PBG1@Z 120bdc70 f   DOMDocumentImpl.obj
 0001:000bcd30       ?release@DOMDocumentImpl@xercesc_2_3@@UAEXXZ 120bdd30 f   DOMDocumentImpl.obj
 0001:000bcdc0       ?releaseDocNotifyUserData@DOMDocumentImpl@xercesc_2_3@@QAEXPAVDOMNode@2@@Z 120bddc0 f   DOMDocumentImpl.obj
 0001:000bce10       ?release@DOMDocumentImpl@xercesc_2_3@@QAEXPAVDOMNode@2@W4NodeObjectType@12@@Z 120bde10 f   DOMDocumentImpl.obj
 0001:000bd070       ?releaseBuffer@DOMDocumentImpl@xercesc_2_3@@QAEXPAVDOMBuffer@2@@Z 120be070 f   DOMDocumentImpl.obj
 0001:000bd190       ?popBuffer@DOMDocumentImpl@xercesc_2_3@@QAEPAVDOMBuffer@2@XZ 120be190 f   DOMDocumentImpl.obj
 0001:000bd260       ?allocate@DOMDocumentImpl@xercesc_2_3@@QAEPAXIW4NodeObjectType@12@@Z 120be260 f   DOMDocumentImpl.obj
 0001:000bd380       ??1?$XMLEnumerator@V?$KeyRefPair@XVDOMUserDataHandler@xercesc_2_3@@@xercesc_2_3@@@xercesc_2_3@@UAE@XZ 120be380 f i DOMDocumentImpl.obj
 0001:000bd390       ??_E?$XMLEnumerator@V?$KeyRefPair@XVDOMUserDataHandler@xercesc_2_3@@@xercesc_2_3@@@xercesc_2_3@@UAEPAXI@Z 120be390 f i DOMDocumentImpl.obj
 0001:000bd390       ??_G?$XMLEnumerator@V?$KeyRefPair@XVDOMUserDataHandler@xercesc_2_3@@@xercesc_2_3@@@xercesc_2_3@@UAEPAXI@Z 120be390 f i DOMDocumentImpl.obj
 0001:000bd3b0       ?put@?$RefHashTableOf@V?$RefHashTableOf@V?$KeyRefPair@XVDOMUserDataHandler@xercesc_2_3@@@xercesc_2_3@@@xercesc_2_3@@@xercesc_2_3@@QAEXPAXQAV?$RefHashTableOf@V?$KeyRefPair@XVDOMUserDataHandler@xercesc_2_3@@@xercesc_2_3@@@2@@Z 120be3b0 f i DOMDocumentImpl.obj
 0001:000bd5e0       ??A?$RefArrayOf@V?$RefStackOf@VDOMNode@xercesc_2_3@@@xercesc_2_3@@@xercesc_2_3@@QAEAAPAV?$RefStackOf@VDOMNode@xercesc_2_3@@@1@I@Z 120be5e0 f i DOMDocumentImpl.obj
 0001:000bd620       ??1?$RefVectorOf@VDOMBuffer@xercesc_2_3@@@xercesc_2_3@@UAE@XZ 120be620 f i DOMDocumentImpl.obj
 0001:000bd6a0       ??1?$BaseRefVectorOf@VDOMBuffer@xercesc_2_3@@@xercesc_2_3@@UAE@XZ 120be6a0 f i DOMDocumentImpl.obj
 0001:000bd6b0       ?isEmpty@?$RefHash2KeysTableOf@VSchemaAttDef@xercesc_2_3@@@xercesc_2_3@@QBE_NXZ 120be6b0 f i DOMDocumentImpl.obj
 0001:000bd6b0       ?isEmpty@?$RefHashTableOf@V?$KeyRefPair@XVDOMUserDataHandler@xercesc_2_3@@@xercesc_2_3@@@xercesc_2_3@@QBE_NXZ 120be6b0 f i DOMDocumentImpl.obj
 0001:000bd6d0       ??1?$RefHashTableOfEnumerator@V?$KeyRefPair@XVDOMUserDataHandler@xercesc_2_3@@@xercesc_2_3@@@xercesc_2_3@@UAE@XZ 120be6d0 f i DOMDocumentImpl.obj
 0001:000bd7c0       ?hasMoreElements@?$RefHashTableOfEnumerator@VDTDAttDef@xercesc_2_3@@@xercesc_2_3@@UBE_NXZ 120be7c0 f i DOMDocumentImpl.obj
 0001:000bd7c0       ?hasMoreElements@?$RefHashTableOfEnumerator@VXMLRefInfo@xercesc_2_3@@@xercesc_2_3@@UBE_NXZ 120be7c0 f i DOMDocumentImpl.obj
 0001:000bd7c0       ?hasMoreElements@?$RefHashTableOfEnumerator@VComplexTypeInfo@xercesc_2_3@@@xercesc_2_3@@UBE_NXZ 120be7c0 f i DOMDocumentImpl.obj
 0001:000bd7c0       ?hasMoreElements@?$RefHashTableOfEnumerator@VXercesGroupInfo@xercesc_2_3@@@xercesc_2_3@@UBE_NXZ 120be7c0 f i DOMDocumentImpl.obj
 0001:000bd7c0       ?hasMoreElements@?$RefHashTableOfEnumerator@VValueStore@xercesc_2_3@@@xercesc_2_3@@UBE_NXZ 120be7c0 f i DOMDocumentImpl.obj
 0001:000bd7c0       ?hasMoreElements@?$RefHashTableOfEnumerator@G@xercesc_2_3@@UBE_NXZ 120be7c0 f i DOMDocumentImpl.obj
 0001:000bd7c0       ?hasMoreElements@?$RefHashTableOfEnumerator@V?$KeyRefPair@XVDOMUserDataHandler@xercesc_2_3@@@xercesc_2_3@@@xercesc_2_3@@UBE_NXZ 120be7c0 f i DOMDocumentImpl.obj
 0001:000bd7c0       ?hasMoreElements@?$RefHashTableOfEnumerator@VKVStringPair@xercesc_2_3@@@xercesc_2_3@@UBE_NXZ 120be7c0 f i DOMDocumentImpl.obj
 0001:000bd7c0       ?hasMoreElements@?$RefHash2KeysTableOfEnumerator@VSchemaAttDef@xercesc_2_3@@@xercesc_2_3@@UBE_NXZ 120be7c0 f i DOMDocumentImpl.obj
 0001:000bd7c0       ?hasMoreElements@?$RefHashTableOfEnumerator@VGrammar@xercesc_2_3@@@xercesc_2_3@@UBE_NXZ 120be7c0 f i DOMDocumentImpl.obj
 0001:000bd7e0       ?Reset@?$RefHashTableOfEnumerator@V?$KeyRefPair@XVDOMUserDataHandler@xercesc_2_3@@@xercesc_2_3@@@xercesc_2_3@@UAEXXZ 120be7e0 f i DOMDocumentImpl.obj
 0001:000bd7e0       ?Reset@?$RefHashTableOfEnumerator@VXercesGroupInfo@xercesc_2_3@@@xercesc_2_3@@UAEXXZ 120be7e0 f i DOMDocumentImpl.obj
 0001:000bd7e0       ?Reset@?$RefHashTableOfEnumerator@VXMLRefInfo@xercesc_2_3@@@xercesc_2_3@@UAEXXZ 120be7e0 f i DOMDocumentImpl.obj
 0001:000bd7e0       ?Reset@?$RefHashTableOfEnumerator@VKVStringPair@xercesc_2_3@@@xercesc_2_3@@UAEXXZ 120be7e0 f i DOMDocumentImpl.obj
 0001:000bd7e0       ?Reset@?$RefHash2KeysTableOfEnumerator@VSchemaAttDef@xercesc_2_3@@@xercesc_2_3@@UAEXXZ 120be7e0 f i DOMDocumentImpl.obj
 0001:000bd7e0       ?Reset@?$RefHashTableOfEnumerator@VGrammar@xercesc_2_3@@@xercesc_2_3@@UAEXXZ 120be7e0 f i DOMDocumentImpl.obj
 0001:000bd7e0       ?Reset@?$RefHashTableOfEnumerator@VDTDAttDef@xercesc_2_3@@@xercesc_2_3@@UAEXXZ 120be7e0 f i DOMDocumentImpl.obj
 0001:000bd7e0       ?Reset@?$RefHashTableOfEnumerator@VValueStore@xercesc_2_3@@@xercesc_2_3@@UAEXXZ 120be7e0 f i DOMDocumentImpl.obj
 0001:000bd7e0       ?Reset@?$RefHashTableOfEnumerator@G@xercesc_2_3@@UAEXXZ 120be7e0 f i DOMDocumentImpl.obj
 0001:000bd7e0       ?Reset@?$RefHashTableOfEnumerator@VComplexTypeInfo@xercesc_2_3@@@xercesc_2_3@@UAEXXZ 120be7e0 f i DOMDocumentImpl.obj
 0001:000bd820       ??1?$RefVectorOf@VDOMNode@xercesc_2_3@@@xercesc_2_3@@UAE@XZ 120be820 f i DOMDocumentImpl.obj
 0001:000bd8a0       ??1?$BaseRefVectorOf@VDOMNode@xercesc_2_3@@@xercesc_2_3@@UAE@XZ 120be8a0 f i DOMDocumentImpl.obj
 0001:000bd8b0       ?pop@?$RefStackOf@VDOMNode@xercesc_2_3@@@xercesc_2_3@@QAEPAVDOMNode@2@XZ 120be8b0 f i DOMDocumentImpl.obj
 0001:000bd960       ??_G?$RefVectorOf@VDOMRangeImpl@xercesc_2_3@@@xercesc_2_3@@UAEPAXI@Z 120be960 f i DOMDocumentImpl.obj
 0001:000bd960       ??_E?$RefVectorOf@VDOMRangeImpl@xercesc_2_3@@@xercesc_2_3@@UAEPAXI@Z 120be960 f i DOMDocumentImpl.obj
 0001:000bd980       ??1?$RefVectorOf@VDOMRangeImpl@xercesc_2_3@@@xercesc_2_3@@UAE@XZ 120be980 f i DOMDocumentImpl.obj
 0001:000bda00       ??1?$BaseRefVectorOf@VDOMRangeImpl@xercesc_2_3@@@xercesc_2_3@@UAE@XZ 120bea00 f i DOMDocumentImpl.obj
 0001:000bda10       ??_G?$RefVectorOf@VDOMNodeIteratorImpl@xercesc_2_3@@@xercesc_2_3@@UAEPAXI@Z 120bea10 f i DOMDocumentImpl.obj
 0001:000bda10       ??_E?$RefVectorOf@VDOMNodeIteratorImpl@xercesc_2_3@@@xercesc_2_3@@UAEPAXI@Z 120bea10 f i DOMDocumentImpl.obj
 0001:000bda30       ??1?$RefVectorOf@VDOMNodeIteratorImpl@xercesc_2_3@@@xercesc_2_3@@UAE@XZ 120bea30 f i DOMDocumentImpl.obj
 0001:000bdab0       ??1?$BaseRefVectorOf@VDOMNodeIteratorImpl@xercesc_2_3@@@xercesc_2_3@@UAE@XZ 120beab0 f i DOMDocumentImpl.obj
 0001:000bdac0       ??_E?$RefVectorOf@VDOMBuffer@xercesc_2_3@@@xercesc_2_3@@UAEPAXI@Z 120beac0 f i DOMDocumentImpl.obj
 0001:000bdac0       ??_G?$RefVectorOf@VDOMBuffer@xercesc_2_3@@@xercesc_2_3@@UAEPAXI@Z 120beac0 f i DOMDocumentImpl.obj
 0001:000bdae0       ??_G?$RefHashTableOfEnumerator@V?$KeyRefPair@XVDOMUserDataHandler@xercesc_2_3@@@xercesc_2_3@@@xercesc_2_3@@UAEPAXI@Z 120beae0 f i DOMDocumentImpl.obj
 0001:000bdae0       ??_E?$RefHashTableOfEnumerator@V?$KeyRefPair@XVDOMUserDataHandler@xercesc_2_3@@@xercesc_2_3@@@xercesc_2_3@@UAEPAXI@Z 120beae0 f i DOMDocumentImpl.obj
 0001:000bdb00       ??_E?$RefVectorOf@VDOMNode@xercesc_2_3@@@xercesc_2_3@@UAEPAXI@Z 120beb00 f i DOMDocumentImpl.obj
 0001:000bdb00       ??_G?$RefVectorOf@VDOMNode@xercesc_2_3@@@xercesc_2_3@@UAEPAXI@Z 120beb00 f i DOMDocumentImpl.obj
 0001:000bdb20       ??0?$DOMDeepNodeListPoolTableBucketElem@VDOMDeepNodeListImpl@xercesc_2_3@@@xercesc_2_3@@QAE@PAXPAG1QAVDOMDeepNodeListImpl@1@PAU01@QAVMemoryManager@1@@Z 120beb20 f i DOMDocumentImpl.obj
 0001:000bdbf0       ?removeAll@?$DOMDeepNodeListPool@VDOMDeepNodeListImpl@xercesc_2_3@@@xercesc_2_3@@QAEXXZ 120bebf0 f i DOMDocumentImpl.obj
 0001:000bdc70       ?findBucketElem@?$DOMDeepNodeListPool@VDOMDeepNodeListImpl@xercesc_2_3@@@xercesc_2_3@@AAEPAU?$DOMDeepNodeListPoolTableBucketElem@VDOMDeepNodeListImpl@xercesc_2_3@@@2@QBXQBG1AAK@Z 120bec70 f i DOMDocumentImpl.obj
 0001:000bdde0       ?removeAll@?$RefHashTableOf@V?$RefHashTableOf@V?$KeyRefPair@XVDOMUserDataHandler@xercesc_2_3@@@xercesc_2_3@@@xercesc_2_3@@@xercesc_2_3@@QAEXXZ 120bede0 f i DOMDocumentImpl.obj
 0001:000bdf00       ?removeBucketElem@?$RefHashTableOf@V?$KeyRefPair@XVDOMUserDataHandler@xercesc_2_3@@@xercesc_2_3@@@xercesc_2_3@@AAEXQBXAAI@Z 120bef00 f i DOMDocumentImpl.obj
 0001:000bdfe0       ?removeAll@?$RefHashTableOf@V?$KeyRefPair@XVDOMUserDataHandler@xercesc_2_3@@@xercesc_2_3@@@xercesc_2_3@@QAEXXZ 120befe0 f i DOMDocumentImpl.obj
 0001:000be050       ??0?$BaseRefVectorOf@VDOMNode@xercesc_2_3@@@xercesc_2_3@@QAE@I_NQAVMemoryManager@1@@Z 120bf050 f i DOMDocumentImpl.obj
 0001:000be0b0       ??_EDOMDocumentImpl@xercesc_2_3@@W3AEPAXI@Z 120bf0b0 f i DOMDocumentImpl.obj
 0001:000be0c0       ??_EDOMDocumentImpl@xercesc_2_3@@W7AEPAXI@Z 120bf0c0 f i DOMDocumentImpl.obj
 0001:000be0f0       ??0DOMDocumentTypeImpl@xercesc_2_3@@QAE@PAVDOMDocument@1@PBG_N@Z 120bf0f0 f   DOMDocumentTypeImpl.obj
 0001:000be360       ??_EDOMDocumentTypeImpl@xercesc_2_3@@UAEPAXI@Z 120bf360 f i DOMDocumentTypeImpl.obj
 0001:000be3c0       ??0DOMDocumentTypeImpl@xercesc_2_3@@QAE@PAVDOMDocument@1@PBG11_N@Z 120bf3c0 f   DOMDocumentTypeImpl.obj
 0001:000be7f0       ??0DOMDocumentTypeImpl@xercesc_2_3@@QAE@ABV01@_N1@Z 120bf7f0 f   DOMDocumentTypeImpl.obj
 0001:000be8f0       ??1DOMDocumentTypeImpl@xercesc_2_3@@UAE@XZ 120bf8f0 f   DOMDocumentTypeImpl.obj
 0001:000be960       ?cloneNode@DOMDocumentTypeImpl@xercesc_2_3@@UBEPAVDOMNode@2@_N@Z 120bf960 f   DOMDocumentTypeImpl.obj
 0001:000beab0       ?setOwnerDocument@DOMDocumentTypeImpl@xercesc_2_3@@UAEXPAVDOMDocument@2@@Z 120bfab0 f   DOMDocumentTypeImpl.obj
 0001:000beb60       ?getNodeType@DOMDocumentTypeImpl@xercesc_2_3@@UBEFXZ 120bfb60 f   DOMDocumentTypeImpl.obj
 0001:000beb60       ?getNodeType@DocumentTypeImpl@xercesc_2_3@@UAEFXZ 120bfb60 f   DOMDocumentTypeImpl.obj
 0001:000beb70       ?getEntities@DocumentTypeImpl@xercesc_2_3@@UAEPAVNamedNodeMapImpl@2@XZ 120bfb70 f   DOMDocumentTypeImpl.obj
 0001:000beb70       ?getAttributes@ElementImpl@xercesc_2_3@@UAEPAVNamedNodeMapImpl@2@XZ 120bfb70 f   DOMDocumentTypeImpl.obj
 0001:000beb70       ?getActualEncoding@DOMEntityImpl@xercesc_2_3@@UBEPBGXZ 120bfb70 f   DOMDocumentTypeImpl.obj
 0001:000beb70       ?getDocumentElement@DocumentImpl@xercesc_2_3@@UAEPAVElementImpl@2@XZ 120bfb70 f   DOMDocumentTypeImpl.obj
 0001:000beb70       ?getElements@DOMDocumentTypeImpl@xercesc_2_3@@UBEPAVDOMNamedNodeMap@2@XZ 120bfb70 f   DOMDocumentTypeImpl.obj
 0001:000beb70       ?getBaseURI@DOMDocumentImpl@xercesc_2_3@@UBEPBGXZ 120bfb70 f   DOMDocumentTypeImpl.obj
 0001:000beb80       ?setReadOnly@DOMDocumentTypeImpl@xercesc_2_3@@UAEX_N0@Z 120bfb80 f   DOMDocumentTypeImpl.obj
 0001:000bebc0       ?getVersion@DOMDocumentImpl@xercesc_2_3@@UBEPBGXZ 120bfbc0 f   DOMDocumentTypeImpl.obj
 0001:000bebc0       ?getPublicId@DOMDocumentTypeImpl@xercesc_2_3@@UBEPBGXZ 120bfbc0 f   DOMDocumentTypeImpl.obj
 0001:000bebc0       ?getEncoding@DOMEntityImpl@xercesc_2_3@@UBEPBGXZ 120bfbc0 f   DOMDocumentTypeImpl.obj
 0001:000bebc0       ?getNamespaceURI@DOMElementNSImpl@xercesc_2_3@@UBEPBGXZ 120bfbc0 f   DOMDocumentTypeImpl.obj
 0001:000bebc0       ?getNotations@DocumentTypeImpl@xercesc_2_3@@UAEPAVNamedNodeMapImpl@2@XZ 120bfbc0 f   DOMDocumentTypeImpl.obj
 0001:000bebd0       ?getSystemId@DOMDocumentTypeImpl@xercesc_2_3@@UBEPBGXZ 120bfbd0 f   DOMDocumentTypeImpl.obj
 0001:000bebd0       ?getDocumentURI@DOMDocumentImpl@xercesc_2_3@@UBEPBGXZ 120bfbd0 f   DOMDocumentTypeImpl.obj
 0001:000bebd0       ?getLocalName@DOMElementNSImpl@xercesc_2_3@@UBEPBGXZ 120bfbd0 f   DOMDocumentTypeImpl.obj
 0001:000bebd0       ?getElements@DocumentTypeImpl@xercesc_2_3@@UAEPAVNamedNodeMapImpl@2@XZ 120bfbd0 f   DOMDocumentTypeImpl.obj
 0001:000bebd0       ?getVersion@DOMEntityImpl@xercesc_2_3@@UBEPBGXZ 120bfbd0 f   DOMDocumentTypeImpl.obj
 0001:000bebe0       ?getContentLeafNameTypeVector@DFAContentModel@xercesc_2_3@@UBEPAVContentLeafNameTypeVector@2@XZ 120bfbe0 f   DOMDocumentTypeImpl.obj
 0001:000bebe0       ?getInternalSubset@DOMDocumentTypeImpl@xercesc_2_3@@UBEPBGXZ 120bfbe0 f   DOMDocumentTypeImpl.obj
 0001:000bebe0       ?getEnumString@UnionDatatypeValidator@xercesc_2_3@@UBEPBV?$RefArrayVectorOf@G@2@XZ 120bfbe0 f   DOMDocumentTypeImpl.obj
 0001:000bebe0       ?getPrefix@DOMElementNSImpl@xercesc_2_3@@UBEPBGXZ 120bfbe0 f   DOMDocumentTypeImpl.obj
 0001:000bebe0       ?getBaseURI@DOMEntityImpl@xercesc_2_3@@UBEPBGXZ 120bfbe0 f   DOMDocumentTypeImpl.obj
 0001:000bebe0       ?getEntityRef@EntityImpl@xercesc_2_3@@UBEPAVEntityReferenceImpl@2@XZ 120bfbe0 f   DOMDocumentTypeImpl.obj
 0001:000bebf0       ?isIntSubsetReading@DOMDocumentTypeImpl@xercesc_2_3@@ABE_NXZ 120bfbf0 f   DOMDocumentTypeImpl.obj
 0001:000bec00       ?setPublicId@DOMDocumentTypeImpl@xercesc_2_3@@EAEXPBG@Z 120bfc00 f   DOMDocumentTypeImpl.obj
 0001:000becf0       ?setSystemId@DOMDocumentTypeImpl@xercesc_2_3@@EAEXPBG@Z 120bfcf0 f   DOMDocumentTypeImpl.obj
 0001:000bedd0       ?setInternalSubset@DOMDocumentTypeImpl@xercesc_2_3@@EAEXPBG@Z 120bfdd0 f   DOMDocumentTypeImpl.obj
 0001:000beeb0       ?release@DOMDocumentTypeImpl@xercesc_2_3@@UAEXXZ 120bfeb0 f   DOMDocumentTypeImpl.obj
 0001:000bef70       ?insertBefore@DOMEntityReferenceImpl@xercesc_2_3@@UAEPAVDOMNode@2@PAV32@0@Z 120bff70 f   DOMDocumentTypeImpl.obj
 0001:000bef70       ?insertBefore@DOMCDATASectionImpl@xercesc_2_3@@UAEPAVDOMNode@2@PAV32@0@Z 120bff70 f   DOMDocumentTypeImpl.obj
 0001:000bef70       ?insertBefore@DOMAttrImpl@xercesc_2_3@@UAEPAVDOMNode@2@PAV32@0@Z 120bff70 f   DOMDocumentTypeImpl.obj
 0001:000bef70       ?insertBefore@DOMDocumentTypeImpl@xercesc_2_3@@UAEPAVDOMNode@2@PAV32@0@Z 120bff70 f   DOMDocumentTypeImpl.obj
 0001:000bef70       ?insertBefore@DOMElementImpl@xercesc_2_3@@UAEPAVDOMNode@2@PAV32@0@Z 120bff70 f   DOMDocumentTypeImpl.obj
 0001:000bef70       ?insertBefore@DOMDocumentFragmentImpl@xercesc_2_3@@UAEPAVDOMNode@2@PAV32@0@Z 120bff70 f   DOMDocumentTypeImpl.obj
 0001:000bef90       ?replaceChild@DOMDocumentFragmentImpl@xercesc_2_3@@UAEPAVDOMNode@2@PAV32@0@Z 120bff90 f   DOMDocumentTypeImpl.obj
 0001:000bef90       ?replaceChild@DOMAttrImpl@xercesc_2_3@@UAEPAVDOMNode@2@PAV32@0@Z 120bff90 f   DOMDocumentTypeImpl.obj
 0001:000bef90       ?replaceChild@DOMCDATASectionImpl@xercesc_2_3@@UAEPAVDOMNode@2@PAV32@0@Z 120bff90 f   DOMDocumentTypeImpl.obj
 0001:000bef90       ?replaceChild@DOMDocumentTypeImpl@xercesc_2_3@@UAEPAVDOMNode@2@PAV32@0@Z 120bff90 f   DOMDocumentTypeImpl.obj
 0001:000bef90       ?replaceChild@DOMElementImpl@xercesc_2_3@@UAEPAVDOMNode@2@PAV32@0@Z 120bff90 f   DOMDocumentTypeImpl.obj
 0001:000bef90       ?replaceChild@DOMEntityReferenceImpl@xercesc_2_3@@UAEPAVDOMNode@2@PAV32@0@Z 120bff90 f   DOMDocumentTypeImpl.obj
 0001:000befb0       ?isEqualNode@DOMDocumentTypeImpl@xercesc_2_3@@UBE_NPBVDOMNode@2@@Z 120bffb0 f   DOMDocumentTypeImpl.obj
 0001:000bf350       ??0DOMElementImpl@xercesc_2_3@@QAE@PAVDOMDocument@1@PBG@Z 120c0350 f   DOMElementImpl.obj
 0001:000bf480       ??_EDOMElementImpl@xercesc_2_3@@UAEPAXI@Z 120c0480 f i DOMElementImpl.obj
 0001:000bf4e0       ??0DOMElementImpl@xercesc_2_3@@QAE@ABV01@_N@Z 120c04e0 f   DOMElementImpl.obj
 0001:000bf680       ??1DOMElementImpl@xercesc_2_3@@UAE@XZ 120c0680 f   DOMElementImpl.obj
 0001:000bf6f0       ?cloneNode@DOMElementImpl@xercesc_2_3@@UBEPAVDOMNode@2@_N@Z 120c06f0 f   DOMElementImpl.obj
 0001:000bf770       ?getNodeType@DOMElementImpl@xercesc_2_3@@UBEFXZ 120c0770 f   DOMElementImpl.obj
 0001:000bf770       ?getNodeType@ElementImpl@xercesc_2_3@@UAEFXZ 120c0770 f   DOMElementImpl.obj
 0001:000bf780       ?getAttribute@DOMElementImpl@xercesc_2_3@@UBEPBGPBG@Z 120c0780 f   DOMElementImpl.obj
 0001:000bf7a0       ?getAttributeNode@DOMElementImpl@xercesc_2_3@@UBEPAVDOMAttr@2@PBG@Z 120c07a0 f   DOMElementImpl.obj
 0001:000bf7b0       ?getElementsByTagName@DOMElementImpl@xercesc_2_3@@UBEPAVDOMNodeList@2@PBG@Z 120c07b0 f   DOMElementImpl.obj
 0001:000bf7d0       ?removeAttribute@DOMElementImpl@xercesc_2_3@@UAEXPBG@Z 120c07d0 f   DOMElementImpl.obj
 0001:000bf840       ?removeAttributeNode@DOMElementImpl@xercesc_2_3@@UAEPAVDOMAttr@2@PAV32@@Z 120c0840 f   DOMElementImpl.obj
 0001:000bf920       ?setAttribute@DOMElementImpl@xercesc_2_3@@UAEXPBG0@Z 120c0920 f   DOMElementImpl.obj
 0001:000bf9a0       ?setIdAttribute@DOMElementImpl@xercesc_2_3@@UAEXPBG@Z 120c09a0 f   DOMElementImpl.obj
 0001:000bfa10       ?setIdAttributeNS@DOMElementImpl@xercesc_2_3@@UAEXPBG0@Z 120c0a10 f   DOMElementImpl.obj
 0001:000bfa80       ?setIdAttributeNode@DOMElementImpl@xercesc_2_3@@UAEXPBVDOMAttr@2@@Z 120c0a80 f   DOMElementImpl.obj
 0001:000bfb20       ?setAttributeNode@DOMElementImpl@xercesc_2_3@@UAEPAVDOMAttr@2@PAV32@@Z 120c0b20 f   DOMElementImpl.obj
 0001:000bfb90       ?setReadOnly@DOMElementImpl@xercesc_2_3@@UAEX_N0@Z 120c0b90 f   DOMElementImpl.obj
 0001:000bfbc0       ?getAttributeNS@DOMElementImpl@xercesc_2_3@@UBEPBGPBG0@Z 120c0bc0 f   DOMElementImpl.obj
 0001:000bfbf0       ?setAttributeNS@DOMElementImpl@xercesc_2_3@@UAEXPBG00@Z 120c0bf0 f   DOMElementImpl.obj
 0001:000bfc70       ?removeAttributeNS@DOMElementImpl@xercesc_2_3@@UAEXPBG0@Z 120c0c70 f   DOMElementImpl.obj
 0001:000bfcd0       ?getAttributeNodeNS@DOMElementImpl@xercesc_2_3@@UBEPAVDOMAttr@2@PBG0@Z 120c0cd0 f   DOMElementImpl.obj
 0001:000bfcf0       ?setAttributeNodeNS@DOMElementImpl@xercesc_2_3@@UAEPAVDOMAttr@2@PAV32@@Z 120c0cf0 f   DOMElementImpl.obj
 0001:000bfd70       ?getElementsByTagNameNS@DOMElementImpl@xercesc_2_3@@UBEPAVDOMNodeList@2@PBG0@Z 120c0d70 f   DOMElementImpl.obj
 0001:000bfd90       ?hasAttributes@DOMElementImpl@xercesc_2_3@@UBE_NXZ 120c0d90 f   DOMElementImpl.obj
 0001:000bfdb0       ?hasAttribute@DOMElementImpl@xercesc_2_3@@UBE_NPBG@Z 120c0db0 f   DOMElementImpl.obj
 0001:000bfdd0       ?hasAttributeNS@DOMElementImpl@xercesc_2_3@@UBE_NPBG0@Z 120c0dd0 f   DOMElementImpl.obj
 0001:000bfdf0       ?setupDefaultAttributes@DOMElementImpl@xercesc_2_3@@MAEXXZ 120c0df0 f   DOMElementImpl.obj
 0001:000bfec0       ?setDefaultAttributeNode@DOMElementImpl@xercesc_2_3@@UAEPAVDOMAttr@2@PAV32@@Z 120c0ec0 f   DOMElementImpl.obj
 0001:000bff40       ?setDefaultAttributeNodeNS@DOMElementImpl@xercesc_2_3@@UAEPAVDOMAttr@2@PAV32@@Z 120c0f40 f   DOMElementImpl.obj
 0001:000bffd0       ?release@DOMElementImpl@xercesc_2_3@@UAEXXZ 120c0fd0 f   DOMElementImpl.obj
 0001:000c0060       ?getBaseURI@DOMElementImpl@xercesc_2_3@@UBEPBGXZ 120c1060 f   DOMElementImpl.obj
 0001:000c01b0       ?isEqualNode@DOMElementImpl@xercesc_2_3@@UBE_NPBVDOMNode@2@@Z 120c11b0 f   DOMElementImpl.obj
 0001:000c02f0       ?rename@DOMElementImpl@xercesc_2_3@@UAEPAVDOMNode@2@PBG0@Z 120c12f0 f   DOMElementImpl.obj
 0001:000c03e0       ?getTypeInfo@DOMElementImpl@xercesc_2_3@@UBEPBVDOMTypeInfo@2@XZ 120c13e0 f   DOMElementImpl.obj
 0001:000c0480       ?setTypeInfo@DOMElementImpl@xercesc_2_3@@UAEXPBG0@Z 120c1480 f   DOMElementImpl.obj
 0001:000c04f0       ??0DOMElementNSImpl@xercesc_2_3@@QAE@PAVDOMDocument@1@PBG@Z 120c14f0 f   DOMElementNSImpl.obj
 0001:000c0520       ??_EDOMElementNSImpl@xercesc_2_3@@UAEPAXI@Z 120c1520 f i DOMElementNSImpl.obj
 0001:000c0580       ??0DOMElementNSImpl@xercesc_2_3@@QAE@PAVDOMDocument@1@PBG1@Z 120c1580 f   DOMElementNSImpl.obj
 0001:000c05e0       ??0DOMElementNSImpl@xercesc_2_3@@QAE@ABV01@_N@Z 120c15e0 f   DOMElementNSImpl.obj
 0001:000c0620       ?cloneNode@DOMElementNSImpl@xercesc_2_3@@UBEPAVDOMNode@2@_N@Z 120c1620 f   DOMElementNSImpl.obj
 0001:000c06c0       ?getBaseURI@DOMElementNSImpl@xercesc_2_3@@UBEPBGXZ 120c16c0 f   DOMElementNSImpl.obj
 0001:000c0800       ?setPrefix@DOMElementNSImpl@xercesc_2_3@@UAEXPBG@Z 120c1800 f   DOMElementNSImpl.obj
 0001:000c0a60       ?release@DOMElementNSImpl@xercesc_2_3@@UAEXXZ 120c1a60 f   DOMElementNSImpl.obj
 0001:000c0af0       ?rename@DOMElementNSImpl@xercesc_2_3@@UAEPAVDOMNode@2@PBG0@Z 120c1af0 f   DOMElementNSImpl.obj
 0001:000c0b20       ?setName@DOMElementNSImpl@xercesc_2_3@@QAEXPBG0@Z 120c1b20 f   DOMElementNSImpl.obj
 0001:000c0cb0       ??0DOMEntityImpl@xercesc_2_3@@QAE@PAVDOMDocument@1@PBG@Z 120c1cb0 f   DOMEntityImpl.obj
 0001:000c0d60       ??_EDOMEntityImpl@xercesc_2_3@@UAEPAXI@Z 120c1d60 f i DOMEntityImpl.obj
 0001:000c0dc0       ??0DOMEntityImpl@xercesc_2_3@@QAE@ABV01@_N@Z 120c1dc0 f   DOMEntityImpl.obj
 0001:000c0e90       ??1DOMEntityImpl@xercesc_2_3@@UAE@XZ 120c1e90 f   DOMEntityImpl.obj
 0001:000c0ef0       ?cloneNode@DOMEntityImpl@xercesc_2_3@@UBEPAVDOMNode@2@_N@Z 120c1ef0 f   DOMEntityImpl.obj
 0001:000c0f70       ?getNodeType@EntityImpl@xercesc_2_3@@UAEFXZ 120c1f70 f   DOMEntityImpl.obj
 0001:000c0f70       ?getNodeType@DOMEntityImpl@xercesc_2_3@@UBEFXZ 120c1f70 f   DOMEntityImpl.obj
 0001:000c0f80       ?getPublicId@DOMEntityImpl@xercesc_2_3@@UBEPBGXZ 120c1f80 f   DOMEntityImpl.obj
 0001:000c0f90       ?setNotationName@DOMEntityImpl@xercesc_2_3@@UAEXPBG@Z 120c1f90 f   DOMEntityImpl.obj
 0001:000c0fb0       ?setPublicId@DOMEntityImpl@xercesc_2_3@@UAEXPBG@Z 120c1fb0 f   DOMEntityImpl.obj
 0001:000c0fd0       ?setSystemId@DOMEntityImpl@xercesc_2_3@@UAEXPBG@Z 120c1fd0 f   DOMEntityImpl.obj
 0001:000c0ff0       ?setBaseURI@DOMEntityImpl@xercesc_2_3@@UAEXPBG@Z 120c1ff0 f   DOMEntityImpl.obj
 0001:000c1050       ?setEntityRef@DOMEntityImpl@xercesc_2_3@@UAEXPAVDOMEntityReference@2@@Z 120c2050 f   DOMEntityImpl.obj
 0001:000c1060       ?cloneEntityRefTree@DOMEntityImpl@xercesc_2_3@@ABEXXZ 120c2060 f   DOMEntityImpl.obj
 0001:000c10b0       ?getFirstChild@DOMEntityImpl@xercesc_2_3@@UBEPAVDOMNode@2@XZ 120c20b0 f   DOMEntityImpl.obj
 0001:000c1100       ?getLastChild@DOMEntityImpl@xercesc_2_3@@UBEPAVDOMNode@2@XZ 120c2100 f   DOMEntityImpl.obj
 0001:000c1150       ?getChildNodes@DOMEntityImpl@xercesc_2_3@@UBEPAVDOMNodeList@2@XZ 120c2150 f   DOMEntityImpl.obj
 0001:000c11a0       ?hasChildNodes@DOMEntityImpl@xercesc_2_3@@UBE_NXZ 120c21a0 f   DOMEntityImpl.obj
 0001:000c11f0       ?release@DOMEntityImpl@xercesc_2_3@@UAEXXZ 120c21f0 f   DOMEntityImpl.obj
 0001:000c1280       ?appendChild@DOMEntityImpl@xercesc_2_3@@UAEPAVDOMNode@2@PAV32@@Z 120c2280 f   DOMEntityImpl.obj
 0001:000c12e0       ?insertBefore@DOMEntityImpl@xercesc_2_3@@UAEPAVDOMNode@2@PAV32@0@Z 120c22e0 f   DOMEntityImpl.obj
 0001:000c1340       ?normalize@DOMEntityImpl@xercesc_2_3@@UAEXXZ 120c2340 f   DOMEntityImpl.obj
 0001:000c1390       ?removeChild@DOMEntityImpl@xercesc_2_3@@UAEPAVDOMNode@2@PAV32@@Z 120c2390 f   DOMEntityImpl.obj
 0001:000c13f0       ?replaceChild@DOMEntityImpl@xercesc_2_3@@UAEPAVDOMNode@2@PAV32@0@Z 120c23f0 f   DOMEntityImpl.obj
 0001:000c1450       ?isEqualNode@DOMEntityImpl@xercesc_2_3@@UBE_NPBVDOMNode@2@@Z 120c2450 f   DOMEntityImpl.obj
 0001:000c14b0       ?setActualEncoding@DOMEntityImpl@xercesc_2_3@@UAEXPBG@Z 120c24b0 f   DOMEntityImpl.obj
 0001:000c14d0       ?setEncoding@DOMEntityImpl@xercesc_2_3@@UAEXPBG@Z 120c24d0 f   DOMEntityImpl.obj
 0001:000c14f0       ?setVersion@DOMEntityImpl@xercesc_2_3@@UAEXPBG@Z 120c24f0 f   DOMEntityImpl.obj
 0001:000c1510       ??0DOMEntityReferenceImpl@xercesc_2_3@@QAE@PAVDOMDocument@1@PBG@Z 120c2510 f   DOMEntityReferenceImpl.obj
 0001:000c1620       ??_EDOMEntityReferenceImpl@xercesc_2_3@@UAEPAXI@Z 120c2620 f i DOMEntityReferenceImpl.obj
 0001:000c1680       ??0DOMEntityReferenceImpl@xercesc_2_3@@QAE@PAVDOMDocument@1@PBG_N@Z 120c2680 f   DOMEntityReferenceImpl.obj
 0001:000c1790       ??0DOMEntityReferenceImpl@xercesc_2_3@@QAE@ABV01@_N@Z 120c2790 f   DOMEntityReferenceImpl.obj
 0001:000c1840       ??1DOMEntityReferenceImpl@xercesc_2_3@@UAE@XZ 120c2840 f   DOMEntityReferenceImpl.obj
 0001:000c18b0       ?cloneNode@DOMEntityReferenceImpl@xercesc_2_3@@UBEPAVDOMNode@2@_N@Z 120c28b0 f   DOMEntityReferenceImpl.obj
 0001:000c1930       ?getNodeType@DOMEntityReferenceImpl@xercesc_2_3@@UBEFXZ 120c2930 f   DOMEntityReferenceImpl.obj
 0001:000c1930       ?getNodeType@EntityReferenceImpl@xercesc_2_3@@UAEFXZ 120c2930 f   DOMEntityReferenceImpl.obj
 0001:000c1940       ?setReadOnly@DOMEntityReferenceImpl@xercesc_2_3@@UAEX_N0@Z 120c2940 f   DOMEntityReferenceImpl.obj
 0001:000c1990       ?release@DOMEntityReferenceImpl@xercesc_2_3@@UAEXXZ 120c2990 f   DOMEntityReferenceImpl.obj
 0001:000c1a20       ??0DOMErrorImpl@xercesc_2_3@@QAE@F@Z 120c2a20 f   DOMErrorImpl.obj
 0001:000c1a50       ??_EDOMErrorImpl@xercesc_2_3@@UAEPAXI@Z 120c2a50 f i DOMErrorImpl.obj
 0001:000c1ab0       ??0DOMErrorImpl@xercesc_2_3@@QAE@FQBGQAVDOMLocator@1@@Z 120c2ab0 f   DOMErrorImpl.obj
 0001:000c1ae0       ??0DOMErrorImpl@xercesc_2_3@@QAE@FPBG0PAX_N@Z 120c2ae0 f   DOMErrorImpl.obj
 0001:000c1b20       ??1DOMErrorImpl@xercesc_2_3@@UAE@XZ 120c2b20 f   DOMErrorImpl.obj
 0001:000c1b90       ?setLocation@DOMErrorImpl@xercesc_2_3@@UAEXQAVDOMLocator@2@@Z 120c2b90 f   DOMErrorImpl.obj
 0001:000c1bd0       ??0DOMImplementationSource@xercesc_2_3@@IAE@XZ 120c2bd0 f i DOMImplementationImpl.obj
 0001:000c1be0       ??1DOMImplementationSource@xercesc_2_3@@UAE@XZ 120c2be0 f i DOMImplementationImpl.obj
 0001:000c1bf0       ??_EDOMImplementationSource@xercesc_2_3@@UAEPAXI@Z 120c2bf0 f i DOMImplementationImpl.obj
 0001:000c1c50       ??0DOMWriterFilter@xercesc_2_3@@IAE@XZ 120c2c50 f i DOMImplementationImpl.obj
 0001:000c1c60       ??_EDOMWriterFilter@xercesc_2_3@@UAEPAXI@Z 120c2c60 f i DOMImplementationImpl.obj
 0001:000c1cc0       ??0DOMWriter@xercesc_2_3@@IAE@XZ 120c2cc0 f i DOMImplementationImpl.obj
 0001:000c1cd0       ??1DOMWriter@xercesc_2_3@@UAE@XZ 120c2cd0 f i DOMImplementationImpl.obj
 0001:000c1ce0       ??_EDOMWriter@xercesc_2_3@@UAEPAXI@Z 120c2ce0 f i DOMImplementationImpl.obj
 0001:000c1d40       ??_FDOMWriterImpl@xercesc_2_3@@QAEXXZ 120c2d40 f i DOMImplementationImpl.obj
 0001:000c1d50       ?setFeature@DOMWriterImpl@xercesc_2_3@@AAEXH_N@Z 120c2d50 f i DOMImplementationImpl.obj
 0001:000c1d80       ?getFeature@DOMWriterImpl@xercesc_2_3@@ABE_NH@Z 120c2d80 f i DOMImplementationImpl.obj
 0001:000c1da0       ?setURCharRef@DOMWriterImpl@xercesc_2_3@@AAEXXZ 120c2da0 f i DOMImplementationImpl.obj
 0001:000c1db0       ?getMsgLoader4DOM@DOMImplementationImpl@xercesc_2_3@@SAPAVXMLMsgLoader@2@XZ 120c2db0 f   DOMImplementationImpl.obj
 0001:000c1ed0       ?getDOMImplementationImpl@DOMImplementationImpl@xercesc_2_3@@SAPAV12@XZ 120c2ed0 f   DOMImplementationImpl.obj
 0001:000c1fd0       ??_EDOMImplementationImpl@xercesc_2_3@@UAEPAXI@Z 120c2fd0 f i DOMImplementationImpl.obj
 0001:000c1fd0       ??_GDOMImplementationImpl@xercesc_2_3@@UAEPAXI@Z 120c2fd0 f i DOMImplementationImpl.obj
 0001:000c1ff0       ??1DOMImplementationImpl@xercesc_2_3@@UAE@XZ 120c2ff0 f i DOMImplementationImpl.obj
 0001:000c2050       ?hasFeature@DOMImplementationImpl@xercesc_2_3@@UBE_NPBG0@Z 120c3050 f   DOMImplementationImpl.obj
 0001:000c2280       ?createDocumentType@DOMImplementationImpl@xercesc_2_3@@UAEPAVDOMDocumentType@2@PBG00@Z 120c3280 f   DOMImplementationImpl.obj
 0001:000c2350       ?createDocument@DOMImplementationImpl@xercesc_2_3@@UAEPAVDOMDocument@2@PBG0PAVDOMDocumentType@2@QAVMemoryManager@2@@Z 120c3350 f   DOMImplementationImpl.obj
 0001:000c23d0       ?createDocument@DOMImplementationImpl@xercesc_2_3@@UAEPAVDOMDocument@2@QAVMemoryManager@2@@Z 120c33d0 f   DOMImplementationImpl.obj
 0001:000c2440       ?getImplementation@DOMImplementation@xercesc_2_3@@SAPAV12@XZ 120c3440 f   DOMImplementationImpl.obj
 0001:000c2450       ?loadDOMExceptionMsg@DOMImplementation@xercesc_2_3@@SA_NW4ExceptionCode@DOMException@2@QAGI@Z 120c3450 f   DOMImplementationImpl.obj
 0001:000c2550       ?loadDOMExceptionMsg@DOMImplementation@xercesc_2_3@@SA_NW4RangeExceptionCode@DOMRangeException@2@QAGI@Z 120c3550 f   DOMImplementationImpl.obj
 0001:000c2650       ?createDOMBuilder@DOMImplementationImpl@xercesc_2_3@@UAEPAVDOMBuilder@2@FQBGQAVMemoryManager@2@@Z 120c3650 f   DOMImplementationImpl.obj
 0001:000c26e0       ?createDOMWriter@DOMImplementationImpl@xercesc_2_3@@UAEPAVDOMWriter@2@QAVMemoryManager@2@@Z 120c36e0 f   DOMImplementationImpl.obj
 0001:000c2740       ?getInterface@DOMImplementationImpl@xercesc_2_3@@UAEPAVDOMImplementation@2@PBG@Z 120c3740 f   DOMImplementationImpl.obj
 0001:000c2740       ?setRelatedException@DOMErrorImpl@xercesc_2_3@@UBEXPAX@Z 120c3740 f   DOMImplementationImpl.obj
 0001:000c2740       ?replaceWholeText@DOMCDATASectionImpl@xercesc_2_3@@UAEPAVDOMText@2@PBG@Z 120c3740 f   DOMImplementationImpl.obj
 0001:000c2740       ?getWholeText@DOMTextImpl@xercesc_2_3@@UAEPBGXZ 120c3740 f   DOMImplementationImpl.obj
 0001:000c2740       ?getWholeText@DOMCDATASectionImpl@xercesc_2_3@@UAEPBGXZ 120c3740 f   DOMImplementationImpl.obj
 0001:000c2740       ?parseWithContext@DOMBuilderImpl@xercesc_2_3@@UAEXABVDOMInputSource@2@QAVDOMNode@2@F@Z 120c3740 f   DOMImplementationImpl.obj
 0001:000c2740       ?getInterface@DOMNodeImpl@xercesc_2_3@@QAEPAVDOMNode@2@PBG@Z 120c3740 f   DOMImplementationImpl.obj
 0001:000c2740       ?setTextContent@DOMNodeImpl@xercesc_2_3@@QAEXPBG@Z 120c3740 f   DOMImplementationImpl.obj
 0001:000c2740       ?replaceWholeText@DOMTextImpl@xercesc_2_3@@UAEPAVDOMText@2@PBG@Z 120c3740 f   DOMImplementationImpl.obj
 0001:000c2740       ?createDOMInputSource@DOMImplementationImpl@xercesc_2_3@@UAEPAVDOMInputSource@2@XZ 120c3740 f   DOMImplementationImpl.obj
 0001:000c2740       ?adoptNode@DOMDocumentImpl@xercesc_2_3@@UAEPAVDOMNode@2@PAV32@@Z 120c3740 f   DOMImplementationImpl.obj
 0001:000c2740       ?setFilter@DOMBuilderImpl@xercesc_2_3@@UAEXQAVDOMBuilderFilter@2@@Z 120c3740 f   DOMImplementationImpl.obj
 0001:000c2760       ?getDOMImplementation@DOMImplementationImpl@xercesc_2_3@@UBEPAVDOMImplementation@2@PBG@Z 120c3760 f   DOMImplementationImpl.obj
 0001:000c2910       ??_EDOMImplementationImpl@xercesc_2_3@@W3AEPAXI@Z 120c3910 f i DOMImplementationImpl.obj
 0001:000c2920       ?getDOMImplSrcVector@xercesc_2_3@@YAPAV?$RefVectorOf@VDOMImplementationSource@xercesc_2_3@@@1@XZ 120c3920 f   DOMImplementationRegistry.obj
 0001:000c2ad0       ?getDOMImplementation@DOMImplementationRegistry@xercesc_2_3@@SAPAVDOMImplementation@2@PBG@Z 120c3ad0 f   DOMImplementationRegistry.obj
 0001:000c2e90       ?addSource@DOMImplementationRegistry@xercesc_2_3@@SAXPAVDOMImplementationSource@2@@Z 120c3e90 f   DOMImplementationRegistry.obj
 0001:000c3150       ??0?$RefVectorOf@VDOMImplementationSource@xercesc_2_3@@@xercesc_2_3@@QAE@I_NQAVMemoryManager@1@@Z 120c4150 f i DOMImplementationRegistry.obj
 0001:000c31b0       ??_G?$RefVectorOf@VDOMImplementationSource@xercesc_2_3@@@xercesc_2_3@@UAEPAXI@Z 120c41b0 f i DOMImplementationRegistry.obj
 0001:000c31b0       ??_E?$RefVectorOf@VDOMImplementationSource@xercesc_2_3@@@xercesc_2_3@@UAEPAXI@Z 120c41b0 f i DOMImplementationRegistry.obj
 0001:000c31d0       ??1?$RefVectorOf@VDOMImplementationSource@xercesc_2_3@@@xercesc_2_3@@UAE@XZ 120c41d0 f i DOMImplementationRegistry.obj
 0001:000c3250       ??1?$BaseRefVectorOf@VDOMImplementationSource@xercesc_2_3@@@xercesc_2_3@@UAE@XZ 120c4250 f i DOMImplementationRegistry.obj
 0001:000c3260       ??0?$BaseRefVectorOf@VDOMImplementationSource@xercesc_2_3@@@xercesc_2_3@@QAE@I_NQAVMemoryManager@1@@Z 120c4260 f i DOMImplementationRegistry.obj
 0001:000c32c0       ??0DOMLocatorImpl@xercesc_2_3@@QAE@XZ 120c42c0 f   DOMLocatorImpl.obj
 0001:000c32e0       ??_EDOMLocatorImpl@xercesc_2_3@@UAEPAXI@Z 120c42e0 f i DOMLocatorImpl.obj
 0001:000c3340       ??0DOMLocatorImpl@xercesc_2_3@@QAE@JJQAVDOMNode@1@QBGJ@Z 120c4340 f   DOMLocatorImpl.obj
 0001:000c3370       ??1DOMLocatorImpl@xercesc_2_3@@UAE@XZ 120c4370 f   DOMLocatorImpl.obj
 0001:000c3380       ??0DOMNamedNodeMapImpl@xercesc_2_3@@QAE@PAVDOMNode@1@@Z 120c4380 f   DOMNamedNodeMapImpl.obj
 0001:000c33a0       ??_EDOMNamedNodeMapImpl@xercesc_2_3@@UAEPAXI@Z 120c43a0 f i DOMNamedNodeMapImpl.obj
 0001:000c3400       ??1DOMNamedNodeMapImpl@xercesc_2_3@@UAE@XZ 120c4400 f   DOMNamedNodeMapImpl.obj
 0001:000c3410       ?readOnly@DOMNamedNodeMapImpl@xercesc_2_3@@IAE_NXZ 120c4410 f   DOMNamedNodeMapImpl.obj
 0001:000c3430       ?cloneMap@DOMNamedNodeMapImpl@xercesc_2_3@@UAEPAV12@PAVDOMNode@2@@Z 120c4430 f   DOMNamedNodeMapImpl.obj
 0001:000c3560       ?removeAll@DOMNamedNodeMapImpl@xercesc_2_3@@UAEXXZ 120c4560 f   DOMNamedNodeMapImpl.obj
 0001:000c35b0       ?findNamePoint@DOMNamedNodeMapImpl@xercesc_2_3@@UBEHPBG@Z 120c45b0 f   DOMNamedNodeMapImpl.obj
 0001:000c3620       ?getNamedItem@DOMNamedNodeMapImpl@xercesc_2_3@@UBEPAVDOMNode@2@PBG@Z 120c4620 f   DOMNamedNodeMapImpl.obj
 0001:000c3650       ?removeNamedItem@DOMNamedNodeMapImpl@xercesc_2_3@@UAEPAVDOMNode@2@PBG@Z 120c4650 f   DOMNamedNodeMapImpl.obj
 0001:000c3700       ?setNamedItem@DOMNamedNodeMapImpl@xercesc_2_3@@UAEPAVDOMNode@2@PAV32@@Z 120c4700 f   DOMNamedNodeMapImpl.obj
 0001:000c38a0       ?setReadOnly@DOMNamedNodeMapImpl@xercesc_2_3@@UAEX_N0@Z 120c48a0 f   DOMNamedNodeMapImpl.obj
 0001:000c38f0       ?findNamePoint@DOMNamedNodeMapImpl@xercesc_2_3@@UBEHPBG0@Z 120c48f0 f   DOMNamedNodeMapImpl.obj
 0001:000c3a40       ?getNamedItemNS@DOMNamedNodeMapImpl@xercesc_2_3@@UBEPAVDOMNode@2@PBG0@Z 120c4a40 f   DOMNamedNodeMapImpl.obj
 0001:000c3a70       ?setNamedItemNS@DOMNamedNodeMapImpl@xercesc_2_3@@UAEPAVDOMNode@2@PAV32@@Z 120c4a70 f   DOMNamedNodeMapImpl.obj
 0001:000c3c10       ?removeNamedItemNS@DOMNamedNodeMapImpl@xercesc_2_3@@UAEPAVDOMNode@2@PBG0@Z 120c4c10 f   DOMNamedNodeMapImpl.obj
 0001:000c3cc0       ?cloneContent@DOMNamedNodeMapImpl@xercesc_2_3@@MAEXPBV12@@Z 120c4cc0 f   DOMNamedNodeMapImpl.obj
 0001:000c3de0       ?removeNamedItemAt@DOMNamedNodeMapImpl@xercesc_2_3@@UAEPAVDOMNode@2@K@Z 120c4de0 f   DOMNamedNodeMapImpl.obj
 0001:000c3e80       ??0DOMNodeIDMap@xercesc_2_3@@QAE@HPAVDOMDocument@1@@Z 120c4e80 f   DOMNodeIDMap.obj
 0001:000c3f70       ??_EDOMNodeIDMap@xercesc_2_3@@UAEPAXI@Z 120c4f70 f i DOMNodeIDMap.obj
 0001:000c3f70       ??_GDOMNodeIDMap@xercesc_2_3@@UAEPAXI@Z 120c4f70 f i DOMNodeIDMap.obj
 0001:000c3fa0       ?add@DOMNodeIDMap@xercesc_2_3@@QAEXPAVDOMAttr@2@@Z 120c4fa0 f   DOMNodeIDMap.obj
 0001:000c4010       ?remove@DOMNodeIDMap@xercesc_2_3@@QAEXPAVDOMAttr@2@@Z 120c5010 f   DOMNodeIDMap.obj
 0001:000c4070       ?find@DOMNodeIDMap@xercesc_2_3@@QAEPAVDOMAttr@2@PBG@Z 120c5070 f   DOMNodeIDMap.obj
 0001:000c4110       ?growTable@DOMNodeIDMap@xercesc_2_3@@AAEXXZ 120c5110 f   DOMNodeIDMap.obj
 0001:000c4250       ??0DOMNodeImpl@xercesc_2_3@@QAE@PAVDOMNode@1@@Z 120c5250 f   DOMNodeImpl.obj
 0001:000c4270       ??0DOMNodeImpl@xercesc_2_3@@QAE@ABV01@@Z 120c5270 f   DOMNodeImpl.obj
 0001:000c4300       ?getChildNodes@DOMNodeImpl@xercesc_2_3@@QBEPAVDOMNodeList@2@XZ 120c5300 f   DOMNodeImpl.obj
 0001:000c4440       ?getOwnerDocument@DOMNodeImpl@xercesc_2_3@@QBEPAVDOMDocument@2@XZ 120c5440 f   DOMNodeImpl.obj
 0001:000c4490       ?setOwnerDocument@DOMNodeImpl@xercesc_2_3@@QAEXPAVDOMDocument@2@@Z 120c5490 f   DOMNodeImpl.obj
 0001:000c44c0       ?isDocumentTypeImpl@NodeImpl@xercesc_2_3@@UAE_NXZ 120c54c0 f   DOMNodeImpl.obj
 0001:000c44c0       ?isAttrImpl@NodeImpl@xercesc_2_3@@UAE_NXZ 120c54c0 f   DOMNodeImpl.obj
 0001:000c44c0       ?hasChildNodes@NodeImpl@xercesc_2_3@@UAE_NXZ 120c54c0 f   DOMNodeImpl.obj
 0001:000c44c0       ?hasChildNodes@DOMNodeImpl@xercesc_2_3@@QBE_NXZ 120c54c0 f   DOMNodeImpl.obj
 0001:000c44c0       ?isEntityReference@NodeImpl@xercesc_2_3@@UAE_NXZ 120c54c0 f   DOMNodeImpl.obj
 0001:000c44c0       ?isElementImpl@NodeImpl@xercesc_2_3@@UAE_NXZ 120c54c0 f   DOMNodeImpl.obj
 0001:000c44c0       ?isDocumentFragmentImpl@NodeImpl@xercesc_2_3@@UAE_NXZ 120c54c0 f   DOMNodeImpl.obj
 0001:000c44c0       ?requiresNamespaces@DTDValidator@xercesc_2_3@@UBE_NXZ 120c54c0 f   DOMNodeImpl.obj
 0001:000c44c0       ?hasAttributes@NodeImpl@xercesc_2_3@@UAE_NXZ 120c54c0 f   DOMNodeImpl.obj
 0001:000c44c0       ?hasAttributes@DOMNodeImpl@xercesc_2_3@@QBE_NXZ 120c54c0 f   DOMNodeImpl.obj
 0001:000c44c0       ?isTextImpl@NodeImpl@xercesc_2_3@@UAE_NXZ 120c54c0 f   DOMNodeImpl.obj
 0001:000c44c0       ?isDocumentImpl@NodeImpl@xercesc_2_3@@UAE_NXZ 120c54c0 f   DOMNodeImpl.obj
 0001:000c44c0       ?isCDATASectionImpl@NodeImpl@xercesc_2_3@@UAE_NXZ 120c54c0 f   DOMNodeImpl.obj
 0001:000c44d0       ?removeChild@DOMNodeImpl@xercesc_2_3@@QAEPAVDOMNode@2@PAV32@@Z 120c54d0 f   DOMNodeImpl.obj
 0001:000c44f0       ?appendChild@DOMNodeImpl@xercesc_2_3@@QAEPAVDOMNode@2@PAV32@@Z 120c54f0 f   DOMNodeImpl.obj
 0001:000c44f0       ?insertBefore@DOMNodeImpl@xercesc_2_3@@QAEPAVDOMNode@2@PAV32@0@Z 120c54f0 f   DOMNodeImpl.obj
 0001:000c44f0       ?replaceChild@DOMNodeImpl@xercesc_2_3@@QAEPAVDOMNode@2@PAV32@0@Z 120c54f0 f   DOMNodeImpl.obj
 0001:000c4510       ?checkAdditionalFacet@ListDatatypeValidator@xercesc_2_3@@MBEXQBG@Z 120c5510 f   DOMNodeImpl.obj
 0001:000c4510       ?checkAdditionalFacet@Base64BinaryDatatypeValidator@xercesc_2_3@@MBEXQBG@Z 120c5510 f   DOMNodeImpl.obj
 0001:000c4510       ?checkAdditionalFacet@HexBinaryDatatypeValidator@xercesc_2_3@@MBEXQBG@Z 120c5510 f   DOMNodeImpl.obj
 0001:000c4510       ?setNodeValue@DOMNodeImpl@xercesc_2_3@@QAEXPBG@Z 120c5510 f   DOMNodeImpl.obj
 0001:000c4510       ?startAttList@DOMParser@xercesc_2_3@@UAEXABVDTDElementDecl@2@@Z 120c5510 f   DOMNodeImpl.obj
 0001:000c4510       ?startAttList@SAX2XMLReaderImpl@xercesc_2_3@@UAEXABVDTDElementDecl@2@@Z 120c5510 f   DOMNodeImpl.obj
 0001:000c4510       ?setLanguageName@XMLMsgLoader@xercesc_2_3@@IAEXQAG@Z 120c5510 f   DOMNodeImpl.obj
 0001:000c4510       ?endInputSource@SAXParser@xercesc_2_3@@UAEXABVInputSource@2@@Z 120c5510 f   DOMNodeImpl.obj
 0001:000c4510       ?checkBlockSize@XMLTranscoder@xercesc_2_3@@IAEXI@Z 120c5510 f   DOMNodeImpl.obj
 0001:000c4510       ?doctypeComment@SAXParser@xercesc_2_3@@UAEXQBG@Z 120c5510 f   DOMNodeImpl.obj
 0001:000c4510       ?checkValueSpace@StringDatatypeValidator@xercesc_2_3@@MAEXQBG@Z 120c5510 f   DOMNodeImpl.obj
 0001:000c4510       ?startInputSource@SAX2XMLReaderImpl@xercesc_2_3@@UAEXABVInputSource@2@@Z 120c5510 f   DOMNodeImpl.obj
 0001:000c4510       ?checkAdditionalFacet@QNameDatatypeValidator@xercesc_2_3@@MBEXQBG@Z 120c5510 f   DOMNodeImpl.obj
 0001:000c4510       ?startAttList@SAXParser@xercesc_2_3@@UAEXABVDTDElementDecl@2@@Z 120c5510 f   DOMNodeImpl.obj
 0001:000c4510       ?endInputSource@SAX2XMLReaderImpl@xercesc_2_3@@UAEXABVInputSource@2@@Z 120c5510 f   DOMNodeImpl.obj
 0001:000c4510       ?checkAdditionalFacet@AnyURIDatatypeValidator@xercesc_2_3@@MBEXQBG@Z 120c5510 f   DOMNodeImpl.obj
 0001:000c4510       ?setNodeValue@NodeImpl@xercesc_2_3@@UAEXABVDOMString@2@@Z 120c5510 f   DOMNodeImpl.obj
 0001:000c4510       ?startInputSource@SAXParser@xercesc_2_3@@UAEXABVInputSource@2@@Z 120c5510 f   DOMNodeImpl.obj
 0001:000c4510       ?endAttList@SAXParser@xercesc_2_3@@UAEXABVDTDElementDecl@2@@Z 120c5510 f   DOMNodeImpl.obj
 0001:000c4510       ?normalizeContent@AbstractStringValidator@xercesc_2_3@@MBEXQAG@Z 120c5510 f   DOMNodeImpl.obj
 0001:000c4510       ?checkAdditionalFacet@NOTATIONDatatypeValidator@xercesc_2_3@@MBEXQBG@Z 120c5510 f   DOMNodeImpl.obj
 0001:000c4510       ?checkValueSpace@ListDatatypeValidator@xercesc_2_3@@MAEXQBG@Z 120c5510 f   DOMNodeImpl.obj
 0001:000c4510       ?endAttList@SAX2XMLReaderImpl@xercesc_2_3@@UAEXABVDTDElementDecl@2@@Z 120c5510 f   DOMNodeImpl.obj
 0001:000c4520       ?setReadOnly@DOMNodeImpl@xercesc_2_3@@QAEX_N0@Z 120c5520 f   DOMNodeImpl.obj
 0001:000c45d0       ?isSupported@DOMNodeImpl@xercesc_2_3@@QBE_NPBG0@Z 120c55d0 f   DOMNodeImpl.obj
 0001:000c45f0       ?setPrefix@DOMNodeImpl@xercesc_2_3@@QAEXPBG@Z 120c55f0 f   DOMNodeImpl.obj
 0001:000c4610       ?getXmlString@DOMNodeImpl@xercesc_2_3@@SAPBGXZ 120c5610 f   DOMNodeImpl.obj
 0001:000c4620       ?getXmlURIString@DOMNodeImpl@xercesc_2_3@@SAPBGXZ 120c5620 f   DOMNodeImpl.obj
 0001:000c4630       ?getXmlnsString@DOMNodeImpl@xercesc_2_3@@SAPBGXZ 120c5630 f   DOMNodeImpl.obj
 0001:000c4640       ?getXmlnsURIString@DOMNodeImpl@xercesc_2_3@@SAPBGXZ 120c5640 f   DOMNodeImpl.obj
 0001:000c4650       ?mapPrefix@DOMNodeImpl@xercesc_2_3@@SAPBGPBG0F@Z 120c5650 f   DOMNodeImpl.obj
 0001:000c4810       ?setUserData@DOMNodeImpl@xercesc_2_3@@QAEPAXPBGPAXPAVDOMUserDataHandler@2@@Z 120c5810 f   DOMNodeImpl.obj
 0001:000c48a0       ?getUserData@DOMNodeImpl@xercesc_2_3@@QBEPAXPBG@Z 120c58a0 f   DOMNodeImpl.obj
 0001:000c4950       ?callUserDataHandlers@DOMNodeImpl@xercesc_2_3@@QBEXW4DOMOperationType@DOMUserDataHandler@2@PBVDOMNode@2@1@Z 120c5950 f   DOMNodeImpl.obj
 0001:000c4a00       ?isSameNode@DOMNodeImpl@xercesc_2_3@@QBE_NPBVDOMNode@2@@Z 120c5a00 f   DOMNodeImpl.obj
 0001:000c4a10       ?isEqualNode@DOMNodeImpl@xercesc_2_3@@QBE_NPBVDOMNode@2@@Z 120c5a10 f   DOMNodeImpl.obj
 0001:000c4c60       ?lookupNamespacePrefix@DOMNodeImpl@xercesc_2_3@@QBEPBGPBG_N@Z 120c5c60 f   DOMNodeImpl.obj
 0001:000c4d50       ?getElementAncestor@DOMNodeImpl@xercesc_2_3@@QBEPAVDOMNode@2@PBV32@@Z 120c5d50 f   DOMNodeImpl.obj
 0001:000c4d90       ?lookupNamespacePrefix@DOMNodeImpl@xercesc_2_3@@QBEPBGQBG_NPAVDOMElement@2@@Z 120c5d90 f   DOMNodeImpl.obj
 0001:000c50b0       ?lookupNamespaceURI@DOMNodeImpl@xercesc_2_3@@QBEPBGPBG@Z 120c60b0 f   DOMNodeImpl.obj
 0001:000c5440       ?getBaseURI@DOMNodeImpl@xercesc_2_3@@QBEPBGXZ 120c6440 f   DOMNodeImpl.obj
 0001:000c5460       ?compareTreePosition@DOMNodeImpl@xercesc_2_3@@QBEFPBVDOMNode@2@@Z 120c6460 f   DOMNodeImpl.obj
 0001:000c5730       ?reverseTreeOrderBitPattern@DOMNodeImpl@xercesc_2_3@@QBEFF@Z 120c6730 f   DOMNodeImpl.obj
 0001:000c5760       ?getTextContent@DOMNodeImpl@xercesc_2_3@@QBEPBGXZ 120c6760 f   DOMNodeImpl.obj
 0001:000c57f0       ?getTextContent@DOMNodeImpl@xercesc_2_3@@QBEPBGPAGAAI@Z 120c67f0 f   DOMNodeImpl.obj
 0001:000c5940       ?isDefaultNamespace@DOMNodeImpl@xercesc_2_3@@QBE_NPBG@Z 120c6940 f   DOMNodeImpl.obj
 0001:000c5b50       ?release@DOMNodeImpl@xercesc_2_3@@QAEXXZ 120c6b50 f   DOMNodeImpl.obj
 0001:000c5b70       ??0DOMNodeIteratorImpl@xercesc_2_3@@QAE@PAVDOMDocument@1@PAVDOMNode@1@KPAVDOMNodeFilter@1@_N@Z 120c6b70 f   DOMNodeIteratorImpl.obj
 0001:000c5bb0       ??_EDOMNodeIteratorImpl@xercesc_2_3@@UAEPAXI@Z 120c6bb0 f i DOMNodeIteratorImpl.obj
 0001:000c5c10       ??0DOMNodeIteratorImpl@xercesc_2_3@@QAE@ABV01@@Z 120c6c10 f   DOMNodeIteratorImpl.obj
 0001:000c5c60       ??4DOMNodeIteratorImpl@xercesc_2_3@@QAEAAV01@ABV01@@Z 120c6c60 f   DOMNodeIteratorImpl.obj
 0001:000c5ca0       ??1DOMNodeIteratorImpl@xercesc_2_3@@UAE@XZ 120c6ca0 f   DOMNodeIteratorImpl.obj
 0001:000c5cb0       ?detach@DOMNodeIteratorImpl@xercesc_2_3@@UAEXXZ 120c6cb0 f   DOMNodeIteratorImpl.obj
 0001:000c5cd0       ?getExpandEntityReferences@DOMTreeWalkerImpl@xercesc_2_3@@UAE_NXZ 120c6cd0 f   DOMNodeIteratorImpl.obj
 0001:000c5cd0       ?getExpandEntityReferences@DOMNodeIteratorImpl@xercesc_2_3@@UAE_NXZ 120c6cd0 f   DOMNodeIteratorImpl.obj
 0001:000c5cd0       ?getExpandEntityReferences@NodeIteratorImpl@xercesc_2_3@@QAE_NXZ 120c6cd0 f   DOMNodeIteratorImpl.obj
 0001:000c5ce0       ?nextNode@DOMNodeIteratorImpl@xercesc_2_3@@UAEPAVDOMNode@2@XZ 120c6ce0 f   DOMNodeIteratorImpl.obj
 0001:000c5dc0       ?previousNode@DOMNodeIteratorImpl@xercesc_2_3@@UAEPAVDOMNode@2@XZ 120c6dc0 f   DOMNodeIteratorImpl.obj
 0001:000c5f30       ?acceptNode@DOMNodeIteratorImpl@xercesc_2_3@@AAE_NPAVDOMNode@2@@Z 120c6f30 f   DOMNodeIteratorImpl.obj
 0001:000c5fd0       ?matchNodeOrParent@DOMNodeIteratorImpl@xercesc_2_3@@AAEPAVDOMNode@2@PAV32@@Z 120c6fd0 f   DOMNodeIteratorImpl.obj
 0001:000c6000       ?nextNode@DOMNodeIteratorImpl@xercesc_2_3@@AAEPAVDOMNode@2@PAV32@_N@Z 120c7000 f   DOMNodeIteratorImpl.obj
 0001:000c60b0       ?previousNode@DOMNodeIteratorImpl@xercesc_2_3@@AAEPAVDOMNode@2@PAV32@@Z 120c70b0 f   DOMNodeIteratorImpl.obj
 0001:000c6140       ?removeNode@DOMNodeIteratorImpl@xercesc_2_3@@QAEXPAVDOMNode@2@@Z 120c7140 f   DOMNodeIteratorImpl.obj
 0001:000c6300       ?release@DOMNodeIteratorImpl@xercesc_2_3@@UAEXXZ 120c7300 f   DOMNodeIteratorImpl.obj
 0001:000c6310       ??0DOMNodeListImpl@xercesc_2_3@@QAE@PAVDOMNode@1@@Z 120c7310 f   DOMNodeListImpl.obj
 0001:000c6330       ??_EDOMNodeListImpl@xercesc_2_3@@UAEPAXI@Z 120c7330 f i DOMNodeListImpl.obj
 0001:000c6390       ?getLength@DOMNodeListImpl@xercesc_2_3@@UBEKXZ 120c7390 f   DOMNodeListImpl.obj
 0001:000c63c0       ?item@DOMNodeListImpl@xercesc_2_3@@UBEPAVDOMNode@2@K@Z 120c73c0 f   DOMNodeListImpl.obj
 0001:000c6400       ??0DOMNodeVector@xercesc_2_3@@QAE@PAVDOMDocument@1@@Z 120c7400 f   DOMNodeVector.obj
 0001:000c6440       ??0DOMNodeVector@xercesc_2_3@@QAE@PAVDOMDocument@1@K@Z 120c7440 f   DOMNodeVector.obj
 0001:000c6480       ?addElement@DOMNodeVector@xercesc_2_3@@QAEXPAVDOMNode@2@@Z 120c7480 f   DOMNodeVector.obj
 0001:000c64f0       ?elementAt@NodeVector@xercesc_2_3@@QAEPAVNodeImpl@2@I@Z 120c74f0 f   DOMNodeVector.obj
 0001:000c64f0       ?elementAt@DOMNodeVector@xercesc_2_3@@QAEPAVDOMNode@2@K@Z 120c74f0 f   DOMNodeVector.obj
 0001:000c6510       ?insertElementAt@DOMNodeVector@xercesc_2_3@@QAEXPAVDOMNode@2@K@Z 120c7510 f   DOMNodeVector.obj
 0001:000c65a0       ?reset@NodeVector@xercesc_2_3@@QAEXXZ 120c75a0 f   DOMNodeVector.obj
 0001:000c65a0       ?reset@DOMNodeVector@xercesc_2_3@@QAEXXZ 120c75a0 f   DOMNodeVector.obj
 0001:000c65b0       ?setElementAt@DOMNodeVector@xercesc_2_3@@QAEXPAVDOMNode@2@K@Z 120c75b0 f   DOMNodeVector.obj
 0001:000c65b0       ?setElementAt@NodeVector@xercesc_2_3@@QAEXPAVNodeImpl@2@I@Z 120c75b0 f   DOMNodeVector.obj
 0001:000c6600       ?reinitMsgLoader@DOMNormalizer@xercesc_2_3@@SAXXZ 120c7600 f   DOMNormalizer.obj
 0001:000c6620       ?reinitNormalizerMutex@DOMNormalizer@xercesc_2_3@@SAXXZ 120c7620 f   DOMNormalizer.obj
 0001:000c6650       ??0DOMNormalizer@xercesc_2_3@@QAE@QAVMemoryManager@1@@Z 120c7650 f   DOMNormalizer.obj
 0001:000c6770       ??1DOMNormalizer@xercesc_2_3@@QAE@XZ 120c7770 f   DOMNormalizer.obj
 0001:000c6790       ?normalizeDocument@DOMNormalizer@xercesc_2_3@@QAEXPAVDOMDocumentImpl@2@@Z 120c7790 f   DOMNormalizer.obj
 0001:000c6810       ?normalizeNode@DOMNormalizer@xercesc_2_3@@ABEPAVDOMNode@2@PAV32@@Z 120c7810 f   DOMNormalizer.obj
 0001:000c6b90       ?namespaceFixUp@DOMNormalizer@xercesc_2_3@@ABEXPAVDOMElementImpl@2@@Z 120c7b90 f   DOMNormalizer.obj
 0001:000c71a0       ?integerToXMLCh@DOMNormalizer@xercesc_2_3@@ABEPBGI@Z 120c81a0 f   DOMNormalizer.obj
 0001:000c7290       ?addOrChangeNamespaceDecl@DOMNormalizer@xercesc_2_3@@ABEXPBG0PAVDOMElementImpl@2@@Z 120c8290 f   DOMNormalizer.obj
 0001:000c7410       ?addCustomNamespaceDecl@DOMNormalizer@xercesc_2_3@@ABEPBGPBGPAVDOMElementImpl@2@@Z 120c8410 f   DOMNormalizer.obj
 0001:000c76c0       ?addOrChangeBinding@InScopeNamespaces@DOMNormalizer@xercesc_2_3@@QAEXPBG0QAVMemoryManager@3@@Z 120c86c0 f   DOMNormalizer.obj
 0001:000c7730       ?addScope@InScopeNamespaces@DOMNormalizer@xercesc_2_3@@QAEXQAVMemoryManager@3@@Z 120c8730 f   DOMNormalizer.obj
 0001:000c77e0       ?addOrChangeBinding@Scope@InScopeNamespaces@DOMNormalizer@xercesc_2_3@@QAEXPBG0QAVMemoryManager@4@@Z 120c87e0 f   DOMNormalizer.obj
 0001:000c7bb0       ?getUri@Scope@InScopeNamespaces@DOMNormalizer@xercesc_2_3@@QBEPBGPBG@Z 120c8bb0 f   DOMNormalizer.obj
 0001:000c7c60       ?getPrefix@Scope@InScopeNamespaces@DOMNormalizer@xercesc_2_3@@QBEPBGPBG@Z 120c8c60 f   DOMNormalizer.obj
 0001:000c7d10       ?error@DOMNormalizer@xercesc_2_3@@ABEXW4Codes@XMLErrs@2@PBVDOMNode@2@@Z 120c8d10 f   DOMNormalizer.obj
 0001:000c7f70       ??1?$XMLEnumerator@G@xercesc_2_3@@UAE@XZ 120c8f70 f i DOMNormalizer.obj
 0001:000c7f80       ??_G?$XMLEnumerator@G@xercesc_2_3@@UAEPAXI@Z 120c8f80 f i DOMNormalizer.obj
 0001:000c7f80       ??_E?$XMLEnumerator@G@xercesc_2_3@@UAEPAXI@Z 120c8f80 f i DOMNormalizer.obj
 0001:000c7fa0       ?put@?$RefHashTableOf@G@xercesc_2_3@@QAEXPAXQAG@Z 120c8fa0 f i DOMNormalizer.obj
 0001:000c81b0       ??1?$RefHashTableOfEnumerator@G@xercesc_2_3@@UAE@XZ 120c91b0 f i DOMNormalizer.obj
 0001:000c82a0       ?nextElementKey@?$RefHashTableOfEnumerator@G@xercesc_2_3@@QAEPAXXZ 120c92a0 f i DOMNormalizer.obj
 0001:000c8320       ??_E?$RefVectorOf@VScope@InScopeNamespaces@DOMNormalizer@xercesc_2_3@@@xercesc_2_3@@UAEPAXI@Z 120c9320 f i DOMNormalizer.obj
 0001:000c8320       ??_G?$RefVectorOf@VScope@InScopeNamespaces@DOMNormalizer@xercesc_2_3@@@xercesc_2_3@@UAEPAXI@Z 120c9320 f i DOMNormalizer.obj
 0001:000c8340       ??1?$RefVectorOf@VScope@InScopeNamespaces@DOMNormalizer@xercesc_2_3@@@xercesc_2_3@@UAE@XZ 120c9340 f i DOMNormalizer.obj
 0001:000c8490       ??1?$BaseRefVectorOf@VScope@InScopeNamespaces@DOMNormalizer@xercesc_2_3@@@xercesc_2_3@@UAE@XZ 120c9490 f i DOMNormalizer.obj
 0001:000c84a0       ??_G?$RefHashTableOfEnumerator@G@xercesc_2_3@@UAEPAXI@Z 120c94a0 f i DOMNormalizer.obj
 0001:000c84a0       ??_E?$RefHashTableOfEnumerator@G@xercesc_2_3@@UAEPAXI@Z 120c94a0 f i DOMNormalizer.obj
 0001:000c84c0       ?removeAll@?$RefHashTableOf@G@xercesc_2_3@@QAEXXZ 120c94c0 f i DOMNormalizer.obj
 0001:000c8530       ?removeBucketElem@?$RefHashTableOf@G@xercesc_2_3@@AAEXQBXAAI@Z 120c9530 f i DOMNormalizer.obj
 0001:000c8610       ?rehash@?$RefHashTableOf@X@xercesc_2_3@@AAEXXZ 120c9610 f i DOMNormalizer.obj
 0001:000c8610       ?rehash@?$RefHashTableOf@VDatatypeValidator@xercesc_2_3@@@xercesc_2_3@@AAEXXZ 120c9610 f i DOMNormalizer.obj
 0001:000c8610       ?rehash@?$RefHashTableOf@VCPMapEntry@xercesc_2_3@@@xercesc_2_3@@AAEXXZ 120c9610 f i DOMNormalizer.obj
 0001:000c8610       ?rehash@?$RefHashTableOf@VValueStore@xercesc_2_3@@@xercesc_2_3@@AAEXXZ 120c9610 f i DOMNormalizer.obj
 0001:000c8610       ?rehash@?$RefHashTableOf@VSchemaInfo@xercesc_2_3@@@xercesc_2_3@@AAEXXZ 120c9610 f i DOMNormalizer.obj
 0001:000c8610       ?rehash@?$RefHashTableOf@G@xercesc_2_3@@AAEXXZ 120c9610 f i DOMNormalizer.obj
 0001:000c8610       ?rehash@?$RefHashTableOf@VXercesAttGroupInfo@xercesc_2_3@@@xercesc_2_3@@AAEXXZ 120c9610 f i DOMNormalizer.obj
 0001:000c8610       ?rehash@?$RefHashTableOf@V?$KeyRefPair@XVDOMUserDataHandler@xercesc_2_3@@@xercesc_2_3@@@xercesc_2_3@@AAEXXZ 120c9610 f i DOMNormalizer.obj
 0001:000c8610       ?rehash@?$RefHashTableOf@VXMLRefInfo@xercesc_2_3@@@xercesc_2_3@@AAEXXZ 120c9610 f i DOMNormalizer.obj
 0001:000c8610       ?rehash@?$RefHashTableOf@V?$RefHashTableOf@V?$KeyRefPair@XVDOMUserDataHandler@xercesc_2_3@@@xercesc_2_3@@@xercesc_2_3@@@xercesc_2_3@@AAEXXZ 120c9610 f i DOMNormalizer.obj
 0001:000c8610       ?rehash@?$RefHashTableOf@VKVStringPair@xercesc_2_3@@@xercesc_2_3@@AAEXXZ 120c9610 f i DOMNormalizer.obj
 0001:000c8610       ?rehash@?$RefHashTableOf@VComplexTypeInfo@xercesc_2_3@@@xercesc_2_3@@AAEXXZ 120c9610 f i DOMNormalizer.obj
 0001:000c8610       ?rehash@?$RefHashTableOf@VENameMap@xercesc_2_3@@@xercesc_2_3@@AAEXXZ 120c9610 f i DOMNormalizer.obj
 0001:000c8610       ?rehash@?$RefHashTableOf@VXMLElementDecl@xercesc_2_3@@@xercesc_2_3@@AAEXXZ 120c9610 f i DOMNormalizer.obj
 0001:000c8610       ?rehash@?$RefHashTableOf@VXercesGroupInfo@xercesc_2_3@@@xercesc_2_3@@AAEXXZ 120c9610 f i DOMNormalizer.obj
 0001:000c86f0       ??0DOMNotationImpl@xercesc_2_3@@QAE@PAVDOMDocument@1@PBG@Z 120c96f0 f   DOMNotationImpl.obj
 0001:000c8780       ??_EDOMNotationImpl@xercesc_2_3@@UAEPAXI@Z 120c9780 f i DOMNotationImpl.obj
 0001:000c87e0       ??0DOMNotationImpl@xercesc_2_3@@QAE@ABV01@_N@Z 120c97e0 f   DOMNotationImpl.obj
 0001:000c8860       ??1DOMNotationImpl@xercesc_2_3@@UAE@XZ 120c9860 f   DOMNotationImpl.obj
 0001:000c88b0       ?cloneNode@DOMNotationImpl@xercesc_2_3@@UBEPAVDOMNode@2@_N@Z 120c98b0 f   DOMNotationImpl.obj
 0001:000c8970       ?getNodeType@DOMNotationImpl@xercesc_2_3@@UBEFXZ 120c9970 f   DOMNotationImpl.obj
 0001:000c8970       ?getNodeType@NotationImpl@xercesc_2_3@@UAEFXZ 120c9970 f   DOMNotationImpl.obj
 0001:000c8980       ?getAttributes@ElementDefinitionImpl@xercesc_2_3@@UAEPAVNamedNodeMapImpl@2@XZ 120c9980 f   DOMNotationImpl.obj
 0001:000c8980       ?getSystemId@DOMNotationImpl@xercesc_2_3@@UBEPBGXZ 120c9980 f   DOMNotationImpl.obj
 0001:000c8980       ?getNextSibling@ChildNode@xercesc_2_3@@UAEPAVNodeImpl@2@XZ 120c9980 f   DOMNotationImpl.obj
 0001:000c8980       ?getSystemId@SAXParseException@xercesc_2_3@@QBEPBGXZ 120c9980 f   DOMNotationImpl.obj
 0001:000c8980       ?getData2@ModifierOp@xercesc_2_3@@UBEHXZ 120c9980 f   DOMNotationImpl.obj
 0001:000c8980       ?getFilter@DOMWriterImpl@xercesc_2_3@@UBEPAVDOMWriterFilter@2@XZ 120c9980 f   DOMNotationImpl.obj
 0001:000c8980       ?getEndOffset@RangeImpl@xercesc_2_3@@QBEIXZ 120c9980 f   DOMNotationImpl.obj
 0001:000c8980       ?getYesFlow@ConditionOp@xercesc_2_3@@UBEPBVOp@2@XZ 120c9980 f   DOMNotationImpl.obj
 0001:000c8990       ?setPublicId@DOMNotationImpl@xercesc_2_3@@UAEXPBG@Z 120c9990 f   DOMNotationImpl.obj
 0001:000c89e0       ?setSystemId@DOMNotationImpl@xercesc_2_3@@UAEXPBG@Z 120c99e0 f   DOMNotationImpl.obj
 0001:000c8a30       ?release@DOMNotationImpl@xercesc_2_3@@UAEXXZ 120c9a30 f   DOMNotationImpl.obj
 0001:000c8ab0       ?setBaseURI@DOMNotationImpl@xercesc_2_3@@UAEXPBG@Z 120c9ab0 f   DOMNotationImpl.obj
 0001:000c8b10       ?getURI@CMAny@xercesc_2_3@@QBEIXZ 120c9b10 f   DOMNotationImpl.obj
 0001:000c8b10       ?getChild@CMUnaryOp@xercesc_2_3@@QAEPAVCMNode@2@XZ 120c9b10 f   DOMNotationImpl.obj
 0001:000c8b10       ?getNoFlow@ConditionOp@xercesc_2_3@@UBEPBVOp@2@XZ 120c9b10 f   DOMNotationImpl.obj
 0001:000c8b10       ?getOwnerDocument@ParentNode@xercesc_2_3@@UAEPAVDocumentImpl@2@XZ 120c9b10 f   DOMNotationImpl.obj
 0001:000c8b10       ?getDocument@DOMRangeImpl@xercesc_2_3@@QAEPAVDOMDocument@2@XZ 120c9b10 f   DOMNotationImpl.obj
 0001:000c8b10       ?getDocument@ParentNode@xercesc_2_3@@UAEPAVDocumentImpl@2@XZ 120c9b10 f   DOMNotationImpl.obj
 0001:000c8b10       ?getLeft@CMBinaryOp@xercesc_2_3@@QAEPAVCMNode@2@XZ 120c9b10 f   DOMNotationImpl.obj
 0001:000c8b10       ?getSign@XMLAbstractDoubleFloat@xercesc_2_3@@UBEHXZ 120c9b10 f   DOMNotationImpl.obj
 0001:000c8b10       ?getBaseURI@DOMNotationImpl@xercesc_2_3@@UBEPBGXZ 120c9b10 f   DOMNotationImpl.obj
 0001:000c8b20       ?insertBefore@DOMCommentImpl@xercesc_2_3@@UAEPAVDOMNode@2@PAV32@0@Z 120c9b20 f   DOMNotationImpl.obj
 0001:000c8b20       ?replaceChild@DOMNotationImpl@xercesc_2_3@@UAEPAVDOMNode@2@PAV32@0@Z 120c9b20 f   DOMNotationImpl.obj
 0001:000c8b20       ?insertBefore@DOMProcessingInstructionImpl@xercesc_2_3@@UAEPAVDOMNode@2@PAV32@0@Z 120c9b20 f   DOMNotationImpl.obj
 0001:000c8b20       ?replaceChild@DOMTextImpl@xercesc_2_3@@UAEPAVDOMNode@2@PAV32@0@Z 120c9b20 f   DOMNotationImpl.obj
 0001:000c8b20       ?replaceChild@DOMCommentImpl@xercesc_2_3@@UAEPAVDOMNode@2@PAV32@0@Z 120c9b20 f   DOMNotationImpl.obj
 0001:000c8b20       ?replaceChild@DOMProcessingInstructionImpl@xercesc_2_3@@UAEPAVDOMNode@2@PAV32@0@Z 120c9b20 f   DOMNotationImpl.obj
 0001:000c8b20       ?insertBefore@DOMNotationImpl@xercesc_2_3@@UAEPAVDOMNode@2@PAV32@0@Z 120c9b20 f   DOMNotationImpl.obj
 0001:000c8b20       ?insertBefore@DOMTextImpl@xercesc_2_3@@UAEPAVDOMNode@2@PAV32@0@Z 120c9b20 f   DOMNotationImpl.obj
 0001:000c8b40       ?isSupported@DOMEntityImpl@xercesc_2_3@@UBE_NPBG0@Z 120c9b40 f   DOMNotationImpl.obj
 0001:000c8b40       ?isSupported@DOMTextImpl@xercesc_2_3@@UBE_NPBG0@Z 120c9b40 f   DOMNotationImpl.obj
 0001:000c8b40       ?isSupported@DOMAttrImpl@xercesc_2_3@@UBE_NPBG0@Z 120c9b40 f   DOMNotationImpl.obj
 0001:000c8b40       ?isSupported@DOMDocumentImpl@xercesc_2_3@@UBE_NPBG0@Z 120c9b40 f   DOMNotationImpl.obj
 0001:000c8b40       ?isSupported@DOMDocumentFragmentImpl@xercesc_2_3@@UBE_NPBG0@Z 120c9b40 f   DOMNotationImpl.obj
 0001:000c8b40       ?isSupported@DOMCDATASectionImpl@xercesc_2_3@@UBE_NPBG0@Z 120c9b40 f   DOMNotationImpl.obj
 0001:000c8b40       ?isSupported@DOMElementImpl@xercesc_2_3@@UBE_NPBG0@Z 120c9b40 f   DOMNotationImpl.obj
 0001:000c8b40       ?isSupported@DOMEntityReferenceImpl@xercesc_2_3@@UBE_NPBG0@Z 120c9b40 f   DOMNotationImpl.obj
 0001:000c8b40       ?isSupported@DOMProcessingInstructionImpl@xercesc_2_3@@UBE_NPBG0@Z 120c9b40 f   DOMNotationImpl.obj
 0001:000c8b40       ?isSupported@DOMNotationImpl@xercesc_2_3@@UBE_NPBG0@Z 120c9b40 f   DOMNotationImpl.obj
 0001:000c8b40       ?isSupported@DOMCommentImpl@xercesc_2_3@@UBE_NPBG0@Z 120c9b40 f   DOMNotationImpl.obj
 0001:000c8b40       ?isSupported@DOMDocumentTypeImpl@xercesc_2_3@@UBE_NPBG0@Z 120c9b40 f   DOMNotationImpl.obj
 0001:000c8b60       ?setUserData@DOMDocumentTypeImpl@xercesc_2_3@@UAEPAXPBGPAXPAVDOMUserDataHandler@2@@Z 120c9b60 f   DOMNotationImpl.obj
 0001:000c8b60       ?setUserData@DOMProcessingInstructionImpl@xercesc_2_3@@UAEPAXPBGPAXPAVDOMUserDataHandler@2@@Z 120c9b60 f   DOMNotationImpl.obj
 0001:000c8b60       ?setUserData@DOMEntityImpl@xercesc_2_3@@UAEPAXPBGPAXPAVDOMUserDataHandler@2@@Z 120c9b60 f   DOMNotationImpl.obj
 0001:000c8b60       ?setUserData@DOMAttrImpl@xercesc_2_3@@UAEPAXPBGPAXPAVDOMUserDataHandler@2@@Z 120c9b60 f   DOMNotationImpl.obj
 0001:000c8b60       ?setUserData@DOMTextImpl@xercesc_2_3@@UAEPAXPBGPAXPAVDOMUserDataHandler@2@@Z 120c9b60 f   DOMNotationImpl.obj
 0001:000c8b60       ?setUserData@DOMCommentImpl@xercesc_2_3@@UAEPAXPBGPAXPAVDOMUserDataHandler@2@@Z 120c9b60 f   DOMNotationImpl.obj
 0001:000c8b60       ?setUserData@DOMNotationImpl@xercesc_2_3@@UAEPAXPBGPAXPAVDOMUserDataHandler@2@@Z 120c9b60 f   DOMNotationImpl.obj
 0001:000c8b60       ?setUserData@DOMCDATASectionImpl@xercesc_2_3@@UAEPAXPBGPAXPAVDOMUserDataHandler@2@@Z 120c9b60 f   DOMNotationImpl.obj
 0001:000c8b60       ?setUserData@DOMElementImpl@xercesc_2_3@@UAEPAXPBGPAXPAVDOMUserDataHandler@2@@Z 120c9b60 f   DOMNotationImpl.obj
 0001:000c8b60       ?setUserData@DOMDocumentFragmentImpl@xercesc_2_3@@UAEPAXPBGPAXPAVDOMUserDataHandler@2@@Z 120c9b60 f   DOMNotationImpl.obj
 0001:000c8b60       ?setUserData@DOMEntityReferenceImpl@xercesc_2_3@@UAEPAXPBGPAXPAVDOMUserDataHandler@2@@Z 120c9b60 f   DOMNotationImpl.obj
 0001:000c8b60       ?setUserData@DOMDocumentImpl@xercesc_2_3@@UAEPAXPBGPAXPAVDOMUserDataHandler@2@@Z 120c9b60 f   DOMNotationImpl.obj
 0001:000c8b80       ?lookupNamespacePrefix@DOMTextImpl@xercesc_2_3@@UBEPBGPBG_N@Z 120c9b80 f   DOMNotationImpl.obj
 0001:000c8b80       ?lookupNamespacePrefix@DOMNotationImpl@xercesc_2_3@@UBEPBGPBG_N@Z 120c9b80 f   DOMNotationImpl.obj
 0001:000c8b80       ?lookupNamespacePrefix@DOMDocumentTypeImpl@xercesc_2_3@@UBEPBGPBG_N@Z 120c9b80 f   DOMNotationImpl.obj
 0001:000c8b80       ?lookupNamespacePrefix@DOMEntityReferenceImpl@xercesc_2_3@@UBEPBGPBG_N@Z 120c9b80 f   DOMNotationImpl.obj
 0001:000c8b80       ?lookupNamespacePrefix@DOMCommentImpl@xercesc_2_3@@UBEPBGPBG_N@Z 120c9b80 f   DOMNotationImpl.obj
 0001:000c8b80       ?lookupNamespacePrefix@DOMProcessingInstructionImpl@xercesc_2_3@@UBEPBGPBG_N@Z 120c9b80 f   DOMNotationImpl.obj
 0001:000c8b80       ?lookupNamespacePrefix@DOMEntityImpl@xercesc_2_3@@UBEPBGPBG_N@Z 120c9b80 f   DOMNotationImpl.obj
 0001:000c8b80       ?lookupNamespacePrefix@DOMAttrImpl@xercesc_2_3@@UBEPBGPBG_N@Z 120c9b80 f   DOMNotationImpl.obj
 0001:000c8b80       ?lookupNamespacePrefix@DOMCDATASectionImpl@xercesc_2_3@@UBEPBGPBG_N@Z 120c9b80 f   DOMNotationImpl.obj
 0001:000c8b80       ?lookupNamespacePrefix@DOMDocumentFragmentImpl@xercesc_2_3@@UBEPBGPBG_N@Z 120c9b80 f   DOMNotationImpl.obj
 0001:000c8b80       ?lookupNamespacePrefix@DOMElementImpl@xercesc_2_3@@UBEPBGPBG_N@Z 120c9b80 f   DOMNotationImpl.obj
 0001:000c8b80       ?lookupNamespacePrefix@DOMDocumentImpl@xercesc_2_3@@UBEPBGPBG_N@Z 120c9b80 f   DOMNotationImpl.obj
 0001:000c8ba0       ??0DOMParentNode@xercesc_2_3@@QAE@PAVDOMDocument@1@@Z 120c9ba0 f   DOMParentNode.obj
 0001:000c8bd0       ??0DOMParentNode@xercesc_2_3@@QAE@ABV01@@Z 120c9bd0 f   DOMParentNode.obj
 0001:000c8c00       ?changed@DOMParentNode@xercesc_2_3@@QAEXXZ 120c9c00 f   DOMParentNode.obj
 0001:000c8c10       ?changes@DOMParentNode@xercesc_2_3@@QBEHXZ 120c9c10 f   DOMParentNode.obj
 0001:000c8c20       ?appendChild@DOMParentNode@xercesc_2_3@@QAEPAVDOMNode@2@PAV32@@Z 120c9c20 f   DOMParentNode.obj
 0001:000c8c30       ?cloneChildren@DOMParentNode@xercesc_2_3@@QAEXPBVDOMNode@2@@Z 120c9c30 f   DOMParentNode.obj
 0001:000c8c70       ?getDocument@DOMParentNode@xercesc_2_3@@QBEPAVDOMDocument@2@XZ 120c9c70 f   DOMParentNode.obj
 0001:000c8c70       ?getOwnerDocument@DOMParentNode@xercesc_2_3@@QBEPAVDOMDocument@2@XZ 120c9c70 f   DOMParentNode.obj
 0001:000c8c80       ?setOwnerDocument@DOMParentNode@xercesc_2_3@@QAEXPAVDOMDocument@2@@Z 120c9c80 f   DOMParentNode.obj
 0001:000c8c90       ?getChildNodes@DOMParentNode@xercesc_2_3@@QBEPAVDOMNodeList@2@XZ 120c9c90 f   DOMParentNode.obj
 0001:000c8ca0       ?getLastChild@DOMParentNode@xercesc_2_3@@QBEPAVDOMNode@2@XZ 120c9ca0 f   DOMParentNode.obj
 0001:000c8ca0       ?lastChild@DOMParentNode@xercesc_2_3@@QBEPAVDOMNode@2@XZ 120c9ca0 f   DOMParentNode.obj
 0001:000c8cd0       ?lastChild@DOMParentNode@xercesc_2_3@@QAEXPAVDOMNode@2@@Z 120c9cd0 f   DOMParentNode.obj
 0001:000c8d00       ?hasChildNodes@DOMParentNode@xercesc_2_3@@QBE_NXZ 120c9d00 f   DOMParentNode.obj
 0001:000c8d10       ?insertBefore@DOMParentNode@xercesc_2_3@@QAEPAVDOMNode@2@PAV32@0@Z 120c9d10 f   DOMParentNode.obj
 0001:000c90b0       ?removeChild@DOMParentNode@xercesc_2_3@@QAEPAVDOMNode@2@PAV32@@Z 120ca0b0 f   DOMParentNode.obj
 0001:000c9310       ?replaceChild@DOMParentNode@xercesc_2_3@@QAEPAVDOMNode@2@PAV32@0@Z 120ca310 f   DOMParentNode.obj
 0001:000c9330       ?normalize@DOMParentNode@xercesc_2_3@@QAEXXZ 120ca330 f   DOMParentNode.obj
 0001:000c93b0       ?isEqualNode@DOMParentNode@xercesc_2_3@@QBE_NPBVDOMNode@2@@Z 120ca3b0 f   DOMParentNode.obj
 0001:000c9440       ?release@DOMParentNode@xercesc_2_3@@QAEXXZ 120ca440 f   DOMParentNode.obj
 0001:000c9480       ??0DOMProcessingInstructionImpl@xercesc_2_3@@QAE@PAVDOMDocument@1@PBG1@Z 120ca480 f   DOMProcessingInstructionImpl.obj
 0001:000c9530       ??_EDOMProcessingInstructionImpl@xercesc_2_3@@UAEPAXI@Z 120ca530 f i DOMProcessingInstructionImpl.obj
 0001:000c9590       ??0DOMProcessingInstructionImpl@xercesc_2_3@@QAE@ABV01@_N@Z 120ca590 f   DOMProcessingInstructionImpl.obj
 0001:000c9630       ??1DOMProcessingInstructionImpl@xercesc_2_3@@UAE@XZ 120ca630 f   DOMProcessingInstructionImpl.obj
 0001:000c96a0       ?cloneNode@DOMProcessingInstructionImpl@xercesc_2_3@@UBEPAVDOMNode@2@_N@Z 120ca6a0 f   DOMProcessingInstructionImpl.obj
 0001:000c9720       ?getNodeType@DOMProcessingInstructionImpl@xercesc_2_3@@UBEFXZ 120ca720 f   DOMProcessingInstructionImpl.obj
 0001:000c9720       ?getNodeType@ProcessingInstructionImpl@xercesc_2_3@@UAEFXZ 120ca720 f   DOMProcessingInstructionImpl.obj
 0001:000c9730       ?release@DOMProcessingInstructionImpl@xercesc_2_3@@UAEXXZ 120ca730 f   DOMProcessingInstructionImpl.obj
 0001:000c97c0       ?setBaseURI@DOMProcessingInstructionImpl@xercesc_2_3@@UAEXPBG@Z 120ca7c0 f   DOMProcessingInstructionImpl.obj
 0001:000c97e0       ?getBaseURI@DOMProcessingInstructionImpl@xercesc_2_3@@UBEPBGXZ 120ca7e0 f   DOMProcessingInstructionImpl.obj
 0001:000c97f0       ?splitText@DOMProcessingInstructionImpl@xercesc_2_3@@QAEPAVDOMProcessingInstruction@2@K@Z 120ca7f0 f   DOMProcessingInstructionImpl.obj
 0001:000c9940       ?deleteData@DOMCommentImpl@xercesc_2_3@@UAEXKK@Z 120ca940 f   DOMProcessingInstructionImpl.obj
 0001:000c9940       ?deleteData@DOMProcessingInstructionImpl@xercesc_2_3@@QAEXKK@Z 120ca940 f   DOMProcessingInstructionImpl.obj
 0001:000c9940       ?deleteData@DOMTextImpl@xercesc_2_3@@UAEXKK@Z 120ca940 f   DOMProcessingInstructionImpl.obj
 0001:000c9960       ?substringData@DOMTextImpl@xercesc_2_3@@UBEPBGKK@Z 120ca960 f   DOMProcessingInstructionImpl.obj
 0001:000c9960       ?substringData@DOMProcessingInstructionImpl@xercesc_2_3@@QBEPBGKK@Z 120ca960 f   DOMProcessingInstructionImpl.obj
 0001:000c9960       ?substringData@DOMCommentImpl@xercesc_2_3@@UBEPBGKK@Z 120ca960 f   DOMProcessingInstructionImpl.obj
 0001:000c9980       ?setData@DOMProcessingInstructionImpl@xercesc_2_3@@UAEXPBG@Z 120ca980 f   DOMProcessingInstructionImpl.obj
 0001:000c9980       ?setData@DOMTextImpl@xercesc_2_3@@UAEXPBG@Z 120ca980 f   DOMProcessingInstructionImpl.obj
 0001:000c9980       ?setData@DOMCommentImpl@xercesc_2_3@@UAEXPBG@Z 120ca980 f   DOMProcessingInstructionImpl.obj
 0001:000c99a0       ?setNodeValue@DOMProcessingInstructionImpl@xercesc_2_3@@UAEXPBG@Z 120ca9a0 f   DOMProcessingInstructionImpl.obj
 0001:000c99a0       ?setNodeValue@DOMTextImpl@xercesc_2_3@@UAEXPBG@Z 120ca9a0 f   DOMProcessingInstructionImpl.obj
 0001:000c99a0       ?setNodeValue@DOMCommentImpl@xercesc_2_3@@UAEXPBG@Z 120ca9a0 f   DOMProcessingInstructionImpl.obj
 0001:000c99c0       ??0DOMRangeImpl@xercesc_2_3@@QAE@PAVDOMDocument@1@@Z 120ca9c0 f   DOMRangeImpl.obj
 0001:000c9a10       ??_EDOMRangeImpl@xercesc_2_3@@UAEPAXI@Z 120caa10 f i DOMRangeImpl.obj
 0001:000c9a70       ??0DOMRangeImpl@xercesc_2_3@@QAE@ABV01@@Z 120caa70 f   DOMRangeImpl.obj
 0001:000c9ab0       ??1DOMRangeImpl@xercesc_2_3@@UAE@XZ 120caab0 f   DOMRangeImpl.obj
 0001:000c9ac0       ?getStartContainer@DOMRangeImpl@xercesc_2_3@@UBEPAVDOMNode@2@XZ 120caac0 f   DOMRangeImpl.obj
 0001:000c9af0       ?getStartOffset@DOMRangeImpl@xercesc_2_3@@UBEKXZ 120caaf0 f   DOMRangeImpl.obj
 0001:000c9b20       ?getEndContainer@DOMRangeImpl@xercesc_2_3@@UBEPAVDOMNode@2@XZ 120cab20 f   DOMRangeImpl.obj
 0001:000c9b50       ?getEndOffset@DOMRangeImpl@xercesc_2_3@@UBEKXZ 120cab50 f   DOMRangeImpl.obj
 0001:000c9b80       ?getCollapsed@DOMRangeImpl@xercesc_2_3@@UBE_NXZ 120cab80 f   DOMRangeImpl.obj
 0001:000c9bd0       ?setStartContainer@DOMRangeImpl@xercesc_2_3@@AAEXPBVDOMNode@2@@Z 120cabd0 f   DOMRangeImpl.obj
 0001:000c9c10       ?setStartOffset@DOMRangeImpl@xercesc_2_3@@AAEXK@Z 120cac10 f   DOMRangeImpl.obj
 0001:000c9c50       ?setEndContainer@DOMRangeImpl@xercesc_2_3@@AAEXPBVDOMNode@2@@Z 120cac50 f   DOMRangeImpl.obj
 0001:000c9c90       ?setEndOffset@DOMRangeImpl@xercesc_2_3@@AAEXK@Z 120cac90 f   DOMRangeImpl.obj
 0001:000c9cd0       ?setStart@DOMRangeImpl@xercesc_2_3@@UAEXPBVDOMNode@2@K@Z 120cacd0 f   DOMRangeImpl.obj
 0001:000c9df0       ?setEnd@DOMRangeImpl@xercesc_2_3@@UAEXPBVDOMNode@2@K@Z 120cadf0 f   DOMRangeImpl.obj
 0001:000c9f10       ?setStartBefore@DOMRangeImpl@xercesc_2_3@@UAEXPBVDOMNode@2@@Z 120caf10 f   DOMRangeImpl.obj
 0001:000ca090       ?setStartAfter@DOMRangeImpl@xercesc_2_3@@UAEXPBVDOMNode@2@@Z 120cb090 f   DOMRangeImpl.obj
 0001:000ca210       ?setEndBefore@DOMRangeImpl@xercesc_2_3@@UAEXPBVDOMNode@2@@Z 120cb210 f   DOMRangeImpl.obj
 0001:000ca390       ?setEndAfter@DOMRangeImpl@xercesc_2_3@@UAEXPBVDOMNode@2@@Z 120cb390 f   DOMRangeImpl.obj
 0001:000ca510       ?detach@DOMRangeImpl@xercesc_2_3@@UAEXXZ 120cb510 f   DOMRangeImpl.obj
 0001:000ca570       ?collapse@DOMRangeImpl@xercesc_2_3@@UAEX_N@Z 120cb570 f   DOMRangeImpl.obj
 0001:000ca5d0       ?selectNode@DOMRangeImpl@xercesc_2_3@@UAEXPBVDOMNode@2@@Z 120cb5d0 f   DOMRangeImpl.obj
 0001:000ca770       ?selectNodeContents@DOMRangeImpl@xercesc_2_3@@UAEXPBVDOMNode@2@@Z 120cb770 f   DOMRangeImpl.obj
 0001:000ca8c0       ?surroundContents@DOMRangeImpl@xercesc_2_3@@UAEXPAVDOMNode@2@@Z 120cb8c0 f   DOMRangeImpl.obj
 0001:000caa30       ?compareBoundaryPoints@DOMRangeImpl@xercesc_2_3@@UBEFW4CompareHow@DOMRange@2@PBV42@@Z 120cba30 f   DOMRangeImpl.obj
 0001:000cad00       ?deleteContents@DOMRangeImpl@xercesc_2_3@@UAEXXZ 120cbd00 f   DOMRangeImpl.obj
 0001:000cad10       ?extractContents@DOMRangeImpl@xercesc_2_3@@UAEPAVDOMDocumentFragment@2@XZ 120cbd10 f   DOMRangeImpl.obj
 0001:000cad40       ?cloneContents@DOMRangeImpl@xercesc_2_3@@UBEPAVDOMDocumentFragment@2@XZ 120cbd40 f   DOMRangeImpl.obj
 0001:000cad50       ?insertNode@DOMRangeImpl@xercesc_2_3@@UAEXPAVDOMNode@2@@Z 120cbd50 f   DOMRangeImpl.obj
 0001:000caf40       ?cloneRange@DOMRangeImpl@xercesc_2_3@@UBEPAVDOMRange@2@XZ 120cbf40 f   DOMRangeImpl.obj
 0001:000cafa0       ?toString@DOMRangeImpl@xercesc_2_3@@UBEPBGXZ 120cbfa0 f   DOMRangeImpl.obj
 0001:000cb360       ?getCommonAncestorContainer@DOMRangeImpl@xercesc_2_3@@UBEPBVDOMNode@2@XZ 120cc360 f   DOMRangeImpl.obj
 0001:000cb370       ?release@DOMRangeImpl@xercesc_2_3@@UAEXXZ 120cc370 f   DOMRangeImpl.obj
 0001:000cb380       ?isValidAncestorType@DOMRangeImpl@xercesc_2_3@@ABE_NPBVDOMNode@2@@Z 120cc380 f   DOMRangeImpl.obj
 0001:000cb3c0       ?isAncestorOf@DOMRangeImpl@xercesc_2_3@@CA_NPBVDOMNode@2@0@Z 120cc3c0 f   DOMRangeImpl.obj
 0001:000cb3f0       ?hasLegalRootContainer@DOMRangeImpl@xercesc_2_3@@ABE_NPBVDOMNode@2@@Z 120cc3f0 f   DOMRangeImpl.obj
 0001:000cb450       ?isLegalContainedNode@DOMRangeImpl@xercesc_2_3@@ABE_NPBVDOMNode@2@@Z 120cc450 f   DOMRangeImpl.obj
 0001:000cb4a0       ?indexOf@DOMRangeImpl@xercesc_2_3@@ABEKPBVDOMNode@2@0@Z 120cc4a0 f   DOMRangeImpl.obj
 0001:000cb4e0       ?validateNode@DOMRangeImpl@xercesc_2_3@@ABEXPBVDOMNode@2@@Z 120cc4e0 f   DOMRangeImpl.obj
 0001:000cb560       ?commonAncestorOf@DOMRangeImpl@xercesc_2_3@@ABEPBVDOMNode@2@PBV32@0@Z 120cc560 f   DOMRangeImpl.obj
 0001:000cb7d0       ?checkIndex@DOMRangeImpl@xercesc_2_3@@ABEXPBVDOMNode@2@K@Z 120cc7d0 f   DOMRangeImpl.obj
 0001:000cb890       ?nextNode@DOMRangeImpl@xercesc_2_3@@ABEPAVDOMNode@2@PBV32@_N@Z 120cc890 f   DOMRangeImpl.obj
 0001:000cb900       ?traverseContents@DOMRangeImpl@xercesc_2_3@@AAEPAVDOMDocumentFragment@2@W4TraversalType@12@@Z 120cc900 f   DOMRangeImpl.obj
 0001:000cba60       ?traverseSameContainer@DOMRangeImpl@xercesc_2_3@@AAEPAVDOMDocumentFragment@2@H@Z 120cca60 f   DOMRangeImpl.obj
 0001:000cbc80       ?traverseCommonStartContainer@DOMRangeImpl@xercesc_2_3@@AAEPAVDOMDocumentFragment@2@PAVDOMNode@2@H@Z 120ccc80 f   DOMRangeImpl.obj
 0001:000cbda0       ?traverseCommonEndContainer@DOMRangeImpl@xercesc_2_3@@AAEPAVDOMDocumentFragment@2@PAVDOMNode@2@H@Z 120ccda0 f   DOMRangeImpl.obj
 0001:000cbea0       ?traverseCommonAncestors@DOMRangeImpl@xercesc_2_3@@AAEPAVDOMDocumentFragment@2@PAVDOMNode@2@0H@Z 120ccea0 f   DOMRangeImpl.obj
 0001:000cc010       ?traverseRightBoundary@DOMRangeImpl@xercesc_2_3@@AAEPAVDOMNode@2@PAV32@H@Z 120cd010 f   DOMRangeImpl.obj
 0001:000cc2d0       ?traverseLeftBoundary@DOMRangeImpl@xercesc_2_3@@AAEPAVDOMNode@2@PAV32@H@Z 120cd2d0 f   DOMRangeImpl.obj
 0001:000cc5a0       ?traverseNode@DOMRangeImpl@xercesc_2_3@@AAEPAVDOMNode@2@PAV32@_N1H@Z 120cd5a0 f   DOMRangeImpl.obj
 0001:000cc650       ?traverseFullySelected@DOMRangeImpl@xercesc_2_3@@AAEPAVDOMNode@2@PAV32@H@Z 120cd650 f   DOMRangeImpl.obj
 0001:000cc6a0       ?traversePartiallySelected@DOMRangeImpl@xercesc_2_3@@AAEPAVDOMNode@2@PAV32@H@Z 120cd6a0 f   DOMRangeImpl.obj
 0001:000cc6c0       ?traverseTextNode@DOMRangeImpl@xercesc_2_3@@AAEPAVDOMNode@2@PAV32@_NH@Z 120cd6c0 f   DOMRangeImpl.obj
 0001:000ccaa0       ?getSelectedNode@DOMRangeImpl@xercesc_2_3@@AAEPAVDOMNode@2@PAV32@H@Z 120cdaa0 f   DOMRangeImpl.obj
 0001:000ccb00       ?checkReadOnly@DOMRangeImpl@xercesc_2_3@@AAEXPAVDOMNode@2@0KK@Z 120cdb00 f   DOMRangeImpl.obj
 0001:000ccc40       ?recurseTreeAndCheck@DOMRangeImpl@xercesc_2_3@@AAEXPAVDOMNode@2@0@Z 120cdc40 f   DOMRangeImpl.obj
 0001:000ccce0       ?removeChild@DOMRangeImpl@xercesc_2_3@@AAEPAVDOMNode@2@PAV32@0@Z 120cdce0 f   DOMRangeImpl.obj
 0001:000ccd00       ?receiveReplacedText@DOMRangeImpl@xercesc_2_3@@QAEXPAVDOMNode@2@@Z 120cdd00 f   DOMRangeImpl.obj
 0001:000ccd70       ?updateRangeForDeletedText@DOMRangeImpl@xercesc_2_3@@QAEXPAVDOMNode@2@KH@Z 120cdd70 f   DOMRangeImpl.obj
 0001:000cce10       ?updateRangeForInsertedText@DOMRangeImpl@xercesc_2_3@@QAEXPAVDOMNode@2@KH@Z 120cde10 f   DOMRangeImpl.obj
 0001:000cce90       ?updateRangeForDeletedNode@DOMRangeImpl@xercesc_2_3@@QAEXPAVDOMNode@2@@Z 120cde90 f   DOMRangeImpl.obj
 0001:000cd060       ?updateRangeForInsertedNode@DOMRangeImpl@xercesc_2_3@@QAEXPAVDOMNode@2@@Z 120ce060 f   DOMRangeImpl.obj
 0001:000cd100       ?updateSplitInfo@DOMRangeImpl@xercesc_2_3@@QAEXPAVDOMNode@2@0K@Z 120ce100 f   DOMRangeImpl.obj
 0001:000cd190       ??0DOMStringPool@xercesc_2_3@@QAE@HPAVDOMDocumentImpl@1@@Z 120ce190 f   DOMStringPool.obj
 0001:000cd1d0       ?getPooledString@DOMStringPool@xercesc_2_3@@QAEPBGPBG@Z 120ce1d0 f   DOMStringPool.obj
 0001:000cd2a0       ??0DOMBuffer@xercesc_2_3@@QAE@PAVDOMDocumentImpl@1@PBG@Z 120ce2a0 f   DOMStringPool.obj
 0001:000cd320       ?append@DOMBuffer@xercesc_2_3@@QAEXQBGI@Z 120ce320 f   DOMStringPool.obj
 0001:000cd3f0       ?set@DOMBuffer@xercesc_2_3@@QAEXQBGI@Z 120ce3f0 f   DOMStringPool.obj
 0001:000cd4b0       ??0DOMTextImpl@xercesc_2_3@@QAE@PAVDOMDocument@1@PBG@Z 120ce4b0 f   DOMTextImpl.obj
 0001:000cd540       ??_EDOMTextImpl@xercesc_2_3@@UAEPAXI@Z 120ce540 f i DOMTextImpl.obj
 0001:000cd5a0       ??0DOMTextImpl@xercesc_2_3@@QAE@ABV01@_N@Z 120ce5a0 f   DOMTextImpl.obj
 0001:000cd630       ??1DOMTextImpl@xercesc_2_3@@UAE@XZ 120ce630 f   DOMTextImpl.obj
 0001:000cd6a0       ?cloneNode@DOMTextImpl@xercesc_2_3@@UBEPAVDOMNode@2@_N@Z 120ce6a0 f   DOMTextImpl.obj
 0001:000cd760       ?getNodeName@DOMTextImpl@xercesc_2_3@@UBEPBGXZ 120ce760 f   DOMTextImpl.obj
 0001:000cd770       ?splitText@DOMTextImpl@xercesc_2_3@@UAEPAVDOMText@2@K@Z 120ce770 f   DOMTextImpl.obj
 0001:000cd8b0       ?isIgnorableWhitespace@DOMCDATASectionImpl@xercesc_2_3@@UBE_NXZ 120ce8b0 f   DOMTextImpl.obj
 0001:000cd8b0       ?isIgnorableWhitespace@DOMTextImpl@xercesc_2_3@@UBE_NXZ 120ce8b0 f   DOMTextImpl.obj
 0001:000cd8d0       ?setIgnorableWhitespace@DOMTextImpl@xercesc_2_3@@MAEX_N@Z 120ce8d0 f   DOMTextImpl.obj
 0001:000cd910       ?release@DOMTextImpl@xercesc_2_3@@UAEXXZ 120ce910 f   DOMTextImpl.obj
 0001:000cd9a0       ??0DOMTreeWalkerImpl@xercesc_2_3@@QAE@PAVDOMNode@1@KPAVDOMNodeFilter@1@_N@Z 120ce9a0 f   DOMTreeWalkerImpl.obj
 0001:000cd9d0       ??_EDOMTreeWalkerImpl@xercesc_2_3@@UAEPAXI@Z 120ce9d0 f i DOMTreeWalkerImpl.obj
 0001:000cda30       ??0DOMTreeWalkerImpl@xercesc_2_3@@QAE@ABV01@@Z 120cea30 f   DOMTreeWalkerImpl.obj
 0001:000cda70       ??4DOMTreeWalkerImpl@xercesc_2_3@@QAEAAV01@ABV01@@Z 120cea70 f   DOMTreeWalkerImpl.obj
 0001:000cdaa0       ?setCurrentNode@DOMTreeWalkerImpl@xercesc_2_3@@UAEXPAVDOMNode@2@@Z 120ceaa0 f   DOMTreeWalkerImpl.obj
 0001:000cdad0       ?parentNode@DOMTreeWalkerImpl@xercesc_2_3@@UAEPAVDOMNode@2@XZ 120cead0 f   DOMTreeWalkerImpl.obj
 0001:000cdb60       ?firstChild@DOMTreeWalkerImpl@xercesc_2_3@@UAEPAVDOMNode@2@XZ 120ceb60 f   DOMTreeWalkerImpl.obj
 0001:000cdc10       ?lastChild@DOMTreeWalkerImpl@xercesc_2_3@@UAEPAVDOMNode@2@XZ 120cec10 f   DOMTreeWalkerImpl.obj
 0001:000cdcc0       ?previousSibling@DOMTreeWalkerImpl@xercesc_2_3@@UAEPAVDOMNode@2@XZ 120cecc0 f   DOMTreeWalkerImpl.obj
 0001:000cdce0       ?nextSibling@DOMTreeWalkerImpl@xercesc_2_3@@UAEPAVDOMNode@2@XZ 120cece0 f   DOMTreeWalkerImpl.obj
 0001:000cdd00       ?previousNode@DOMTreeWalkerImpl@xercesc_2_3@@UAEPAVDOMNode@2@XZ 120ced00 f   DOMTreeWalkerImpl.obj
 0001:000cde50       ?nextNode@DOMTreeWalkerImpl@xercesc_2_3@@UAEPAVDOMNode@2@XZ 120cee50 f   DOMTreeWalkerImpl.obj
 0001:000ce010       ?getParentNode@DOMTreeWalkerImpl@xercesc_2_3@@IAEPAVDOMNode@2@PAV32@@Z 120cf010 f   DOMTreeWalkerImpl.obj
 0001:000ce090       ?getNextSibling@DOMTreeWalkerImpl@xercesc_2_3@@IAEPAVDOMNode@2@PAV32@@Z 120cf090 f   DOMTreeWalkerImpl.obj
 0001:000ce280       ?getPreviousSibling@DOMTreeWalkerImpl@xercesc_2_3@@IAEPAVDOMNode@2@PAV32@@Z 120cf280 f   DOMTreeWalkerImpl.obj
 0001:000ce470       ?getFirstChild@DOMTreeWalkerImpl@xercesc_2_3@@IAEPAVDOMNode@2@PAV32@@Z 120cf470 f   DOMTreeWalkerImpl.obj
 0001:000ce510       ?getLastChild@DOMTreeWalkerImpl@xercesc_2_3@@IAEPAVDOMNode@2@PAV32@@Z 120cf510 f   DOMTreeWalkerImpl.obj
 0001:000ce5b0       ?acceptNode@DOMTreeWalkerImpl@xercesc_2_3@@IAEFPAVDOMNode@2@@Z 120cf5b0 f   DOMTreeWalkerImpl.obj
 0001:000ce630       ??0DOMTypeInfoImpl@xercesc_2_3@@QAE@PBG0PAVDOMDocumentImpl@1@@Z 120cf630 f   DOMTypeInfoImpl.obj
 0001:000ce6a0       ??_EDOMTypeInfoImpl@xercesc_2_3@@UAEPAXI@Z 120cf6a0 f i DOMTypeInfoImpl.obj
 0001:000ce700       ??0DOMTypeInfoImpl@xercesc_2_3@@QAE@XZ 120cf700 f   DOMTypeInfoImpl.obj
 0001:000ce760       ??1DOMWriterImpl@xercesc_2_3@@UAE@XZ 120cf760 f   DOMWriterImpl.obj
 0001:000ce7d0       ??_EDOMWriterImpl@xercesc_2_3@@UAEPAXI@Z 120cf7d0 f i DOMWriterImpl.obj
 0001:000ce830       ??0DOMWriterImpl@xercesc_2_3@@QAE@QAVMemoryManager@1@@Z 120cf830 f   DOMWriterImpl.obj
 0001:000ce8f0       ?canSetFeature@DOMWriterImpl@xercesc_2_3@@UBE_NQBG_N@Z 120cf8f0 f   DOMWriterImpl.obj
 0001:000ce930       ?setFeature@DOMWriterImpl@xercesc_2_3@@UAEXQBG_N@Z 120cf930 f   DOMWriterImpl.obj
 0001:000cea40       ?getFeature@DOMWriterImpl@xercesc_2_3@@UBE_NQBG@Z 120cfa40 f   DOMWriterImpl.obj
 0001:000cea80       ?setEncoding@DOMWriterImpl@xercesc_2_3@@UAEXQBG@Z 120cfa80 f   DOMWriterImpl.obj
 0001:000ceaf0       ?setNewLine@DOMWriterImpl@xercesc_2_3@@UAEXQBG@Z 120cfaf0 f   DOMWriterImpl.obj
 0001:000ceb60       ?setFilter@DOMWriterImpl@xercesc_2_3@@UAEXPAVDOMWriterFilter@2@@Z 120cfb60 f   DOMWriterImpl.obj
 0001:000ceb70       ?writeNode@DOMWriterImpl@xercesc_2_3@@UAE_NQAVXMLFormatTarget@2@ABVDOMNode@2@@Z 120cfb70 f   DOMWriterImpl.obj
 0001:000cecf0       ?writeToString@DOMWriterImpl@xercesc_2_3@@UAEPAGABVDOMNode@2@@Z 120cfcf0 f   DOMWriterImpl.obj
 0001:000cee00       ?initSession@DOMWriterImpl@xercesc_2_3@@AAEXQBVDOMNode@2@@Z 120cfe00 f   DOMWriterImpl.obj
 0001:000ceec0       ?processNode@DOMWriterImpl@xercesc_2_3@@AAEXQBVDOMNode@2@H@Z 120cfec0 f   DOMWriterImpl.obj
 0001:000d0760       ?checkFilter@DOMWriterImpl@xercesc_2_3@@ABE?AW4FilterAction@DOMNodeFilter@2@QBVDOMNode@2@@Z 120d1760 f   DOMWriterImpl.obj
 0001:000d07b0       ?checkFeature@DOMWriterImpl@xercesc_2_3@@ABE_NQBG_NAAH@Z 120d17b0 f   DOMWriterImpl.obj
 0001:000d0a50       ?reportError@DOMWriterImpl@xercesc_2_3@@AAE_NQBVDOMNode@2@W4ErrorSeverity@DOMError@2@QBG@Z 120d1a50 f   DOMWriterImpl.obj
 0001:000d0b00       ?reportError@DOMWriterImpl@xercesc_2_3@@AAE_NQBVDOMNode@2@W4ErrorSeverity@DOMError@2@W4Codes@XMLDOMMsg@2@@Z 120d1b00 f   DOMWriterImpl.obj
 0001:000d0c10       ?procCdataSection@DOMWriterImpl@xercesc_2_3@@AAEXQBGQBVDOMNode@2@H@Z 120d1c10 f   DOMWriterImpl.obj
 0001:000d0ea0       ?procUnrepCharInCdataSection@DOMWriterImpl@xercesc_2_3@@AAEXQBGQBVDOMNode@2@H@Z 120d1ea0 f   DOMWriterImpl.obj
 0001:000d11f0       ?processNode@DOMWriterImpl@xercesc_2_3@@AAEXQBVDOMNode@2@@Z 120d21f0 f   DOMWriterImpl.obj
 0001:000d1200       ?canSetFeature@DOMWriterImpl@xercesc_2_3@@ABE_NH_N@Z 120d2200 f   DOMWriterImpl.obj
 0001:000d1220       ?printNewLine@DOMWriterImpl@xercesc_2_3@@AAEXXZ 120d2220 f   DOMWriterImpl.obj
 0001:000d1240       ?printIndent@DOMWriterImpl@xercesc_2_3@@ABEXH@Z 120d2240 f   DOMWriterImpl.obj
 0001:000d1280       ?release@DOMWriterImpl@xercesc_2_3@@UAEXXZ 120d2280 f   DOMWriterImpl.obj
 0001:000d1280       ?unreferenced@DeepNodeListImpl@xercesc_2_3@@EAEXXZ 120d2280 f   DOMWriterImpl.obj
 0001:000d1280       ?release@Wrapper4InputSource@xercesc_2_3@@UAEXXZ 120d2280 f   DOMWriterImpl.obj
 0001:000d1290       ?processBOM@DOMWriterImpl@xercesc_2_3@@AAEXXZ 120d2290 f   DOMWriterImpl.obj
 0001:000d1460       ??1?$Janitor@VXMLFormatter@xercesc_2_3@@@xercesc_2_3@@QAE@XZ 120d2460 f i DOMWriterImpl.obj
 0001:000d1490       ??_E?$RefVectorOf@V?$RefHashTableOf@G@xercesc_2_3@@@xercesc_2_3@@UAEPAXI@Z 120d2490 f i DOMWriterImpl.obj
 0001:000d1490       ??_G?$RefVectorOf@V?$RefHashTableOf@G@xercesc_2_3@@@xercesc_2_3@@UAEPAXI@Z 120d2490 f i DOMWriterImpl.obj
 0001:000d14b0       ??1?$RefVectorOf@V?$RefHashTableOf@G@xercesc_2_3@@@xercesc_2_3@@UAE@XZ 120d24b0 f i DOMWriterImpl.obj
 0001:000d15b0       ??1?$BaseRefVectorOf@V?$RefHashTableOf@G@xercesc_2_3@@@xercesc_2_3@@UAE@XZ 120d25b0 f i DOMWriterImpl.obj
 0001:000d15c0       ??0?$BaseRefVectorOf@V?$RefHashTableOf@G@xercesc_2_3@@@xercesc_2_3@@QAE@I_NQAVMemoryManager@1@@Z 120d25c0 f i DOMWriterImpl.obj
 0001:000d1620       ??1?$RefHashTableOf@G@xercesc_2_3@@QAE@XZ 120d2620 f i DOMWriterImpl.obj
 0001:000d16a0       ??0XSDElementNSImpl@xercesc_2_3@@QAE@PAVDOMDocument@1@PBG@Z 120d26a0 f   XSDElementNSImpl.obj
 0001:000d16d0       ??_EXSDElementNSImpl@xercesc_2_3@@UAEPAXI@Z 120d26d0 f i XSDElementNSImpl.obj
 0001:000d1730       ??0XSDElementNSImpl@xercesc_2_3@@QAE@PAVDOMDocument@1@PBG1JJ@Z 120d2730 f   XSDElementNSImpl.obj
 0001:000d1770       ??0XSDElementNSImpl@xercesc_2_3@@QAE@ABV01@_N@Z 120d2770 f   XSDElementNSImpl.obj
 0001:000d17a0       ?cloneNode@XSDElementNSImpl@xercesc_2_3@@UBEPAVDOMNode@2@_N@Z 120d27a0 f   XSDElementNSImpl.obj
 0001:000d1830       ?isReadOnly@NodeImpl@xercesc_2_3@@QBE_NXZ 120d2830 f i AttrImpl.obj
 0001:000d1850       ?isReadOnly@NodeImpl@xercesc_2_3@@QAEX_N@Z 120d2850 f i AttrImpl.obj
 0001:000d1890       ?needsSyncData@NodeImpl@xercesc_2_3@@QBE_NXZ 120d2890 f i AttrImpl.obj
 0001:000d18b0       ?needsSyncData@NodeImpl@xercesc_2_3@@QAEX_N@Z 120d28b0 f i AttrImpl.obj
 0001:000d18f0       ?needsSyncChildren@NodeImpl@xercesc_2_3@@QBE_NXZ 120d28f0 f i AttrImpl.obj
 0001:000d1910       ?needsSyncChildren@NodeImpl@xercesc_2_3@@QAEX_N@Z 120d2910 f i AttrImpl.obj
 0001:000d1950       ?isOwned@NodeImpl@xercesc_2_3@@QBE_NXZ 120d2950 f i AttrImpl.obj
 0001:000d1970       ?isOwned@NodeImpl@xercesc_2_3@@QAEX_N@Z 120d2970 f i AttrImpl.obj
 0001:000d19b0       ?isFirstChild@NodeImpl@xercesc_2_3@@QBE_NXZ 120d29b0 f i AttrImpl.obj
 0001:000d19d0       ?isFirstChild@NodeImpl@xercesc_2_3@@QAEX_N@Z 120d29d0 f i AttrImpl.obj
 0001:000d1a10       ?isSpecified@NodeImpl@xercesc_2_3@@QBE_NXZ 120d2a10 f i AttrImpl.obj
 0001:000d1a30       ?isSpecified@NodeImpl@xercesc_2_3@@QAEX_N@Z 120d2a30 f i AttrImpl.obj
 0001:000d1a70       ?ignorableWhitespace@NodeImpl@xercesc_2_3@@QBE_NXZ 120d2a70 f i AttrImpl.obj
 0001:000d1a90       ?ignorableWhitespace@NodeImpl@xercesc_2_3@@QAEX_N@Z 120d2a90 f i AttrImpl.obj
 0001:000d1ad0       ?setValueCalled@NodeImpl@xercesc_2_3@@QBE_NXZ 120d2ad0 f i AttrImpl.obj
 0001:000d1af0       ?setValueCalled@NodeImpl@xercesc_2_3@@QAEX_N@Z 120d2af0 f i AttrImpl.obj
 0001:000d1b30       ?isIdAttr@NodeImpl@xercesc_2_3@@QBE_NXZ 120d2b30 f i AttrImpl.obj
 0001:000d1b50       ?isIdAttr@NodeImpl@xercesc_2_3@@QAEX_N@Z 120d2b50 f i AttrImpl.obj
 0001:000d1b90       ?hasUserData@NodeImpl@xercesc_2_3@@QBE_NXZ 120d2b90 f i AttrImpl.obj
 0001:000d1bb0       ?hasUserData@NodeImpl@xercesc_2_3@@QAEX_N@Z 120d2bb0 f i AttrImpl.obj
 0001:000d1bf0       ?hasStringValue@NodeImpl@xercesc_2_3@@QBE_NXZ 120d2bf0 f i AttrImpl.obj
 0001:000d1c10       ?hasStringValue@NodeImpl@xercesc_2_3@@QAEX_N@Z 120d2c10 f i AttrImpl.obj
 0001:000d1c50       ??_OAttrImpl@xercesc_2_3@@QAEXABV01@@Z 120d2c50 f i AttrImpl.obj
 0001:000d1c60       ??4DOM_DOMException@xercesc_2_3@@QAEAAV01@ABV01@@Z 120d2c60 f i AttrImpl.obj
 0001:000d1c80       ??1ParentNode@xercesc_2_3@@UAE@XZ 120d2c80 f i AttrImpl.obj
 0001:000d1c90       ??_OXMLDeclImpl@xercesc_2_3@@QAEXABV01@@Z 120d2c90 f i AttrImpl.obj
 0001:000d1ca0       ?getNodeIDMap@DocumentImpl@xercesc_2_3@@QAEPAVNodeIDMap@2@XZ 120d2ca0 f i AttrImpl.obj
 0001:000d1ca0       ?getNamespaceList@SchemaAttDef@xercesc_2_3@@QBEPAV?$ValueVectorOf@I@2@XZ 120d2ca0 f i AttrImpl.obj
 0001:000d1ca0       ?getContentSpec@ComplexTypeInfo@xercesc_2_3@@QBEPAVContentSpecNode@2@XZ 120d2ca0 f i AttrImpl.obj
 0001:000d1ca0       ?getGrammarResolver@AbstractDOMParser@xercesc_2_3@@IBEPAVGrammarResolver@2@XZ 120d2ca0 f i AttrImpl.obj
 0001:000d1ca0       ?getRecursingAnonTypes@SchemaInfo@xercesc_2_3@@QBEPAV?$ValueVectorOf@PBVDOMElement@xercesc_2_3@@@2@XZ 120d2ca0 f i AttrImpl.obj
 0001:000d1ca0       ?getLength@AbstractStringValidator@xercesc_2_3@@QBEIXZ 120d2ca0 f i AttrImpl.obj
 0001:000d1cb0       ?setErrorChecking@DocumentImpl@xercesc_2_3@@QAEX_N@Z 120d2cb0 f i AttrImpl.obj
 0001:000d1cc0       ?getErrorChecking@DocumentImpl@xercesc_2_3@@QAE_NXZ 120d2cc0 f i AttrImpl.obj
 0001:000d1cd0       ?getErrorHandler@SAX2XMLReaderImpl@xercesc_2_3@@UBEPAVErrorHandler@2@XZ 120d2cd0 f i AttrImpl.obj
 0001:000d1cd0       ?getMemoryManager@DocumentImpl@xercesc_2_3@@QBEPAVMemoryManager@2@XZ 120d2cd0 f i AttrImpl.obj
 0001:000d1cd0       ?getIDRefList@XMLScanner@xercesc_2_3@@QBEPBV?$RefHashTableOf@VXMLRefInfo@xercesc_2_3@@@2@XZ 120d2cd0 f i AttrImpl.obj
 0001:000d1cd0       ?getIDRefList@XMLScanner@xercesc_2_3@@QAEPAV?$RefHashTableOf@VXMLRefInfo@xercesc_2_3@@@2@XZ 120d2cd0 f i AttrImpl.obj
 0001:000d1ce0       ??0DocumentImpl@xercesc_2_3@@QAE@ABV01@@Z 120d2ce0 f i AttrImpl.obj
 0001:000d1d40       ??_FDocumentImpl@xercesc_2_3@@QAEXXZ 120d2d40 f i AttrImpl.obj
 0001:000d1d50       ??_EDocumentImpl@xercesc_2_3@@UAEPAXI@Z 120d2d50 f i AttrImpl.obj
 0001:000d1db0       ??_OCharacterDataImpl@xercesc_2_3@@QAEXABV01@@Z 120d2db0 f i AttrImpl.obj
 0001:000d1dc0       ??_OTextImpl@xercesc_2_3@@QAEXABV01@@Z 120d2dc0 f i AttrImpl.obj
 0001:000d1dd0       ?getIssueFatalErrorIfNotFound@InputSource@xercesc_2_3@@UBE?B_NXZ 120d2dd0 f i AttrImpl.obj
 0001:000d1dd0       ?getCreateCommentNodes@AbstractDOMParser@xercesc_2_3@@QBE_NXZ 120d2dd0 f i AttrImpl.obj
 0001:000d1dd0       ?hasDefaults@AttrMapImpl@xercesc_2_3@@UAE_NXZ 120d2dd0 f i AttrImpl.obj
 0001:000d1dd0       ?isExternal@XMLElementDecl@xercesc_2_3@@QBE_NXZ 120d2dd0 f i AttrImpl.obj
 0001:000d1de0       ?setCreateCommentNodes@AbstractDOMParser@xercesc_2_3@@QAEX_N@Z 120d2de0 f i AttrImpl.obj
 0001:000d1de0       ?setIssueFatalErrorIfNotFound@InputSource@xercesc_2_3@@UAEX_N@Z 120d2de0 f i AttrImpl.obj
 0001:000d1de0       ?hasDefaults@AttrMapImpl@xercesc_2_3@@UAEX_N@Z 120d2de0 f i AttrImpl.obj
 0001:000d1de0       ?setExternalElemDeclaration@XMLElementDecl@xercesc_2_3@@QAEX_N@Z 120d2de0 f i AttrImpl.obj
 0001:000d1df0       ??_OElementImpl@xercesc_2_3@@QAEXABV01@@Z 120d2df0 f i AttrImpl.obj
 0001:000d1e00       ??0AttrImpl@xercesc_2_3@@QAE@PAVDocumentImpl@1@ABVDOMString@1@@Z 120d2e00 f   AttrImpl.obj
 0001:000d1eb0       ??_EAttrImpl@xercesc_2_3@@UAEPAXI@Z 120d2eb0 f i AttrImpl.obj
 0001:000d1f10       ??0AttrImpl@xercesc_2_3@@QAE@ABV01@_N@Z 120d2f10 f   AttrImpl.obj
 0001:000d2110       ??1AttrImpl@xercesc_2_3@@UAE@XZ 120d3110 f   AttrImpl.obj
 0001:000d21b0       ?makeChildNode@AttrImpl@xercesc_2_3@@IAEXXZ 120d31b0 f   AttrImpl.obj
 0001:000d2230       ?cloneNode@AttrImpl@xercesc_2_3@@UAEPAVNodeImpl@2@_N@Z 120d3230 f   AttrImpl.obj
 0001:000d22b0       ?getNodeValue@AttrImpl@xercesc_2_3@@UAE?AVDOMString@2@XZ 120d32b0 f   AttrImpl.obj
 0001:000d22d0       ?getSpecified@AttrImpl@xercesc_2_3@@UAE_NXZ 120d32d0 f   AttrImpl.obj
 0001:000d22f0       ?getValue@AttrImpl@xercesc_2_3@@UAE?AVDOMString@2@XZ 120d32f0 f   AttrImpl.obj
 0001:000d2450       ?setNodeValue@AttrImpl@xercesc_2_3@@UAEXABVDOMString@2@@Z 120d3450 f   AttrImpl.obj
 0001:000d2460       ?setSpecified@AttrImpl@xercesc_2_3@@UAEX_N@Z 120d3460 f   AttrImpl.obj
 0001:000d24a0       ?setValue@AttrImpl@xercesc_2_3@@UAEXABVDOMString@2@@Z 120d34a0 f   AttrImpl.obj
 0001:000d2650       ?toString@AttrImpl@xercesc_2_3@@UAE?AVDOMString@2@XZ 120d3650 f   AttrImpl.obj
 0001:000d2750       ?setOwnerElement@AttrImpl@xercesc_2_3@@QAEXPAVElementImpl@2@@Z 120d3750 f   AttrImpl.obj
 0001:000d2770       ?getChildNodes@ParentNode@xercesc_2_3@@UAEPAVNodeListImpl@2@XZ 120d3770 f   AttrImpl.obj
 0001:000d2770       ?getChildNodes@AttrImpl@xercesc_2_3@@UAEPAVNodeListImpl@2@XZ 120d3770 f   AttrImpl.obj
 0001:000d2770       ??0DOM_DOMImplementation@xercesc_2_3@@QAE@XZ 120d3770 f   AttrImpl.obj
 0001:000d2770       ?getChildNodes@NodeImpl@xercesc_2_3@@UAEPAVNodeListImpl@2@XZ 120d3770 f   AttrImpl.obj
 0001:000d2780       ?getFirstChild@AttrImpl@xercesc_2_3@@UAEPAVNodeImpl@2@XZ 120d3780 f   AttrImpl.obj
 0001:000d2790       ?lastChild@AttrImpl@xercesc_2_3@@IAEPAVChildNode@2@XZ 120d3790 f   AttrImpl.obj
 0001:000d2790       ?getLastChild@AttrImpl@xercesc_2_3@@UAEPAVNodeImpl@2@XZ 120d3790 f   AttrImpl.obj
 0001:000d27b0       ?lastChild@AttrImpl@xercesc_2_3@@IAEXPAVChildNode@2@@Z 120d37b0 f   AttrImpl.obj
 0001:000d27d0       ?getLength@AttrImpl@xercesc_2_3@@UAEIXZ 120d37d0 f   AttrImpl.obj
 0001:000d2800       ?hasChildNodes@AttrImpl@xercesc_2_3@@UAE_NXZ 120d3800 f   AttrImpl.obj
 0001:000d2810       ?insertBefore@AttrImpl@xercesc_2_3@@UAEPAVNodeImpl@2@PAV32@0@Z 120d3810 f   AttrImpl.obj
 0001:000d2b80       ?item@AttrImpl@xercesc_2_3@@UAEPAVNodeImpl@2@I@Z 120d3b80 f   AttrImpl.obj
 0001:000d2bd0       ?removeChild@AttrImpl@xercesc_2_3@@UAEPAVNodeImpl@2@PAV32@@Z 120d3bd0 f   AttrImpl.obj
 0001:000d2db0       ?setReadOnly@AttrImpl@xercesc_2_3@@UAEX_N0@Z 120d3db0 f   AttrImpl.obj
 0001:000d2e00       ?normalize@AttrImpl@xercesc_2_3@@UAEXXZ 120d3e00 f   AttrImpl.obj
 0001:000d2eb0       ??0AttrMapImpl@xercesc_2_3@@QAE@PAVNodeImpl@1@@Z 120d3eb0 f   AttrMapImpl.obj
 0001:000d2ed0       ??_EAttrMapImpl@xercesc_2_3@@UAEPAXI@Z 120d3ed0 f i AttrMapImpl.obj
 0001:000d2f30       ??0AttrMapImpl@xercesc_2_3@@QAE@PAVNodeImpl@1@PAVNamedNodeMapImpl@1@@Z 120d3f30 f   AttrMapImpl.obj
 0001:000d2fa0       ??1AttrMapImpl@xercesc_2_3@@UAE@XZ 120d3fa0 f   AttrMapImpl.obj
 0001:000d2fb0       ?cloneAttrMap@AttrMapImpl@xercesc_2_3@@UAEPAV12@PAVNodeImpl@2@@Z 120d3fb0 f   AttrMapImpl.obj
 0001:000d3040       ?removeNamedItem@AttrMapImpl@xercesc_2_3@@UAEPAVNodeImpl@2@ABVDOMString@2@@Z 120d4040 f   AttrMapImpl.obj
 0001:000d3090       ?removeNamedItemNS@AttrMapImpl@xercesc_2_3@@UAEPAVNodeImpl@2@ABVDOMString@2@0@Z 120d4090 f   AttrMapImpl.obj
 0001:000d30f0       ??1AttrNSImpl@xercesc_2_3@@UAE@XZ 120d40f0 f i AttrNSImpl.obj
 0001:000d3150       ??_OAttrNSImpl@xercesc_2_3@@QAEXABV01@@Z 120d4150 f i AttrNSImpl.obj
 0001:000d3160       ??0AttrNSImpl@xercesc_2_3@@QAE@PAVDocumentImpl@1@ABVDOMString@1@@Z 120d4160 f   AttrNSImpl.obj
 0001:000d31f0       ??_EAttrNSImpl@xercesc_2_3@@UAEPAXI@Z 120d41f0 f i AttrNSImpl.obj
 0001:000d3250       ??0AttrNSImpl@xercesc_2_3@@QAE@PAVDocumentImpl@1@ABVDOMString@1@1@Z 120d4250 f   AttrNSImpl.obj
 0001:000d3500       ??0AttrNSImpl@xercesc_2_3@@QAE@ABV01@_N@Z 120d4500 f   AttrNSImpl.obj
 0001:000d35d0       ?cloneNode@AttrNSImpl@xercesc_2_3@@UAEPAVNodeImpl@2@_N@Z 120d45d0 f   AttrNSImpl.obj
 0001:000d3650       ?getPrefix@AttrNSImpl@xercesc_2_3@@UAE?AVDOMString@2@XZ 120d4650 f   AttrNSImpl.obj
 0001:000d36a0       ?setPrefix@AttrNSImpl@xercesc_2_3@@UAEXABVDOMString@2@@Z 120d46a0 f   AttrNSImpl.obj
 0001:000d3990       ??_OCDATASectionImpl@xercesc_2_3@@QAEXABV01@@Z 120d4990 f i CDATASectionImpl.obj
 0001:000d39c0       ??0CDATASectionImpl@xercesc_2_3@@QAE@PAVDocumentImpl@1@ABVDOMString@1@@Z 120d49c0 f   CDATASectionImpl.obj
 0001:000d39e0       ??_ECDATASectionImpl@xercesc_2_3@@UAEPAXI@Z 120d49e0 f i CDATASectionImpl.obj
 0001:000d3a40       ??0CDATASectionImpl@xercesc_2_3@@QAE@ABV01@_N@Z 120d4a40 f   CDATASectionImpl.obj
 0001:000d3a60       ??1CDATASectionImpl@xercesc_2_3@@UAE@XZ 120d4a60 f   CDATASectionImpl.obj
 0001:000d3a70       ?cloneNode@CDATASectionImpl@xercesc_2_3@@UAEPAVNodeImpl@2@_N@Z 120d4a70 f   CDATASectionImpl.obj
 0001:000d3ae0       ?getNodeName@CDATASectionImpl@xercesc_2_3@@UAE?AVDOMString@2@XZ 120d4ae0 f   CDATASectionImpl.obj
 0001:000d3b20       ?reinitCDATASectionImpl@CDATASectionImpl@xercesc_2_3@@SAXXZ 120d4b20 f   CDATASectionImpl.obj
 0001:000d3b50       ??0CharacterDataImpl@xercesc_2_3@@QAE@PAVDocumentImpl@1@ABVDOMString@1@@Z 120d4b50 f   CharacterDataImpl.obj
 0001:000d3be0       ??_ECharacterDataImpl@xercesc_2_3@@UAEPAXI@Z 120d4be0 f i CharacterDataImpl.obj
 0001:000d3c40       ??0CharacterDataImpl@xercesc_2_3@@QAE@ABV01@_N@Z 120d4c40 f   CharacterDataImpl.obj
 0001:000d3cd0       ??1CharacterDataImpl@xercesc_2_3@@UAE@XZ 120d4cd0 f   CharacterDataImpl.obj
 0001:000d3d30       ?setNodeValue@CharacterDataImpl@xercesc_2_3@@UAEXABVDOMString@2@@Z 120d4d30 f   CharacterDataImpl.obj
 0001:000d3e60       ?appendData@CharacterDataImpl@xercesc_2_3@@UAEXABVDOMString@2@@Z 120d4e60 f   CharacterDataImpl.obj
 0001:000d3ee0       ?deleteData@CharacterDataImpl@xercesc_2_3@@UAEXII@Z 120d4ee0 f   CharacterDataImpl.obj
 0001:000d4020       ?getData@CharacterDataImpl@xercesc_2_3@@UAEAAVDOMString@2@XZ 120d5020 f   CharacterDataImpl.obj
 0001:000d4030       ?getCharDataLength@CharacterDataImpl@xercesc_2_3@@UAEIXZ 120d5030 f   CharacterDataImpl.obj
 0001:000d4040       ?insertData@CharacterDataImpl@xercesc_2_3@@UAEXIABVDOMString@2@@Z 120d5040 f   CharacterDataImpl.obj
 0001:000d40c0       ?replaceData@CharacterDataImpl@xercesc_2_3@@UAEXIIABVDOMString@2@@Z 120d50c0 f   CharacterDataImpl.obj
 0001:000d4160       ?setData@CharacterDataImpl@xercesc_2_3@@UAEXABVDOMString@2@@Z 120d5160 f   CharacterDataImpl.obj
 0001:000d4200       ?substringData@CharacterDataImpl@xercesc_2_3@@UAE?AVDOMString@2@II@Z 120d5200 f   CharacterDataImpl.obj
 0001:000d4230       ??0ChildNode@xercesc_2_3@@QAE@PAVDocumentImpl@1@@Z 120d5230 f   ChildNode.obj
 0001:000d4260       ??_EChildNode@xercesc_2_3@@UAEPAXI@Z 120d5260 f i ChildNode.obj
 0001:000d42c0       ??0ChildNode@xercesc_2_3@@QAE@ABV01@@Z 120d52c0 f   ChildNode.obj
 0001:000d42f0       ??1ChildNode@xercesc_2_3@@UAE@XZ 120d52f0 f   ChildNode.obj
 0001:000d4300       ?getOwnerElement@AttrImpl@xercesc_2_3@@QAEPAVElementImpl@2@XZ 120d5300 f   ChildNode.obj
 0001:000d4300       ?getParentNode@ChildNode@xercesc_2_3@@UAEPAVNodeImpl@2@XZ 120d5300 f   ChildNode.obj
 0001:000d4320       ?getPreviousSibling@ChildNode@xercesc_2_3@@UAEPAVNodeImpl@2@XZ 120d5320 f   ChildNode.obj
 0001:000d4340       ??0CommentImpl@xercesc_2_3@@QAE@ABV01@@Z 120d5340 f i CommentImpl.obj
 0001:000d4360       ??_ECommentImpl@xercesc_2_3@@UAEPAXI@Z 120d5360 f i CommentImpl.obj
 0001:000d43e0       ??0CommentImpl@xercesc_2_3@@QAE@PAVDocumentImpl@1@ABVDOMString@1@@Z 120d53e0 f   CommentImpl.obj
 0001:000d4400       ??0CommentImpl@xercesc_2_3@@QAE@ABV01@_N@Z 120d5400 f   CommentImpl.obj
 0001:000d4420       ??1CommentImpl@xercesc_2_3@@UAE@XZ 120d5420 f   CommentImpl.obj
 0001:000d4430       ?cloneNode@CommentImpl@xercesc_2_3@@UAEPAVNodeImpl@2@_N@Z 120d5430 f   CommentImpl.obj
 0001:000d44a0       ?getNodeName@CommentImpl@xercesc_2_3@@UAE?AVDOMString@2@XZ 120d54a0 f   CommentImpl.obj
 0001:000d44e0       ?reinitCommentImpl@CommentImpl@xercesc_2_3@@SAXXZ 120d54e0 f   CommentImpl.obj
 0001:000d4530       ??0DeepNodeListImpl@xercesc_2_3@@QAE@PAVNodeImpl@1@ABVDOMString@1@@Z 120d5530 f   DeepNodeListImpl.obj
 0001:000d4630       ??_EDeepNodeListImpl@xercesc_2_3@@UAEPAXI@Z 120d5630 f i DeepNodeListImpl.obj
 0001:000d4690       ??0DeepNodeListImpl@xercesc_2_3@@QAE@PAVNodeImpl@1@ABVDOMString@1@1@Z 120d5690 f   DeepNodeListImpl.obj
 0001:000d47b0       ??1DeepNodeListImpl@xercesc_2_3@@UAE@XZ 120d57b0 f   DeepNodeListImpl.obj
 0001:000d4830       ?getLength@DeepNodeListImpl@xercesc_2_3@@UAEIXZ 120d5830 f   DeepNodeListImpl.obj
 0001:000d4850       ?item@DeepNodeListImpl@xercesc_2_3@@UAEPAVNodeImpl@2@I@Z 120d5850 f   DeepNodeListImpl.obj
 0001:000d48e0       ?nextMatchingElementAfter@DeepNodeListImpl@xercesc_2_3@@EAEPAVNodeImpl@2@PAV32@@Z 120d58e0 f   DeepNodeListImpl.obj
 0001:000d4a70       ?reinitDeepNodeListImpl@DeepNodeListImpl@xercesc_2_3@@SAXXZ 120d5a70 f   DeepNodeListImpl.obj
 0001:000d4aa0       ??0DocumentFragmentImpl@xercesc_2_3@@QAE@ABV01@@Z 120d5aa0 f i DocumentFragmentImpl.obj
 0001:000d4ac0       ??_EDocumentFragmentImpl@xercesc_2_3@@UAEPAXI@Z 120d5ac0 f i DocumentFragmentImpl.obj
 0001:000d4b40       ??0DocumentFragmentImpl@xercesc_2_3@@IAE@PAVDocumentImpl@1@@Z 120d5b40 f   DocumentFragmentImpl.obj
 0001:000d4b60       ??0DocumentFragmentImpl@xercesc_2_3@@AAE@ABV01@_N@Z 120d5b60 f   DocumentFragmentImpl.obj
 0001:000d4bc0       ??1DocumentFragmentImpl@xercesc_2_3@@UAE@XZ 120d5bc0 f   DocumentFragmentImpl.obj
 0001:000d4bd0       ?cloneNode@DocumentFragmentImpl@xercesc_2_3@@UAEPAVNodeImpl@2@_N@Z 120d5bd0 f   DocumentFragmentImpl.obj
 0001:000d4c70       ?getNodeName@DocumentFragmentImpl@xercesc_2_3@@UAE?AVDOMString@2@XZ 120d5c70 f   DocumentFragmentImpl.obj
 0001:000d4cb0       ?reinitDocumentFragmentImpl@DocumentFragmentImpl@xercesc_2_3@@SAXXZ 120d5cb0 f   DocumentFragmentImpl.obj
 0001:000d4ce0       ??_ODocumentTypeImpl@xercesc_2_3@@QAEXABV01@@Z 120d5ce0 f i DocumentImpl.obj
 0001:000d4cf0       ??1ElementNSImpl@xercesc_2_3@@UAE@XZ 120d5cf0 f i DocumentImpl.obj
 0001:000d4d50       ??_OElementNSImpl@xercesc_2_3@@QAEXABV01@@Z 120d5d50 f i DocumentImpl.obj
 0001:000d4d60       ??_OEntityReferenceImpl@xercesc_2_3@@QAEXABV01@@Z 120d5d60 f i DocumentImpl.obj
 0001:000d4d70       ??_OEntityImpl@xercesc_2_3@@QAEXABV01@@Z 120d5d70 f i DocumentImpl.obj
 0001:000d4d80       ??_ONotationImpl@xercesc_2_3@@QAEXABV01@@Z 120d5d80 f i DocumentImpl.obj
 0001:000d4d90       ??_OProcessingInstructionImpl@xercesc_2_3@@QAEXABV01@@Z 120d5d90 f i DocumentImpl.obj
 0001:000d4da0       ??1TreeWalkerImpl@xercesc_2_3@@UAE@XZ 120d5da0 f i DocumentImpl.obj
 0001:000d4e20       ??0DocumentImpl@xercesc_2_3@@QAE@QAVMemoryManager@1@@Z 120d5e20 f   DocumentImpl.obj
 0001:000d4ec0       ??0DocumentImpl@xercesc_2_3@@QAE@ABVDOMString@1@0PAVDocumentTypeImpl@1@QAVMemoryManager@1@@Z 120d5ec0 f   DocumentImpl.obj
 0001:000d5000       ?setDocumentType@DocumentImpl@xercesc_2_3@@AAEXPAVDocumentTypeImpl@2@@Z 120d6000 f   DocumentImpl.obj
 0001:000d50d0       ??1DocumentImpl@xercesc_2_3@@UAE@XZ 120d60d0 f   DocumentImpl.obj
 0001:000d5200       ?cloneNode@DocumentImpl@xercesc_2_3@@UAEPAVNodeImpl@2@_N@Z 120d6200 f   DocumentImpl.obj
 0001:000d52a0       ?getNodeName@DocumentImpl@xercesc_2_3@@UAE?AVDOMString@2@XZ 120d62a0 f   DocumentImpl.obj
 0001:000d52e0       ?createAttribute@DocumentImpl@xercesc_2_3@@UAEPAVAttrImpl@2@ABVDOMString@2@@Z 120d62e0 f   DocumentImpl.obj
 0001:000d53b0       ?createCDATASection@DocumentImpl@xercesc_2_3@@UAEPAVCDATASectionImpl@2@ABVDOMString@2@@Z 120d63b0 f   DocumentImpl.obj
 0001:000d5420       ?createComment@DocumentImpl@xercesc_2_3@@UAEPAVCommentImpl@2@ABVDOMString@2@@Z 120d6420 f   DocumentImpl.obj
 0001:000d5490       ?createDocumentFragment@DocumentImpl@xercesc_2_3@@UAEPAVDocumentFragmentImpl@2@XZ 120d6490 f   DocumentImpl.obj
 0001:000d5500       ?createDocumentType@DocumentImpl@xercesc_2_3@@UAEPAVDocumentTypeImpl@2@ABVDOMString@2@@Z 120d6500 f   DocumentImpl.obj
 0001:000d55d0       ?createDocumentType@DocumentImpl@xercesc_2_3@@UAEPAVDocumentTypeImpl@2@ABVDOMString@2@00@Z 120d65d0 f   DocumentImpl.obj
 0001:000d56b0       ?createElement@DocumentImpl@xercesc_2_3@@UAEPAVElementImpl@2@ABVDOMString@2@@Z 120d66b0 f   DocumentImpl.obj
 0001:000d57a0       ?createElement@DocumentImpl@xercesc_2_3@@UAEPAVElementImpl@2@PBG@Z 120d67a0 f   DocumentImpl.obj
 0001:000d5840       ?createEntity@DocumentImpl@xercesc_2_3@@UAEPAVEntityImpl@2@ABVDOMString@2@@Z 120d6840 f   DocumentImpl.obj
 0001:000d5910       ?createEntityReference@DocumentImpl@xercesc_2_3@@UAEPAVEntityReferenceImpl@2@ABVDOMString@2@@Z 120d6910 f   DocumentImpl.obj
 0001:000d59e0       ?createNotation@DocumentImpl@xercesc_2_3@@UAEPAVNotationImpl@2@ABVDOMString@2@@Z 120d69e0 f   DocumentImpl.obj
 0001:000d5ab0       ?createProcessingInstruction@DocumentImpl@xercesc_2_3@@UAEPAVProcessingInstructionImpl@2@ABVDOMString@2@0@Z 120d6ab0 f   DocumentImpl.obj
 0001:000d5b80       ?createTextNode@DocumentImpl@xercesc_2_3@@UAEPAVTextImpl@2@ABVDOMString@2@@Z 120d6b80 f   DocumentImpl.obj
 0001:000d5bf0       ?createNodeIterator@DocumentImpl@xercesc_2_3@@SAPAVNodeIteratorImpl@2@VDOM_Node@2@KPAVDOM_NodeFilter@2@_NQAVMemoryManager@2@@Z 120d6bf0 f   DocumentImpl.obj
 0001:000d5da0       ?createTreeWalker@DocumentImpl@xercesc_2_3@@SAPAVTreeWalkerImpl@2@VDOM_Node@2@KPAVDOM_NodeFilter@2@_NQAVMemoryManager@2@@Z 120d6da0 f   DocumentImpl.obj
 0001:000d5f50       ?getElementsByTagName@DocumentImpl@xercesc_2_3@@UAEPAVDeepNodeListImpl@2@ABVDOMString@2@@Z 120d6f50 f   DocumentImpl.obj
 0001:000d5fc0       ?insertBefore@DocumentImpl@xercesc_2_3@@UAEPAVNodeImpl@2@PAV32@0@Z 120d6fc0 f   DocumentImpl.obj
 0001:000d6080       ?isXMLName@DocumentImpl@xercesc_2_3@@QAE_NABVDOMString@2@@Z 120d7080 f   DocumentImpl.obj
 0001:000d60b0       ?removeChild@DocumentImpl@xercesc_2_3@@UAEPAVNodeImpl@2@PAV32@@Z 120d70b0 f   DocumentImpl.obj
 0001:000d60f0       ?unreferenced@DocumentImpl@xercesc_2_3@@UAEXXZ 120d70f0 f   DocumentImpl.obj
 0001:000d6100       ?importNode@DocumentImpl@xercesc_2_3@@UAEPAVNodeImpl@2@PAV32@_N@Z 120d7100 f   DocumentImpl.obj
 0001:000d69c0       ?createElementNS@DocumentImpl@xercesc_2_3@@UAEPAVElementImpl@2@ABVDOMString@2@0@Z 120d79c0 f   DocumentImpl.obj
 0001:000d6a90       ?createAttributeNS@DocumentImpl@xercesc_2_3@@UAEPAVAttrImpl@2@ABVDOMString@2@0@Z 120d7a90 f   DocumentImpl.obj
 0001:000d6b60       ?getElementsByTagNameNS@DocumentImpl@xercesc_2_3@@UAEPAVDeepNodeListImpl@2@ABVDOMString@2@0@Z 120d7b60 f   DocumentImpl.obj
 0001:000d6be0       ?getElementById@DocumentImpl@xercesc_2_3@@UAEPAVElementImpl@2@ABVDOMString@2@@Z 120d7be0 f   DocumentImpl.obj
 0001:000d6c10       ?indexofQualifiedName@DocumentImpl@xercesc_2_3@@SAHABVDOMString@2@@Z 120d7c10 f   DocumentImpl.obj
 0001:000d6c70       ?createXMLDecl@DocumentImpl@xercesc_2_3@@UAEPAVXMLDeclImpl@2@ABVDOMString@2@00@Z 120d7c70 f   DocumentImpl.obj
 0001:000d6cf0       ?createRange@DocumentImpl@xercesc_2_3@@UAEPAVRangeImpl@2@XZ 120d7cf0 f   DocumentImpl.obj
 0001:000d6e40       ?removeRange@DocumentImpl@xercesc_2_3@@UAEXPAVRangeImpl@2@@Z 120d7e40 f   DocumentImpl.obj
 0001:000d6f50       ?isKidOK@DocumentImpl@xercesc_2_3@@SA_NPAVNodeImpl@2@0@Z 120d7f50 f   DocumentImpl.obj
 0001:000d6fe0       ?setUserData@DocumentImpl@xercesc_2_3@@UAEXPAVNodeImpl@2@PAX@Z 120d7fe0 f   DocumentImpl.obj
 0001:000d7280       ?getUserData@DocumentImpl@xercesc_2_3@@UAEPAXPAVNodeImpl@2@@Z 120d8280 f   DocumentImpl.obj
 0001:000d7320       ?getUserData@DocumentImpl@xercesc_2_3@@UAEPAXXZ 120d8320 f   DocumentImpl.obj
 0001:000d7340       ?setUserData@DocumentImpl@xercesc_2_3@@UAEXPAX@Z 120d8340 f   DocumentImpl.obj
 0001:000d7380       ?changed@DocumentImpl@xercesc_2_3@@UAEXXZ 120d8380 f   DocumentImpl.obj
 0001:000d7390       ?changes@DocumentImpl@xercesc_2_3@@UAEHXZ 120d8390 f   DocumentImpl.obj
 0001:000d73a0       ?reinitDocumentImpl@DocumentImpl@xercesc_2_3@@SAXXZ 120d83a0 f   DocumentImpl.obj
 0001:000d73d0       ??_G?$RefVectorOf@VNodeIteratorImpl@xercesc_2_3@@@xercesc_2_3@@UAEPAXI@Z 120d83d0 f i DocumentImpl.obj
 0001:000d73d0       ??_E?$RefVectorOf@VNodeIteratorImpl@xercesc_2_3@@@xercesc_2_3@@UAEPAXI@Z 120d83d0 f i DocumentImpl.obj
 0001:000d73f0       ??1?$RefVectorOf@VNodeIteratorImpl@xercesc_2_3@@@xercesc_2_3@@UAE@XZ 120d83f0 f i DocumentImpl.obj
 0001:000d7470       ??1?$BaseRefVectorOf@VNodeIteratorImpl@xercesc_2_3@@@xercesc_2_3@@UAE@XZ 120d8470 f i DocumentImpl.obj
 0001:000d7480       ??_G?$RefVectorOf@VTreeWalkerImpl@xercesc_2_3@@@xercesc_2_3@@UAEPAXI@Z 120d8480 f i DocumentImpl.obj
 0001:000d7480       ??_E?$RefVectorOf@VTreeWalkerImpl@xercesc_2_3@@@xercesc_2_3@@UAEPAXI@Z 120d8480 f i DocumentImpl.obj
 0001:000d74a0       ??1?$RefVectorOf@VTreeWalkerImpl@xercesc_2_3@@@xercesc_2_3@@UAE@XZ 120d84a0 f i DocumentImpl.obj
 0001:000d7520       ??1?$BaseRefVectorOf@VTreeWalkerImpl@xercesc_2_3@@@xercesc_2_3@@UAE@XZ 120d8520 f i DocumentImpl.obj
 0001:000d7530       ??_E?$RefVectorOf@VRangeImpl@xercesc_2_3@@@xercesc_2_3@@UAEPAXI@Z 120d8530 f i DocumentImpl.obj
 0001:000d7530       ??_G?$RefVectorOf@VRangeImpl@xercesc_2_3@@@xercesc_2_3@@UAEPAXI@Z 120d8530 f i DocumentImpl.obj
 0001:000d7550       ??1?$RefVectorOf@VRangeImpl@xercesc_2_3@@@xercesc_2_3@@UAE@XZ 120d8550 f i DocumentImpl.obj
 0001:000d75d0       ??1?$BaseRefVectorOf@VRangeImpl@xercesc_2_3@@@xercesc_2_3@@UAE@XZ 120d85d0 f i DocumentImpl.obj
 0001:000d75e0       ??0?$RefHashTableBucketElem@V?$RefHashTableOf@V?$KeyRefPair@XVDOMUserDataHandler@xercesc_2_3@@@xercesc_2_3@@@xercesc_2_3@@@xercesc_2_3@@QAE@PAXQAV?$RefHashTableOf@V?$KeyRefPair@XVDOMUserDataHandler@xercesc_2_3@@@xercesc_2_3@@@1@PAU01@@Z 120d85e0 f i DocumentImpl.obj
 0001:000d75e0       ??0?$RefHashTableBucketElem@VXMLRefInfo@xercesc_2_3@@@xercesc_2_3@@QAE@PAXQAVXMLRefInfo@1@PAU01@@Z 120d85e0 f i DocumentImpl.obj
 0001:000d75e0       ??0?$RefHashTableBucketElem@VKVStringPair@xercesc_2_3@@@xercesc_2_3@@QAE@PAXQAVKVStringPair@1@PAU01@@Z 120d85e0 f i DocumentImpl.obj
 0001:000d75e0       ??0?$RefHashTableBucketElem@VDatatypeValidator@xercesc_2_3@@@xercesc_2_3@@QAE@PAXQAVDatatypeValidator@1@PAU01@@Z 120d85e0 f i DocumentImpl.obj
 0001:000d75e0       ??0?$RefHashTableBucketElem@VSchemaInfo@xercesc_2_3@@@xercesc_2_3@@QAE@PAXQAVSchemaInfo@1@PAU01@@Z 120d85e0 f i DocumentImpl.obj
 0001:000d75e0       ??0?$RefHashTableBucketElem@X@xercesc_2_3@@QAE@PAXQAXPAU01@@Z 120d85e0 f i DocumentImpl.obj
 0001:000d75e0       ??0?$RefHashTableBucketElem@VXercesAttGroupInfo@xercesc_2_3@@@xercesc_2_3@@QAE@PAXQAVXercesAttGroupInfo@1@PAU01@@Z 120d85e0 f i DocumentImpl.obj
 0001:000d75e0       ??0?$RefHashTableBucketElem@VXercesGroupInfo@xercesc_2_3@@@xercesc_2_3@@QAE@PAXQAVXercesGroupInfo@1@PAU01@@Z 120d85e0 f i DocumentImpl.obj
 0001:000d75e0       ??0?$RefHashTableBucketElem@VXMLInteger@xercesc_2_3@@@xercesc_2_3@@QAE@PAXQAVXMLInteger@1@PAU01@@Z 120d85e0 f i DocumentImpl.obj
 0001:000d75e0       ??0?$RefHashTableBucketElem@VENameMap@xercesc_2_3@@@xercesc_2_3@@QAE@PAXQAVENameMap@1@PAU01@@Z 120d85e0 f i DocumentImpl.obj
 0001:000d75e0       ??0?$RefHashTableBucketElem@VValueStore@xercesc_2_3@@@xercesc_2_3@@QAE@PAXQAVValueStore@1@PAU01@@Z 120d85e0 f i DocumentImpl.obj
 0001:000d75e0       ??0?$RefHashTableBucketElem@V?$KeyRefPair@XVDOMUserDataHandler@xercesc_2_3@@@xercesc_2_3@@@xercesc_2_3@@QAE@PAXQAV?$KeyRefPair@XVDOMUserDataHandler@xercesc_2_3@@@1@PAU01@@Z 120d85e0 f i DocumentImpl.obj
 0001:000d75e0       ??0?$RefHashTableBucketElem@G@xercesc_2_3@@QAE@PAXQAGPAU01@@Z 120d85e0 f i DocumentImpl.obj
 0001:000d75e0       ??0?$RefHashTableBucketElem@VComplexTypeInfo@xercesc_2_3@@@xercesc_2_3@@QAE@PAXQAVComplexTypeInfo@1@PAU01@@Z 120d85e0 f i DocumentImpl.obj
 0001:000d75e0       ??0?$RefHashTableBucketElem@VCPMapEntry@xercesc_2_3@@@xercesc_2_3@@QAE@PAXQAVCPMapEntry@1@PAU01@@Z 120d85e0 f i DocumentImpl.obj
 0001:000d7600       ??0DocumentTypeImpl@xercesc_2_3@@QAE@PAVDocumentImpl@1@ABVDOMString@1@@Z 120d8600 f   DocumentTypeImpl.obj
 0001:000d7730       ??_EDocumentTypeImpl@xercesc_2_3@@UAEPAXI@Z 120d8730 f i DocumentTypeImpl.obj
 0001:000d7790       ??0DocumentTypeImpl@xercesc_2_3@@QAE@PAVDocumentImpl@1@ABVDOMString@1@11@Z 120d8790 f   DocumentTypeImpl.obj
 0001:000d7910       ??0DocumentTypeImpl@xercesc_2_3@@QAE@ABV01@_N@Z 120d8910 f   DocumentTypeImpl.obj
 0001:000d7a80       ??1DocumentTypeImpl@xercesc_2_3@@UAE@XZ 120d8a80 f   DocumentTypeImpl.obj
 0001:000d7b50       ?cloneNode@DocumentTypeImpl@xercesc_2_3@@UAEPAVNodeImpl@2@_N@Z 120d8b50 f   DocumentTypeImpl.obj
 0001:000d7bc0       ?setOwnerDocument@DocumentTypeImpl@xercesc_2_3@@UAEXPAVDocumentImpl@2@@Z 120d8bc0 f   DocumentTypeImpl.obj
 0001:000d7bf0       ?getNodeName@EntityReferenceImpl@xercesc_2_3@@UAE?AVDOMString@2@XZ 120d8bf0 f   DocumentTypeImpl.obj
 0001:000d7bf0       ?getNodeName@ElementImpl@xercesc_2_3@@UAE?AVDOMString@2@XZ 120d8bf0 f   DocumentTypeImpl.obj
 0001:000d7bf0       ?getName@DocumentTypeImpl@xercesc_2_3@@UAE?AVDOMString@2@XZ 120d8bf0 f   DocumentTypeImpl.obj
 0001:000d7bf0       ?getNodeName@EntityImpl@xercesc_2_3@@UAE?AVDOMString@2@XZ 120d8bf0 f   DocumentTypeImpl.obj
 0001:000d7bf0       ?getNodeName@DocumentTypeImpl@xercesc_2_3@@UAE?AVDOMString@2@XZ 120d8bf0 f   DocumentTypeImpl.obj
 0001:000d7bf0       ?getTagName@ElementImpl@xercesc_2_3@@UAE?AVDOMString@2@XZ 120d8bf0 f   DocumentTypeImpl.obj
 0001:000d7c10       ?setReadOnly@DocumentTypeImpl@xercesc_2_3@@UAEX_N0@Z 120d8c10 f   DocumentTypeImpl.obj
 0001:000d7c40       ?getPublicId@DocumentTypeImpl@xercesc_2_3@@UAE?AVDOMString@2@XZ 120d8c40 f   DocumentTypeImpl.obj
 0001:000d7c60       ?getSystemId@DocumentTypeImpl@xercesc_2_3@@UAE?AVDOMString@2@XZ 120d8c60 f   DocumentTypeImpl.obj
 0001:000d7c80       ?getInternalSubset@DocumentTypeImpl@xercesc_2_3@@UAE?AVDOMString@2@XZ 120d8c80 f   DocumentTypeImpl.obj
 0001:000d7ca0       ?isIntSubsetReading@DocumentTypeImpl@xercesc_2_3@@AAE_NXZ 120d8ca0 f   DocumentTypeImpl.obj
 0001:000d7cb0       ?setPublicId@DocumentTypeImpl@xercesc_2_3@@EAEXABVDOMString@2@@Z 120d8cb0 f   DocumentTypeImpl.obj
 0001:000d7d20       ?setSystemId@DocumentTypeImpl@xercesc_2_3@@EAEXABVDOMString@2@@Z 120d8d20 f   DocumentTypeImpl.obj
 0001:000d7d90       ?setInternalSubset@DocumentTypeImpl@xercesc_2_3@@EAEXABVDOMString@2@@Z 120d8d90 f   DocumentTypeImpl.obj
 0001:000d7e00       ??0DOM_ProcessingInstruction@xercesc_2_3@@QAE@ABV01@@Z 120d8e00 f   DOM_Attr.obj
 0001:000d7e00       ??0DOM_Entity@xercesc_2_3@@QAE@ABV01@@Z 120d8e00 f   DOM_Attr.obj
 0001:000d7e00       ??0DOM_DocumentFragment@xercesc_2_3@@QAE@ABV01@@Z 120d8e00 f   DOM_Attr.obj
 0001:000d7e00       ??0DOM_Notation@xercesc_2_3@@QAE@ABV01@@Z 120d8e00 f   DOM_Attr.obj
 0001:000d7e00       ??0DOM_Attr@xercesc_2_3@@QAE@ABV01@@Z 120d8e00 f   DOM_Attr.obj
 0001:000d7e00       ??0DOM_EntityReference@xercesc_2_3@@QAE@ABV01@@Z 120d8e00 f   DOM_Attr.obj
 0001:000d7e00       ??0DOM_XMLDecl@xercesc_2_3@@QAE@ABV01@@Z 120d8e00 f   DOM_Attr.obj
 0001:000d7e00       ??0DOM_DocumentType@xercesc_2_3@@QAE@ABV01@@Z 120d8e00 f   DOM_Attr.obj
 0001:000d7e00       ??0DOM_Document@xercesc_2_3@@QAE@ABV01@@Z 120d8e00 f   DOM_Attr.obj
 0001:000d7e00       ??0DOM_CharacterData@xercesc_2_3@@QAE@ABV01@@Z 120d8e00 f   DOM_Attr.obj
 0001:000d7e00       ??0DOM_Element@xercesc_2_3@@QAE@ABV01@@Z 120d8e00 f   DOM_Attr.obj
 0001:000d7e20       ?getName@DOM_Attr@xercesc_2_3@@QBE?AVDOMString@2@XZ 120d8e20 f   DOM_Attr.obj
 0001:000d7e90       ?getSpecified@DOM_Attr@xercesc_2_3@@QBE_NXZ 120d8e90 f   DOM_Attr.obj
 0001:000d7ea0       ?getValue@DOM_Attr@xercesc_2_3@@QBE?AVDOMString@2@XZ 120d8ea0 f   DOM_Attr.obj
 0001:000d7ec0       ?setValue@DOM_Attr@xercesc_2_3@@QAEXABVDOMString@2@@Z 120d8ec0 f   DOM_Attr.obj
 0001:000d7ec0       ?removeAttribute@DOM_Element@xercesc_2_3@@QAEXABVDOMString@2@@Z 120d8ec0 f   DOM_Attr.obj
 0001:000d7ee0       ?getOwnerElement@DOM_Attr@xercesc_2_3@@QBE?AVDOM_Element@2@XZ 120d8ee0 f   DOM_Attr.obj
 0001:000d7f10       ??0DOM_CDATASection@xercesc_2_3@@QAE@XZ 120d8f10 f   DOM_CDATASection.obj
 0001:000d7f20       ??0DOM_CDATASection@xercesc_2_3@@QAE@ABV01@@Z 120d8f20 f   DOM_CDATASection.obj
 0001:000d7f40       ??0DOM_CDATASection@xercesc_2_3@@IAE@PAVCDATASectionImpl@1@@Z 120d8f40 f   DOM_CDATASection.obj
 0001:000d7f60       ??1DOM_CDATASection@xercesc_2_3@@QAE@XZ 120d8f60 f   DOM_CDATASection.obj
 0001:000d7f70       ??4DOM_CDATASection@xercesc_2_3@@QAEAAV01@ABV01@@Z 120d8f70 f   DOM_CDATASection.obj
 0001:000d7f80       ?getData@DOM_CharacterData@xercesc_2_3@@QBE?AVDOMString@2@XZ 120d8f80 f   DOM_CharacterData.obj
 0001:000d7fb0       ?setData@DOM_CharacterData@xercesc_2_3@@QAEXABVDOMString@2@@Z 120d8fb0 f   DOM_CharacterData.obj
 0001:000d7fd0       ?getLength@DOM_CharacterData@xercesc_2_3@@QBEIXZ 120d8fd0 f   DOM_CharacterData.obj
 0001:000d7fe0       ?substringData@DOM_CharacterData@xercesc_2_3@@QBE?AVDOMString@2@II@Z 120d8fe0 f   DOM_CharacterData.obj
 0001:000d8010       ?appendData@DOM_CharacterData@xercesc_2_3@@QAEXABVDOMString@2@@Z 120d9010 f   DOM_CharacterData.obj
 0001:000d8030       ?insertData@DOM_CharacterData@xercesc_2_3@@QAEXIABVDOMString@2@@Z 120d9030 f   DOM_CharacterData.obj
 0001:000d8050       ?deleteData@DOM_CharacterData@xercesc_2_3@@QAEXII@Z 120d9050 f   DOM_CharacterData.obj
 0001:000d8070       ?replaceData@DOM_CharacterData@xercesc_2_3@@QAEXIIABVDOMString@2@@Z 120d9070 f   DOM_CharacterData.obj
 0001:000d8090       ?createDocument@DOM_Document@xercesc_2_3@@SA?AV12@QAVMemoryManager@2@@Z 120d9090 f   DOM_Document.obj
 0001:000d8100       ?createNotation@DOM_Document@xercesc_2_3@@QAE?AVDOM_Notation@2@ABVDOMString@2@@Z 120d9100 f   DOM_Document.obj
 0001:000d8130       ?getDoctype@DOM_Document@xercesc_2_3@@QBE?AVDOM_DocumentType@2@XZ 120d9130 f   DOM_Document.obj
 0001:000d8160       ?getImplementation@DOM_Document@xercesc_2_3@@QBEAAVDOM_DOMImplementation@2@XZ 120d9160 f   DOM_Document.obj
 0001:000d8170       ?getDocumentElement@DOM_Document@xercesc_2_3@@QBE?AVDOM_Element@2@XZ 120d9170 f   DOM_Document.obj
 0001:000d81a0       ?createElement@DOM_Document@xercesc_2_3@@QAE?AVDOM_Element@2@ABVDOMString@2@@Z 120d91a0 f   DOM_Document.obj
 0001:000d81d0       ?createElement@DOM_Document@xercesc_2_3@@QAE?AVDOM_Element@2@PBG@Z 120d91d0 f   DOM_Document.obj
 0001:000d8200       ?createDocumentFragment@DOM_Document@xercesc_2_3@@QAE?AVDOM_DocumentFragment@2@XZ 120d9200 f   DOM_Document.obj
 0001:000d8230       ?createDocumentType@DOM_Document@xercesc_2_3@@QAE?AVDOM_DocumentType@2@ABVDOMString@2@@Z 120d9230 f   DOM_Document.obj
 0001:000d8260       ?createTextNode@DOM_Document@xercesc_2_3@@QAE?AVDOM_Text@2@ABVDOMString@2@@Z 120d9260 f   DOM_Document.obj
 0001:000d8290       ?createComment@DOM_Document@xercesc_2_3@@QAE?AVDOM_Comment@2@ABVDOMString@2@@Z 120d9290 f   DOM_Document.obj
 0001:000d82c0       ?createCDATASection@DOM_Document@xercesc_2_3@@QAE?AVDOM_CDATASection@2@ABVDOMString@2@@Z 120d92c0 f   DOM_Document.obj
 0001:000d82f0       ?getAttributeNodeNS@DOM_Element@xercesc_2_3@@QBE?AVDOM_Attr@2@ABVDOMString@2@0@Z 120d92f0 f   DOM_Document.obj
 0001:000d82f0       ?createProcessingInstruction@DOM_Document@xercesc_2_3@@QAE?AVDOM_ProcessingInstruction@2@ABVDOMString@2@0@Z 120d92f0 f   DOM_Document.obj
 0001:000d8330       ?createAttribute@DOM_Document@xercesc_2_3@@QAE?AVDOM_Attr@2@ABVDOMString@2@@Z 120d9330 f   DOM_Document.obj
 0001:000d8360       ?createEntityReference@DOM_Document@xercesc_2_3@@QAE?AVDOM_EntityReference@2@ABVDOMString@2@@Z 120d9360 f   DOM_Document.obj
 0001:000d8390       ?createNodeIterator@DOM_Document@xercesc_2_3@@QAE?AVDOM_NodeIterator@2@VDOM_Node@2@KPAVDOM_NodeFilter@2@_N@Z 120d9390 f   DOM_Document.obj
 0001:000d8420       ?createTreeWalker@DOM_Document@xercesc_2_3@@QAE?AVDOM_TreeWalker@2@VDOM_Node@2@KPAVDOM_NodeFilter@2@_N@Z 120d9420 f   DOM_Document.obj
 0001:000d84b0       ?getElementsByTagName@DOM_Document@xercesc_2_3@@QBE?AVDOM_NodeList@2@ABVDOMString@2@@Z 120d94b0 f   DOM_Document.obj
 0001:000d84e0       ?importNode@DOM_Document@xercesc_2_3@@QAE?AVDOM_Node@2@ABV32@_N@Z 120d94e0 f   DOM_Document.obj
 0001:000d8520       ?createElementNS@DOM_Document@xercesc_2_3@@QAE?AVDOM_Element@2@ABVDOMString@2@0@Z 120d9520 f   DOM_Document.obj
 0001:000d8560       ?createAttributeNS@DOM_Document@xercesc_2_3@@QAE?AVDOM_Attr@2@ABVDOMString@2@0@Z 120d9560 f   DOM_Document.obj
 0001:000d85a0       ?getElementsByTagNameNS@DOM_Document@xercesc_2_3@@QBE?AVDOM_NodeList@2@ABVDOMString@2@0@Z 120d95a0 f   DOM_Document.obj
 0001:000d85e0       ?getElementById@DOM_Document@xercesc_2_3@@QAE?AVDOM_Element@2@ABVDOMString@2@@Z 120d95e0 f   DOM_Document.obj
 0001:000d8610       ?createXMLDecl@DOM_Document@xercesc_2_3@@QAE?AVDOM_XMLDecl@2@ABVDOMString@2@00@Z 120d9610 f   DOM_Document.obj
 0001:000d8650       ?createRange@DOM_Document@xercesc_2_3@@QAE?AVDOM_Range@2@XZ 120d9650 f   DOM_Document.obj
 0001:000d8680       ?setErrorChecking@DOM_Document@xercesc_2_3@@QAEX_N@Z 120d9680 f   DOM_Document.obj
 0001:000d8690       ?getErrorChecking@DOM_Document@xercesc_2_3@@QAE_NXZ 120d9690 f   DOM_Document.obj
 0001:000d86a0       ??0DOM_DocumentType@xercesc_2_3@@QAE@H@Z 120d96a0 f   DOM_DocumentType.obj
 0001:000d86b0       ?getName@DOM_DocumentType@xercesc_2_3@@QBE?AVDOMString@2@XZ 120d96b0 f   DOM_DocumentType.obj
 0001:000d8720       ?getEntities@DOM_DocumentType@xercesc_2_3@@QBE?AVDOM_NamedNodeMap@2@XZ 120d9720 f   DOM_DocumentType.obj
 0001:000d8750       ?getNotations@DOM_DocumentType@xercesc_2_3@@QBE?AVDOM_NamedNodeMap@2@XZ 120d9750 f   DOM_DocumentType.obj
 0001:000d8780       ?getPublicId@DOM_DocumentType@xercesc_2_3@@QBE?AVDOMString@2@XZ 120d9780 f   DOM_DocumentType.obj
 0001:000d87f0       ?getSystemId@DOM_DocumentType@xercesc_2_3@@QBE?AVDOMString@2@XZ 120d97f0 f   DOM_DocumentType.obj
 0001:000d8860       ?getInternalSubset@DOM_DocumentType@xercesc_2_3@@QBE?AVDOMString@2@XZ 120d9860 f   DOM_DocumentType.obj
 0001:000d88d0       ??0DOM_DOMException@xercesc_2_3@@QAE@XZ 120d98d0 f   DOM_DOMException.obj
 0001:000d88f0       ??_EDOM_DOMException@xercesc_2_3@@UAEPAXI@Z 120d98f0 f i DOM_DOMException.obj
 0001:000d8950       ??0DOM_DOMException@xercesc_2_3@@QAE@FABVDOMString@1@@Z 120d9950 f   DOM_DOMException.obj
 0001:000d8980       ??0DOM_DOMException@xercesc_2_3@@QAE@ABV01@@Z 120d9980 f   DOM_DOMException.obj
 0001:000d89b0       ??1DOM_DOMException@xercesc_2_3@@UAE@XZ 120d99b0 f   DOM_DOMException.obj
 0001:000d89e0       ??0DOM_DOMImplementation@xercesc_2_3@@AAE@ABV01@@Z 120d99e0 f   DOM_DOMImplementation.obj
 0001:000d89e0       ??4DOM_DOMImplementation@xercesc_2_3@@QAEAAV01@ABV01@@Z 120d99e0 f   DOM_DOMImplementation.obj
 0001:000d89f0       ?getImplementation@DOM_DOMImplementation@xercesc_2_3@@SAAAV12@XZ 120d99f0 f   DOM_DOMImplementation.obj
 0001:000d8b00       ?hasFeature@DOM_DOMImplementation@xercesc_2_3@@QAE_NABVDOMString@2@0@Z 120d9b00 f   DOM_DOMImplementation.obj
 0001:000d8cd0       ?createDocumentType@DOM_DOMImplementation@xercesc_2_3@@QAE?AVDOM_DocumentType@2@ABVDOMString@2@00@Z 120d9cd0 f   DOM_DOMImplementation.obj
 0001:000d8dd0       ?createDocument@DOM_DOMImplementation@xercesc_2_3@@QAE?AVDOM_Document@2@ABVDOMString@2@0ABVDOM_DocumentType@2@QAVMemoryManager@2@@Z 120d9dd0 f   DOM_DOMImplementation.obj
 0001:000d8e70       ?reinitDOM_DOMImplementation@DOM_DOMImplementation@xercesc_2_3@@SAXXZ 120d9e70 f   DOM_DOMImplementation.obj
 0001:000d8f40       ?getTagName@DOM_Element@xercesc_2_3@@QBE?AVDOMString@2@XZ 120d9f40 f   DOM_Element.obj
 0001:000d8fb0       ?getAttribute@DOM_Element@xercesc_2_3@@QBE?AVDOMString@2@ABV32@@Z 120d9fb0 f   DOM_Element.obj
 0001:000d9030       ?setAttribute@DOM_Element@xercesc_2_3@@QAEXABVDOMString@2@0@Z 120da030 f   DOM_Element.obj
 0001:000d9050       ?getAttributeNode@DOM_Element@xercesc_2_3@@QBE?AVDOM_Attr@2@ABVDOMString@2@@Z 120da050 f   DOM_Element.obj
 0001:000d9080       ?setAttributeNode@DOM_Element@xercesc_2_3@@QAE?AVDOM_Attr@2@V32@@Z 120da080 f   DOM_Element.obj
 0001:000d90f0       ?removeAttributeNode@DOM_Element@xercesc_2_3@@QAE?AVDOM_Attr@2@V32@@Z 120da0f0 f   DOM_Element.obj
 0001:000d9160       ?getElementsByTagName@DOM_Element@xercesc_2_3@@QBE?AVDOM_NodeList@2@ABVDOMString@2@@Z 120da160 f   DOM_Element.obj
 0001:000d9190       ?getAttributeNS@DOM_Element@xercesc_2_3@@QBE?AVDOMString@2@ABV32@0@Z 120da190 f   DOM_Element.obj
 0001:000d9210       ?setAttributeNS@DOM_Element@xercesc_2_3@@QAEXABVDOMString@2@00@Z 120da210 f   DOM_Element.obj
 0001:000d9230       ?removeAttributeNS@DOM_Element@xercesc_2_3@@QAEXABVDOMString@2@0@Z 120da230 f   DOM_Element.obj
 0001:000d9250       ?setAttributeNodeNS@DOM_Element@xercesc_2_3@@QAE?AVDOM_Attr@2@V32@@Z 120da250 f   DOM_Element.obj
 0001:000d92c0       ?getElementsByTagNameNS@DOM_Element@xercesc_2_3@@QBE?AVDOM_NodeList@2@ABVDOMString@2@0@Z 120da2c0 f   DOM_Element.obj
 0001:000d9300       ?hasAttributes@DOM_Node@xercesc_2_3@@QBE_NXZ 120da300 f   DOM_Element.obj
 0001:000d9300       ?hasAttributes@DOM_Element@xercesc_2_3@@QBE_NXZ 120da300 f   DOM_Element.obj
 0001:000d9310       ?hasAttribute@DOM_Element@xercesc_2_3@@QBE_NABVDOMString@2@@Z 120da310 f   DOM_Element.obj
 0001:000d9330       ?hasAttributeNS@DOM_Element@xercesc_2_3@@QBE_NABVDOMString@2@0@Z 120da330 f   DOM_Element.obj
 0001:000d9350       ?getPublicId@DOM_Entity@xercesc_2_3@@QBE?AVDOMString@2@XZ 120da350 f   DOM_Entity.obj
 0001:000d93c0       ?getSystemId@DOM_Entity@xercesc_2_3@@QBE?AVDOMString@2@XZ 120da3c0 f   DOM_Entity.obj
 0001:000d9430       ?getNotationName@DOM_Entity@xercesc_2_3@@QBE?AVDOMString@2@XZ 120da430 f   DOM_Entity.obj
 0001:000d94a0       ?getFirstChild@DOM_Entity@xercesc_2_3@@QBE?AVDOM_Node@2@XZ 120da4a0 f   DOM_Entity.obj
 0001:000d94d0       ?getLastChild@DOM_Entity@xercesc_2_3@@QBE?AVDOM_Node@2@XZ 120da4d0 f   DOM_Entity.obj
 0001:000d9500       ?getChildNodes@DOM_Node@xercesc_2_3@@QBE?AVDOM_NodeList@2@XZ 120da500 f   DOM_Entity.obj
 0001:000d9500       ?getChildNodes@DOM_Entity@xercesc_2_3@@QBE?AVDOM_NodeList@2@XZ 120da500 f   DOM_Entity.obj
 0001:000d9520       ?hasChildNodes@DOM_Entity@xercesc_2_3@@QBE_NXZ 120da520 f   DOM_Entity.obj
 0001:000d9520       ?hasChildNodes@DOM_Node@xercesc_2_3@@QBE_NXZ 120da520 f   DOM_Entity.obj
 0001:000d9530       ?getPreviousSibling@DOM_Entity@xercesc_2_3@@QBE?AVDOM_Node@2@XZ 120da530 f   DOM_Entity.obj
 0001:000d9560       ?getNextSibling@DOM_Entity@xercesc_2_3@@QBE?AVDOM_Node@2@XZ 120da560 f   DOM_Entity.obj
 0001:000d9590       ??0DOM_NamedNodeMap@xercesc_2_3@@QAE@XZ 120da590 f   DOM_NamedNodeMap.obj
 0001:000d95a0       ??0DOM_NamedNodeMap@xercesc_2_3@@QAE@ABV01@@Z 120da5a0 f   DOM_NamedNodeMap.obj
 0001:000d95e0       ??0DOM_NamedNodeMap@xercesc_2_3@@IAE@PAVNamedNodeMapImpl@1@@Z 120da5e0 f   DOM_NamedNodeMap.obj
 0001:000d9610       ??0DOM_NamedNodeMap@xercesc_2_3@@IAE@PAVNodeImpl@1@@Z 120da610 f   DOM_NamedNodeMap.obj
 0001:000d9630       ??1DOM_NamedNodeMap@xercesc_2_3@@QAE@XZ 120da630 f   DOM_NamedNodeMap.obj
 0001:000d9650       ??8DOM_Node@xercesc_2_3@@QBE_NABV01@@Z 120da650 f   DOM_NamedNodeMap.obj
 0001:000d9650       ??8DOM_NamedNodeMap@xercesc_2_3@@QBE_NABV01@@Z 120da650 f   DOM_NamedNodeMap.obj
 0001:000d9650       ??8DOM_Range@xercesc_2_3@@QBE_NABV01@@Z 120da650 f   DOM_NamedNodeMap.obj
 0001:000d9650       ??8DOMString@xercesc_2_3@@QBE_NABV01@@Z 120da650 f   DOM_NamedNodeMap.obj
 0001:000d9650       ??8DOM_NodeList@xercesc_2_3@@QBE_NABV01@@Z 120da650 f   DOM_NamedNodeMap.obj
 0001:000d9650       ??8DOM_NodeIterator@xercesc_2_3@@QBE_NABV01@@Z 120da650 f   DOM_NamedNodeMap.obj
 0001:000d9650       ??8DOM_TreeWalker@xercesc_2_3@@QBE_NABV01@@Z 120da650 f   DOM_NamedNodeMap.obj
 0001:000d9660       ??4DOM_NamedNodeMap@xercesc_2_3@@QAEAAV01@ABV01@@Z 120da660 f   DOM_NamedNodeMap.obj
 0001:000d96c0       ??4DOM_NamedNodeMap@xercesc_2_3@@QAEAAV01@PBVDOM_NullPtr@1@@Z 120da6c0 f   DOM_NamedNodeMap.obj
 0001:000d9700       ?getNamedItem@DOM_NamedNodeMap@xercesc_2_3@@QBE?AVDOM_Node@2@ABVDOMString@2@@Z 120da700 f   DOM_NamedNodeMap.obj
 0001:000d97d0       ?setNamedItem@DOM_NamedNodeMap@xercesc_2_3@@QAE?AVDOM_Node@2@V32@@Z 120da7d0 f   DOM_NamedNodeMap.obj
 0001:000d98c0       ?removeNamedItem@DOM_NamedNodeMap@xercesc_2_3@@QAE?AVDOM_Node@2@ABVDOMString@2@@Z 120da8c0 f   DOM_NamedNodeMap.obj
 0001:000d9990       ?item@DOM_NamedNodeMap@xercesc_2_3@@QBE?AVDOM_Node@2@I@Z 120da990 f   DOM_NamedNodeMap.obj
 0001:000d9a60       ?getLength@DOM_NamedNodeMap@xercesc_2_3@@QBEIXZ 120daa60 f   DOM_NamedNodeMap.obj
 0001:000d9a80       ?getNamedItemNS@DOM_NamedNodeMap@xercesc_2_3@@QAE?AVDOM_Node@2@ABVDOMString@2@0@Z 120daa80 f   DOM_NamedNodeMap.obj
 0001:000d9b50       ?setNamedItemNS@DOM_NamedNodeMap@xercesc_2_3@@QAE?AVDOM_Node@2@V32@@Z 120dab50 f   DOM_NamedNodeMap.obj
 0001:000d9c40       ?removeNamedItemNS@DOM_NamedNodeMap@xercesc_2_3@@QAE?AVDOM_Node@2@ABVDOMString@2@0@Z 120dac40 f   DOM_NamedNodeMap.obj
 0001:000d9d10       ?appendChild@DOM_Node@xercesc_2_3@@QAE?AV12@ABV12@@Z 120dad10 f   DOM_Node.obj
 0001:000d9d40       ?cloneNode@DOM_Node@xercesc_2_3@@QBE?AV12@_N@Z 120dad40 f   DOM_Node.obj
 0001:000d9d70       ?getNodeName@DOM_Node@xercesc_2_3@@QBE?AVDOMString@2@XZ 120dad70 f   DOM_Node.obj
 0001:000d9de0       ?getNodeValue@DOM_Node@xercesc_2_3@@QBE?AVDOMString@2@XZ 120dade0 f   DOM_Node.obj
 0001:000d9e50       ?getNodeType@DOM_Node@xercesc_2_3@@QBEFXZ 120dae50 f   DOM_Node.obj
 0001:000d9e60       ?getParentNode@DOM_Node@xercesc_2_3@@QBE?AV12@XZ 120dae60 f   DOM_Node.obj
 0001:000d9e90       ?getFirstChild@DOM_Node@xercesc_2_3@@QBE?AV12@XZ 120dae90 f   DOM_Node.obj
 0001:000d9ec0       ?getLastChild@DOM_Node@xercesc_2_3@@QBE?AV12@XZ 120daec0 f   DOM_Node.obj
 0001:000d9ef0       ?getPreviousSibling@DOM_Node@xercesc_2_3@@QBE?AV12@XZ 120daef0 f   DOM_Node.obj
 0001:000d9f20       ?getNextSibling@DOM_Node@xercesc_2_3@@QBE?AV12@XZ 120daf20 f   DOM_Node.obj
 0001:000d9f50       ?getUserData@DOM_Node@xercesc_2_3@@QBEPAXXZ 120daf50 f   DOM_Node.obj
 0001:000d9f60       ?getAttributes@DOM_Node@xercesc_2_3@@QBE?AVDOM_NamedNodeMap@2@XZ 120daf60 f   DOM_Node.obj
 0001:000da060       ?getOwnerDocument@DOM_Node@xercesc_2_3@@QBE?AVDOM_Document@2@XZ 120db060 f   DOM_Node.obj
 0001:000da090       ?insertBefore@DOM_Node@xercesc_2_3@@QAE?AV12@ABV12@0@Z 120db090 f   DOM_Node.obj
 0001:000da0d0       ?isNull@DOM_Node@xercesc_2_3@@QBE_NXZ 120db0d0 f   DOM_Node.obj
 0001:000da0e0       ?replaceChild@DOM_Node@xercesc_2_3@@QAE?AV12@ABV12@0@Z 120db0e0 f   DOM_Node.obj
 0001:000da120       ?removeChild@DOM_Node@xercesc_2_3@@QAE?AV12@ABV12@@Z 120db120 f   DOM_Node.obj
 0001:000da150       ?setNodeValue@DOM_Node@xercesc_2_3@@QAEXABVDOMString@2@@Z 120db150 f   DOM_Node.obj
 0001:000da170       ?setUserData@DOM_Node@xercesc_2_3@@QAEXPAX@Z 120db170 f   DOM_Node.obj
 0001:000da190       ?normalize@DOM_Node@xercesc_2_3@@QAEXXZ 120db190 f   DOM_Node.obj
 0001:000da1a0       ?isSupported@DOM_Node@xercesc_2_3@@QBE_NABVDOMString@2@0@Z 120db1a0 f   DOM_Node.obj
 0001:000da1c0       ?getNamespaceURI@DOM_Node@xercesc_2_3@@QBE?AVDOMString@2@XZ 120db1c0 f   DOM_Node.obj
 0001:000da230       ?getPrefix@DOM_Node@xercesc_2_3@@QBE?AVDOMString@2@XZ 120db230 f   DOM_Node.obj
 0001:000da2a0       ?getLocalName@DOM_Node@xercesc_2_3@@QBE?AVDOMString@2@XZ 120db2a0 f   DOM_Node.obj
 0001:000da310       ?setPrefix@DOM_Node@xercesc_2_3@@QAEXABVDOMString@2@@Z 120db310 f   DOM_Node.obj
 0001:000da330       ??0DOM_NodeFilter@xercesc_2_3@@QAE@XZ 120db330 f   DOM_NodeFilter.obj
 0001:000da340       ??_EDOM_NodeFilter@xercesc_2_3@@UAEPAXI@Z 120db340 f i DOM_NodeFilter.obj
 0001:000da3a0       ??1DOM_NodeFilter@xercesc_2_3@@UAE@XZ 120db3a0 f   DOM_NodeFilter.obj
 0001:000da3b0       ?detach@DOM_NodeIterator@xercesc_2_3@@QAEXXZ 120db3b0 f   DOM_NodeIterator.obj
 0001:000da3c0       ?getFilter@DOM_NodeIterator@xercesc_2_3@@QAEPAVDOM_NodeFilter@2@XZ 120db3c0 f   DOM_NodeIterator.obj
 0001:000da3d0       ?getExpandEntityReferences@DOM_NodeIterator@xercesc_2_3@@QAE_NXZ 120db3d0 f   DOM_NodeIterator.obj
 0001:000da3e0       ?nextNode@DOM_NodeIterator@xercesc_2_3@@QAE?AVDOM_Node@2@XZ 120db3e0 f   DOM_NodeIterator.obj
 0001:000da400       ?previousNode@DOM_NodeIterator@xercesc_2_3@@QAE?AVDOM_Node@2@XZ 120db400 f   DOM_NodeIterator.obj
 0001:000da420       ??4DOM_NodeList@xercesc_2_3@@QAEAAV01@ABV01@@Z 120db420 f   DOM_NodeList.obj
 0001:000da420       ??4DOM_Range@xercesc_2_3@@QAEAAV01@ABV01@@Z 120db420 f   DOM_NodeList.obj
 0001:000da420       ??4DOM_Node@xercesc_2_3@@QAEAAV01@ABV01@@Z 120db420 f   DOM_NodeList.obj
 0001:000da420       ??4DOM_TreeWalker@xercesc_2_3@@QAEAAV01@ABV01@@Z 120db420 f   DOM_NodeList.obj
 0001:000da420       ??4DOM_NodeIterator@xercesc_2_3@@QAEAAV01@ABV01@@Z 120db420 f   DOM_NodeList.obj
 0001:000da450       ??9DOM_NodeList@xercesc_2_3@@QBE_NABV01@@Z 120db450 f   DOM_NodeList.obj
 0001:000da450       ??9DOMString@xercesc_2_3@@QBE_NABV01@@Z 120db450 f   DOM_NodeList.obj
 0001:000da450       ??9DOM_Node@xercesc_2_3@@QBE_NABV01@@Z 120db450 f   DOM_NodeList.obj
 0001:000da450       ??9DOM_Range@xercesc_2_3@@QBE_NABV01@@Z 120db450 f   DOM_NodeList.obj
 0001:000da450       ??9DOM_TreeWalker@xercesc_2_3@@QBE_NABV01@@Z 120db450 f   DOM_NodeList.obj
 0001:000da450       ??9DOM_NamedNodeMap@xercesc_2_3@@QBE_NABV01@@Z 120db450 f   DOM_NodeList.obj
 0001:000da450       ??9DOM_NodeIterator@xercesc_2_3@@QBE_NABV01@@Z 120db450 f   DOM_NodeList.obj
 0001:000da470       ??8DOMString@xercesc_2_3@@QBE_NPBVDOM_NullPtr@1@@Z 120db470 f   DOM_NodeList.obj
 0001:000da470       ??8DOM_NodeIterator@xercesc_2_3@@QBE_NPBVDOM_NullPtr@1@@Z 120db470 f   DOM_NodeList.obj
 0001:000da470       ??8DOM_Node@xercesc_2_3@@QBE_NPBVDOM_NullPtr@1@@Z 120db470 f   DOM_NodeList.obj
 0001:000da470       ??8DOM_NodeList@xercesc_2_3@@QBE_NPBVDOM_NullPtr@1@@Z 120db470 f   DOM_NodeList.obj
 0001:000da470       ??8DOM_NamedNodeMap@xercesc_2_3@@QBE_NPBVDOM_NullPtr@1@@Z 120db470 f   DOM_NodeList.obj
 0001:000da470       ??8DOM_Range@xercesc_2_3@@QBE_NPBVDOM_NullPtr@1@@Z 120db470 f   DOM_NodeList.obj
 0001:000da470       ??8DOM_TreeWalker@xercesc_2_3@@QBE_NPBVDOM_NullPtr@1@@Z 120db470 f   DOM_NodeList.obj
 0001:000da480       ??9DOM_TreeWalker@xercesc_2_3@@QBE_NPBVDOM_NullPtr@1@@Z 120db480 f   DOM_NodeList.obj
 0001:000da480       ??9DOM_NodeList@xercesc_2_3@@QBE_NPBVDOM_NullPtr@1@@Z 120db480 f   DOM_NodeList.obj
 0001:000da480       ??9DOM_Range@xercesc_2_3@@QBE_NPBVDOM_NullPtr@1@@Z 120db480 f   DOM_NodeList.obj
 0001:000da480       ??9DOM_NamedNodeMap@xercesc_2_3@@QBE_NPBVDOM_NullPtr@1@@Z 120db480 f   DOM_NodeList.obj
 0001:000da480       ??9DOM_NodeIterator@xercesc_2_3@@QBE_NPBVDOM_NullPtr@1@@Z 120db480 f   DOM_NodeList.obj
 0001:000da480       ??9DOMString@xercesc_2_3@@QBE_NPBVDOM_NullPtr@1@@Z 120db480 f   DOM_NodeList.obj
 0001:000da480       ??9DOM_Node@xercesc_2_3@@QBE_NPBVDOM_NullPtr@1@@Z 120db480 f   DOM_NodeList.obj
 0001:000da490       ?item@DOM_NodeList@xercesc_2_3@@QBE?AVDOM_Node@2@I@Z 120db490 f   DOM_NodeList.obj
 0001:000da4c0       ?getLength@DOM_NodeList@xercesc_2_3@@QBEIXZ 120db4c0 f   DOM_NodeList.obj
 0001:000da4d0       ?getPublicId@DOM_Notation@xercesc_2_3@@QBE?AVDOMString@2@XZ 120db4d0 f   DOM_Notation.obj
 0001:000da4f0       ?getSystemId@DOM_Notation@xercesc_2_3@@QBE?AVDOMString@2@XZ 120db4f0 f   DOM_Notation.obj
 0001:000da510       ??0DOM_Document@xercesc_2_3@@IAE@PAVDocumentImpl@1@@Z 120db510 f   DOM_ProcessingInstruction.obj
 0001:000da510       ??0DOM_Entity@xercesc_2_3@@IAE@PAVEntityImpl@1@@Z 120db510 f   DOM_ProcessingInstruction.obj
 0001:000da510       ??0DOM_DocumentFragment@xercesc_2_3@@IAE@PAVDocumentFragmentImpl@1@@Z 120db510 f   DOM_ProcessingInstruction.obj
 0001:000da510       ??0DOM_EntityReference@xercesc_2_3@@IAE@PAVEntityReferenceImpl@1@@Z 120db510 f   DOM_ProcessingInstruction.obj
 0001:000da510       ??0DOM_ProcessingInstruction@xercesc_2_3@@IAE@PAVProcessingInstructionImpl@1@@Z 120db510 f   DOM_ProcessingInstruction.obj
 0001:000da510       ??0DOM_Attr@xercesc_2_3@@IAE@PAVAttrImpl@1@@Z 120db510 f   DOM_ProcessingInstruction.obj
 0001:000da510       ??0DOM_DocumentType@xercesc_2_3@@IAE@PAVDocumentTypeImpl@1@@Z 120db510 f   DOM_ProcessingInstruction.obj
 0001:000da510       ??0DOM_Element@xercesc_2_3@@IAE@PAVElementImpl@1@@Z 120db510 f   DOM_ProcessingInstruction.obj
 0001:000da510       ??0DOM_CharacterData@xercesc_2_3@@IAE@PAVCharacterDataImpl@1@@Z 120db510 f   DOM_ProcessingInstruction.obj
 0001:000da510       ??0DOM_Notation@xercesc_2_3@@IAE@PAVNotationImpl@1@@Z 120db510 f   DOM_ProcessingInstruction.obj
 0001:000da510       ??0DOM_XMLDecl@xercesc_2_3@@IAE@PAVXMLDeclImpl@1@@Z 120db510 f   DOM_ProcessingInstruction.obj
 0001:000da530       ?getTarget@DOM_ProcessingInstruction@xercesc_2_3@@QBE?AVDOMString@2@XZ 120db530 f   DOM_ProcessingInstruction.obj
 0001:000da5a0       ?getData@DOM_ProcessingInstruction@xercesc_2_3@@QBE?AVDOMString@2@XZ 120db5a0 f   DOM_ProcessingInstruction.obj
 0001:000da610       ?setData@DOM_ProcessingInstruction@xercesc_2_3@@QAEXABVDOMString@2@@Z 120db610 f   DOM_ProcessingInstruction.obj
 0001:000da670       ??0DOM_NodeIterator@xercesc_2_3@@QAE@XZ 120db670 f   DOM_Range.obj
 0001:000da670       ??0DOMString@xercesc_2_3@@QAE@XZ 120db670 f   DOM_Range.obj
 0001:000da670       ??0DOM_TreeWalker@xercesc_2_3@@QAE@XZ 120db670 f   DOM_Range.obj
 0001:000da670       ??0DOM_NodeList@xercesc_2_3@@QAE@XZ 120db670 f   DOM_Range.obj
 0001:000da670       ??0DOM_Range@xercesc_2_3@@QAE@XZ 120db670 f   DOM_Range.obj
 0001:000da670       ??0DOM_Node@xercesc_2_3@@QAE@XZ 120db670 f   DOM_Range.obj
 0001:000da680       ??0DOM_NodeList@xercesc_2_3@@IAE@PAVNodeListImpl@1@@Z 120db680 f   DOM_Range.obj
 0001:000da680       ??0DOM_NodeIterator@xercesc_2_3@@IAE@PAVNodeIteratorImpl@1@@Z 120db680 f   DOM_Range.obj
 0001:000da680       ??0DOM_Node@xercesc_2_3@@IAE@PAVNodeImpl@1@@Z 120db680 f   DOM_Range.obj
 0001:000da680       ??0DOM_Range@xercesc_2_3@@IAE@PAVRangeImpl@1@@Z 120db680 f   DOM_Range.obj
 0001:000da680       ??0DOM_TreeWalker@xercesc_2_3@@IAE@PAVTreeWalkerImpl@1@@Z 120db680 f   DOM_Range.obj
 0001:000da6a0       ??0DOM_NodeList@xercesc_2_3@@QAE@ABV01@@Z 120db6a0 f   DOM_Range.obj
 0001:000da6a0       ??0DOM_TreeWalker@xercesc_2_3@@QAE@ABV01@@Z 120db6a0 f   DOM_Range.obj
 0001:000da6a0       ??0DOM_Node@xercesc_2_3@@QAE@ABV01@@Z 120db6a0 f   DOM_Range.obj
 0001:000da6a0       ??0DOM_NodeIterator@xercesc_2_3@@QAE@ABV01@@Z 120db6a0 f   DOM_Range.obj
 0001:000da6a0       ??0DOM_Range@xercesc_2_3@@QAE@ABV01@@Z 120db6a0 f   DOM_Range.obj
 0001:000da6c0       ??1DOM_NodeIterator@xercesc_2_3@@QAE@XZ 120db6c0 f   DOM_Range.obj
 0001:000da6c0       ??1DOM_TreeWalker@xercesc_2_3@@QAE@XZ 120db6c0 f   DOM_Range.obj
 0001:000da6c0       ??1DOM_Node@xercesc_2_3@@QAE@XZ 120db6c0 f   DOM_Range.obj
 0001:000da6c0       ??1DOM_NodeList@xercesc_2_3@@QAE@XZ 120db6c0 f   DOM_Range.obj
 0001:000da6c0       ??1DOM_Range@xercesc_2_3@@QAE@XZ 120db6c0 f   DOM_Range.obj
 0001:000da6e0       ??4DOM_NodeIterator@xercesc_2_3@@QAEAAV01@PBVDOM_NullPtr@1@@Z 120db6e0 f   DOM_Range.obj
 0001:000da6e0       ??4DOM_NodeList@xercesc_2_3@@QAEAAV01@PBVDOM_NullPtr@1@@Z 120db6e0 f   DOM_Range.obj
 0001:000da6e0       ??4DOM_TreeWalker@xercesc_2_3@@QAEAAV01@PBVDOM_NullPtr@1@@Z 120db6e0 f   DOM_Range.obj
 0001:000da6e0       ??4DOM_Node@xercesc_2_3@@QAEAAV01@PBVDOM_NullPtr@1@@Z 120db6e0 f   DOM_Range.obj
 0001:000da6e0       ??4DOM_Range@xercesc_2_3@@QAEAAV01@PBVDOM_NullPtr@1@@Z 120db6e0 f   DOM_Range.obj
 0001:000da700       ?getRoot@DOM_NodeIterator@xercesc_2_3@@QAE?AVDOM_Node@2@XZ 120db700 f   DOM_Range.obj
 0001:000da700       ?getStartContainer@DOM_Range@xercesc_2_3@@QBE?AVDOM_Node@2@XZ 120db700 f   DOM_Range.obj
 0001:000da720       ?getEndContainer@DOM_Range@xercesc_2_3@@QBE?AVDOM_Node@2@XZ 120db720 f   DOM_Range.obj
 0001:000da720       ?getCurrentNode@DOM_TreeWalker@xercesc_2_3@@QAE?AVDOM_Node@2@XZ 120db720 f   DOM_Range.obj
 0001:000da740       ?getEndOffset@DOM_Range@xercesc_2_3@@QBEIXZ 120db740 f   DOM_Range.obj
 0001:000da750       ?getCommonAncestorContainer@DOM_Range@xercesc_2_3@@QBE?BVDOM_Node@2@XZ 120db750 f   DOM_Range.obj
 0001:000da770       ?setStart@DOM_Range@xercesc_2_3@@QAEXABVDOM_Node@2@I@Z 120db770 f   DOM_Range.obj
 0001:000da790       ?setEnd@DOM_Range@xercesc_2_3@@QAEXABVDOM_Node@2@I@Z 120db790 f   DOM_Range.obj
 0001:000da7b0       ?setStartBefore@DOM_Range@xercesc_2_3@@QAEXABVDOM_Node@2@@Z 120db7b0 f   DOM_Range.obj
 0001:000da7c0       ?setStartAfter@DOM_Range@xercesc_2_3@@QAEXABVDOM_Node@2@@Z 120db7c0 f   DOM_Range.obj
 0001:000da7d0       ?setEndBefore@DOM_Range@xercesc_2_3@@QAEXABVDOM_Node@2@@Z 120db7d0 f   DOM_Range.obj
 0001:000da7e0       ?setEndAfter@DOM_Range@xercesc_2_3@@QAEXABVDOM_Node@2@@Z 120db7e0 f   DOM_Range.obj
 0001:000da7f0       ?collapse@DOM_Range@xercesc_2_3@@QAEX_N@Z 120db7f0 f   DOM_Range.obj
 0001:000da800       ?getCollapsed@DOM_Range@xercesc_2_3@@QBE_NXZ 120db800 f   DOM_Range.obj
 0001:000da810       ?selectNode@DOM_Range@xercesc_2_3@@QAEXABVDOM_Node@2@@Z 120db810 f   DOM_Range.obj
 0001:000da820       ?selectNodeContents@DOM_Range@xercesc_2_3@@QAEXABVDOM_Node@2@@Z 120db820 f   DOM_Range.obj
 0001:000da830       ?compareBoundaryPoints@DOM_Range@xercesc_2_3@@QBEFW4CompareHow@12@ABV12@@Z 120db830 f   DOM_Range.obj
 0001:000da850       ?deleteContents@DOM_Range@xercesc_2_3@@QAEXXZ 120db850 f   DOM_Range.obj
 0001:000da860       ?extractContents@DOM_Range@xercesc_2_3@@QAE?AVDOM_DocumentFragment@2@XZ 120db860 f   DOM_Range.obj
 0001:000da880       ?cloneContents@DOM_Range@xercesc_2_3@@QBE?AVDOM_DocumentFragment@2@XZ 120db880 f   DOM_Range.obj
 0001:000da8a0       ?insertNode@DOM_Range@xercesc_2_3@@QAEXAAVDOM_Node@2@@Z 120db8a0 f   DOM_Range.obj
 0001:000da8b0       ?surroundContents@DOM_Range@xercesc_2_3@@QAEXAAVDOM_Node@2@@Z 120db8b0 f   DOM_Range.obj
 0001:000da8c0       ?cloneRange@DOM_Range@xercesc_2_3@@QBE?AV12@XZ 120db8c0 f   DOM_Range.obj
 0001:000da8f0       ?toString@DOM_Range@xercesc_2_3@@QBE?AVDOMString@2@XZ 120db8f0 f   DOM_Range.obj
 0001:000da910       ?detach@DOM_Range@xercesc_2_3@@QAEXXZ 120db910 f   DOM_Range.obj
 0001:000da920       ??4DOM_RangeException@xercesc_2_3@@QAEAAV01@ABV01@@Z 120db920 f i DOM_RangeException.obj
 0001:000da950       ??0DOM_RangeException@xercesc_2_3@@QAE@XZ 120db950 f   DOM_RangeException.obj
 0001:000da970       ??_EDOM_RangeException@xercesc_2_3@@UAEPAXI@Z 120db970 f i DOM_RangeException.obj
 0001:000da9d0       ??0DOM_RangeException@xercesc_2_3@@QAE@W4RangeExceptionCode@01@ABVDOMString@1@@Z 120db9d0 f   DOM_RangeException.obj
 0001:000daa00       ??0DOM_RangeException@xercesc_2_3@@QAE@ABV01@@Z 120dba00 f   DOM_RangeException.obj
 0001:000daa30       ??1DOM_RangeException@xercesc_2_3@@UAE@XZ 120dba30 f   DOM_RangeException.obj
 0001:000daa40       ??0DOM_Text@xercesc_2_3@@QAE@XZ 120dba40 f   DOM_Text.obj
 0001:000daa40       ??0DOM_Comment@xercesc_2_3@@QAE@XZ 120dba40 f   DOM_Text.obj
 0001:000daa50       ??0DOM_Comment@xercesc_2_3@@QAE@ABV01@@Z 120dba50 f   DOM_Text.obj
 0001:000daa50       ??0DOM_Text@xercesc_2_3@@QAE@ABV01@@Z 120dba50 f   DOM_Text.obj
 0001:000daa70       ??0DOM_Text@xercesc_2_3@@IAE@PAVTextImpl@1@@Z 120dba70 f   DOM_Text.obj
 0001:000daa70       ??0DOM_Comment@xercesc_2_3@@IAE@PAVCommentImpl@1@@Z 120dba70 f   DOM_Text.obj
 0001:000daa90       ??1DOM_Text@xercesc_2_3@@QAE@XZ 120dba90 f   DOM_Text.obj
 0001:000daa90       ??1DOM_Comment@xercesc_2_3@@QAE@XZ 120dba90 f   DOM_Text.obj
 0001:000daaa0       ??4DOM_Text@xercesc_2_3@@QAEAAV01@ABV01@@Z 120dbaa0 f   DOM_Text.obj
 0001:000daaa0       ??4DOM_Comment@xercesc_2_3@@QAEAAV01@ABV01@@Z 120dbaa0 f   DOM_Text.obj
 0001:000daab0       ?createEntity@DOM_Document@xercesc_2_3@@QAE?AVDOM_Entity@2@ABVDOMString@2@@Z 120dbab0 f   DOM_Text.obj
 0001:000daab0       ?splitText@DOM_Text@xercesc_2_3@@QAE?AV12@I@Z 120dbab0 f   DOM_Text.obj
 0001:000daae0       ?isIgnorableWhitespace@DOM_Text@xercesc_2_3@@QAE_NXZ 120dbae0 f   DOM_Text.obj
 0001:000daaf0       ?getRoot@DOM_TreeWalker@xercesc_2_3@@QAE?AVDOM_Node@2@XZ 120dbaf0 f   DOM_TreeWalker.obj
 0001:000dab10       ?getWhatToShow@DOM_TreeWalker@xercesc_2_3@@QAEKXZ 120dbb10 f   DOM_TreeWalker.obj
 0001:000dab20       ?getStartOffset@DOM_Range@xercesc_2_3@@QBEIXZ 120dbb20 f   DOM_TreeWalker.obj
 0001:000dab20       ?getWhatToShow@DOM_NodeIterator@xercesc_2_3@@QAEKXZ 120dbb20 f   DOM_TreeWalker.obj
 0001:000dab20       ?getFilter@DOM_TreeWalker@xercesc_2_3@@QAEPAVDOM_NodeFilter@2@XZ 120dbb20 f   DOM_TreeWalker.obj
 0001:000dab30       ?setCurrentNode@DOM_TreeWalker@xercesc_2_3@@QAEXVDOM_Node@2@@Z 120dbb30 f   DOM_TreeWalker.obj
 0001:000dab90       ?parentNode@DOM_TreeWalker@xercesc_2_3@@QAE?AVDOM_Node@2@XZ 120dbb90 f   DOM_TreeWalker.obj
 0001:000dabb0       ?firstChild@DOM_TreeWalker@xercesc_2_3@@QAE?AVDOM_Node@2@XZ 120dbbb0 f   DOM_TreeWalker.obj
 0001:000dabd0       ?lastChild@DOM_TreeWalker@xercesc_2_3@@QAE?AVDOM_Node@2@XZ 120dbbd0 f   DOM_TreeWalker.obj
 0001:000dabf0       ?previousSibling@DOM_TreeWalker@xercesc_2_3@@QAE?AVDOM_Node@2@XZ 120dbbf0 f   DOM_TreeWalker.obj
 0001:000dac10       ?nextSibling@DOM_TreeWalker@xercesc_2_3@@QAE?AVDOM_Node@2@XZ 120dbc10 f   DOM_TreeWalker.obj
 0001:000dac30       ?previousNode@DOM_TreeWalker@xercesc_2_3@@QAE?AVDOM_Node@2@XZ 120dbc30 f   DOM_TreeWalker.obj
 0001:000dac50       ?nextNode@DOM_TreeWalker@xercesc_2_3@@QAE?AVDOM_Node@2@XZ 120dbc50 f   DOM_TreeWalker.obj
 0001:000dac70       ??0DOM_EntityReference@xercesc_2_3@@QAE@XZ 120dbc70 f   DOM_XMLDecl.obj
 0001:000dac70       ??0DOM_XMLDecl@xercesc_2_3@@QAE@XZ 120dbc70 f   DOM_XMLDecl.obj
 0001:000dac70       ??0DOM_Attr@xercesc_2_3@@QAE@XZ 120dbc70 f   DOM_XMLDecl.obj
 0001:000dac70       ??0DOM_DocumentType@xercesc_2_3@@QAE@XZ 120dbc70 f   DOM_XMLDecl.obj
 0001:000dac70       ??0DOM_ProcessingInstruction@xercesc_2_3@@QAE@XZ 120dbc70 f   DOM_XMLDecl.obj
 0001:000dac70       ??0DOM_DocumentFragment@xercesc_2_3@@QAE@XZ 120dbc70 f   DOM_XMLDecl.obj
 0001:000dac70       ??0DOM_Entity@xercesc_2_3@@QAE@XZ 120dbc70 f   DOM_XMLDecl.obj
 0001:000dac70       ??0DOM_Notation@xercesc_2_3@@QAE@XZ 120dbc70 f   DOM_XMLDecl.obj
 0001:000dac70       ??0DOM_CharacterData@xercesc_2_3@@QAE@XZ 120dbc70 f   DOM_XMLDecl.obj
 0001:000dac70       ??0DOM_Element@xercesc_2_3@@QAE@XZ 120dbc70 f   DOM_XMLDecl.obj
 0001:000dac70       ??0DOM_Document@xercesc_2_3@@QAE@XZ 120dbc70 f   DOM_XMLDecl.obj
 0001:000dac80       ??1DOM_Entity@xercesc_2_3@@QAE@XZ 120dbc80 f   DOM_XMLDecl.obj
 0001:000dac80       ??1DOM_XMLDecl@xercesc_2_3@@QAE@XZ 120dbc80 f   DOM_XMLDecl.obj
 0001:000dac80       ??1DOM_Attr@xercesc_2_3@@QAE@XZ 120dbc80 f   DOM_XMLDecl.obj
 0001:000dac80       ??1DOM_DocumentFragment@xercesc_2_3@@QAE@XZ 120dbc80 f   DOM_XMLDecl.obj
 0001:000dac80       ??1DOM_CharacterData@xercesc_2_3@@QAE@XZ 120dbc80 f   DOM_XMLDecl.obj
 0001:000dac80       ??1DOM_EntityReference@xercesc_2_3@@QAE@XZ 120dbc80 f   DOM_XMLDecl.obj
 0001:000dac80       ??1DOM_Notation@xercesc_2_3@@QAE@XZ 120dbc80 f   DOM_XMLDecl.obj
 0001:000dac80       ??1DOM_DocumentType@xercesc_2_3@@QAE@XZ 120dbc80 f   DOM_XMLDecl.obj
 0001:000dac80       ??1DOM_Document@xercesc_2_3@@QAE@XZ 120dbc80 f   DOM_XMLDecl.obj
 0001:000dac80       ??1DOM_Element@xercesc_2_3@@QAE@XZ 120dbc80 f   DOM_XMLDecl.obj
 0001:000dac80       ??1DOM_ProcessingInstruction@xercesc_2_3@@QAE@XZ 120dbc80 f   DOM_XMLDecl.obj
 0001:000dac90       ??4DOM_Entity@xercesc_2_3@@QAEAAV01@ABV01@@Z 120dbc90 f   DOM_XMLDecl.obj
 0001:000dac90       ??4DOM_Element@xercesc_2_3@@QAEAAV01@ABV01@@Z 120dbc90 f   DOM_XMLDecl.obj
 0001:000dac90       ??4DOM_Notation@xercesc_2_3@@QAEAAV01@ABV01@@Z 120dbc90 f   DOM_XMLDecl.obj
 0001:000dac90       ??4DOM_DocumentFragment@xercesc_2_3@@QAEAAV01@ABV01@@Z 120dbc90 f   DOM_XMLDecl.obj
 0001:000dac90       ??4DOM_XMLDecl@xercesc_2_3@@QAEAAV01@ABV01@@Z 120dbc90 f   DOM_XMLDecl.obj
 0001:000dac90       ??4DOM_Attr@xercesc_2_3@@QAEAAV01@ABV01@@Z 120dbc90 f   DOM_XMLDecl.obj
 0001:000dac90       ??4DOM_DocumentType@xercesc_2_3@@QAEAAV01@ABV01@@Z 120dbc90 f   DOM_XMLDecl.obj
 0001:000dac90       ??4DOM_CharacterData@xercesc_2_3@@QAEAAV01@ABV01@@Z 120dbc90 f   DOM_XMLDecl.obj
 0001:000dac90       ??4DOM_Document@xercesc_2_3@@QAEAAV01@ABV01@@Z 120dbc90 f   DOM_XMLDecl.obj
 0001:000dac90       ??4DOM_ProcessingInstruction@xercesc_2_3@@QAEAAV01@ABV01@@Z 120dbc90 f   DOM_XMLDecl.obj
 0001:000dac90       ??4DOM_EntityReference@xercesc_2_3@@QAEAAV01@ABV01@@Z 120dbc90 f   DOM_XMLDecl.obj
 0001:000daca0       ??4DOM_CharacterData@xercesc_2_3@@QAEAAV01@PBVDOM_NullPtr@1@@Z 120dbca0 f   DOM_XMLDecl.obj
 0001:000daca0       ??4DOM_Entity@xercesc_2_3@@QAEAAV01@PBVDOM_NullPtr@1@@Z 120dbca0 f   DOM_XMLDecl.obj
 0001:000daca0       ??4DOM_CDATASection@xercesc_2_3@@QAEAAV01@PBVDOM_NullPtr@1@@Z 120dbca0 f   DOM_XMLDecl.obj
 0001:000daca0       ??4DOM_DocumentFragment@xercesc_2_3@@QAEAAV01@PBVDOM_NullPtr@1@@Z 120dbca0 f   DOM_XMLDecl.obj
 0001:000daca0       ??4DOM_Element@xercesc_2_3@@QAEAAV01@PBVDOM_NullPtr@1@@Z 120dbca0 f   DOM_XMLDecl.obj
 0001:000daca0       ??4DOM_Attr@xercesc_2_3@@QAEAAV01@PBVDOM_NullPtr@1@@Z 120dbca0 f   DOM_XMLDecl.obj
 0001:000daca0       ??4DOM_DocumentType@xercesc_2_3@@QAEAAV01@PBVDOM_NullPtr@1@@Z 120dbca0 f   DOM_XMLDecl.obj
 0001:000daca0       ??4DOM_Document@xercesc_2_3@@QAEAAV01@PBVDOM_NullPtr@1@@Z 120dbca0 f   DOM_XMLDecl.obj
 0001:000daca0       ??4DOM_ProcessingInstruction@xercesc_2_3@@QAEAAV01@PBVDOM_NullPtr@1@@Z 120dbca0 f   DOM_XMLDecl.obj
 0001:000daca0       ??4DOM_EntityReference@xercesc_2_3@@QAEAAV01@PBVDOM_NullPtr@1@@Z 120dbca0 f   DOM_XMLDecl.obj
 0001:000daca0       ??4DOM_Notation@xercesc_2_3@@QAEAAV01@PBVDOM_NullPtr@1@@Z 120dbca0 f   DOM_XMLDecl.obj
 0001:000daca0       ??4DOM_Comment@xercesc_2_3@@QAEAAV01@PBVDOM_NullPtr@1@@Z 120dbca0 f   DOM_XMLDecl.obj
 0001:000daca0       ??4DOM_XMLDecl@xercesc_2_3@@QAEAAV01@PBVDOM_NullPtr@1@@Z 120dbca0 f   DOM_XMLDecl.obj
 0001:000daca0       ??4DOM_Text@xercesc_2_3@@QAEAAV01@PBVDOM_NullPtr@1@@Z 120dbca0 f   DOM_XMLDecl.obj
 0001:000dacb0       ?getVersion@DOM_XMLDecl@xercesc_2_3@@QBE?AVDOMString@2@XZ 120dbcb0 f   DOM_XMLDecl.obj
 0001:000dad20       ?getEncoding@DOM_XMLDecl@xercesc_2_3@@QBE?AVDOMString@2@XZ 120dbd20 f   DOM_XMLDecl.obj
 0001:000dad90       ?getStandalone@DOM_XMLDecl@xercesc_2_3@@QBE?AVDOMString@2@XZ 120dbd90 f   DOM_XMLDecl.obj
 0001:000dae00       ??0DomMemDebug@xercesc_2_3@@QAE@XZ 120dbe00 f   DomMemDebug.obj
 0001:000dae50       ??8DomMemDebug@xercesc_2_3@@QAE_NABV01@@Z 120dbe50 f   DomMemDebug.obj
 0001:000dae80       ??9DomMemDebug@xercesc_2_3@@QAE_NABV01@@Z 120dbe80 f   DomMemDebug.obj
 0001:000daec0       ??4DomMemDebug@xercesc_2_3@@QAEXABV01@@Z 120dbec0 f   DomMemDebug.obj
 0001:000daf00       ?print@DomMemDebug@xercesc_2_3@@QAEXXZ 120dbf00 f   DomMemDebug.obj
 0001:000daf30       ?printDifference@DomMemDebug@xercesc_2_3@@QAEXABV12@@Z 120dbf30 f   DomMemDebug.obj
 0001:000dafa0       ??_FDOMParser@xercesc_2_3@@QAEXXZ 120dbfa0 f i DOMParser.obj
 0001:000dafb0       ?getDocument@DOMParser@xercesc_2_3@@QAE?AVDOM_Document@2@XZ 120dbfb0 f i DOMParser.obj
 0001:000dafd0       ?getExpandEntityReferences@DOMParser@xercesc_2_3@@QBE_NXZ 120dbfd0 f i DOMParser.obj
 0001:000dafe0       ?setExpandEntityReferences@DOMParser@xercesc_2_3@@QAEX_N@Z 120dbfe0 f i DOMParser.obj
 0001:000daff0       ?getCurrentNode@DOMParser@xercesc_2_3@@IAE?AVDOM_Node@2@XZ 120dbff0 f i DOMParser.obj
 0001:000db010       ?setCurrentNode@DOMParser@xercesc_2_3@@IAEXVDOM_Node@2@@Z 120dc010 f i DOMParser.obj
 0001:000db060       ?setDocument@DOMParser@xercesc_2_3@@IAEXVDOM_Document@2@@Z 120dc060 f i DOMParser.obj
 0001:000db0b0       ??0DOMParser@xercesc_2_3@@QAE@QAVXMLValidator@1@QAVMemoryManager@1@@Z 120dc0b0 f   DOMParser.obj
 0001:000db200       ??_EDOMParser@xercesc_2_3@@UAEPAXI@Z 120dc200 f i DOMParser.obj
 0001:000db260       ??1DOMParser@xercesc_2_3@@UAE@XZ 120dc260 f   DOMParser.obj
 0001:000db380       ?initialize@DOMParser@xercesc_2_3@@AAEXXZ 120dc380 f   DOMParser.obj
 0001:000db520       ?cleanUp@DOMParser@xercesc_2_3@@AAEXXZ 120dc520 f   DOMParser.obj
 0001:000db590       ?reset@DOMParser@xercesc_2_3@@QAEXXZ 120dc590 f   DOMParser.obj
 0001:000db620       ?getValidator@DOMParser@xercesc_2_3@@QBEABVXMLValidator@2@XZ 120dc620 f   DOMParser.obj
 0001:000db630       ?getDoNamespaces@DOMParser@xercesc_2_3@@QBE_NXZ 120dc630 f   DOMParser.obj
 0001:000db640       ?getExitOnFirstFatalError@DOMParser@xercesc_2_3@@QBE_NXZ 120dc640 f   DOMParser.obj
 0001:000db650       ?getValidationConstraintFatal@DOMParser@xercesc_2_3@@QBE_NXZ 120dc650 f   DOMParser.obj
 0001:000db660       ?getValidationScheme@DOMParser@xercesc_2_3@@QBE?AW4ValSchemes@12@XZ 120dc660 f   DOMParser.obj
 0001:000db680       ?getDoSchema@DOMParser@xercesc_2_3@@QBE_NXZ 120dc680 f   DOMParser.obj
 0001:000db690       ?getValidationSchemaFullChecking@DOMParser@xercesc_2_3@@QBE_NXZ 120dc690 f   DOMParser.obj
 0001:000db6a0       ?getErrorCount@DOMParser@xercesc_2_3@@QBEHXZ 120dc6a0 f   DOMParser.obj
 0001:000db6b0       ?getExternalSchemaLocation@DOMParser@xercesc_2_3@@QBEPAGXZ 120dc6b0 f   DOMParser.obj
 0001:000db6c0       ?getExternalNoNamespaceSchemaLocation@DOMParser@xercesc_2_3@@QBEPAGXZ 120dc6c0 f   DOMParser.obj
 0001:000db6d0       ?isCachingGrammarFromParse@DOMParser@xercesc_2_3@@QBE_NXZ 120dc6d0 f   DOMParser.obj
 0001:000db6e0       ?isUsingCachedGrammarInParse@DOMParser@xercesc_2_3@@QBE_NXZ 120dc6e0 f   DOMParser.obj
 0001:000db6f0       ?getGrammar@XercesDOMParser@xercesc_2_3@@QAEPAVGrammar@2@QBG@Z 120dc6f0 f   DOMParser.obj
 0001:000db6f0       ?getGrammar@DOMParser@xercesc_2_3@@QAEPAVGrammar@2@QBG@Z 120dc6f0 f   DOMParser.obj
 0001:000db700       ?getRootGrammar@DOMParser@xercesc_2_3@@QAEPAVGrammar@2@XZ 120dc700 f   DOMParser.obj
 0001:000db710       ?getURIText@DOMParser@xercesc_2_3@@QBEPBGI@Z 120dc710 f   DOMParser.obj
 0001:000db720       ?getCalculateSrcOfs@DOMParser@xercesc_2_3@@QBE_NXZ 120dc720 f   DOMParser.obj
 0001:000db730       ?getStandardUriConformant@DOMParser@xercesc_2_3@@QBE_NXZ 120dc730 f   DOMParser.obj
 0001:000db740       ?getSrcOffset@DOMParser@xercesc_2_3@@QBEIXZ 120dc740 f   DOMParser.obj
 0001:000db750       ?setDoNamespaces@DOMParser@xercesc_2_3@@QAEX_N@Z 120dc750 f   DOMParser.obj
 0001:000db760       ?setErrorHandler@DOMParser@xercesc_2_3@@QAEXQAVErrorHandler@2@@Z 120dc760 f   DOMParser.obj
 0001:000db7a0       ?setEntityResolver@DOMParser@xercesc_2_3@@QAEXQAVEntityResolver@2@@Z 120dc7a0 f   DOMParser.obj
 0001:000db7c0       ?setExitOnFirstFatalError@DOMParser@xercesc_2_3@@QAEX_N@Z 120dc7c0 f   DOMParser.obj
 0001:000db7d0       ?setValidationConstraintFatal@DOMParser@xercesc_2_3@@QAEX_N@Z 120dc7d0 f   DOMParser.obj
 0001:000db7e0       ?setValidationScheme@DOMParser@xercesc_2_3@@QAEXW4ValSchemes@12@@Z 120dc7e0 f   DOMParser.obj
 0001:000db830       ?setDoSchema@DOMParser@xercesc_2_3@@QAEX_N@Z 120dc830 f   DOMParser.obj
 0001:000db840       ?setValidationSchemaFullChecking@DOMParser@xercesc_2_3@@QAEX_N@Z 120dc840 f   DOMParser.obj
 0001:000db850       ?setExternalSchemaLocation@DOMParser@xercesc_2_3@@QAEXQBG@Z 120dc850 f   DOMParser.obj
 0001:000db8d0       ?setExternalNoNamespaceSchemaLocation@DOMParser@xercesc_2_3@@QAEXQBG@Z 120dc8d0 f   DOMParser.obj
 0001:000db950       ?setExternalSchemaLocation@DOMParser@xercesc_2_3@@QAEXQBD@Z 120dc950 f   DOMParser.obj
 0001:000db990       ?setExternalNoNamespaceSchemaLocation@DOMParser@xercesc_2_3@@QAEXQBD@Z 120dc990 f   DOMParser.obj
 0001:000db9d0       ?cacheGrammarFromParse@DOMParser@xercesc_2_3@@QAEX_N@Z 120dc9d0 f   DOMParser.obj
 0001:000db9f0       ?useCachedGrammarInParse@DOMParser@xercesc_2_3@@QAEX_N@Z 120dc9f0 f   DOMParser.obj
 0001:000dba10       ?setCalculateSrcOfs@DOMParser@xercesc_2_3@@QAEX_N@Z 120dca10 f   DOMParser.obj
 0001:000dba20       ?setStandardUriConformant@DOMParser@xercesc_2_3@@QAEX_N@Z 120dca20 f   DOMParser.obj
 0001:000dba30       ?useScanner@DOMParser@xercesc_2_3@@QAEXQBG@Z 120dca30 f   DOMParser.obj
 0001:000dba90       ?parse@DOMParser@xercesc_2_3@@QAEXABVInputSource@2@@Z 120dca90 f   DOMParser.obj
 0001:000dbb40       ?parse@DOMParser@xercesc_2_3@@QAEXQBG@Z 120dcb40 f   DOMParser.obj
 0001:000dbbf0       ?parse@DOMParser@xercesc_2_3@@QAEXQBD@Z 120dcbf0 f   DOMParser.obj
 0001:000dbca0       ?parseFirst@DOMParser@xercesc_2_3@@QAE_NQBGAAVXMLPScanToken@2@@Z 120dcca0 f   DOMParser.obj
 0001:000dbcf0       ?parseFirst@DOMParser@xercesc_2_3@@QAE_NQBDAAVXMLPScanToken@2@@Z 120dccf0 f   DOMParser.obj
 0001:000dbd40       ?parseFirst@DOMParser@xercesc_2_3@@QAE_NABVInputSource@2@AAVXMLPScanToken@2@@Z 120dcd40 f   DOMParser.obj
 0001:000dbd90       ?parseNext@DOMParser@xercesc_2_3@@QAE_NAAVXMLPScanToken@2@@Z 120dcd90 f   DOMParser.obj
 0001:000dbda0       ?parseReset@DOMParser@xercesc_2_3@@QAEXAAVXMLPScanToken@2@@Z 120dcda0 f   DOMParser.obj
 0001:000dbdc0       ?error@DOMParser@xercesc_2_3@@UAEXIQBGW4ErrTypes@XMLErrorReporter@2@000JJ@Z 120dcdc0 f   DOMParser.obj
 0001:000dbe80       ?resolveEntity@DOMParser@xercesc_2_3@@UAEPAVInputSource@2@QBG00@Z 120dce80 f   DOMParser.obj
 0001:000dbea0       ?docCharacters@DOMParser@xercesc_2_3@@UAEXQBGI_N@Z 120dcea0 f   DOMParser.obj
 0001:000dc040       ?docComment@DOMParser@xercesc_2_3@@UAEXQBG@Z 120dd040 f   DOMParser.obj
 0001:000dc0e0       ?docPI@DOMParser@xercesc_2_3@@UAEXQBG0@Z 120dd0e0 f   DOMParser.obj
 0001:000dc1b0       ?endEntityReference@DOMParser@xercesc_2_3@@UAEXABVXMLEntityDecl@2@@Z 120dd1b0 f   DOMParser.obj
 0001:000dc240       ?endElement@DOMParser@xercesc_2_3@@UAEXABVXMLElementDecl@2@I_NQBG@Z 120dd240 f   DOMParser.obj
 0001:000dc2c0       ?ignorableWhitespace@DOMParser@xercesc_2_3@@UAEXQBGI_N@Z 120dd2c0 f   DOMParser.obj
 0001:000dc3f0       ?resetDocument@DOMParser@xercesc_2_3@@UAEXXZ 120dd3f0 f   DOMParser.obj
 0001:000dc400       ?startDocument@DOMParser@xercesc_2_3@@UAEXXZ 120dd400 f   DOMParser.obj
 0001:000dc430       ?endDocument@DOMParser@xercesc_2_3@@UAEXXZ 120dd430 f   DOMParser.obj
 0001:000dc440       ?startElement@DOMParser@xercesc_2_3@@UAEXABVXMLElementDecl@2@IQBGABV?$RefVectorOf@VXMLAttr@xercesc_2_3@@@2@I_N3@Z 120dd440 f   DOMParser.obj
 0001:000dca70       ?startEntityReference@DOMParser@xercesc_2_3@@UAEXABVXMLEntityDecl@2@@Z 120dda70 f   DOMParser.obj
 0001:000dcc00       ?XMLDecl@DOMParser@xercesc_2_3@@UAEXQBG000@Z 120ddc00 f   DOMParser.obj
 0001:000dccf0       ?getDoValidation@DOMParser@xercesc_2_3@@QBE_NXZ 120ddcf0 f   DOMParser.obj
 0001:000dcd00       ?setDoValidation@DOMParser@xercesc_2_3@@QAEX_N@Z 120ddd00 f   DOMParser.obj
 0001:000dcd30       ?attDef@DOMParser@xercesc_2_3@@UAEXABVDTDElementDecl@2@ABVDTDAttDef@2@_N@Z 120ddd30 f   DOMParser.obj
 0001:000dd090       ?doctypeComment@DOMParser@xercesc_2_3@@UAEXQBG@Z 120de090 f   DOMParser.obj
 0001:000dd160       ?doctypeDecl@DOMParser@xercesc_2_3@@UAEXABVDTDElementDecl@2@QBG1_N2@Z 120de160 f   DOMParser.obj
 0001:000dd270       ?doctypePI@DOMParser@xercesc_2_3@@UAEXQBG0@Z 120de270 f   DOMParser.obj
 0001:000dd330       ?doctypeWhitespace@DOMParser@xercesc_2_3@@UAEXQBGI@Z 120de330 f   DOMParser.obj
 0001:000dd360       ?elementDecl@DOMParser@xercesc_2_3@@UAEXABVDTDElementDecl@2@_N@Z 120de360 f   DOMParser.obj
 0001:000dd450       ?endAttList@DOMParser@xercesc_2_3@@UAEXABVDTDElementDecl@2@@Z 120de450 f   DOMParser.obj
 0001:000dd770       ?endIntSubset@DOMParser@xercesc_2_3@@UAEXXZ 120de770 f   DOMParser.obj
 0001:000dd780       ?entityDecl@DOMParser@xercesc_2_3@@UAEXABVDTDEntityDecl@2@_N1@Z 120de780 f   DOMParser.obj
 0001:000ddb20       ?resetDocType@DOMParser@xercesc_2_3@@UAEXXZ 120deb20 f   DOMParser.obj
 0001:000ddb30       ?notationDecl@DOMParser@xercesc_2_3@@UAEXABVXMLNotationDecl@2@_N@Z 120deb30 f   DOMParser.obj
 0001:000ddc30       ?startIntSubset@DOMParser@xercesc_2_3@@UAEXXZ 120dec30 f   DOMParser.obj
 0001:000ddc40       ?loadGrammar@DOMParser@xercesc_2_3@@QAEPAVGrammar@2@QBDF_N@Z 120dec40 f   DOMParser.obj
 0001:000ddcf0       ?loadGrammar@DOMParser@xercesc_2_3@@QAEPAVGrammar@2@QBGF_N@Z 120decf0 f   DOMParser.obj
 0001:000ddda0       ?loadGrammar@DOMParser@xercesc_2_3@@QAEPAVGrammar@2@ABVInputSource@2@F_N@Z 120deda0 f   DOMParser.obj
 0001:000dde50       ?resetCachedGrammarPool@XercesDOMParser@xercesc_2_3@@QAEXXZ 120dee50 f   DOMParser.obj
 0001:000dde50       ?resetCachedGrammarPool@DOMParser@xercesc_2_3@@QAEXXZ 120dee50 f   DOMParser.obj
 0001:000dde60       ?pop@?$ValueStackOf@VDOM_Node@xercesc_2_3@@@xercesc_2_3@@QAE?AVDOM_Node@2@XZ 120dee60 f i DOMParser.obj
 0001:000ddfe0       ??_EDOMParser@xercesc_2_3@@W3AEPAXI@Z 120defe0 f i DOMParser.obj
 0001:000ddff0       ??_EDOMParser@xercesc_2_3@@W7AEPAXI@Z 120deff0 f i DOMParser.obj
 0001:000de000       ??_EDOMParser@xercesc_2_3@@WM@AEPAXI@Z 120df000 f i DOMParser.obj
 0001:000de050       ?allocateBuffer@DOMStringData@xercesc_2_3@@SAPAV12@I@Z 120df050 f   DOMString.obj
 0001:000de150       ??2DOMStringHandle@xercesc_2_3@@SAPAXI@Z 120df150 f   DOMString.obj
 0001:000de2c0       ??3DOMStringHandle@xercesc_2_3@@SAXPAX@Z 120df2c0 f   DOMString.obj
 0001:000de420       ?createNewStringHandle@DOMStringHandle@xercesc_2_3@@SAPAV12@I@Z 120df420 f   DOMString.obj
 0001:000de5b0       ?cloneStringHandle@DOMStringHandle@xercesc_2_3@@QAEPAV12@XZ 120df5b0 f   DOMString.obj
 0001:000de730       ??0DOMString@xercesc_2_3@@QAE@ABV01@@Z 120df730 f   DOMString.obj
 0001:000de760       ??0DOMString@xercesc_2_3@@QAE@PBG@Z 120df760 f   DOMString.obj
 0001:000de7d0       ??0DOMString@xercesc_2_3@@QAE@PBGI@Z 120df7d0 f   DOMString.obj
 0001:000de830       ??0DOMString@xercesc_2_3@@QAE@PBD@Z 120df830 f   DOMString.obj
 0001:000dea00       ??0DOMString@xercesc_2_3@@QAE@H@Z 120dfa00 f   DOMString.obj
 0001:000dea10       ??1DOMString@xercesc_2_3@@QAE@XZ 120dfa10 f   DOMString.obj
 0001:000dea80       ??4DOMString@xercesc_2_3@@QAEAAV01@ABV01@@Z 120dfa80 f   DOMString.obj
 0001:000deb10       ??4DOMString@xercesc_2_3@@QAEAAV01@PAVDOM_NullPtr@1@@Z 120dfb10 f   DOMString.obj
 0001:000deb90       ?reserve@DOMString@xercesc_2_3@@QAEXI@Z 120dfb90 f   DOMString.obj
 0001:000debb0       ?appendData@DOMString@xercesc_2_3@@QAEXABV12@@Z 120dfbb0 f   DOMString.obj
 0001:000ded20       ?appendData@DOMString@xercesc_2_3@@QAEXG@Z 120dfd20 f   DOMString.obj
 0001:000dede0       ?appendData@DOMString@xercesc_2_3@@QAEXPBG@Z 120dfde0 f   DOMString.obj
 0001:000defd0       ??YDOMString@xercesc_2_3@@QAEAAV01@ABV01@@Z 120dffd0 f   DOMString.obj
 0001:000deff0       ??YDOMString@xercesc_2_3@@QAEAAV01@PBG@Z 120dfff0 f   DOMString.obj
 0001:000df010       ??YDOMString@xercesc_2_3@@QAEAAV01@G@Z 120e0010 f   DOMString.obj
 0001:000df030       ?charAt@DOMString@xercesc_2_3@@QBEGI@Z 120e0030 f   DOMString.obj
 0001:000df050       ?clone@DOMString@xercesc_2_3@@QBE?AV12@XZ 120e0050 f   DOMString.obj
 0001:000df2f0       ?getMutex@DOMStringHandle@xercesc_2_3@@CAAAVXMLMutex@2@XZ 120e02f0 f i DOMString.obj
 0001:000df3d0       ?deleteData@DOMString@xercesc_2_3@@QAEXII@Z 120e03d0 f   DOMString.obj
 0001:000df570       ?equals@DOMString@xercesc_2_3@@QBE_NABV12@@Z 120e0570 f   DOMString.obj
 0001:000df5e0       ?equals@DOMString@xercesc_2_3@@QBE_NPBG@Z 120e05e0 f   DOMString.obj
 0001:000df660       ?insertData@DOMString@xercesc_2_3@@QAEXIABV12@@Z 120e0660 f   DOMString.obj
 0001:000df920       ?removeRef@DOMStringData@xercesc_2_3@@QAEXXZ 120e0920 f i DOMString.obj
 0001:000df960       ?length@DOMString@xercesc_2_3@@QBEIXZ 120e0960 f   DOMString.obj
 0001:000df970       ?print@DOMString@xercesc_2_3@@QBEXXZ 120e0970 f   DOMString.obj
 0001:000df9b0       ?println@DOMString@xercesc_2_3@@QBEXXZ 120e09b0 f   DOMString.obj
 0001:000dfa00       ?rawBuffer@DOMString@xercesc_2_3@@QBEPBGXZ 120e0a00 f   DOMString.obj
 0001:000dfa10       ?transcode@DOMString@xercesc_2_3@@QBEPADXZ 120e0a10 f   DOMString.obj
 0001:000dfd10       ?transcode@DOMString@xercesc_2_3@@QBEPADQAVMemoryManager@2@@Z 120e0d10 f   DOMString.obj
 0001:000e0030       ?transcode@DOMString@xercesc_2_3@@SA?AV12@PBD@Z 120e1030 f   DOMString.obj
 0001:000e0050       ?compareString@DOMString@xercesc_2_3@@QBEHABV12@@Z 120e1050 f   DOMString.obj
 0001:000e00c0       ?substringData@DOMString@xercesc_2_3@@QBE?AV12@II@Z 120e10c0 f   DOMString.obj
 0001:000e0280       ??Hxercesc_2_3@@YA?AVDOMString@0@ABV10@0@Z 120e1280 f   DOMString.obj
 0001:000e04a0       ??Hxercesc_2_3@@YA?AVDOMString@0@ABV10@PBG@Z 120e14a0 f   DOMString.obj
 0001:000e06f0       ??_GXMLMutex@xercesc_2_3@@QAEPAXI@Z 120e16f0 f i DOMString.obj
 0001:000e0710       ??Hxercesc_2_3@@YA?AVDOMString@0@PBGABV10@@Z 120e1710 f   DOMString.obj
 0001:000e0930       ??Hxercesc_2_3@@YA?AVDOMString@0@ABV10@G@Z 120e1930 f   DOMString.obj
 0001:000e0b50       ??Hxercesc_2_3@@YA?AVDOMString@0@GABV10@@Z 120e1b50 f   DOMString.obj
 0001:000e0dc0       ??0DStringPool@xercesc_2_3@@QAE@HQAVMemoryManager@1@@Z 120e1dc0 f   DStringPool.obj
 0001:000e0e00       ??1DStringPool@xercesc_2_3@@QAE@XZ 120e1e00 f   DStringPool.obj
 0001:000e0e60       ??1DStringPoolEntry@xercesc_2_3@@QAE@XZ 120e1e60 f i DStringPool.obj
 0001:000e0e70       ?getPooledString@DStringPool@xercesc_2_3@@QAEABVDOMString@2@PBG@Z 120e1e70 f   DStringPool.obj
 0001:000e0f60       ?getPooledString@DStringPool@xercesc_2_3@@QAEABVDOMString@2@ABV32@@Z 120e1f60 f   DStringPool.obj
 0001:000e1060       ?getStaticString@DStringPool@xercesc_2_3@@SAABVDOMString@2@PBDPAPAV32@P6AXXZAAVXMLRegisterCleanup@2@@Z 120e2060 f   DStringPool.obj
 0001:000e1150       ??_OElementDefinitionImpl@xercesc_2_3@@QAEXABV01@@Z 120e2150 f i ElementDefinitionImpl.obj
 0001:000e1160       ??0ElementDefinitionImpl@xercesc_2_3@@QAE@PAVDocumentImpl@1@ABVDOMString@1@@Z 120e2160 f   ElementDefinitionImpl.obj
 0001:000e11f0       ??_EElementDefinitionImpl@xercesc_2_3@@UAEPAXI@Z 120e21f0 f i ElementDefinitionImpl.obj
 0001:000e1250       ??0ElementDefinitionImpl@xercesc_2_3@@QAE@ABV01@_N@Z 120e2250 f   ElementDefinitionImpl.obj
 0001:000e12f0       ??1ElementDefinitionImpl@xercesc_2_3@@UAE@XZ 120e22f0 f   ElementDefinitionImpl.obj
 0001:000e1350       ?cloneNode@ElementDefinitionImpl@xercesc_2_3@@UAEPAVNodeImpl@2@_N@Z 120e2350 f   ElementDefinitionImpl.obj
 0001:000e1410       ?getNodeType@ElementDefinitionImpl@xercesc_2_3@@UAEFXZ 120e2410 f   ElementDefinitionImpl.obj
 0001:000e1440       ??0ElementImpl@xercesc_2_3@@QAE@PAVDocumentImpl@1@ABVDOMString@1@@Z 120e2440 f   ElementImpl.obj
 0001:000e14e0       ??_EElementImpl@xercesc_2_3@@UAEPAXI@Z 120e24e0 f i ElementImpl.obj
 0001:000e1540       ??0ElementImpl@xercesc_2_3@@QAE@ABV01@_N@Z 120e2540 f   ElementImpl.obj
 0001:000e1610       ??1ElementImpl@xercesc_2_3@@UAE@XZ 120e2610 f   ElementImpl.obj
 0001:000e1680       ?cloneNode@ElementImpl@xercesc_2_3@@UAEPAVNodeImpl@2@_N@Z 120e2680 f   ElementImpl.obj
 0001:000e1700       ?setOwnerDocument@ElementImpl@xercesc_2_3@@UAEXPAVDocumentImpl@2@@Z 120e2700 f   ElementImpl.obj
 0001:000e1720       ?getAttribute@ElementImpl@xercesc_2_3@@UAE?AVDOMString@2@ABV32@@Z 120e2720 f   ElementImpl.obj
 0001:000e17d0       ?getAttributeNode@ElementImpl@xercesc_2_3@@UAEPAVAttrImpl@2@ABVDOMString@2@@Z 120e27d0 f   ElementImpl.obj
 0001:000e17f0       ?getElementsByTagName@ElementImpl@xercesc_2_3@@UAEPAVDeepNodeListImpl@2@ABVDOMString@2@@Z 120e27f0 f   ElementImpl.obj
 0001:000e1870       ?removeAttribute@ElementImpl@xercesc_2_3@@UAEXABVDOMString@2@@Z 120e2870 f   ElementImpl.obj
 0001:000e1920       ?removeAttributeNode@ElementImpl@xercesc_2_3@@UAEPAVAttrImpl@2@PAV32@@Z 120e2920 f   ElementImpl.obj
 0001:000e1a60       ?setAttribute@ElementImpl@xercesc_2_3@@UAEPAVAttrImpl@2@ABVDOMString@2@0@Z 120e2a60 f   ElementImpl.obj
 0001:000e1b70       ?setAttributeNode@ElementImpl@xercesc_2_3@@UAEPAVAttrImpl@2@PAV32@@Z 120e2b70 f   ElementImpl.obj
 0001:000e1cc0       ?setReadOnly@ElementImpl@xercesc_2_3@@UAEX_N0@Z 120e2cc0 f   ElementImpl.obj
 0001:000e1cf0       ?getAttributeNS@ElementImpl@xercesc_2_3@@UAE?AVDOMString@2@ABV32@0@Z 120e2cf0 f   ElementImpl.obj
 0001:000e1dc0       ?setAttributeNS@ElementImpl@xercesc_2_3@@UAEPAVAttrImpl@2@ABVDOMString@2@00@Z 120e2dc0 f   ElementImpl.obj
 0001:000e1ed0       ?removeAttributeNS@ElementImpl@xercesc_2_3@@UAEXABVDOMString@2@0@Z 120e2ed0 f   ElementImpl.obj
 0001:000e1f90       ?getAttributeNodeNS@ElementImpl@xercesc_2_3@@UAEPAVAttrImpl@2@ABVDOMString@2@0@Z 120e2f90 f   ElementImpl.obj
 0001:000e1fb0       ?setAttributeNodeNS@ElementImpl@xercesc_2_3@@UAEPAVAttrImpl@2@PAV32@@Z 120e2fb0 f   ElementImpl.obj
 0001:000e2130       ?getElementsByTagNameNS@ElementImpl@xercesc_2_3@@UAEPAVDeepNodeListImpl@2@ABVDOMString@2@0@Z 120e3130 f   ElementImpl.obj
 0001:000e21b0       ?hasAttributes@ElementImpl@xercesc_2_3@@UAE_NXZ 120e31b0 f   ElementImpl.obj
 0001:000e21d0       ?hasAttribute@ElementImpl@xercesc_2_3@@UAE_NABVDOMString@2@@Z 120e31d0 f   ElementImpl.obj
 0001:000e21f0       ?hasAttributeNS@ElementImpl@xercesc_2_3@@UAE_NABVDOMString@2@0@Z 120e31f0 f   ElementImpl.obj
 0001:000e2210       ?NNM_cloneMap@ElementImpl@xercesc_2_3@@UAEPAVNamedNodeMapImpl@2@PAVNodeImpl@2@@Z 120e3210 f   ElementImpl.obj
 0001:000e2240       ?NNM_findNamePoint@ElementImpl@xercesc_2_3@@UAEHABVDOMString@2@@Z 120e3240 f   ElementImpl.obj
 0001:000e2270       ?NNM_getLength@ElementImpl@xercesc_2_3@@UAEIXZ 120e3270 f   ElementImpl.obj
 0001:000e2290       ?NNM_getNamedItem@ElementImpl@xercesc_2_3@@UAEPAVNodeImpl@2@ABVDOMString@2@@Z 120e3290 f   ElementImpl.obj
 0001:000e22c0       ?NNM_item@ElementImpl@xercesc_2_3@@UAEPAVNodeImpl@2@I@Z 120e32c0 f   ElementImpl.obj
 0001:000e22f0       ?NNM_removeAll@ElementImpl@xercesc_2_3@@UAEXXZ 120e32f0 f   ElementImpl.obj
 0001:000e2310       ?NNM_removeNamedItem@ElementImpl@xercesc_2_3@@UAEPAVNodeImpl@2@ABVDOMString@2@@Z 120e3310 f   ElementImpl.obj
 0001:000e2390       ?NNM_setNamedItem@ElementImpl@xercesc_2_3@@UAEPAVNodeImpl@2@PAV32@@Z 120e3390 f   ElementImpl.obj
 0001:000e2420       ?NNM_setReadOnly@ElementImpl@xercesc_2_3@@UAEX_N0@Z 120e3420 f   ElementImpl.obj
 0001:000e2450       ?NNM_findNamePoint@ElementImpl@xercesc_2_3@@UAEHABVDOMString@2@0@Z 120e3450 f   ElementImpl.obj
 0001:000e2480       ?NNM_getNamedItemNS@ElementImpl@xercesc_2_3@@UAEPAVNodeImpl@2@ABVDOMString@2@0@Z 120e3480 f   ElementImpl.obj
 0001:000e24b0       ?NNM_setNamedItemNS@ElementImpl@xercesc_2_3@@UAEPAVNodeImpl@2@PAV32@@Z 120e34b0 f   ElementImpl.obj
 0001:000e2540       ?NNM_removeNamedItemNS@ElementImpl@xercesc_2_3@@UAEPAVNodeImpl@2@ABVDOMString@2@0@Z 120e3540 f   ElementImpl.obj
 0001:000e25c0       ?NNM_setOwnerDocument@ElementImpl@xercesc_2_3@@UAEXPAVDocumentImpl@2@@Z 120e35c0 f   ElementImpl.obj
 0001:000e25f0       ?getDefaultAttributes@ElementImpl@xercesc_2_3@@UAEPAVAttrMapImpl@2@XZ 120e35f0 f   ElementImpl.obj
 0001:000e26b0       ?setupDefaultAttributes@ElementImpl@xercesc_2_3@@UAEXXZ 120e36b0 f   ElementImpl.obj
 0001:000e2770       ?reinitElementImpl@ElementImpl@xercesc_2_3@@SAXXZ 120e3770 f   ElementImpl.obj
 0001:000e27a0       ??0ElementNSImpl@xercesc_2_3@@QAE@PAVDocumentImpl@1@ABVDOMString@1@@Z 120e37a0 f   ElementNSImpl.obj
 0001:000e2830       ??_EElementNSImpl@xercesc_2_3@@UAEPAXI@Z 120e3830 f i ElementNSImpl.obj
 0001:000e2890       ??0ElementNSImpl@xercesc_2_3@@QAE@PAVDocumentImpl@1@ABVDOMString@1@1@Z 120e3890 f   ElementNSImpl.obj
 0001:000e2aa0       ??0ElementNSImpl@xercesc_2_3@@QAE@ABV01@_N@Z 120e3aa0 f   ElementNSImpl.obj
 0001:000e2b70       ?cloneNode@ElementNSImpl@xercesc_2_3@@UAEPAVNodeImpl@2@_N@Z 120e3b70 f   ElementNSImpl.obj
 0001:000e2bf0       ?getPrefix@ElementNSImpl@xercesc_2_3@@UAE?AVDOMString@2@XZ 120e3bf0 f   ElementNSImpl.obj
 0001:000e2c40       ?setPrefix@ElementNSImpl@xercesc_2_3@@UAEXABVDOMString@2@@Z 120e3c40 f   ElementNSImpl.obj
 0001:000e2ec0       ??0EntityImpl@xercesc_2_3@@QAE@PAVDocumentImpl@1@ABVDOMString@1@@Z 120e3ec0 f   EntityImpl.obj
 0001:000e2f80       ??_EEntityImpl@xercesc_2_3@@UAEPAXI@Z 120e3f80 f i EntityImpl.obj
 0001:000e2fe0       ??0EntityImpl@xercesc_2_3@@QAE@ABV01@_N@Z 120e3fe0 f   EntityImpl.obj
 0001:000e3140       ??1EntityImpl@xercesc_2_3@@UAE@XZ 120e4140 f   EntityImpl.obj
 0001:000e31c0       ?cloneNode@EntityImpl@xercesc_2_3@@UAEPAVNodeImpl@2@_N@Z 120e41c0 f   EntityImpl.obj
 0001:000e3240       ?getNotationName@EntityImpl@xercesc_2_3@@UAE?AVDOMString@2@XZ 120e4240 f   EntityImpl.obj
 0001:000e3240       ?getLocalName@ElementNSImpl@xercesc_2_3@@UAE?AVDOMString@2@XZ 120e4240 f   EntityImpl.obj
 0001:000e3260       ?getPublicId@EntityImpl@xercesc_2_3@@UAE?AVDOMString@2@XZ 120e4260 f   EntityImpl.obj
 0001:000e3280       ?getNamespaceURI@ElementNSImpl@xercesc_2_3@@UAE?AVDOMString@2@XZ 120e4280 f   EntityImpl.obj
 0001:000e3280       ?getSystemId@EntityImpl@xercesc_2_3@@UAE?AVDOMString@2@XZ 120e4280 f   EntityImpl.obj
 0001:000e32a0       ?setNotationName@EntityImpl@xercesc_2_3@@UAEXABVDOMString@2@@Z 120e42a0 f   EntityImpl.obj
 0001:000e32b0       ?setPublicId@EntityImpl@xercesc_2_3@@UAEXABVDOMString@2@@Z 120e42b0 f   EntityImpl.obj
 0001:000e32c0       ?setSystemId@EntityImpl@xercesc_2_3@@UAEXABVDOMString@2@@Z 120e42c0 f   EntityImpl.obj
 0001:000e32d0       ?setEntityRef@EntityImpl@xercesc_2_3@@UAEXPAVEntityReferenceImpl@2@@Z 120e42d0 f   EntityImpl.obj
 0001:000e32f0       ?cloneEntityRefTree@EntityImpl@xercesc_2_3@@AAEXXZ 120e42f0 f   EntityImpl.obj
 0001:000e3330       ?getFirstChild@EntityImpl@xercesc_2_3@@UAEPAVNodeImpl@2@XZ 120e4330 f   EntityImpl.obj
 0001:000e3370       ?getLastChild@EntityImpl@xercesc_2_3@@UAEPAVNodeImpl@2@XZ 120e4370 f   EntityImpl.obj
 0001:000e33b0       ?getChildNodes@EntityImpl@xercesc_2_3@@UAEPAVNodeListImpl@2@XZ 120e43b0 f   EntityImpl.obj
 0001:000e33f0       ?hasChildNodes@EntityImpl@xercesc_2_3@@UAE_NXZ 120e43f0 f   EntityImpl.obj
 0001:000e3440       ?item@EntityImpl@xercesc_2_3@@UAEPAVNodeImpl@2@I@Z 120e4440 f   EntityImpl.obj
 0001:000e34a0       ??0EntityReferenceImpl@xercesc_2_3@@QAE@PAVDocumentImpl@1@ABVDOMString@1@@Z 120e44a0 f   EntityReferenceImpl.obj
 0001:000e35a0       ??_EEntityReferenceImpl@xercesc_2_3@@UAEPAXI@Z 120e45a0 f i EntityReferenceImpl.obj
 0001:000e3600       ??0EntityReferenceImpl@xercesc_2_3@@QAE@ABV01@_N@Z 120e4600 f   EntityReferenceImpl.obj
 0001:000e36b0       ??1EntityReferenceImpl@xercesc_2_3@@UAE@XZ 120e46b0 f   EntityReferenceImpl.obj
 0001:000e3710       ?cloneNode@EntityReferenceImpl@xercesc_2_3@@UAEPAVNodeImpl@2@_N@Z 120e4710 f   EntityReferenceImpl.obj
 0001:000e37e0       ?setReadOnly@EntityReferenceImpl@xercesc_2_3@@UAEX_N0@Z 120e47e0 f   EntityReferenceImpl.obj
 0001:000e3860       ??0NamedNodeMapImpl@xercesc_2_3@@QAE@PAVNodeImpl@1@@Z 120e4860 f   NamedNodeMapImpl.obj
 0001:000e3890       ??_ENamedNodeMapImpl@xercesc_2_3@@UAEPAXI@Z 120e4890 f i NamedNodeMapImpl.obj
 0001:000e3910       ??1NamedNodeMapImpl@xercesc_2_3@@UAE@XZ 120e4910 f   NamedNodeMapImpl.obj
 0001:000e3950       ?addRef@NamedNodeMapImpl@xercesc_2_3@@SAXPAV12@@Z 120e4950 f   NamedNodeMapImpl.obj
 0001:000e3960       ?cloneMap@NamedNodeMapImpl@xercesc_2_3@@UAEPAV12@PAVNodeImpl@2@@Z 120e4960 f   NamedNodeMapImpl.obj
 0001:000e3ac0       ?removeAll@NamedNodeMapImpl@xercesc_2_3@@UAEXXZ 120e4ac0 f   NamedNodeMapImpl.obj
 0001:000e3b30       ?findNamePoint@NamedNodeMapImpl@xercesc_2_3@@UAEHABVDOMString@2@@Z 120e4b30 f   NamedNodeMapImpl.obj
 0001:000e3bf0       ?getLength@DOMNamedNodeMapImpl@xercesc_2_3@@UBEKXZ 120e4bf0 f   NamedNodeMapImpl.obj
 0001:000e3bf0       ?getLength@NamedNodeMapImpl@xercesc_2_3@@UAEIXZ 120e4bf0 f   NamedNodeMapImpl.obj
 0001:000e3c00       ?getNamedItem@NamedNodeMapImpl@xercesc_2_3@@UAEPAVNodeImpl@2@ABVDOMString@2@@Z 120e4c00 f   NamedNodeMapImpl.obj
 0001:000e3c30       ?item@DOMNamedNodeMapImpl@xercesc_2_3@@UBEPAVDOMNode@2@K@Z 120e4c30 f   NamedNodeMapImpl.obj
 0001:000e3c30       ?item@NamedNodeMapImpl@xercesc_2_3@@UAEPAVNodeImpl@2@I@Z 120e4c30 f   NamedNodeMapImpl.obj
 0001:000e3c60       ?removeNamedItem@NamedNodeMapImpl@xercesc_2_3@@UAEPAVNodeImpl@2@ABVDOMString@2@@Z 120e4c60 f   NamedNodeMapImpl.obj
 0001:000e3d40       ?removeRef@NamedNodeMapImpl@xercesc_2_3@@SAXPAV12@@Z 120e4d40 f   NamedNodeMapImpl.obj
 0001:000e3d60       ?setNamedItem@NamedNodeMapImpl@xercesc_2_3@@UAEPAVNodeImpl@2@PAV32@@Z 120e4d60 f   NamedNodeMapImpl.obj
 0001:000e3f50       ?setReadOnly@NamedNodeMapImpl@xercesc_2_3@@UAEX_N0@Z 120e4f50 f   NamedNodeMapImpl.obj
 0001:000e3fa0       ?findNamePoint@NamedNodeMapImpl@xercesc_2_3@@UAEHABVDOMString@2@0@Z 120e4fa0 f   NamedNodeMapImpl.obj
 0001:000e4160       ?getNamedItemNS@NamedNodeMapImpl@xercesc_2_3@@UAEPAVNodeImpl@2@ABVDOMString@2@0@Z 120e5160 f   NamedNodeMapImpl.obj
 0001:000e4190       ?setNamedItemNS@NamedNodeMapImpl@xercesc_2_3@@UAEPAVNodeImpl@2@PAV32@@Z 120e5190 f   NamedNodeMapImpl.obj
 0001:000e43d0       ?removeNamedItemNS@NamedNodeMapImpl@xercesc_2_3@@UAEPAVNodeImpl@2@ABVDOMString@2@0@Z 120e53d0 f   NamedNodeMapImpl.obj
 0001:000e44c0       ?setOwnerDocument@NamedNodeMapImpl@xercesc_2_3@@UAEXPAVDocumentImpl@2@@Z 120e54c0 f   NamedNodeMapImpl.obj
 0001:000e4510       ?cloneContent@NamedNodeMapImpl@xercesc_2_3@@MAEXPAV12@@Z 120e5510 f   NamedNodeMapImpl.obj
 0001:000e4640       ??0NodeIDMap@xercesc_2_3@@QAE@HQAVMemoryManager@1@@Z 120e5640 f   NodeIDMap.obj
 0001:000e4730       ??_ENodeIDMap@xercesc_2_3@@UAEPAXI@Z 120e5730 f i NodeIDMap.obj
 0001:000e4730       ??_GNodeIDMap@xercesc_2_3@@UAEPAXI@Z 120e5730 f i NodeIDMap.obj
 0001:000e4760       ?add@NodeIDMap@xercesc_2_3@@QAEXPAVAttrImpl@2@@Z 120e5760 f   NodeIDMap.obj
 0001:000e4820       ?remove@NodeIDMap@xercesc_2_3@@QAEXPAVAttrImpl@2@@Z 120e5820 f   NodeIDMap.obj
 0001:000e48d0       ?find@NodeIDMap@xercesc_2_3@@QAEPAVAttrImpl@2@ABVDOMString@2@@Z 120e58d0 f   NodeIDMap.obj
 0001:000e49a0       ?growTable@NodeIDMap@xercesc_2_3@@AAEXXZ 120e59a0 f   NodeIDMap.obj
 0001:000e4aa0       ??0NodeImpl@xercesc_2_3@@QAE@PAVDocumentImpl@1@@Z 120e5aa0 f   NodeImpl.obj
 0001:000e4ae0       ??_ENodeImpl@xercesc_2_3@@UAEPAXI@Z 120e5ae0 f i NodeImpl.obj
 0001:000e4b40       ??0NodeImpl@xercesc_2_3@@QAE@ABV01@@Z 120e5b40 f   NodeImpl.obj
 0001:000e4be0       ??1NodeImpl@xercesc_2_3@@UAE@XZ 120e5be0 f   NodeImpl.obj
 0001:000e4c70       ?changed@NodeImpl@xercesc_2_3@@UAEXXZ 120e5c70 f   NodeImpl.obj
 0001:000e4c80       ?changes@NodeImpl@xercesc_2_3@@UAEHXZ 120e5c80 f   NodeImpl.obj
 0001:000e4c90       ?appendChild@NodeImpl@xercesc_2_3@@UAEPAV12@PAV12@@Z 120e5c90 f   NodeImpl.obj
 0001:000e4ca0       ?deleteIf@NodeImpl@xercesc_2_3@@SAXPAV12@@Z 120e5ca0 f   NodeImpl.obj
 0001:000e4d40       ?getNamespaceURI@NodeImpl@xercesc_2_3@@UAE?AVDOMString@2@XZ 120e5d40 f   NodeImpl.obj
 0001:000e4d40       ?getPrefix@NodeImpl@xercesc_2_3@@UAE?AVDOMString@2@XZ 120e5d40 f   NodeImpl.obj
 0001:000e4d40       ?getNodeValue@NodeImpl@xercesc_2_3@@UAE?AVDOMString@2@XZ 120e5d40 f   NodeImpl.obj
 0001:000e4d40       ?getLocalName@NodeImpl@xercesc_2_3@@UAE?AVDOMString@2@XZ 120e5d40 f   NodeImpl.obj
 0001:000e4d60       ?getOwnerDocument@NodeImpl@xercesc_2_3@@UAEPAVDocumentImpl@2@XZ 120e5d60 f   NodeImpl.obj
 0001:000e4d60       ?getDocument@NodeImpl@xercesc_2_3@@UAEPAVDocumentImpl@2@XZ 120e5d60 f   NodeImpl.obj
 0001:000e4d80       ?setOwnerDocument@NodeImpl@xercesc_2_3@@UAEXPAVDocumentImpl@2@@Z 120e5d80 f   NodeImpl.obj
 0001:000e4da0       ?getUserData@NodeImpl@xercesc_2_3@@UAEPAXXZ 120e5da0 f   NodeImpl.obj
 0001:000e4dd0       ?insertBefore@NodeImpl@xercesc_2_3@@UAEPAV12@PAV12@0@Z 120e5dd0 f   NodeImpl.obj
 0001:000e4e20       ?item@NodeImpl@xercesc_2_3@@UAEPAV12@I@Z 120e5e20 f   NodeImpl.obj
 0001:000e4e30       ?removeChild@NodeImpl@xercesc_2_3@@UAEPAV12@PAV12@@Z 120e5e30 f   NodeImpl.obj
 0001:000e4e80       ?replaceChild@NodeImpl@xercesc_2_3@@UAEPAV12@PAV12@0@Z 120e5e80 f   NodeImpl.obj
 0001:000e4ed0       ?referenced@NodeImpl@xercesc_2_3@@UAEXXZ 120e5ed0 f   NodeImpl.obj
 0001:000e4ee0       ?unreferenced@NodeImpl@xercesc_2_3@@UAEXXZ 120e5ee0 f   NodeImpl.obj
 0001:000e4f00       ?setReadOnly@NodeImpl@xercesc_2_3@@UAEX_N0@Z 120e5f00 f   NodeImpl.obj
 0001:000e4f40       ?setUserData@NodeImpl@xercesc_2_3@@UAEXPAX@Z 120e5f40 f   NodeImpl.obj
 0001:000e4f80       ?toString@NodeImpl@xercesc_2_3@@UAE?AVDOMString@2@XZ 120e5f80 f   NodeImpl.obj
 0001:000e50e0       ?isSupported@NodeImpl@xercesc_2_3@@UAE_NABVDOMString@2@0@Z 120e60e0 f   NodeImpl.obj
 0001:000e5100       ?setPrefix@NodeImpl@xercesc_2_3@@UAEXABVDOMString@2@@Z 120e6100 f   NodeImpl.obj
 0001:000e5150       ?getXmlnsString@NodeImpl@xercesc_2_3@@KA?AVDOMString@2@XZ 120e6150 f   NodeImpl.obj
 0001:000e5190       ?getXmlnsURIString@NodeImpl@xercesc_2_3@@KA?AVDOMString@2@XZ 120e6190 f   NodeImpl.obj
 0001:000e51d0       ?getXmlString@NodeImpl@xercesc_2_3@@KA?AVDOMString@2@XZ 120e61d0 f   NodeImpl.obj
 0001:000e5210       ?getXmlURIString@NodeImpl@xercesc_2_3@@KA?AVDOMString@2@XZ 120e6210 f   NodeImpl.obj
 0001:000e5250       ?mapPrefix@NodeImpl@xercesc_2_3@@KAABVDOMString@2@ABV32@0F@Z 120e6250 f   NodeImpl.obj
 0001:000e54e0       ?reinitNodeImpl@NodeImpl@xercesc_2_3@@SAXXZ 120e64e0 f   NodeImpl.obj
 0001:000e5570       ??0NodeIteratorImpl@xercesc_2_3@@IAE@XZ 120e6570 f   NodeIteratorImpl.obj
 0001:000e55e0       ??_ENodeIteratorImpl@xercesc_2_3@@UAEPAXI@Z 120e65e0 f i NodeIteratorImpl.obj
 0001:000e5640       ??1NodeIteratorImpl@xercesc_2_3@@UAE@XZ 120e6640 f   NodeIteratorImpl.obj
 0001:000e56b0       ?detach@NodeIteratorImpl@xercesc_2_3@@QAEXXZ 120e66b0 f   NodeIteratorImpl.obj
 0001:000e56c0       ??0NodeIteratorImpl@xercesc_2_3@@QAE@VDOM_Node@1@KPAVDOM_NodeFilter@1@_N@Z 120e66c0 f   NodeIteratorImpl.obj
 0001:000e5760       ??0NodeIteratorImpl@xercesc_2_3@@QAE@ABV01@@Z 120e6760 f   NodeIteratorImpl.obj
 0001:000e57f0       ??4NodeIteratorImpl@xercesc_2_3@@QAEAAV01@ABV01@@Z 120e67f0 f   NodeIteratorImpl.obj
 0001:000e5840       ?getStartContainer@RangeImpl@xercesc_2_3@@QBE?AVDOM_Node@2@XZ 120e6840 f   NodeIteratorImpl.obj
 0001:000e5840       ?getRoot@NodeIteratorImpl@xercesc_2_3@@QAE?AVDOM_Node@2@XZ 120e6840 f   NodeIteratorImpl.obj
 0001:000e5860       ?nextNode@NodeIteratorImpl@xercesc_2_3@@QAE?AVDOM_Node@2@XZ 120e6860 f   NodeIteratorImpl.obj
 0001:000e59f0       ?previousNode@NodeIteratorImpl@xercesc_2_3@@QAE?AVDOM_Node@2@XZ 120e69f0 f   NodeIteratorImpl.obj
 0001:000e5b90       ?acceptNode@NodeIteratorImpl@xercesc_2_3@@QAE_NVDOM_Node@2@@Z 120e6b90 f   NodeIteratorImpl.obj
 0001:000e5c60       ?matchNodeOrParent@NodeIteratorImpl@xercesc_2_3@@QAE?AVDOM_Node@2@V32@@Z 120e6c60 f   NodeIteratorImpl.obj
 0001:000e5d90       ?nextNode@NodeIteratorImpl@xercesc_2_3@@QAE?AVDOM_Node@2@V32@_N@Z 120e6d90 f   NodeIteratorImpl.obj
 0001:000e6020       ?previousNode@NodeIteratorImpl@xercesc_2_3@@QAE?AVDOM_Node@2@V32@@Z 120e7020 f   NodeIteratorImpl.obj
 0001:000e61c0       ?removeNode@NodeIteratorImpl@xercesc_2_3@@QAEXVDOM_Node@2@@Z 120e71c0 f   NodeIteratorImpl.obj
 0001:000e6360       ?unreferenced@NodeIteratorImpl@xercesc_2_3@@UAEXXZ 120e7360 f   NodeIteratorImpl.obj
 0001:000e64e0       ??0NodeListImpl@xercesc_2_3@@IAE@XZ 120e74e0 f   NodeListImpl.obj
 0001:000e6500       ??_ENodeListImpl@xercesc_2_3@@UAEPAXI@Z 120e7500 f i NodeListImpl.obj
 0001:000e6560       ??1NodeListImpl@xercesc_2_3@@UAE@XZ 120e7560 f   NodeListImpl.obj
 0001:000e6570       ??0NodeVector@xercesc_2_3@@QAE@QAVMemoryManager@1@@Z 120e7570 f   NodeVector.obj
 0001:000e65a0       ??0NodeVector@xercesc_2_3@@QAE@IQAVMemoryManager@1@@Z 120e75a0 f   NodeVector.obj
 0001:000e65d0       ??1NodeVector@xercesc_2_3@@QAE@XZ 120e75d0 f   NodeVector.obj
 0001:000e65e0       ?addElement@NodeVector@xercesc_2_3@@QAEXPAVNodeImpl@2@@Z 120e75e0 f   NodeVector.obj
 0001:000e6600       ?checkSpace@NodeVector@xercesc_2_3@@AAEXXZ 120e7600 f   NodeVector.obj
 0001:000e6660       ?lastElement@NodeVector@xercesc_2_3@@QAEPAVNodeImpl@2@XZ 120e7660 f   NodeVector.obj
 0001:000e6670       ?insertElementAt@NodeVector@xercesc_2_3@@QAEXPAVNodeImpl@2@I@Z 120e7670 f   NodeVector.obj
 0001:000e66b0       ?removeElementAt@NodeVector@xercesc_2_3@@QAEXI@Z 120e76b0 f   NodeVector.obj
 0001:000e66b0       ?removeElementAt@DOMNodeVector@xercesc_2_3@@QAEXK@Z 120e76b0 f   NodeVector.obj
 0001:000e66e0       ??0NotationImpl@xercesc_2_3@@QAE@PAVDocumentImpl@1@ABVDOMString@1@@Z 120e76e0 f   NotationImpl.obj
 0001:000e6780       ??_ENotationImpl@xercesc_2_3@@UAEPAXI@Z 120e7780 f i NotationImpl.obj
 0001:000e67e0       ??0NotationImpl@xercesc_2_3@@QAE@ABV01@_N@Z 120e77e0 f   NotationImpl.obj
 0001:000e6880       ??1NotationImpl@xercesc_2_3@@UAE@XZ 120e7880 f   NotationImpl.obj
 0001:000e68f0       ?cloneNode@NotationImpl@xercesc_2_3@@UAEPAVNodeImpl@2@_N@Z 120e78f0 f   NotationImpl.obj
 0001:000e6960       ?getName@AttrImpl@xercesc_2_3@@UAE?AVDOMString@2@XZ 120e7960 f   NotationImpl.obj
 0001:000e6960       ?getNodeName@NotationImpl@xercesc_2_3@@UAE?AVDOMString@2@XZ 120e7960 f   NotationImpl.obj
 0001:000e6960       ?getNodeName@ElementDefinitionImpl@xercesc_2_3@@UAE?AVDOMString@2@XZ 120e7960 f   NotationImpl.obj
 0001:000e6960       ?getNodeName@AttrImpl@xercesc_2_3@@UAE?AVDOMString@2@XZ 120e7960 f   NotationImpl.obj
 0001:000e6980       ?getPublicId@NotationImpl@xercesc_2_3@@UAE?AVDOMString@2@XZ 120e7980 f   NotationImpl.obj
 0001:000e69a0       ?getSystemId@NotationImpl@xercesc_2_3@@UAE?AVDOMString@2@XZ 120e79a0 f   NotationImpl.obj
 0001:000e69a0       ?getTarget@ProcessingInstructionImpl@xercesc_2_3@@UAE?AVDOMString@2@XZ 120e79a0 f   NotationImpl.obj
 0001:000e69c0       ?setPublicId@NotationImpl@xercesc_2_3@@UAEXABVDOMString@2@@Z 120e79c0 f   NotationImpl.obj
 0001:000e6a60       ?setSystemId@NotationImpl@xercesc_2_3@@UAEXABVDOMString@2@@Z 120e7a60 f   NotationImpl.obj
 0001:000e6b00       ??0ParentNode@xercesc_2_3@@QAE@PAVDocumentImpl@1@@Z 120e7b00 f   ParentNode.obj
 0001:000e6b30       ??_EParentNode@xercesc_2_3@@UAEPAXI@Z 120e7b30 f i ParentNode.obj
 0001:000e6b90       ??0ParentNode@xercesc_2_3@@QAE@ABV01@@Z 120e7b90 f   ParentNode.obj
 0001:000e6bd0       ?cloneChildren@ParentNode@xercesc_2_3@@IAEXABVNodeImpl@2@@Z 120e7bd0 f   ParentNode.obj
 0001:000e6bd0       ?cloneChildren@AttrImpl@xercesc_2_3@@IAEXABVNodeImpl@2@@Z 120e7bd0 f   ParentNode.obj
 0001:000e6c10       ?setOwnerDocument@ParentNode@xercesc_2_3@@UAEXPAVDocumentImpl@2@@Z 120e7c10 f   ParentNode.obj
 0001:000e6c40       ?lastChild@ParentNode@xercesc_2_3@@IAEPAVChildNode@2@XZ 120e7c40 f   ParentNode.obj
 0001:000e6c40       ?getLastChild@ParentNode@xercesc_2_3@@UAEPAVNodeImpl@2@XZ 120e7c40 f   ParentNode.obj
 0001:000e6c50       ?lastChild@ParentNode@xercesc_2_3@@IAEXPAVChildNode@2@@Z 120e7c50 f   ParentNode.obj
 0001:000e6c70       ?getLength@ParentNode@xercesc_2_3@@UAEIXZ 120e7c70 f   ParentNode.obj
 0001:000e6cb0       ?hasChildNodes@ParentNode@xercesc_2_3@@UAE_NXZ 120e7cb0 f   ParentNode.obj
 0001:000e6cc0       ?insertBefore@ParentNode@xercesc_2_3@@UAEPAVNodeImpl@2@PAV32@0@Z 120e7cc0 f   ParentNode.obj
 0001:000e7050       ?item@ParentNode@xercesc_2_3@@UAEPAVNodeImpl@2@I@Z 120e8050 f   ParentNode.obj
 0001:000e70f0       ?removeChild@ParentNode@xercesc_2_3@@UAEPAVNodeImpl@2@PAV32@@Z 120e80f0 f   ParentNode.obj
 0001:000e7300       ?replaceChild@ParentNode@xercesc_2_3@@UAEPAVNodeImpl@2@PAV32@0@Z 120e8300 f   ParentNode.obj
 0001:000e7300       ?replaceChild@AttrImpl@xercesc_2_3@@UAEPAVNodeImpl@2@PAV32@0@Z 120e8300 f   ParentNode.obj
 0001:000e7330       ?setReadOnly@ParentNode@xercesc_2_3@@UAEX_N0@Z 120e8330 f   ParentNode.obj
 0001:000e7380       ?normalize@ParentNode@xercesc_2_3@@UAEXXZ 120e8380 f   ParentNode.obj
 0001:000e7420       ??0ProcessingInstructionImpl@xercesc_2_3@@QAE@PAVDocumentImpl@1@ABVDOMString@1@1@Z 120e8420 f   ProcessingInstructionImpl.obj
 0001:000e74e0       ??_EProcessingInstructionImpl@xercesc_2_3@@UAEPAXI@Z 120e84e0 f i ProcessingInstructionImpl.obj
 0001:000e7540       ??0ProcessingInstructionImpl@xercesc_2_3@@QAE@ABV01@_N@Z 120e8540 f   ProcessingInstructionImpl.obj
 0001:000e7600       ??1ProcessingInstructionImpl@xercesc_2_3@@UAE@XZ 120e8600 f   ProcessingInstructionImpl.obj
 0001:000e7660       ?cloneNode@ProcessingInstructionImpl@xercesc_2_3@@UAEPAVNodeImpl@2@_N@Z 120e8660 f   ProcessingInstructionImpl.obj
 0001:000e76d0       ?getData@ProcessingInstructionImpl@xercesc_2_3@@UAE?AVDOMString@2@XZ 120e86d0 f   ProcessingInstructionImpl.obj
 0001:000e76d0       ?getNodeValue@ProcessingInstructionImpl@xercesc_2_3@@UAE?AVDOMString@2@XZ 120e86d0 f   ProcessingInstructionImpl.obj
 0001:000e76f0       ?setNodeValue@ProcessingInstructionImpl@xercesc_2_3@@UAEXABVDOMString@2@@Z 120e86f0 f   ProcessingInstructionImpl.obj
 0001:000e7790       ?setData@ProcessingInstructionImpl@xercesc_2_3@@UAEXABVDOMString@2@@Z 120e8790 f   ProcessingInstructionImpl.obj
 0001:000e7830       ??0RangeImpl@xercesc_2_3@@QAE@VDOM_Document@1@@Z 120e8830 f   RangeImpl.obj
 0001:000e78e0       ??_ERangeImpl@xercesc_2_3@@UAEPAXI@Z 120e88e0 f i RangeImpl.obj
 0001:000e7940       ??0RangeImpl@xercesc_2_3@@QAE@ABV01@@Z 120e8940 f   RangeImpl.obj
 0001:000e7a10       ??1RangeImpl@xercesc_2_3@@UAE@XZ 120e8a10 f   RangeImpl.obj
 0001:000e7a90       ?unreferenced@RangeImpl@xercesc_2_3@@UAEXXZ 120e8a90 f   RangeImpl.obj
 0001:000e7b90       ?getCollapsed@RangeImpl@xercesc_2_3@@QBE_NXZ 120e8b90 f   RangeImpl.obj
 0001:000e7c30       ?setStartContainer@RangeImpl@xercesc_2_3@@AAEXABVDOM_Node@2@@Z 120e8c30 f   RangeImpl.obj
 0001:000e7ca0       ?setStartOffset@RangeImpl@xercesc_2_3@@AAEXI@Z 120e8ca0 f   RangeImpl.obj
 0001:000e7d10       ?setEndContainer@RangeImpl@xercesc_2_3@@AAEXABVDOM_Node@2@@Z 120e8d10 f   RangeImpl.obj
 0001:000e7d80       ?setEndOffset@RangeImpl@xercesc_2_3@@AAEXI@Z 120e8d80 f   RangeImpl.obj
 0001:000e7df0       ?setStart@RangeImpl@xercesc_2_3@@QAEXABVDOM_Node@2@I@Z 120e8df0 f   RangeImpl.obj
 0001:000e8090       ?setEnd@RangeImpl@xercesc_2_3@@QAEXABVDOM_Node@2@I@Z 120e9090 f   RangeImpl.obj
 0001:000e8330       ?setStartBefore@RangeImpl@xercesc_2_3@@QAEXABVDOM_Node@2@@Z 120e9330 f   RangeImpl.obj
 0001:000e8630       ?setStartAfter@RangeImpl@xercesc_2_3@@QAEXABVDOM_Node@2@@Z 120e9630 f   RangeImpl.obj
 0001:000e8920       ?setEndBefore@RangeImpl@xercesc_2_3@@QAEXABVDOM_Node@2@@Z 120e9920 f   RangeImpl.obj
 0001:000e8c20       ?setEndAfter@RangeImpl@xercesc_2_3@@QAEXABVDOM_Node@2@@Z 120e9c20 f   RangeImpl.obj
 0001:000e8f20       ?detach@RangeImpl@xercesc_2_3@@QAEXXZ 120e9f20 f   RangeImpl.obj
 0001:000e8fc0       ?collapse@RangeImpl@xercesc_2_3@@QAEX_N@Z 120e9fc0 f   RangeImpl.obj
 0001:000e9060       ?selectNode@RangeImpl@xercesc_2_3@@QAEXABVDOM_Node@2@@Z 120ea060 f   RangeImpl.obj
 0001:000e9320       ?selectNodeContents@RangeImpl@xercesc_2_3@@QAEXABVDOM_Node@2@@Z 120ea320 f   RangeImpl.obj
 0001:000e9550       ?surroundContents@RangeImpl@xercesc_2_3@@QAEXAAVDOM_Node@2@@Z 120ea550 f   RangeImpl.obj
 0001:000e9820       ?compareBoundaryPoints@RangeImpl@xercesc_2_3@@QBEFW4CompareHow@DOM_Range@2@PAV12@@Z 120ea820 f   RangeImpl.obj
 0001:000e9fd0       ?deleteContents@RangeImpl@xercesc_2_3@@QAEXXZ 120eafd0 f   RangeImpl.obj
 0001:000e9ff0       ?extractContents@RangeImpl@xercesc_2_3@@QAE?AVDOM_DocumentFragment@2@XZ 120eaff0 f   RangeImpl.obj
 0001:000ea030       ?cloneContents@RangeImpl@xercesc_2_3@@QBE?AVDOM_DocumentFragment@2@XZ 120eb030 f   RangeImpl.obj
 0001:000ea050       ?insertNode@RangeImpl@xercesc_2_3@@QAEXAAVDOM_Node@2@@Z 120eb050 f   RangeImpl.obj
 0001:000ea4b0       ?cloneRange@RangeImpl@xercesc_2_3@@QBEPAV12@XZ 120eb4b0 f   RangeImpl.obj
 0001:000ea550       ?toString@RangeImpl@xercesc_2_3@@QBE?AVDOMString@2@XZ 120eb550 f   RangeImpl.obj
 0001:000eaa30       ?getDocument@RangeImpl@xercesc_2_3@@QAE?AVDOM_Document@2@XZ 120eba30 f   RangeImpl.obj
 0001:000eaa50       ?getCommonAncestorContainer@RangeImpl@xercesc_2_3@@QBE?BVDOM_Node@2@XZ 120eba50 f   RangeImpl.obj
 0001:000eaa80       ?isValidAncestorType@RangeImpl@xercesc_2_3@@ABE_NABVDOM_Node@2@@Z 120eba80 f   RangeImpl.obj
 0001:000eab60       ?isAncestorOf@RangeImpl@xercesc_2_3@@CA_NABVDOM_Node@2@0@Z 120ebb60 f   RangeImpl.obj
 0001:000eac30       ?hasLegalRootContainer@RangeImpl@xercesc_2_3@@ABE_NABVDOM_Node@2@@Z 120ebc30 f   RangeImpl.obj
 0001:000ead80       ?isLegalContainedNode@RangeImpl@xercesc_2_3@@ABE_NABVDOM_Node@2@@Z 120ebd80 f   RangeImpl.obj
 0001:000eade0       ?indexOf@RangeImpl@xercesc_2_3@@ABEGABVDOM_Node@2@0@Z 120ebde0 f   RangeImpl.obj
 0001:000eaed0       ?validateNode@RangeImpl@xercesc_2_3@@ABEXABVDOM_Node@2@@Z 120ebed0 f   RangeImpl.obj
 0001:000eb000       ?commonAncestorOf@RangeImpl@xercesc_2_3@@ABE?BVDOM_Node@2@ABV32@0@Z 120ec000 f   RangeImpl.obj
 0001:000eb470       ?checkIndex@RangeImpl@xercesc_2_3@@ABEXABVDOM_Node@2@I@Z 120ec470 f   RangeImpl.obj
 0001:000eb5e0       ?nextNode@RangeImpl@xercesc_2_3@@ABE?AVDOM_Node@2@ABV32@_N@Z 120ec5e0 f   RangeImpl.obj
 0001:000eb820       ?traverseContents@RangeImpl@xercesc_2_3@@AAE?AVDOM_DocumentFragment@2@W4TraversalType@12@@Z 120ec820 f   RangeImpl.obj
 0001:000ebbc0       ?traverseSameContainer@RangeImpl@xercesc_2_3@@AAE?AVDOM_DocumentFragment@2@H@Z 120ecbc0 f   RangeImpl.obj
 0001:000ebec0       ?traverseCommonStartContainer@RangeImpl@xercesc_2_3@@AAE?AVDOM_DocumentFragment@2@VDOM_Node@2@H@Z 120ecec0 f   RangeImpl.obj
 0001:000ec240       ?traverseCommonEndContainer@RangeImpl@xercesc_2_3@@AAE?AVDOM_DocumentFragment@2@VDOM_Node@2@H@Z 120ed240 f   RangeImpl.obj
 0001:000ec530       ?traverseCommonAncestors@RangeImpl@xercesc_2_3@@AAE?AVDOM_DocumentFragment@2@VDOM_Node@2@0H@Z 120ed530 f   RangeImpl.obj
 0001:000ec970       ?traverseRightBoundary@RangeImpl@xercesc_2_3@@AAE?AVDOM_Node@2@V32@H@Z 120ed970 f   RangeImpl.obj
 0001:000ecc90       ?traverseLeftBoundary@RangeImpl@xercesc_2_3@@AAE?AVDOM_Node@2@V32@H@Z 120edc90 f   RangeImpl.obj
 0001:000ecfb0       ?traverseNode@RangeImpl@xercesc_2_3@@AAE?AVDOM_Node@2@V32@_N1H@Z 120edfb0 f   RangeImpl.obj
 0001:000ed090       ?traverseFullySelected@RangeImpl@xercesc_2_3@@AAE?AVDOM_Node@2@V32@H@Z 120ee090 f   RangeImpl.obj
 0001:000ed1b0       ?traversePartiallySelected@RangeImpl@xercesc_2_3@@AAE?AVDOM_Node@2@V32@H@Z 120ee1b0 f   RangeImpl.obj
 0001:000ed240       ?traverseTextNode@RangeImpl@xercesc_2_3@@AAE?AVDOM_Node@2@V32@_NH@Z 120ee240 f   RangeImpl.obj
 0001:000ed480       ?getSelectedNode@RangeImpl@xercesc_2_3@@AAE?AVDOM_Node@2@V32@H@Z 120ee480 f   RangeImpl.obj
 0001:000ed5b0       ?checkReadOnly@RangeImpl@xercesc_2_3@@AAEXAAVDOM_Node@2@0II@Z 120ee5b0 f   RangeImpl.obj
 0001:000ed770       ?recurseTreeAndCheck@RangeImpl@xercesc_2_3@@AAEXAAVDOM_Node@2@0@Z 120ee770 f   RangeImpl.obj
 0001:000ed8c0       ?removeChild@RangeImpl@xercesc_2_3@@AAE?AVDOM_Node@2@AAV32@0@Z 120ee8c0 f   RangeImpl.obj
 0001:000ed950       ?receiveReplacedText@RangeImpl@xercesc_2_3@@QAEXPAVNodeImpl@2@@Z 120ee950 f   RangeImpl.obj
 0001:000eda00       ?updateRangeForDeletedText@RangeImpl@xercesc_2_3@@QAEXAAVDOM_Node@2@IH@Z 120eea00 f   RangeImpl.obj
 0001:000edaa0       ?updateRangeForDeletedNode@RangeImpl@xercesc_2_3@@QAEXPAVNodeImpl@2@@Z 120eeaa0 f   RangeImpl.obj
 0001:000ee010       ?updateRangeForInsertedNode@RangeImpl@xercesc_2_3@@QAEXPAVNodeImpl@2@@Z 120ef010 f   RangeImpl.obj
 0001:000ee230       ?updateSplitInfo@RangeImpl@xercesc_2_3@@QAEXPAVTextImpl@2@0I@Z 120ef230 f   RangeImpl.obj
 0001:000ee310       ??_E?$RefVectorOf@VNodeImpl@xercesc_2_3@@@xercesc_2_3@@UAEPAXI@Z 120ef310 f i RangeImpl.obj
 0001:000ee310       ??_G?$RefVectorOf@VNodeImpl@xercesc_2_3@@@xercesc_2_3@@UAEPAXI@Z 120ef310 f i RangeImpl.obj
 0001:000ee330       ??1?$RefVectorOf@VNodeImpl@xercesc_2_3@@@xercesc_2_3@@UAE@XZ 120ef330 f i RangeImpl.obj
 0001:000ee3b0       ??1?$BaseRefVectorOf@VNodeImpl@xercesc_2_3@@@xercesc_2_3@@UAE@XZ 120ef3b0 f i RangeImpl.obj
 0001:000ee3c0       ??0?$BaseRefVectorOf@VNodeImpl@xercesc_2_3@@@xercesc_2_3@@QAE@I_NQAVMemoryManager@1@@Z 120ef3c0 f i RangeImpl.obj
 0001:000ee420       ??0RefCountedImpl@xercesc_2_3@@QAE@XZ 120ef420 f   RefCountedImpl.obj
 0001:000ee430       ??_ERefCountedImpl@xercesc_2_3@@UAEPAXI@Z 120ef430 f i RefCountedImpl.obj
 0001:000ee490       ??1RefCountedImpl@xercesc_2_3@@UAE@XZ 120ef490 f   RefCountedImpl.obj
 0001:000ee4a0       ?addRef@RefCountedImpl@xercesc_2_3@@SAXPAV12@@Z 120ef4a0 f   RefCountedImpl.obj
 0001:000ee4c0       ?removeRef@RefCountedImpl@xercesc_2_3@@SAXPAV12@@Z 120ef4c0 f   RefCountedImpl.obj
 0001:000ee500       ??0TextImpl@xercesc_2_3@@QAE@PAVDocumentImpl@1@ABVDOMString@1@@Z 120ef500 f   TextImpl.obj
 0001:000ee520       ??_ETextImpl@xercesc_2_3@@UAEPAXI@Z 120ef520 f i TextImpl.obj
 0001:000ee580       ??0TextImpl@xercesc_2_3@@QAE@ABV01@_N@Z 120ef580 f   TextImpl.obj
 0001:000ee5a0       ??1TextImpl@xercesc_2_3@@UAE@XZ 120ef5a0 f   TextImpl.obj
 0001:000ee5b0       ?cloneNode@TextImpl@xercesc_2_3@@UAEPAVNodeImpl@2@_N@Z 120ef5b0 f   TextImpl.obj
 0001:000ee620       ?getNodeName@TextImpl@xercesc_2_3@@UAE?AVDOMString@2@XZ 120ef620 f   TextImpl.obj
 0001:000ee660       ?getNodeType@TextImpl@xercesc_2_3@@UAEFXZ 120ef660 f   TextImpl.obj
 0001:000ee660       ?getNodeType@DOMTextImpl@xercesc_2_3@@UBEFXZ 120ef660 f   TextImpl.obj
 0001:000ee670       ?splitText@TextImpl@xercesc_2_3@@UAEPAV12@I@Z 120ef670 f   TextImpl.obj
 0001:000ee870       ?isIgnorableWhitespace@TextImpl@xercesc_2_3@@UAE_NXZ 120ef870 f   TextImpl.obj
 0001:000ee890       ?setIgnorableWhitespace@TextImpl@xercesc_2_3@@MAEX_N@Z 120ef890 f   TextImpl.obj
 0001:000ee8d0       ?reinitTextImpl@TextImpl@xercesc_2_3@@SAXXZ 120ef8d0 f   TextImpl.obj
 0001:000ee900       ??0TreeWalkerImpl@xercesc_2_3@@QAE@VDOM_Node@1@KPAVDOM_NodeFilter@1@_N@Z 120ef900 f   TreeWalkerImpl.obj
 0001:000ee990       ??_ETreeWalkerImpl@xercesc_2_3@@UAEPAXI@Z 120ef990 f i TreeWalkerImpl.obj
 0001:000ee9f0       ??0TreeWalkerImpl@xercesc_2_3@@QAE@ABV01@@Z 120ef9f0 f   TreeWalkerImpl.obj
 0001:000eea70       ??4TreeWalkerImpl@xercesc_2_3@@QAEAAV01@ABV01@@Z 120efa70 f   TreeWalkerImpl.obj
 0001:000eeab0       ?unreferenced@TreeWalkerImpl@xercesc_2_3@@UAEXXZ 120efab0 f   TreeWalkerImpl.obj
 0001:000eec30       ?getRoot@TreeWalkerImpl@xercesc_2_3@@QAE?AVDOM_Node@2@XZ 120efc30 f   TreeWalkerImpl.obj
 0001:000eec50       ?getExpandEntityReferences@TreeWalkerImpl@xercesc_2_3@@QAE_NXZ 120efc50 f   TreeWalkerImpl.obj
 0001:000eec60       ?getEndContainer@RangeImpl@xercesc_2_3@@QBE?AVDOM_Node@2@XZ 120efc60 f   TreeWalkerImpl.obj
 0001:000eec60       ?getCurrentNode@TreeWalkerImpl@xercesc_2_3@@QAE?AVDOM_Node@2@XZ 120efc60 f   TreeWalkerImpl.obj
 0001:000eec80       ?setCurrentNode@TreeWalkerImpl@xercesc_2_3@@QAEXVDOM_Node@2@@Z 120efc80 f   TreeWalkerImpl.obj
 0001:000eecd0       ?parentNode@TreeWalkerImpl@xercesc_2_3@@QAE?AVDOM_Node@2@XZ 120efcd0 f   TreeWalkerImpl.obj
 0001:000eedb0       ?firstChild@TreeWalkerImpl@xercesc_2_3@@QAE?AVDOM_Node@2@XZ 120efdb0 f   TreeWalkerImpl.obj
 0001:000eee90       ?lastChild@TreeWalkerImpl@xercesc_2_3@@QAE?AVDOM_Node@2@XZ 120efe90 f   TreeWalkerImpl.obj
 0001:000eef70       ?previousSibling@TreeWalkerImpl@xercesc_2_3@@QAE?AVDOM_Node@2@XZ 120eff70 f   TreeWalkerImpl.obj
 0001:000ef050       ?nextSibling@TreeWalkerImpl@xercesc_2_3@@QAE?AVDOM_Node@2@XZ 120f0050 f   TreeWalkerImpl.obj
 0001:000ef130       ?previousNode@TreeWalkerImpl@xercesc_2_3@@QAE?AVDOM_Node@2@XZ 120f0130 f   TreeWalkerImpl.obj
 0001:000ef2f0       ?nextNode@TreeWalkerImpl@xercesc_2_3@@QAE?AVDOM_Node@2@XZ 120f02f0 f   TreeWalkerImpl.obj
 0001:000ef520       ?getParentNode@TreeWalkerImpl@xercesc_2_3@@IAE?AVDOM_Node@2@V32@@Z 120f0520 f   TreeWalkerImpl.obj
 0001:000ef6b0       ?getNextSibling@TreeWalkerImpl@xercesc_2_3@@IAE?AVDOM_Node@2@V32@@Z 120f06b0 f   TreeWalkerImpl.obj
 0001:000ef940       ?getPreviousSibling@TreeWalkerImpl@xercesc_2_3@@IAE?AVDOM_Node@2@V32@@Z 120f0940 f   TreeWalkerImpl.obj
 0001:000efbd0       ?getFirstChild@TreeWalkerImpl@xercesc_2_3@@IAE?AVDOM_Node@2@V32@@Z 120f0bd0 f   TreeWalkerImpl.obj
 0001:000efdb0       ?getLastChild@TreeWalkerImpl@xercesc_2_3@@IAE?AVDOM_Node@2@V32@@Z 120f0db0 f   TreeWalkerImpl.obj
 0001:000eff90       ?acceptNode@TreeWalkerImpl@xercesc_2_3@@IAEFVDOM_Node@2@@Z 120f0f90 f   TreeWalkerImpl.obj
 0001:000f00c0       ??0XMLDeclImpl@xercesc_2_3@@QAE@PAVDocumentImpl@1@@Z 120f10c0 f   XMLDeclImpl.obj
 0001:000f0140       ??_EXMLDeclImpl@xercesc_2_3@@UAEPAXI@Z 120f1140 f i XMLDeclImpl.obj
 0001:000f01a0       ??0XMLDeclImpl@xercesc_2_3@@QAE@PAVDocumentImpl@1@ABVDOMString@1@11@Z 120f11a0 f   XMLDeclImpl.obj
 0001:000f0220       ??0XMLDeclImpl@xercesc_2_3@@QAE@ABV01@_N@Z 120f1220 f   XMLDeclImpl.obj
 0001:000f0320       ??1XMLDeclImpl@xercesc_2_3@@UAE@XZ 120f1320 f   XMLDeclImpl.obj
 0001:000f0390       ?cloneNode@XMLDeclImpl@xercesc_2_3@@UAEPAVNodeImpl@2@_N@Z 120f1390 f   XMLDeclImpl.obj
 0001:000f0410       ?getNodeName@XMLDeclImpl@xercesc_2_3@@UAE?AVDOMString@2@XZ 120f1410 f   XMLDeclImpl.obj
 0001:000f0450       ?getNodeType@XMLDeclImpl@xercesc_2_3@@UAEFXZ 120f1450 f   XMLDeclImpl.obj
 0001:000f0460       ?getNodeValue@CharacterDataImpl@xercesc_2_3@@UAE?AVDOMString@2@XZ 120f1460 f   XMLDeclImpl.obj
 0001:000f0460       ?getVersion@XMLDeclImpl@xercesc_2_3@@UBE?AVDOMString@2@XZ 120f1460 f   XMLDeclImpl.obj
 0001:000f0460       ?getNamespaceURI@AttrNSImpl@xercesc_2_3@@UAE?AVDOMString@2@XZ 120f1460 f   XMLDeclImpl.obj
 0001:000f0460       ?getNodeName@ProcessingInstructionImpl@xercesc_2_3@@UAE?AVDOMString@2@XZ 120f1460 f   XMLDeclImpl.obj
 0001:000f0480       ?getLocalName@AttrNSImpl@xercesc_2_3@@UAE?AVDOMString@2@XZ 120f1480 f   XMLDeclImpl.obj
 0001:000f0480       ?getEncoding@XMLDeclImpl@xercesc_2_3@@UBE?AVDOMString@2@XZ 120f1480 f   XMLDeclImpl.obj
 0001:000f04a0       ?getStandalone@XMLDeclImpl@xercesc_2_3@@UBE?AVDOMString@2@XZ 120f14a0 f   XMLDeclImpl.obj
 0001:000f04c0       ?setVersion@XMLDeclImpl@xercesc_2_3@@UAEXABVDOMString@2@@Z 120f14c0 f   XMLDeclImpl.obj
 0001:000f0520       ?setEncoding@XMLDeclImpl@xercesc_2_3@@UAEXABVDOMString@2@@Z 120f1520 f   XMLDeclImpl.obj
 0001:000f0580       ?setStandalone@XMLDeclImpl@xercesc_2_3@@UAEXABVDOMString@2@@Z 120f1580 f   XMLDeclImpl.obj
 0001:000f05e0       ?reinitXMLDeclImpl@XMLDeclImpl@xercesc_2_3@@SAXXZ 120f15e0 f   XMLDeclImpl.obj
 0001:000f0610       ??0DOMException@xercesc_2_3@@QAE@XZ 120f1610 f   DOMException.obj
 0001:000f0630       ??_EDOMException@xercesc_2_3@@UAEPAXI@Z 120f1630 f i DOMException.obj
 0001:000f0690       ??0DOMException@xercesc_2_3@@QAE@FPBG@Z 120f1690 f   DOMException.obj
 0001:000f06b0       ??0DOMException@xercesc_2_3@@QAE@ABV01@@Z 120f16b0 f   DOMException.obj
 0001:000f06d0       ??1DOMException@xercesc_2_3@@UAE@XZ 120f16d0 f   DOMException.obj
 0001:000f06e0       ??0DOMRangeException@xercesc_2_3@@QAE@XZ 120f16e0 f   DOMRangeException.obj
 0001:000f0700       ??_EDOMRangeException@xercesc_2_3@@UAEPAXI@Z 120f1700 f i DOMRangeException.obj
 0001:000f0760       ??0DOMRangeException@xercesc_2_3@@QAE@W4RangeExceptionCode@01@PBG@Z 120f1760 f   DOMRangeException.obj
 0001:000f0790       ??0DOMRangeException@xercesc_2_3@@QAE@ABV01@@Z 120f1790 f   DOMRangeException.obj
 0001:000f07c0       ??1DOMRangeException@xercesc_2_3@@UAE@XZ 120f17c0 f   DOMRangeException.obj
 0001:000f07d0       __purecall                 120f17d0 f   MSVCRT:MSVCRT.dll
 0001:000f07d6       ??3@YAXPAX@Z               120f17d6 f   MSVCRT:MSVCRT.dll
 0001:000f07dc       ??_M@YGXPAXIHP6EX0@Z@Z     120f17dc f   MSVCRT:ehvecdtr.obj
 0001:000f085c       ?__ArrayUnwind@@YGXPAXIHP6EX0@Z@Z 120f185c f   MSVCRT:ehvecdtr.obj
 0001:000f08d0       ___CxxFrameHandler         120f18d0 f   MSVCRT:MSVCRT.dll
 0001:000f08e0       ??2@YAPAXI@Z               120f18e0 f   MSVCRT:MSVCRT.dll
 0001:000f08e6       ??_Gtype_info@@UAEPAXI@Z   120f18e6 f i MSVCRT:ti_inst.obj
 0001:000f08e6       ??_Etype_info@@UAEPAXI@Z   120f18e6 f i MSVCRT:ti_inst.obj
 0001:000f0902       __CxxThrowException@8      120f1902 f   MSVCRT:MSVCRT.dll
 0001:000f0908       __ftol                     120f1908 f   MSVCRT:MSVCRT.dll
 0001:000f090e       __onexit                   120f190e f   MSVCRT:atonexit.obj
 0001:000f093a       _atexit                    120f193a f   MSVCRT:atonexit.obj
 0001:000f0950       __alloca_probe             120f1950 f   MSVCRT:chkstk.obj
 0001:000f0950       __chkstk                   120f1950 f   MSVCRT:chkstk.obj
 0001:000f097f       __CRT_INIT@12              120f197f f   MSVCRT:crtdll.obj
 0001:000f0a2a       __DllMainCRTStartup@12     120f1a2a f   MSVCRT:crtdll.obj
 0001:000f0ac8       __except_handler3          120f1ac8 f   MSVCRT:MSVCRT.dll
 0001:000f0ace       ?terminate@@YAXXZ          120f1ace f   MSVCRT:MSVCRT.dll
 0001:000f0ad4       ??1type_info@@UAE@XZ       120f1ad4 f   MSVCRT:MSVCRT.dll
 0001:000f0ada       ___dllonexit               120f1ada f   MSVCRT:MSVCRT.dll
 0001:000f0ae0       __initterm                 120f1ae0 f   MSVCRT:MSVCRT.dll
 0002:00000000       __imp__RegOpenKeyExA@20    12103000     advapi32:ADVAPI32.dll
 0002:00000004       __imp__RegEnumKeyExA@32    12103004     advapi32:ADVAPI32.dll
 0002:00000008       __imp__RegCloseKey@4       12103008     advapi32:ADVAPI32.dll
 0002:0000000c       __imp__RegQueryValueExA@24 1210300c     advapi32:ADVAPI32.dll
 0002:00000010       \177ADVAPI32_NULL_THUNK_DATA 12103010     advapi32:ADVAPI32.dll
 0002:00000014       __imp__GetStdHandle@4      12103014     kernel32:KERNEL32.dll
 0002:00000018       __imp__GetLastError@0      12103018     kernel32:KERNEL32.dll
 0002:0000001c       __imp__ReadFile@20         1210301c     kernel32:KERNEL32.dll
 0002:00000020       __imp__WriteFile@20        12103020     kernel32:KERNEL32.dll
 0002:00000024       __imp__GetCurrentProcess@0 12103024     kernel32:KERNEL32.dll
 0002:00000028       __imp__DuplicateHandle@28  12103028     kernel32:KERNEL32.dll
 0002:0000002c       __imp__GetFullPathNameA@16 1210302c     kernel32:KERNEL32.dll
 0002:00000030       __imp__GetCurrentDirectoryA@8 12103030     kernel32:KERNEL32.dll
 0002:00000034       __imp__GetCurrentDirectoryW@8 12103034     kernel32:KERNEL32.dll
 0002:00000038       __imp__GetTickCount@0      12103038     kernel32:KERNEL32.dll
 0002:0000003c       __imp__DeleteCriticalSection@4 1210303c     kernel32:KERNEL32.dll
 0002:00000040       __imp__EnterCriticalSection@4 12103040     kernel32:KERNEL32.dll
 0002:00000044       __imp__InitializeCriticalSection@4 12103044     kernel32:KERNEL32.dll
 0002:00000048       __imp__GetFullPathNameW@16 12103048     kernel32:KERNEL32.dll
 0002:0000004c       __imp__CloseHandle@4       1210304c     kernel32:KERNEL32.dll
 0002:00000050       __imp__InterlockedDecrement@4 12103050     kernel32:KERNEL32.dll
 0002:00000054       __imp__GetVersionExA@4     12103054     kernel32:KERNEL32.dll
 0002:00000058       __imp__GetModuleHandleA@4  12103058     kernel32:KERNEL32.dll
 0002:0000005c       __imp__LockResource@4      1210305c     kernel32:KERNEL32.dll
 0002:00000060       __imp__LoadResource@8      12103060     kernel32:KERNEL32.dll
 0002:00000064       __imp__FindResourceExA@16  12103064     kernel32:KERNEL32.dll
 0002:00000068       __imp__IsValidCodePage@4   12103068     kernel32:KERNEL32.dll
 0002:0000006c       __imp__MultiByteToWideChar@24 1210306c     kernel32:KERNEL32.dll
 0002:00000070       __imp__IsDBCSLeadByteEx@8  12103070     kernel32:KERNEL32.dll
 0002:00000074       __imp__WideCharToMultiByte@32 12103074     kernel32:KERNEL32.dll
 0002:00000078       __imp__FreeLibrary@4       12103078     kernel32:KERNEL32.dll
 0002:0000007c       __imp__GetProcAddress@8    1210307c     kernel32:KERNEL32.dll
 0002:00000080       __imp__LoadLibraryA@4      12103080     kernel32:KERNEL32.dll
 0002:00000084       __imp__CreateFileW@28      12103084     kernel32:KERNEL32.dll
 0002:00000088       __imp__CreateFileA@28      12103088     kernel32:KERNEL32.dll
 0002:0000008c       __imp__LeaveCriticalSection@4 1210308c     kernel32:KERNEL32.dll
 0002:00000090       __imp__SetFilePointer@16   12103090     kernel32:KERNEL32.dll
 0002:00000094       __imp__InterlockedIncrement@4 12103094     kernel32:KERNEL32.dll
 0002:00000098       \177KERNEL32_NULL_THUNK_DATA 12103098     kernel32:KERNEL32.dll
 0002:0000009c       __imp_?write@ostream@@QAEAAV1@PBDH@Z 1210309c     msvcirt:MSVCIRT.dll
 0002:000000a0       __imp_?cout@@3Vostream_withassign@@A 121030a0     msvcirt:MSVCIRT.dll
 0002:000000a4       __imp_?flush@ostream@@QAEAAV1@XZ 121030a4     msvcirt:MSVCIRT.dll
 0002:000000a8       \177MSVCIRT_NULL_THUNK_DATA 121030a8     msvcirt:MSVCIRT.dll
 0002:000000ac       __imp___purecall           121030ac     MSVCRT:MSVCRT.dll
 0002:000000b0       __imp____CxxFrameHandler   121030b0     MSVCRT:MSVCRT.dll
 0002:000000b4       __imp___wcsupr             121030b4     MSVCRT:MSVCRT.dll
 0002:000000b8       __imp__mbstowcs            121030b8     MSVCRT:MSVCRT.dll
 0002:000000bc       __imp__mblen               121030bc     MSVCRT:MSVCRT.dll
 0002:000000c0       __imp____mb_cur_max        121030c0     MSVCRT:MSVCRT.dll
 0002:000000c4       __imp__wcscmp              121030c4     MSVCRT:MSVCRT.dll
 0002:000000c8       __imp___wcsicmp            121030c8     MSVCRT:MSVCRT.dll
 0002:000000cc       __imp___wcsnicmp           121030cc     MSVCRT:MSVCRT.dll
 0002:000000d0       __imp__iswspace            121030d0     MSVCRT:MSVCRT.dll
 0002:000000d4       __imp___wcslwr             121030d4     MSVCRT:MSVCRT.dll
 0002:000000d8       __imp__wcstombs            121030d8     MSVCRT:MSVCRT.dll
 0002:000000dc       __imp__atoi                121030dc     MSVCRT:MSVCRT.dll
 0002:000000e0       __imp__strchr              121030e0     MSVCRT:MSVCRT.dll
 0002:000000e4       __imp__strstr              121030e4     MSVCRT:MSVCRT.dll
 0002:000000e8       __imp___itoa               121030e8     MSVCRT:MSVCRT.dll
 0002:000000ec       __imp___ftol               121030ec     MSVCRT:MSVCRT.dll
 0002:000000f0       __imp__exit                121030f0     MSVCRT:MSVCRT.dll
 0002:000000f4       __imp__fprintf             121030f4     MSVCRT:MSVCRT.dll
 0002:000000f8       __imp_??3@YAXPAX@Z         121030f8     MSVCRT:MSVCRT.dll
 0002:000000fc       __imp__div                 121030fc     MSVCRT:MSVCRT.dll
 0002:00000100       __imp__strtod              12103100     MSVCRT:MSVCRT.dll
 0002:00000104       __imp___errno              12103104     MSVCRT:MSVCRT.dll
 0002:00000108       __imp__strncmp             12103108     MSVCRT:MSVCRT.dll
 0002:0000010c       __imp__isspace             1210310c     MSVCRT:MSVCRT.dll
 0002:00000110       __imp__strtoul             12103110     MSVCRT:MSVCRT.dll
 0002:00000114       __imp__strtol              12103114     MSVCRT:MSVCRT.dll
 0002:00000118       __imp__printf              12103118     MSVCRT:MSVCRT.dll
 0002:0000011c       __imp__fputs               1210311c     MSVCRT:MSVCRT.dll
 0002:00000120       __imp__putchar             12103120     MSVCRT:MSVCRT.dll
 0002:00000124       __imp___except_handler3    12103124     MSVCRT:MSVCRT.dll
 0002:00000128       __imp_?terminate@@YAXXZ    12103128     MSVCRT:MSVCRT.dll
 0002:0000012c       __imp_??1type_info@@UAE@XZ 1210312c     MSVCRT:MSVCRT.dll
 0002:00000130       __imp____dllonexit         12103130     MSVCRT:MSVCRT.dll
 0002:00000134       __imp___onexit             12103134     MSVCRT:MSVCRT.dll
 0002:00000138       __imp__free                12103138     MSVCRT:MSVCRT.dll
 0002:0000013c       __imp___initterm           1210313c     MSVCRT:MSVCRT.dll
 0002:00000140       __imp__malloc              12103140     MSVCRT:MSVCRT.dll
 0002:00000144       __imp___adjust_fdiv        12103144     MSVCRT:MSVCRT.dll
 0002:00000148       __imp___iob                12103148     MSVCRT:MSVCRT.dll
 0002:0000014c       __imp_??2@YAPAXI@Z         1210314c     MSVCRT:MSVCRT.dll
 0002:00000150       __imp___CxxThrowException@8 12103150     MSVCRT:MSVCRT.dll
 0002:00000154       __imp__wcsncpy             12103154     MSVCRT:MSVCRT.dll
 0002:00000158       __imp__stricmp             12103158     MSVCRT:MSVCRT.dll
 0002:00000158       __imp___stricmp            12103158     MSVCRT:MSVCRT.dll
 0002:0000015c       __imp__strnicmp            1210315c     MSVCRT:MSVCRT.dll
 0002:0000015c       __imp___strnicmp           1210315c     MSVCRT:MSVCRT.dll
 0002:00000160       \177MSVCRT_NULL_THUNK_DATA 12103160     MSVCRT:MSVCRT.dll
 0002:00000168       ??_7MemoryManager@xercesc_2_3@@6B@ 12103168     Win32PlatformUtils.obj
 0002:00000174       ??_7DOMError@xercesc_2_3@@6B@ 12103174     Win32PlatformUtils.obj
 0002:000001a8       ??_7XMLErrorReporter@xercesc_2_3@@6B@ 121031a8     Win32PlatformUtils.obj
 0002:000001b4       ??_7PanicHandler@xercesc_2_3@@6B@ 121031b4     Win32PlatformUtils.obj
 0002:000001bc       ??_7XMLPlatformUtilsException@xercesc_2_3@@6B@ 121031bc     Win32PlatformUtils.obj
 0002:000001c8       ??_7XMLDeleter@xercesc_2_3@@6B@ 121031c8     Win32PlatformUtils.obj
 0002:000001cc       ??_7RuntimeException@xercesc_2_3@@6B@ 121031cc     Win32PlatformUtils.obj
 0002:000001d8       ??_7ArrayIndexOutOfBoundsException@xercesc_2_3@@6B@ 121031d8     Win32PlatformUtils.obj
 0002:000001e4       ??_7HashBase@xercesc_2_3@@6B@ 121031e4     Win32PlatformUtils.obj
 0002:000001ec       ??_7IllegalArgumentException@xercesc_2_3@@6B@ 121031ec     Win32PlatformUtils.obj
 0002:000001f8       ??_7NoSuchElementException@xercesc_2_3@@6B@ 121031f8     Win32PlatformUtils.obj
 0002:00000204       ??_7NullPointerException@xercesc_2_3@@6B@ 12103204     Win32PlatformUtils.obj
 0002:00000210       ??_7XMLMsgLoader@xercesc_2_3@@6B@ 12103210     Win32PlatformUtils.obj
 0002:00000224       ??_7MalformedURLException@xercesc_2_3@@6B@ 12103224     Win32PlatformUtils.obj
 0002:00000230       ??_7XMLNetAccessor@xercesc_2_3@@6B@ 12103230     Win32PlatformUtils.obj
 0002:0000023c       ??_7NetAccessorException@xercesc_2_3@@6B@ 1210323c     Win32PlatformUtils.obj
 0002:0000024c       ??_7Win32MsgLoader@xercesc_2_3@@6B@ 1210324c     Win32MsgLoader.obj
 0002:0000026c       ??_7TranscodingException@xercesc_2_3@@6B@ 1210326c     Win32TransService.obj
 0002:00000278       ??_7Win32TransService@xercesc_2_3@@6B@ 12103278     Win32TransService.obj
 0002:000002a0       ??_7Win32LCPTranscoder@xercesc_2_3@@6B@ 121032a0     Win32TransService.obj
 0002:000002c4       ??_7Win32Transcoder@xercesc_2_3@@6B@ 121032c4     Win32TransService.obj
 0002:000002d4       ??_7BinHTTPURLInputStream@xercesc_2_3@@6B@ 121032d4     BinHTTPURLInputStream.obj
 0002:000002e0       ?fgMyName@WinSockNetAccessor@xercesc_2_3@@0QBGB 121032e0     WinSockNetAccessor.obj
 0002:00000308       ??_7WinSockNetAccessor@xercesc_2_3@@6B@ 12103308     WinSockNetAccessor.obj
 0002:000003b0       ??_7ASCIIRangeFactory@xercesc_2_3@@6B@ 121033b0     ASCIIRangeFactory.obj
 0002:00004a7c       ??_7BlockRangeFactory@xercesc_2_3@@6B@ 12107a7c     BlockRangeFactory.obj
 0002:00004a88       ??_7CharToken@xercesc_2_3@@6B@ 12107a88     CharToken.obj
 0002:00004ad0       ??_7ClosureToken@xercesc_2_3@@6B@ 12107ad0     ClosureToken.obj
 0002:00004b18       ??_7ConcatToken@xercesc_2_3@@6B@ 12107b18     ConcatToken.obj
 0002:00004b60       ??_7ConditionToken@xercesc_2_3@@6B@ 12107b60     ConditionToken.obj
 0002:00004ba8       ??_7Match@xercesc_2_3@@6B@ 12107ba8     Match.obj
 0002:00004bac       ??_7ModifierToken@xercesc_2_3@@6B@ 12107bac     ModifierToken.obj
 0002:00004bf4       ??_7Op@xercesc_2_3@@6B@    12107bf4     Op.obj
 0002:00004c24       ??_7UnionOp@xercesc_2_3@@6B@ 12107c24     Op.obj
 0002:00004c54       ??_7StringOp@xercesc_2_3@@6B@ 12107c54     Op.obj
 0002:00004c84       ??_7CharOp@xercesc_2_3@@6B@ 12107c84     Op.obj
 0002:00004cb4       ??_7?$RefVectorOf@VOp@xercesc_2_3@@@xercesc_2_3@@6B@ 12107cb4     Op.obj
 0002:00004cb8       ??_7?$BaseRefVectorOf@VOp@xercesc_2_3@@@xercesc_2_3@@6B@ 12107cb8     Op.obj
 0002:00004cbc       ??_7ChildOp@xercesc_2_3@@6B@ 12107cbc     Op.obj
 0002:00004cec       ??_7ModifierOp@xercesc_2_3@@6B@ 12107cec     Op.obj
 0002:00004d1c       ??_7RangeOp@xercesc_2_3@@6B@ 12107d1c     Op.obj
 0002:00004d4c       ??_7ConditionOp@xercesc_2_3@@6B@ 12107d4c     Op.obj
 0002:00004d7c       ??_7ParenToken@xercesc_2_3@@6B@ 12107d7c     ParenToken.obj
 0002:00004e5c       ??_7ParseException@xercesc_2_3@@6B@ 12107e5c     ParserForXMLSchema.obj
 0002:00004e68       ??_7ParserForXMLSchema@xercesc_2_3@@6B@ 12107e68     ParserForXMLSchema.obj
 0002:00004ee8       ??_7RangeFactory@xercesc_2_3@@6B@ 12107ee8     RangeFactory.obj
 0002:00004ef4       ?MAPSIZE@RangeToken@xercesc_2_3@@2HB 12107ef4     RangeToken.obj
 0002:00004ef8       ?INITIALSIZE@RangeToken@xercesc_2_3@@2IB 12107ef8     RangeToken.obj
 0002:00004efc       ??_7RangeToken@xercesc_2_3@@6B@ 12107efc     RangeToken.obj
 0002:00004f48       __real@8@3fffa000000000000000 12107f48     RangeToken.obj
 0002:00004f64       ?MARK_PARENS@RegularExpression@xercesc_2_3@@2IB 12107f64     RegularExpression.obj
 0002:00004f68       ?IGNORE_CASE@RegularExpression@xercesc_2_3@@2IB 12107f68     RegularExpression.obj
 0002:00004f6c       ?SINGLE_LINE@RegularExpression@xercesc_2_3@@2IB 12107f6c     RegularExpression.obj
 0002:00004f70       ?MULTIPLE_LINE@RegularExpression@xercesc_2_3@@2IB 12107f70     RegularExpression.obj
 0002:00004f74       ?EXTENDED_COMMENT@RegularExpression@xercesc_2_3@@2IB 12107f74     RegularExpression.obj
 0002:00004f78       ?USE_UNICODE_CATEGORY@RegularExpression@xercesc_2_3@@2IB 12107f78     RegularExpression.obj
 0002:00004f7c       ?UNICODE_WORD_BOUNDARY@RegularExpression@xercesc_2_3@@2IB 12107f7c     RegularExpression.obj
 0002:00004f80       ?PROHIBIT_HEAD_CHARACTER_OPTIMIZATION@RegularExpression@xercesc_2_3@@2IB 12107f80     RegularExpression.obj
 0002:00004f84       ?PROHIBIT_FIXED_STRING_OPTIMIZATION@RegularExpression@xercesc_2_3@@2IB 12107f84     RegularExpression.obj
 0002:00004f88       ?XMLSCHEMA_MODE@RegularExpression@xercesc_2_3@@2IB 12107f88     RegularExpression.obj
 0002:00004f8c       ?SPECIAL_COMMA@RegularExpression@xercesc_2_3@@2IB 12107f8c     RegularExpression.obj
 0002:00004f90       ?WT_IGNORE@RegularExpression@xercesc_2_3@@2GB 12107f90     RegularExpression.obj
 0002:00004f92       ?WT_LETTER@RegularExpression@xercesc_2_3@@2GB 12107f92     RegularExpression.obj
 0002:00004f94       ?WT_OTHER@RegularExpression@xercesc_2_3@@2GB 12107f94     RegularExpression.obj
 0002:00004f98       ??_7?$RefArrayVectorOf@G@xercesc_2_3@@6B@ 12107f98     RegularExpression.obj
 0002:00004f9c       ??_7?$BaseRefVectorOf@G@xercesc_2_3@@6B@ 12107f9c     RegularExpression.obj
 0002:00004fa0       ??_7?$RefVectorOf@VMatch@xercesc_2_3@@@xercesc_2_3@@6B@ 12107fa0     RegularExpression.obj
 0002:00004fa4       ??_7?$BaseRefVectorOf@VMatch@xercesc_2_3@@@xercesc_2_3@@6B@ 12107fa4     RegularExpression.obj
 0002:00005022       ?S_NORMAL@RegxParser@xercesc_2_3@@2GB 12108022     RegxParser.obj
 0002:00005024       ?S_INBRACKETS@RegxParser@xercesc_2_3@@2GB 12108024     RegxParser.obj
 0002:00005026       ?S_INXBRACKETS@RegxParser@xercesc_2_3@@2GB 12108026     RegxParser.obj
 0002:00005028       ??_7RegxParser@xercesc_2_3@@6B@ 12108028     RegxParser.obj
 0002:000050a8       ??_7?$RefVectorOf@VReferencePosition@RegxParser@xercesc_2_3@@@xercesc_2_3@@6B@ 121080a8     RegxParser.obj
 0002:000050ac       ??_7?$BaseRefVectorOf@VReferencePosition@RegxParser@xercesc_2_3@@@xercesc_2_3@@6B@ 121080ac     RegxParser.obj
 0002:000050b0       ??_7StringToken@xercesc_2_3@@6B@ 121080b0     StringToken.obj
 0002:000050f8       ?UTF16_MAX@Token@xercesc_2_3@@2HB 121080f8     Token.obj
 0002:000050fc       ?FC_CONTINUE@Token@xercesc_2_3@@2GB 121080fc     Token.obj
 0002:000050fe       ?FC_TERMINAL@Token@xercesc_2_3@@2GB 121080fe     Token.obj
 0002:00005100       ?FC_ANY@Token@xercesc_2_3@@2GB 12108100     Token.obj
 0002:00005104       ??_7Token@xercesc_2_3@@6B@ 12108104     Token.obj
 0002:0000519c       ??_7?$RefVectorOf@VToken@xercesc_2_3@@@xercesc_2_3@@6B@ 1210819c     TokenFactory.obj
 0002:000051a0       ??_7?$BaseRefVectorOf@VToken@xercesc_2_3@@@xercesc_2_3@@6B@ 121081a0     TokenFactory.obj
 0002:00005cb4       ??_7UnicodeRangeFactory@xercesc_2_3@@6B@ 12108cb4     UnicodeRangeFactory.obj
 0002:00005cc0       ?INITIALSIZE@UnionToken@xercesc_2_3@@0GB 12108cc0     UnionToken.obj
 0002:00005cc4       ??_7UnionToken@xercesc_2_3@@6B@ 12108cc4     UnionToken.obj
 0002:00006230       ??_7XMLRangeFactory@xercesc_2_3@@6B@ 12109230     XMLRangeFactory.obj
 0002:0001623c       ?base64Alphabet@Base64@xercesc_2_3@@0QBEB 1211923c     Base64.obj
 0002:0001627d       ?base64Padding@Base64@xercesc_2_3@@0EB 1211927d     Base64.obj
 0002:00016280       ?quadsPerLine@Base64@xercesc_2_3@@0IB 12119280     Base64.obj
 0002:00016284       ??_7BinFileInputStream@xercesc_2_3@@6B@ 12119284     BinFileInputStream.obj
 0002:00016290       ??_7BinInputStream@xercesc_2_3@@6B@ 12119290     BinInputStream.obj
 0002:0001629c       ??_7BinMemInputStream@xercesc_2_3@@6B@ 1211929c     BinMemInputStream.obj
 0002:000162a8       ??_7DefaultPanicHandler@xercesc_2_3@@6B@ 121192a8     DefaultPanicHandler.obj
 0002:00027ef4       ??_7HashPtr@xercesc_2_3@@6B@ 1212aef4     HashPtr.obj
 0002:00027f00       ??_7HashXMLCh@xercesc_2_3@@6B@ 1212af00     HashXMLCh.obj
 0002:00027f0c       ??_7EmptyStackException@xercesc_2_3@@6B@ 1212af0c     HeaderDummy.obj
 0002:00027f18       ??_7InvalidCastException@xercesc_2_3@@6B@ 1212af18     HeaderDummy.obj
 0002:00027f24       ??_7IOException@xercesc_2_3@@6B@ 1212af24     HeaderDummy.obj
 0002:00027f30       ??_7UnexpectedEOFException@xercesc_2_3@@6B@ 1212af30     HeaderDummy.obj
 0002:00027f3c       ??_7UnsupportedEncodingException@xercesc_2_3@@6B@ 1212af3c     HeaderDummy.obj
 0002:00027f48       ??_7UTFDataFormatException@xercesc_2_3@@6B@ 1212af48     HeaderDummy.obj
 0002:00027f54       ??_7MemoryManagerImpl@xercesc_2_3@@6B@ 1212af54     PlatformUtils.obj
 0002:00027f60       __real@8@3fffc000000000000000 1212af60     StringPool.obj
 0002:00027f68       ??_7?$RefVectorOf@VENameMap@xercesc_2_3@@@xercesc_2_3@@6B@ 1212af68     TransService.obj
 0002:00027f6c       ??_7?$BaseRefVectorOf@VENameMap@xercesc_2_3@@@xercesc_2_3@@6B@ 1212af6c     TransService.obj
 0002:00027f70       ??_7XMLTransService@xercesc_2_3@@6B@ 1212af70     TransService.obj
 0002:00027f98       ??_7?$ENameMapFor@VXML88591Transcoder@xercesc_2_3@@@xercesc_2_3@@6B@ 1212af98     TransService.obj
 0002:00027fa0       ??_7?$ENameMapFor@VXMLUTF8Transcoder@xercesc_2_3@@@xercesc_2_3@@6B@ 1212afa0     TransService.obj
 0002:00027fa8       ??_7?$ENameMapFor@VXMLASCIITranscoder@xercesc_2_3@@@xercesc_2_3@@6B@ 1212afa8     TransService.obj
 0002:00027fb0       ??_7?$ENameMapFor@VXMLChTranscoder@xercesc_2_3@@@xercesc_2_3@@6B@ 1212afb0     TransService.obj
 0002:00027fb8       ??_7ENameMap@xercesc_2_3@@6B@ 1212afb8     TransService.obj
 0002:00027fc0       ??_7XMLTranscoder@xercesc_2_3@@6B@ 1212afc0     TransService.obj
 0002:00027fd0       ??_7XMLLCPTranscoder@xercesc_2_3@@6B@ 1212afd0     TransService.obj
 0002:00027ff4       ??_7?$EEndianNameMapFor@VXMLUTF16Transcoder@xercesc_2_3@@@xercesc_2_3@@6B@ 1212aff4     TransService.obj
 0002:00027ffc       ??_7?$EEndianNameMapFor@VXMLUCS4Transcoder@xercesc_2_3@@@xercesc_2_3@@6B@ 1212affc     TransService.obj
 0002:00028004       ??_7?$ENameMapFor@VXMLEBCDICTranscoder@xercesc_2_3@@@xercesc_2_3@@6B@ 1212b004     TransService.obj
 0002:0002800c       ??_7?$ENameMapFor@VXMLIBM1140Transcoder@xercesc_2_3@@@xercesc_2_3@@6B@ 1212b00c     TransService.obj
 0002:00028014       ??_7?$ENameMapFor@VXMLWin1252Transcoder@xercesc_2_3@@@xercesc_2_3@@6B@ 1212b014     TransService.obj
 0002:0002801c       ??_7XML256TableTranscoder@xercesc_2_3@@6B@ 1212b01c     XML256TableTranscoder.obj
 0002:0002802c       ??_7XML88591Transcoder@xercesc_2_3@@6B@ 1212b02c     XML88591Transcoder.obj
 0002:0002803c       ??_7NumberFormatException@xercesc_2_3@@6B@ 1212b03c     XMLAbstractDoubleFloat.obj
 0002:00028048       ??_7XMLAbstractDoubleFloat@xercesc_2_3@@6B@ 1212b048     XMLAbstractDoubleFloat.obj
 0002:00028060       ??_7XMLASCIITranscoder@xercesc_2_3@@6B@ 1212b060     XMLASCIITranscoder.obj
 0002:00028070       ??_7XMLBigDecimal@xercesc_2_3@@6B@ 1212b070     XMLBigDecimal.obj
 0002:000280a4       ??_7XMLChTranscoder@xercesc_2_3@@6B@ 1212b0a4     XMLChTranscoder.obj
 0002:0002813c       ??_7SchemaDateTimeException@xercesc_2_3@@6B@ 1212b13c     XMLDateTime.obj
 0002:00028148       ??_7XMLDateTime@xercesc_2_3@@6B@ 1212b148     XMLDateTime.obj
 0002:0002815c       ??_7XMLDouble@xercesc_2_3@@6B@ 1212b15c     XMLDouble.obj
 0002:00028178       __real@8@3c018000000000000000 1212b178     XMLDouble.obj
 0002:00028180       __real@8@bc018000000000000000 1212b180     XMLDouble.obj
 0002:00028188       __real@8@00000000000000000000 1212b188     XMLDouble.obj
 0002:00028910       ??_7XMLEBCDICTranscoder@xercesc_2_3@@6B@ 1212b910     XMLEBCDICTranscoder.obj
 0002:00028950       ??_7XMLException@xercesc_2_3@@6B@ 1212b950     XMLException.obj
 0002:00028958       ??_7XMLFloat@xercesc_2_3@@6B@ 1212b958     XMLFloat.obj
 0002:00028970       __real@8@407effffff0000000000 1212b970     XMLFloat.obj
 0002:00028978       __real@8@3f818000000000000000 1212b978     XMLFloat.obj
 0002:00028980       __real@8@bf818000000000000000 1212b980     XMLFloat.obj
 0002:00028988       __real@8@c07effffff0000000000 1212b988     XMLFloat.obj
 0002:0002910c       ??_7XMLIBM1140Transcoder@xercesc_2_3@@6B@ 1212c10c     XMLIBM1140Transcoder.obj
 0002:0002911c       ??_7XMLNumber@xercesc_2_3@@6B@ 1212c11c     XMLNumber.obj
 0002:0002916c       ??_7XMLUCS4Transcoder@xercesc_2_3@@6B@ 1212c16c     XMLUCSTranscoder.obj
 0002:0002917c       ?fgAnyString@XMLUni@xercesc_2_3@@2QBGB 1212c17c     XMLUni.obj
 0002:00029184       ?fgAttListString@XMLUni@xercesc_2_3@@2QBGB 1212c184     XMLUni.obj
 0002:00029194       ?fgCommentString@XMLUni@xercesc_2_3@@2QBGB 1212c194     XMLUni.obj
 0002:000291a0       ?fgCDATAString@XMLUni@xercesc_2_3@@2QBGB 1212c1a0     XMLUni.obj
 0002:000291ac       ?fgDefaultString@XMLUni@xercesc_2_3@@2QBGB 1212c1ac     XMLUni.obj
 0002:000291c0       ?fgDocTypeString@XMLUni@xercesc_2_3@@2QBGB 1212c1c0     XMLUni.obj
 0002:000291d4       ?fgEBCDICEncodingString@XMLUni@xercesc_2_3@@2QBGB 1212c1d4     XMLUni.obj
 0002:000291e4       ?fgElemString@XMLUni@xercesc_2_3@@2QBGB 1212c1e4     XMLUni.obj
 0002:000291f4       ?fgEmptyString@XMLUni@xercesc_2_3@@2QBGB 1212c1f4     XMLUni.obj
 0002:00029200       ?fgEncodingString@XMLUni@xercesc_2_3@@2QBGB 1212c200     XMLUni.obj
 0002:00029214       ?fgEntitString@XMLUni@xercesc_2_3@@2QBGB 1212c214     XMLUni.obj
 0002:00029220       ?fgEntityString@XMLUni@xercesc_2_3@@2QBGB 1212c220     XMLUni.obj
 0002:00029230       ?fgEntitiesString@XMLUni@xercesc_2_3@@2QBGB 1212c230     XMLUni.obj
 0002:00029244       ?fgEnumerationString@XMLUni@xercesc_2_3@@2QBGB 1212c244     XMLUni.obj
 0002:0002925c       ?fgExceptDomain@XMLUni@xercesc_2_3@@2QBGB 1212c25c     XMLUni.obj
 0002:000292b4       ?fgFixedString@XMLUni@xercesc_2_3@@2QBGB 1212c2b4     XMLUni.obj
 0002:000292c4       ?fgIBM037EncodingString@XMLUni@xercesc_2_3@@2QBGB 1212c2c4     XMLUni.obj
 0002:000292e0       ?fgIBM037EncodingString2@XMLUni@xercesc_2_3@@2QBGB 1212c2e0     XMLUni.obj
 0002:000292f0       ?fgIBM1140EncodingString@XMLUni@xercesc_2_3@@2QBGB 1212c2f0     XMLUni.obj
 0002:00029300       ?fgIBM1140EncodingString2@XMLUni@xercesc_2_3@@2QBGB 1212c300     XMLUni.obj
 0002:00029314       ?fgIBM1140EncodingString3@XMLUni@xercesc_2_3@@2QBGB 1212c314     XMLUni.obj
 0002:0002932c       ?fgIBM1140EncodingString4@XMLUni@xercesc_2_3@@2QBGB 1212c32c     XMLUni.obj
 0002:0002933c       ?fgIESString@XMLUni@xercesc_2_3@@2QBGB 1212c33c     XMLUni.obj
 0002:00029344       ?fgIDString@XMLUni@xercesc_2_3@@2QBGB 1212c344     XMLUni.obj
 0002:0002934c       ?fgIDRefString@XMLUni@xercesc_2_3@@2QBGB 1212c34c     XMLUni.obj
 0002:00029358       ?fgIDRefsString@XMLUni@xercesc_2_3@@2QBGB 1212c358     XMLUni.obj
 0002:00029368       ?fgImpliedString@XMLUni@xercesc_2_3@@2QBGB 1212c368     XMLUni.obj
 0002:0002937c       ?fgIgnoreString@XMLUni@xercesc_2_3@@2QBGB 1212c37c     XMLUni.obj
 0002:0002938c       ?fgIncludeString@XMLUni@xercesc_2_3@@2QBGB 1212c38c     XMLUni.obj
 0002:0002939c       ?fgISO88591EncodingString@XMLUni@xercesc_2_3@@2QBGB 1212c39c     XMLUni.obj
 0002:000293b0       ?fgISO88591EncodingString2@XMLUni@xercesc_2_3@@2QBGB 1212c3b0     XMLUni.obj
 0002:000293c8       ?fgISO88591EncodingString3@XMLUni@xercesc_2_3@@2QBGB 1212c3c8     XMLUni.obj
 0002:000293e0       ?fgISO88591EncodingString4@XMLUni@xercesc_2_3@@2QBGB 1212c3e0     XMLUni.obj
 0002:000293f0       ?fgISO88591EncodingString5@XMLUni@xercesc_2_3@@2QBGB 1212c3f0     XMLUni.obj
 0002:00029400       ?fgISO88591EncodingString6@XMLUni@xercesc_2_3@@2QBGB 1212c400     XMLUni.obj
 0002:00029410       ?fgISO88591EncodingString7@XMLUni@xercesc_2_3@@2QBGB 1212c410     XMLUni.obj
 0002:00029420       ?fgISO88591EncodingString8@XMLUni@xercesc_2_3@@2QBGB 1212c420     XMLUni.obj
 0002:00029430       ?fgISO88591EncodingString9@XMLUni@xercesc_2_3@@2QBGB 1212c430     XMLUni.obj
 0002:0002943c       ?fgISO88591EncodingString10@XMLUni@xercesc_2_3@@2QBGB 1212c43c     XMLUni.obj
 0002:00029454       ?fgISO88591EncodingString11@XMLUni@xercesc_2_3@@2QBGB 1212c454     XMLUni.obj
 0002:0002946c       ?fgISO88591EncodingString12@XMLUni@xercesc_2_3@@2QBGB 1212c46c     XMLUni.obj
 0002:00029474       ?fgLocalHostString@XMLUni@xercesc_2_3@@2QBGB 1212c474     XMLUni.obj
 0002:00029488       ?fgNoString@XMLUni@xercesc_2_3@@2QBGB 1212c488     XMLUni.obj
 0002:00029490       ?fgNotationString@XMLUni@xercesc_2_3@@2QBGB 1212c490     XMLUni.obj
 0002:000294a4       ?fgNDATAString@XMLUni@xercesc_2_3@@2QBGB 1212c4a4     XMLUni.obj
 0002:000294b0       ?fgNmTokenString@XMLUni@xercesc_2_3@@2QBGB 1212c4b0     XMLUni.obj
 0002:000294c0       ?fgNmTokensString@XMLUni@xercesc_2_3@@2QBGB 1212c4c0     XMLUni.obj
 0002:000294d4       ?fgPCDATAString@XMLUni@xercesc_2_3@@2QBGB 1212c4d4     XMLUni.obj
 0002:000294e4       ?fgPIString@XMLUni@xercesc_2_3@@2QBGB 1212c4e4     XMLUni.obj
 0002:000294ec       ?fgPubIDString@XMLUni@xercesc_2_3@@2QBGB 1212c4ec     XMLUni.obj
 0002:000294fc       ?fgRefString@XMLUni@xercesc_2_3@@2QBGB 1212c4fc     XMLUni.obj
 0002:00029504       ?fgRequiredString@XMLUni@xercesc_2_3@@2QBGB 1212c504     XMLUni.obj
 0002:00029518       ?fgStandaloneString@XMLUni@xercesc_2_3@@2QBGB 1212c518     XMLUni.obj
 0002:00029530       ?fgVersion1_0@XMLUni@xercesc_2_3@@2QBGB 1212c530     XMLUni.obj
 0002:00029538       ?fgVersion1_1@XMLUni@xercesc_2_3@@2QBGB 1212c538     XMLUni.obj
 0002:00029540       ?fgSysIDString@XMLUni@xercesc_2_3@@2QBGB 1212c540     XMLUni.obj
 0002:00029550       ?fgUnknownURIName@XMLUni@xercesc_2_3@@2QBGB 1212c550     XMLUni.obj
 0002:00029590       ?fgUCS4EncodingString@XMLUni@xercesc_2_3@@2QBGB 1212c590     XMLUni.obj
 0002:0002959c       ?fgUCS4EncodingString2@XMLUni@xercesc_2_3@@2QBGB 1212c59c     XMLUni.obj
 0002:000295a8       ?fgUCS4EncodingString3@XMLUni@xercesc_2_3@@2QBGB 1212c5a8     XMLUni.obj
 0002:000295b4       ?fgUCS4BEncodingString@XMLUni@xercesc_2_3@@2QBGB 1212c5b4     XMLUni.obj
 0002:000295cc       ?fgUCS4BEncodingString2@XMLUni@xercesc_2_3@@2QBGB 1212c5cc     XMLUni.obj
 0002:000295dc       ?fgUCS4LEncodingString@XMLUni@xercesc_2_3@@2QBGB 1212c5dc     XMLUni.obj
 0002:000295f4       ?fgUCS4LEncodingString2@XMLUni@xercesc_2_3@@2QBGB 1212c5f4     XMLUni.obj
 0002:00029604       ?fgUSASCIIEncodingString@XMLUni@xercesc_2_3@@2QBGB 1212c604     XMLUni.obj
 0002:00029618       ?fgUSASCIIEncodingString2@XMLUni@xercesc_2_3@@2QBGB 1212c618     XMLUni.obj
 0002:00029628       ?fgUSASCIIEncodingString3@XMLUni@xercesc_2_3@@2QBGB 1212c628     XMLUni.obj
 0002:00029634       ?fgUSASCIIEncodingString4@XMLUni@xercesc_2_3@@2QBGB 1212c634     XMLUni.obj
 0002:00029648       ?fgUTF8EncodingString@XMLUni@xercesc_2_3@@2QBGB 1212c648     XMLUni.obj
 0002:00029654       ?fgUTF8EncodingString2@XMLUni@xercesc_2_3@@2QBGB 1212c654     XMLUni.obj
 0002:00029660       ?fgUTF16EncodingString@XMLUni@xercesc_2_3@@2QBGB 1212c660     XMLUni.obj
 0002:00029670       ?fgUTF16EncodingString2@XMLUni@xercesc_2_3@@2QBGB 1212c670     XMLUni.obj
 0002:0002967c       ?fgUTF16EncodingString3@XMLUni@xercesc_2_3@@2QBGB 1212c67c     XMLUni.obj
 0002:0002968c       ?fgUTF16EncodingString4@XMLUni@xercesc_2_3@@2QBGB 1212c68c     XMLUni.obj
 0002:000296a0       ?fgUTF16EncodingString5@XMLUni@xercesc_2_3@@2QBGB 1212c6a0     XMLUni.obj
 0002:000296ac       ?fgUTF16BEncodingString@XMLUni@xercesc_2_3@@2QBGB 1212c6ac     XMLUni.obj
 0002:000296c4       ?fgUTF16BEncodingString2@XMLUni@xercesc_2_3@@2QBGB 1212c6c4     XMLUni.obj
 0002:000296d8       ?fgUTF16LEncodingString@XMLUni@xercesc_2_3@@2QBGB 1212c6d8     XMLUni.obj
 0002:000296f0       ?fgUTF16LEncodingString2@XMLUni@xercesc_2_3@@2QBGB 1212c6f0     XMLUni.obj
 0002:00029704       ?fgVersionString@XMLUni@xercesc_2_3@@2QBGB 1212c704     XMLUni.obj
 0002:00029714       ?fgValidityDomain@XMLUni@xercesc_2_3@@2QBGB 1212c714     XMLUni.obj
 0002:0002976c       ?fgWin1252EncodingString@XMLUni@xercesc_2_3@@2QBGB 1212c76c     XMLUni.obj
 0002:00029788       ?fgXMLChEncodingString@XMLUni@xercesc_2_3@@2QBGB 1212c788     XMLUni.obj
 0002:000297a4       ?fgXMLString@XMLUni@xercesc_2_3@@2QBGB 1212c7a4     XMLUni.obj
 0002:000297ac       ?fgXMLStringSpace@XMLUni@xercesc_2_3@@2QBGB 1212c7ac     XMLUni.obj
 0002:000297b8       ?fgXMLStringHTab@XMLUni@xercesc_2_3@@2QBGB 1212c7b8     XMLUni.obj
 0002:000297c4       ?fgXMLStringCR@XMLUni@xercesc_2_3@@2QBGB 1212c7c4     XMLUni.obj
 0002:000297d0       ?fgXMLStringLF@XMLUni@xercesc_2_3@@2QBGB 1212c7d0     XMLUni.obj
 0002:000297dc       ?fgXMLStringSpaceU@XMLUni@xercesc_2_3@@2QBGB 1212c7dc     XMLUni.obj
 0002:000297e8       ?fgXMLStringHTabU@XMLUni@xercesc_2_3@@2QBGB 1212c7e8     XMLUni.obj
 0002:000297f4       ?fgXMLStringCRU@XMLUni@xercesc_2_3@@2QBGB 1212c7f4     XMLUni.obj
 0002:00029800       ?fgXMLStringLFU@XMLUni@xercesc_2_3@@2QBGB 1212c800     XMLUni.obj
 0002:0002980c       ?fgXMLDeclString@XMLUni@xercesc_2_3@@2QBGB 1212c80c     XMLUni.obj
 0002:00029818       ?fgXMLDeclStringSpace@XMLUni@xercesc_2_3@@2QBGB 1212c818     XMLUni.obj
 0002:00029828       ?fgXMLDeclStringHTab@XMLUni@xercesc_2_3@@2QBGB 1212c828     XMLUni.obj
 0002:00029838       ?fgXMLDeclStringLF@XMLUni@xercesc_2_3@@2QBGB 1212c838     XMLUni.obj
 0002:00029848       ?fgXMLDeclStringCR@XMLUni@xercesc_2_3@@2QBGB 1212c848     XMLUni.obj
 0002:00029858       ?fgXMLDeclStringSpaceU@XMLUni@xercesc_2_3@@2QBGB 1212c858     XMLUni.obj
 0002:00029868       ?fgXMLDeclStringHTabU@XMLUni@xercesc_2_3@@2QBGB 1212c868     XMLUni.obj
 0002:00029878       ?fgXMLDeclStringLFU@XMLUni@xercesc_2_3@@2QBGB 1212c878     XMLUni.obj
 0002:00029888       ?fgXMLDeclStringCRU@XMLUni@xercesc_2_3@@2QBGB 1212c888     XMLUni.obj
 0002:00029898       ?fgXMLNSString@XMLUni@xercesc_2_3@@2QBGB 1212c898     XMLUni.obj
 0002:000298a4       ?fgXMLNSColonString@XMLUni@xercesc_2_3@@2QBGB 1212c8a4     XMLUni.obj
 0002:000298b4       ?fgXMLNSURIName@XMLUni@xercesc_2_3@@2QBGB 1212c8b4     XMLUni.obj
 0002:000298f0       ?fgXMLErrDomain@XMLUni@xercesc_2_3@@2QBGB 1212c8f0     XMLUni.obj
 0002:00029944       ?fgXMLURIName@XMLUni@xercesc_2_3@@2QBGB 1212c944     XMLUni.obj
 0002:00029990       ?fgYesString@XMLUni@xercesc_2_3@@2QBGB 1212c990     XMLUni.obj
 0002:00029998       ?fgZeroLenString@XMLUni@xercesc_2_3@@2QBGB 1212c998     XMLUni.obj
 0002:0002999c       ?fgDTDEntityString@XMLUni@xercesc_2_3@@2QBGB 1212c99c     XMLUni.obj
 0002:000299a8       ?fgAmp@XMLUni@xercesc_2_3@@2QBGB 1212c9a8     XMLUni.obj
 0002:000299b0       ?fgLT@XMLUni@xercesc_2_3@@2QBGB 1212c9b0     XMLUni.obj
 0002:000299b8       ?fgGT@XMLUni@xercesc_2_3@@2QBGB 1212c9b8     XMLUni.obj
 0002:000299c0       ?fgQuot@XMLUni@xercesc_2_3@@2QBGB 1212c9c0     XMLUni.obj
 0002:000299cc       ?fgApos@XMLUni@xercesc_2_3@@2QBGB 1212c9cc     XMLUni.obj
 0002:000299d8       ?fgWFXMLScanner@XMLUni@xercesc_2_3@@2QBGB 1212c9d8     XMLUni.obj
 0002:000299f4       ?fgIGXMLScanner@XMLUni@xercesc_2_3@@2QBGB 1212c9f4     XMLUni.obj
 0002:00029a10       ?fgSGXMLScanner@XMLUni@xercesc_2_3@@2QBGB 1212ca10     XMLUni.obj
 0002:00029a2c       ?fgDGXMLScanner@XMLUni@xercesc_2_3@@2QBGB 1212ca2c     XMLUni.obj
 0002:00029a48       ?fgArrayIndexOutOfBoundsException_Name@XMLUni@xercesc_2_3@@2QBGB 1212ca48     XMLUni.obj
 0002:00029a88       ?fgEmptyStackException_Name@XMLUni@xercesc_2_3@@2QBGB 1212ca88     XMLUni.obj
 0002:00029ab0       ?fgIllegalArgumentException_Name@XMLUni@xercesc_2_3@@2QBGB 1212cab0     XMLUni.obj
 0002:00029ae4       ?fgInvalidCastException_Name@XMLUni@xercesc_2_3@@2QBGB 1212cae4     XMLUni.obj
 0002:00029b10       ?fgIOException_Name@XMLUni@xercesc_2_3@@2QBGB 1212cb10     XMLUni.obj
 0002:00029b28       ?fgNoSuchElementException_Name@XMLUni@xercesc_2_3@@2QBGB 1212cb28     XMLUni.obj
 0002:00029b58       ?fgNullPointerException_Name@XMLUni@xercesc_2_3@@2QBGB 1212cb58     XMLUni.obj
 0002:00029b84       ?fgXMLPlatformUtilsException_Name@XMLUni@xercesc_2_3@@2QBGB 1212cb84     XMLUni.obj
 0002:00029bb0       ?fgRuntimeException_Name@XMLUni@xercesc_2_3@@2QBGB 1212cbb0     XMLUni.obj
 0002:00029bd4       ?fgTranscodingException_Name@XMLUni@xercesc_2_3@@2QBGB 1212cbd4     XMLUni.obj
 0002:00029c00       ?fgUnexpectedEOFException_Name@XMLUni@xercesc_2_3@@2QBGB 1212cc00     XMLUni.obj
 0002:00029c30       ?fgUnsupportedEncodingException_Name@XMLUni@xercesc_2_3@@2QBGB 1212cc30     XMLUni.obj
 0002:00029c6c       ?fgUTFDataFormatException_Name@XMLUni@xercesc_2_3@@2QBGB 1212cc6c     XMLUni.obj
 0002:00029c9c       ?fgNetAccessorException_Name@XMLUni@xercesc_2_3@@2QBGB 1212cc9c     XMLUni.obj
 0002:00029cc8       ?fgMalformedURLException_Name@XMLUni@xercesc_2_3@@2QBGB 1212ccc8     XMLUni.obj
 0002:00029cf4       ?fgNumberFormatException_Name@XMLUni@xercesc_2_3@@2QBGB 1212ccf4     XMLUni.obj
 0002:00029d20       ?fgParseException_Name@XMLUni@xercesc_2_3@@2QBGB 1212cd20     XMLUni.obj
 0002:00029d40       ?fgInvalidDatatypeFacetException_Name@XMLUni@xercesc_2_3@@2QBGB 1212cd40     XMLUni.obj
 0002:00029d7c       ?fgInvalidDatatypeValueException_Name@XMLUni@xercesc_2_3@@2QBGB 1212cd7c     XMLUni.obj
 0002:00029db8       ?fgSchemaDateTimeException_Name@XMLUni@xercesc_2_3@@2QBGB 1212cdb8     XMLUni.obj
 0002:00029de8       ?fgXPathException_Name@XMLUni@xercesc_2_3@@2QBGB 1212cde8     XMLUni.obj
 0002:00029e08       ?fgNegINFString@XMLUni@xercesc_2_3@@2QBGB 1212ce08     XMLUni.obj
 0002:00029e14       ?fgNegZeroString@XMLUni@xercesc_2_3@@2QBGB 1212ce14     XMLUni.obj
 0002:00029e1c       ?fgPosZeroString@XMLUni@xercesc_2_3@@2QBGB 1212ce1c     XMLUni.obj
 0002:00029e20       ?fgPosINFString@XMLUni@xercesc_2_3@@2QBGB 1212ce20     XMLUni.obj
 0002:00029e28       ?fgNaNString@XMLUni@xercesc_2_3@@2QBGB 1212ce28     XMLUni.obj
 0002:00029e30       ?fgEString@XMLUni@xercesc_2_3@@2QBGB 1212ce30     XMLUni.obj
 0002:00029e34       ?fgZeroString@XMLUni@xercesc_2_3@@2QBGB 1212ce34     XMLUni.obj
 0002:00029e38       ?fgNullString@XMLUni@xercesc_2_3@@2QBGB 1212ce38     XMLUni.obj
 0002:00029e44       ?fgSAX2CoreValidation@XMLUni@xercesc_2_3@@2QBGB 1212ce44     XMLUni.obj
 0002:00029e94       ?fgSAX2CoreNameSpaces@XMLUni@xercesc_2_3@@2QBGB 1212ce94     XMLUni.obj
 0002:00029ee4       ?fgSAX2CoreNameSpacePrefixes@XMLUni@xercesc_2_3@@2QBGB 1212cee4     XMLUni.obj
 0002:00029f44       ?fgXercesDynamic@XMLUni@xercesc_2_3@@2QBGB 1212cf44     XMLUni.obj
 0002:00029fa8       ?fgXercesSchema@XMLUni@xercesc_2_3@@2QBGB 1212cfa8     XMLUni.obj
 0002:0002a00c       ?fgXercesSchemaFullChecking@XMLUni@xercesc_2_3@@2QBGB 1212d00c     XMLUni.obj
 0002:0002a08c       ?fgXercesLoadExternalDTD@XMLUni@xercesc_2_3@@2QBGB 1212d08c     XMLUni.obj
 0002:0002a10c       ?fgXercesContinueAfterFatalError@XMLUni@xercesc_2_3@@2QBGB 1212d10c     XMLUni.obj
 0002:0002a180       ?fgXercesValidationErrorAsFatal@XMLUni@xercesc_2_3@@2QBGB 1212d180     XMLUni.obj
 0002:0002a1f4       ?fgXercesCalculateSrcOfs@XMLUni@xercesc_2_3@@2QBGB 1212d1f4     XMLUni.obj
 0002:0002a258       ?fgXercesStandardUriConformant@XMLUni@xercesc_2_3@@2QBGB 1212d258     XMLUni.obj
 0002:0002a2c8       ?fgXercesSchemaExternalSchemaLocation@XMLUni@xercesc_2_3@@2QBGB 1212d2c8     XMLUni.obj
 0002:0002a348       ?fgXercesSecurityManager@XMLUni@xercesc_2_3@@2QBGB 1212d348     XMLUni.obj
 0002:0002a3ac       ?fgXercesSchemaExternalNoNameSpaceSchemaLocation@XMLUni@xercesc_2_3@@2QBGB 1212d3ac     XMLUni.obj
 0002:0002a444       ?fgXercesScannerName@XMLUni@xercesc_2_3@@2QBGB 1212d444     XMLUni.obj
 0002:0002a4a0       ?fgXercesUserAdoptsDOMDocument@XMLUni@xercesc_2_3@@2QBGB 1212d4a0     XMLUni.obj
 0002:0002a518       ?fgXercesCacheGrammarFromParse@XMLUni@xercesc_2_3@@2QBGB 1212d518     XMLUni.obj
 0002:0002a59c       ?fgXercesUseCachedGrammarInParse@XMLUni@xercesc_2_3@@2QBGB 1212d59c     XMLUni.obj
 0002:0002a620       ?fgDOMCanonicalForm@XMLUni@xercesc_2_3@@2QBGB 1212d620     XMLUni.obj
 0002:0002a640       ?fgDOMCDATASections@XMLUni@xercesc_2_3@@2QBGB 1212d640     XMLUni.obj
 0002:0002a660       ?fgDOMComments@XMLUni@xercesc_2_3@@2QBGB 1212d660     XMLUni.obj
 0002:0002a674       ?fgDOMCharsetOverridesXMLEncoding@XMLUni@xercesc_2_3@@2QBGB 1212d674     XMLUni.obj
 0002:0002a6b4       ?fgDOMDatatypeNormalization@XMLUni@xercesc_2_3@@2QBGB 1212d6b4     XMLUni.obj
 0002:0002a6e4       ?fgDOMEntities@XMLUni@xercesc_2_3@@2QBGB 1212d6e4     XMLUni.obj
 0002:0002a6f8       ?fgDOMInfoset@XMLUni@xercesc_2_3@@2QBGB 1212d6f8     XMLUni.obj
 0002:0002a708       ?fgDOMNamespaces@XMLUni@xercesc_2_3@@2QBGB 1212d708     XMLUni.obj
 0002:0002a720       ?fgDOMNamespaceDeclarations@XMLUni@xercesc_2_3@@2QBGB 1212d720     XMLUni.obj
 0002:0002a750       ?fgDOMSupportedMediatypesOnly@XMLUni@xercesc_2_3@@2QBGB 1212d750     XMLUni.obj
 0002:0002a784       ?fgDOMValidateIfSchema@XMLUni@xercesc_2_3@@2QBGB 1212d784     XMLUni.obj
 0002:0002a7ac       ?fgDOMValidation@XMLUni@xercesc_2_3@@2QBGB 1212d7ac     XMLUni.obj
 0002:0002a7c4       ?fgDOMWhitespaceInElementContent@XMLUni@xercesc_2_3@@2QBGB 1212d7c4     XMLUni.obj
 0002:0002a800       ?fgDOMWRTCanonicalForm@XMLUni@xercesc_2_3@@2QBGB 1212d800     XMLUni.obj
 0002:0002a820       ?fgDOMWRTDiscardDefaultContent@XMLUni@xercesc_2_3@@2QBGB 1212d820     XMLUni.obj
 0002:0002a854       ?fgDOMWRTEntities@XMLUni@xercesc_2_3@@2QBGB 1212d854     XMLUni.obj
 0002:0002a868       ?fgDOMWRTFormatPrettyPrint@XMLUni@xercesc_2_3@@2QBGB 1212d868     XMLUni.obj
 0002:0002a890       ?fgDOMWRTNormalizeCharacters@XMLUni@xercesc_2_3@@2QBGB 1212d890     XMLUni.obj
 0002:0002a8bc       ?fgDOMWRTSplitCdataSections@XMLUni@xercesc_2_3@@2QBGB 1212d8bc     XMLUni.obj
 0002:0002a8e8       ?fgDOMWRTValidation@XMLUni@xercesc_2_3@@2QBGB 1212d8e8     XMLUni.obj
 0002:0002a900       ?fgDOMWRTWhitespaceInElementContent@XMLUni@xercesc_2_3@@2QBGB 1212d900     XMLUni.obj
 0002:0002a93c       ?fgDOMWRTBOM@XMLUni@xercesc_2_3@@2QBGB 1212d93c     XMLUni.obj
 0002:0002a9a4       ?fgXercescDefaultLocale@XMLUni@xercesc_2_3@@2QBDB 1212d9a4     XMLUni.obj
 0002:0002a9ac       ?fgXMLDOMMsgDomain@XMLUni@xercesc_2_3@@2QBGB 1212d9ac     XMLUni.obj
 0002:0002aa00       ?RESERVED_CHARACTERS@XMLUri@xercesc_2_3@@0QBGB 1212da00     XMLUri.obj
 0002:0002aa18       ?MARK_CHARACTERS@XMLUri@xercesc_2_3@@0QBGB 1212da18     XMLUri.obj
 0002:0002aa2c       ?SCHEME_CHARACTERS@XMLUri@xercesc_2_3@@0QBGB 1212da2c     XMLUri.obj
 0002:0002aa34       ?USERINFO_CHARACTERS@XMLUri@xercesc_2_3@@0QBGB 1212da34     XMLUri.obj
 0002:0002ab00       ??_7XMLUri@xercesc_2_3@@6B@ 1212db00     XMLUri.obj
 0002:0002ab44       ??_7XMLURL@xercesc_2_3@@6B@ 1212db44     XMLURL.obj
 0002:0002ab48       ??_7XMLUTF16Transcoder@xercesc_2_3@@6B@ 1212db48     XMLUTF16Transcoder.obj
 0002:0002ac88       ??_7XMLUTF8Transcoder@xercesc_2_3@@6B@ 1212dc88     XMLUTF8Transcoder.obj
 0002:0002b410       ??_7XMLWin1252Transcoder@xercesc_2_3@@6B@ 1212e410     XMLWin1252Transcoder.obj
 0002:0002b420       ??_7XMLFormatTarget@xercesc_2_3@@6B@ 1212e420     LocalFileFormatTarget.obj
 0002:0002b42c       ??_7LocalFileFormatTarget@xercesc_2_3@@6B@ 1212e42c     LocalFileFormatTarget.obj
 0002:0002b438       ??_7LocalFileInputSource@xercesc_2_3@@6B@ 1212e438     LocalFileInputSource.obj
 0002:0002b460       ??_7MemBufFormatTarget@xercesc_2_3@@6B@ 1212e460     MemBufFormatTarget.obj
 0002:0002b46c       ??_7MemBufInputSource@xercesc_2_3@@6B@ 1212e46c     MemBufInputSource.obj
 0002:0002b494       ??_7StdInInputSource@xercesc_2_3@@6B@ 1212e494     StdInInputSource.obj
 0002:0002b4bc       ??_7StdOutFormatTarget@xercesc_2_3@@6B@ 1212e4bc     StdOutFormatTarget.obj
 0002:0002b4c8       ??_7URLInputSource@xercesc_2_3@@6B@ 1212e4c8     URLInputSource.obj
 0002:0002b4f0       ??_7DOMInputSource@xercesc_2_3@@6B@ 1212e4f0     Wrapper4DOMInputSource.obj
 0002:0002b524       ??_7Wrapper4DOMInputSource@xercesc_2_3@@6B@ 1212e524     Wrapper4DOMInputSource.obj
 0002:0002b54c       ??_7Wrapper4InputSource@xercesc_2_3@@6B@ 1212e54c     Wrapper4InputSource.obj
 0002:0002b5dc       ?fgInvalidAttrId@XMLAttDef@xercesc_2_3@@2IB 1212e5dc     XMLAttDef.obj
 0002:0002b5e0       ??_7XMLAttDef@xercesc_2_3@@6B@ 1212e5e0     XMLAttDef.obj
 0002:0002b5f4       ?gInvalidTrans@XMLContentModel@xercesc_2_3@@2IB 1212e5f4     XMLContentModel.obj
 0002:0002b5f8       ?gEOCFakeId@XMLContentModel@xercesc_2_3@@2IB 1212e5f8     XMLContentModel.obj
 0002:0002b5fc       ?gEpsilonFakeId@XMLContentModel@xercesc_2_3@@2IB 1212e5fc     XMLContentModel.obj
 0002:0002b600       ??_7XMLContentModel@xercesc_2_3@@6B@ 1212e600     XMLContentModel.obj
 0002:0002b618       ?fgInvalidElemId@XMLElementDecl@xercesc_2_3@@2IB 1212e618     XMLElementDecl.obj
 0002:0002b61c       ?fgPCDataElemId@XMLElementDecl@xercesc_2_3@@2IB 1212e61c     XMLElementDecl.obj
 0002:0002b620       ?fgPCDataElemName@XMLElementDecl@xercesc_2_3@@2QBGB 1212e620     XMLElementDecl.obj
 0002:0002b630       ??_7XMLAttDefList@xercesc_2_3@@6B@ 1212e630     XMLElementDecl.obj
 0002:0002b654       ??_7XMLElementDecl@xercesc_2_3@@6B@ 1212e654     XMLElementDecl.obj
 0002:0002b68c       ??_7XMLEntityDecl@xercesc_2_3@@6B@ 1212e68c     XMLEntityDecl.obj
 0002:0002b710       ?fgASCIIPre@XMLRecognizer@xercesc_2_3@@2QBDB 1212e710     XMLRecognizer.obj
 0002:0002b718       ?fgASCIIPreLen@XMLRecognizer@xercesc_2_3@@2IB 1212e718     XMLRecognizer.obj
 0002:0002b71c       ?fgEBCDICPre@XMLRecognizer@xercesc_2_3@@2QBEB 1212e71c     XMLRecognizer.obj
 0002:0002b724       ?fgEBCDICPreLen@XMLRecognizer@xercesc_2_3@@2IB 1212e724     XMLRecognizer.obj
 0002:0002b728       ?fgUTF16BPre@XMLRecognizer@xercesc_2_3@@2QBEB 1212e728     XMLRecognizer.obj
 0002:0002b734       ?fgUTF16LPre@XMLRecognizer@xercesc_2_3@@2QBEB 1212e734     XMLRecognizer.obj
 0002:0002b740       ?fgUTF16PreLen@XMLRecognizer@xercesc_2_3@@2IB 1212e740     XMLRecognizer.obj
 0002:0002b744       ?fgUCS4BPre@XMLRecognizer@xercesc_2_3@@2QBEB 1212e744     XMLRecognizer.obj
 0002:0002b75c       ?fgUCS4LPre@XMLRecognizer@xercesc_2_3@@2QBEB 1212e75c     XMLRecognizer.obj
 0002:0002b774       ?fgUCS4PreLen@XMLRecognizer@xercesc_2_3@@2IB 1212e774     XMLRecognizer.obj
 0002:0002b778       ?fgUTF8BOM@XMLRecognizer@xercesc_2_3@@2QBDB 1212e778     XMLRecognizer.obj
 0002:0002b77c       ?fgUTF8BOMLen@XMLRecognizer@xercesc_2_3@@2IB 1212e77c     XMLRecognizer.obj
 0002:0002b780       ??_7XMLValidator@xercesc_2_3@@6B@ 1212e780     XMLValidator.obj
 0002:0002b7b4       ??_7SecurityManager@xercesc_2_3@@6B@ 1212e7b4     XMLValidator.obj
 0002:0002b7c0       ??_7Locator@xercesc_2_3@@6B@ 1212e7c0     XMLValidator.obj
 0002:0002b7d4       ??_7DTDEntityDecl@xercesc_2_3@@6B@ 1212e7d4     XMLValidator.obj
 0002:0002b800       ??_7Grammar@xercesc_2_3@@6B@ 1212e800     DGXMLScanner.obj
 0002:0002b844       ??_7XMLDocumentHandler@xercesc_2_3@@6B@ 1212e844     DGXMLScanner.obj
 0002:0002b878       ??_7XMLEntityHandler@xercesc_2_3@@6B@ 1212e878     DGXMLScanner.obj
 0002:0002b890       ??_7DocTypeHandler@xercesc_2_3@@6B@ 1212e890     DGXMLScanner.obj
 0002:0002b8d4       ??_7?$NameIdPoolEnumerator@VDTDElementDecl@xercesc_2_3@@@xercesc_2_3@@6B@ 1212e8d4     DGXMLScanner.obj
 0002:0002b8e4       ??_7?$NameIdPoolEnumerator@VDTDEntityDecl@xercesc_2_3@@@xercesc_2_3@@6B@ 1212e8e4     DGXMLScanner.obj
 0002:0002b8f4       ??_7?$NameIdPoolEnumerator@VXMLNotationDecl@xercesc_2_3@@@xercesc_2_3@@6B@ 1212e8f4     DGXMLScanner.obj
 0002:0002b904       ??_7DGXMLScanner@xercesc_2_3@@6B@ 1212e904     DGXMLScanner.obj
 0002:0002b93c       ??_7?$XMLEnumerator@VDTDElementDecl@xercesc_2_3@@@xercesc_2_3@@6B@ 1212e93c     DGXMLScanner.obj
 0002:0002b94c       ??_7?$XMLEnumerator@VDTDEntityDecl@xercesc_2_3@@@xercesc_2_3@@6B@ 1212e94c     DGXMLScanner.obj
 0002:0002b95c       ??_7?$XMLEnumerator@VXMLNotationDecl@xercesc_2_3@@@xercesc_2_3@@6B@ 1212e95c     DGXMLScanner.obj
 0002:0002b994       ??_7?$RefVectorOf@VSchemaElementDecl@xercesc_2_3@@@xercesc_2_3@@6B@ 1212e994     IGXMLScanner.obj
 0002:0002b998       ??_7?$BaseRefVectorOf@VSchemaElementDecl@xercesc_2_3@@@xercesc_2_3@@6B@ 1212e998     IGXMLScanner.obj
 0002:0002b99c       ??_7?$RefHash2KeysTableOfEnumerator@VSchemaAttDef@xercesc_2_3@@@xercesc_2_3@@6B@ 1212e99c     IGXMLScanner.obj
 0002:0002b9ac       ??_7FieldMatcher@xercesc_2_3@@6B@ 1212e9ac     IGXMLScanner.obj
 0002:0002b9c4       ??_7?$RefVectorOf@VIC_Field@xercesc_2_3@@@xercesc_2_3@@6B@ 1212e9c4     IGXMLScanner.obj
 0002:0002b9c8       ??_7?$BaseRefVectorOf@VIC_Field@xercesc_2_3@@@xercesc_2_3@@6B@ 1212e9c8     IGXMLScanner.obj
 0002:0002b9cc       ??_7?$RefVectorOf@VIdentityConstraint@xercesc_2_3@@@xercesc_2_3@@6B@ 1212e9cc     IGXMLScanner.obj
 0002:0002b9d0       ??_7?$BaseRefVectorOf@VIdentityConstraint@xercesc_2_3@@@xercesc_2_3@@6B@ 1212e9d0     IGXMLScanner.obj
 0002:0002b9d4       ??_7?$RefHash3KeysIdPoolEnumerator@VSchemaElementDecl@xercesc_2_3@@@xercesc_2_3@@6B@ 1212e9d4     IGXMLScanner.obj
 0002:0002b9e4       ??_7XSDErrorReporter@xercesc_2_3@@6B@ 1212e9e4     IGXMLScanner.obj
 0002:0002b9e8       ??_7SelectorMatcher@xercesc_2_3@@6B@ 1212e9e8     IGXMLScanner.obj
 0002:0002ba00       ??_7IGXMLScanner@xercesc_2_3@@6B@ 1212ea00     IGXMLScanner.obj
 0002:0002ba38       ??_7?$RefVectorOf@VKVStringPair@xercesc_2_3@@@xercesc_2_3@@6B@ 1212ea38     IGXMLScanner.obj
 0002:0002ba3c       ??_7?$BaseRefVectorOf@VKVStringPair@xercesc_2_3@@@xercesc_2_3@@6B@ 1212ea3c     IGXMLScanner.obj
 0002:0002ba40       ??_7?$XMLEnumerator@VSchemaAttDef@xercesc_2_3@@@xercesc_2_3@@6B@ 1212ea40     IGXMLScanner.obj
 0002:0002ba50       ??_7?$XMLEnumerator@VSchemaElementDecl@xercesc_2_3@@@xercesc_2_3@@6B@ 1212ea50     IGXMLScanner.obj
 0002:0002ba68       ??_7DOMNode@xercesc_2_3@@6B@ 1212ea68     IGXMLScanner2.obj
 0002:0002bb04       ??_7DOMElement@xercesc_2_3@@6B@ 1212eb04     IGXMLScanner2.obj
 0002:0002bbf0       ??_7DOMAttr@xercesc_2_3@@6B@ 1212ebf0     IGXMLScanner2.obj
 0002:0002bca8       ??_7?$BaseRefVectorEnumerator@VSchemaInfo@xercesc_2_3@@@xercesc_2_3@@6B@ 1212eca8     IGXMLScanner2.obj
 0002:0002bcb8       ??_7?$BaseRefVectorOf@VSchemaInfo@xercesc_2_3@@@xercesc_2_3@@6B@ 1212ecb8     IGXMLScanner2.obj
 0002:0002bcbc       ??_7?$RefVectorOf@VSchemaInfo@xercesc_2_3@@@xercesc_2_3@@6B@ 1212ecbc     IGXMLScanner2.obj
 0002:0002bcc0       ??_7DOMDocumentRange@xercesc_2_3@@6B@ 1212ecc0     IGXMLScanner2.obj
 0002:0002bcc8       ??_7DOMDocumentTraversal@xercesc_2_3@@6B@ 1212ecc8     IGXMLScanner2.obj
 0002:0002bcd4       ??_7DOMDocument@xercesc_2_3@@6BDOMNode@1@@ 1212ecd4     IGXMLScanner2.obj
 0002:0002bd70       ??_7DOMDocument@xercesc_2_3@@6BDOMDocumentTraversal@1@@ 1212ed70     IGXMLScanner2.obj
 0002:0002bd7c       ??_7DOMDocument@xercesc_2_3@@6BDOMDocumentRange@1@@ 1212ed7c     IGXMLScanner2.obj
 0002:0002be18       ??_7DOMDocumentType@xercesc_2_3@@6B@ 1212ee18     IGXMLScanner2.obj
 0002:0002becc       ??_7?$XMLEnumerator@VSchemaInfo@xercesc_2_3@@@xercesc_2_3@@6B@ 1212eecc     IGXMLScanner2.obj
 0002:0002bedc       ??_7ReaderMgr@xercesc_2_3@@6B@ 1212eedc     ReaderMgr.obj
 0002:0002bef0       ??_7?$BaseRefVectorOf@VXMLEntityDecl@xercesc_2_3@@@xercesc_2_3@@6B@ 1212eef0     ReaderMgr.obj
 0002:0002bef4       ??_7?$RefVectorOf@VXMLEntityDecl@xercesc_2_3@@@xercesc_2_3@@6B@ 1212eef4     ReaderMgr.obj
 0002:0002bef8       ??_7?$BaseRefVectorOf@VXMLReader@xercesc_2_3@@@xercesc_2_3@@6B@ 1212eef8     ReaderMgr.obj
 0002:0002befc       ??_7?$RefVectorOf@VXMLReader@xercesc_2_3@@@xercesc_2_3@@6B@ 1212eefc     ReaderMgr.obj
 0002:0002bf30       ??_7SGXMLScanner@xercesc_2_3@@6B@ 1212ef30     SGXMLScanner.obj
 0002:0002bf68       ??_7Attributes@xercesc_2_3@@6B@ 1212ef68     VecAttributesImpl.obj
 0002:0002bf9c       ??_7VecAttributesImpl@xercesc_2_3@@6B@ 1212ef9c     VecAttributesImpl.obj
 0002:0002bfd0       ??_7AttributeList@xercesc_2_3@@6B@ 1212efd0     VecAttrListImpl.obj
 0002:0002bff0       ??_7VecAttrListImpl@xercesc_2_3@@6B@ 1212eff0     VecAttrListImpl.obj
 0002:0002c054       ??_7WFXMLScanner@xercesc_2_3@@6B@ 1212f054     WFXMLScanner.obj
 0002:0002c08c       ??_7?$RefVectorOf@VXMLElementDecl@xercesc_2_3@@@xercesc_2_3@@6B@ 1212f08c     WFXMLScanner.obj
 0002:0002c090       ??_7?$BaseRefVectorOf@VXMLElementDecl@xercesc_2_3@@@xercesc_2_3@@6B@ 1212f090     WFXMLScanner.obj
 0002:0002c0ac       ??_7XMLScanner@xercesc_2_3@@6B@ 1212f0ac     XMLScanner.obj
 0002:0002c0e4       ??_7?$RefVectorOf@VXMLAttr@xercesc_2_3@@@xercesc_2_3@@6B@ 1212f0e4     XMLScanner.obj
 0002:0002c0e8       ??_7?$BaseRefVectorOf@VXMLAttr@xercesc_2_3@@@xercesc_2_3@@6B@ 1212f0e8     XMLScanner.obj
 0002:0002c0ec       ??_7?$RefHashTableOfEnumerator@VXMLRefInfo@xercesc_2_3@@@xercesc_2_3@@6B@ 1212f0ec     XMLScanner.obj
 0002:0002c0fc       ??_7?$XMLEnumerator@VXMLRefInfo@xercesc_2_3@@@xercesc_2_3@@6B@ 1212f0fc     XMLScanner.obj
 0002:0002c10c       ??_7DocumentHandler@xercesc_2_3@@6B@ 1212f10c     Dummy.obj
 0002:0002c134       ??_7DTDHandler@xercesc_2_3@@6B@ 1212f134     Dummy.obj
 0002:0002c144       ??_7EntityResolver@xercesc_2_3@@6B@ 1212f144     Dummy.obj
 0002:0002c14c       ??_7ErrorHandler@xercesc_2_3@@6B@ 1212f14c     Dummy.obj
 0002:0002c160       ??_7SAXException@xercesc_2_3@@6B@ 1212f160     Dummy.obj
 0002:0002c168       ??_7SAXNotSupportedException@xercesc_2_3@@6B@ 1212f168     Dummy.obj
 0002:0002c170       ??_7SAXNotRecognizedException@xercesc_2_3@@6B@ 1212f170     Dummy.obj
 0002:0002c178       ??_7HandlerBase@xercesc_2_3@@6BErrorHandler@1@@ 1212f178     Dummy.obj
 0002:0002c18c       ??_7HandlerBase@xercesc_2_3@@6BDocumentHandler@1@@ 1212f18c     Dummy.obj
 0002:0002c1b4       ??_7HandlerBase@xercesc_2_3@@6BDTDHandler@1@@ 1212f1b4     Dummy.obj
 0002:0002c1c4       ??_7HandlerBase@xercesc_2_3@@6BEntityResolver@1@@ 1212f1c4     Dummy.obj
 0002:0002c1cc       ??_7Parser@xercesc_2_3@@6B@ 1212f1cc     Dummy.obj
 0002:0002c1ec       ??_7InputSource@xercesc_2_3@@6B@ 1212f1ec     InputSource.obj
 0002:0002c214       ??_7SAXParseException@xercesc_2_3@@6B@ 1212f214     SAXParseException.obj
 0002:0002c23c       ??_7DOMImplementationLS@xercesc_2_3@@6B@ 1212f23c     AbstractDOMParser.obj
 0002:0002c24c       ??_7DOMImplementation@xercesc_2_3@@6B@ 1212f24c     AbstractDOMParser.obj
 0002:0002c270       ??_7DOMNodeList@xercesc_2_3@@6B@ 1212f270     AbstractDOMParser.obj
 0002:0002c27c       ??_7DOMUserDataHandler@xercesc_2_3@@6B@ 1212f27c     AbstractDOMParser.obj
 0002:0002c284       ??_7DOMTypeInfo@xercesc_2_3@@6B@ 1212f284     AbstractDOMParser.obj
 0002:0002c290       ??_7DOMCharacterData@xercesc_2_3@@6B@ 1212f290     AbstractDOMParser.obj
 0002:0002c34c       ??_7DOMText@xercesc_2_3@@6B@ 1212f34c     AbstractDOMParser.obj
 0002:0002c41c       ??_7DOMCDATASection@xercesc_2_3@@6B@ 1212f41c     AbstractDOMParser.obj
 0002:0002c4ec       ??_7DOMComment@xercesc_2_3@@6B@ 1212f4ec     AbstractDOMParser.obj
 0002:0002c5a8       ??_7DOMNamedNodeMap@xercesc_2_3@@6B@ 1212f5a8     AbstractDOMParser.obj
 0002:0002c5cc       ??_7DOMEntity@xercesc_2_3@@6B@ 1212f5cc     AbstractDOMParser.obj
 0002:0002c68c       ??_7DOMEntityReference@xercesc_2_3@@6B@ 1212f68c     AbstractDOMParser.obj
 0002:0002c728       ??_7DOMNotation@xercesc_2_3@@6B@ 1212f728     AbstractDOMParser.obj
 0002:0002c7cc       ??_7DOMProcessingInstruction@xercesc_2_3@@6B@ 1212f7cc     AbstractDOMParser.obj
 0002:0002c874       ??_7AbstractDOMParser@xercesc_2_3@@6BDocTypeHandler@1@@ 1212f874     AbstractDOMParser.obj
 0002:0002c8b8       ??_7AbstractDOMParser@xercesc_2_3@@6BXMLEntityHandler@1@@ 1212f8b8     AbstractDOMParser.obj
 0002:0002c8d0       ??_7AbstractDOMParser@xercesc_2_3@@6BXMLErrorReporter@1@@ 1212f8d0     AbstractDOMParser.obj
 0002:0002c8dc       ??_7AbstractDOMParser@xercesc_2_3@@6BXMLDocumentHandler@1@@ 1212f8dc     AbstractDOMParser.obj
 0002:0002c914       ??_7?$RefVectorOf@VDOMDocumentImpl@xercesc_2_3@@@xercesc_2_3@@6B@ 1212f914     AbstractDOMParser.obj
 0002:0002c918       ??_7?$BaseRefVectorOf@VDOMDocumentImpl@xercesc_2_3@@@xercesc_2_3@@6B@ 1212f918     AbstractDOMParser.obj
 0002:0002c91c       ??_7DOMBuilder@xercesc_2_3@@6B@ 1212f91c     DOMBuilderImpl.obj
 0002:0002c990       ??_7DOMEntityResolver@xercesc_2_3@@6B@ 1212f990     DOMBuilderImpl.obj
 0002:0002c998       ??_7DOMErrorHandler@xercesc_2_3@@6B@ 1212f998     DOMBuilderImpl.obj
 0002:0002c9a0       ??_7DOMLocator@xercesc_2_3@@6B@ 1212f9a0     DOMBuilderImpl.obj
 0002:0002c9cc       ??_7DOMBuilderImpl@xercesc_2_3@@6B@ 1212f9cc     DOMBuilderImpl.obj
 0002:0002ca40       ??_7DOMBuilderImpl@xercesc_2_3@@6BDocTypeHandler@1@@ 1212fa40     DOMBuilderImpl.obj
 0002:0002ca84       ??_7DOMBuilderImpl@xercesc_2_3@@6BXMLEntityHandler@1@@ 1212fa84     DOMBuilderImpl.obj
 0002:0002ca9c       ??_7DOMBuilderImpl@xercesc_2_3@@6BXMLErrorReporter@1@@ 1212fa9c     DOMBuilderImpl.obj
 0002:0002caa8       ??_7DOMBuilderImpl@xercesc_2_3@@6BXMLDocumentHandler@1@@ 1212faa8     DOMBuilderImpl.obj
 0002:0002caec       ??_7ContentHandler@xercesc_2_3@@6B@ 1212faec     SAX2XMLReaderImpl.obj
 0002:0002cb1c       ??_7LexicalHandler@xercesc_2_3@@6B@ 1212fb1c     SAX2XMLReaderImpl.obj
 0002:0002cb3c       ??_7DeclHandler@xercesc_2_3@@6B@ 1212fb3c     SAX2XMLReaderImpl.obj
 0002:0002cb50       ??_7SAX2XMLReader@xercesc_2_3@@6B@ 1212fb50     SAX2XMLReaderImpl.obj
 0002:0002cbf8       ??_7SAX2XMLReaderImpl@xercesc_2_3@@6BDocTypeHandler@1@@ 1212fbf8     SAX2XMLReaderImpl.obj
 0002:0002cc3c       ??_7SAX2XMLReaderImpl@xercesc_2_3@@6BXMLEntityHandler@1@@ 1212fc3c     SAX2XMLReaderImpl.obj
 0002:0002cc54       ??_7SAX2XMLReaderImpl@xercesc_2_3@@6BXMLErrorReporter@1@@ 1212fc54     SAX2XMLReaderImpl.obj
 0002:0002cc60       ??_7SAX2XMLReaderImpl@xercesc_2_3@@6BXMLDocumentHandler@1@@ 1212fc60     SAX2XMLReaderImpl.obj
 0002:0002cc94       ??_7SAX2XMLReaderImpl@xercesc_2_3@@6BSAX2XMLReader@1@@ 1212fc94     SAX2XMLReaderImpl.obj
 0002:0002cd3c       ??_7?$RefVectorOf@VXMLBuffer@xercesc_2_3@@@xercesc_2_3@@6B@ 1212fd3c     SAX2XMLReaderImpl.obj
 0002:0002cd40       ??_7?$BaseRefVectorOf@VXMLBuffer@xercesc_2_3@@@xercesc_2_3@@6B@ 1212fd40     SAX2XMLReaderImpl.obj
 0002:0002cd44       ??_7SAXParser@xercesc_2_3@@6BDocTypeHandler@1@@ 1212fd44     SAXParser.obj
 0002:0002cd88       ??_7SAXParser@xercesc_2_3@@6BXMLEntityHandler@1@@ 1212fd88     SAXParser.obj
 0002:0002cda0       ??_7SAXParser@xercesc_2_3@@6BXMLErrorReporter@1@@ 1212fda0     SAXParser.obj
 0002:0002cdac       ??_7SAXParser@xercesc_2_3@@6BXMLDocumentHandler@1@@ 1212fdac     SAXParser.obj
 0002:0002cde0       ??_7SAXParser@xercesc_2_3@@6BParser@1@@ 1212fde0     SAXParser.obj
 0002:0002ce00       ??_7XercesDOMParser@xercesc_2_3@@6BDocTypeHandler@1@@ 1212fe00     XercesDOMParser.obj
 0002:0002ce44       ??_7XercesDOMParser@xercesc_2_3@@6BXMLEntityHandler@1@@ 1212fe44     XercesDOMParser.obj
 0002:0002ce5c       ??_7XercesDOMParser@xercesc_2_3@@6BXMLErrorReporter@1@@ 1212fe5c     XercesDOMParser.obj
 0002:0002ce68       ??_7XercesDOMParser@xercesc_2_3@@6BXMLDocumentHandler@1@@ 1212fe68     XercesDOMParser.obj
 0002:0002cea0       ??_7AllContentModel@xercesc_2_3@@6B@ 1212fea0     AllContentModel.obj
 0002:0002ceb8       ??_7CMAny@xercesc_2_3@@6B@ 1212feb8     CMAny.obj
 0002:0002cec8       ??_7CMNode@xercesc_2_3@@6B@ 1212fec8     CMAny.obj
 0002:0002ced8       ??_7CMBinaryOp@xercesc_2_3@@6B@ 1212fed8     CMBinaryOp.obj
 0002:0002cee8       ??_7CMUnaryOp@xercesc_2_3@@6B@ 1212fee8     CMUnaryOp.obj
 0002:0002cef8       ??_7HashCMStateSet@xercesc_2_3@@6B@ 1212fef8     DFAContentModel.obj
 0002:0002cf04       ??_7DFAContentModel@xercesc_2_3@@6B@ 1212ff04     DFAContentModel.obj
 0002:0002cf1c       ??_7CMLeaf@xercesc_2_3@@6B@ 1212ff1c     DFAContentModel.obj
 0002:0002cf2c       ??_7?$RefHashTableOfEnumerator@VGrammar@xercesc_2_3@@@xercesc_2_3@@6B@ 1212ff2c     GrammarResolver.obj
 0002:0002cf3c       ??_7?$XMLEnumerator@VGrammar@xercesc_2_3@@@xercesc_2_3@@6B@ 1212ff3c     GrammarResolver.obj
 0002:0002cf4c       ??_7MixedContentModel@xercesc_2_3@@6B@ 1212ff4c     MixedContentModel.obj
 0002:0002cf64       ?INDETERMINATE@AbstractNumericFacetValidator@xercesc_2_3@@1HB 1212ff64     AbstractNumericFacetValidator.obj
 0002:0002cf68       ??_7InvalidDatatypeFacetException@xercesc_2_3@@6B@ 1212ff68     AbstractNumericFacetValidator.obj
 0002:0002cf74       ??_7AbstractNumericFacetValidator@xercesc_2_3@@6B@ 1212ff74     AbstractNumericFacetValidator.obj
 0002:0002cfc0       ??_7?$RefHashTableOfEnumerator@VKVStringPair@xercesc_2_3@@@xercesc_2_3@@6B@ 1212ffc0     AbstractNumericFacetValidator.obj
 0002:0002cfd0       ??_7?$XMLEnumerator@VKVStringPair@xercesc_2_3@@@xercesc_2_3@@6B@ 1212ffd0     AbstractNumericFacetValidator.obj
 0002:0002cfe0       ??_7InvalidDatatypeValueException@xercesc_2_3@@6B@ 1212ffe0     AbstractNumericValidator.obj
 0002:0002cfec       ??_7AbstractNumericValidator@xercesc_2_3@@6B@ 1212ffec     AbstractNumericValidator.obj
 0002:0002d038       ??_7AbstractStringValidator@xercesc_2_3@@6B@ 12130038     AbstractStringValidator.obj
 0002:0002d084       ??_7AnySimpleTypeDatatypeValidator@xercesc_2_3@@6B@ 12130084     AnySimpleTypeDatatypeValidator.obj
 0002:0002d0d4       ??_7AnyURIDatatypeValidator@xercesc_2_3@@6B@ 121300d4     AnyURIDatatypeValidator.obj
 0002:0002d120       ??_7Base64BinaryDatatypeValidator@xercesc_2_3@@6B@ 12130120     Base64BinaryDatatypeValidator.obj
 0002:0002d26c       ??_7BooleanDatatypeValidator@xercesc_2_3@@6B@ 1213026c     BooleanDatatypeValidator.obj
 0002:0002d28c       ??_7DatatypeValidator@xercesc_2_3@@6B@ 1213028c     DatatypeValidator.obj
 0002:0002d434       ??_7DateDatatypeValidator@xercesc_2_3@@6B@ 12130434     DateDatatypeValidator.obj
 0002:0002d488       ??_7DateTimeDatatypeValidator@xercesc_2_3@@6B@ 12130488     DateTimeDatatypeValidator.obj
 0002:0002d4dc       ??_7DateTimeValidator@xercesc_2_3@@6B@ 121304dc     DateTimeValidator.obj
 0002:0002d530       ??_7?$RefVectorOf@VXMLNumber@xercesc_2_3@@@xercesc_2_3@@6B@ 12130530     DateTimeValidator.obj
 0002:0002d534       ??_7?$BaseRefVectorOf@VXMLNumber@xercesc_2_3@@@xercesc_2_3@@6B@ 12130534     DateTimeValidator.obj
 0002:0002d538       ??_7DayDatatypeValidator@xercesc_2_3@@6B@ 12130538     DayDatatypeValidator.obj
 0002:0002d58c       ??_7DecimalDatatypeValidator@xercesc_2_3@@6B@ 1213058c     DecimalDatatypeValidator.obj
 0002:0002d5d8       ??_7DoubleDatatypeValidator@xercesc_2_3@@6B@ 121305d8     DoubleDatatypeValidator.obj
 0002:0002d624       ??_7DurationDatatypeValidator@xercesc_2_3@@6B@ 12130624     DurationDatatypeValidator.obj
 0002:0002d678       ??_7ENTITYDatatypeValidator@xercesc_2_3@@6B@ 12130678     ENTITYDatatypeValidator.obj
 0002:0002d6c4       ??_7FloatDatatypeValidator@xercesc_2_3@@6B@ 121306c4     FloatDatatypeValidator.obj
 0002:0002d710       ??_7HexBinaryDatatypeValidator@xercesc_2_3@@6B@ 12130710     HexBinaryDatatypeValidator.obj
 0002:0002d75c       ??_7IDDatatypeValidator@xercesc_2_3@@6B@ 1213075c     IDDatatypeValidator.obj
 0002:0002d7a8       ??_7IDREFDatatypeValidator@xercesc_2_3@@6B@ 121307a8     IDREFDatatypeValidator.obj
 0002:0002d7f4       ??_7ListDatatypeValidator@xercesc_2_3@@6B@ 121307f4     ListDatatypeValidator.obj
 0002:0002d840       ??_7MonthDatatypeValidator@xercesc_2_3@@6B@ 12130840     MonthDatatypeValidator.obj
 0002:0002d894       ??_7MonthDayDatatypeValidator@xercesc_2_3@@6B@ 12130894     MonthDayDatatypeValidator.obj
 0002:0002d8e8       ??_7NameDatatypeValidator@xercesc_2_3@@6B@ 121308e8     NameDatatypeValidator.obj
 0002:0002d934       ??_7NCNameDatatypeValidator@xercesc_2_3@@6B@ 12130934     NCNameDatatypeValidator.obj
 0002:0002d980       ??_7NOTATIONDatatypeValidator@xercesc_2_3@@6B@ 12130980     NOTATIONDatatypeValidator.obj
 0002:0002d9cc       ??_7QNameDatatypeValidator@xercesc_2_3@@6B@ 121309cc     QNameDatatypeValidator.obj
 0002:0002da18       ??_7StringDatatypeValidator@xercesc_2_3@@6B@ 12130a18     StringDatatypeValidator.obj
 0002:0002da64       ??_7TimeDatatypeValidator@xercesc_2_3@@6B@ 12130a64     TimeDatatypeValidator.obj
 0002:0002dab8       ??_7UnionDatatypeValidator@xercesc_2_3@@6B@ 12130ab8     UnionDatatypeValidator.obj
 0002:0002dad8       ??_7YearDatatypeValidator@xercesc_2_3@@6B@ 12130ad8     YearDatatypeValidator.obj
 0002:0002db2c       ??_7YearMonthDatatypeValidator@xercesc_2_3@@6B@ 12130b2c     YearMonthDatatypeValidator.obj
 0002:0002db80       ??_7DTDAttDef@xercesc_2_3@@6B@ 12130b80     DTDAttDef.obj
 0002:0002db94       ??_7DTDAttDefList@xercesc_2_3@@6B@ 12130b94     DTDAttDefList.obj
 0002:0002dbb8       ??_7?$RefHashTableOfEnumerator@VDTDAttDef@xercesc_2_3@@@xercesc_2_3@@6B@ 12130bb8     DTDAttDefList.obj
 0002:0002dbc8       ??_7?$XMLEnumerator@VDTDAttDef@xercesc_2_3@@@xercesc_2_3@@6B@ 12130bc8     DTDAttDefList.obj
 0002:0002dbd8       ??_7DTDElementDecl@xercesc_2_3@@6B@ 12130bd8     DTDElementDecl.obj
 0002:0002dc10       ??_7SimpleContentModel@xercesc_2_3@@6B@ 12130c10     DTDElementDecl.obj
 0002:0002dc28       ??_7DTDGrammar@xercesc_2_3@@6B@ 12130c28     DTDGrammar.obj
 0002:0002dc7c       ??_7DTDScanner@xercesc_2_3@@6B@ 12130c7c     DTDScanner.obj
 0002:0002dc80       ??_7DTDValidator@xercesc_2_3@@6B@ 12130c80     DTDValidator.obj
 0002:0002dcb4       ??_7XPathScanner@xercesc_2_3@@6B@ 12130cb4     IC_Field.obj
 0002:0002dcbc       ??_7IC_Key@xercesc_2_3@@6B@ 12130cbc     IC_Key.obj
 0002:0002dcc4       ??_7IC_KeyRef@xercesc_2_3@@6B@ 12130cc4     IC_KeyRef.obj
 0002:0002dccc       ??_7IC_Unique@xercesc_2_3@@6B@ 12130ccc     IC_Unique.obj
 0002:0002dcd4       ??_7IdentityConstraint@xercesc_2_3@@6B@ 12130cd4     IdentityConstraint.obj
 0002:0002dcdc       ??_7?$RefVectorOf@VFieldValueMap@xercesc_2_3@@@xercesc_2_3@@6B@ 12130cdc     ValueStore.obj
 0002:0002dce0       ??_7?$BaseRefVectorOf@VFieldValueMap@xercesc_2_3@@@xercesc_2_3@@6B@ 12130ce0     ValueStore.obj
 0002:0002dce4       ??_7?$BaseRefVectorOf@V?$RefHashTableOf@VValueStore@xercesc_2_3@@@xercesc_2_3@@@xercesc_2_3@@6B@ 12130ce4     ValueStoreCache.obj
 0002:0002dce8       ??_7?$RefVectorOf@V?$RefHashTableOf@VValueStore@xercesc_2_3@@@xercesc_2_3@@@xercesc_2_3@@6B@ 12130ce8     ValueStoreCache.obj
 0002:0002dcec       ??_7?$RefHashTableOfEnumerator@VValueStore@xercesc_2_3@@@xercesc_2_3@@6B@ 12130cec     ValueStoreCache.obj
 0002:0002dcfc       ??_7?$RefVectorOf@VValueStore@xercesc_2_3@@@xercesc_2_3@@6B@ 12130cfc     ValueStoreCache.obj
 0002:0002dd00       ??_7?$BaseRefVectorOf@VValueStore@xercesc_2_3@@@xercesc_2_3@@6B@ 12130d00     ValueStoreCache.obj
 0002:0002dd04       ??_7?$XMLEnumerator@VValueStore@xercesc_2_3@@@xercesc_2_3@@6B@ 12130d04     ValueStoreCache.obj
 0002:0002dd14       ?fASCIICharMap@XPathScanner@xercesc_2_3@@0QBEB 12130d14     XercesXPath.obj
 0002:0002dd94       ??_7XPathException@xercesc_2_3@@6B@ 12130d94     XercesXPath.obj
 0002:0002dda0       ??_7?$RefVectorOf@VXercesLocationPath@xercesc_2_3@@@xercesc_2_3@@6B@ 12130da0     XercesXPath.obj
 0002:0002dda4       ??_7?$RefVectorOf@VXercesStep@xercesc_2_3@@@xercesc_2_3@@6B@ 12130da4     XercesXPath.obj
 0002:0002dda8       ??_7XPathScannerForSchema@xercesc_2_3@@6B@ 12130da8     XercesXPath.obj
 0002:0002ddb0       ??_7?$BaseRefVectorOf@VXercesStep@xercesc_2_3@@@xercesc_2_3@@6B@ 12130db0     XercesXPath.obj
 0002:0002ddb4       ??_7?$BaseRefVectorOf@VXercesLocationPath@xercesc_2_3@@@xercesc_2_3@@6B@ 12130db4     XercesXPath.obj
 0002:0002ddb8       ??_7XPathMatcher@xercesc_2_3@@6B@ 12130db8     XPathMatcher.obj
 0002:0002ddd0       ??_7?$RefVectorOf@V?$ValueStackOf@H@xercesc_2_3@@@xercesc_2_3@@6B@ 12130dd0     XPathMatcher.obj
 0002:0002ddd4       ??_7?$BaseRefVectorOf@V?$ValueStackOf@H@xercesc_2_3@@@xercesc_2_3@@6B@ 12130dd4     XPathMatcher.obj
 0002:0002ddd8       ??_7?$RefVectorOf@VXPathMatcher@xercesc_2_3@@@xercesc_2_3@@6B@ 12130dd8     XPathMatcherStack.obj
 0002:0002dddc       ??_7?$BaseRefVectorOf@VXPathMatcher@xercesc_2_3@@@xercesc_2_3@@6B@ 12130ddc     XPathMatcherStack.obj
 0002:0002dde0       ?fgSYMBOL_AND@XPathSymbols@xercesc_2_3@@2QBGB 12130de0     XPathSymbols.obj
 0002:0002dde8       ?fgSYMBOL_OR@XPathSymbols@xercesc_2_3@@2QBGB 12130de8     XPathSymbols.obj
 0002:0002ddf0       ?fgSYMBOL_MOD@XPathSymbols@xercesc_2_3@@2QBGB 12130df0     XPathSymbols.obj
 0002:0002ddf8       ?fgSYMBOL_DIV@XPathSymbols@xercesc_2_3@@2QBGB 12130df8     XPathSymbols.obj
 0002:0002de00       ?fgSYMBOL_COMMENT@XPathSymbols@xercesc_2_3@@2QBGB 12130e00     XPathSymbols.obj
 0002:0002de10       ?fgSYMBOL_TEXT@XPathSymbols@xercesc_2_3@@2QBGB 12130e10     XPathSymbols.obj
 0002:0002de1c       ?fgSYMBOL_PI@XPathSymbols@xercesc_2_3@@2QBGB 12130e1c     XPathSymbols.obj
 0002:0002de4c       ?fgSYMBOL_NODE@XPathSymbols@xercesc_2_3@@2QBGB 12130e4c     XPathSymbols.obj
 0002:0002de58       ?fgSYMBOL_ANCESTOR@XPathSymbols@xercesc_2_3@@2QBGB 12130e58     XPathSymbols.obj
 0002:0002de6c       ?fgSYMBOL_ANCESTOR_OR_SELF@XPathSymbols@xercesc_2_3@@2QBGB 12130e6c     XPathSymbols.obj
 0002:0002de90       ?fgSYMBOL_ATTRIBUTE@XPathSymbols@xercesc_2_3@@2QBGB 12130e90     XPathSymbols.obj
 0002:0002dea4       ?fgSYMBOL_CHILD@XPathSymbols@xercesc_2_3@@2QBGB 12130ea4     XPathSymbols.obj
 0002:0002deb0       ?fgSYMBOL_DESCENDANT@XPathSymbols@xercesc_2_3@@2QBGB 12130eb0     XPathSymbols.obj
 0002:0002dec8       ?fgSYMBOL_DESCENDANT_OR_SELF@XPathSymbols@xercesc_2_3@@2QBGB 12130ec8     XPathSymbols.obj
 0002:0002def0       ?fgSYMBOL_FOLLOWING@XPathSymbols@xercesc_2_3@@2QBGB 12130ef0     XPathSymbols.obj
 0002:0002df04       ?fgSYMBOL_FOLLOWING_SIBLING@XPathSymbols@xercesc_2_3@@2QBGB 12130f04     XPathSymbols.obj
 0002:0002df28       ?fgSYMBOL_NAMESPACE@XPathSymbols@xercesc_2_3@@2QBGB 12130f28     XPathSymbols.obj
 0002:0002df3c       ?fgSYMBOL_PARENT@XPathSymbols@xercesc_2_3@@2QBGB 12130f3c     XPathSymbols.obj
 0002:0002df4c       ?fgSYMBOL_PRECEDING@XPathSymbols@xercesc_2_3@@2QBGB 12130f4c     XPathSymbols.obj
 0002:0002df60       ?fgSYMBOL_PRECEDING_SIBLING@XPathSymbols@xercesc_2_3@@2QBGB 12130f60     XPathSymbols.obj
 0002:0002df84       ?fgSYMBOL_SELF@XPathSymbols@xercesc_2_3@@2QBGB 12130f84     XPathSymbols.obj
 0002:0002df90       ??_7SchemaAttDefList@xercesc_2_3@@6B@ 12130f90     ComplexTypeInfo.obj
 0002:0002dfb4       ??_7?$RefVectorOf@VContentSpecNode@xercesc_2_3@@@xercesc_2_3@@6B@ 12130fb4     ComplexTypeInfo.obj
 0002:0002dfb8       ??_7?$BaseRefVectorOf@VContentSpecNode@xercesc_2_3@@@xercesc_2_3@@6B@ 12130fb8     ComplexTypeInfo.obj
 0002:0002dff4       ??_7SchemaAttDef@xercesc_2_3@@6B@ 12130ff4     SchemaAttDef.obj
 0002:0002e008       ??_7SchemaElementDecl@xercesc_2_3@@6B@ 12131008     SchemaElementDecl.obj
 0002:0002e044       ??_7?$RefVectorOf@VSchemaAttDef@xercesc_2_3@@@xercesc_2_3@@6B@ 12131044     SchemaGrammar.obj
 0002:0002e048       ??_7?$BaseRefVectorOf@VSchemaAttDef@xercesc_2_3@@@xercesc_2_3@@6B@ 12131048     SchemaGrammar.obj
 0002:0002e04c       ??_7SchemaGrammar@xercesc_2_3@@6B@ 1213104c     SchemaGrammar.obj
 0002:0002e090       ?fgURI_XSI@SchemaSymbols@xercesc_2_3@@2QBGB 12131090     SchemaSymbols.obj
 0002:0002e0e4       ?fgURI_SCHEMAFORSCHEMA@SchemaSymbols@xercesc_2_3@@2QBGB 121310e4     SchemaSymbols.obj
 0002:0002e128       ?fgXSI_SCHEMALOCACTION@SchemaSymbols@xercesc_2_3@@2QBGB 12131128     SchemaSymbols.obj
 0002:0002e148       ?fgXSI_NONAMESPACESCHEMALOCACTION@SchemaSymbols@xercesc_2_3@@2QBGB 12131148     SchemaSymbols.obj
 0002:0002e17c       ?fgXSI_TYPE@SchemaSymbols@xercesc_2_3@@2QBGB 1213117c     SchemaSymbols.obj
 0002:0002e188       ?fgELT_ALL@SchemaSymbols@xercesc_2_3@@2QBGB 12131188     SchemaSymbols.obj
 0002:0002e190       ?fgELT_ANNOTATION@SchemaSymbols@xercesc_2_3@@2QBGB 12131190     SchemaSymbols.obj
 0002:0002e1a8       ?fgELT_ANY@SchemaSymbols@xercesc_2_3@@2QBGB 121311a8     SchemaSymbols.obj
 0002:0002e1b0       ?fgELT_WILDCARD@SchemaSymbols@xercesc_2_3@@2QBGB 121311b0     SchemaSymbols.obj
 0002:0002e1b8       ?fgELT_ANYATTRIBUTE@SchemaSymbols@xercesc_2_3@@2QBGB 121311b8     SchemaSymbols.obj
 0002:0002e1d4       ?fgELT_APPINFO@SchemaSymbols@xercesc_2_3@@2QBGB 121311d4     SchemaSymbols.obj
 0002:0002e1e4       ?fgELT_ATTRIBUTE@SchemaSymbols@xercesc_2_3@@2QBGB 121311e4     SchemaSymbols.obj
 0002:0002e1f8       ?fgELT_ATTRIBUTEGROUP@SchemaSymbols@xercesc_2_3@@2QBGB 121311f8     SchemaSymbols.obj
 0002:0002e218       ?fgELT_CHOICE@SchemaSymbols@xercesc_2_3@@2QBGB 12131218     SchemaSymbols.obj
 0002:0002e228       ?fgELT_COMPLEXTYPE@SchemaSymbols@xercesc_2_3@@2QBGB 12131228     SchemaSymbols.obj
 0002:0002e240       ?fgELT_CONTENT@SchemaSymbols@xercesc_2_3@@2QBGB 12131240     SchemaSymbols.obj
 0002:0002e250       ?fgELT_DOCUMENTATION@SchemaSymbols@xercesc_2_3@@2QBGB 12131250     SchemaSymbols.obj
 0002:0002e26c       ?fgELT_DURATION@SchemaSymbols@xercesc_2_3@@2QBGB 1213126c     SchemaSymbols.obj
 0002:0002e280       ?fgELT_ELEMENT@SchemaSymbols@xercesc_2_3@@2QBGB 12131280     SchemaSymbols.obj
 0002:0002e290       ?fgELT_ENCODING@SchemaSymbols@xercesc_2_3@@2QBGB 12131290     SchemaSymbols.obj
 0002:0002e2a4       ?fgELT_ENUMERATION@SchemaSymbols@xercesc_2_3@@2QBGB 121312a4     SchemaSymbols.obj
 0002:0002e2bc       ?fgELT_FIELD@SchemaSymbols@xercesc_2_3@@2QBGB 121312bc     SchemaSymbols.obj
 0002:0002e2c8       ?fgELT_WHITESPACE@SchemaSymbols@xercesc_2_3@@2QBGB 121312c8     SchemaSymbols.obj
 0002:0002e2e0       ?fgELT_GROUP@SchemaSymbols@xercesc_2_3@@2QBGB 121312e0     SchemaSymbols.obj
 0002:0002e2ec       ?fgELT_IMPORT@SchemaSymbols@xercesc_2_3@@2QBGB 121312ec     SchemaSymbols.obj
 0002:0002e2fc       ?fgELT_INCLUDE@SchemaSymbols@xercesc_2_3@@2QBGB 121312fc     SchemaSymbols.obj
 0002:0002e30c       ?fgELT_REDEFINE@SchemaSymbols@xercesc_2_3@@2QBGB 1213130c     SchemaSymbols.obj
 0002:0002e320       ?fgELT_KEY@SchemaSymbols@xercesc_2_3@@2QBGB 12131320     SchemaSymbols.obj
 0002:0002e328       ?fgELT_KEYREF@SchemaSymbols@xercesc_2_3@@2QBGB 12131328     SchemaSymbols.obj
 0002:0002e338       ?fgELT_LENGTH@SchemaSymbols@xercesc_2_3@@2QBGB 12131338     SchemaSymbols.obj
 0002:0002e348       ?fgELT_MAXEXCLUSIVE@SchemaSymbols@xercesc_2_3@@2QBGB 12131348     SchemaSymbols.obj
 0002:0002e364       ?fgELT_MAXINCLUSIVE@SchemaSymbols@xercesc_2_3@@2QBGB 12131364     SchemaSymbols.obj
 0002:0002e380       ?fgELT_MAXLENGTH@SchemaSymbols@xercesc_2_3@@2QBGB 12131380     SchemaSymbols.obj
 0002:0002e394       ?fgELT_MINEXCLUSIVE@SchemaSymbols@xercesc_2_3@@2QBGB 12131394     SchemaSymbols.obj
 0002:0002e3b0       ?fgELT_MININCLUSIVE@SchemaSymbols@xercesc_2_3@@2QBGB 121313b0     SchemaSymbols.obj
 0002:0002e3cc       ?fgELT_MINLENGTH@SchemaSymbols@xercesc_2_3@@2QBGB 121313cc     SchemaSymbols.obj
 0002:0002e3e0       ?fgELT_NOTATION@SchemaSymbols@xercesc_2_3@@2QBGB 121313e0     SchemaSymbols.obj
 0002:0002e3f4       ?fgELT_PATTERN@SchemaSymbols@xercesc_2_3@@2QBGB 121313f4     SchemaSymbols.obj
 0002:0002e404       ?fgELT_PERIOD@SchemaSymbols@xercesc_2_3@@2QBGB 12131404     SchemaSymbols.obj
 0002:0002e414       ?fgELT_TOTALDIGITS@SchemaSymbols@xercesc_2_3@@2QBGB 12131414     SchemaSymbols.obj
 0002:0002e42c       ?fgELT_FRACTIONDIGITS@SchemaSymbols@xercesc_2_3@@2QBGB 1213142c     SchemaSymbols.obj
 0002:0002e44c       ?fgELT_SCHEMA@SchemaSymbols@xercesc_2_3@@2QBGB 1213144c     SchemaSymbols.obj
 0002:0002e45c       ?fgELT_SELECTOR@SchemaSymbols@xercesc_2_3@@2QBGB 1213145c     SchemaSymbols.obj
 0002:0002e470       ?fgELT_SEQUENCE@SchemaSymbols@xercesc_2_3@@2QBGB 12131470     SchemaSymbols.obj
 0002:0002e484       ?fgELT_SIMPLETYPE@SchemaSymbols@xercesc_2_3@@2QBGB 12131484     SchemaSymbols.obj
 0002:0002e49c       ?fgELT_UNION@SchemaSymbols@xercesc_2_3@@2QBGB 1213149c     SchemaSymbols.obj
 0002:0002e4a8       ?fgELT_LIST@SchemaSymbols@xercesc_2_3@@2QBGB 121314a8     SchemaSymbols.obj
 0002:0002e4b4       ?fgELT_UNIQUE@SchemaSymbols@xercesc_2_3@@2QBGB 121314b4     SchemaSymbols.obj
 0002:0002e4c4       ?fgELT_COMPLEXCONTENT@SchemaSymbols@xercesc_2_3@@2QBGB 121314c4     SchemaSymbols.obj
 0002:0002e4e4       ?fgELT_SIMPLECONTENT@SchemaSymbols@xercesc_2_3@@2QBGB 121314e4     SchemaSymbols.obj
 0002:0002e500       ?fgELT_RESTRICTION@SchemaSymbols@xercesc_2_3@@2QBGB 12131500     SchemaSymbols.obj
 0002:0002e518       ?fgELT_EXTENSION@SchemaSymbols@xercesc_2_3@@2QBGB 12131518     SchemaSymbols.obj
 0002:0002e52c       ?fgATT_ABSTRACT@SchemaSymbols@xercesc_2_3@@2QBGB 1213152c     SchemaSymbols.obj
 0002:0002e540       ?fgATT_ATTRIBUTEFORMDEFAULT@SchemaSymbols@xercesc_2_3@@2QBGB 12131540     SchemaSymbols.obj
 0002:0002e56c       ?fgATT_BASE@SchemaSymbols@xercesc_2_3@@2QBGB 1213156c     SchemaSymbols.obj
 0002:0002e578       ?fgATT_ITEMTYPE@SchemaSymbols@xercesc_2_3@@2QBGB 12131578     SchemaSymbols.obj
 0002:0002e58c       ?fgATT_MEMBERTYPES@SchemaSymbols@xercesc_2_3@@2QBGB 1213158c     SchemaSymbols.obj
 0002:0002e5a4       ?fgATT_BLOCK@SchemaSymbols@xercesc_2_3@@2QBGB 121315a4     SchemaSymbols.obj
 0002:0002e5b0       ?fgATT_BLOCKDEFAULT@SchemaSymbols@xercesc_2_3@@2QBGB 121315b0     SchemaSymbols.obj
 0002:0002e5cc       ?fgATT_DEFAULT@SchemaSymbols@xercesc_2_3@@2QBGB 121315cc     SchemaSymbols.obj
 0002:0002e5dc       ?fgATT_ELEMENTFORMDEFAULT@SchemaSymbols@xercesc_2_3@@2QBGB 121315dc     SchemaSymbols.obj
 0002:0002e604       ?fgATT_SUBSTITUTIONGROUP@SchemaSymbols@xercesc_2_3@@2QBGB 12131604     SchemaSymbols.obj
 0002:0002e628       ?fgATT_FINAL@SchemaSymbols@xercesc_2_3@@2QBGB 12131628     SchemaSymbols.obj
 0002:0002e634       ?fgATT_FINALDEFAULT@SchemaSymbols@xercesc_2_3@@2QBGB 12131634     SchemaSymbols.obj
 0002:0002e650       ?fgATT_FIXED@SchemaSymbols@xercesc_2_3@@2QBGB 12131650     SchemaSymbols.obj
 0002:0002e65c       ?fgATT_FORM@SchemaSymbols@xercesc_2_3@@2QBGB 1213165c     SchemaSymbols.obj
 0002:0002e668       ?fgATT_ID@SchemaSymbols@xercesc_2_3@@2QBGB 12131668     SchemaSymbols.obj
 0002:0002e670       ?fgATT_MAXOCCURS@SchemaSymbols@xercesc_2_3@@2QBGB 12131670     SchemaSymbols.obj
 0002:0002e684       ?fgATT_MINOCCURS@SchemaSymbols@xercesc_2_3@@2QBGB 12131684     SchemaSymbols.obj
 0002:0002e698       ?fgATT_NAME@SchemaSymbols@xercesc_2_3@@2QBGB 12131698     SchemaSymbols.obj
 0002:0002e6a4       ?fgATT_NAMESPACE@SchemaSymbols@xercesc_2_3@@2QBGB 121316a4     SchemaSymbols.obj
 0002:0002e6b8       ?fgATT_NILL@SchemaSymbols@xercesc_2_3@@2QBGB 121316b8     SchemaSymbols.obj
 0002:0002e6c0       ?fgATT_NILLABLE@SchemaSymbols@xercesc_2_3@@2QBGB 121316c0     SchemaSymbols.obj
 0002:0002e6d4       ?fgATT_PROCESSCONTENTS@SchemaSymbols@xercesc_2_3@@2QBGB 121316d4     SchemaSymbols.obj
 0002:0002e6f4       ?fgATT_REF@SchemaSymbols@xercesc_2_3@@2QBGB 121316f4     SchemaSymbols.obj
 0002:0002e6fc       ?fgATT_REFER@SchemaSymbols@xercesc_2_3@@2QBGB 121316fc     SchemaSymbols.obj
 0002:0002e708       ?fgATT_SCHEMALOCATION@SchemaSymbols@xercesc_2_3@@2QBGB 12131708     SchemaSymbols.obj
 0002:0002e728       ?fgATT_SOURCE@SchemaSymbols@xercesc_2_3@@2QBGB 12131728     SchemaSymbols.obj
 0002:0002e738       ?fgATT_SYSTEM@SchemaSymbols@xercesc_2_3@@2QBGB 12131738     SchemaSymbols.obj
 0002:0002e748       ?fgATT_PUBLIC@SchemaSymbols@xercesc_2_3@@2QBGB 12131748     SchemaSymbols.obj
 0002:0002e758       ?fgATT_TARGETNAMESPACE@SchemaSymbols@xercesc_2_3@@2QBGB 12131758     SchemaSymbols.obj
 0002:0002e778       ?fgATT_TYPE@SchemaSymbols@xercesc_2_3@@2QBGB 12131778     SchemaSymbols.obj
 0002:0002e784       ?fgATT_USE@SchemaSymbols@xercesc_2_3@@2QBGB 12131784     SchemaSymbols.obj
 0002:0002e78c       ?fgATT_VALUE@SchemaSymbols@xercesc_2_3@@2QBGB 1213178c     SchemaSymbols.obj
 0002:0002e798       ?fgATT_MIXED@SchemaSymbols@xercesc_2_3@@2QBGB 12131798     SchemaSymbols.obj
 0002:0002e7a4       ?fgATT_VERSION@SchemaSymbols@xercesc_2_3@@2QBGB 121317a4     SchemaSymbols.obj
 0002:0002e7b4       ?fgATT_XPATH@SchemaSymbols@xercesc_2_3@@2QBGB 121317b4     SchemaSymbols.obj
 0002:0002e7c0       ?fgATTVAL_TWOPOUNDANY@SchemaSymbols@xercesc_2_3@@2QBGB 121317c0     SchemaSymbols.obj
 0002:0002e7cc       ?fgATTVAL_TWOPOUNDLOCAL@SchemaSymbols@xercesc_2_3@@2QBGB 121317cc     SchemaSymbols.obj
 0002:0002e7dc       ?fgATTVAL_TWOPOUNDOTHER@SchemaSymbols@xercesc_2_3@@2QBGB 121317dc     SchemaSymbols.obj
 0002:0002e7ec       ?fgATTVAL_TWOPOUNDTRAGETNAMESPACE@SchemaSymbols@xercesc_2_3@@2QBGB 121317ec     SchemaSymbols.obj
 0002:0002e810       ?fgATTVAL_POUNDALL@SchemaSymbols@xercesc_2_3@@2QBGB 12131810     SchemaSymbols.obj
 0002:0002e81c       ?fgATTVAL_BASE64@SchemaSymbols@xercesc_2_3@@2QBGB 1213181c     SchemaSymbols.obj
 0002:0002e82c       ?fgATTVAL_BOOLEAN@SchemaSymbols@xercesc_2_3@@2QBGB 1213182c     SchemaSymbols.obj
 0002:0002e83c       ?fgATTVAL_DEFAULT@SchemaSymbols@xercesc_2_3@@2QBGB 1213183c     SchemaSymbols.obj
 0002:0002e84c       ?fgATTVAL_ELEMENTONLY@SchemaSymbols@xercesc_2_3@@2QBGB 1213184c     SchemaSymbols.obj
 0002:0002e864       ?fgATTVAL_EMPTY@SchemaSymbols@xercesc_2_3@@2QBGB 12131864     SchemaSymbols.obj
 0002:0002e870       ?fgATTVAL_EXTENSION@SchemaSymbols@xercesc_2_3@@2QBGB 12131870     SchemaSymbols.obj
 0002:0002e884       ?fgATTVAL_FALSE@SchemaSymbols@xercesc_2_3@@2QBGB 12131884     SchemaSymbols.obj
 0002:0002e890       ?fgATTVAL_FIXED@SchemaSymbols@xercesc_2_3@@2QBGB 12131890     SchemaSymbols.obj
 0002:0002e89c       ?fgATTVAL_HEX@SchemaSymbols@xercesc_2_3@@2QBGB 1213189c     SchemaSymbols.obj
 0002:0002e8a4       ?fgATTVAL_ID@SchemaSymbols@xercesc_2_3@@2QBGB 121318a4     SchemaSymbols.obj
 0002:0002e8ac       ?fgATTVAL_LAX@SchemaSymbols@xercesc_2_3@@2QBGB 121318ac     SchemaSymbols.obj
 0002:0002e8b4       ?fgATTVAL_MAXLENGTH@SchemaSymbols@xercesc_2_3@@2QBGB 121318b4     SchemaSymbols.obj
 0002:0002e8c8       ?fgATTVAL_MINLENGTH@SchemaSymbols@xercesc_2_3@@2QBGB 121318c8     SchemaSymbols.obj
 0002:0002e8dc       ?fgATTVAL_MIXED@SchemaSymbols@xercesc_2_3@@2QBGB 121318dc     SchemaSymbols.obj
 0002:0002e8e8       ?fgATTVAL_NCNAME@SchemaSymbols@xercesc_2_3@@2QBGB 121318e8     SchemaSymbols.obj
 0002:0002e8f8       ?fgATTVAL_OPTIONAL@SchemaSymbols@xercesc_2_3@@2QBGB 121318f8     SchemaSymbols.obj
 0002:0002e90c       ?fgATTVAL_PROHIBITED@SchemaSymbols@xercesc_2_3@@2QBGB 1213190c     SchemaSymbols.obj
 0002:0002e924       ?fgATTVAL_QNAME@SchemaSymbols@xercesc_2_3@@2QBGB 12131924     SchemaSymbols.obj
 0002:0002e930       ?fgATTVAL_QUALIFIED@SchemaSymbols@xercesc_2_3@@2QBGB 12131930     SchemaSymbols.obj
 0002:0002e944       ?fgATTVAL_REQUIRED@SchemaSymbols@xercesc_2_3@@2QBGB 12131944     SchemaSymbols.obj
 0002:0002e958       ?fgATTVAL_RESTRICTION@SchemaSymbols@xercesc_2_3@@2QBGB 12131958     SchemaSymbols.obj
 0002:0002e970       ?fgATTVAL_SKIP@SchemaSymbols@xercesc_2_3@@2QBGB 12131970     SchemaSymbols.obj
 0002:0002e97c       ?fgATTVAL_STRICT@SchemaSymbols@xercesc_2_3@@2QBGB 1213197c     SchemaSymbols.obj
 0002:0002e98c       ?fgATTVAL_STRING@SchemaSymbols@xercesc_2_3@@2QBGB 1213198c     SchemaSymbols.obj
 0002:0002e99c       ?fgATTVAL_TEXTONLY@SchemaSymbols@xercesc_2_3@@2QBGB 1213199c     SchemaSymbols.obj
 0002:0002e9b0       ?fgATTVAL_TIMEDURATION@SchemaSymbols@xercesc_2_3@@2QBGB 121319b0     SchemaSymbols.obj
 0002:0002e9cc       ?fgATTVAL_TRUE@SchemaSymbols@xercesc_2_3@@2QBGB 121319cc     SchemaSymbols.obj
 0002:0002e9d8       ?fgATTVAL_UNQUALIFIED@SchemaSymbols@xercesc_2_3@@2QBGB 121319d8     SchemaSymbols.obj
 0002:0002e9f0       ?fgATTVAL_URI@SchemaSymbols@xercesc_2_3@@2QBGB 121319f0     SchemaSymbols.obj
 0002:0002e9f8       ?fgATTVAL_URIREFERENCE@SchemaSymbols@xercesc_2_3@@2QBGB 121319f8     SchemaSymbols.obj
 0002:0002ea14       ?fgATTVAL_SUBSTITUTIONGROUP@SchemaSymbols@xercesc_2_3@@2QBGB 12131a14     SchemaSymbols.obj
 0002:0002ea38       ?fgATTVAL_SUBSTITUTION@SchemaSymbols@xercesc_2_3@@2QBGB 12131a38     SchemaSymbols.obj
 0002:0002ea54       ?fgATTVAL_ANYTYPE@SchemaSymbols@xercesc_2_3@@2QBGB 12131a54     SchemaSymbols.obj
 0002:0002ea64       ?fgWS_PRESERVE@SchemaSymbols@xercesc_2_3@@2QBGB 12131a64     SchemaSymbols.obj
 0002:0002ea78       ?fgWS_COLLAPSE@SchemaSymbols@xercesc_2_3@@2QBGB 12131a78     SchemaSymbols.obj
 0002:0002ea8c       ?fgWS_REPLACE@SchemaSymbols@xercesc_2_3@@2QBGB 12131a8c     SchemaSymbols.obj
 0002:0002ea9c       ?fgDT_STRING@SchemaSymbols@xercesc_2_3@@2QBGB 12131a9c     SchemaSymbols.obj
 0002:0002eaac       ?fgDT_TOKEN@SchemaSymbols@xercesc_2_3@@2QBGB 12131aac     SchemaSymbols.obj
 0002:0002eab8       ?fgDT_LANGUAGE@SchemaSymbols@xercesc_2_3@@2QBGB 12131ab8     SchemaSymbols.obj
 0002:0002eacc       ?fgDT_NAME@SchemaSymbols@xercesc_2_3@@2QBGB 12131acc     SchemaSymbols.obj
 0002:0002ead8       ?fgDT_NCNAME@SchemaSymbols@xercesc_2_3@@2QBGB 12131ad8     SchemaSymbols.obj
 0002:0002eae8       ?fgDT_INTEGER@SchemaSymbols@xercesc_2_3@@2QBGB 12131ae8     SchemaSymbols.obj
 0002:0002eaf8       ?fgDT_DECIMAL@SchemaSymbols@xercesc_2_3@@2QBGB 12131af8     SchemaSymbols.obj
 0002:0002eb08       ?fgDT_BOOLEAN@SchemaSymbols@xercesc_2_3@@2QBGB 12131b08     SchemaSymbols.obj
 0002:0002eb18       ?fgDT_NONPOSITIVEINTEGER@SchemaSymbols@xercesc_2_3@@2QBGB 12131b18     SchemaSymbols.obj
 0002:0002eb40       ?fgDT_NEGATIVEINTEGER@SchemaSymbols@xercesc_2_3@@2QBGB 12131b40     SchemaSymbols.obj
 0002:0002eb60       ?fgDT_LONG@SchemaSymbols@xercesc_2_3@@2QBGB 12131b60     SchemaSymbols.obj
 0002:0002eb6c       ?fgDT_INT@SchemaSymbols@xercesc_2_3@@2QBGB 12131b6c     SchemaSymbols.obj
 0002:0002eb74       ?fgDT_SHORT@SchemaSymbols@xercesc_2_3@@2QBGB 12131b74     SchemaSymbols.obj
 0002:0002eb80       ?fgDT_BYTE@SchemaSymbols@xercesc_2_3@@2QBGB 12131b80     SchemaSymbols.obj
 0002:0002eb8c       ?fgDT_NONNEGATIVEINTEGER@SchemaSymbols@xercesc_2_3@@2QBGB 12131b8c     SchemaSymbols.obj
 0002:0002ebb4       ?fgDT_ULONG@SchemaSymbols@xercesc_2_3@@2QBGB 12131bb4     SchemaSymbols.obj
 0002:0002ebd0       ?fgDT_UINT@SchemaSymbols@xercesc_2_3@@2QBGB 12131bd0     SchemaSymbols.obj
 0002:0002ebe8       ?fgDT_USHORT@SchemaSymbols@xercesc_2_3@@2QBGB 12131be8     SchemaSymbols.obj
 0002:0002ec04       ?fgDT_UBYTE@SchemaSymbols@xercesc_2_3@@2QBGB 12131c04     SchemaSymbols.obj
 0002:0002ec20       ?fgDT_POSITIVEINTEGER@SchemaSymbols@xercesc_2_3@@2QBGB 12131c20     SchemaSymbols.obj
 0002:0002ec40       ?fgDT_DATETIME@SchemaSymbols@xercesc_2_3@@2QBGB 12131c40     SchemaSymbols.obj
 0002:0002ec54       ?fgDT_DATE@SchemaSymbols@xercesc_2_3@@2QBGB 12131c54     SchemaSymbols.obj
 0002:0002ec60       ?fgDT_TIME@SchemaSymbols@xercesc_2_3@@2QBGB 12131c60     SchemaSymbols.obj
 0002:0002ec6c       ?fgDT_DURATION@SchemaSymbols@xercesc_2_3@@2QBGB 12131c6c     SchemaSymbols.obj
 0002:0002ec80       ?fgDT_DAY@SchemaSymbols@xercesc_2_3@@2QBGB 12131c80     SchemaSymbols.obj
 0002:0002ec8c       ?fgDT_MONTH@SchemaSymbols@xercesc_2_3@@2QBGB 12131c8c     SchemaSymbols.obj
 0002:0002ec9c       ?fgDT_MONTHDAY@SchemaSymbols@xercesc_2_3@@2QBGB 12131c9c     SchemaSymbols.obj
 0002:0002ecb0       ?fgDT_YEAR@SchemaSymbols@xercesc_2_3@@2QBGB 12131cb0     SchemaSymbols.obj
 0002:0002ecbc       ?fgDT_YEARMONTH@SchemaSymbols@xercesc_2_3@@2QBGB 12131cbc     SchemaSymbols.obj
 0002:0002ecd4       ?fgDT_BASE64BINARY@SchemaSymbols@xercesc_2_3@@2QBGB 12131cd4     SchemaSymbols.obj
 0002:0002ecf0       ?fgDT_HEXBINARY@SchemaSymbols@xercesc_2_3@@2QBGB 12131cf0     SchemaSymbols.obj
 0002:0002ed04       ?fgDT_FLOAT@SchemaSymbols@xercesc_2_3@@2QBGB 12131d04     SchemaSymbols.obj
 0002:0002ed10       ?fgDT_DOUBLE@SchemaSymbols@xercesc_2_3@@2QBGB 12131d10     SchemaSymbols.obj
 0002:0002ed20       ?fgDT_URIREFERENCE@SchemaSymbols@xercesc_2_3@@2QBGB 12131d20     SchemaSymbols.obj
 0002:0002ed3c       ?fgDT_ANYURI@SchemaSymbols@xercesc_2_3@@2QBGB 12131d3c     SchemaSymbols.obj
 0002:0002ed4c       ?fgDT_QNAME@SchemaSymbols@xercesc_2_3@@2QBGB 12131d4c     SchemaSymbols.obj
 0002:0002ed58       ?fgDT_NORMALIZEDSTRING@SchemaSymbols@xercesc_2_3@@2QBGB 12131d58     SchemaSymbols.obj
 0002:0002ed7c       ?fgDT_ANYSIMPLETYPE@SchemaSymbols@xercesc_2_3@@2QBGB 12131d7c     SchemaSymbols.obj
 0002:0002ed98       ?fgRegEx_XOption@SchemaSymbols@xercesc_2_3@@2QBGB 12131d98     SchemaSymbols.obj
 0002:0002ed9c       ?fgRedefIdentifier@SchemaSymbols@xercesc_2_3@@2QBGB 12131d9c     SchemaSymbols.obj
 0002:0002eda8       ?fgINT_MIN_VALUE@SchemaSymbols@xercesc_2_3@@2HB 12131da8     SchemaSymbols.obj
 0002:0002edac       ?fgINT_MAX_VALUE@SchemaSymbols@xercesc_2_3@@2HB 12131dac     SchemaSymbols.obj
 0002:0002edb0       ??_7SchemaValidator@xercesc_2_3@@6B@ 12131db0     SchemaValidator.obj
 0002:0002ede4       ??_7?$XMLEnumerator@VComplexTypeInfo@xercesc_2_3@@@xercesc_2_3@@6B@ 12131de4     SchemaValidator.obj
 0002:0002edf4       ??_7?$XMLEnumerator@VXercesGroupInfo@xercesc_2_3@@@xercesc_2_3@@6B@ 12131df4     SchemaValidator.obj
 0002:0002ee04       ??_7?$RefHashTableOfEnumerator@VXercesGroupInfo@xercesc_2_3@@@xercesc_2_3@@6B@ 12131e04     SchemaValidator.obj
 0002:0002ee14       ??_7?$RefHashTableOfEnumerator@VComplexTypeInfo@xercesc_2_3@@@xercesc_2_3@@6B@ 12131e14     SchemaValidator.obj
 0002:0002ee8c       ??_7?$RefVectorOf@VDatatypeValidator@xercesc_2_3@@@xercesc_2_3@@6B@ 12131e8c     TraverseSchema.obj
 0002:0002ee90       ??_7?$BaseRefVectorOf@VDatatypeValidator@xercesc_2_3@@@xercesc_2_3@@6B@ 12131e90     TraverseSchema.obj
 0002:0002ee94       ??_7XSDDOMParser@xercesc_2_3@@6BDocTypeHandler@1@@ 12131e94     XSDDOMParser.obj
 0002:0002eed8       ??_7XSDDOMParser@xercesc_2_3@@6BXMLEntityHandler@1@@ 12131ed8     XSDDOMParser.obj
 0002:0002eef0       ??_7XSDDOMParser@xercesc_2_3@@6BXMLErrorReporter@1@@ 12131ef0     XSDDOMParser.obj
 0002:0002eefc       ??_7XSDDOMParser@xercesc_2_3@@6BXMLDocumentHandler@1@@ 12131efc     XSDDOMParser.obj
 0002:0002ef34       ??_7XSDLocator@xercesc_2_3@@6B@ 12131f34     XSDLocator.obj
 0002:0002ef48       ??_7DefaultHandler@xercesc_2_3@@6BDeclHandler@1@@ 12131f48     sax2Dummy.obj
 0002:0002ef5c       ??_7DefaultHandler@xercesc_2_3@@6BLexicalHandler@1@@ 12131f5c     sax2Dummy.obj
 0002:0002ef7c       ??_7DefaultHandler@xercesc_2_3@@6BErrorHandler@1@@ 12131f7c     sax2Dummy.obj
 0002:0002ef90       ??_7DefaultHandler@xercesc_2_3@@6BContentHandler@1@@ 12131f90     sax2Dummy.obj
 0002:0002efc0       ??_7DefaultHandler@xercesc_2_3@@6BDTDHandler@1@@ 12131fc0     sax2Dummy.obj
 0002:0002efd0       ??_7DefaultHandler@xercesc_2_3@@6BEntityResolver@1@@ 12131fd0     sax2Dummy.obj
 0002:0002efdc       ??_7DOMAttrImpl@xercesc_2_3@@6B@ 12131fdc     DOMAttrImpl.obj
 0002:0002f0a8       ??_7DOMAttrMapImpl@xercesc_2_3@@6B@ 121320a8     DOMAttrMapImpl.obj
 0002:0002f0f4       ??_7DOMAttrNSImpl@xercesc_2_3@@6B@ 121320f4     DOMAttrNSImpl.obj
 0002:0002f1e0       ??_7DOMRange@xercesc_2_3@@6B@ 121321e0     DOMCDATASectionImpl.obj
 0002:0002f248       ??_7DOMCDATASectionImpl@xercesc_2_3@@6B@ 12132248     DOMCDATASectionImpl.obj
 0002:0002f32c       ??_7DOMCommentImpl@xercesc_2_3@@6B@ 1213232c     DOMCommentImpl.obj
 0002:0002f3e8       ?fgCANONICAL_FORM@DOMConfigurationImpl@xercesc_2_3@@2QBGB 121323e8     DOMConfigurationImpl.obj
 0002:0002f408       ?fgCDATA_SECTIONS@DOMConfigurationImpl@xercesc_2_3@@2QBGB 12132408     DOMConfigurationImpl.obj
 0002:0002f428       ?fgCOMMENTS@DOMConfigurationImpl@xercesc_2_3@@2QBGB 12132428     DOMConfigurationImpl.obj
 0002:0002f43c       ?fgDATATYPE_NORMALIZATION@DOMConfigurationImpl@xercesc_2_3@@2QBGB 1213243c     DOMConfigurationImpl.obj
 0002:0002f46c       ?fgDISCARD_DEFAULT_CONTENT@DOMConfigurationImpl@xercesc_2_3@@2QBGB 1213246c     DOMConfigurationImpl.obj
 0002:0002f49c       ?fgENTITIES@DOMConfigurationImpl@xercesc_2_3@@2QBGB 1213249c     DOMConfigurationImpl.obj
 0002:0002f4b0       ?fgINFOSET@DOMConfigurationImpl@xercesc_2_3@@2QBGB 121324b0     DOMConfigurationImpl.obj
 0002:0002f4c0       ?fgNAMESPACES@DOMConfigurationImpl@xercesc_2_3@@2QBGB 121324c0     DOMConfigurationImpl.obj
 0002:0002f4d8       ?fgNAMESPACE_DECLARATIONS@DOMConfigurationImpl@xercesc_2_3@@2QBGB 121324d8     DOMConfigurationImpl.obj
 0002:0002f508       ?fgNORMALIZE_CHARACTERS@DOMConfigurationImpl@xercesc_2_3@@2QBGB 12132508     DOMConfigurationImpl.obj
 0002:0002f534       ?fgSPLIT_CDATA_SECTIONS@DOMConfigurationImpl@xercesc_2_3@@2QBGB 12132534     DOMConfigurationImpl.obj
 0002:0002f560       ?fgVALIDATE@DOMConfigurationImpl@xercesc_2_3@@2QBGB 12132560     DOMConfigurationImpl.obj
 0002:0002f574       ?fgVALIDATE_IF_SCHEMA@DOMConfigurationImpl@xercesc_2_3@@2QBGB 12132574     DOMConfigurationImpl.obj
 0002:0002f59c       ?fgWHITESPACE_IN_ELEMENT_CONTENT@DOMConfigurationImpl@xercesc_2_3@@2QBGB 1213259c     DOMConfigurationImpl.obj
 0002:0002f5d8       ?fgERROR_HANDLER@DOMConfigurationImpl@xercesc_2_3@@2QBGB 121325d8     DOMConfigurationImpl.obj
 0002:0002f5f4       ?fgSCHEMA_TYPE@DOMConfigurationImpl@xercesc_2_3@@2QBGB 121325f4     DOMConfigurationImpl.obj
 0002:0002f60c       ?fgSCHEMA_LOCATION@DOMConfigurationImpl@xercesc_2_3@@2QBGB 1213260c     DOMConfigurationImpl.obj
 0002:0002f62c       ?fDEFAULT_VALUES@DOMConfigurationImpl@xercesc_2_3@@2GB 1213262c     DOMConfigurationImpl.obj
 0002:0002f630       ??_7DOMConfiguration@xercesc_2_3@@6B@ 12132630     DOMConfigurationImpl.obj
 0002:0002f63c       ??_7DOMConfigurationImpl@xercesc_2_3@@6B@ 1213263c     DOMConfigurationImpl.obj
 0002:0002f64c       ??_7DOMDeepNodeListImpl@xercesc_2_3@@6B@ 1213264c     DOMDeepNodeListImpl.obj
 0002:0002f680       ??_7DOMDocumentFragment@xercesc_2_3@@6B@ 12132680     DOMDocumentFragmentImpl.obj
 0002:0002f71c       ??_7DOMDocumentFragmentImpl@xercesc_2_3@@6B@ 1213271c     DOMDocumentFragmentImpl.obj
 0002:0002f7cc       ??_7DOMNodeFilter@xercesc_2_3@@6B@ 121327cc     DOMDocumentImpl.obj
 0002:0002f7d4       ??_7DOMTreeWalker@xercesc_2_3@@6B@ 121327d4     DOMDocumentImpl.obj
 0002:0002f810       ??_7DOMNodeIterator@xercesc_2_3@@6B@ 12132810     DOMDocumentImpl.obj
 0002:0002f834       ??_7DOMDocumentImpl@xercesc_2_3@@6BDOMNode@1@@ 12132834     DOMDocumentImpl.obj
 0002:0002f8d0       ??_7DOMDocumentImpl@xercesc_2_3@@6BDOMDocumentTraversal@1@@ 121328d0     DOMDocumentImpl.obj
 0002:0002f8dc       ??_7DOMDocumentImpl@xercesc_2_3@@6BDOMDocumentRange@1@@ 121328dc     DOMDocumentImpl.obj
 0002:0002f9a0       ??_7?$RefVectorOf@VDOMNodeIteratorImpl@xercesc_2_3@@@xercesc_2_3@@6B@ 121329a0     DOMDocumentImpl.obj
 0002:0002f9a4       ??_7?$BaseRefVectorOf@VDOMNodeIteratorImpl@xercesc_2_3@@@xercesc_2_3@@6B@ 121329a4     DOMDocumentImpl.obj
 0002:0002f9a8       ??_7?$RefVectorOf@VDOMRangeImpl@xercesc_2_3@@@xercesc_2_3@@6B@ 121329a8     DOMDocumentImpl.obj
 0002:0002f9ac       ??_7?$BaseRefVectorOf@VDOMRangeImpl@xercesc_2_3@@@xercesc_2_3@@6B@ 121329ac     DOMDocumentImpl.obj
 0002:0002f9b0       ??_7?$RefHashTableOfEnumerator@V?$KeyRefPair@XVDOMUserDataHandler@xercesc_2_3@@@xercesc_2_3@@@xercesc_2_3@@6B@ 121329b0     DOMDocumentImpl.obj
 0002:0002f9c0       ??_7?$RefVectorOf@VDOMNode@xercesc_2_3@@@xercesc_2_3@@6B@ 121329c0     DOMDocumentImpl.obj
 0002:0002f9c4       ??_7?$RefVectorOf@VDOMBuffer@xercesc_2_3@@@xercesc_2_3@@6B@ 121329c4     DOMDocumentImpl.obj
 0002:0002f9c8       ??_7?$BaseRefVectorOf@VDOMBuffer@xercesc_2_3@@@xercesc_2_3@@6B@ 121329c8     DOMDocumentImpl.obj
 0002:0002f9cc       ??_7?$XMLEnumerator@V?$KeyRefPair@XVDOMUserDataHandler@xercesc_2_3@@@xercesc_2_3@@@xercesc_2_3@@6B@ 121329cc     DOMDocumentImpl.obj
 0002:0002f9dc       ??_7?$BaseRefVectorOf@VDOMNode@xercesc_2_3@@@xercesc_2_3@@6B@ 121329dc     DOMDocumentImpl.obj
 0002:0002f9ec       ??_7DOMDocumentTypeImpl@xercesc_2_3@@6B@ 121329ec     DOMDocumentTypeImpl.obj
 0002:0002fabc       ??_7DOMElementImpl@xercesc_2_3@@6B@ 12132abc     DOMElementImpl.obj
 0002:0002fbc4       ??_7DOMElementNSImpl@xercesc_2_3@@6B@ 12132bc4     DOMElementNSImpl.obj
 0002:0002fccc       ??_7DOMEntityImpl@xercesc_2_3@@6B@ 12132ccc     DOMEntityImpl.obj
 0002:0002fda4       ??_7DOMEntityReferenceImpl@xercesc_2_3@@6B@ 12132da4     DOMEntityReferenceImpl.obj
 0002:0002fe44       ??_7DOMErrorImpl@xercesc_2_3@@6B@ 12132e44     DOMErrorImpl.obj
 0002:0002fecc       ??_7DOMImplementationSource@xercesc_2_3@@6B@ 12132ecc     DOMImplementationImpl.obj
 0002:0002fed4       ??_7DOMWriterFilter@xercesc_2_3@@6B@ 12132ed4     DOMImplementationImpl.obj
 0002:0002fee4       ??_7DOMWriter@xercesc_2_3@@6B@ 12132ee4     DOMImplementationImpl.obj
 0002:0002ff20       ??_7DOMImplementationImpl@xercesc_2_3@@6BDOMImplementationSource@1@@ 12132f20     DOMImplementationImpl.obj
 0002:0002ff28       ??_7DOMImplementationImpl@xercesc_2_3@@6BDOMImplementation@1@@ 12132f28     DOMImplementationImpl.obj
 0002:0002ff4c       ??_7?$RefVectorOf@VDOMImplementationSource@xercesc_2_3@@@xercesc_2_3@@6B@ 12132f4c     DOMImplementationRegistry.obj
 0002:0002ff50       ??_7?$BaseRefVectorOf@VDOMImplementationSource@xercesc_2_3@@@xercesc_2_3@@6B@ 12132f50     DOMImplementationRegistry.obj
 0002:0002ff54       ??_7DOMLocatorImpl@xercesc_2_3@@6B@ 12132f54     DOMLocatorImpl.obj
 0002:0002ff80       ??_7DOMNamedNodeMapImpl@xercesc_2_3@@6B@ 12132f80     DOMNamedNodeMapImpl.obj
 0002:0002ffd8       ??_7DOMNodeIDMap@xercesc_2_3@@6B@ 12132fd8     DOMNodeIDMap.obj
 0002:0002ffdc       ?READONLY@DOMNodeImpl@xercesc_2_3@@2GB 12132fdc     DOMNodeImpl.obj
 0002:0002ffde       ?SYNCDATA@DOMNodeImpl@xercesc_2_3@@2GB 12132fde     DOMNodeImpl.obj
 0002:0002ffe0       ?SYNCCHILDREN@DOMNodeImpl@xercesc_2_3@@2GB 12132fe0     DOMNodeImpl.obj
 0002:0002ffe2       ?OWNED@DOMNodeImpl@xercesc_2_3@@2GB 12132fe2     DOMNodeImpl.obj
 0002:0002ffe4       ?FIRSTCHILD@DOMNodeImpl@xercesc_2_3@@2GB 12132fe4     DOMNodeImpl.obj
 0002:0002ffe6       ?SPECIFIED@DOMNodeImpl@xercesc_2_3@@2GB 12132fe6     DOMNodeImpl.obj
 0002:0002ffe8       ?IGNORABLEWS@DOMNodeImpl@xercesc_2_3@@2GB 12132fe8     DOMNodeImpl.obj
 0002:0002ffea       ?SETVALUE@DOMNodeImpl@xercesc_2_3@@2GB 12132fea     DOMNodeImpl.obj
 0002:0002ffec       ?ID_ATTR@DOMNodeImpl@xercesc_2_3@@2GB 12132fec     DOMNodeImpl.obj
 0002:0002ffee       ?USERDATA@DOMNodeImpl@xercesc_2_3@@2GB 12132fee     DOMNodeImpl.obj
 0002:0002fff0       ?LEAFNODETYPE@DOMNodeImpl@xercesc_2_3@@2GB 12132ff0     DOMNodeImpl.obj
 0002:0002fff2       ?CHILDNODE@DOMNodeImpl@xercesc_2_3@@2GB 12132ff2     DOMNodeImpl.obj
 0002:0002fff4       ?TOBERELEASED@DOMNodeImpl@xercesc_2_3@@2GB 12132ff4     DOMNodeImpl.obj
 0002:00030130       ??_7DOMNodeIteratorImpl@xercesc_2_3@@6B@ 12133130     DOMNodeIteratorImpl.obj
 0002:00030154       ??_7DOMNodeListImpl@xercesc_2_3@@6B@ 12133154     DOMNodeListImpl.obj
 0002:00030160       ??_7?$RefVectorOf@VScope@InScopeNamespaces@DOMNormalizer@xercesc_2_3@@@xercesc_2_3@@6B@ 12133160     DOMNormalizer.obj
 0002:00030164       ??_7?$BaseRefVectorOf@VScope@InScopeNamespaces@DOMNormalizer@xercesc_2_3@@@xercesc_2_3@@6B@ 12133164     DOMNormalizer.obj
 0002:00030168       ??_7?$RefHashTableOfEnumerator@G@xercesc_2_3@@6B@ 12133168     DOMNormalizer.obj
 0002:00030178       ??_7?$XMLEnumerator@G@xercesc_2_3@@6B@ 12133178     DOMNormalizer.obj
 0002:00030188       ??_7DOMNotationImpl@xercesc_2_3@@6B@ 12133188     DOMNotationImpl.obj
 0002:00030238       ??_7DOMProcessingInstructionImpl@xercesc_2_3@@6B@ 12133238     DOMProcessingInstructionImpl.obj
 0002:000302e4       ??_7DOMRangeImpl@xercesc_2_3@@6B@ 121332e4     DOMRangeImpl.obj
 0002:00030358       ??_7DOMTextImpl@xercesc_2_3@@6B@ 12133358     DOMTextImpl.obj
 0002:0003042c       ??_7DOMTreeWalkerImpl@xercesc_2_3@@6B@ 1213342c     DOMTreeWalkerImpl.obj
 0002:00030468       ??_7DOMTypeInfoImpl@xercesc_2_3@@6B@ 12133468     DOMTypeInfoImpl.obj
 0002:000306bc       ??_7DOMWriterImpl@xercesc_2_3@@6B@ 121336bc     DOMWriterImpl.obj
 0002:000306f8       ??_7?$RefVectorOf@V?$RefHashTableOf@G@xercesc_2_3@@@xercesc_2_3@@6B@ 121336f8     DOMWriterImpl.obj
 0002:000306fc       ??_7?$BaseRefVectorOf@V?$RefHashTableOf@G@xercesc_2_3@@@xercesc_2_3@@6B@ 121336fc     DOMWriterImpl.obj
 0002:00030700       ??_7XSDElementNSImpl@xercesc_2_3@@6B@ 12133700     XSDElementNSImpl.obj
 0002:00030808       ??_7DocumentImpl@xercesc_2_3@@6B@ 12133808     AttrImpl.obj
 0002:0003092c       ??_7AttrImpl@xercesc_2_3@@6B@ 1213392c     AttrImpl.obj
 0002:000309f8       ??_7AttrMapImpl@xercesc_2_3@@6B@ 121339f8     AttrMapImpl.obj
 0002:00030a44       ??_7AttrNSImpl@xercesc_2_3@@6B@ 12133a44     AttrNSImpl.obj
 0002:00030b10       ??_7CDATASectionImpl@xercesc_2_3@@6B@ 12133b10     CDATASectionImpl.obj
 0002:00030bf4       ??_7CharacterDataImpl@xercesc_2_3@@6B@ 12133bf4     CharacterDataImpl.obj
 0002:00030ccc       ??_7ChildNode@xercesc_2_3@@6B@ 12133ccc     ChildNode.obj
 0002:00030d84       ??_7CommentImpl@xercesc_2_3@@6B@ 12133d84     CommentImpl.obj
 0002:00030e5c       ??_7DeepNodeListImpl@xercesc_2_3@@6B@ 12133e5c     DeepNodeListImpl.obj
 0002:00030e74       ??_7DocumentFragmentImpl@xercesc_2_3@@6B@ 12133e74     DocumentFragmentImpl.obj
 0002:00030f2c       ??_7?$RefVectorOf@VNodeIteratorImpl@xercesc_2_3@@@xercesc_2_3@@6B@ 12133f2c     DocumentImpl.obj
 0002:00030f30       ??_7?$BaseRefVectorOf@VNodeIteratorImpl@xercesc_2_3@@@xercesc_2_3@@6B@ 12133f30     DocumentImpl.obj
 0002:00030f34       ??_7?$RefVectorOf@VTreeWalkerImpl@xercesc_2_3@@@xercesc_2_3@@6B@ 12133f34     DocumentImpl.obj
 0002:00030f38       ??_7?$BaseRefVectorOf@VTreeWalkerImpl@xercesc_2_3@@@xercesc_2_3@@6B@ 12133f38     DocumentImpl.obj
 0002:00030f3c       ??_7?$RefVectorOf@VRangeImpl@xercesc_2_3@@@xercesc_2_3@@6B@ 12133f3c     DocumentImpl.obj
 0002:00030f40       ??_7?$BaseRefVectorOf@VRangeImpl@xercesc_2_3@@@xercesc_2_3@@6B@ 12133f40     DocumentImpl.obj
 0002:00030f44       ??_7DocumentTypeImpl@xercesc_2_3@@6B@ 12133f44     DocumentTypeImpl.obj
 0002:00031024       ??_7DOM_DOMException@xercesc_2_3@@6B@ 12134024     DOM_DOMException.obj
 0002:00031028       ?NNM_ELEMENT@DOM_NamedNodeMap@xercesc_2_3@@0GB 12134028     DOM_NamedNodeMap.obj
 0002:0003102a       ?NNM_OTHER@DOM_NamedNodeMap@xercesc_2_3@@0GB 1213402a     DOM_NamedNodeMap.obj
 0002:0003102c       ??_7DOM_NodeFilter@xercesc_2_3@@6B@ 1213402c     DOM_NodeFilter.obj
 0002:00031034       ??_7DOM_RangeException@xercesc_2_3@@6B@ 12134034     DOM_RangeException.obj
 0002:00031050       ??_7DOMParser@xercesc_2_3@@6BDocTypeHandler@1@@ 12134050     DOMParser.obj
 0002:00031094       ??_7DOMParser@xercesc_2_3@@6BXMLEntityHandler@1@@ 12134094     DOMParser.obj
 0002:000310ac       ??_7DOMParser@xercesc_2_3@@6BXMLErrorReporter@1@@ 121340ac     DOMParser.obj
 0002:000310b8       ??_7DOMParser@xercesc_2_3@@6BXMLDocumentHandler@1@@ 121340b8     DOMParser.obj
 0002:000310ec       ??_7ElementDefinitionImpl@xercesc_2_3@@6B@ 121340ec     ElementDefinitionImpl.obj
 0002:000311a4       ??_7ElementImpl@xercesc_2_3@@6B@ 121341a4     ElementImpl.obj
 0002:000312dc       ??_7ElementNSImpl@xercesc_2_3@@6B@ 121342dc     ElementNSImpl.obj
 0002:00031414       ??_7EntityImpl@xercesc_2_3@@6B@ 12134414     EntityImpl.obj
 0002:000314ec       ??_7EntityReferenceImpl@xercesc_2_3@@6B@ 121344ec     EntityReferenceImpl.obj
 0002:000315a4       ??_7NamedNodeMapImpl@xercesc_2_3@@6B@ 121345a4     NamedNodeMapImpl.obj
 0002:000315fc       ??_7NodeIDMap@xercesc_2_3@@6B@ 121345fc     NodeIDMap.obj
 0002:00031600       ?READONLY@NodeImpl@xercesc_2_3@@2GB 12134600     NodeImpl.obj
 0002:00031602       ?SYNCDATA@NodeImpl@xercesc_2_3@@2GB 12134602     NodeImpl.obj
 0002:00031604       ?SYNCCHILDREN@NodeImpl@xercesc_2_3@@2GB 12134604     NodeImpl.obj
 0002:00031606       ?OWNED@NodeImpl@xercesc_2_3@@2GB 12134606     NodeImpl.obj
 0002:00031608       ?FIRSTCHILD@NodeImpl@xercesc_2_3@@2GB 12134608     NodeImpl.obj
 0002:0003160a       ?SPECIFIED@NodeImpl@xercesc_2_3@@2GB 1213460a     NodeImpl.obj
 0002:0003160c       ?IGNORABLEWS@NodeImpl@xercesc_2_3@@2GB 1213460c     NodeImpl.obj
 0002:0003160e       ?SETVALUE@NodeImpl@xercesc_2_3@@2GB 1213460e     NodeImpl.obj
 0002:00031610       ?ID_ATTR@NodeImpl@xercesc_2_3@@2GB 12134610     NodeImpl.obj
 0002:00031612       ?USERDATA@NodeImpl@xercesc_2_3@@2GB 12134612     NodeImpl.obj
 0002:00031614       ?HASSTRING@NodeImpl@xercesc_2_3@@2GB 12134614     NodeImpl.obj
 0002:00031618       ??_7NodeImpl@xercesc_2_3@@6B@ 12134618     NodeImpl.obj
 0002:000316d0       ??_7NodeIteratorImpl@xercesc_2_3@@6B@ 121346d0     NodeIteratorImpl.obj
 0002:000316dc       ??_7NodeListImpl@xercesc_2_3@@6B@ 121346dc     NodeListImpl.obj
 0002:000316f0       ??_7NotationImpl@xercesc_2_3@@6B@ 121346f0     NotationImpl.obj
 0002:000317b8       ??_7ParentNode@xercesc_2_3@@6B@ 121347b8     ParentNode.obj
 0002:00031870       ??_7ProcessingInstructionImpl@xercesc_2_3@@6B@ 12134870     ProcessingInstructionImpl.obj
 0002:00031934       ??_7RangeImpl@xercesc_2_3@@6B@ 12134934     RangeImpl.obj
 0002:00031940       ??_7?$BaseRefVectorOf@VNodeImpl@xercesc_2_3@@@xercesc_2_3@@6B@ 12134940     RangeImpl.obj
 0002:00031944       ??_7?$RefVectorOf@VNodeImpl@xercesc_2_3@@@xercesc_2_3@@6B@ 12134944     RangeImpl.obj
 0002:00031948       ??_7RefCountedImpl@xercesc_2_3@@6B@ 12134948     RefCountedImpl.obj
 0002:00031954       ??_7TextImpl@xercesc_2_3@@6B@ 12134954     TextImpl.obj
 0002:00031a38       ??_7TreeWalkerImpl@xercesc_2_3@@6B@ 12134a38     TreeWalkerImpl.obj
 0002:00031a44       ??_7XMLDeclImpl@xercesc_2_3@@6B@ 12134a44     XMLDeclImpl.obj
 0002:00031b14       ??_7DOMException@xercesc_2_3@@6B@ 12134b14     DOMException.obj
 0002:00031b18       ??_7DOMRangeException@xercesc_2_3@@6B@ 12134b18     DOMRangeException.obj
 0002:00031b40       ??_7type_info@@6B@         12134b40     MSVCRT:ti_inst.obj
 0002:00031b48       ??_R1A@?0A@A@type_info@@8  12134b48     MSVCRT:ti_inst.obj
 0002:00031b60       ??_R2type_info@@8          12134b60     MSVCRT:ti_inst.obj
 0002:00031b68       ??_R3type_info@@8          12134b68     MSVCRT:ti_inst.obj
 0002:00031b78       ??_R4type_info@@6B@        12134b78     MSVCRT:ti_inst.obj
 0002:00032090       __CT??_R0?AVXMLException@xercesc_2_3@@@8??0XMLException@xercesc_2_3@@QAE@ABV01@@Z20 12135090     Win32PlatformUtils.obj
 0002:000320b0       __CT??_R0?AVXMLPlatformUtilsException@xercesc_2_3@@@8??0XMLPlatformUtilsException@xercesc_2_3@@QAE@ABV01@@Z20 121350b0     Win32PlatformUtils.obj
 0002:000320d0       __CTA2?AVXMLPlatformUtilsException@xercesc_2_3@@ 121350d0     Win32PlatformUtils.obj
 0002:000320e0       __TI2?AVXMLPlatformUtilsException@xercesc_2_3@@ 121350e0     Win32PlatformUtils.obj
 0002:000322b0       __CT??_R0?AVRuntimeException@xercesc_2_3@@@8??0RuntimeException@xercesc_2_3@@QAE@ABV01@@Z20 121352b0     Win32TransService.obj
 0002:000322d0       __CTA2?AVRuntimeException@xercesc_2_3@@ 121352d0     Win32TransService.obj
 0002:000322e0       __TI2?AVRuntimeException@xercesc_2_3@@ 121352e0     Win32TransService.obj
 0002:000323c0       __CT??_R0?AVTranscodingException@xercesc_2_3@@@8??0TranscodingException@xercesc_2_3@@QAE@ABV01@@Z20 121353c0     Win32TransService.obj
 0002:000323e0       __CTA2?AVTranscodingException@xercesc_2_3@@ 121353e0     Win32TransService.obj
 0002:000323f0       __TI2?AVTranscodingException@xercesc_2_3@@ 121353f0     Win32TransService.obj
 0002:00032400       __CT??_R0?AVNetAccessorException@xercesc_2_3@@@8??0NetAccessorException@xercesc_2_3@@QAE@ABV01@@Z20 12135400     BinHTTPURLInputStream.obj
 0002:00032420       __CTA2?AVNetAccessorException@xercesc_2_3@@ 12135420     BinHTTPURLInputStream.obj
 0002:00032430       __TI2?AVNetAccessorException@xercesc_2_3@@ 12135430     BinHTTPURLInputStream.obj
 0002:00032538       __CT??_R0?AVMalformedURLException@xercesc_2_3@@@8??0MalformedURLException@xercesc_2_3@@QAE@ABV01@@Z20 12135538     WinSockNetAccessor.obj
 0002:00032558       __CTA2?AVMalformedURLException@xercesc_2_3@@ 12135558     WinSockNetAccessor.obj
 0002:00032568       __TI2?AVMalformedURLException@xercesc_2_3@@ 12135568     WinSockNetAccessor.obj
 0002:00032680       __CT??_R0?AVArrayIndexOutOfBoundsException@xercesc_2_3@@@8??0ArrayIndexOutOfBoundsException@xercesc_2_3@@QAE@ABV01@@Z20 12135680     Match.obj
 0002:000326a0       __CTA2?AVArrayIndexOutOfBoundsException@xercesc_2_3@@ 121356a0     Match.obj
 0002:000326b0       __TI2?AVArrayIndexOutOfBoundsException@xercesc_2_3@@ 121356b0     Match.obj
 0002:00032ab0       __CT??_R0?AVParseException@xercesc_2_3@@@8??0ParseException@xercesc_2_3@@QAE@ABV01@@Z20 12135ab0     ParserForXMLSchema.obj
 0002:00032ad0       __CTA2?AVParseException@xercesc_2_3@@ 12135ad0     ParserForXMLSchema.obj
 0002:00032ae0       __TI2?AVParseException@xercesc_2_3@@ 12135ae0     ParserForXMLSchema.obj
 0002:00032b18       __CT??_R0?AVIllegalArgumentException@xercesc_2_3@@@8??0IllegalArgumentException@xercesc_2_3@@QAE@ABV01@@Z20 12135b18     RangeToken.obj
 0002:00032b38       __CTA2?AVIllegalArgumentException@xercesc_2_3@@ 12135b38     RangeToken.obj
 0002:00032b48       __TI2?AVIllegalArgumentException@xercesc_2_3@@ 12135b48     RangeToken.obj
 0002:00033268       __CT??_R0?AW4Codes@XMLErrs@xercesc_2_3@@@84 12136268     RegxParser.obj
 0002:00033288       __CTA1?AW4Codes@XMLErrs@xercesc_2_3@@ 12136288     RegxParser.obj
 0002:00033290       __TI1?AW4Codes@XMLErrs@xercesc_2_3@@ 12136290     RegxParser.obj
 0002:000333f0       __CT??_R0H@84              121363f0     RegxParser.obj
 0002:00033410       __CTA1H                    12136410     RegxParser.obj
 0002:00033418       __TI1H                     12136418     RegxParser.obj
 0002:000343d0       __CT??_R0?AVNumberFormatException@xercesc_2_3@@@8??0NumberFormatException@xercesc_2_3@@QAE@ABV01@@Z20 121373d0     XMLAbstractDoubleFloat.obj
 0002:000343f0       __CTA2?AVNumberFormatException@xercesc_2_3@@ 121373f0     XMLAbstractDoubleFloat.obj
 0002:00034400       __TI2?AVNumberFormatException@xercesc_2_3@@ 12137400     XMLAbstractDoubleFloat.obj
 0002:000345a0       __CT??_R0?AVSchemaDateTimeException@xercesc_2_3@@@8??0SchemaDateTimeException@xercesc_2_3@@QAE@ABV01@@Z20 121375a0     XMLDateTime.obj
 0002:000345c0       __CTA2?AVSchemaDateTimeException@xercesc_2_3@@ 121375c0     XMLDateTime.obj
 0002:000345d0       __TI2?AVSchemaDateTimeException@xercesc_2_3@@ 121375d0     XMLDateTime.obj
 0002:000350a0       __CT??_R0?AVUTFDataFormatException@xercesc_2_3@@@8??0UTFDataFormatException@xercesc_2_3@@QAE@ABV01@@Z20 121380a0     XMLUTF8Transcoder.obj
 0002:000350c0       __CTA2?AVUTFDataFormatException@xercesc_2_3@@ 121380c0     XMLUTF8Transcoder.obj
 0002:000350d0       __TI2?AVUTFDataFormatException@xercesc_2_3@@ 121380d0     XMLUTF8Transcoder.obj
 0002:000350e0       __CT??_R0?AVIOException@xercesc_2_3@@@8??0IOException@xercesc_2_3@@QAE@ABV01@@Z20 121380e0     LocalFileFormatTarget.obj
 0002:00035100       __CTA2?AVIOException@xercesc_2_3@@ 12138100     LocalFileFormatTarget.obj
 0002:00035110       __TI2?AVIOException@xercesc_2_3@@ 12138110     LocalFileFormatTarget.obj
 0002:00035400       __CT??_R0?AVNullPointerException@xercesc_2_3@@@8??0NullPointerException@xercesc_2_3@@QAE@ABV01@@Z20 12138400     Wrapper4DOMInputSource.obj
 0002:00035420       __CTA2?AVNullPointerException@xercesc_2_3@@ 12138420     Wrapper4DOMInputSource.obj
 0002:00035430       __TI2?AVNullPointerException@xercesc_2_3@@ 12138430     Wrapper4DOMInputSource.obj
 0002:00035808       __CT??_R0?AW4Codes@XMLValid@xercesc_2_3@@@84 12138808     XMLValidator.obj
 0002:00035828       __CTA1?AW4Codes@XMLValid@xercesc_2_3@@ 12138828     XMLValidator.obj
 0002:00035830       __TI1?AW4Codes@XMLValid@xercesc_2_3@@ 12138830     XMLValidator.obj
 0002:00035870       __CT??_R0?AVNoSuchElementException@xercesc_2_3@@@8??0NoSuchElementException@xercesc_2_3@@QAE@ABV01@@Z20 12138870     DGXMLScanner.obj
 0002:00035890       __CTA2?AVNoSuchElementException@xercesc_2_3@@ 12138890     DGXMLScanner.obj
 0002:000358a0       __TI2?AVNoSuchElementException@xercesc_2_3@@ 121388a0     DGXMLScanner.obj
 0002:00035c78       __CT??_R0?AVUnexpectedEOFException@xercesc_2_3@@@8??0UnexpectedEOFException@xercesc_2_3@@QAE@ABV01@@Z20 12138c78     DGXMLScanner.obj
 0002:00035c98       __CTA2?AVUnexpectedEOFException@xercesc_2_3@@ 12138c98     DGXMLScanner.obj
 0002:00035ca8       __TI2?AVUnexpectedEOFException@xercesc_2_3@@ 12138ca8     DGXMLScanner.obj
 0002:00036150       __CT??_R0?AVEmptyStackException@xercesc_2_3@@@8??0EmptyStackException@xercesc_2_3@@QAE@ABV01@@Z20 12139150     ElemStack.obj
 0002:00036170       __CTA2?AVEmptyStackException@xercesc_2_3@@ 12139170     ElemStack.obj
 0002:00036180       __TI2?AVEmptyStackException@xercesc_2_3@@ 12139180     ElemStack.obj
 0002:00037280       __CT??_R0?AVEndOfEntityException@xercesc_2_3@@@8??0EndOfEntityException@xercesc_2_3@@QAE@ABV01@@Z8 1213a280     ReaderMgr.obj
 0002:000372a0       __CTA1?AVEndOfEntityException@xercesc_2_3@@ 1213a2a0     ReaderMgr.obj
 0002:000372a8       __TI1?AVEndOfEntityException@xercesc_2_3@@ 1213a2a8     ReaderMgr.obj
 0002:00038a58       __CT??_R0?AVSAXException@xercesc_2_3@@@8??0SAXException@xercesc_2_3@@QAE@ABV01@@Z8 1213ba58     Dummy.obj
 0002:00038a78       __CT??_R0?AVSAXParseException@xercesc_2_3@@@8??0SAXParseException@xercesc_2_3@@QAE@ABV01@@Z24 1213ba78     Dummy.obj
 0002:00038a98       __CTA2?AVSAXParseException@xercesc_2_3@@ 1213ba98     Dummy.obj
 0002:00038aa8       __TI2?AVSAXParseException@xercesc_2_3@@ 1213baa8     Dummy.obj
 0002:00038e68       __CT??_R0?AVDOMException@xercesc_2_3@@@8??0DOMException@xercesc_2_3@@QAE@ABV01@@Z12 1213be68     DOMBuilderImpl.obj
 0002:00038e88       __CTA1?AVDOMException@xercesc_2_3@@ 1213be88     DOMBuilderImpl.obj
 0002:00038e90       __TI1?AVDOMException@xercesc_2_3@@ 1213be90     DOMBuilderImpl.obj
 0002:00039380       __CT??_R0?AVSAXNotRecognizedException@xercesc_2_3@@@8??0SAXNotRecognizedException@xercesc_2_3@@QAE@ABV01@@Z8 1213c380     SAX2XMLReaderImpl.obj
 0002:000393a0       __CTA2?AVSAXNotRecognizedException@xercesc_2_3@@ 1213c3a0     SAX2XMLReaderImpl.obj
 0002:000393b0       __CT??_R0?AVSAXNotSupportedException@xercesc_2_3@@@8??0SAXNotSupportedException@xercesc_2_3@@QAE@ABV01@@Z8 1213c3b0     SAX2XMLReaderImpl.obj
 0002:000393d0       __CTA2?AVSAXNotSupportedException@xercesc_2_3@@ 1213c3d0     SAX2XMLReaderImpl.obj
 0002:000393e0       __TI2?AVSAXNotRecognizedException@xercesc_2_3@@ 1213c3e0     SAX2XMLReaderImpl.obj
 0002:000393f0       __TI2?AVSAXNotSupportedException@xercesc_2_3@@ 1213c3f0     SAX2XMLReaderImpl.obj
 0002:0003a230       __CT??_R0?AVInvalidDatatypeFacetException@xercesc_2_3@@@8??0InvalidDatatypeFacetException@xercesc_2_3@@QAE@ABV01@@Z20 1213d230     AbstractNumericFacetValidator.obj
 0002:0003a250       __CTA2?AVInvalidDatatypeFacetException@xercesc_2_3@@ 1213d250     AbstractNumericFacetValidator.obj
 0002:0003a260       __TI2?AVInvalidDatatypeFacetException@xercesc_2_3@@ 1213d260     AbstractNumericFacetValidator.obj
 0002:0003a6c0       __CT??_R0?AVInvalidDatatypeValueException@xercesc_2_3@@@8??0InvalidDatatypeValueException@xercesc_2_3@@QAE@ABV01@@Z20 1213d6c0     AbstractNumericValidator.obj
 0002:0003a6e0       __CTA2?AVInvalidDatatypeValueException@xercesc_2_3@@ 1213d6e0     AbstractNumericValidator.obj
 0002:0003a6f0       __TI2?AVInvalidDatatypeValueException@xercesc_2_3@@ 1213d6f0     AbstractNumericValidator.obj
 0002:0003d9e0       __CT??_R0?AVXPathException@xercesc_2_3@@@8??0XPathException@xercesc_2_3@@QAE@ABV01@@Z20 121409e0     XercesXPath.obj
 0002:0003da00       __CTA2?AVXPathException@xercesc_2_3@@ 12140a00     XercesXPath.obj
 0002:0003da10       __TI2?AVXPathException@xercesc_2_3@@ 12140a10     XercesXPath.obj
 0002:0003f588       __CT??_R0?AW4ExceptionCodes@TraverseSchema@xercesc_2_3@@@84 12142588     TraverseSchema.obj
 0002:0003f5a8       __CTA1?AW4ExceptionCodes@TraverseSchema@xercesc_2_3@@ 121425a8     TraverseSchema.obj
 0002:0003f5b0       __TI1?AW4ExceptionCodes@TraverseSchema@xercesc_2_3@@ 121425b0     TraverseSchema.obj
 0002:00041b50       __CT??_R0?AVDOMRangeException@xercesc_2_3@@@8??0DOMRangeException@xercesc_2_3@@QAE@ABV01@@Z16 12144b50     DOMRangeImpl.obj
 0002:00041b70       __CTA2?AVDOMRangeException@xercesc_2_3@@ 12144b70     DOMRangeImpl.obj
 0002:00041b80       __TI2?AVDOMRangeException@xercesc_2_3@@ 12144b80     DOMRangeImpl.obj
 0002:00042190       __CT??_R0?AW4Codes@XMLDOMMsg@xercesc_2_3@@@84 12145190     DOMWriterImpl.obj
 0002:000421b0       __CTA1?AW4Codes@XMLDOMMsg@xercesc_2_3@@ 121451b0     DOMWriterImpl.obj
 0002:000421b8       __TI1?AW4Codes@XMLDOMMsg@xercesc_2_3@@ 121451b8     DOMWriterImpl.obj
 0002:00042488       __CT??_R0?AVDOM_DOMException@xercesc_2_3@@@8??0DOM_DOMException@xercesc_2_3@@QAE@ABV01@@Z12 12145488     AttrImpl.obj
 0002:000424a8       __CTA1?AVDOM_DOMException@xercesc_2_3@@ 121454a8     AttrImpl.obj
 0002:000424b0       __TI1?AVDOM_DOMException@xercesc_2_3@@ 121454b0     AttrImpl.obj
 0002:00045d38       __CT??_R0?AVDOM_RangeException@xercesc_2_3@@@8??0DOM_RangeException@xercesc_2_3@@QAE@ABV01@@Z16 12148d38     RangeImpl.obj
 0002:00045d58       __CTA2?AVDOM_RangeException@xercesc_2_3@@ 12148d58     RangeImpl.obj
 0002:00045d68       __TI2?AVDOM_RangeException@xercesc_2_3@@ 12148d68     RangeImpl.obj
 0002:000473a0       __IMPORT_DESCRIPTOR_KERNEL32 1214a3a0     kernel32:KERNEL32.dll
 0002:000473b4       __IMPORT_DESCRIPTOR_ADVAPI32 1214a3b4     advapi32:ADVAPI32.dll
 0002:000473c8       __IMPORT_DESCRIPTOR_MSVCRT 1214a3c8     MSVCRT:MSVCRT.dll
 0002:000473dc       __IMPORT_DESCRIPTOR_MSVCIRT 1214a3dc     msvcirt:MSVCIRT.dll
 0002:000473f0       __NULL_IMPORT_DESCRIPTOR   1214a3f0     kernel32:KERNEL32.dll
 0003:00000000       ___xc_a                    121b9000     MSVCRT:cinitexe.obj
 0003:00000060       ___xc_z                    121b9060     MSVCRT:cinitexe.obj
 0003:00000064       ___xi_a                    121b9064     MSVCRT:cinitexe.obj
 0003:00000068       ___xi_z                    121b9068     MSVCRT:cinitexe.obj
 0003:00000070       ??_R0?AVXMLException@xercesc_2_3@@@8 121b9070     Win32PlatformUtils.obj
 0003:00000098       ??_R0?AVXMLPlatformUtilsException@xercesc_2_3@@@8 121b9098     Win32PlatformUtils.obj
 0003:000000cc       ??_C@_0FJ@BODP@c?3?2xml4c_root?2xerces?9c?9src_2_3_0@ 121b90cc     Win32PlatformUtils.obj
 0003:00000128       ??_C@_06FFNI@IXUTIL?$AA@   121b9128     Win32MsgLoader.obj
 0003:00000130       ??_R0?AVRuntimeException@xercesc_2_3@@@8 121b9130     Win32TransService.obj
 0003:0000015c       ??_C@_0DB@IMPN@?4?4?2?4?4?2?4?4?2?4?4?2?4?4?2src?2xercesc?1util?1@ 121b915c     Win32TransService.obj
 0003:00000190       ??_C@_0BB@GMML@InternetEncoding?$AA@ 121b9190     Win32TransService.obj
 0003:000001a4       ??_C@_08GJEK@Codepage?$AA@ 121b91a4     Win32TransService.obj
 0003:000001b0       ??_C@_0BA@OCEI@AliasForCharset?$AA@ 121b91b0     Win32TransService.obj
 0003:000001c0       ??_C@_0BG@EHIG@MIME?2Database?2Charset?$AA@ 121b91c0     Win32TransService.obj
 0003:000001d8       ??_R0?AVTranscodingException@xercesc_2_3@@@8 121b91d8     Win32TransService.obj
 0003:00000208       ??_C@_0FK@CDNJ@c?3?2xml4c_root?2xerces?9c?9src_2_3_0@ 121b9208     Win32TransService.obj
 0003:00000268       ??_R0?AVNetAccessorException@xercesc_2_3@@@8 121b9268     BinHTTPURLInputStream.obj
 0003:00000298       ??_C@_0M@BGOH@closesocket?$AA@ 121b9298     BinHTTPURLInputStream.obj
 0003:000002a4       ??_C@_08DHEI@shutdown?$AA@ 121b92a4     BinHTTPURLInputStream.obj
 0003:000002b0       ??_C@_04NJFL@recv?$AA@     121b92b0     BinHTTPURLInputStream.obj
 0003:000002b8       ??_C@_04PJAD@send?$AA@     121b92b8     BinHTTPURLInputStream.obj
 0003:000002c0       ??_C@_07DHIJ@connect?$AA@  121b92c0     BinHTTPURLInputStream.obj
 0003:000002c8       ??_C@_06KDPK@socket?$AA@   121b92c8     BinHTTPURLInputStream.obj
 0003:000002d0       ??_C@_05MHGE@htons?$AA@    121b92d0     BinHTTPURLInputStream.obj
 0003:000002d8       ??_C@_0O@IOIG@gethostbyaddr?$AA@ 121b92d8     BinHTTPURLInputStream.obj
 0003:000002e8       ??_C@_09NHDB@inet_addr?$AA@ 121b92e8     BinHTTPURLInputStream.obj
 0003:000002f4       ??_C@_0O@BLIP@gethostbyname?$AA@ 121b92f4     BinHTTPURLInputStream.obj
 0003:00000304       ??_C@_0L@KLBB@WSACleanup?$AA@ 121b9304     BinHTTPURLInputStream.obj
 0003:00000310       ??_C@_0L@BKPI@WSAStartup?$AA@ 121b9310     BinHTTPURLInputStream.obj
 0003:0000031c       ??_C@_0GB@MNDM@c?3?2xml4c_root?2xerces?9c?9src_2_3_0@ 121b931c     BinHTTPURLInputStream.obj
 0003:00000380       ??_C@_07JDFI@WSOCK32?$AA@  121b9380     BinHTTPURLInputStream.obj
 0003:00000388       ??_C@_04EJJ@HTTP?$AA@      121b9388     BinHTTPURLInputStream.obj
 0003:00000390       ??_C@_02JJJH@?6?6?$AA@     121b9390     BinHTTPURLInputStream.obj
 0003:00000394       ??_C@_04FGNA@?$AN?6?$AN?6?$AA@ 121b9394     BinHTTPURLInputStream.obj
 0003:0000039c       ??_C@_01PKAG@?3?$AA@       121b939c     BinHTTPURLInputStream.obj
 0003:000003a0       ??_C@_06LGGD@Host?3?5?$AA@ 121b93a0     BinHTTPURLInputStream.obj
 0003:000003a8       ??_C@_0M@BGOJ@?5HTTP?11?40?$AN?6?$AA@ 121b93a8     BinHTTPURLInputStream.obj
 0003:000003b4       ??_C@_01PKMN@?$DP?$AA@     121b93b4     BinHTTPURLInputStream.obj
 0003:000003b8       ??_C@_04PJJL@GET?5?$AA@    121b93b8     BinHTTPURLInputStream.obj
 0003:000003c0       ??_R0?AVMalformedURLException@xercesc_2_3@@@8 121b93c0     WinSockNetAccessor.obj
 0003:000003f0       ??_C@_0FO@JLCO@c?3?2xml4c_root?2xerces?9c?9src_2_3_0@ 121b93f0     WinSockNetAccessor.obj
 0003:00000450       ??_C@_0CP@JDCL@?4?4?2?4?4?2?4?4?2?4?4?2?4?4?2src?2xercesc?1util?1@ 121b9450     ASCIIRangeFactory.obj
 0003:00000480       ??_C@_0DI@JHFM@?4?4?2?4?4?2?4?4?2?4?4?2?4?4?2src?2xercesc?1util?1@ 121b9480     ConditionToken.obj
 0003:000004b8       ??_C@_0CP@HPDD@?4?4?2?4?4?2?4?4?2?4?4?2?4?4?2src?2xercesc?1util?1@ 121b94b8     Match.obj
 0003:000004e8       ??_R0?AVArrayIndexOutOfBoundsException@xercesc_2_3@@@8 121b94e8     Match.obj
 0003:00000524       ??_C@_0CM@JAIE@?4?4?2?4?4?2?4?4?2?4?4?2?4?4?2src?2xercesc?1util?1@ 121b9524     Op.obj
 0003:00000550       ??_C@_0DO@JEFD@c?3?2xml4c_root?2xerces?9c?9src_2_3_0@ 121b9550     Op.obj
 0003:00000590       ??_C@_0DC@MEPO@?4?4?2?4?4?2?4?4?2?4?4?2?4?4?2src?2xercesc?1util?1@ 121b9590     Op.obj
 0003:000005c8       ??_R0?AVParseException@xercesc_2_3@@@8 121b95c8     ParserForXMLSchema.obj
 0003:000005f4       ??_C@_0EO@CBHP@c?3?2xml4c_root?2xerces?9c?9src_2_3_0@ 121b95f4     ParserForXMLSchema.obj
 0003:00000648       ??_R0?AVIllegalArgumentException@xercesc_2_3@@@8 121b9648     RangeToken.obj
 0003:0000067c       ??_C@_0EG@NPAP@c?3?2xml4c_root?2xerces?9c?9src_2_3_0@ 121b967c     RangeToken.obj
 0003:000006c4       ??_C@_0EJ@OKNC@c?3?2xml4c_root?2xerces?9c?9src_2_3_0@ 121b96c4     RangeTokenMap.obj
 0003:00000710       ??_C@_0EN@BPHB@c?3?2xml4c_root?2xerces?9c?9src_2_3_0@ 121b9710     RegularExpression.obj
 0003:00000760       ??_C@_0EG@FGHG@c?3?2xml4c_root?2xerces?9c?9src_2_3_0@ 121b9760     RegxParser.obj
 0003:000007a8       ??_R0?AW4Codes@XMLErrs@xercesc_2_3@@@8 121b97a8     RegxParser.obj
 0003:000007d8       ??_R0H@8                   121b97d8     RegxParser.obj
 0003:000007e4       ??_C@_03HHKO@?$CFs?6?$AA@  121b97e4     DefaultPanicHandler.obj
 0003:000007e8       ??_C@_0DD@FBDC@?4?4?2?4?4?2?4?4?2?4?4?2?4?4?2src?2xercesc?1util?1@ 121b97e8     EncodingValidator.obj
 0003:0000081c       ??_C@_0P@BFFG@Unknown?5reason?$AA@ 121b981c     PanicHandler.obj
 0003:0000082c       ??_C@_0CG@NDGG@Cannot?5initialize?5the?5system?5or?5@ 121b982c     PanicHandler.obj
 0003:00000854       ??_C@_0CD@KFKN@Cannot?5synchronize?5system?5or?5mut@ 121b9854     PanicHandler.obj
 0003:00000878       ??_C@_0BL@HHGI@Cannot?5load?5message?5domain?$AA@ 121b9878     PanicHandler.obj
 0003:00000894       ??_C@_0BH@NKGC@Unknown?5message?5domain?$AA@ 121b9894     PanicHandler.obj
 0003:000008ac       ??_C@_0CA@LBJK@Could?5not?5find?5the?5xerces?9c?5DLL?$AA@ 121b98ac     PanicHandler.obj
 0003:000008cc       ??_C@_0CM@CIGD@Could?5not?5load?5a?5local?5code?5page@ 121b98cc     PanicHandler.obj
 0003:000008f8       ??_C@_0CF@CLOA@Could?5not?5load?5a?5transcoding?5ser@ 121b98f8     PanicHandler.obj
 0003:00000920       ?fgMemMgrAdopted@XMLPlatformUtils@xercesc_2_3@@0_NA 121b9920     PlatformUtils.obj
 0003:00000924       ??_C@_0EE@MFDA@c?3?2xml4c_root?2xerces?9c?9src_2_3_0@ 121b9924     PlatformUtils.obj
 0003:00000968       ??_C@_0EB@GJFO@c?3?2xml4c_root?2xerces?9c?9src_2_3_0@ 121b9968     StringPool.obj
 0003:000009ac       ??_C@_0EM@FPKH@c?3?2xml4c_root?2xerces?9c?9src_2_3_0@ 121b99ac     XML256TableTranscoder.obj
 0003:000009f8       ??_C@_0EJ@NLIO@c?3?2xml4c_root?2xerces?9c?9src_2_3_0@ 121b99f8     XML88591Transcoder.obj
 0003:00000a48       ??_R0?AVNumberFormatException@xercesc_2_3@@@8 121b9a48     XMLAbstractDoubleFloat.obj
 0003:00000a78       ??_C@_0EN@KAEN@c?3?2xml4c_root?2xerces?9c?9src_2_3_0@ 121b9a78     XMLAbstractDoubleFloat.obj
 0003:00000ac8       ??_C@_0EJ@EAMG@c?3?2xml4c_root?2xerces?9c?9src_2_3_0@ 121b9ac8     XMLASCIITranscoder.obj
 0003:00000b14       ??_C@_0EE@GMJN@c?3?2xml4c_root?2xerces?9c?9src_2_3_0@ 121b9b14     XMLBigDecimal.obj
 0003:00000b58       ??_C@_0EE@CABF@c?3?2xml4c_root?2xerces?9c?9src_2_3_0@ 121b9b58     XMLBigInteger.obj
 0003:00000b9c       ?fgCharCharsTable1_0@XMLChar1_0@xercesc_2_3@@0PAEA 121b9b9c     XMLChar.obj
 0003:00010b9c       ?fgCharCharsTable1_1@XMLChar1_1@xercesc_2_3@@0PAEA 121c9b9c     XMLChar.obj
 0003:00020ba0       ??_R0?AVSchemaDateTimeException@xercesc_2_3@@@8 121d9ba0     XMLDateTime.obj
 0003:00020bd4       ??_C@_0DA@JBEC@?4?4?2?4?4?2?4?4?2?4?4?2?4?4?2src?2xercesc?1util?1@ 121d9bd4     XMLDateTime.obj
 0003:00020c04       ??_C@_0EC@NDON@c?3?2xml4c_root?2xerces?9c?9src_2_3_0@ 121d9c04     XMLDateTime.obj
 0003:00020c48       ??_C@_0EA@PKNB@c?3?2xml4c_root?2xerces?9c?9src_2_3_0@ 121d9c48     XMLDouble.obj
 0003:00020c88       ??_C@_0DP@OPOL@c?3?2xml4c_root?2xerces?9c?9src_2_3_0@ 121d9c88     XMLFloat.obj
 0003:00020cc8       ?fLanguage@XMLMsgLoader@xercesc_2_3@@0PAGA 121d9cc8     XMLMsgLoader.obj
 0003:00020ce0       ??_C@_0EA@ENHB@c?3?2xml4c_root?2xerces?9c?9src_2_3_0@ 121d9ce0     XMLString.obj
 0003:00020d20       ??_C@_0EH@JANK@c?3?2xml4c_root?2xerces?9c?9src_2_3_0@ 121d9d20     XMLUCSTranscoder.obj
 0003:00020d68       ??_C@_0DN@GFFM@c?3?2xml4c_root?2xerces?9c?9src_2_3_0@ 121d9d68     XMLUri.obj
 0003:00020dcc       ??_C@_0DN@PFEC@c?3?2xml4c_root?2xerces?9c?9src_2_3_0@ 121d9dcc     XMLURL.obj
 0003:00020e10       ??_R0?AVUTFDataFormatException@xercesc_2_3@@@8 121d9e10     XMLUTF8Transcoder.obj
 0003:00020e44       ??_C@_0EI@MCEC@c?3?2xml4c_root?2xerces?9c?9src_2_3_0@ 121d9e44     XMLUTF8Transcoder.obj
 0003:00020e90       ??_R0?AVIOException@xercesc_2_3@@@8 121d9e90     LocalFileFormatTarget.obj
 0003:00020eb8       ??_C@_0FB@PIKH@c?3?2xml4c_root?2xerces?9c?9src_2_3_0@ 121d9eb8     LocalFileFormatTarget.obj
 0003:00020f0c       ??_C@_05NOKM@stdin?$AA@    121d9f0c     StdInInputSource.obj
 0003:00020f18       ??_R0?AVNullPointerException@xercesc_2_3@@@8 121d9f18     Wrapper4DOMInputSource.obj
 0003:00020f48       ??_C@_0FC@CKDI@c?3?2xml4c_root?2xerces?9c?9src_2_3_0@ 121d9f48     Wrapper4DOMInputSource.obj
 0003:00020f9c       ??_C@_0EP@FHNK@c?3?2xml4c_root?2xerces?9c?9src_2_3_0@ 121d9f9c     Wrapper4InputSource.obj
 0003:00020fec       ??_C@_0EF@LFEJ@c?3?2xml4c_root?2xerces?9c?9src_2_3_0@ 121d9fec     XMLAttDef.obj
 0003:00021034       ??_C@_0EI@FBJI@c?3?2xml4c_root?2xerces?9c?9src_2_3_0@ 121da034     XMLBufferMgr.obj
 0003:0002107c       ??_C@_0EI@GBMA@c?3?2xml4c_root?2xerces?9c?9src_2_3_0@ 121da07c     XMLFormatter.obj
 0003:000210e4       ??_C@_0EJ@HKMB@c?3?2xml4c_root?2xerces?9c?9src_2_3_0@ 121da0e4     XMLRecognizer.obj
 0003:00021130       ??_R0?AW4Codes@XMLValid@xercesc_2_3@@@8 121da130     XMLValidator.obj
 0003:00021160       ??_R0?AVNoSuchElementException@xercesc_2_3@@@8 121da160     DGXMLScanner.obj
 0003:00021194       ??_C@_0CN@GFNC@?4?4?2?4?4?2?4?4?2?4?4?2?4?4?2src?2xercesc?1util?1@ 121da194     DGXMLScanner.obj
 0003:000211c4       ??_C@_0EH@JEKI@c?3?2xml4c_root?2xerces?9c?9src_2_3_0@ 121da1c4     DGXMLScanner.obj
 0003:00021210       ??_R0?AVEndOfEntityException@xercesc_2_3@@@8 121da210     DGXMLScanner.obj
 0003:00021240       ??_R0?AVUnexpectedEOFException@xercesc_2_3@@@8 121da240     DGXMLScanner.obj
 0003:00021274       ??_C@_0DA@CACO@?4?4?2?4?4?2?4?4?2?4?4?2?4?4?2src?2xercesc?1util?1@ 121da274     DGXMLScanner.obj
 0003:000212a8       ??_R0?AVEmptyStackException@xercesc_2_3@@@8 121da2a8     ElemStack.obj
 0003:000212d8       ??_C@_0EE@LDDC@c?3?2xml4c_root?2xerces?9c?9src_2_3_0@ 121da2d8     ElemStack.obj
 0003:0002131c       ??_C@_0DG@GENG@?4?4?2?4?4?2?4?4?2?4?4?2?4?4?2src?2xercesc?1util?1@ 121da31c     IGXMLScanner.obj
 0003:00021354       ??_C@_0DF@DOIO@?4?4?2?4?4?2?4?4?2?4?4?2?4?4?2src?2xercesc?1util?1@ 121da354     IGXMLScanner.obj
 0003:0002138c       ??_C@_0CP@NCIM@?4?4?2?4?4?2?4?4?2?4?4?2?4?4?2src?2xercesc?1util?1@ 121da38c     IGXMLScanner.obj
 0003:000213bc       ??_C@_0EH@DMHF@c?3?2xml4c_root?2xerces?9c?9src_2_3_0@ 121da3bc     IGXMLScanner.obj
 0003:00021404       ??_C@_0EI@LHNI@c?3?2xml4c_root?2xerces?9c?9src_2_3_0@ 121da404     IGXMLScanner2.obj
 0003:0002144c       ??_C@_0CN@LDGJ@?4?4?2?4?4?2?4?4?2?4?4?2?4?4?2src?2xercesc?1util?1@ 121da44c     ReaderMgr.obj
 0003:0002147c       ??_C@_0EE@PDPJ@c?3?2xml4c_root?2xerces?9c?9src_2_3_0@ 121da47c     ReaderMgr.obj
 0003:000214c0       ??_C@_0EH@GNMP@c?3?2xml4c_root?2xerces?9c?9src_2_3_0@ 121da4c0     SGXMLScanner.obj
 0003:00021508       ??_C@_0EH@CIGF@c?3?2xml4c_root?2xerces?9c?9src_2_3_0@ 121da508     WFXMLScanner.obj
 0003:00021550       ??_C@_0EE@JAMI@c?3?2xml4c_root?2xerces?9c?9src_2_3_0@ 121da550     XMLReader.obj
 0003:00021594       ??_C@_0EF@PKHK@c?3?2xml4c_root?2xerces?9c?9src_2_3_0@ 121da594     XMLScanner.obj
 0003:000215dc       ??_C@_09NHPD@in?5prolog?$AA@ 121da5dc     XMLScanner.obj
 0003:000215e8       ??_R0?AVSAXException@xercesc_2_3@@@8 121da5e8     Dummy.obj
 0003:00021610       ??_R0?AVSAXParseException@xercesc_2_3@@@8 121da610     Dummy.obj
 0003:0002163c       ??_C@_0EL@HNBC@c?3?2xml4c_root?2xerces?9c?9src_2_3_0@ 121da63c     AbstractDOMParser.obj
 0003:00021688       ??_R0?AVDOMException@xercesc_2_3@@@8 121da688     DOMBuilderImpl.obj
 0003:000216b0       ??_C@_0EI@EILA@c?3?2xml4c_root?2xerces?9c?9src_2_3_0@ 121da6b0     DOMBuilderImpl.obj
 0003:000216f8       ??_C@_0EL@KNID@c?3?2xml4c_root?2xerces?9c?9src_2_3_0@ 121da6f8     SAX2XMLReaderImpl.obj
 0003:00021748       ??_R0?AVSAXNotRecognizedException@xercesc_2_3@@@8 121da748     SAX2XMLReaderImpl.obj
 0003:00021780       ??_R0?AVSAXNotSupportedException@xercesc_2_3@@@8 121da780     SAX2XMLReaderImpl.obj
 0003:000217b4       ??_C@_0BA@IJFN@Unknown?5Feature?$AA@ 121da7b4     SAX2XMLReaderImpl.obj
 0003:000217c4       ??_C@_0DE@KAIE@Feature?5modification?5is?5not?5supp@ 121da7c4     SAX2XMLReaderImpl.obj
 0003:000217f8       ??_C@_0BB@MDM@Unknown?5Property?$AA@ 121da7f8     SAX2XMLReaderImpl.obj
 0003:0002180c       ??_C@_0DF@CGAC@Property?5modification?5is?5not?5sup@ 121da80c     SAX2XMLReaderImpl.obj
 0003:00021844       ??_C@_0ED@IACG@c?3?2xml4c_root?2xerces?9c?9src_2_3_0@ 121da844     SAXParser.obj
 0003:00021888       ??_C@_0EJ@EIFN@c?3?2xml4c_root?2xerces?9c?9src_2_3_0@ 121da888     XercesDOMParser.obj
 0003:000218d4       ??_C@_0FD@FGMC@c?3?2xml4c_root?2xerces?9c?9src_2_3_0@ 121da8d4     AllContentModel.obj
 0003:00021928       ??_C@_05ONKL@CMAny?$AA@    121da928     CMAny.obj
 0003:00021930       ??_C@_0EJ@PFAA@c?3?2xml4c_root?2xerces?9c?9src_2_3_0@ 121da930     CMAny.obj
 0003:0002197c       ??_C@_0DM@NIED@?4?4?2?4?4?2?4?4?2?4?4?2?4?4?2src?2xercesc?1valid@ 121da97c     CMAny.obj
 0003:000219b8       ??_C@_0EO@NKKC@c?3?2xml4c_root?2xerces?9c?9src_2_3_0@ 121da9b8     CMBinaryOp.obj
 0003:00021a08       ??_C@_0EN@DOJL@c?3?2xml4c_root?2xerces?9c?9src_2_3_0@ 121daa08     CMUnaryOp.obj
 0003:00021a58       ??_C@_0FN@PBCH@c?3?2xml4c_root?2xerces?9c?9src_2_3_0@ 121daa58     ContentLeafNameTypeVector.obj
 0003:00021ab8       ??_C@_0EB@DCJN@?4?4?2?4?4?2?4?4?2?4?4?2?4?4?2src?2xercesc?1valid@ 121daab8     DFAContentModel.obj
 0003:00021afc       ??_C@_0FD@GLNN@c?3?2xml4c_root?2xerces?9c?9src_2_3_0@ 121daafc     DFAContentModel.obj
 0003:00021b50       ??_C@_0FD@GMOI@c?3?2xml4c_root?2xerces?9c?9src_2_3_0@ 121dab50     GrammarResolver.obj
 0003:00021ba4       ??_C@_0FF@ILND@c?3?2xml4c_root?2xerces?9c?9src_2_3_0@ 121daba4     MixedContentModel.obj
 0003:00021bfc       ??_C@_0FG@CIFB@c?3?2xml4c_root?2xerces?9c?9src_2_3_0@ 121dabfc     SimpleContentModel.obj
 0003:00021c58       ??_R0?AVInvalidDatatypeFacetException@xercesc_2_3@@@8 121dac58     AbstractNumericFacetValidator.obj
 0003:00021c90       ??_C@_0GD@BFAE@c?3?2xml4c_root?2xerces?9c?9src_2_3_0@ 121dac90     AbstractNumericFacetValidator.obj
 0003:00021cf8       ??_R0?AVInvalidDatatypeValueException@xercesc_2_3@@@8 121dacf8     AbstractNumericValidator.obj
 0003:00021d30       ??_C@_0FO@IBJN@c?3?2xml4c_root?2xerces?9c?9src_2_3_0@ 121dad30     AbstractNumericValidator.obj
 0003:00021d90       ??_C@_0FN@DAJF@c?3?2xml4c_root?2xerces?9c?9src_2_3_0@ 121dad90     AbstractStringValidator.obj
 0003:00021df0       ??_C@_0GE@GIME@c?3?2xml4c_root?2xerces?9c?9src_2_3_0@ 121dadf0     AnySimpleTypeDatatypeValidator.obj
 0003:00021e54       ??_C@_0FN@COIB@c?3?2xml4c_root?2xerces?9c?9src_2_3_0@ 121dae54     AnyURIDatatypeValidator.obj
 0003:00021eb4       ??_C@_0GD@OMDH@c?3?2xml4c_root?2xerces?9c?9src_2_3_0@ 121daeb4     Base64BinaryDatatypeValidator.obj
 0003:00021f18       ??_C@_0M@NIGK@enumeration?$AA@ 121daf18     BooleanDatatypeValidator.obj
 0003:00021f24       ??_C@_0FO@KGOA@c?3?2xml4c_root?2xerces?9c?9src_2_3_0@ 121daf24     BooleanDatatypeValidator.obj
 0003:00021f84       ??_C@_0FH@DGDC@c?3?2xml4c_root?2xerces?9c?9src_2_3_0@ 121daf84     DateTimeValidator.obj
 0003:00021fdc       ??_C@_0FO@JHBG@c?3?2xml4c_root?2xerces?9c?9src_2_3_0@ 121dafdc     DecimalDatatypeValidator.obj
 0003:0002203c       ??_C@_0FN@GHJN@c?3?2xml4c_root?2xerces?9c?9src_2_3_0@ 121db03c     DoubleDatatypeValidator.obj
 0003:0002209c       ??_C@_0FN@JOMD@c?3?2xml4c_root?2xerces?9c?9src_2_3_0@ 121db09c     ENTITYDatatypeValidator.obj
 0003:000220fc       ??_C@_0FM@LFOO@c?3?2xml4c_root?2xerces?9c?9src_2_3_0@ 121db0fc     FloatDatatypeValidator.obj
 0003:00022158       ??_C@_0GA@CPNL@c?3?2xml4c_root?2xerces?9c?9src_2_3_0@ 121db158     HexBinaryDatatypeValidator.obj
 0003:000221b8       ??_C@_0FJ@MAGB@c?3?2xml4c_root?2xerces?9c?9src_2_3_0@ 121db1b8     IDDatatypeValidator.obj
 0003:00022214       ??_C@_0FM@MNGI@c?3?2xml4c_root?2xerces?9c?9src_2_3_0@ 121db214     IDREFDatatypeValidator.obj
 0003:00022270       ??_C@_0FL@CLEI@c?3?2xml4c_root?2xerces?9c?9src_2_3_0@ 121db270     ListDatatypeValidator.obj
 0003:000222cc       ??_C@_0FL@BJEF@c?3?2xml4c_root?2xerces?9c?9src_2_3_0@ 121db2cc     NameDatatypeValidator.obj
 0003:00022328       ??_C@_0FN@LLPN@c?3?2xml4c_root?2xerces?9c?9src_2_3_0@ 121db328     NCNameDatatypeValidator.obj
 0003:00022388       ??_C@_0FP@DMJD@c?3?2xml4c_root?2xerces?9c?9src_2_3_0@ 121db388     NOTATIONDatatypeValidator.obj
 0003:000223e8       ??_C@_0FM@CGJL@c?3?2xml4c_root?2xerces?9c?9src_2_3_0@ 121db3e8     QNameDatatypeValidator.obj
 0003:00022444       ??_C@_0FN@HCNH@c?3?2xml4c_root?2xerces?9c?9src_2_3_0@ 121db444     StringDatatypeValidator.obj
 0003:000224a4       ??_C@_0FM@OKCE@c?3?2xml4c_root?2xerces?9c?9src_2_3_0@ 121db4a4     UnionDatatypeValidator.obj
 0003:00022500       ??_C@_0EP@NEFM@c?3?2xml4c_root?2xerces?9c?9src_2_3_0@ 121db500     DTDElementDecl.obj
 0003:00022550       ??_C@_0EL@BBDF@c?3?2xml4c_root?2xerces?9c?9src_2_3_0@ 121db550     DTDScanner.obj
 0003:0002259c       ??_C@_0EN@NKBC@c?3?2xml4c_root?2xerces?9c?9src_2_3_0@ 121db59c     DTDValidator.obj
 0003:000225f0       ??_R0?AVXPathException@xercesc_2_3@@@8 121db5f0     XercesXPath.obj
 0003:0002261c       ??_C@_0FI@FLIN@c?3?2xml4c_root?2xerces?9c?9src_2_3_0@ 121db61c     XercesXPath.obj
 0003:00022674       ??_C@_0FJ@EGPE@c?3?2xml4c_root?2xerces?9c?9src_2_3_0@ 121db674     XPathMatcher.obj
 0003:000226d0       ??_C@_0FD@ICOF@c?3?2xml4c_root?2xerces?9c?9src_2_3_0@ 121db6d0     ComplexTypeInfo.obj
 0003:00022724       ?fgElemAttTable@GeneralAttributeCheck@xercesc_2_3@@0PAY0CC@GA 121db724     GeneralAttributeCheck.obj
 0003:0002346c       ?fAttNames@GeneralAttributeCheck@xercesc_2_3@@0PAPBGA 121dc46c     GeneralAttributeCheck.obj
 0003:000234f4       ??_C@_0FC@IFNE@c?3?2xml4c_root?2xerces?9c?9src_2_3_0@ 121dc4f4     NamespaceScope.obj
 0003:00023548       ??_C@_0FE@OLKP@c?3?2xml4c_root?2xerces?9c?9src_2_3_0@ 121dc548     SchemaAttDefList.obj
 0003:0002359c       ??_C@_0FF@GABI@c?3?2xml4c_root?2xerces?9c?9src_2_3_0@ 121dc59c     SchemaElementDecl.obj
 0003:000235f4       ??_C@_0FD@GIJ@c?3?2xml4c_root?2xerces?9c?9src_2_3_0@ 121dc5f4     SchemaValidator.obj
 0003:00023648       ??_C@_0FP@IIHP@c?3?2xml4c_root?2xerces?9c?9src_2_3_0@ 121dc648     SubstitutionGroupComparator.obj
 0003:000236a8       ?fgIdentityConstraints@xercesc_2_3@@3PAPBGA 121dc6a8     TraverseSchema.obj
 0003:000236b8       ??_R0?AW4ExceptionCodes@TraverseSchema@xercesc_2_3@@@8 121dc6b8     TraverseSchema.obj
 0003:000236f4       ??_C@_0FC@LFHM@c?3?2xml4c_root?2xerces?9c?9src_2_3_0@ 121dc6f4     TraverseSchema.obj
 0003:00023748       ??_C@_0CN@FACH@?4?4?2?4?4?2?4?4?2?4?4?2?4?4?2src?2xercesc?1util?1@ 121dc748     DOMDocumentImpl.obj
 0003:00023778       ??_C@_0EK@OOPP@c?3?2xml4c_root?2xerces?9c?9src_2_3_0@ 121dc778     DOMDocumentImpl.obj
 0003:000237c4       ??_C@_0DK@LODD@?4?4?2?4?4?2?4?4?2?4?4?2?4?4?2src?2xercesc?1dom?1i@ 121dc7c4     DOMDocumentImpl.obj
 0003:00023800       ??_C@_0EH@LDJB@c?3?2xml4c_root?2xerces?9c?9src_2_3_0@ 121dc800     DOMNodeIDMap.obj
 0003:00023848       ??_R0?AVDOMRangeException@xercesc_2_3@@@8 121dc848     DOMRangeImpl.obj
 0003:00023878       ??_R0?AW4Codes@XMLDOMMsg@xercesc_2_3@@@8 121dc878     DOMWriterImpl.obj
 0003:000238a8       ??_R0?AVDOM_DOMException@xercesc_2_3@@@8 121dc8a8     AttrImpl.obj
 0003:000238d4       ??_C@_01HMO@?$CC?$AA@      121dc8d4     AttrImpl.obj
 0003:000238d8       ??_C@_02EBGB@?$DN?$CC?$AA@ 121dc8d8     AttrImpl.obj
 0003:000238dc       ??_C@_0P@CKBI@?$CDcdata?9section?$AA@ 121dc8dc     CDATASectionImpl.obj
 0003:000238ec       ??_C@_08JMOF@?$CDcomment?$AA@ 121dc8ec     CommentImpl.obj
 0003:000238f8       ??_C@_01FDHG@?$CK?$AA@     121dc8f8     DeepNodeListImpl.obj
 0003:000238fc       ??_C@_0BD@CBIP@?$CDdocument?9fragment?$AA@ 121dc8fc     DocumentFragmentImpl.obj
 0003:00023910       ??_C@_09FGFB@?$CDdocument?$AA@ 121dc910     DocumentImpl.obj
 0003:0002391c       ??_C@_05MCCK@Range?$AA@    121dc91c     DOM_DOMImplementation.obj
 0003:00023924       ??_C@_09LNFH@Traversal?$AA@ 121dc924     DOM_DOMImplementation.obj
 0003:00023930       ??_C@_04BNDI@Core?$AA@     121dc930     DOM_DOMImplementation.obj
 0003:00023938       ??_C@_03DMKA@XML?$AA@      121dc938     DOM_DOMImplementation.obj
 0003:0002393c       ??_C@_03CLPL@2?40?$AA@     121dc93c     DOM_DOMImplementation.obj
 0003:00023940       ??_C@_03NNMA@1?40?$AA@     121dc940     DOM_DOMImplementation.obj
 0003:00023944       ??_C@_0BCM@GHMG@DOM?5reference?5counted?5memory?5all@ 121dc944     DomMemDebug.obj
 0003:00023a70       ??_C@_01BJG@?6?$AA@        121dca70     DomMemDebug.obj
 0003:00023a74       ??_C@_0BF@JFNJ@?5?5?5?$CFd?5NamedNodeMaps?4?$AA@ 121dca74     DomMemDebug.obj
 0003:00023a8c       ??_C@_0BB@IEON@?5?5?5?$CFd?5NodeImpls?4?$AA@ 121dca8c     DomMemDebug.obj
 0003:00023aa0       ??_C@_0BF@IGHB@?5?5?5?$CFd?5StringBuffers?4?$AA@ 121dcaa0     DomMemDebug.obj
 0003:00023ab8       ??_C@_0BF@HJNG@?5?5?5?$CFd?5StringHandles?4?$AA@ 121dcab8     DomMemDebug.obj
 0003:00023ad0       ??_C@_0EK@CGEP@c?3?2xml4c_root?2xerces?9c?9src_2_3_0@ 121dcad0     DOMParser.obj
 0003:00023b1c       ??_C@_0EK@KIDL@c?3?2xml4c_root?2xerces?9c?9src_2_3_0@ 121dcb1c     DOMString.obj
 0003:00023b68       ??_C@_0EK@DLGJ@c?3?2xml4c_root?2xerces?9c?9src_2_3_0@ 121dcb68     NodeIDMap.obj
 0003:00023bb4       ??_C@_01KHLB@?$FL?$AA@     121dcbb4     NodeImpl.obj
 0003:00023bb8       ??_C@_02HFBK@?3?5?$AA@     121dcbb8     NodeImpl.obj
 0003:00023bbc       ??_C@_01FIMD@?$FN?$AA@     121dcbbc     NodeImpl.obj
 0003:00023bc0       ??_C@_05GJOJ@xmlns?$AA@    121dcbc0     NodeImpl.obj
 0003:00023bc8       ??_C@_0BO@DOBD@http?3?1?1www?4w3?4org?12000?1xmlns?1?$AA@ 121dcbc8     NodeImpl.obj
 0003:00023be8       ??_C@_03PJMH@xml?$AA@      121dcbe8     NodeImpl.obj
 0003:00023bec       ??_C@_0CF@JEIF@http?3?1?1www?4w3?4org?1XML?11998?1names@ 121dcbec     NodeImpl.obj
 0003:00023c18       ??_R0?AVDOM_RangeException@xercesc_2_3@@@8 121dcc18     RangeImpl.obj
 0003:00023c48       ??_C@_05FDFO@?$CDtext?$AA@ 121dcc48     TextImpl.obj
 0003:00023c50       ??_C@_08PCJH@?$CDxmldecl?$AA@ 121dcc50     XMLDeclImpl.obj
 0003:00023c60       ??_R0?AVtype_info@@@8      121dcc60     MSVCRT:ti_inst.obj
 0003:00023c80       ??_C@_00A@?$AA@            121dcc80     Win32PlatformUtils.obj
 0003:00023c88       ?globalModuleHandle@@3PAUHINSTANCE__@@A 121dcc88     Win32MsgLoader.obj
 0003:00023c8c       ?gWinsockLib@xercesc_2_3@@3PAUHINSTANCE__@@A 121dcc8c     BinHTTPURLInputStream.obj
 0003:00023c90       ?gWSgethostbyname@xercesc_2_3@@3P6GPAUhostent@@PBD@ZA 121dcc90     BinHTTPURLInputStream.obj
 0003:00023c94       ?gWSinet_addr@xercesc_2_3@@3P6GKPBD@ZA 121dcc94     BinHTTPURLInputStream.obj
 0003:00023c98       ?gWSgethostbyaddr@xercesc_2_3@@3P6GPAUhostent@@PBDHH@ZA 121dcc98     BinHTTPURLInputStream.obj
 0003:00023c9c       ?gWShtons@xercesc_2_3@@3P6GGG@ZA 121dcc9c     BinHTTPURLInputStream.obj
 0003:00023ca0       ?gWSsocket@xercesc_2_3@@3P6GIHHH@ZA 121dcca0     BinHTTPURLInputStream.obj
 0003:00023ca4       ?gWSconnect@xercesc_2_3@@3P6GHIPBUsockaddr@@H@ZA 121dcca4     BinHTTPURLInputStream.obj
 0003:00023ca8       ?gWSsend@xercesc_2_3@@3P6GHIPBDHH@ZA 121dcca8     BinHTTPURLInputStream.obj
 0003:00023cac       ?gWSrecv@xercesc_2_3@@3P6GHIPADHH@ZA 121dccac     BinHTTPURLInputStream.obj
 0003:00023cb0       ?gWSshutdown@xercesc_2_3@@3P6GHIH@ZA 121dccb0     BinHTTPURLInputStream.obj
 0003:00023cb4       ?gWSclosesocket@xercesc_2_3@@3P6GHI@ZA 121dccb4     BinHTTPURLInputStream.obj
 0003:00023cb8       ?gWSACleanup@xercesc_2_3@@3P6GHXZA 121dccb8     BinHTTPURLInputStream.obj
 0003:00023cbc       ?fInitialized@BinHTTPURLInputStream@xercesc_2_3@@0_NA 121dccbc     BinHTTPURLInputStream.obj
 0003:00023cc0       ?fInitMutex@BinHTTPURLInputStream@xercesc_2_3@@0PAVXMLMutex@2@A 121dccc0     BinHTTPURLInputStream.obj
 0003:00023cdc       ?fInstance@RangeTokenMap@xercesc_2_3@@0PAV12@A 121dccdc     RangeTokenMap.obj
 0003:00023ce0       ?fWordRange@RegularExpression@xercesc_2_3@@0PAVRangeToken@2@A 121dcce0     RegularExpression.obj
 0003:00023ce4       ?fRangeInitialized@TokenFactory@xercesc_2_3@@0_NA 121dcce4     TokenFactory.obj
 0003:00023ce8       ?base64Inverse@Base64@xercesc_2_3@@0PAEA 121dcce8     Base64.obj
 0003:00023de7       ?isInitialized@Base64@xercesc_2_3@@0_NA 121dcde7     Base64.obj
 0003:00023dfc       ?fInstance@EncodingValidator@xercesc_2_3@@0PAV12@A 121dcdfc     EncodingValidator.obj
 0003:00023e00       ?hexNumberTable@HexBin@xercesc_2_3@@0PA_NA 121dce00     HexBin.obj
 0003:00023eff       ?isInitialized@HexBin@xercesc_2_3@@0_NA 121dceff     HexBin.obj
 0003:00023f08       ?gXMLCleanupList@xercesc_2_3@@3PAVXMLRegisterCleanup@1@A 121dcf08     PlatformUtils.obj
 0003:00023f0c       ?gXMLCleanupListMutex@xercesc_2_3@@3PAVXMLMutex@1@A 121dcf0c     PlatformUtils.obj
 0003:00023f10       ?fgNetAccessor@XMLPlatformUtils@xercesc_2_3@@2PAVXMLNetAccessor@2@A 121dcf10     PlatformUtils.obj
 0003:00023f14       ?fgTransService@XMLPlatformUtils@xercesc_2_3@@2PAVXMLTransService@2@A 121dcf14     PlatformUtils.obj
 0003:00023f18       ?fgUserPanicHandler@XMLPlatformUtils@xercesc_2_3@@2PAVPanicHandler@2@A 121dcf18     PlatformUtils.obj
 0003:00023f1c       ?fgDefaultPanicHandler@XMLPlatformUtils@xercesc_2_3@@2PAVPanicHandler@2@A 121dcf1c     PlatformUtils.obj
 0003:00023f20       ?fgMemoryManager@XMLPlatformUtils@xercesc_2_3@@2PAVMemoryManager@2@A 121dcf20     PlatformUtils.obj
 0003:00023fd8       ?enableNEL@XMLChar1_0@xercesc_2_3@@0_NA 121dcfd8     XMLChar.obj
 0003:00024004       ?fLocale@XMLMsgLoader@xercesc_2_3@@0PADA 121dd004     XMLMsgLoader.obj
 0003:00024008       ?fPath@XMLMsgLoader@xercesc_2_3@@0PADA 121dd008     XMLMsgLoader.obj
 0003:00024010       ?fgMemoryManager@XMLString@xercesc_2_3@@0PAVMemoryManager@2@A 121dd010     XMLString.obj
 0003:0002420c       ?fBuiltInRegistry@DatatypeValidatorFactory@xercesc_2_3@@0PAV?$RefHashTableOf@VDatatypeValidator@xercesc_2_3@@@2@A 121dd20c     DatatypeValidatorFactory.obj
 0003:00024534       ?fAttMap@GeneralAttributeCheck@xercesc_2_3@@0PAV?$ValueHashTableOf@G@2@A 121dd534     GeneralAttributeCheck.obj
 0003:00024538       ?fFacetsMap@GeneralAttributeCheck@xercesc_2_3@@0PAV?$ValueHashTableOf@G@2@A 121dd538     GeneralAttributeCheck.obj
 0003:0002453c       ?fNonNegIntDV@GeneralAttributeCheck@xercesc_2_3@@0PAVDatatypeValidator@2@A 121dd53c     GeneralAttributeCheck.obj
 0003:00024540       ?fBooleanDV@GeneralAttributeCheck@xercesc_2_3@@0PAVDatatypeValidator@2@A 121dd540     GeneralAttributeCheck.obj
 0003:00024544       ?fAnyURIDV@GeneralAttributeCheck@xercesc_2_3@@0PAVDatatypeValidator@2@A 121dd544     GeneralAttributeCheck.obj
 0003:00024744       ?freeListPtr@DOMStringHandle@xercesc_2_3@@0PAXA 121dd744     DOMString.obj
 0003:00024748       ?blockListPtr@DOMStringHandle@xercesc_2_3@@0PAV12@A 121dd748     DOMString.obj
 0003:0002474c       ?gLiveStringDataCount@DOMString@xercesc_2_3@@0HA 121dd74c     DOMString.obj
 0003:00024750       ?gTotalStringDataCount@DOMString@xercesc_2_3@@0HA 121dd750     DOMString.obj
 0003:00024754       ?gLiveStringHandleCount@DOMString@xercesc_2_3@@0HA 121dd754     DOMString.obj
 0003:00024758       ?gTotalStringHandleCount@DOMString@xercesc_2_3@@0HA 121dd758     DOMString.obj
 0003:00024770       ?gLiveNamedNodeMaps@NamedNodeMapImpl@xercesc_2_3@@1HA 121dd770     NamedNodeMapImpl.obj
 0003:00024774       ?gTotalNamedNodeMaps@NamedNodeMapImpl@xercesc_2_3@@1HA 121dd774     NamedNodeMapImpl.obj
 0003:00024794       ?gLiveNodeImpls@NodeImpl@xercesc_2_3@@2HA 121dd794     NodeImpl.obj
 0003:00024798       ?gTotalNodeImpls@NodeImpl@xercesc_2_3@@2HA 121dd798     NodeImpl.obj
 0003:000247c4       __adjust_fdiv              121dd7c4     <common>
 0003:000247c8       __pRawDllMain              121dd7c8     <common>
 0003:000247cc       ___onexitend               121dd7cc     <common>
 0003:000247d0       ___onexitbegin             121dd7d0     <common>

 entry point at        0001:000f0a2a

 Static symbols

 0001:000f00a0       _$E215                     120f10a0 f   XMLDeclImpl.obj
 0001:000ee4e0       _$E215                     120ef4e0 f   TextImpl.obj
 0001:000e4a80       _$E215                     120e5a80 f   NodeImpl.obj
 0001:000e1420       _$E217                     120e2420 f   ElementImpl.obj
 0001:000de010       _$E216                     120df010 f   DOMString.obj
 0001:000de030       _$E219                     120df030 f   DOMString.obj
 0001:000e0d70       ?reinitDomConverter@xercesc_2_3@@YAXXZ 120e1d70 f   DOMString.obj
 0001:000e0d90       ?reinitDomMutex@xercesc_2_3@@YAXXZ 120e1d90 f   DOMString.obj
 0001:000d89c0       _$E218                     120d99c0 f   DOM_DOMImplementation.obj
 0001:000d8ad0       ?reinitImplementation@xercesc_2_3@@YAXXZ 120d9ad0 f   DOM_DOMImplementation.obj
 0001:000d8af0       _$E221                     120d9af0 f   DOM_DOMImplementation.obj
 0001:000d4e00       _$E232                     120d5e00 f   DocumentImpl.obj
 0001:000d4b20       _$E215                     120d5b20 f   DocumentFragmentImpl.obj
 0001:000d4510       _$E217                     120d5510 f   DeepNodeListImpl.obj
 0001:000d43c0       _$E215                     120d53c0 f   CommentImpl.obj
 0001:000d39a0       _$E215                     120d49a0 f   CDATASectionImpl.obj
 0001:000ce720       _$E213                     120cf720 f   DOMWriterImpl.obj
 0001:000c65c0       _$E232                     120c75c0 f   DOMNormalizer.obj
 0001:000c65e0       _$E235                     120c75e0 f   DOMNormalizer.obj
 0001:000c4410       ?reinitEmptyNodeList@xercesc_2_3@@YAXXZ 120c5410 f   DOMNodeImpl.obj
 0001:000c4430       _$E211                     120c5430 f   DOMNodeImpl.obj
 0001:000c2a60       ?reinitDOMImplSrcVector@xercesc_2_3@@YAXXZ 120c3a60 f   DOMImplementationRegistry.obj
 0001:000c2a80       _$E197                     120c3a80 f   DOMImplementationRegistry.obj
 0001:000c2a90       ?reinitDOMImplSrcVectorMutex@xercesc_2_3@@YAXXZ 120c3a90 f   DOMImplementationRegistry.obj
 0001:000c2ac0       _$E199                     120c3ac0 f   DOMImplementationRegistry.obj
 0001:000c1ea0       ?reinitMsgLoader4DOM@xercesc_2_3@@YAXXZ 120c2ea0 f   DOMImplementationImpl.obj
 0001:000c1ec0       _$E224                     120c2ec0 f   DOMImplementationImpl.obj
 0001:000c2020       ?reinitImplementation@xercesc_2_3@@YAXXZ 120c3020 f   DOMImplementationImpl.obj
 0001:000c2040       _$E226                     120c3040 f   DOMImplementationImpl.obj
 0001:000be0d0       _$E214                     120bf0d0 f   DOMDocumentTypeImpl.obj
 0001:000be340       ?reinitDocument@xercesc_2_3@@YAXXZ 120bf340 f   DOMDocumentTypeImpl.obj
 0001:000b32f0       ?reinitErrMsgLoader@xercesc_2_3@@YAXXZ 120b42f0 f   XSDErrorReporter.obj
 0001:000b3310       ?reinitValidMsgLoader@xercesc_2_3@@YAXXZ 120b4310 f   XSDErrorReporter.obj
 0001:000b3330       _$E201                     120b4330 f   XSDErrorReporter.obj
 0001:000b3340       _$E203                     120b4340 f   XSDErrorReporter.obj
 0001:000906e0       _$E403                     120916e0 f   GeneralAttributeCheck.obj
 0001:00081d00       ?makeRepNode@xercesc_2_3@@YAPAVContentSpecNode@1@GQAV21@QAVMemoryManager@1@@Z 12082d00 f   DTDScanner.obj
 0001:00074250       _$E394                     12075250 f   DatatypeValidatorFactory.obj
 0001:000675f0       ?formatNode@xercesc_2_3@@YAXQBVContentSpecNode@1@W4NodeTypes@21@AAVXMLBuffer@1@@Z 120685f0 f   ContentSpecNode.obj
 0001:00056eb0       _$E223                     12057eb0 f   XMLScanner.obj
 0001:00056ed0       _$E226                     12057ed0 f   XMLScanner.obj
 0001:00058500       ?gScannerMsgLoader@xercesc_2_3@@YAAAVXMLMsgLoader@1@XZ 12059500 f   XMLScanner.obj
 0001:000315f0       _$E217                     120325f0 f   XMLValidator.obj
 0001:00031610       _$E220                     12032610 f   XMLValidator.obj
 0001:00031730       ?getMsgLoader@xercesc_2_3@@YAAAVXMLMsgLoader@1@XZ 12032730 f   XMLValidator.obj
 0001:00023750       _$E201                     12024750 f   XMLException.obj
 0001:00023770       _$E204                     12024770 f   XMLException.obj
 0001:00023b30       ?gGetMsgLoader@xercesc_2_3@@YAAAVXMLMsgLoader@1@XZ 12024b30 f   XMLException.obj
 0001:0001bbd0       ?reinitMappings@xercesc_2_3@@YAXXZ 1201cbd0 f   TransService.obj
 0001:0001bc90       ?reinitMappingsRecognizer@xercesc_2_3@@YAXXZ 1201cc90 f   TransService.obj
 0001:0001bcb0       _$E212                     1201ccb0 f   TransService.obj
 0001:0001bcc0       _$E211                     1201ccc0 f   TransService.obj
 0001:00018a00       _$E199                     12019a00 f   EncodingValidator.obj
 0001:0000b1f0       _$E206                     1200c1f0 f   RangeTokenMap.obj
 0001:000f08ba       ?ArrayUnwindFilter@@YAHPAU_EXCEPTION_POINTERS@@@Z 120f18ba f   MSVCRT:ehvecdtr.obj

 57968 bytes saved through ICF

